 phylip

 Timestamp is 5dee3632 (Mon Dec 09 18:55:30 2019)

 Preferred load address is 10000000

 Start         Length     Name                   Class
 0001:00000000 00005a68H .text$di                CODE
 0001:00005a70 000353f6H .text$mn                CODE
 0001:0003ae70 00004544H .text$x                 CODE
 0001:0003f3c0 000011ebH .text$yd                CODE
 0002:00000000 00000b50H .idata$5                DATA
 0002:00000b50 00000004H .CRT$XCA                DATA
 0002:00000b54 000003a8H .CRT$XCU                DATA
 0002:00000efc 00000004H .CRT$XCZ                DATA
 0002:00000f00 00000004H .CRT$XIA                DATA
 0002:00000f04 00000004H .CRT$XIAA               DATA
 0002:00000f08 00000008H .CRT$XIC                DATA
 0002:00000f10 00000004H .CRT$XIZ                DATA
 0002:00000f20 00005848H .rdata                  DATA
 0002:00006768 0000006cH .rdata$debug            DATA
 0002:000067d4 000012c0H .rdata$r                DATA
 0002:00007aa0 00000474H .rdata$sxdata           DATA
 0002:00007f14 00000004H .rtc$IAA                DATA
 0002:00007f18 00000004H .rtc$IZZ                DATA
 0002:00007f1c 00000004H .rtc$TAA                DATA
 0002:00007f20 00000004H .rtc$TZZ                DATA
 0002:00007f28 0000492cH .xdata$x                DATA
 0002:0000c860 0000004fH .edata                  DATA
 0002:0000c8b0 000000c8H .idata$2                DATA
 0002:0000c978 00000014H .idata$3                DATA
 0002:0000c98c 00000b50H .idata$4                DATA
 0002:0000d4dc 00007e4cH .idata$6                DATA
 0003:00000000 00009fa4H .data                   DATA
 0003:00009fa4 00000890H .data$r                 DATA
 0003:0000a838 000038f0H .bss                    DATA
 0004:00000000 00000058H .rsrc$01                DATA
 0004:00000060 00000180H .rsrc$02                DATA

  Address         Publics by Value              Rva+Base       Lib:Object

 0000:00000000       __except_list              00000000     <absolute>
 0000:00000000       ___guard_flags             00000000     <absolute>
 0000:00000000       ___guard_fids_table        00000000     <absolute>
 0000:00000000       ___guard_fids_count        00000000     <absolute>
 0000:0000011d       ___safe_se_handler_count   0000011d     <absolute>
 0000:00009876       __ldused                   00009876     <absolute>
 0000:00009876       __fltused                  00009876     <absolute>
 0000:00000000       ___ImageBase               10000000     <linker-defined>
 0001:00005a70       ??$?6U?$char_traits@D@std@@@std@@YAAAV?$basic_ostream@DU?$char_traits@D@std@@@0@AAV10@PBD@Z 10006a70 f i DistanceMatrix.obj
 0001:00005ca0       ??$_Allocate@D@std@@YAPADIPAD@Z 10006ca0 f i DistanceMatrix.obj
 0001:00005cd0       ??$_Move@AAPAU?$QMapData@VQString@@H@@@std@@YA$$QAPAU?$QMapData@VQString@@H@@AAPAU1@@Z 10006cd0 f i DistanceMatrix.obj
 0001:00005ce0       ??$_Move@AAPAU?$QTypedArrayData@M@@@std@@YA$$QAPAU?$QTypedArrayData@M@@AAPAU1@@Z 10006ce0 f i DistanceMatrix.obj
 0001:00005cf0       ??$_Move@AAPAU?$QTypedArrayData@V?$QVector@M@@@@@std@@YA$$QAPAU?$QTypedArrayData@V?$QVector@M@@@@AAPAU1@@Z 10006cf0 f i DistanceMatrix.obj
 0001:00005d00       ??$_Move@AAPAUData@QListData@@@std@@YA$$QAPAUData@QListData@@AAPAU12@@Z 10006d00 f i DistanceMatrix.obj
 0001:00005d10       ??$addressof@D@std@@YAPADAAD@Z 10006d10 f i DistanceMatrix.obj
 0001:00005d20       ??$atomic@H@?$QAtomicOpsBySize@$03@@CAPAJPAH@Z 10006d20 f i DistanceMatrix.obj
 0001:00005d30       ??$construct@PADAAPAD@?$_Wrap_alloc@V?$allocator@D@std@@@std@@QAEXPAPADAAPAD@Z 10006d30 f i DistanceMatrix.obj
 0001:00005d50       ??$construct@PADAAPAD@?$allocator@D@std@@QAEXPAPADAAPAD@Z 10006d50 f i DistanceMatrix.obj
 0001:00005d70       ??$construct@PADAAPAD@?$allocator_traits@V?$allocator@D@std@@@std@@SAXAAV?$allocator@D@1@PAPADAAPAD@Z 10006d70 f i DistanceMatrix.obj
 0001:00005d90       ??$deref@H@?$QAtomicOpsBySize@$03@@SA_NAAH@Z 10006d90 f i DistanceMatrix.obj
 0001:00005db0       ??$destroy@PAD@?$_Wrap_alloc@V?$allocator@D@std@@@std@@QAEXPAPAD@Z 10006db0 f i DistanceMatrix.obj
 0001:00005dc0       ??$destroy@PAD@?$allocator@D@std@@QAEXPAPAD@Z 10006dc0 f i DistanceMatrix.obj
 0001:00005dd0       ??$destroy@PAD@?$allocator_traits@V?$allocator@D@std@@@std@@SAXAAV?$allocator@D@1@PAPAD@Z 10006dd0 f i DistanceMatrix.obj
 0001:00005de0       ??$endl@DU?$char_traits@D@std@@@std@@YAAAV?$basic_ostream@DU?$char_traits@D@std@@@0@AAV10@@Z 10006de0 f i DistanceMatrix.obj
 0001:00005e10       ??$forward@AAPAD@std@@YAAAPADAAPAD@Z 10006e10 f i DistanceMatrix.obj
 0001:00005e20       ??$load@H@?$QGenericAtomicOps@U?$QAtomicOpsBySize@$03@@@@SAHABH@Z 10006e20 f i DistanceMatrix.obj
 0001:00005e30       ??$qMapLessThanKey@VQString@@@@YA_NABVQString@@0@Z 10006e30 f i DistanceMatrix.obj
 0001:00005e40       ??$qMax@H@@YAABHABH0@Z     10006e40 f i DistanceMatrix.obj
 0001:00005e60       ??$qSwap@PAU?$QMapData@VQString@@H@@@@YAXAAPAU?$QMapData@VQString@@H@@0@Z 10006e60 f i DistanceMatrix.obj
 0001:00005e80       ??$qSwap@PAU?$QTypedArrayData@M@@@@YAXAAPAU?$QTypedArrayData@M@@0@Z 10006e80 f i DistanceMatrix.obj
 0001:00005ea0       ??$qSwap@PAU?$QTypedArrayData@V?$QVector@M@@@@@@YAXAAPAU?$QTypedArrayData@V?$QVector@M@@@@0@Z 10006ea0 f i DistanceMatrix.obj
 0001:00005ec0       ??$qSwap@PAUData@QListData@@@@YAXAAPAUData@QListData@@0@Z 10006ec0 f i DistanceMatrix.obj
 0001:00005ee0       ??$ref@H@?$QAtomicOpsBySize@$03@@SA_NAAH@Z 10006ee0 f i DistanceMatrix.obj
 0001:00005f00       ??$swap@PAU?$QMapData@VQString@@H@@@std@@YAXAAPAU?$QMapData@VQString@@H@@0@Z 10006f00 f i DistanceMatrix.obj
 0001:00005f20       ??$swap@PAU?$QTypedArrayData@M@@@std@@YAXAAPAU?$QTypedArrayData@M@@0@Z 10006f20 f i DistanceMatrix.obj
 0001:00005f40       ??$swap@PAU?$QTypedArrayData@V?$QVector@M@@@@@std@@YAXAAPAU?$QTypedArrayData@V?$QVector@M@@@@0@Z 10006f40 f i DistanceMatrix.obj
 0001:00005f60       ??$swap@PAUData@QListData@@@std@@YAXAAPAUData@QListData@@0@Z 10006f60 f i DistanceMatrix.obj
 0001:00005f80       ??0?$QFlags@W4AllocationOption@QArrayData@@@@QAE@W4AllocationOption@QArrayData@@@Z 10006f80 f i DistanceMatrix.obj
 0001:00005f90       ??0?$QForeachContainer@$$CBV?$QList@VMultipleSequenceAlignmentRow@U2@@@@@@QAE@ABV?$QList@VMultipleSequenceAlignmentRow@U2@@@@@Z 10006f90 f i DistanceMatrix.obj
 0001:00005fd0       ??0?$QList@PAVPhyBranch@U2@@@@QAE@XZ 10006fd0 f i DistanceMatrix.obj
 0001:00005fe0       ??0?$QList@PAVPhyNode@U2@@@@QAE@XZ 10006fe0 f i DistanceMatrix.obj
 0001:00005ff0       ??0?$QList@VMultipleSequenceAlignmentRow@U2@@@@QAE@ABV0@@Z 10006ff0 f i DistanceMatrix.obj
 0001:000060b0       ??0?$QList@VQString@@@@QAE@$$QAV0@@Z 100070b0 f i DistanceMatrix.obj
 0001:000060d0       ??0?$QList@VQString@@@@QAE@XZ 100070d0 f i DistanceMatrix.obj
 0001:000060e0       ??0?$QMap@VQString@@H@@QAE@XZ 100070e0 f i DistanceMatrix.obj
 0001:000060f0       ??0?$QVector@M@@QAE@ABV0@@Z 100070f0 f i DistanceMatrix.obj
 0001:000061b0       ??0?$QVector@M@@QAE@XZ     100071b0 f i DistanceMatrix.obj
 0001:000061c0       ??0?$QVector@V?$QVector@M@@@@QAE@ABV0@@Z 100071c0 f i DistanceMatrix.obj
 0001:00006280       ??0?$QVector@V?$QVector@M@@@@QAE@XZ 10007280 f i DistanceMatrix.obj
 0001:00006290       ??0?$_String_alloc@$0A@U?$_String_base_types@DV?$allocator@D@std@@@std@@@std@@QAE@ABV?$allocator@D@1@@Z 10007290 f i DistanceMatrix.obj
 0001:000062b0       ??0?$_String_val@U?$_Simple_types@D@std@@@std@@QAE@XZ 100072b0 f i DistanceMatrix.obj
 0001:000062d0       ??0?$_Wrap_alloc@V?$allocator@D@std@@@std@@QAE@XZ 100072d0 f i DistanceMatrix.obj
 0001:000062e0       ??0?$allocator@D@std@@QAE@XZ 100072e0 f i DistanceMatrix.obj
 0001:000062f0       ??0?$basic_string@DU?$char_traits@D@std@@V?$allocator@D@2@@std@@QAE@PBD@Z 100072f0 f i DistanceMatrix.obj
 0001:00006350       ??0DistanceMatrix@U2@@QAE@XZ 10007350 f   DistanceMatrix.obj
 0001:00006470       ??0MemoryLocker@U2@@QAE@HW4MemoryLockType@AppResource@1@@Z 10007470 f i DistanceMatrix.obj
 0001:00006520       ??0QLatin1Char@@QAE@D@Z    10007520 f i DistanceMatrix.obj
 0001:00006530       ??0_Generic_error_category@std@@QAE@XZ 10007530 f i DistanceMatrix.obj
 0001:00006540       ??0_Ignore@std@@QAE@XZ     10007540 f i DistanceMatrix.obj
 0001:00006550       ??0_Iostream_error_category@std@@QAE@XZ 10007550 f i DistanceMatrix.obj
 0001:00006560       ??0_Sentry_base@?$basic_ostream@DU?$char_traits@D@std@@@std@@QAE@AAV12@@Z 10007560 f i DistanceMatrix.obj
 0001:00006590       ??0_System_error_category@std@@QAE@XZ 10007590 f i DistanceMatrix.obj
 0001:000065a0       ??0const_iterator@?$QList@VMultipleSequenceAlignmentRow@U2@@@@QAE@PAUNode@1@@Z 100075a0 f i DistanceMatrix.obj
 0001:000065b0       ??0const_iterator@?$QMap@VQString@@H@@QAE@PBU?$QMapNode@VQString@@H@@@Z 100075b0 f i DistanceMatrix.obj
 0001:000065c0       ??0error_category@std@@QAE@XZ 100075c0 f i DistanceMatrix.obj
 0001:000065d0       ??0error_condition@std@@QAE@HABVerror_category@1@@Z 100075d0 f i DistanceMatrix.obj
 0001:000065f0       ??0iterator@?$QMap@VQString@@H@@QAE@PAU?$QMapNode@VQString@@H@@@Z 100075f0 f i DistanceMatrix.obj
 0001:00006600       ??0iterator@?$QMap@VQString@@H@@QAE@XZ 10007600 f i DistanceMatrix.obj
 0001:00006610       ??0sentry@?$basic_ostream@DU?$char_traits@D@std@@@std@@QAE@AAV12@@Z 10007610 f i DistanceMatrix.obj
 0001:000066a0       ??1?$QForeachContainer@$$CBV?$QList@VMultipleSequenceAlignmentRow@U2@@@@@@QAE@XZ 100076a0 f i DistanceMatrix.obj
 0001:000066d0       ??1?$QList@PAVPhyBranch@U2@@@@QAE@XZ 100076d0 f i DistanceMatrix.obj
 0001:00006700       ??1?$QList@PAVPhyNode@U2@@@@QAE@XZ 10007700 f i DistanceMatrix.obj
 0001:00006730       ??1?$QList@VMultipleSequenceAlignmentRow@U2@@@@QAE@XZ 10007730 f i DistanceMatrix.obj
 0001:00006760       ??1?$QList@VQString@@@@QAE@XZ 10007760 f i DistanceMatrix.obj
 0001:000067c0       ??1?$QMap@VQString@@H@@QAE@XZ 100077c0 f i DistanceMatrix.obj
 0001:00006830       ??1?$QVector@M@@QAE@XZ     10007830 f i DistanceMatrix.obj
 0001:00006870       ??1?$QVector@V?$QVector@M@@@@QAE@XZ 10007870 f i DistanceMatrix.obj
 0001:000068d0       ??1?$basic_string@DU?$char_traits@D@std@@V?$allocator@D@2@@std@@QAE@XZ 100078d0 f i DistanceMatrix.obj
 0001:00006900       ??1DistanceMatrix@U2@@QAE@XZ 10007900 f   DistanceMatrix.obj
 0001:00006da0       ??1MemoryLocker@U2@@UAE@XZ 10007da0 f i DistanceMatrix.obj
 0001:00006e00       ??1_Generic_error_category@std@@UAE@XZ 10007e00 f i DistanceMatrix.obj
 0001:00006e10       ??1_Iostream_error_category@std@@UAE@XZ 10007e10 f i DistanceMatrix.obj
 0001:00006e20       ??1_Sentry_base@?$basic_ostream@DU?$char_traits@D@std@@@std@@QAE@XZ 10007e20 f i DistanceMatrix.obj
 0001:00006e40       ??1_System_error_category@std@@UAE@XZ 10007e40 f i DistanceMatrix.obj
 0001:00006e50       ??1error_category@std@@UAE@XZ 10007e50 f i DistanceMatrix.obj
 0001:00006e60       ??1sentry@?$basic_ostream@DU?$char_traits@D@std@@@std@@QAE@XZ 10007e60 f i DistanceMatrix.obj
 0001:00006e90       ??2@YAPAXIPAX@Z            10007e90 f i DistanceMatrix.obj
 0001:00006ea0       ??3@YAXPAX0@Z              10007ea0 f i DistanceMatrix.obj
 0001:00006eb0       ??4?$QList@VQString@@@@QAEAAV0@$$QAV0@@Z 10007eb0 f i DistanceMatrix.obj
 0001:00006ed0       ??4?$QMap@VQString@@H@@QAEAAV0@$$QAV0@@Z 10007ed0 f i DistanceMatrix.obj
 0001:00006ef0       ??4?$QVector@M@@QAEAAV0@ABV0@@Z 10007ef0 f i DistanceMatrix.obj
 0001:00006f60       ??4?$QVector@V?$QVector@M@@@@QAE?AV0@$$QAV0@@Z 10007f60 f i DistanceMatrix.obj
 0001:00006f90       ??8const_iterator@?$QMap@VQString@@H@@QBE_NABV01@@Z 10007f90 f i DistanceMatrix.obj
 0001:00006fb0       ??8error_category@std@@QBE_NABV01@@Z 10007fb0 f i DistanceMatrix.obj
 0001:00006fc0       ??8error_condition@std@@QBE_NABV01@@Z 10007fc0 f i DistanceMatrix.obj
 0001:00006fe0       ??9@YA_NABVQString@@0@Z    10007fe0 f i DistanceMatrix.obj
 0001:00007000       ??9const_iterator@?$QList@VMultipleSequenceAlignmentRow@U2@@@@QBE_NABV01@@Z 10008000 f i DistanceMatrix.obj
 0001:00007020       ??9const_iterator@?$QMap@VQString@@H@@QBE_NABV01@@Z 10008020 f i DistanceMatrix.obj
 0001:00007040       ??9iterator@?$QMap@VQString@@H@@QBE_NABV01@@Z 10008040 f i DistanceMatrix.obj
 0001:00007060       ??A?$QList@PAVPhyNode@U2@@@@QAEAAPAVPhyNode@U2@@H@Z 10008060 f i DistanceMatrix.obj
 0001:00007090       ??A?$QList@VQString@@@@QAEAAVQString@@H@Z 10008090 f i DistanceMatrix.obj
 0001:000070c0       ??A?$QMap@VQString@@H@@QAEAAHABVQString@@@Z 100080c0 f i DistanceMatrix.obj
 0001:00007140       ??A?$QVector@M@@QAEAAMH@Z  10008140 f i DistanceMatrix.obj
 0001:000071c0       ??A?$QVector@V?$QVector@M@@@@QAEAAV?$QVector@M@@H@Z 100081c0 f i DistanceMatrix.obj
 0001:00007240       ??Bsentry@?$basic_ostream@DU?$char_traits@D@std@@@std@@QBE_NXZ 10008240 f i DistanceMatrix.obj
 0001:00007250       ??Dconst_iterator@?$QList@VMultipleSequenceAlignmentRow@U2@@@@QBEABVMultipleSequenceAlignmentRow@U2@@XZ 10008250 f i DistanceMatrix.obj
 0001:00007260       ??Diterator@?$QMap@VQString@@H@@QBEAAHXZ 10008260 f i DistanceMatrix.obj
 0001:00007270       ??Econst_iterator@?$QList@VMultipleSequenceAlignmentRow@U2@@@@QAEAAV01@XZ 10008270 f i DistanceMatrix.obj
 0001:00007280       ??Econst_iterator@?$QMap@VQString@@H@@QAEAAV01@XZ 10008280 f i DistanceMatrix.obj
 0001:000072a0       ??Eiterator@?$QMap@VQString@@H@@QAEAAV01@XZ 100082a0 f i DistanceMatrix.obj
 0001:000072c0       ??_G?$QVector@M@@QAEPAXI@Z 100082c0 f i DistanceMatrix.obj
 0001:00007320       ??_GMemoryLocker@U2@@UAEPAXI@Z 10008320 f i DistanceMatrix.obj
 0001:00007320       ??_EMemoryLocker@U2@@UAEPAXI@Z 10008320 f i DistanceMatrix.obj
 0001:00007390       ??_EMultipleSequenceAlignmentRow@U2@@UAEPAXI@Z 10008390 f i DistanceMatrix.obj
 0001:00007390       ??_GMultipleSequenceAlignmentRow@U2@@UAEPAXI@Z 10008390 f i DistanceMatrix.obj
 0001:000073c0       ??_GPhyTreeData@U2@@QAEPAXI@Z 100083c0 f i DistanceMatrix.obj
 0001:000073f0       ??_GQString@@QAEPAXI@Z     100083f0 f i DistanceMatrix.obj
 0001:00007420       ??_E_Generic_error_category@std@@UAEPAXI@Z 10008420 f i DistanceMatrix.obj
 0001:00007420       ??_G_Generic_error_category@std@@UAEPAXI@Z 10008420 f i DistanceMatrix.obj
 0001:00007450       ??_E_Iostream_error_category@std@@UAEPAXI@Z 10008450 f i DistanceMatrix.obj
 0001:00007450       ??_G_Iostream_error_category@std@@UAEPAXI@Z 10008450 f i DistanceMatrix.obj
 0001:00007480       ??_G_System_error_category@std@@UAEPAXI@Z 10008480 f i DistanceMatrix.obj
 0001:00007480       ??_E_System_error_category@std@@UAEPAXI@Z 10008480 f i DistanceMatrix.obj
 0001:000074b0       ??_Gerror_category@std@@UAEPAXI@Z 100084b0 f i DistanceMatrix.obj
 0001:000074b0       ??_Eerror_category@std@@UAEPAXI@Z 100084b0 f i DistanceMatrix.obj
 0001:000074e0       ?_Copy@?$basic_string@DU?$char_traits@D@std@@V?$allocator@D@2@@std@@QAEXII@Z 100084e0 f i DistanceMatrix.obj
 0001:00007630       ?_Eos@?$basic_string@DU?$char_traits@D@std@@V?$allocator@D@2@@std@@QAEXI@Z 10008630 f i DistanceMatrix.obj
 0001:00007660       ?_Getal@?$_String_alloc@$0A@U?$_String_base_types@DV?$allocator@D@std@@@std@@@std@@QBE?AU?$_Wrap_alloc@V?$allocator@D@std@@@2@XZ 10008660 f i DistanceMatrix.obj
 0001:00007670       ?_Grow@?$basic_string@DU?$char_traits@D@std@@V?$allocator@D@2@@std@@QAE_NI_N@Z 10008670 f i DistanceMatrix.obj
 0001:00007720       ?_Inside@?$basic_string@DU?$char_traits@D@std@@V?$allocator@D@2@@std@@QAE_NPBD@Z 10008720 f i DistanceMatrix.obj
 0001:00007760       ?_Myptr@?$_String_val@U?$_Simple_types@D@std@@@std@@QAEPADXZ 10008760 f i DistanceMatrix.obj
 0001:00007770       ?_Myptr@?$_String_val@U?$_Simple_types@D@std@@@std@@QBEPBDXZ 10008770 f i DistanceMatrix.obj
 0001:00007780       ?_Tidy@?$basic_string@DU?$char_traits@D@std@@V?$allocator@D@2@@std@@QAEX_NI@Z 10008780 f i DistanceMatrix.obj
 0001:000077d0       ?_Xlen@?$basic_string@DU?$char_traits@D@std@@V?$allocator@D@2@@std@@QBEXXZ 100087d0 f i DistanceMatrix.obj
 0001:000077e0       ?_Xran@?$basic_string@DU?$char_traits@D@std@@V?$allocator@D@2@@std@@QBEXXZ 100087e0 f i DistanceMatrix.obj
 0001:000077f0       ?abs@@YANN@Z               100087f0 f i DistanceMatrix.obj
 0001:00007810       ?addNodeToList@DistanceMatrix@U2@@CAXAAV?$QList@PAVPhyNode@U2@@@@AAV?$QMap@VQString@@H@@AAV?$QList@PAVPhyBranch@U2@@@@PAVPhyNode@2@@Z 10008810 f   DistanceMatrix.obj
 0001:000079c0       ?addPairToTree@DistanceMatrix@U2@@AAEXPAU?$QPair@HH@@@Z 100089c0 f   DistanceMatrix.obj
 0001:00008a10       ?allocate@?$QTypedArrayData@M@@SAPAU1@IV?$QFlags@W4AllocationOption@QArrayData@@@@@Z 10009a10 f i DistanceMatrix.obj
 0001:00008a30       ?allocate@?$QTypedArrayData@V?$QVector@M@@@@SAPAU1@IV?$QFlags@W4AllocationOption@QArrayData@@@@@Z 10009a30 f i DistanceMatrix.obj
 0001:00008a50       ?allocate@?$_Wrap_alloc@V?$allocator@D@std@@@std@@QAEPADI@Z 10009a50 f i DistanceMatrix.obj
 0001:00008a80       ?allocate@?$allocator@D@std@@QAEPADI@Z 10009a80 f i DistanceMatrix.obj
 0001:00008ab0       ?append@?$QList@PAVPhyBranch@U2@@@@QAEXABQAVPhyBranch@U2@@@Z 10009ab0 f i DistanceMatrix.obj
 0001:00008b40       ?append@?$QList@PAVPhyNode@U2@@@@QAEXABQAVPhyNode@U2@@@Z 10009b40 f i DistanceMatrix.obj
 0001:00008bd0       ?append@?$QList@VQString@@@@QAEXABVQString@@@Z 10009bd0 f i DistanceMatrix.obj
 0001:00008cc0       ?append@?$QVector@M@@QAEXABM@Z 10009cc0 f i DistanceMatrix.obj
 0001:00008d40       ?append@?$QVector@V?$QVector@M@@@@QAEXABV?$QVector@M@@@Z 10009d40 f i DistanceMatrix.obj
 0001:00008e40       ?areTreesEqual@DistanceMatrix@U2@@CA_NPAV?$QSharedDataPointer@VPhyTreeData@U2@@@@0@Z 10009e40 f   DistanceMatrix.obj
 0001:00009230       ?assign@?$basic_string@DU?$char_traits@D@std@@V?$allocator@D@2@@std@@QAEAAV12@ABV12@II@Z 1000a230 f i DistanceMatrix.obj
 0001:00009350       ?assign@?$basic_string@DU?$char_traits@D@std@@V?$allocator@D@2@@std@@QAEAAV12@PBD@Z 1000a350 f i DistanceMatrix.obj
 0001:00009390       ?assign@?$basic_string@DU?$char_traits@D@std@@V?$allocator@D@2@@std@@QAEAAV12@PBDI@Z 1000a390 f i DistanceMatrix.obj
 0001:00009490       ?assign@?$char_traits@D@std@@SAXAADABD@Z 1000a490 f i DistanceMatrix.obj
 0001:000094a0       ?begin@?$QList@VMultipleSequenceAlignmentRow@U2@@@@QBE?AVconst_iterator@1@XZ 1000a4a0 f i DistanceMatrix.obj
 0001:000094c0       ?begin@?$QMap@VQString@@H@@QAE?AViterator@1@XZ 1000a4c0 f i DistanceMatrix.obj
 0001:00009500       ?begin@?$QMap@VQString@@H@@QBE?AVconst_iterator@1@XZ 1000a500 f i DistanceMatrix.obj
 0001:00009520       ?begin@?$QMapData@VQString@@H@@QAEPAU?$QMapNode@VQString@@H@@XZ 1000a520 f i DistanceMatrix.obj
 0001:00009530       ?begin@?$QTypedArrayData@M@@QAEPAMPAM@Z 1000a530 f i DistanceMatrix.obj
 0001:00009540       ?begin@?$QTypedArrayData@V?$QVector@M@@@@QAEPAV?$QVector@M@@PAV2@@Z 1000a540 f i DistanceMatrix.obj
 0001:00009550       ?calculateAdjacentDistance@DistanceMatrix@U2@@AAEMHHM@Z 1000a550 f   DistanceMatrix.obj
 0001:00009580       ?calculateNewDistance@DistanceMatrix@U2@@AAEMPAU?$QPair@HH@@H@Z 1000a580 f   DistanceMatrix.obj
 0001:00009600       ?calculateOutOfAlignment@DistanceMatrix@U2@@QAEXABVMultipleSequenceAlignment@2@ABVCreatePhyTreeSettings@2@@Z 1000a600 f   DistanceMatrix.obj
 0001:0000a0e0       ?calculateQMatrix@DistanceMatrix@U2@@AAEXXZ 1000b0e0 f   DistanceMatrix.obj
 0001:0000a5a0       ?calculateRawDivergence@DistanceMatrix@U2@@AAEMH@Z 1000b5a0 f   DistanceMatrix.obj
 0001:0000a790       ?calculateRootDistance@DistanceMatrix@U2@@AAEMHH@Z 1000b790 f   DistanceMatrix.obj
 0001:0000a810       ?category@error_code@std@@QBEABVerror_category@2@XZ 1000b810 f i DistanceMatrix.obj
 0001:0000a820       ?category@error_condition@std@@QBEABVerror_category@2@XZ 1000b820 f i DistanceMatrix.obj
 0001:0000a830       ?clear@?$QList@VQString@@@@QAEXXZ 1000b830 f i DistanceMatrix.obj
 0001:0000a850       ?clear@?$QMap@VQString@@H@@QAEXXZ 1000b850 f i DistanceMatrix.obj
 0001:0000a870       ?clear@?$QVector@V?$QVector@M@@@@QAEXXZ 1000b870 f i DistanceMatrix.obj
 0001:0000a960       ?clone@?$QSharedDataPointer@VPhyTreeData@U2@@@@IAEPAVPhyTreeData@U2@@XZ 1000b960 f i DistanceMatrix.obj
 0001:0000a9d0       ?contains@?$QList@PAVPhyBranch@U2@@@@QBE_NABQAVPhyBranch@U2@@@Z 1000b9d0 f i DistanceMatrix.obj
 0001:0000aa10       ?contains@?$QList@PAVPhyNode@U2@@@@QBE_NABQAVPhyNode@U2@@@Z 1000ba10 f i DistanceMatrix.obj
 0001:0000aa50       ?contains@?$QList@VQString@@@@QBE_NABVQString@@@Z 1000ba50 f i DistanceMatrix.obj
 0001:0000aaa0       ?contains@?$QMap@VQString@@H@@QBE_NABVQString@@@Z 1000baa0 f i DistanceMatrix.obj
 0001:0000aae0       ?copy@?$QMapNode@VQString@@H@@QBEPAU1@PAU?$QMapData@VQString@@H@@@Z 1000bae0 f i DistanceMatrix.obj
 0001:0000ab70       ?copy@?$char_traits@D@std@@SAPADPADPBDI@Z 1000bb70 f i DistanceMatrix.obj
 0001:0000ab90       ?copyConstruct@?$QVector@M@@AAEXPBM0PAM@Z 1000bb90 f i DistanceMatrix.obj
 0001:0000abb0       ?copyConstruct@?$QVector@V?$QVector@M@@@@AAEXPBV?$QVector@M@@0PAV2@@Z 1000bbb0 f i DistanceMatrix.obj
 0001:0000ace0       ?count@?$QMap@VQString@@H@@QBEHXZ 1000bce0 f i DistanceMatrix.obj
 0001:0000acf0       ?count@?$QVector@M@@QBEHXZ 1000bcf0 f i DistanceMatrix.obj
 0001:0000ad00       ?count@?$QVector@V?$QVector@M@@@@QBEHXZ 1000bd00 f i DistanceMatrix.obj
 0001:0000ad10       ?create@?$QMapData@VQString@@H@@SAPAU1@XZ 1000bd10 f i DistanceMatrix.obj
 0001:0000ad20       ?createNode@?$QMapData@VQString@@H@@QAEPAU?$QMapNode@VQString@@H@@ABVQString@@ABHPAU2@_N@Z 1000bd20 f i DistanceMatrix.obj
 0001:0000adc0       ?data@?$QSharedDataPointer@VPhyTreeData@U2@@@@QAEPAVPhyTreeData@U2@@XZ 1000bdc0 f i DistanceMatrix.obj
 0001:0000ade0       ?data@?$QTypedArrayData@M@@QAEPAMXZ 1000bde0 f i DistanceMatrix.obj
 0001:0000adf0       ?data@?$QTypedArrayData@V?$QVector@M@@@@QAEPAV?$QVector@M@@XZ 1000bdf0 f i DistanceMatrix.obj
 0001:0000ae00       ?data@?$QVector@M@@QAEPAMXZ 1000be00 f i DistanceMatrix.obj
 0001:0000ae60       ?data@?$QVector@V?$QVector@M@@@@QAEPAV?$QVector@M@@XZ 1000be60 f i DistanceMatrix.obj
 0001:0000aec0       ?dealloc@?$QList@PAVPhyBranch@U2@@@@AAEXPAUData@QListData@@@Z 1000bec0 f i DistanceMatrix.obj
 0001:0000aee0       ?dealloc@?$QList@PAVPhyNode@U2@@@@AAEXPAUData@QListData@@@Z 1000bee0 f i DistanceMatrix.obj
 0001:0000af00       ?dealloc@?$QList@VMultipleSequenceAlignmentRow@U2@@@@AAEXPAUData@QListData@@@Z 1000bf00 f i DistanceMatrix.obj
 0001:0000af50       ?dealloc@?$QList@VQString@@@@AAEXPAUData@QListData@@@Z 1000bf50 f i DistanceMatrix.obj
 0001:0000af90       ?deallocate@?$QTypedArrayData@M@@SAXPAUQArrayData@@@Z 1000bf90 f i DistanceMatrix.obj
 0001:0000afb0       ?deallocate@?$QTypedArrayData@V?$QVector@M@@@@SAXPAUQArrayData@@@Z 1000bfb0 f i DistanceMatrix.obj
 0001:0000afd0       ?deallocate@?$_Wrap_alloc@V?$allocator@D@std@@@std@@QAEXPADI@Z 1000bfd0 f i DistanceMatrix.obj
 0001:0000aff0       ?deallocate@?$allocator@D@std@@QAEXPADI@Z 1000bff0 f i DistanceMatrix.obj
 0001:0000b010       ?defaultConstruct@?$QVector@M@@AAEXPAM0@Z 1000c010 f i DistanceMatrix.obj
 0001:0000b030       ?defaultConstruct@?$QVector@V?$QVector@M@@@@AAEXPAV?$QVector@M@@0@Z 1000c030 f i DistanceMatrix.obj
 0001:0000b060       ?default_error_condition@_System_error_category@std@@UBE?AVerror_condition@2@H@Z 1000c060 f i DistanceMatrix.obj
 0001:0000b0a0       ?default_error_condition@error_category@std@@UBE?AVerror_condition@2@H@Z 1000c0a0 f i DistanceMatrix.obj
 0001:0000b0c0       ?deref@?$QBasicAtomicInteger@H@@QAE_NXZ 1000c0c0 f i DistanceMatrix.obj
 0001:0000b0d0       ?deref@RefCount@QtPrivate@@QAE_NXZ 1000c0d0 f i DistanceMatrix.obj
 0001:0000b0f0       ?destroy@?$QMapData@VQString@@H@@QAEXXZ 1000c0f0 f i DistanceMatrix.obj
 0001:0000b140       ?destroySubTree@?$QMapNode@VQString@@H@@QAEXXZ 1000c140 f i DistanceMatrix.obj
 0001:0000b170       ?destruct@?$QVector@M@@AAEXPAM0@Z 1000c170 f i DistanceMatrix.obj
 0001:0000b180       ?destruct@?$QVector@V?$QVector@M@@@@AAEXPAV?$QVector@M@@0@Z 1000c180 f i DistanceMatrix.obj
 0001:0000b1e0       ?detach@?$QList@PAVPhyNode@U2@@@@QAEXXZ 1000c1e0 f i DistanceMatrix.obj
 0001:0000b200       ?detach@?$QList@VQString@@@@QAEXXZ 1000c200 f i DistanceMatrix.obj
 0001:0000b220       ?detach@?$QMap@VQString@@H@@QAEXXZ 1000c220 f i DistanceMatrix.obj
 0001:0000b240       ?detach@?$QSharedDataPointer@VPhyTreeData@U2@@@@QAEXXZ 1000c240 f i DistanceMatrix.obj
 0001:0000b250       ?detach@?$QVector@M@@QAEXXZ 1000c250 f i DistanceMatrix.obj
 0001:0000b2a0       ?detach@?$QVector@V?$QVector@M@@@@QAEXXZ 1000c2a0 f i DistanceMatrix.obj
 0001:0000b2f0       ?detach_helper@?$QList@PAVPhyNode@U2@@@@AAEXH@Z 1000c2f0 f i DistanceMatrix.obj
 0001:0000b3c0       ?detach_helper@?$QList@PAVPhyNode@U2@@@@AAEXXZ 1000c3c0 f i DistanceMatrix.obj
 0001:0000b3d0       ?detach_helper@?$QList@VQString@@@@AAEXH@Z 1000c3d0 f i DistanceMatrix.obj
 0001:0000b4c0       ?detach_helper@?$QList@VQString@@@@AAEXXZ 1000c4c0 f i DistanceMatrix.obj
 0001:0000b4d0       ?detach_helper@?$QMap@VQString@@H@@AAEXXZ 1000c4d0 f i DistanceMatrix.obj
 0001:0000b580       ?detach_helper@?$QSharedDataPointer@VPhyTreeData@U2@@@@AAEXXZ 1000c580 f i DistanceMatrix.obj
 0001:0000b620       ?detach_helper_grow@?$QList@PAVPhyBranch@U2@@@@AAEPAUNode@1@HH@Z 1000c620 f i DistanceMatrix.obj
 0001:0000b730       ?detach_helper_grow@?$QList@PAVPhyNode@U2@@@@AAEPAUNode@1@HH@Z 1000c730 f i DistanceMatrix.obj
 0001:0000b840       ?detach_helper_grow@?$QList@VQString@@@@AAEPAUNode@1@HH@Z 1000c840 f i DistanceMatrix.obj
 0001:0000b9c0       ?dumpQData@DistanceMatrix@U2@@AAEXXZ 1000c9c0 f   DistanceMatrix.obj
 0001:0000bb30       ?dumpRawData@DistanceMatrix@U2@@AAEXAAV?$QVector@V?$QVector@M@@@@@Z 1000cb30 f   DistanceMatrix.obj
 0001:0000bca0       ?dumpRawData@DistanceMatrix@U2@@AAEXXZ 1000cca0 f   DistanceMatrix.obj
 0001:0000bcb0       ?end@?$QList@VMultipleSequenceAlignmentRow@U2@@@@QBE?AVconst_iterator@1@XZ 1000ccb0 f i DistanceMatrix.obj
 0001:0000bcd0       ?end@?$QMap@VQString@@H@@QAE?AViterator@1@XZ 1000ccd0 f i DistanceMatrix.obj
 0001:0000bd00       ?end@?$QMap@VQString@@H@@QBE?AVconst_iterator@1@XZ 1000cd00 f i DistanceMatrix.obj
 0001:0000bd20       ?end@?$QMapData@VQString@@H@@QAEPAU?$QMapNode@VQString@@H@@XZ 1000cd20 f i DistanceMatrix.obj
 0001:0000bd30       ?end@?$QTypedArrayData@M@@QAEPAMPAM@Z 1000cd30 f i DistanceMatrix.obj
 0001:0000bd50       ?end@?$QTypedArrayData@V?$QVector@M@@@@QAEPAV?$QVector@M@@PAV2@@Z 1000cd50 f i DistanceMatrix.obj
 0001:0000bd70       ?eof@?$char_traits@D@std@@SAHXZ 1000cd70 f i DistanceMatrix.obj
 0001:0000bd80       ?eq_int_type@?$char_traits@D@std@@SA_NABH0@Z 1000cd80 f i DistanceMatrix.obj
 0001:0000bda0       ?equivalent@error_category@std@@UBE_NABVerror_code@2@H@Z 1000cda0 f i DistanceMatrix.obj
 0001:0000bdc0       ?equivalent@error_category@std@@UBE_NHABVerror_condition@2@@Z 1000cdc0 f i DistanceMatrix.obj
 0001:0000be00       ?erase@?$QVector@M@@QAEPAMPAM0@Z 1000ce00 f i DistanceMatrix.obj
 0001:0000be80       ?erase@?$QVector@V?$QVector@M@@@@QAEPAV?$QVector@M@@PAV2@0@Z 1000ce80 f i DistanceMatrix.obj
 0001:0000bf20       ?erase@?$basic_string@DU?$char_traits@D@std@@V?$allocator@D@2@@std@@QAEAAV12@I@Z 1000cf20 f i DistanceMatrix.obj
 0001:0000bf60       ?erase@?$basic_string@DU?$char_traits@D@std@@V?$allocator@D@2@@std@@QAEAAV12@II@Z 1000cf60 f i DistanceMatrix.obj
 0001:0000c000       ?findNode@?$QMapData@VQString@@H@@QBEPAU?$QMapNode@VQString@@H@@ABVQString@@@Z 1000d000 f i DistanceMatrix.obj
 0001:0000c040       ?findNode@DistanceMatrix@U2@@AAEPAVPhyNode@2@PAV32@VQString@@@Z 1000d040 f   DistanceMatrix.obj
 0001:0000c160       ?freeData@?$QVector@M@@AAEXPAU?$QTypedArrayData@M@@@Z 1000d160 f i DistanceMatrix.obj
 0001:0000c190       ?freeData@?$QVector@V?$QVector@M@@@@AAEXPAU?$QTypedArrayData@V?$QVector@M@@@@@Z 1000d190 f i DistanceMatrix.obj
 0001:0000c1d0       ?generateNodeName@DistanceMatrix@U2@@AAE?AVQString@@V3@0@Z 1000d1d0 f   DistanceMatrix.obj
 0001:0000c290       ?generic_category@std@@YAABVerror_category@1@XZ 1000d290 f i DistanceMatrix.obj
 0001:0000c2a0       ?getError@MemoryLocker@U2@@QAEABVQString@@XZ 1000d2a0 f i DistanceMatrix.obj
 0001:0000c2b0       ?getNewIndex@DistanceMatrix@U2@@AAEHVQString@@U?$QPair@HH@@AAV?$QMap@VQString@@H@@@Z 1000d2b0 f   DistanceMatrix.obj
 0001:0000c330       ?getNodeByName@DistanceMatrix@U2@@AAEPAVPhyNode@2@VQString@@@Z 1000d330 f   DistanceMatrix.obj
 0001:0000c3c0       ?getTaxaName@DistanceMatrix@U2@@AAE?AVQString@@H@Z 1000d3c0 f   DistanceMatrix.obj
 0001:0000c470       ?hasError@MemoryLocker@U2@@QAE_NXZ 1000d470 f i DistanceMatrix.obj
 0001:0000c480       ?indexOf@?$QList@VQString@@@@QBEHABVQString@@H@Z 1000d480 f i DistanceMatrix.obj
 0001:0000c520       ?insert@?$QMap@VQString@@H@@QAE?AViterator@1@ABVQString@@ABH@Z 1000d520 f i DistanceMatrix.obj
 0001:0000c5e0       ?isDetached@?$QVector@M@@QBE_NXZ 1000d5e0 f i DistanceMatrix.obj
 0001:0000c610       ?isDetached@?$QVector@V?$QVector@M@@@@QBE_NXZ 1000d610 f i DistanceMatrix.obj
 0001:0000c640       ?isFiniteNumber@U2@@YA_NN@Z 1000d640 f i DistanceMatrix.obj
 0001:0000c670       ?isShared@RefCount@QtPrivate@@QBE_NXZ 1000d670 f i DistanceMatrix.obj
 0001:0000c690       ?isValid@DistanceMatrix@U2@@QAE_NXZ 1000d690 f   DistanceMatrix.obj
 0001:0000c840       ?key@const_iterator@?$QMap@VQString@@H@@QBEABVQString@@XZ 1000d840 f i DistanceMatrix.obj
 0001:0000c850       ?key@iterator@?$QMap@VQString@@H@@QBEABVQString@@XZ 1000d850 f i DistanceMatrix.obj
 0001:0000c860       ?keys@?$QMap@VQString@@H@@QBE?AV?$QList@VQString@@@@ABH@Z 1000d860 f i DistanceMatrix.obj
 0001:0000c910       ?keys@?$QMap@VQString@@H@@QBE?AV?$QList@VQString@@@@XZ 1000d910 f i DistanceMatrix.obj
 0001:0000c9d0       ?leftNode@?$QMapNode@VQString@@H@@QBEPAU1@XZ 1000d9d0 f i DistanceMatrix.obj
 0001:0000c9e0       ?length@?$char_traits@D@std@@SAIPBD@Z 1000d9e0 f i DistanceMatrix.obj
 0001:0000ca00       ?load@?$QBasicAtomicInteger@H@@QBEHXZ 1000da00 f i DistanceMatrix.obj
 0001:0000ca10       ?lowerBound@?$QMapNode@VQString@@H@@QAEPAU1@ABVQString@@@Z 1000da10 f i DistanceMatrix.obj
 0001:0000ca50       ?max_size@?$_Wrap_alloc@V?$allocator@D@std@@@std@@QBEIXZ 1000da50 f i DistanceMatrix.obj
 0001:0000ca60       ?max_size@?$allocator@D@std@@QBEIXZ 1000da60 f i DistanceMatrix.obj
 0001:0000ca70       ?max_size@?$allocator_traits@V?$allocator@D@std@@@std@@SAIABV?$allocator@D@2@@Z 1000da70 f i DistanceMatrix.obj
 0001:0000ca80       ?max_size@?$basic_string@DU?$char_traits@D@std@@V?$allocator@D@2@@std@@QBEIXZ 1000da80 f i DistanceMatrix.obj
 0001:0000ca90       ?message@_Generic_error_category@std@@UBE?AV?$basic_string@DU?$char_traits@D@std@@V?$allocator@D@2@@2@H@Z 1000da90 f i DistanceMatrix.obj
 0001:0000cb10       ?message@_Iostream_error_category@std@@UBE?AV?$basic_string@DU?$char_traits@D@std@@V?$allocator@D@2@@2@H@Z 1000db10 f i DistanceMatrix.obj
 0001:0000cb60       ?message@_System_error_category@std@@UBE?AV?$basic_string@DU?$char_traits@D@std@@V?$allocator@D@2@@2@H@Z 1000db60 f i DistanceMatrix.obj
 0001:0000cbe0       ?move@?$char_traits@D@std@@SAPADPADPBDI@Z 1000dbe0 f i DistanceMatrix.obj
 0001:0000cc00       ?name@_Generic_error_category@std@@UBEPBDXZ 1000dc00 f i DistanceMatrix.obj
 0001:0000cc10       ?name@_Iostream_error_category@std@@UBEPBDXZ 1000dc10 f i DistanceMatrix.obj
 0001:0000cc20       ?name@_System_error_category@std@@UBEPBDXZ 1000dc20 f i DistanceMatrix.obj
 0001:0000cc30       ?nextNode@?$QMapNode@VQString@@H@@QAEPAU1@XZ 1000dc30 f i DistanceMatrix.obj
 0001:0000cc40       ?nextNode@?$QMapNode@VQString@@H@@QBEPBU1@XZ 1000dc40 f i DistanceMatrix.obj
 0001:0000cc50       ?node_construct@?$QList@PAVPhyBranch@U2@@@@AAEXPAUNode@1@ABQAVPhyBranch@U2@@@Z 1000dc50 f i DistanceMatrix.obj
 0001:0000cc70       ?node_construct@?$QList@PAVPhyNode@U2@@@@AAEXPAUNode@1@ABQAVPhyNode@U2@@@Z 1000dc70 f i DistanceMatrix.obj
 0001:0000cc90       ?node_construct@?$QList@VQString@@@@AAEXPAUNode@1@ABVQString@@@Z 1000dc90 f i DistanceMatrix.obj
 0001:0000cce0       ?node_copy@?$QList@PAVPhyBranch@U2@@@@AAEXPAUNode@1@00@Z 1000dce0 f i DistanceMatrix.obj
 0001:0000cd10       ?node_copy@?$QList@PAVPhyNode@U2@@@@AAEXPAUNode@1@00@Z 1000dd10 f i DistanceMatrix.obj
 0001:0000cd40       ?node_copy@?$QList@VMultipleSequenceAlignmentRow@U2@@@@AAEXPAUNode@1@00@Z 1000dd40 f i DistanceMatrix.obj
 0001:0000ce10       ?node_copy@?$QList@VQString@@@@AAEXPAUNode@1@00@Z 1000de10 f i DistanceMatrix.obj
 0001:0000ceb0       ?node_destruct@?$QList@PAVPhyBranch@U2@@@@AAEXPAUNode@1@0@Z 1000deb0 f i DistanceMatrix.obj
 0001:0000cec0       ?node_destruct@?$QList@PAVPhyBranch@U2@@@@AAEXPAUNode@1@@Z 1000dec0 f i DistanceMatrix.obj
 0001:0000ced0       ?node_destruct@?$QList@PAVPhyNode@U2@@@@AAEXPAUNode@1@0@Z 1000ded0 f i DistanceMatrix.obj
 0001:0000cee0       ?node_destruct@?$QList@PAVPhyNode@U2@@@@AAEXPAUNode@1@@Z 1000dee0 f i DistanceMatrix.obj
 0001:0000cef0       ?node_destruct@?$QList@VMultipleSequenceAlignmentRow@U2@@@@AAEXPAUNode@1@0@Z 1000def0 f i DistanceMatrix.obj
 0001:0000cf20       ?node_destruct@?$QList@VQString@@@@AAEXPAUNode@1@0@Z 1000df20 f i DistanceMatrix.obj
 0001:0000cf50       ?node_destruct@?$QList@VQString@@@@AAEXPAUNode@1@@Z 1000df50 f i DistanceMatrix.obj
 0001:0000cf60       ?printIndex@DistanceMatrix@U2@@AAEXXZ 1000df60 f   DistanceMatrix.obj
 0001:0000d110       ?printPhyNode@DistanceMatrix@U2@@CAXPAVPhyNode@2@HAAV?$QList@PAVPhyNode@U2@@@@@Z 1000e110 f   DistanceMatrix.obj
 0001:0000d250       ?printPhyTree@DistanceMatrix@U2@@AAEXXZ 1000e250 f   DistanceMatrix.obj
 0001:0000d260       ?printPhyTree@DistanceMatrix@U2@@CAXPAVPhyTreeData@2@@Z 1000e260 f   DistanceMatrix.obj
 0001:0000d270       ?qt_noop@@YAXXZ            1000e270 f i DistanceMatrix.obj
 0001:0000d280       ?reallocData@?$QVector@M@@AAEXHHV?$QFlags@W4AllocationOption@QArrayData@@@@@Z 1000e280 f i DistanceMatrix.obj
 0001:0000d4c0       ?reallocData@?$QVector@V?$QVector@M@@@@AAEXHHV?$QFlags@W4AllocationOption@QArrayData@@@@@Z 1000e4c0 f i DistanceMatrix.obj
 0001:0000d7a0       ?ref@?$QBasicAtomicInteger@H@@QAE_NXZ 1000e7a0 f i DistanceMatrix.obj
 0001:0000d7c0       ?ref@RefCount@QtPrivate@@QAE_NXZ 1000e7c0 f i DistanceMatrix.obj
 0001:0000d7e0       ?release@MemoryLocker@U2@@QAEXXZ 1000e7e0 f i DistanceMatrix.obj
 0001:0000d890       ?remove@?$QVector@M@@QAEXH@Z 1000e890 f i DistanceMatrix.obj
 0001:0000d8d0       ?remove@?$QVector@V?$QVector@M@@@@QAEXH@Z 1000e8d0 f i DistanceMatrix.obj
 0001:0000d910       ?removeAll@?$QList@VQString@@@@QAEHABVQString@@@Z 1000e910 f i DistanceMatrix.obj
 0001:0000da10       ?reserve@?$QList@VQString@@@@QAEXH@Z 1000ea10 f i DistanceMatrix.obj
 0001:0000da40       ?reserve@?$QVector@M@@QAEXH@Z 1000ea40 f i DistanceMatrix.obj
 0001:0000da90       ?rightNode@?$QMapNode@VQString@@H@@QBEPAU1@XZ 1000ea90 f i DistanceMatrix.obj
 0001:0000daa0       ?root@?$QMapData@VQString@@H@@QBEPAU?$QMapNode@VQString@@H@@XZ 1000eaa0 f i DistanceMatrix.obj
 0001:0000dab0       ?sharedNull@?$QTypedArrayData@M@@SAPAU1@XZ 1000eab0 f i DistanceMatrix.obj
 0001:0000dac0       ?sharedNull@?$QTypedArrayData@V?$QVector@M@@@@SAPAU1@XZ 1000eac0 f i DistanceMatrix.obj
 0001:0000dad0       ?size@?$QList@PAVPhyNode@U2@@@@QBEHXZ 1000ead0 f i DistanceMatrix.obj
 0001:0000dae0       ?size@?$QList@VQString@@@@QBEHXZ 1000eae0 f i DistanceMatrix.obj
 0001:0000daf0       ?size@?$QMap@VQString@@H@@QBEHXZ 1000eaf0 f i DistanceMatrix.obj
 0001:0000db00       ?size@?$basic_string@DU?$char_traits@D@std@@V?$allocator@D@2@@std@@QBEIXZ 1000eb00 f i DistanceMatrix.obj
 0001:0000db10       ?swap@?$QVector@M@@QAEXAAV1@@Z 1000eb10 f i DistanceMatrix.obj
 0001:0000db30       ?switchName@DistanceMatrix@U2@@AAEXPAVPhyNode@2@@Z 1000eb30 f   DistanceMatrix.obj
 0001:0000dcf0       ?switchNamesToAllNodes@DistanceMatrix@U2@@AAEXXZ 1000ecf0 f   DistanceMatrix.obj
 0001:0000de70       ?system_category@std@@YAABVerror_category@1@XZ 1000ee70 f i DistanceMatrix.obj
 0001:0000de80       ?t@Node@?$QList@PAVPhyBranch@U2@@@@QAEAAPAVPhyBranch@U2@@XZ 1000ee80 f i DistanceMatrix.obj
 0001:0000de90       ?t@Node@?$QList@PAVPhyNode@U2@@@@QAEAAPAVPhyNode@U2@@XZ 1000ee90 f i DistanceMatrix.obj
 0001:0000dea0       ?t@Node@?$QList@VMultipleSequenceAlignmentRow@U2@@@@QAEAAVMultipleSequenceAlignmentRow@U2@@XZ 1000eea0 f i DistanceMatrix.obj
 0001:0000deb0       ?t@Node@?$QList@VQString@@@@QAEAAVQString@@XZ 1000eeb0 f i DistanceMatrix.obj
 0001:0000dec0       ?tryAcquire@MemoryLocker@U2@@QAE_N_J@Z 1000eec0 f i DistanceMatrix.obj
 0001:0000e040       ?uniqueKeys@?$QMap@VQString@@H@@QBE?AV?$QList@VQString@@@@XZ 1000f040 f i DistanceMatrix.obj
 0001:0000e140       ?unsharableEmpty@?$QTypedArrayData@M@@SAPAU1@XZ 1000f140 f i DistanceMatrix.obj
 0001:0000e160       ?unsharableEmpty@?$QTypedArrayData@V?$QVector@M@@@@SAPAU1@XZ 1000f160 f i DistanceMatrix.obj
 0001:0000e180       ?value@const_iterator@?$QMap@VQString@@H@@QBEABHXZ 1000f180 f i DistanceMatrix.obj
 0001:0000e190       ?value@error_code@std@@QBEHXZ 1000f190 f i DistanceMatrix.obj
 0001:0000e1a0       ?value@error_condition@std@@QBEHXZ 1000f1a0 f i DistanceMatrix.obj
 0001:0000e1b0       ?value@iterator@?$QMap@VQString@@H@@QBEAAHXZ 1000f1b0 f i DistanceMatrix.obj
 0001:0000e1c0       _hypot                     1000f1c0 f i DistanceMatrix.obj
 0001:0000e1f0       ??0?$QScopedPointer@VDistanceMatrix@U2@@U?$QScopedPointerDeleter@VDistanceMatrix@U2@@@@@@QAE@PAVDistanceMatrix@U2@@@Z 1000f1f0 f i NeighborJoinAdapter.obj
 0001:0000e200       ??0?$QScopedPointer@VSeqBoot@U2@@U?$QScopedPointerDeleter@VSeqBoot@U2@@@@@@QAE@PAVSeqBoot@U2@@@Z 1000f200 f i NeighborJoinAdapter.obj
 0001:0000e210       ??0?$QSharedDataPointer@VPhyTreeData@U2@@@@QAE@PAVPhyTreeData@U2@@@Z 1000f210 f i NeighborJoinAdapter.obj
 0001:0000e230       ??0MemoryLocker@U2@@QAE@AAVU2OpStatus@1@HW4MemoryLockType@AppResource@1@@Z 1000f230 f i NeighborJoinAdapter.obj
 0001:0000e2e0       ??0NeighborJoinCalculateTreeTask@U2@@QAE@ABVMultipleSequenceAlignment@1@ABVCreatePhyTreeSettings@1@@Z 1000f2e0 f   NeighborJoinAdapter.obj
 0001:0000e3e0       ??1?$QScopedPointer@VDistanceMatrix@U2@@U?$QScopedPointerDeleter@VDistanceMatrix@U2@@@@@@QAE@XZ 1000f3e0 f i NeighborJoinAdapter.obj
 0001:0000e400       ??1?$QScopedPointer@VSeqBoot@U2@@U?$QScopedPointerDeleter@VSeqBoot@U2@@@@@@QAE@XZ 1000f400 f i NeighborJoinAdapter.obj
 0001:0000e420       ??1?$QSharedDataPointer@VPhyTreeData@U2@@@@QAE@XZ 1000f420 f i NeighborJoinAdapter.obj
 0001:0000e450       ??1NeighborJoinCalculateTreeTask@U2@@UAE@XZ 1000f450 f i NeighborJoinAdapter.obj
 0001:0000e4d0       ??4?$QSharedDataPointer@VPhyTreeData@U2@@@@QAEAAV0@ABV0@@Z 1000f4d0 f i NeighborJoinAdapter.obj
 0001:0000e520       ??4?$QSharedDataPointer@VPhyTreeData@U2@@@@QAEAAV0@PAVPhyTreeData@U2@@@Z 1000f520 f i NeighborJoinAdapter.obj
 0001:0000e570       ??C?$QScopedPointer@VDistanceMatrix@U2@@U?$QScopedPointerDeleter@VDistanceMatrix@U2@@@@@@QBEPAVDistanceMatrix@U2@@XZ 1000f570 f i NeighborJoinAdapter.obj
 0001:0000e580       ??C?$QScopedPointer@VSeqBoot@U2@@U?$QScopedPointerDeleter@VSeqBoot@U2@@@@@@QBEPAVSeqBoot@U2@@XZ 1000f580 f i NeighborJoinAdapter.obj
 0001:0000e590       ??_GDistanceMatrix@U2@@QAEPAXI@Z 1000f590 f i NeighborJoinAdapter.obj
 0001:0000e5c0       ??_GNeighborJoinCalculateTreeTask@U2@@UAEPAXI@Z 1000f5c0 f i NeighborJoinAdapter.obj
 0001:0000e5c0       ??_ENeighborJoinCalculateTreeTask@U2@@UAEPAXI@Z 1000f5c0 f i NeighborJoinAdapter.obj
 0001:0000e650       ??_GSeqBoot@U2@@QAEPAXI@Z  1000f650 f i NeighborJoinAdapter.obj
 0001:0000e680       ?c_str@?$basic_string@DU?$char_traits@D@std@@V?$allocator@D@2@@std@@QBEPBDXZ 1000f680 f i NeighborJoinAdapter.obj
 0001:0000e690       ?cleanup@?$QScopedPointerDeleter@VDistanceMatrix@U2@@@@SAXPAVDistanceMatrix@U2@@@Z 1000f690 f i NeighborJoinAdapter.obj
 0001:0000e6b0       ?cleanup@?$QScopedPointerDeleter@VSeqBoot@U2@@@@SAXPAVSeqBoot@U2@@@Z 1000f6b0 f i NeighborJoinAdapter.obj
 0001:0000e6d0       ?createCalculatePhyTreeTask@NeighborJoinAdapter@U2@@UAEPAVTask@2@ABVMultipleSequenceAlignment@2@ABVCreatePhyTreeSettings@2@@Z 1000f6d0 f   NeighborJoinAdapter.obj
 0001:0000e740       ?createPhyTreeFromPhylipTree@U2@@YAXABVMultipleSequenceAlignment@1@PAUnode@@NE1PAVPhyNode@1@H@Z 1000f740 f   NeighborJoinAdapter.obj
 0001:0000e9d0       ?createPhyTreeSettingsWidget@NeighborJoinAdapter@U2@@UAEPAVCreatePhyTreeWidget@2@ABVMultipleSequenceAlignment@2@PAVQWidget@@@Z 1000f9d0 f   NeighborJoinAdapter.obj
 0001:0000ea40       ?getErrorMessage@DistanceMatrix@U2@@QAEABVQString@@XZ 1000fa40 f i NeighborJoinAdapter.obj
 0001:0000ea50       ?replacePhylipRestrictedSymbols@U2@@YAXAAVQByteArray@@@Z 1000fa50 f   NeighborJoinAdapter.obj
 0001:0000ea90       ?run@NeighborJoinCalculateTreeTask@U2@@UAEXXZ 1000fa90 f   NeighborJoinAdapter.obj
 0001:0000fac0       ??$move@AAV?$QList@VQString@@@@@std@@YA$$QAV?$QList@VQString@@@@AAV1@@Z 10010ac0 f i NeighborJoinWidget.obj
 0001:0000fad0       ??$qAbs@H@@YAHABH@Z        10010ad0 f i NeighborJoinWidget.obj
 0001:0000fae0       ??0?$QFlags@W4AlignmentFlag@Qt@@@@QAE@PQPrivate@0@H@Z 10010ae0 f i NeighborJoinWidget.obj
 0001:0000faf0       ??0?$QFlags@W4MatchFlag@Qt@@@@QAE@VQFlag@@@Z 10010af0 f i NeighborJoinWidget.obj
 0001:0000fb00       ??0?$QFlags@W4MatchFlag@Qt@@@@QAE@W4MatchFlag@Qt@@@Z 10010b00 f i NeighborJoinWidget.obj
 0001:0000fb10       ??0?$QFlags@W4WindowType@Qt@@@@QAE@PQPrivate@0@H@Z 10010b10 f i NeighborJoinWidget.obj
 0001:0000fb20       ??0?$QList@VQString@@@@QAE@ABV0@@Z 10010b20 f i NeighborJoinWidget.obj
 0001:0000fbe0       ??0NeighborJoinWidget@U2@@QAE@ABVMultipleSequenceAlignment@1@PAVQWidget@@@Z 10010be0 f   NeighborJoinWidget.obj
 0001:0000fca0       ??0QFlag@@QAE@H@Z          10010ca0 f i NeighborJoinWidget.obj
 0001:0000fcb0       ??0QStringList@@QAE@$$QAV?$QList@VQString@@@@@Z 10010cb0 f i NeighborJoinWidget.obj
 0001:0000fcd0       ??1NeighborJoinWidget@U2@@UAE@XZ 10010cd0 f i NeighborJoinWidget.obj
 0001:0000fce0       ??1QStringList@@QAE@XZ     10010ce0 f i NeighborJoinWidget.obj
 0001:0000fcf0       ??BQFlag@@QBEHXZ           10010cf0 f i NeighborJoinWidget.obj
 0001:0000fd00       ??H@YA?BVQString@@ABV0@PBD@Z 10010d00 f i NeighborJoinWidget.obj
 0001:00010200       ??U?$QFlags@W4MatchFlag@Qt@@@@QBE?AV0@W4MatchFlag@Qt@@@Z 10011200 f i NeighborJoinWidget.obj
 0001:00010220       ??U@YA?AV?$QFlags@W4MatchFlag@Qt@@@@W4MatchFlag@Qt@@0@Z 10011220 f i NeighborJoinWidget.obj
 0001:00010230       ??_ENeighborJoinWidget@U2@@W7AEPAXI@Z 10011230 f i NeighborJoinWidget.obj
 0001:00010238       ??_EPhyTreeDisplayOptionsWidget@U2@@W7AEPAXI@Z 10011238 f i NeighborJoinWidget.obj
 0001:00010240       ??_EQCheckBox@@W7AEPAXI@Z  10011240 f i NeighborJoinWidget.obj
 0001:00010248       ??_EQComboBox@@W7AEPAXI@Z  10011248 f i NeighborJoinWidget.obj
 0001:00010250       ??_EQDoubleSpinBox@@W7AEPAXI@Z 10011250 f i NeighborJoinWidget.obj
 0001:00010258       ??_EQGridLayout@@W7AEPAXI@Z 10011258 f i NeighborJoinWidget.obj
 0001:00010260       ??_EQHBoxLayout@@W7AEPAXI@Z 10011260 f i NeighborJoinWidget.obj
 0001:00010268       ??_EQLabel@@W7AEPAXI@Z     10011268 f i NeighborJoinWidget.obj
 0001:00010270       ??_EQSpinBox@@W7AEPAXI@Z   10011270 f i NeighborJoinWidget.obj
 0001:00010278       ??_EQTabWidget@@W7AEPAXI@Z 10011278 f i NeighborJoinWidget.obj
 0001:00010280       ??_EQVBoxLayout@@W7AEPAXI@Z 10011280 f i NeighborJoinWidget.obj
 0001:00010288       ??_EQWidget@@W7AEPAXI@Z    10011288 f i NeighborJoinWidget.obj
 0001:00010290       ??_GNeighborJoinWidget@U2@@UAEPAXI@Z 10011290 f i NeighborJoinWidget.obj
 0001:00010290       ??_ENeighborJoinWidget@U2@@UAEPAXI@Z 10011290 f i NeighborJoinWidget.obj
 0001:000102c0       ??_EPhyTreeDisplayOptionsWidget@U2@@UAEPAXI@Z 100112c0 f i NeighborJoinWidget.obj
 0001:000102c0       ??_GPhyTreeDisplayOptionsWidget@U2@@UAEPAXI@Z 100112c0 f i NeighborJoinWidget.obj
 0001:000102f0       ??_EQCheckBox@@UAEPAXI@Z   100112f0 f i NeighborJoinWidget.obj
 0001:000102f0       ??_GQCheckBox@@UAEPAXI@Z   100112f0 f i NeighborJoinWidget.obj
 0001:00010320       ??_GQComboBox@@UAEPAXI@Z   10011320 f i NeighborJoinWidget.obj
 0001:00010320       ??_EQComboBox@@UAEPAXI@Z   10011320 f i NeighborJoinWidget.obj
 0001:00010350       ??_GQDoubleSpinBox@@UAEPAXI@Z 10011350 f i NeighborJoinWidget.obj
 0001:00010350       ??_EQDoubleSpinBox@@UAEPAXI@Z 10011350 f i NeighborJoinWidget.obj
 0001:00010380       ??_GQGridLayout@@UAEPAXI@Z 10011380 f i NeighborJoinWidget.obj
 0001:00010380       ??_EQGridLayout@@UAEPAXI@Z 10011380 f i NeighborJoinWidget.obj
 0001:000103b0       ??_EQHBoxLayout@@UAEPAXI@Z 100113b0 f i NeighborJoinWidget.obj
 0001:000103b0       ??_GQHBoxLayout@@UAEPAXI@Z 100113b0 f i NeighborJoinWidget.obj
 0001:000103e0       ??_GQLabel@@UAEPAXI@Z      100113e0 f i NeighborJoinWidget.obj
 0001:000103e0       ??_EQLabel@@UAEPAXI@Z      100113e0 f i NeighborJoinWidget.obj
 0001:00010410       ??_GQSpacerItem@@UAEPAXI@Z 10011410 f i NeighborJoinWidget.obj
 0001:00010410       ??_EQSpacerItem@@UAEPAXI@Z 10011410 f i NeighborJoinWidget.obj
 0001:00010440       ??_GQSpinBox@@UAEPAXI@Z    10011440 f i NeighborJoinWidget.obj
 0001:00010440       ??_EQSpinBox@@UAEPAXI@Z    10011440 f i NeighborJoinWidget.obj
 0001:00010470       ??_EQTabWidget@@UAEPAXI@Z  10011470 f i NeighborJoinWidget.obj
 0001:00010470       ??_GQTabWidget@@UAEPAXI@Z  10011470 f i NeighborJoinWidget.obj
 0001:000104a0       ??_EQVBoxLayout@@UAEPAXI@Z 100114a0 f i NeighborJoinWidget.obj
 0001:000104a0       ??_GQVBoxLayout@@UAEPAXI@Z 100114a0 f i NeighborJoinWidget.obj
 0001:000104d0       ??_GQWidget@@UAEPAXI@Z     100114d0 f i NeighborJoinWidget.obj
 0001:000104d0       ??_EQWidget@@UAEPAXI@Z     100114d0 f i NeighborJoinWidget.obj
 0001:00010500       ?checkMemoryEstimation@NeighborJoinWidget@U2@@UAE_NAAVQString@@ABVMultipleSequenceAlignment@2@ABVCreatePhyTreeSettings@2@@Z 10011500 f   NeighborJoinWidget.obj
 0001:00010660       ?checkSeed@NeighborJoinWidget@U2@@CA_NH@Z 10011660 f   NeighborJoinWidget.obj
 0001:00010690       ?checkSettings@NeighborJoinWidget@U2@@UAE_NAAVQString@@ABVCreatePhyTreeSettings@2@@Z 10011690 f   NeighborJoinWidget.obj
 0001:00010750       ?connectSignals@NeighborJoinWidget@U2@@AAEXXZ 10011750 f   NeighborJoinWidget.obj
 0001:000107b0       ?data_ptr@?$QStaticStringData@$05@@QBEPAU?$QTypedArrayData@G@@XZ 100117b0 f i NeighborJoinWidget.obj
 0001:000107c0       ?data_ptr@?$QStaticStringData@$06@@QBEPAU?$QTypedArrayData@G@@XZ 100117c0 f i NeighborJoinWidget.obj
 0001:000107d0       ?data_ptr@?$QStaticStringData@$07@@QBEPAU?$QTypedArrayData@G@@XZ 100117d0 f i NeighborJoinWidget.obj
 0001:000107e0       ?data_ptr@?$QStaticStringData@$08@@QBEPAU?$QTypedArrayData@G@@XZ 100117e0 f i NeighborJoinWidget.obj
 0001:000107f0       ?data_ptr@?$QStaticStringData@$09@@QBEPAU?$QTypedArrayData@G@@XZ 100117f0 f i NeighborJoinWidget.obj
 0001:00010800       ?data_ptr@?$QStaticStringData@$0BA@@@QBEPAU?$QTypedArrayData@G@@XZ 10011800 f i NeighborJoinWidget.obj
 0001:00010810       ?data_ptr@?$QStaticStringData@$0BB@@@QBEPAU?$QTypedArrayData@G@@XZ 10011810 f i NeighborJoinWidget.obj
 0001:00010820       ?data_ptr@?$QStaticStringData@$0BC@@@QBEPAU?$QTypedArrayData@G@@XZ 10011820 f i NeighborJoinWidget.obj
 0001:00010830       ?data_ptr@?$QStaticStringData@$0BD@@@QBEPAU?$QTypedArrayData@G@@XZ 10011830 f i NeighborJoinWidget.obj
 0001:00010840       ?data_ptr@?$QStaticStringData@$0BG@@@QBEPAU?$QTypedArrayData@G@@XZ 10011840 f i NeighborJoinWidget.obj
 0001:00010850       ?data_ptr@?$QStaticStringData@$0BJ@@@QBEPAU?$QTypedArrayData@G@@XZ 10011850 f i NeighborJoinWidget.obj
 0001:00010860       ?data_ptr@?$QStaticStringData@$0L@@@QBEPAU?$QTypedArrayData@G@@XZ 10011860 f i NeighborJoinWidget.obj
 0001:00010870       ?data_ptr@?$QStaticStringData@$0M@@@QBEPAU?$QTypedArrayData@G@@XZ 10011870 f i NeighborJoinWidget.obj
 0001:00010880       ?data_ptr@?$QStaticStringData@$0N@@@QBEPAU?$QTypedArrayData@G@@XZ 10011880 f i NeighborJoinWidget.obj
 0001:00010890       ?data_ptr@?$QStaticStringData@$0O@@@QBEPAU?$QTypedArrayData@G@@XZ 10011890 f i NeighborJoinWidget.obj
 0001:000108a0       ?data_ptr@?$QStaticStringData@$0P@@@QBEPAU?$QTypedArrayData@G@@XZ 100118a0 f i NeighborJoinWidget.obj
 0001:000108b0       ?fillSettings@NeighborJoinWidget@U2@@UAEXAAVCreatePhyTreeSettings@2@@Z 100118b0 f   NeighborJoinWidget.obj
 0001:000109d0       ?getConsensusModelTypes@ConsensusModelTypes@U2@@SA?AV?$QList@VQString@@@@XZ 100119d0 f   NeighborJoinWidget.obj
 0001:00010a60       ?getRandomSeed@NeighborJoinWidget@U2@@CAHXZ 10011a60 f   NeighborJoinWidget.obj
 0001:00010ae0       ?init@NeighborJoinWidget@U2@@AAEXABVMultipleSequenceAlignment@2@@Z 10011ae0 f   NeighborJoinWidget.obj
 0001:000112d0       ?isEmpty@?$QList@VQString@@@@QBE_NXZ 100122d0 f i NeighborJoinWidget.obj
 0001:000112e0       ?restoreDefault@NeighborJoinWidget@U2@@UAEXXZ 100122e0 f   NeighborJoinWidget.obj
 0001:000116a0       ?retranslateUi@Ui_NeighborJoinWidget@@QAEXPAVQWidget@@@Z 100126a0 f i NeighborJoinWidget.obj
 0001:000119d0       ?setupUi@Ui_NeighborJoinWidget@@QAEXPAVQWidget@@@Z 100129d0 f i NeighborJoinWidget.obj
 0001:00012e90       ?sl_onConsensusTypeChanged@NeighborJoinWidget@U2@@AAEXABVQString@@@Z 10013e90 f   NeighborJoinWidget.obj
 0001:00012f60       ?sl_onMatrixModelChanged@NeighborJoinWidget@U2@@AAEXABVQString@@@Z 10013f60 f   NeighborJoinWidget.obj
 0001:00012fc0       ?storeSettings@NeighborJoinWidget@U2@@UAEXXZ 10013fc0 f   NeighborJoinWidget.obj
 0001:000134d0       ?tr@NeighborJoinWidget@U2@@SA?AVQString@@PBD0H@Z 100144d0 f i NeighborJoinWidget.obj
 0001:00013500       ??0?$QHash@VQString@@V1@@@QAE@XZ 10014500 f i PhylipCmdlineTask.obj
 0001:00013510       ??0?$QHashNode@VQString@@V1@@@QAE@ABVQString@@0IPAU0@@Z 10014510 f i PhylipCmdlineTask.obj
 0001:00013580       ??0?$QList@VQByteArray@@@@QAE@ABV0@@Z 10014580 f i PhylipCmdlineTask.obj
 0001:00013640       ??0?$QMap@VQString@@VQVariant@@@@QAE@XZ 10014640 f i PhylipCmdlineTask.obj
 0001:00013650       ??0PhylipCmdlineTask@U2@@QAE@ABVMultipleSequenceAlignment@1@ABVCreatePhyTreeSettings@1@@Z 10014650 f   PhylipCmdlineTask.obj
 0001:00013760       ??0iterator@?$QList@VQByteArray@@@@QAE@PAUNode@1@@Z 10014760 f i PhylipCmdlineTask.obj
 0001:00013770       ??1?$QHash@VQString@@V1@@@QAE@XZ 10014770 f i PhylipCmdlineTask.obj
 0001:000137a0       ??1?$QHashNode@VQString@@V1@@@QAE@XZ 100147a0 f i PhylipCmdlineTask.obj
 0001:00013800       ??1?$QList@VQByteArray@@@@QAE@XZ 10014800 f i PhylipCmdlineTask.obj
 0001:00013860       ??1?$QMap@VQString@@VQVariant@@@@QAE@XZ 10014860 f i PhylipCmdlineTask.obj
 0001:000138b0       ??1PhylipCmdlineTask@U2@@UAE@XZ 100148b0 f   PhylipCmdlineTask.obj
 0001:00013940       ??6?$QList@PAVGObject@U2@@@@QAEAAV0@ABQAVGObject@U2@@@Z 10014940 f i PhylipCmdlineTask.obj
 0001:00013960       ??6QStringList@@QAEAAV0@ABVQString@@@Z 10014960 f i PhylipCmdlineTask.obj
 0001:00013980       ??A?$QHash@VQString@@V1@@@QAEAAVQString@@ABV1@@Z 10014980 f i PhylipCmdlineTask.obj
 0001:00013aa0       ??Diterator@?$QList@VQByteArray@@@@QBEAAVQByteArray@@XZ 10014aa0 f i PhylipCmdlineTask.obj
 0001:00013ab0       ??H@YA?BVQString@@PBDABV0@@Z 10014ab0 f i PhylipCmdlineTask.obj
 0001:00013b20       ??_G?$QHashNode@VQString@@V1@@@QAEPAXI@Z 10014b20 f i PhylipCmdlineTask.obj
 0001:00013b90       ??_GCmdlineInOutTaskRunner@U2@@UAEPAXI@Z 10014b90 f i PhylipCmdlineTask.obj
 0001:00013b90       ??_ECmdlineInOutTaskRunner@U2@@UAEPAXI@Z 10014b90 f i PhylipCmdlineTask.obj
 0001:00013bc0       ??_EPhyTreeObject@U2@@UAEPAXI@Z 10014bc0 f i PhylipCmdlineTask.obj
 0001:00013bc0       ??_GPhyTreeObject@U2@@UAEPAXI@Z 10014bc0 f i PhylipCmdlineTask.obj
 0001:00013bf0       ??_EPhylipCmdlineTask@U2@@UAEPAXI@Z 10014bf0 f i PhylipCmdlineTask.obj
 0001:00013bf0       ??_GPhylipCmdlineTask@U2@@UAEPAXI@Z 10014bf0 f i PhylipCmdlineTask.obj
 0001:00013ca0       ??_GQByteArray@@QAEPAXI@Z  10014ca0 f i PhylipCmdlineTask.obj
 0001:00013cd0       ??_GQVariant@@QAEPAXI@Z    10014cd0 f i PhylipCmdlineTask.obj
 0001:00013d00       ?alignOfNode@?$QHash@VQString@@V1@@@CAHXZ 10014d00 f i PhylipCmdlineTask.obj
 0001:00013d10       ?append@?$QList@PAVGObject@U2@@@@QAEXABQAVGObject@U2@@@Z 10014d10 f i PhylipCmdlineTask.obj
 0001:00013da0       ?begin@?$QList@VQByteArray@@@@QAE?AViterator@1@XZ 10014da0 f i PhylipCmdlineTask.obj
 0001:00013de0       ?concrete@?$QHash@VQString@@V1@@@CAPAU?$QHashNode@VQString@@V1@@@PAUNode@QHashData@@@Z 10014de0 f i PhylipCmdlineTask.obj
 0001:00013df0       ?createCmdlineTask@PhylipCmdlineTask@U2@@AAEXXZ 10014df0 f   PhylipCmdlineTask.obj
 0001:000143d0       ?createNode@?$QHash@VQString@@V1@@@AAEPAU?$QHashNode@VQString@@V1@@@IABVQString@@0PAPAU2@@Z 100153d0 f i PhylipCmdlineTask.obj
 0001:00014470       ?dealloc@?$QList@PAVGObject@U2@@@@AAEXPAUData@QListData@@@Z 10015470 f i PhylipCmdlineTask.obj
 0001:00014490       ?dealloc@?$QList@VQByteArray@@@@AAEXPAUData@QListData@@@Z 10015490 f i PhylipCmdlineTask.obj
 0001:000144d0       ?deleteNode2@?$QHash@VQString@@V1@@@CAXPAUNode@QHashData@@@Z 100154d0 f i PhylipCmdlineTask.obj
 0001:00014530       ?destroy@?$QMapData@VQString@@VQVariant@@@@QAEXXZ 10015530 f i PhylipCmdlineTask.obj
 0001:00014560       ?destroySubTree@?$QMapNode@VQString@@VQVariant@@@@QAEXXZ 10015560 f i PhylipCmdlineTask.obj
 0001:000145a0       ?detach@?$QHash@VQString@@V1@@@QAEXXZ 100155a0 f i PhylipCmdlineTask.obj
 0001:00014600       ?detach@?$QList@VQByteArray@@@@QAEXXZ 10015600 f i PhylipCmdlineTask.obj
 0001:00014620       ?detach_helper@?$QHash@VQString@@V1@@@AAEXXZ 10015620 f i PhylipCmdlineTask.obj
 0001:00014670       ?detach_helper@?$QList@VQByteArray@@@@AAEXH@Z 10015670 f i PhylipCmdlineTask.obj
 0001:00014760       ?detach_helper@?$QList@VQByteArray@@@@AAEXXZ 10015760 f i PhylipCmdlineTask.obj
 0001:00014770       ?detach_helper_grow@?$QList@PAVGObject@U2@@@@AAEPAUNode@1@HH@Z 10015770 f i PhylipCmdlineTask.obj
 0001:00014880       ?duplicateNode@?$QHash@VQString@@V1@@@CAXPAUNode@QHashData@@PAX@Z 10015880 f i PhylipCmdlineTask.obj
 0001:00014900       ?findNode@?$QHash@VQString@@V1@@@ABEPAPAU?$QHashNode@VQString@@V1@@@ABVQString@@PAI@Z 10015900 f i PhylipCmdlineTask.obj
 0001:00014990       ?first@?$QList@VQByteArray@@@@QAEAAVQByteArray@@XZ 10015990 f i PhylipCmdlineTask.obj
 0001:000149c0       ?freeData@?$QHash@VQString@@V1@@@AAEXPAUQHashData@@@Z 100159c0 f i PhylipCmdlineTask.obj
 0001:000149e0       ?isEmpty@?$QList@VQByteArray@@@@QBE_NXZ 100159e0 f i PhylipCmdlineTask.obj
 0001:000149f0       ?leftNode@?$QMapNode@VQString@@VQVariant@@@@QBEPAU1@XZ 100159f0 f i PhylipCmdlineTask.obj
 0001:00014a00       ?node_construct@?$QList@PAVGObject@U2@@@@AAEXPAUNode@1@ABQAVGObject@U2@@@Z 10015a00 f i PhylipCmdlineTask.obj
 0001:00014a20       ?node_copy@?$QList@PAVGObject@U2@@@@AAEXPAUNode@1@00@Z 10015a20 f i PhylipCmdlineTask.obj
 0001:00014a50       ?node_copy@?$QList@VQByteArray@@@@AAEXPAUNode@1@00@Z 10015a50 f i PhylipCmdlineTask.obj
 0001:00014af0       ?node_destruct@?$QList@PAVGObject@U2@@@@AAEXPAUNode@1@0@Z 10015af0 f i PhylipCmdlineTask.obj
 0001:00014b00       ?node_destruct@?$QList@PAVGObject@U2@@@@AAEXPAUNode@1@@Z 10015b00 f i PhylipCmdlineTask.obj
 0001:00014b10       ?node_destruct@?$QList@VQByteArray@@@@AAEXPAUNode@1@0@Z 10015b10 f i PhylipCmdlineTask.obj
 0001:00014b40       ?prepare@PhylipCmdlineTask@U2@@UAEXXZ 10015b40 f   PhylipCmdlineTask.obj
 0001:00014b80       ?prepareTempDbi@PhylipCmdlineTask@U2@@AAEXXZ 10015b80 f   PhylipCmdlineTask.obj
 0001:00014d70       ?report@PhylipCmdlineTask@U2@@UAE?AW4ReportResult@Task@2@XZ 10015d70 f   PhylipCmdlineTask.obj
 0001:00014f40       ?rightNode@?$QMapNode@VQString@@VQVariant@@@@QBEPAU1@XZ 10015f40 f i PhylipCmdlineTask.obj
 0001:00014f50       ?root@?$QMapData@VQString@@VQVariant@@@@QBEPAU?$QMapNode@VQString@@VQVariant@@@@XZ 10015f50 f i PhylipCmdlineTask.obj
 0001:00014f60       ?same_key@?$QHashNode@VQString@@V1@@@QBE_NIABVQString@@@Z 10015f60 f i PhylipCmdlineTask.obj
 0001:00014f90       ?t@Node@?$QList@VQByteArray@@@@QAEAAVQByteArray@@XZ 10015f90 f i PhylipCmdlineTask.obj
 0001:00014fa0       ?tr@PhylipCmdlineTask@U2@@SA?AVQString@@PBD0H@Z 10015fa0 f i PhylipCmdlineTask.obj
 0001:00014fd0       ??$qDeleteAll@V?$QList@PAVXMLTestFactory@U2@@@@@@YAXABV?$QList@PAVXMLTestFactory@U2@@@@@Z 10015fd0 f i PhylipPlugin.obj
 0001:00015010       ??$qDeleteAll@Vconst_iterator@?$QList@PAVXMLTestFactory@U2@@@@@@YAXVconst_iterator@?$QList@PAVXMLTestFactory@U2@@@@0@Z 10016010 f i PhylipPlugin.obj
 0001:00015040       ??$qobject_cast@PAVXMLTestFormat@U2@@@@YAPAVXMLTestFormat@U2@@PAVQObject@@@Z 10016040 f i PhylipPlugin.obj
 0001:00015060       ??0?$AbstractId@H@U2@@IAE@ABH@Z 10016060 f i PhylipPlugin.obj
 0001:00015080       ??0?$GAutoDeleteList@VXMLTestFactory@U2@@@U2@@QAE@PAVQObject@@@Z 10016080 f i PhylipPlugin.obj
 0001:000150b0       ??0?$QForeachContainer@V?$QList@PAVXMLTestFactory@U2@@@@@@QAE@ABV?$QList@PAVXMLTestFactory@U2@@@@@Z 100160b0 f i PhylipPlugin.obj
 0001:000150f0       ??0?$QList@PAVXMLTestFactory@U2@@@@QAE@ABV0@@Z 100160f0 f i PhylipPlugin.obj
 0001:000151b0       ??0?$QList@PAVXMLTestFactory@U2@@@@QAE@XZ 100161b0 f i PhylipPlugin.obj
 0001:000151c0       ??0AbstractInt32Id@U2@@IAE@H@Z 100161c0 f i PhylipPlugin.obj
 0001:000151e0       ??0NeighborJoinAdapter@U2@@QAE@XZ 100161e0 f i PhylipPlugin.obj
 0001:000151f0       ??0PhylipPlugin@U2@@QAE@XZ 100161f0 f   PhylipPlugin.obj
 0001:00015420       ??0ServiceType@U2@@QAE@H@Z 10016420 f i PhylipPlugin.obj
 0001:00015440       ??0const_iterator@?$QList@PAVXMLTestFactory@U2@@@@QAE@PAUNode@1@@Z 10016440 f i PhylipPlugin.obj
 0001:00015450       ??1?$AbstractId@H@U2@@MAE@XZ 10016450 f i PhylipPlugin.obj
 0001:00015460       ??1?$GAutoDeleteList@VXMLTestFactory@U2@@@U2@@UAE@XZ 10016460 f i PhylipPlugin.obj
 0001:00015520       ??1?$QForeachContainer@V?$QList@PAVXMLTestFactory@U2@@@@@@QAE@XZ 10016520 f i PhylipPlugin.obj
 0001:00015550       ??1?$QList@PAVXMLTestFactory@U2@@@@QAE@XZ 10016550 f i PhylipPlugin.obj
 0001:00015580       ??1AbstractInt32Id@U2@@UAE@XZ 10016580 f i PhylipPlugin.obj
 0001:00015590       ??1NeighborJoinAdapter@U2@@UAE@XZ 10016590 f i PhylipPlugin.obj
 0001:000155a0       ??1PhylipPlugin@U2@@UAE@XZ 100165a0 f i PhylipPlugin.obj
 0001:000155b0       ??1ServiceType@U2@@UAE@XZ  100165b0 f i PhylipPlugin.obj
 0001:000155c0       ??4?$QList@PAVXMLTestFactory@U2@@@@QAEAAV0@$$QAV0@@Z 100165c0 f i PhylipPlugin.obj
 0001:000155e0       ??9const_iterator@?$QList@PAVXMLTestFactory@U2@@@@QBE_NABV01@@Z 100165e0 f i PhylipPlugin.obj
 0001:00015600       ??Dconst_iterator@?$QList@PAVXMLTestFactory@U2@@@@QBEABQAVXMLTestFactory@U2@@XZ 10016600 f i PhylipPlugin.obj
 0001:00015610       ??Econst_iterator@?$QList@PAVXMLTestFactory@U2@@@@QAEAAV01@XZ 10016610 f i PhylipPlugin.obj
 0001:00015620       ??_E?$AbstractId@H@U2@@MAEPAXI@Z 10016620 f i PhylipPlugin.obj
 0001:00015620       ??_G?$AbstractId@H@U2@@MAEPAXI@Z 10016620 f i PhylipPlugin.obj
 0001:00015650       ??_G?$GAutoDeleteList@VXMLTestFactory@U2@@@U2@@UAEPAXI@Z 10016650 f i PhylipPlugin.obj
 0001:00015650       ??_E?$GAutoDeleteList@VXMLTestFactory@U2@@@U2@@UAEPAXI@Z 10016650 f i PhylipPlugin.obj
 0001:00015680       ??_GAbstractInt32Id@U2@@UAEPAXI@Z 10016680 f i PhylipPlugin.obj
 0001:00015680       ??_EAbstractInt32Id@U2@@UAEPAXI@Z 10016680 f i PhylipPlugin.obj
 0001:000156b0       ??_GNeighborJoinAdapter@U2@@UAEPAXI@Z 100166b0 f i PhylipPlugin.obj
 0001:000156b0       ??_ENeighborJoinAdapter@U2@@UAEPAXI@Z 100166b0 f i PhylipPlugin.obj
 0001:000156e0       ??_EPhylipPlugin@U2@@UAEPAXI@Z 100166e0 f i PhylipPlugin.obj
 0001:000156e0       ??_GPhylipPlugin@U2@@UAEPAXI@Z 100166e0 f i PhylipPlugin.obj
 0001:00015710       ??_GServiceType@U2@@UAEPAXI@Z 10016710 f i PhylipPlugin.obj
 0001:00015710       ??_EServiceType@U2@@UAEPAXI@Z 10016710 f i PhylipPlugin.obj
 0001:00015740       ??_ETaskStarter@U2@@UAEPAXI@Z 10016740 f i PhylipPlugin.obj
 0001:00015740       ??_GTaskStarter@U2@@UAEPAXI@Z 10016740 f i PhylipPlugin.obj
 0001:00015770       ?begin@?$QList@PAVXMLTestFactory@U2@@@@QBE?AVconst_iterator@1@XZ 10016770 f i PhylipPlugin.obj
 0001:00015790       ?dealloc@?$QList@PAVXMLTestFactory@U2@@@@AAEXPAUData@QListData@@@Z 10016790 f i PhylipPlugin.obj
 0001:000157b0       ?end@?$QList@PAVXMLTestFactory@U2@@@@QBE?AVconst_iterator@1@XZ 100167b0 f i PhylipPlugin.obj
 0001:000157d0       ?fetchSettings@?A0xabc90af7@U2@@YA?AVCreatePhyTreeSettings@2@XZ 100167d0 f   PhylipPlugin.obj
 0001:00015ab0       ?isValid@AbstractInt32Id@U2@@UBE_NXZ 10016ab0 f i PhylipPlugin.obj
 0001:00015ac0       ?node_copy@?$QList@PAVXMLTestFactory@U2@@@@AAEXPAUNode@1@00@Z 10016ac0 f i PhylipPlugin.obj
 0001:00015af0       ?node_destruct@?$QList@PAVXMLTestFactory@U2@@@@AAEXPAUNode@1@0@Z 10016af0 f i PhylipPlugin.obj
 0001:00015b00       ?processCmdlineOptions@PhylipPlugin@U2@@AAEXXZ 10016b00 f   PhylipPlugin.obj
 0001:00015db0       ?t@Node@?$QList@PAVXMLTestFactory@U2@@@@QAEAAPAVXMLTestFactory@U2@@XZ 10016db0 f i PhylipPlugin.obj
 0001:00015dc0       ?tr@PhylipPlugin@U2@@SA?AVQString@@PBD0H@Z 10016dc0 f i PhylipPlugin.obj
 0001:00015df0       _ugene_plugin_init         10016df0 f   PhylipPlugin.obj
 0001:00015e10       ??$getContext@VDocument@U2@@@GTest@U2@@SAPAVDocument@1@PBV01@ABVQString@@@Z 10016e10 f i PhylipPluginTests.obj
 0001:00015e30       ??$qobject_cast@PAVDocument@U2@@@@YAPAVDocument@U2@@PAVQObject@@@Z 10016e30 f i PhylipPluginTests.obj
 0001:00015e50       ??$qobject_cast@PAVMultipleSequenceAlignmentObject@U2@@@@YAPAVMultipleSequenceAlignmentObject@U2@@PAVQObject@@@Z 10016e50 f i PhylipPluginTests.obj
 0001:00015e70       ??$qobject_cast@PAVPhyTreeObject@U2@@@@YAPAVPhyTreeObject@U2@@PAVQObject@@@Z 10016e70 f i PhylipPluginTests.obj
 0001:00015e90       ??0?$QFlags@W4TaskFlag@U2@@@@QAE@VQFlag@@@Z 10016e90 f i PhylipPluginTests.obj
 0001:00015ea0       ??0?$QFlags@W4TaskFlag@U2@@@@QAE@W4TaskFlag@U2@@@Z 10016ea0 f i PhylipPluginTests.obj
 0001:00015eb0       ??0?$QList@PAVXMLTestFactory@U2@@@@QAE@$$QAV0@@Z 10016eb0 f i PhylipPluginTests.obj
 0001:00015ed0       ??0GTest_NeighborJoin@U2@@QAE@PAVXMLTestFormat@1@ABVQString@@PAVGTest@1@PBVGTestEnvironment@1@ABV?$QList@PAVGTest@U2@@@@ABVQDomElement@@@Z 10016ed0 f i PhylipPluginTests.obj
 0001:00015f60       ??0GTest_NeighborJoinFactory@GTest_NeighborJoin@U2@@QAE@XZ 10016f60 f i PhylipPluginTests.obj
 0001:00015fe0       ??0iterator@?$QList@PAVGObject@U2@@@@QAE@PAUNode@1@@Z 10016fe0 f i PhylipPluginTests.obj
 0001:00015ff0       ??1?$QList@PAVGObject@U2@@@@QAE@XZ 10016ff0 f i PhylipPluginTests.obj
 0001:00016020       ??1GTest_NeighborJoin@U2@@UAE@XZ 10017020 f i PhylipPluginTests.obj
 0001:00016090       ??1GTest_NeighborJoinFactory@GTest_NeighborJoin@U2@@UAE@XZ 10017090 f i PhylipPluginTests.obj
 0001:000160a0       ??B?$QSharedDataPointer@VPhyTreeData@U2@@@@QBEPBVPhyTreeData@U2@@XZ 100170a0 f i PhylipPluginTests.obj
 0001:000160b0       ??Diterator@?$QList@PAVGObject@U2@@@@QBEAAPAVGObject@U2@@XZ 100170b0 f i PhylipPluginTests.obj
 0001:000160c0       ??U?$QFlags@W4TaskFlag@U2@@@@QBE?AV0@W4TaskFlag@U2@@@Z 100170c0 f i PhylipPluginTests.obj
 0001:000160e0       ??_GGTest_NeighborJoin@U2@@UAEPAXI@Z 100170e0 f i PhylipPluginTests.obj
 0001:000160e0       ??_EGTest_NeighborJoin@U2@@UAEPAXI@Z 100170e0 f i PhylipPluginTests.obj
 0001:00016160       ??_EGTest_NeighborJoinFactory@GTest_NeighborJoin@U2@@UAEPAXI@Z 10017160 f i PhylipPluginTests.obj
 0001:00016160       ??_GGTest_NeighborJoinFactory@GTest_NeighborJoin@U2@@UAEPAXI@Z 10017160 f i PhylipPluginTests.obj
 0001:00016190       ??_EPhyTreeGeneratorLauncherTask@U2@@UAEPAXI@Z 10017190 f i PhylipPluginTests.obj
 0001:00016190       ??_GPhyTreeGeneratorLauncherTask@U2@@UAEPAXI@Z 10017190 f i PhylipPluginTests.obj
 0001:000161c0       ?append@?$QList@PAVXMLTestFactory@U2@@@@QAEXABQAVXMLTestFactory@U2@@@Z 100171c0 f i PhylipPluginTests.obj
 0001:00016250       ?begin@?$QList@PAVGObject@U2@@@@QAE?AViterator@1@XZ 10017250 f i PhylipPluginTests.obj
 0001:00016290       ?createFactory@GTest_NeighborJoin@U2@@SAPAVXMLTestFactory@2@XZ 10017290 f i PhylipPluginTests.obj
 0001:00016330       ?createTest@GTest_NeighborJoinFactory@GTest_NeighborJoin@U2@@UAEPAVGTest@3@PAVXMLTestFormat@3@ABVQString@@PAV43@PBVGTestEnvironment@3@ABV?$QList@PAVGTest@U2@@@@ABVQDomElement@@@Z 10017330 f i PhylipPluginTests.obj
 0001:000163f0       ?createTestFactories@PhylipPluginTests@U2@@SA?AV?$QList@PAVXMLTestFactory@U2@@@@XZ 100173f0 f   PhylipPluginTests.obj
 0001:00016460       ?detach@?$QList@PAVGObject@U2@@@@QAEXXZ 10017460 f i PhylipPluginTests.obj
 0001:00016480       ?detach_helper@?$QList@PAVGObject@U2@@@@AAEXH@Z 10017480 f i PhylipPluginTests.obj
 0001:00016550       ?detach_helper@?$QList@PAVGObject@U2@@@@AAEXXZ 10017550 f i PhylipPluginTests.obj
 0001:00016560       ?detach_helper_grow@?$QList@PAVXMLTestFactory@U2@@@@AAEPAUNode@1@HH@Z 10017560 f i PhylipPluginTests.obj
 0001:00016670       ?first@?$QList@PAVGObject@U2@@@@QAEAAPAVGObject@U2@@XZ 10017670 f i PhylipPluginTests.obj
 0001:000166a0       ?init@GTest_NeighborJoin@U2@@QAEXPAVXMLTestFormat@2@ABVQDomElement@@@Z 100176a0 f   PhylipPluginTests.obj
 0001:000168d0       ?node_construct@?$QList@PAVXMLTestFactory@U2@@@@AAEXPAUNode@1@ABQAVXMLTestFactory@U2@@@Z 100178d0 f i PhylipPluginTests.obj
 0001:000168f0       ?node_destruct@?$QList@PAVXMLTestFactory@U2@@@@AAEXPAUNode@1@@Z 100178f0 f i PhylipPluginTests.obj
 0001:00016900       ?prepare@GTest_NeighborJoin@U2@@UAEXXZ 10017900 f   PhylipPluginTests.obj
 0001:00016e00       ?report@GTest_NeighborJoin@U2@@UAE?AW4ReportResult@Task@2@XZ 10017e00 f   PhylipPluginTests.obj
 0001:00016f10       ?size@?$QList@PAVGObject@U2@@@@QBEHXZ 10017f10 f i PhylipPluginTests.obj
 0001:00016f20       ?t@Node@?$QList@PAVGObject@U2@@@@QAEAAPAVGObject@U2@@XZ 10017f20 f i PhylipPluginTests.obj
 0001:00016f30       ??0?$QList@VMultipleSequenceAlignmentRow@U2@@@@QAE@XZ 10017f30 f i PhylipTask.obj
 0001:00016f40       ??0PhylipTask@U2@@QAE@ABVU2EntityRef@1@ABVU2DbiRef@1@ABVCreatePhyTreeSettings@1@@Z 10017f40 f   PhylipTask.obj
 0001:00017000       ??1PhylipTask@U2@@UAE@XZ   10018000 f i PhylipTask.obj
 0001:00017080       ??_EMultipleSequenceAlignmentObject@U2@@UAEPAXI@Z 10018080 f i PhylipTask.obj
 0001:00017080       ??_GMultipleSequenceAlignmentObject@U2@@UAEPAXI@Z 10018080 f i PhylipTask.obj
 0001:000170b0       ??_GPhylipTask@U2@@UAEPAXI@Z 100180b0 f i PhylipTask.obj
 0001:000170b0       ??_EPhylipTask@U2@@UAEPAXI@Z 100180b0 f i PhylipTask.obj
 0001:00017140       ?prepare@PhylipTask@U2@@UAEXXZ 10018140 f   PhylipTask.obj
 0001:00017390       ?report@PhylipTask@U2@@UAE?AW4ReportResult@Task@2@XZ 10018390 f   PhylipTask.obj
 0001:00017410       ?saveTree@PhylipTask@U2@@AAE?AVQByteArray@@XZ 10018410 f   PhylipTask.obj
 0001:00017590       ?tr@PhylipTask@U2@@SA?AVQString@@PBD0H@Z 10018590 f i PhylipTask.obj
 0001:000175c0       ??$_Move@AAPAU?$QTypedArrayData@VMultipleSequenceAlignment@U2@@@@@std@@YA$$QAPAU?$QTypedArrayData@VMultipleSequenceAlignment@U2@@@@AAPAU1@@Z 100185c0 f i SeqBootAdapter.obj
 0001:000175d0       ??$qSwap@PAU?$QTypedArrayData@VMultipleSequenceAlignment@U2@@@@@@YAXAAPAU?$QTypedArrayData@VMultipleSequenceAlignment@U2@@@@0@Z 100185d0 f i SeqBootAdapter.obj
 0001:000175f0       ??$swap@PAU?$QTypedArrayData@VMultipleSequenceAlignment@U2@@@@@std@@YAXAAPAU?$QTypedArrayData@VMultipleSequenceAlignment@U2@@@@0@Z 100185f0 f i SeqBootAdapter.obj
 0001:00017610       ??0?$QVector@VMultipleSequenceAlignment@U2@@@@QAE@ABV0@@Z 10018610 f i SeqBootAdapter.obj
 0001:000176d0       ??0?$QVector@VMultipleSequenceAlignment@U2@@@@QAE@H@Z 100186d0 f i SeqBootAdapter.obj
 0001:00017730       ??0?$QVector@VMultipleSequenceAlignment@U2@@@@QAE@XZ 10018730 f i SeqBootAdapter.obj
 0001:00017740       ??0SeqBoot@U2@@QAE@XZ      10018740 f   SeqBootAdapter.obj
 0001:00017800       ??1?$QVector@VMultipleSequenceAlignment@U2@@@@QAE@XZ 10018800 f i SeqBootAdapter.obj
 0001:00017830       ??1SeqBoot@U2@@QAE@XZ      10018830 f   SeqBootAdapter.obj
 0001:000178c0       ??4?$QVector@VMultipleSequenceAlignment@U2@@@@QAE?AV0@$$QAV0@@Z 100188c0 f i SeqBootAdapter.obj
 0001:000178f0       ??A?$QVector@VMultipleSequenceAlignment@U2@@@@QAEAAVMultipleSequenceAlignment@U2@@H@Z 100188f0 f i SeqBootAdapter.obj
 0001:00017960       ??A?$QVector@VMultipleSequenceAlignment@U2@@@@QBEABVMultipleSequenceAlignment@U2@@H@Z 10018960 f i SeqBootAdapter.obj
 0001:00017980       ??_GMultipleSequenceAlignment@U2@@UAEPAXI@Z 10018980 f i SeqBootAdapter.obj
 0001:00017980       ??_EMultipleSequenceAlignment@U2@@UAEPAXI@Z 10018980 f i SeqBootAdapter.obj
 0001:000179b0       ?allocate@?$QTypedArrayData@VMultipleSequenceAlignment@U2@@@@SAPAU1@IV?$QFlags@W4AllocationOption@QArrayData@@@@@Z 100189b0 f i SeqBootAdapter.obj
 0001:000179d0       ?begin@?$QTypedArrayData@VMultipleSequenceAlignment@U2@@@@QAEPAVMultipleSequenceAlignment@U2@@PAV23@@Z 100189d0 f i SeqBootAdapter.obj
 0001:000179e0       ?clear@?$QVector@VMultipleSequenceAlignment@U2@@@@QAEXXZ 100189e0 f i SeqBootAdapter.obj
 0001:00017a90       ?clearGenratedSequences@SeqBoot@U2@@QAEXXZ 10018a90 f   SeqBootAdapter.obj
 0001:00017aa0       ?copyConstruct@?$QVector@VMultipleSequenceAlignment@U2@@@@AAEXPBVMultipleSequenceAlignment@U2@@0PAV23@@Z 10018aa0 f i SeqBootAdapter.obj
 0001:00017b20       ?data@?$QTypedArrayData@VMultipleSequenceAlignment@U2@@@@QAEPAVMultipleSequenceAlignment@U2@@XZ 10018b20 f i SeqBootAdapter.obj
 0001:00017b30       ?data@?$QVector@VMultipleSequenceAlignment@U2@@@@QAEPAVMultipleSequenceAlignment@U2@@XZ 10018b30 f i SeqBootAdapter.obj
 0001:00017b90       ?deallocate@?$QTypedArrayData@VMultipleSequenceAlignment@U2@@@@SAXPAUQArrayData@@@Z 10018b90 f i SeqBootAdapter.obj
 0001:00017bb0       ?defaultConstruct@?$QVector@VMultipleSequenceAlignment@U2@@@@AAEXPAVMultipleSequenceAlignment@U2@@0@Z 10018bb0 f i SeqBootAdapter.obj
 0001:00017d00       ?destruct@?$QVector@VMultipleSequenceAlignment@U2@@@@AAEXPAVMultipleSequenceAlignment@U2@@0@Z 10018d00 f i SeqBootAdapter.obj
 0001:00017d30       ?detach@?$QVector@VMultipleSequenceAlignment@U2@@@@QAEXXZ 10018d30 f i SeqBootAdapter.obj
 0001:00017d80       ?end@?$QTypedArrayData@VMultipleSequenceAlignment@U2@@@@QAEPAVMultipleSequenceAlignment@U2@@PAV23@@Z 10018d80 f i SeqBootAdapter.obj
 0001:00017da0       ?freeData@?$QVector@VMultipleSequenceAlignment@U2@@@@AAEXPAU?$QTypedArrayData@VMultipleSequenceAlignment@U2@@@@@Z 10018da0 f i SeqBootAdapter.obj
 0001:00017df0       ?generateSequencesFromAlignment@SeqBoot@U2@@QAEXABVMultipleSequenceAlignment@2@ABVCreatePhyTreeSettings@2@@Z 10018df0 f   SeqBootAdapter.obj
 0001:00017ff0       ?getMSA@SeqBoot@U2@@QBEABVMultipleSequenceAlignment@2@H@Z 10018ff0 f   SeqBootAdapter.obj
 0001:00018010       ?getTmpFileTemplate@SeqBoot@U2@@QAE?AVQString@@XZ 10019010 f   SeqBootAdapter.obj
 0001:00018120       ?initGenerSeq@SeqBoot@U2@@QAEXHHH@Z 10019120 f   SeqBootAdapter.obj
 0001:000183b0       ?isDetached@?$QVector@VMultipleSequenceAlignment@U2@@@@QBE_NXZ 100193b0 f i SeqBootAdapter.obj
 0001:000183e0       ?reallocData@?$QVector@VMultipleSequenceAlignment@U2@@@@AAEXHHV?$QFlags@W4AllocationOption@QArrayData@@@@@Z 100193e0 f i SeqBootAdapter.obj
 0001:00018620       ?sharedNull@?$QTypedArrayData@VMultipleSequenceAlignment@U2@@@@SAPAU1@XZ 10019620 f i SeqBootAdapter.obj
 0001:00018630       ?unsharableEmpty@?$QTypedArrayData@VMultipleSequenceAlignment@U2@@@@SAPAU1@XZ 10019630 f i SeqBootAdapter.obj
 0001:00018650       ?accumulate@@YAXPAUnode@@@Z 10019650 f   cons.obj
 0001:00018a80       ?bigsubset@@YAXPAHJ@Z      10019a80 f   cons.obj
 0001:00018c30       ?censor@@YAXXZ             10019c30 f   cons.obj
 0001:00018d20       ?clean_up_final@@YAXXZ     10019d20 f   cons.obj
 0001:00018df0       ?compatible@@YAEJJ@Z       10019df0 f   cons.obj
 0001:00018f10       ?compress@@YAXPAJ@Z        10019f10 f   cons.obj
 0001:00019030       ?consens_free_res@@YAXXZ   1001a030 f   cons.obj
 0001:000190f0       ?consens_starter@@YAXPBDN_N111@Z 1001a0f0 f   cons.obj
 0001:00019310       ?consensus@@YAXPAPAPAUpattern_elm@@J@Z 1001a310 f   cons.obj
 0001:00019630       ?coordinates@@YAXPAUnode@@PAJ@Z 1001a630 f   cons.obj
 0001:00019720       ?drawline@@YAXJ@Z          1001a720 f   cons.obj
 0001:00019ad0       ?dupname2@@YAXPADPAUnode@@1@Z 1001aad0 f   cons.obj
 0001:00019b60       ?dupname@@YAXPAUnode@@@Z   1001ab60 f   cons.obj
 0001:00019be0       ?elimboth@@YAXJ@Z          1001abe0 f   cons.obj
 0001:00019e40       ?eliminate@@YAXPAJ0@Z      1001ae40 f   cons.obj
 0001:00019fe0       ?enternodeset@@YAXPAUnode@@@Z 1001afe0 f   cons.obj
 0001:0001a330       ?enterpartition@@YAXPAHPAJ@Z 1001b330 f   cons.obj
 0001:0001a460       ?gdispose@@YAXPAUnode@@@Z  1001b460 f   cons.obj
 0001:0001a4c0       ?initconsnode@@YAXPAPAUnode@@0PAU1@JJPAJ2W4initops@@00PAD4PAU_iobuf@@@Z 1001b4c0 f   cons.obj
 0001:0001a760       ?initreenode@@YAXPAUnode@@@Z 1001b760 f   cons.obj
 0001:0001a7d0       ?missingname@@YAXPAUnode@@@Z 1001b7d0 f   cons.obj
 0001:0001a7f0       ?missingnameRecurs@@YAXPAUnode@@@Z 1001b7f0 f   cons.obj
 0001:0001a850       ?namesAdd@@YAXQAD@Z        1001b850 f   cons.obj
 0001:0001a8b0       ?namesCheckTable@@YAXXZ    1001b8b0 f   cons.obj
 0001:0001a940       ?namesClearTable@@YAXXZ    1001b940 f   cons.obj
 0001:0001a990       ?namesGetBucket@@YAJQAD@Z  1001b990 f   cons.obj
 0001:0001aa10       ?namesSearch@@YAEQAD@Z     1001ba10 f   cons.obj
 0001:0001aa80       ?printree@@YAXXZ           1001ba80 f   cons.obj
 0001:0001ac00       ?printset@@YAXJ@Z          1001bc00 f   cons.obj
 0001:0001ae30       ?read_groups@@YAXPAPAPAPAUpattern_elm@@JJPAU_iobuf@@@Z 1001be30 f   cons.obj
 0001:0001b2e0       ?reconstruct@@YAXJ@Z       1001c2e0 f   cons.obj
 0001:0001b340       ?recontraverse@@YAXPAPAUnode@@PAHJPAJ@Z 1001c340 f   cons.obj
 0001:0001b6c0       ?rehash@@YAXXZ             1001c6c0 f   cons.obj
 0001:0001ba50       ?reordertips@@YAXXZ        1001ca50 f   cons.obj
 0001:0001bb20       ?reorient@@YAXPAUnode@@@Z  1001cb20 f   cons.obj
 0001:0001bb80       ?reroot@@YAXPAUnode@@PAJ@Z 1001cb80 f   cons.obj
 0001:0001bd30       ?samename@@YAEQAD0@Z       1001cd30 f   cons.obj
 0001:0001bd50       ?sort@@YAXJ@Z              1001cd50 f   cons.obj
 0001:0001beb0       ?store_pattern@@YAXPAPAPAUpattern_elm@@H@Z 1001ceb0 f   cons.obj
 0001:0001c120       ?allocd@@YAXJPAPAUnode@@@Z 1001d120 f   dist.obj
 0001:0001c1c0       ?allocw@@YAXJPAPAUnode@@@Z 1001d1c0 f   dist.obj
 0001:0001c260       ?dist_alloctree@@YAXPAPAPAUnode@@JAAVMemoryLocker@U2@@@Z 1001d260 f   dist.obj
 0001:0001c310       ?dist_coordinates@@YAXPAUnode@@NPAJPAN0E@Z 1001d310 f   dist.obj
 0001:0001c460       ?dist_drawline@@YAXJNPAUnode@@E@Z 1001d460 f   dist.obj
 0001:0001c7c0       ?dist_freetree@@YAXPAPAPAUnode@@J@Z 1001d7c0 f   dist.obj
 0001:0001c860       ?dist_inputdata@@YAXEEEEPAPANPAPAJ@Z 1001d860 f   dist.obj
 0001:0001ccc0       ?dist_inputdata_modified@@YAXEEEEPAPANPAPAJ@Z 1001dcc0 f   dist.obj
 0001:0001cee0       ?dist_printree@@YAXPAUnode@@EEE@Z 1001dee0 f   dist.obj
 0001:0001cfb0       ?dist_setuptree@@YAXPAUtree@@J@Z 1001dfb0 f   dist.obj
 0001:0001d0b0       ?dist_treeout@@YAXPAUnode@@PAJNE0@Z 1001e0b0 f   dist.obj
 0001:0001d3d0       ?freed@@YAXJPAPAUnode@@@Z  1001e3d0 f   dist.obj
 0001:0001d450       ?freew@@YAXJPAPAUnode@@@Z  1001e450 f   dist.obj
 0001:0001d4d0       ?initname_modified@@YAXJ@Z 1001e4d0 f   dist.obj
 0001:0001d580       ?treeoutr@@YAXPAUnode@@PAJPAUtree@@@Z 1001e580 f   dist.obj
 0001:0001d830       ?allocrest@@YAXAAVMemoryLocker@U2@@@Z 1001e830 f   dnadist.obj
 0001:0001d9d0       ?dnadist_empiricalfreqs@@YAXXZ 1001e9d0 f   dnadist.obj
 0001:0001dba0       ?dnadist_makevalues@@YAXXZ 1001eba0 f   dnadist.obj
 0001:0001de50       ?dnadist_sitecombine@@YAXXZ 1001ee50 f   dnadist.obj
 0001:0001df60       ?dnadist_sitescrunch@@YAXXZ 1001ef60 f   dnadist.obj
 0001:0001e010       ?dnadist_sitesort@@YAXXZ   1001f010 f   dnadist.obj
 0001:0001e1a0       ?doinit@@YAXAAVMemoryLocker@U2@@@Z 1001f1a0 f   dnadist.obj
 0001:0001e1e0       ?getDNADistModelTypes@DNADistModelTypes@@SA?AV?$QList@VQString@@@@XZ 1001f1e0 f   dnadist.obj
 0001:0001e270       ?getDNADistSettings@@YAABVCreatePhyTreeSettings@U2@@XZ 1001f270 f   dnadist.obj
 0001:0001e280       ?getinput@@YAXXZ           1001f280 f   dnadist.obj
 0001:0001e540       ?getoptions@@YAXXZ         1001f540 f   dnadist.obj
 0001:0001e780       ?inittable@@YAXXZ          1001f780 f   dnadist.obj
 0001:0001e860       ?inputcategories@@YAXXZ    1001f860 f   dnadist.obj
 0001:0001e8f0       ?inputoptions@@YAXXZ       1001f8f0 f   dnadist.obj
 0001:0001ebc0       ?lndet@@YANPAY03N@Z        1001fbc0 f   dnadist.obj
 0001:0001ecb0       ?makedists@@YAXXZ          1001fcb0 f   dnadist.obj
 0001:0001ef80       ?makev@@YAXJJPAN@Z         1001ff80 f   dnadist.obj
 0001:00020680       ?makeweights@@YAXXZ        10021680 f   dnadist.obj
 0001:00020950       ?printcategories@@YAXXZ    10021950 f   dnadist.obj
 0001:00020a60       ?reallocsites@@YAXXZ       10021a60 f   dnadist.obj
 0001:00020b60       ?setDNADistSettings@U2@@YAXABVCreatePhyTreeSettings@1@@Z 10021b60 f   dnadist.obj
 0001:00020b80       ?writedists@@YAXXZ         10021b80 f   dnadist.obj
 0001:00020be0       ?describe@@YAXPAUnode@@N@Z 10021be0 f   neighbor.obj
 0001:00020d40       ?freerest@@YAXXZ           10021d40 f   neighbor.obj
 0001:00020dc0       ?getMtx@@YAPAPANXZ         10021dc0 f   neighbor.obj
 0001:00020dd0       ?getNayme@@YAPAY0BO@DXZ    10021dd0 f   neighbor.obj
 0001:00020de0       ?inputnumbers2_modified@@YAXPAJ0J@Z 10021de0 f   neighbor.obj
 0001:00020e00       ?jointree@@YAXXZ           10021e00 f   neighbor.obj
 0001:00021860       ?maketree@@YAXXZ           10022860 f   neighbor.obj
 0001:00021a50       ?neighbor_allocrest@@YAXXZ 10022a50 f   neighbor.obj
 0001:00021b20       ?neighbor_doinit@@YAXAAVMemoryLocker@U2@@@Z 10022b20 f   neighbor.obj
 0001:00021b90       ?neighbor_doinit_modified@@YAXAAVMemoryLocker@U2@@@Z 10022b90 f   neighbor.obj
 0001:00021c10       ?neighbor_getoptions@@YAXXZ 10022c10 f   neighbor.obj
 0001:00021c80       ?neighbor_inputoptions@@YAXXZ 10022c80 f   neighbor.obj
 0001:00021cb0       ?neighbour_calc_tree@@YAPBUtree@@XZ 10022cb0 f   neighbor.obj
 0001:00021d50       ?neighbour_free_resources@@YAXXZ 10022d50 f   neighbor.obj
 0001:00021da0       ?neighbour_init@@YAXHAAVMemoryLocker@U2@@ABVQString@@@Z 10022da0 f   neighbor.obj
 0001:00021e60       ?nodelabel@@YAXE@Z         10022e60 f   neighbor.obj
 0001:00021e90       ?summarize@@YAXXZ          10022e90 f   neighbor.obj
 0001:00021fa0       ??E@YAAAW4bases@@AAW40@H@Z 10022fa0 f   phylip.obj
 0001:00021fc0       ?EOF_error@@YAXXZ          10022fc0 f   phylip.obj
 0001:00021fe0       ?addelement2@@YAXPAUnode@@PADPAJPAU_iobuf@@PAPAU1@EPANPAE22J6EJ@Z 10022fe0 f   phylip.obj
 0001:00022370       ?addelement@@YAXPAPAUnode@@PAU1@PADPAJPAU_iobuf@@0PAE503350P6AX001JJ33W4initops@@00224@ZEJ@Z 10023370 f   phylip.obj
 0001:000226f0       ?addtree@@YAXJPAJE0PAUbestelm@@@Z 100236f0 f   phylip.obj
 0001:000227a0       ?allocate_nodep@@YAXPAPAPAUnode@@PAPAU_iobuf@@PAJ@Z 100237a0 f   phylip.obj
 0001:00022800       ?allocdiscnode@@YAXPAPAUnode@@PAJPAEJ@Z 10023800 f   phylip.obj
 0001:00022830       ?allocdiscnontip@@YAXPAUnode@@PAJPAEJ@Z 10023830 f   phylip.obj
 0001:00022980       ?allocnode@@YAXPAPAUnode@@PAJJ@Z 10023980 f   phylip.obj
 0001:000229b0       ?allocnontip@@YAXPAUnode@@PAJJ@Z 100239b0 f   phylip.obj
 0001:00022af0       ?chuck@@YAXPAPAUnode@@PAU1@@Z 10023af0 f   phylip.obj
 0001:00022b10       ?clear_connections@@YAXPAUtree@@J@Z 10023b10 f   phylip.obj
 0001:00022b70       ?cleerhome@@YAXXZ          10023b70 f   phylip.obj
 0001:00022ba0       ?commentskipper@@YAXPAPAPAU_iobuf@@PAJ@Z 10023ba0 f   phylip.obj
 0001:00022c80       ?count_sibs@@YAJPAUnode@@@Z 10023c80 f   phylip.obj
 0001:00022cd0       ?countcomma@@YAJPAPAU_iobuf@@PAJ@Z 10023cd0 f   phylip.obj
 0001:00022e70       ?countsemic@@YAJPAPAU_iobuf@@@Z 10023e70 f   phylip.obj
 0001:00022fb0       ?countup@@YAXPAJJ@Z        10023fb0 f   phylip.obj
 0001:00023080       ?eoff@@YAEPAU_iobuf@@@Z    10024080 f   phylip.obj
 0001:000230d0       ?eoln@@YAEPAU_iobuf@@@Z    100240d0 f   phylip.obj
 0001:00023110       ?exxit@@YAXH@Z             10024110 f   phylip.obj
 0001:00023130       ?fieldwidth_double@@YAHNI@Z 10024130 f   phylip.obj
 0001:000231a0       ?filexists@@YAHPAD@Z       100241a0 f   phylip.obj
 0001:000231d0       ?findch2@@YAXDPAJ0PAD@Z    100241d0 f   phylip.obj
 0001:00023310       ?findch@@YAXDPADJ@Z        10024310 f   phylip.obj
 0001:000233f0       ?findtree@@YAXPAEPAJJ1PAUbestelm@@@Z 100243f0 f   phylip.obj
 0001:000234c0       ?findunrearranged@@YAJPAUbestelm@@JE@Z 100244c0 f   phylip.obj
 0001:00023510       ?getTaskInfo@U2@@YAPAVTaskStateInfo@1@XZ 10024510 f   phylip.obj
 0001:00023520       ?get_command_name@@YAPBDPBD@Z 10024520 f   phylip.obj
 0001:00023540       ?getch2@@YAXPADPAJ@Z       10024540 f   phylip.obj
 0001:00023630       ?getch@@YAXPADPAJPAU_iobuf@@@Z 10024630 f   phylip.obj
 0001:00023700       ?getstryng@@YAXPAD@Z       10024700 f   phylip.obj
 0001:00023750       ?gettc@@YADPAU_iobuf@@@Z   10024750 f   phylip.obj
 0001:000237a0       ?glaguerre@@YANJNN@Z       100247a0 f   phylip.obj
 0001:00023860       ?gnu@@YAXPAPAUnode@@0@Z    10024860 f   phylip.obj
 0001:000238f0       ?gnudisctreenode@@YAXPAPAUnode@@0JJPAJPAE@Z 100248f0 f   phylip.obj
 0001:000239e0       ?gnutreenode@@YAXPAPAUnode@@0JJPAJ@Z 100249e0 f   phylip.obj
 0001:00023ad0       ?halfroot@@YANP6ANJN@ZJNN@Z 10024ad0 f   phylip.obj
 0001:00023cf0       ?headings@@YAXJPBD0@Z      10024cf0 f   phylip.obj
 0001:00023dd0       ?hermite@@YANJN@Z          10024dd0 f   phylip.obj
 0001:00023f70       ?hermite_weight@@YAXJPAN0@Z 10024f70 f   phylip.obj
 0001:00024020       ?hookup@@YAXPAUnode@@0@Z   10025020 f   phylip.obj
 0001:00024040       ?init@@YAXHPAPAD@Z         10025040 f   phylip.obj
 0001:00024090       ?initbestrees@@YAXPAUbestelm@@JE@Z 10025090 f   phylip.obj
 0001:000240d0       ?initcategs@@YAXJPAN@Z     100250d0 f   phylip.obj
 0001:000242d0       ?initcatn@@YAXPAJ@Z        100252d0 f   phylip.obj
 0001:00024350       ?initdatasets@@YAXPAJ@Z    10025350 f   phylip.obj
 0001:000243d0       ?initfreqs@@YAXPAN000@Z    100253d0 f   phylip.obj
 0001:00024500       ?initgammacat@@YAXJNPAN0@Z 10025500 f   phylip.obj
 0001:00024540       ?inithermitcat@@YAXJNPAN0@Z 10025540 f   phylip.obj
 0001:000247f0       ?inithowmany@@YAXPAJJ@Z    100257f0 f   phylip.obj
 0001:00024860       ?inithowoften@@YAXPAJ@Z    10025860 f   phylip.obj
 0001:000248d0       ?initjumble@@YAXPAJ0QAJ0@Z 100258d0 f   phylip.obj
 0001:00024950       ?initlaguerrecat@@YAXJNPAN0@Z 10025950 f   phylip.obj
 0001:00024be0       ?initlambda@@YAXPAN@Z      10025be0 f   phylip.obj
 0001:00024c60       ?initname@@YAXJ@Z          10025c60 f   phylip.obj
 0001:00024df0       ?initnumlines@@YAXPAJ@Z    10025df0 f   phylip.obj
 0001:00024e40       ?initoutgroup@@YAXPAJJ@Z   10025e40 f   phylip.obj
 0001:00024ed0       ?initpower@@YAXPAN@Z       10025ed0 f   phylip.obj
 0001:00024f20       ?initprobcat@@YAXJPAN0@Z   10025f20 f   phylip.obj
 0001:000251e0       ?initratio@@YAXPAN@Z       100261e0 f   phylip.obj
 0001:00025260       ?initseed@@YAXPAJ0QAJ@Z    10026260 f   phylip.obj
 0001:00025330       ?initterminal@@YAXPAE0@Z   10026330 f   phylip.obj
 0001:00025360       ?initthreshold@@YAXPAN@Z   10026360 f   phylip.obj
 0001:00025410       ?inittrav@@YAXPAUnode@@@Z  10026410 f   phylip.obj
 0001:00025450       ?inputcategs@@YAXJJPAJJPBD@Z 10026450 f   phylip.obj
 0001:00025550       ?inputfactors@@YAXJPADPAE@Z 10026550 f   phylip.obj
 0001:00025610       ?inputnumbers2@@YAXPAJ0J@Z 10026610 f   phylip.obj
 0001:00025680       ?inputnumbers3@@YAXPAJ0@Z  10026680 f   phylip.obj
 0001:000256e0       ?inputnumbers@@YAXPAJ00J@Z 100266e0 f   phylip.obj
 0001:00025740       ?inputnumbersold@@YAXPAJ00J@Z 10026740 f   phylip.obj
 0001:000257a0       ?inputweights2@@YAXJJPAJ0PAEPBD@Z 100267a0 f   phylip.obj
 0001:000258b0       ?inputweights@@YAXJPAJPAE@Z 100268b0 f   phylip.obj
 0001:00025a00       ?inputweightsold@@YAXJPAJPAE@Z 10026a00 f   phylip.obj
 0001:00025b70       ?isBootstr@U2@@YA_NXZ      10026b70 f   phylip.obj
 0001:00025b80       ?justweights@@YAXPAJ@Z     10026b80 f   phylip.obj
 0001:00025c00       ?lgr@@YAXJNQAY0L@N@Z       10026c00 f   phylip.obj
 0001:00025dd0       ?link_trees@@YAXJJJPAPAUnode@@@Z 10026dd0 f   phylip.obj
 0001:00025e40       ?logfac@@YANJ@Z            10026e40 f   phylip.obj
 0001:00025f60       ?malloc_pheno@@YAXPAUnode@@JJ@Z 10026f60 f   phylip.obj
 0001:00026010       ?malloc_ppheno@@YAXPAUnode@@JJ@Z 10027010 f   phylip.obj
 0001:000260d0       ?match_names_to_data@@YAXPADPAPAUnode@@1J@Z 100270d0 f   phylip.obj
 0001:00026220       ?matchoptions@@YAXPADPBD@Z 10027220 f   phylip.obj
 0001:000262d0       ?memerror@@YAXXZ           100272d0 f   phylip.obj
 0001:00026310       ?mymalloc@@YAPAXJ@Z        10027310 f   phylip.obj
 0001:00026340       ?newline@@YAXPAU_iobuf@@JJJ@Z 10027340 f   phylip.obj
 0001:00026390       ?normrand@@YANQAJ@Z        10027390 f   phylip.obj
 0001:00026440       ?odd_malloc@@YAXJ@Z        10027440 f   phylip.obj
 0001:000264a0       ?openfile@@YAXPAPAU_iobuf@@PBD111PAD@Z 100274a0 f   phylip.obj
 0001:00026a70       ?output_matrix_d@@YAXPAU_iobuf@@PAPANKKPAPAD2H@Z 10027a70 f   phylip.obj
 0001:000270c0       ?phyClearScreen@@YAXXZ     100280c0 f   phylip.obj
 0001:00027150       ?phyFillScreenColor@@YAXXZ 10028150 f   phylip.obj
 0001:000271b0       ?phyRestoreConsoleAttributes@@YAXXZ 100281b0 f   phylip.obj
 0001:00027230       ?phySaveConsoleAttributes@@YAXXZ 10028230 f   phylip.obj
 0001:00027260       ?phySetConsoleAttributes@@YAXXZ 10028260 f   phylip.obj
 0001:000272c0       ?pnode@@YAPAUnode@@PAUtree@@PAU1@@Z 100282c0 f   phylip.obj
 0001:000272e0       ?printcategs@@YAXPAU_iobuf@@JPAJPBD@Z 100282e0 f   phylip.obj
 0001:000273a0       ?printfactors@@YAXPAU_iobuf@@JPADPBD@Z 100283a0 f   phylip.obj
 0001:00027470       ?printweights@@YAXPAU_iobuf@@JJPAJPBD@Z 10028470 f   phylip.obj
 0001:000275a0       ?processlength@@YAXPAN0PADPAEPAU_iobuf@@PAJ@Z 100285a0 f   phylip.obj
 0001:000277a0       ?randum@@YANQAJ@Z          100287a0 f   phylip.obj
 0001:00027a40       ?randumize@@YAXQAJPAJ@Z    10028a40 f   phylip.obj
 0001:00027d40       ?readlong@@YAJPBD@Z        10028d40 f   phylip.obj
 0001:00027e50       ?readoptions@@YAXPAJPBD@Z  10028e50 f   phylip.obj
 0001:00027f60       ?reducebestrees@@YAXPAUbestelm@@PAJ@Z 10028f60 f   phylip.obj
 0001:00028000       ?root_hermite@@YAXJPAN@Z   10029000 f   phylip.obj
 0001:000280d0       ?samenumsp2@@YAXJ@Z        100290d0 f   phylip.obj
 0001:00028190       ?samenumsp@@YAXPAJJ@Z      10029190 f   phylip.obj
 0001:00028240       ?scan_eoln@@YAXPAU_iobuf@@@Z 10029240 f   phylip.obj
 0001:00028330       ?setBootstr@U2@@YAX_N@Z    10029330 f   phylip.obj
 0001:00028340       ?setTaskInfo@U2@@YAXPAVTaskStateInfo@1@@Z 10029340 f   phylip.obj
 0001:00028350       ?setupnode@@YAXPAUnode@@J@Z 10029350 f   phylip.obj
 0001:00028380       ?shellsort@@YAXPANPAJJ@Z   10029380 f   phylip.obj
 0001:000284a0       ?stringnames_delete@@YAXPAPAD@Z 100294a0 f   phylip.obj
 0001:000284e0       ?stringnames_new@@YAPAPADXZ 100294e0 f   phylip.obj
 0001:000285a0       ?strpbrk@@YAPADPADPBD@Z    100295a0 f i phylip.obj
 0001:000285b0       ?take_name_from_tree@@YAJPAD0PAU_iobuf@@@Z 100295b0 f   phylip.obj
 0001:00028680       ?torearrange@@YAEPAUbestelm@@J@Z 10029680 f   phylip.obj
 0001:000286e0       ?treeread2@@YAXPAU_iobuf@@PAPAUnode@@1EPANPAE3PAJEJ@Z 100296e0 f   phylip.obj
 0001:000288a0       ?treeread@@YAXPAU_iobuf@@PAPAUnode@@1PAE21PAJ21P6AX11PAU2@JJ33W4initops@@11PAD60@ZEJ@Z 100298a0 f   phylip.obj
 0001:00028a60       ?ugene_exit@@YAXPBD@Z      10029a60 f   phylip.obj
 0001:00028a80       ?unhookup@@YAXPAUnode@@0@Z 10029a80 f   phylip.obj
 0001:00028aa0       ?unroot@@YAXPAUtree@@J@Z   10029aa0 f   phylip.obj
 0001:00028b30       ?unroot_here@@YAXPAUnode@@PAPAU1@J@Z 10029b30 f   phylip.obj
 0001:00028bf0       ?unroot_r@@YAXPAUnode@@PAPAU1@J@Z 10029bf0 f   phylip.obj
 0001:00028cf0       ?uppercase@@YAXPAD@Z       10029cf0 f   phylip.obj
 0001:00028d20       ?writename@@YAXJJPAJ@Z     10029d20 f   phylip.obj
 0001:00028da0       ?zerodiscnumnuc@@YAXPAUnode@@J@Z 10029da0 f   phylip.obj
 0001:00028e30       ?zeronumnuc@@YAXPAUnode@@J@Z 10029e30 f   phylip.obj
 0001:00028ea0       ?code@@YAXXZ               10029ea0 f   protdist.obj
 0001:00029020       ?coeffs@@YAXNNPAN0N@Z      1002a020 f   protdist.obj
 0001:000290a0       ?doinput@@YAXXZ            1002a0a0 f   protdist.obj
 0001:00029330       ?getProtDistModelTypes@ProtDistModelTypes@@SA?AV?$QList@VQString@@@@XZ 1002a330 f   protdist.obj
 0001:000293c0       ?givens@@YAXQAY0BE@NJJJNNE@Z 1002a3c0 f   protdist.obj
 0001:000294b0       ?jtteigen@@YAXXZ           1002a4b0 f   protdist.obj
 0001:000294f0       ?maketrans@@YAXXZ          1002a4f0 f   protdist.obj
 0001:00029a60       ?pameigen@@YAXXZ           1002aa60 f   protdist.obj
 0001:00029aa0       ?pmbeigen@@YAXXZ           1002aaa0 f   protdist.obj
 0001:00029ae0       ?predict@@YAXJJJ@Z         1002aae0 f   protdist.obj
 0001:00029d90       ?prot_doinit@@YAXABVCreatePhyTreeSettings@U2@@AAVMemoryLocker@2@@Z 1002ad90 f   protdist.obj
 0001:00029dd0       ?prot_getoptions@@YAXABVQString@@@Z 1002add0 f   protdist.obj
 0001:00029f90       ?prot_inputoptions@@YAXXZ  1002af90 f   protdist.obj
 0001:0002a1e0       ?prot_makedists@@YAXXZ     1002b1e0 f   protdist.obj
 0001:0002a9c0       ?prot_printcategories@@YAXXZ 1002b9c0 f   protdist.obj
 0001:0002a9d0       ?protdist_cats@@YAXXZ      1002b9d0 f   protdist.obj
 0001:0002ab30       ?protdist_inputdata@@YAXXZ 1002bb30 f   protdist.obj
 0001:0002b3a0       ?protdist_inputnumbers@@YAXAAVMemoryLocker@U2@@@Z 1002c3a0 f   protdist.obj
 0001:0002b500       ?protdist_uppercase@@YAXPAD@Z 1002c500 f   protdist.obj
 0001:0002b530       ?qreigen@@YAXQAY0BE@NJ@Z   1002c530 f   protdist.obj
 0001:0002b6a0       ?reallocchars@@YAXXZ       1002c6a0 f   protdist.obj
 0001:0002b740       ?shiftqr@@YAXQAY0BE@NJN@Z  1002c740 f   protdist.obj
 0001:0002baa0       ?transition@@YAXXZ         1002caa0 f   protdist.obj
 0001:0002bb80       ?tridiag@@YAXQAY0BE@NJN@Z  1002cb80 f   protdist.obj
 0001:0002bd50       ?add@@YAXPAUnode@@00PAPAU1@E11PAJ@Z 1002cd50 f   seq.obj
 0001:0002c160       ?addbestever@@YAXPAJ0JE0PAUbestelm@@@Z 1002d160 f   seq.obj
 0001:0002c1b0       ?addnsave@@YAXPAUnode@@00PAPAU1@1E1PAJ2@Z 1002d1b0 f   seq.obj
 0001:0002c220       ?addtiedtree@@YAXJPAJJE0PAUbestelm@@@Z 1002d220 f   seq.obj
 0001:0002c250       ?allcommonbases@@YAEPAUnode@@0PAE@Z 1002d250 f   seq.obj
 0001:0002c2b0       ?alloctemp@@YAXPAPAUnode@@PAJJ@Z 1002d2b0 f   seq.obj
 0001:0002c340       ?alloctip@@YAXPAUnode@@PAJ@Z 1002d340 f   seq.obj
 0001:0002c400       ?alloctree@@YAXPAPAPAUnode@@JE@Z 1002d400 f   seq.obj
 0001:0002c500       ?allocx@@YAXJJPAPAUnode@@E@Z 1002d500 f   seq.obj
 0001:0002c630       ?alltips@@YAEPAUnode@@0@Z  1002d630 f   seq.obj
 0001:0002c670       ?backtobinary@@YAXPAPAUnode@@PAU1@0@Z 1002d670 f   seq.obj
 0001:0002c6e0       ?bintomulti@@YAXPAPAUnode@@00PAJ@Z 1002d6e0 f   seq.obj
 0001:0002c790       ?branchlength@@YAXPAUnode@@0PANPAPAU1@@Z 1002d790 f   seq.obj
 0001:0002c920       ?branchlentrav@@YAXPAUnode@@0JJPANPAPAU1@@Z 1002d920 f   seq.obj
 0001:0002cb70       ?chuckbase@@YAXPAUgbases@@PAPAU1@@Z 1002db70 f   seq.obj
 0001:0002cb90       ?clearbottom@@YAXPAPAUnode@@@Z 1002db90 f   seq.obj
 0001:0002cbe0       ?clearcollapse@@YAXPAPAUnode@@@Z 1002dbe0 f   seq.obj
 0001:0002cc30       ?clearvisited@@YAXPAPAUnode@@@Z 1002dc30 f   seq.obj
 0001:0002cc80       ?collabranch@@YAXPAUnode@@00@Z 1002dc80 f   seq.obj
 0001:0002cfd0       ?collapsebestrees@@YAXPAPAUnode@@00PAUbestelm@@PAJ2JEE@Z 1002dfd0 f   seq.obj
 0001:0002d2d0       ?collapsetree@@YAXPAUnode@@0PAPAU1@1PAJ@Z 1002e2d0 f   seq.obj
 0001:0002d4a0       ?collapsible@@YAEPAUnode@@0000000E0PAJPAPAU1@@Z 1002e4a0 f   seq.obj
 0001:0002d7f0       ?compmin@@YAXPAUnode@@0@Z  1002e7f0 f   seq.obj
 0001:0002d8d0       ?coordinates@@YAXPAUnode@@PAJN1@Z 1002e8d0 f   seq.obj
 0001:0002da50       ?copy_@@YAXPAUtree@@0JJ@Z  1002ea50 f   seq.obj
 0001:0002dbc0       ?copynode@@YAXPAUnode@@0J@Z 1002ebc0 f   seq.obj
 0001:0002dcc0       ?drawline2@@YAXJNUtree@@@Z 1002ecc0 f   seq.obj
 0001:0002dcf0       ?drawline3@@YAXJNPAUnode@@@Z 1002ecf0 f   seq.obj
 0001:0002dfd0       ?drawline@@YAXJNPAUnode@@@Z 1002efd0 f   seq.obj
 0001:0002e2b0       ?empiricalfreqs@@YAXPAN000PAJPAPAUnode@@@Z 1002f2b0 f   seq.obj
 0001:0002e4c0       ?fdrawline2@@YAXPAU_iobuf@@JNPAUtree@@@Z 1002f4c0 f   seq.obj
 0001:0002e7e0       ?fillin@@YAXPAUnode@@00@Z  1002f7e0 f   seq.obj
 0001:0002ea70       ?findbelow@@YAXPAPAUnode@@PAU1@1@Z 1002fa70 f   seq.obj
 0001:0002ea90       ?findbottom@@YAXPAUnode@@PAPAU1@@Z 1002fa90 f   seq.obj
 0001:0002ead0       ?fix_protx@@YAXPAUnode@@JNJ@Z 1002fad0 f   seq.obj
 0001:0002eb80       ?fix_x@@YAXPAUnode@@JNJ@Z  1002fb80 f   seq.obj
 0001:0002ec20       ?flipindexes@@YAXJPAPAUnode@@@Z 1002fc20 f   seq.obj
 0001:0002eca0       ?flipnodes@@YAXPAUnode@@0@Z 1002fca0 f   seq.obj
 0001:0002ecc0       ?freegarbage@@YAXPAPAUgbases@@@Z 1002fcc0 f   seq.obj
 0001:0002ecf0       ?freegrbg@@YAXPAPAUnode@@@Z 1002fcf0 f   seq.obj
 0001:0002ed50       ?freenode@@YAXPAPAUnode@@@Z 1002fd50 f   seq.obj
 0001:0002eda0       ?freenodes@@YAXJPAPAUnode@@@Z 1002fda0 f   seq.obj
 0001:0002ee80       ?freenontip@@YAXPAUnode@@@Z 1002fe80 f   seq.obj
 0001:0002eec0       ?freetemp@@YAXPAPAUnode@@@Z 1002fec0 f   seq.obj
 0001:0002ef00       ?freetip@@YAXPAUnode@@@Z   1002ff00 f   seq.obj
 0001:0002ef40       ?freetree2@@YAXPAPAUnode@@J@Z 1002ff40 f   seq.obj
 0001:0002efc0       ?freetree@@YAXJPAPAUnode@@@Z 1002ffc0 f   seq.obj
 0001:0002f040       ?freex@@YAXJPAPAUnode@@@Z  10030040 f   seq.obj
 0001:0002f130       ?freex_notip@@YAXJPAPAUnode@@@Z 10030130 f   seq.obj
 0001:0002f1c0       ?gdispose@@YAXPAUnode@@PAPAU1@1@Z 100301c0 f   seq.obj
 0001:0002f230       ?getbasefreqs@@YAXNNNNPAN000000000EE@Z 10030230 f   seq.obj
 0001:0002f4f0       ?getlargest@@YAJPAJ@Z      100304f0 f   seq.obj
 0001:0002f530       ?getnufork@@YAXPAPAUnode@@00PAJ@Z 10030530 f   seq.obj
 0001:0002f580       ?gnubase@@YAXPAPAUgbases@@0J@Z 10030580 f   seq.obj
 0001:0002f5d0       ?hyprint@@YAXJJPAULOC_hyptrav@@PAPAUnode@@PAD@Z 100305d0 f   seq.obj
 0001:0002f860       ?hypstates@@YAXJPAUnode@@PAPAU1@PAPAUgbases@@PAD@Z 10030860 f   seq.obj
 0001:0002f950       ?hyptrav@@YAXPAUnode@@PAJJJEPAPAU1@PAPAUgbases@@PAD@Z 10030950 f   seq.obj
 0001:0002fe40       ?initbase@@YAXPAUnode@@J@Z 10030e40 f   seq.obj
 0001:000300a0       ?initbranchlen@@YAXPAUnode@@@Z 100310a0 f   seq.obj
 0001:00030110       ?initmin@@YAXPAUnode@@JE@Z 10031110 f   seq.obj
 0001:00030290       ?inittreetrav@@YAXPAUnode@@J@Z 10031290 f   seq.obj
 0001:00030390       ?inputdata@@YAXJ@Z         10031390 f   seq.obj
 0001:000307e0       ?makevalues2@@YAXJPAPAUnode@@JJPAPADPAJ@Z 100317e0 f   seq.obj
 0001:00030b20       ?makevalues@@YAXPAPAUnode@@PAJE@Z 10031b20 f   seq.obj
 0001:00030d10       ?minpostorder@@YAXPAUnode@@PAPAU1@@Z 10031d10 f   seq.obj
 0001:00030e50       ?moresteps@@YAEPAUnode@@0@Z 10031e50 f   seq.obj
 0001:00030e90       ?moveleft@@YAXPAUnode@@0PAPAU1@@Z 10031e90 f   seq.obj
 0001:00030ee0       ?multifillin@@YAXPAUnode@@0J@Z 10031ee0 f   seq.obj
 0001:00031270       ?multisumnsteps2@@YAXPAUnode@@@Z 10032270 f   seq.obj
 0001:00031460       ?multisumnsteps@@YAXPAUnode@@0JJPAJ@Z 10032460 f   seq.obj
 0001:00031670       ?newindex@@YAXJPAUnode@@@Z 10032670 f   seq.obj
 0001:00031690       ?outgrin@@YAEPAUnode@@0@Z  10032690 f   seq.obj
 0001:000316c0       ?parentinmulti@@YAEPAUnode@@@Z 100326c0 f   seq.obj
 0001:00031710       ?passdown@@YAEPAUnode@@00000000E@Z 10032710 f   seq.obj
 0001:000319c0       ?postorder@@YAXPAUnode@@@Z 100329c0 f   seq.obj
 0001:00031a30       ?preorder@@YAXPAUnode@@00000J@Z 10032a30 f   seq.obj
 0001:00031b90       ?printbranchlengths@@YAXPAUnode@@@Z 10032b90 f   seq.obj
 0001:00031c70       ?printree@@YAXPAUnode@@N@Z 10032c70 f   seq.obj
 0001:00031d60       ?prot_allocx@@YAXJJPAPAUnode@@E@Z 10032d60 f   seq.obj
 0001:00031ea0       ?prot_copy_@@YAXPAUtree@@0JJ@Z 10032ea0 f   seq.obj
 0001:00032010       ?prot_copynode@@YAXPAUnode@@0J@Z 10033010 f   seq.obj
 0001:00032110       ?prot_freex@@YAXJPAPAUnode@@@Z 10033110 f   seq.obj
 0001:00032200       ?prot_freex_notip@@YAXJPAPAUnode@@@Z 10033200 f   seq.obj
 0001:000322b0       ?putback@@YAXPAUnode@@00PAPAU1@@Z 100332b0 f   seq.obj
 0001:00032300       ?re_move@@YAXPAUnode@@PAPAU1@1E11PAJ@Z 10033300 f   seq.obj
 0001:00032700       ?replaceback@@YAXPAPAUnode@@PAU1@10PAJ@Z 10033700 f   seq.obj
 0001:00032770       ?reroot2@@YAXPAUnode@@0@Z  10033770 f   seq.obj
 0001:00032790       ?reroot3@@YAXPAUnode@@000PAPAU1@@Z 10033790 f   seq.obj
 0001:000327d0       ?reroot@@YAXPAUnode@@0@Z   100337d0 f   seq.obj
 0001:00032820       ?savelocrearr@@YAXPAUnode@@00000000PAPAU1@JPAJEEPAE2PAUbestelm@@112@Z 10033820 f   seq.obj
 0001:00032ac0       ?savetraverse@@YAXPAUnode@@@Z 10033ac0 f   seq.obj
 0001:00032b00       ?savetree@@YAXPAUnode@@PAJPAPAU1@21@Z 10033b00 f   seq.obj
 0001:00032f50       ?setbottom@@YAXPAUnode@@@Z 10033f50 f   seq.obj
 0001:00032f70       ?setuptree2@@YAXPAUtree@@@Z 10033f70 f   seq.obj
 0001:00032fa0       ?setuptree@@YAXPAPAUnode@@JE@Z 10033fa0 f   seq.obj
 0001:00033080       ?sibsvisited@@YAJPAUnode@@PAJ@Z 10034080 f   seq.obj
 0001:000330d0       ?sitecombine2@@YAXJPAJ@Z   100340d0 f   seq.obj
 0001:000331f0       ?sitecombine@@YAXJ@Z       100341f0 f   seq.obj
 0001:000332f0       ?sitescrunch2@@YAXJJJPAJ@Z 100342f0 f   seq.obj
 0001:000333a0       ?sitescrunch@@YAXJ@Z       100343a0 f   seq.obj
 0001:00033470       ?sitesort2@@YAXJPAJ@Z      10034470 f   seq.obj
 0001:000335f0       ?sitesort@@YAXJPAJ@Z       100345f0 f   seq.obj
 0001:00033760       ?smallest@@YAJPAUnode@@PAJ@Z 10034760 f   seq.obj
 0001:000337e0       ?standev2@@YAXJJJJNPANPAPANPAJQAJ@Z 100347e0 f   seq.obj
 0001:000342c0       ?standev@@YAXJJJNPANPAPAJQAJ@Z 100352c0 f   seq.obj
 0001:00034e20       ?sumnsteps2@@YAXPAUnode@@00JJPAJ@Z 10035e20 f   seq.obj
 0001:00034f50       ?sumnsteps@@YAXPAUnode@@00JJ@Z 10035f50 f   seq.obj
 0001:00035090       ?treelength@@YAXPAUnode@@JPAPAU1@@Z 10036090 f   seq.obj
 0001:000350f0       ?treeout3@@YAXPAUnode@@JPAJ0@Z 100360f0 f   seq.obj
 0001:00035330       ?treeout@@YAXPAUnode@@JPAJ0@Z 10036330 f   seq.obj
 0001:000354b0       ?trycollapdesc@@YAEPAUnode@@00000000EPAJ@Z 100364b0 f   seq.obj
 0001:000357e0       ?updatenumdesc@@YAXPAUnode@@0J@Z 100367e0 f   seq.obj
 0001:00035810       ?writesteps@@YAXJEPAJPAUnode@@@Z 10036810 f   seq.obj
 0001:000359a0       ?zeroinsubtree@@YAEPAUnode@@0000000E0PAJ@Z 100369a0 f   seq.obj
 0001:00035b20       ?allocnew@@YAXXZ           10036b20 f   seqboot.obj
 0001:00035b50       ?allocnewer@@YAXJJ@Z       10036b50 f   seqboot.obj
 0001:00035c90       ?bootweights@@YAXXZ        10036c90 f   seqboot.obj
 0001:00036070       ?bootwrite@@YAXAAV?$QVector@VMultipleSequenceAlignment@U2@@@@ABVMultipleSequenceAlignment@U2@@@Z 10037070 f   seqboot.obj
 0001:00036240       ?charpermute@@YAXJJ@Z      10037240 f   seqboot.obj
 0001:00036260       ?doinput@@YAXHQAPAD@Z      10037260 f   seqboot.obj
 0001:00036470       ?freenew@@YAXXZ            10037470 f   seqboot.obj
 0001:000364a0       ?freenewer@@YAXXZ          100374a0 f   seqboot.obj
 0001:00036520       ?getData@@YAPAPADXZ        10037520 f   seqboot.obj
 0001:00036530       ?matrix_char_delete@@YAXPAPADJ@Z 10037530 f   seqboot.obj
 0001:00036560       ?matrix_char_new@@YAPAPADJJ@Z 10037560 f   seqboot.obj
 0001:000365a0       ?matrix_double_delete@@YAXPAPANJ@Z 100375a0 f   seqboot.obj
 0001:000365d0       ?matrix_double_new@@YAPAPANJJ@Z 100375d0 f   seqboot.obj
 0001:00036620       ?permute_vec@@YAXPAJJ@Z    10037620 f   seqboot.obj
 0001:00036690       ?seq_allocrest@@YAXXZ      10037690 f   seqboot.obj
 0001:00036780       ?seq_freerest@@YAXXZ       10037780 f   seqboot.obj
 0001:00036830       ?seq_inputoptions@@YAXXZ   10037830 f   seqboot.obj
 0001:00036bb0       ?seqboot_getoptions@@YAXXZ 10037bb0 f   seqboot.obj
 0001:00036c70       ?seqboot_inputdata@@YAXXZ  10037c70 f   seqboot.obj
 0001:00037690       ?seqboot_inputfactors@@YAXXZ 10038690 f   seqboot.obj
 0001:00037700       ?seqboot_inputnumbers@@YAXXZ 10038700 f   seqboot.obj
 0001:00037720       ?sppermute@@YAXJ@Z         10038720 f   seqboot.obj
 0001:00037740       ?writeauxdata@@YAXPAJPAU_iobuf@@@Z 10038740 f   seqboot.obj
 0001:000379a0       ?writecategories@@YAXXZ    100389a0 f   seqboot.obj
 0001:00037c00       ?writedata@@YAXAAV?$QVector@VMultipleSequenceAlignment@U2@@@@HABVMultipleSequenceAlignment@U2@@@Z 10038c00 f   seqboot.obj
 0001:00038480       ?writefactors@@YAXXZ       10039480 f   seqboot.obj
 0001:00038650       ?writeweights@@YAXXZ       10039650 f   seqboot.obj
 0001:00038800       ??C?$QScopedPointer@VQObjectData@@U?$QScopedPointerDeleter@VQObjectData@@@@@@QBEPAVQObjectData@@XZ 10039800 f i moc_NeighborJoinWidget.obj
 0001:00038810       ?metaObject@NeighborJoinWidget@U2@@UBEPBUQMetaObject@@XZ 10039810 f   moc_NeighborJoinWidget.obj
 0001:00038830       ?qt_metacall@NeighborJoinWidget@U2@@UAEHW4Call@QMetaObject@@HPAPAX@Z 10039830 f   moc_NeighborJoinWidget.obj
 0001:000388c0       ?qt_metacast@NeighborJoinWidget@U2@@UAEPAXPBD@Z 100398c0 f   moc_NeighborJoinWidget.obj
 0001:00038960       ?qt_static_metacall@NeighborJoinWidget@U2@@CAXPAVQObject@@W4Call@QMetaObject@@HPAPAX@Z 10039960 f   moc_NeighborJoinWidget.obj
 0001:000389a0       ?metaObject@PhylipCmdlineTask@U2@@UBEPBUQMetaObject@@XZ 100399a0 f   moc_PhylipCmdlineTask.obj
 0001:000389c0       ?qt_metacall@PhylipCmdlineTask@U2@@UAEHW4Call@QMetaObject@@HPAPAX@Z 100399c0 f   moc_PhylipCmdlineTask.obj
 0001:000389d0       ?qt_metacast@PhylipCmdlineTask@U2@@UAEPAXPBD@Z 100399d0 f   moc_PhylipCmdlineTask.obj
 0001:00038a30       ?qt_static_metacall@PhylipCmdlineTask@U2@@CAXPAVQObject@@W4Call@QMetaObject@@HPAPAX@Z 10039a30 f   moc_PhylipCmdlineTask.obj
 0001:00038a40       ?metaObject@PhylipPlugin@U2@@UBEPBUQMetaObject@@XZ 10039a40 f   moc_PhylipPlugin.obj
 0001:00038a60       ?qt_metacall@PhylipPlugin@U2@@UAEHW4Call@QMetaObject@@HPAPAX@Z 10039a60 f   moc_PhylipPlugin.obj
 0001:00038a70       ?qt_metacast@PhylipPlugin@U2@@UAEPAXPBD@Z 10039a70 f   moc_PhylipPlugin.obj
 0001:00038ad0       ?qt_static_metacall@PhylipPlugin@U2@@CAXPAVQObject@@W4Call@QMetaObject@@HPAPAX@Z 10039ad0 f   moc_PhylipPlugin.obj
 0001:00038ae0       ?metaObject@GTest_NeighborJoin@U2@@UBEPBUQMetaObject@@XZ 10039ae0 f   moc_PhylipPluginTests.obj
 0001:00038b00       ?qt_metacall@GTest_NeighborJoin@U2@@UAEHW4Call@QMetaObject@@HPAPAX@Z 10039b00 f   moc_PhylipPluginTests.obj
 0001:00038b10       ?qt_metacast@GTest_NeighborJoin@U2@@UAEPAXPBD@Z 10039b10 f   moc_PhylipPluginTests.obj
 0001:00038b70       ?qt_static_metacall@GTest_NeighborJoin@U2@@CAXPAVQObject@@W4Call@QMetaObject@@HPAPAX@Z 10039b70 f   moc_PhylipPluginTests.obj
 0001:00038b80       ?metaObject@PhylipTask@U2@@UBEPBUQMetaObject@@XZ 10039b80 f   moc_PhylipTask.obj
 0001:00038ba0       ?qt_metacall@PhylipTask@U2@@UAEHW4Call@QMetaObject@@HPAPAX@Z 10039ba0 f   moc_PhylipTask.obj
 0001:00038bb0       ?qt_metacast@PhylipTask@U2@@UAEPAXPBD@Z 10039bb0 f   moc_PhylipTask.obj
 0001:00038c10       ?qt_static_metacall@PhylipTask@U2@@CAXPAVQObject@@W4Call@QMetaObject@@HPAPAX@Z 10039c10 f   moc_PhylipTask.obj
 0001:00038c12       ??0Logger@U2@@QAE@ABVQString@@@Z 10039c12 f   U2Core:U2Core.dll
 0001:00038c18       ??1Logger@U2@@UAE@XZ       10039c18 f   U2Core:U2Core.dll
 0001:00038c1e       ?getResource@AppResourcePool@U2@@QBEPAVAppResource@2@H@Z 10039c1e f   U2Core:U2Core.dll
 0001:00038c24       ?instance@AppResourcePool@U2@@SAPAV12@XZ 10039c24 f   U2Core:U2Core.dll
 0001:00038c2a       ??1MultipleAlignmentRow@U2@@UAE@XZ 10039c2a f   U2Core:U2Core.dll
 0001:00038c30       ?getName@MultipleAlignmentData@U2@@QBE?AVQString@@XZ 10039c30 f   U2Core:U2Core.dll
 0001:00038c36       ?getAlphabet@MultipleAlignmentData@U2@@QBEPBVDNAAlphabet@2@XZ 10039c36 f   U2Core:U2Core.dll
 0001:00038c3c       ?getLength@MultipleAlignmentData@U2@@QBEHXZ 10039c3c f   U2Core:U2Core.dll
 0001:00038c42       ??CMultipleSequenceAlignmentRow@U2@@QBEPBVMultipleSequenceAlignmentRowData@1@XZ 10039c42 f   U2Core:U2Core.dll
 0001:00038c48       ??1MultipleSequenceAlignmentRow@U2@@UAE@XZ 10039c48 f   U2Core:U2Core.dll
 0001:00038c4e       ??0MultipleSequenceAlignmentRow@U2@@QAE@ABV01@@Z 10039c4e f   U2Core:U2Core.dll
 0001:00038c54       ??CMultipleSequenceAlignment@U2@@QBEPBVMultipleSequenceAlignmentData@1@XZ 10039c54 f   U2Core:U2Core.dll
 0001:00038c5a       ?getNumRows@MultipleSequenceAlignmentData@U2@@QBEHXZ 10039c5a f   U2Core:U2Core.dll
 0001:00038c60       ?getMsaRow@MultipleSequenceAlignmentData@U2@@QBE?BVMultipleSequenceAlignmentRow@2@H@Z 10039c60 f   U2Core:U2Core.dll
 0001:00038c66       ?getMsaRows@MultipleSequenceAlignmentData@U2@@QBE?BV?$QList@VMultipleSequenceAlignmentRow@U2@@@@XZ 10039c66 f   U2Core:U2Core.dll
 0001:00038c6c       ??0PhyTreeData@U2@@QAE@ABV01@@Z 10039c6c f   U2Core:U2Core.dll
 0001:00038c72       ??1PhyTreeData@U2@@QAE@XZ  10039c72 f   U2Core:U2Core.dll
 0001:00038c78       ?print@PhyTreeData@U2@@QBEXXZ 10039c78 f   U2Core:U2Core.dll
 0001:00038c7e       ?addBranch@PhyTreeData@U2@@SAPAVPhyBranch@2@PAVPhyNode@2@0N@Z 10039c7e f   U2Core:U2Core.dll
 0001:00038c84       ?removeBranch@PhyTreeData@U2@@SAXPAVPhyNode@2@0@Z 10039c84 f   U2Core:U2Core.dll
 0001:00038c8a       ??0PhyNode@U2@@QAE@XZ      10039c8a f   U2Core:U2Core.dll
 0001:00038c90       ?branchCount@PhyNode@U2@@QBEHXZ 10039c90 f   U2Core:U2Core.dll
 0001:00038c96       ?getBranchesDistance@PhyNode@U2@@QBENH@Z 10039c96 f   U2Core:U2Core.dll
 0001:00038c9c       ?isConnected@PhyNode@U2@@QBE_NPBV12@@Z 10039c9c f   U2Core:U2Core.dll
 0001:00038ca2       ?getBranch@PhyNode@U2@@QBEPAVPhyBranch@2@H@Z 10039ca2 f   U2Core:U2Core.dll
 0001:00038ca8       ?getParentNode@PhyNode@U2@@QAEPAV12@XZ 10039ca8 f   U2Core:U2Core.dll
 0001:00038cae       ?setBranchesDistance@PhyNode@U2@@QAEXHN@Z 10039cae f   U2Core:U2Core.dll
 0001:00038cb4       ??1GCounter@U2@@UAE@XZ     10039cb4 f   U2Core:U2Core.dll
 0001:00038cba       ??0GReportableCounter@U2@@QAE@ABVQString@@0N@Z 10039cba f   U2Core:U2Core.dll
 0001:00038cc0       ??1SimpleEventCounter@U2@@UAE@XZ 10039cc0 f   U2Core:U2Core.dll
 0001:00038cc6       ?setError@Task@U2@@QAEXABVQString@@@Z 10039cc6 f   U2Core:U2Core.dll
 0001:00038ccc       ?setTaskName@Task@U2@@IAEXABVQString@@@Z 10039ccc f   U2Core:U2Core.dll
 0001:00038cd2       ??0PhyTreeData@U2@@QAE@XZ  10039cd2 f   U2Core:U2Core.dll
 0001:00038cd8       ?cleanup@Task@U2@@UAEXXZ   10039cd8 f   U2Core:U2Core.dll
 0001:00038cde       ?generateReport@Task@U2@@UBE?AVQString@@XZ 10039cde f   U2Core:U2Core.dll
 0001:00038ce4       ?getNumParallelSubtasks@Task@U2@@UBEHXZ 10039ce4 f   U2Core:U2Core.dll
 0001:00038cea       ?getParentTask@Task@U2@@UBEPAV12@XZ 10039cea f   U2Core:U2Core.dll
 0001:00038cf0       ?getSubtaskWithErrors@Task@U2@@UBEPAV12@XZ 10039cf0 f   U2Core:U2Core.dll
 0001:00038cf6       ?getTaskId@Task@U2@@UBE_JXZ 10039cf6 f   U2Core:U2Core.dll
 0001:00038cfc       ?getTopLevelParentTask@Task@U2@@UAEPAV12@XZ 10039cfc f   U2Core:U2Core.dll
 0001:00038d02       ?getWarnings@Task@U2@@UBE?AVQStringList@@XZ 10039d02 f   U2Core:U2Core.dll
 0001:00038d08       ?hasSubtasksWithErrors@Task@U2@@UBE_NXZ 10039d08 f   U2Core:U2Core.dll
 0001:00038d0e       ?hasWarning@Task@U2@@UBE_NXZ 10039d0e f   U2Core:U2Core.dll
 0001:00038d14       ?isNotificationReport@Task@U2@@UBE_NXZ 10039d14 f   U2Core:U2Core.dll
 0001:00038d1a       ?isReportingEnabled@Task@U2@@UBE_NXZ 10039d1a f   U2Core:U2Core.dll
 0001:00038d20       ?isReportingSupported@Task@U2@@UBE_NXZ 10039d20 f   U2Core:U2Core.dll
 0001:00038d26       ?isTopLevelTask@Task@U2@@UBE_NXZ 10039d26 f   U2Core:U2Core.dll
 0001:00038d2c       ?onSubTaskFinished@Task@U2@@MAE?AV?$QList@PAVTask@U2@@@@PAV12@@Z 10039d2c f   U2Core:U2Core.dll
 0001:00038d32       ?prepare@Task@U2@@UAEXXZ   10039d32 f   U2Core:U2Core.dll
 0001:00038d38       ?propagateSubtaskError@Task@U2@@UAE_NXZ 10039d38 f   U2Core:U2Core.dll
 0001:00038d3e       ?setCollectChildrensWarningsFlag@Task@U2@@UAEX_N@Z 10039d3e f   U2Core:U2Core.dll
 0001:00038d44       ?setNoAutoDelete@Task@U2@@UAEX_N@Z 10039d44 f   U2Core:U2Core.dll
 0001:00038d4a       ?setNotificationReport@Task@U2@@UAEX_N@Z 10039d4a f   U2Core:U2Core.dll
 0001:00038d50       ?setReportingEnabled@Task@U2@@UAEX_N@Z 10039d50 f   U2Core:U2Core.dll
 0001:00038d56       ?setReportingSupported@Task@U2@@UAEX_N@Z 10039d56 f   U2Core:U2Core.dll
 0001:00038d5c       ?getSettings@AppContext@U2@@SAPAVSettings@2@XZ 10039d5c f   U2Core:U2Core.dll
 0001:00038d62       ?getAppSettings@AppContext@U2@@SAPAVAppSettings@2@XZ 10039d62 f   U2Core:U2Core.dll
 0001:00038d68       ??0U2DbiRef@U2@@QAE@ABVQString@@0@Z 10039d68 f   U2Core:U2Core.dll
 0001:00038d6e       ??1U2DbiRef@U2@@QAE@XZ     10039d6e f   U2Core:U2Core.dll
 0001:00038d74       ??0U2EntityRef@U2@@QAE@ABVU2DbiRef@1@ABVQByteArray@@@Z 10039d74 f   U2Core:U2Core.dll
 0001:00038d7a       ??1U2EntityRef@U2@@QAE@XZ  10039d7a f   U2Core:U2Core.dll
 0001:00038d80       ?addSubTask@Task@U2@@QAEXPAV12@@Z 10039d80 f   U2Core:U2Core.dll
 0001:00038d86       ??0CmdlineInOutTaskConfig@U2@@QAE@XZ 10039d86 f   U2Core:U2Core.dll
 0001:00038d8c       ??1CmdlineInOutTaskConfig@U2@@QAE@XZ 10039d8c f   U2Core:U2Core.dll
 0001:00038d92       ??0CmdlineInOutTaskRunner@U2@@QAE@ABVCmdlineInOutTaskConfig@1@@Z 10039d92 f   U2Core:U2Core.dll
 0001:00038d98       ?getOutputObjects@CmdlineInOutTaskRunner@U2@@QBEABV?$QList@VQByteArray@@@@XZ 10039d98 f   U2Core:U2Core.dll
 0001:00038d9e       ??1CmdlineInOutTaskRunner@U2@@UAE@XZ 10039d9e f   U2Core:U2Core.dll
 0001:00038da4       ?prepareTmpFileLocation@GUrlUtils@U2@@SA?AVQString@@ABV3@00AAVU2OpStatus@2@@Z 10039da4 f   U2Core:U2Core.dll
 0001:00038daa       ?createAlignment@MultipleSequenceAlignmentImporter@U2@@SAPAVMultipleSequenceAlignmentObject@2@ABVU2DbiRef@2@AAVMultipleSequenceAlignment@2@AAVU2OpStatus@2@@Z 10039daa f   U2Core:U2Core.dll
 0001:00038db0       ??0PhyTreeObject@U2@@QAE@ABVQString@@ABVU2EntityRef@1@ABV?$QMap@VQString@@VQVariant@@@@@Z 10039db0 f   U2Core:U2Core.dll
 0001:00038db6       ??1PhyTreeObject@U2@@UAE@XZ 10039db6 f   U2Core:U2Core.dll
 0001:00038dbc       ??0DbiConnection@U2@@QAE@ABVU2DbiRef@1@_NAAVU2OpStatus@1@ABV?$QHash@VQString@@V1@@@@Z 10039dbc f   U2Core:U2Core.dll
 0001:00038dc2       ??1DbiConnection@U2@@QAE@XZ 10039dc2 f   U2Core:U2Core.dll
 0001:00038dc8       ?getCurrentProcessTemporaryDirPath@UserAppsSettings@U2@@QBE?AVQString@@ABV3@@Z 10039dc8 f   U2Core:U2Core.dll
 0001:00038dce       ?checkConstraints@GObject@U2@@UBE_NPBVGObjectConstraints@2@@Z 10039dce f   U2Core:U2Core.dll
 0001:00038dd4       ?clone@PhyTreeObject@U2@@UBEPAVGObject@2@ABVU2DbiRef@2@AAVU2OpStatus@2@ABV?$QMap@VQString@@VQVariant@@@@@Z 10039dd4 f   U2Core:U2Core.dll
 0001:00038dda       ?getDocument@GObject@U2@@UBEPAVDocument@2@XZ 10039dda f   U2Core:U2Core.dll
 0001:00038de0       ?getModificationVersion@StateLockableItem@U2@@UBEHXZ 10039de0 f   U2Core:U2Core.dll
 0001:00038de6       ?getTree@PhyTreeObject@U2@@UBEABV?$QSharedDataPointer@VPhyTreeData@U2@@@@XZ 10039de6 f   U2Core:U2Core.dll
 0001:00038dec       ?hasModifiedChildren@StateLockableTreeItem@U2@@UBE_NXZ 10039dec f   U2Core:U2Core.dll
 0001:00038df2       ?isCommandLogLine@CmdlineInOutTaskRunner@U2@@EBE_NABVQString@@@Z 10039df2 f   U2Core:U2Core.dll
 0001:00038df8       ?isItemModified@StateLockableItem@U2@@UBE_NXZ 10039df8 f   U2Core:U2Core.dll
 0001:00038dfe       ?isMainThreadModificationOnly@StateLockableTreeItem@U2@@UBE_NXZ 10039dfe f   U2Core:U2Core.dll
 0001:00038e04       ?isMainThreadObject@StateLockableItem@U2@@UBE_NXZ 10039e04 f   U2Core:U2Core.dll
 0001:00038e0a       ?isModificationAllowed@StateLockableItem@U2@@UAE_NABVQString@@@Z 10039e0a f   U2Core:U2Core.dll
 0001:00038e10       ?isModificationTracked@StateLockableItem@U2@@UBE_NXZ 10039e10 f   U2Core:U2Core.dll
 0001:00038e16       ?isStateLocked@StateLockableTreeItem@U2@@UBE_NXZ 10039e16 f   U2Core:U2Core.dll
 0001:00038e1c       ?isTreeItemModified@StateLockableTreeItem@U2@@UBE_NXZ 10039e1c f   U2Core:U2Core.dll
 0001:00038e22       ?loadDataCore@PhyTreeObject@U2@@MAEXAAVU2OpStatus@2@@Z 10039e22 f   U2Core:U2Core.dll
 0001:00038e28       ?lockState@StateLockableTreeItem@U2@@UAEXPAVStateLock@2@@Z 10039e28 f   U2Core:U2Core.dll
 0001:00038e2e       ?metaObject@CmdlineInOutTaskRunner@U2@@UBEPBUQMetaObject@@XZ 10039e2e f   U2Core:U2Core.dll
 0001:00038e34       ?metaObject@PhyTreeObject@U2@@UBEPBUQMetaObject@@XZ 10039e34 f   U2Core:U2Core.dll
 0001:00038e3a       ?parseCommandLogWord@CmdlineInOutTaskRunner@U2@@EAE_NABVQString@@@Z 10039e3a f   U2Core:U2Core.dll
 0001:00038e40       ?prepare@CmdlineTaskRunner@U2@@UAEXXZ 10039e40 f   U2Core:U2Core.dll
 0001:00038e46       ?qt_metacall@CmdlineInOutTaskRunner@U2@@UAEHW4Call@QMetaObject@@HPAPAX@Z 10039e46 f   U2Core:U2Core.dll
 0001:00038e4c       ?qt_metacall@PhyTreeObject@U2@@UAEHW4Call@QMetaObject@@HPAPAX@Z 10039e4c f   U2Core:U2Core.dll
 0001:00038e52       ?qt_metacast@CmdlineInOutTaskRunner@U2@@UAEPAXPBD@Z 10039e52 f   U2Core:U2Core.dll
 0001:00038e58       ?qt_metacast@PhyTreeObject@U2@@UAEPAXPBD@Z 10039e58 f   U2Core:U2Core.dll
 0001:00038e5e       ?report@CmdlineInOutTaskRunner@U2@@UAE?AW4ReportResult@Task@2@XZ 10039e5e f   U2Core:U2Core.dll
 0001:00038e64       ?run@Task@U2@@UAEXXZ       10039e64 f   U2Core:U2Core.dll
 0001:00038e6a       ?setGObjectName@GObject@U2@@UAEXABVQString@@@Z 10039e6a f   U2Core:U2Core.dll
 0001:00038e70       ?setMainThreadModificationOnly@StateLockableItem@U2@@UAEX_N@Z 10039e70 f   U2Core:U2Core.dll
 0001:00038e76       ?setModificationTrack@StateLockableTreeItem@U2@@UAEX_N@Z 10039e76 f   U2Core:U2Core.dll
 0001:00038e7c       ?setModified@StateLockableTreeItem@U2@@UAEX_NABVQString@@@Z 10039e7c f   U2Core:U2Core.dll
 0001:00038e82       ?setParentStateLockItem@GObject@U2@@EAEXPAVStateLockableTreeItem@2@@Z 10039e82 f   U2Core:U2Core.dll
 0001:00038e88       ?unlockState@StateLockableTreeItem@U2@@UAEXPAVStateLock@2@@Z 10039e88 f   U2Core:U2Core.dll
 0001:00038e8e       ?isCoR@U2OpStatus@U2@@UBE_NXZ 10039e8e f   U2Core:U2Core.dll
 0001:00038e94       ?getPluginSupport@AppContext@U2@@SAPAVPluginSupport@2@XZ 10039e94 f   U2Core:U2Core.dll
 0001:00038e9a       ?getTestFramework@AppContext@U2@@SAPAVTestFramework@2@XZ 10039e9a f   U2Core:U2Core.dll
 0001:00038ea0       ?getPhyTreeGeneratorRegistry@AppContext@U2@@SAPAVPhyTreeGeneratorRegistry@2@XZ 10039ea0 f   U2Core:U2Core.dll
 0001:00038ea6       ?getCMDLineRegistry@AppContext@U2@@SAPAVCMDLineRegistry@2@XZ 10039ea6 f   U2Core:U2Core.dll
 0001:00038eac       ?hasParameter@CMDLineRegistry@U2@@QBE_NABVQString@@H@Z 10039eac f   U2Core:U2Core.dll
 0001:00038eb2       ?getParameterValue@CMDLineRegistry@U2@@QBE?AVQString@@ABV3@H@Z 10039eb2 f   U2Core:U2Core.dll
 0001:00038eb8       ?parseDbiRef@CmdlineInOutTaskRunner@U2@@SA?AVU2DbiRef@2@ABVQString@@AAVU2OpStatus@2@@Z 10039eb8 f   U2Core:U2Core.dll
 0001:00038ebe       ?parseDataId@CmdlineInOutTaskRunner@U2@@SA?AVQByteArray@@ABVQString@@ABVU2DbiRef@2@AAVU2OpStatus@2@@Z 10039ebe f   U2Core:U2Core.dll
 0001:00038ec4       ??0U2OpStatus2Log@U2@@QAE@W4LogLevel@1@@Z 10039ec4 f   U2Core:U2Core.dll
 0001:00038eca       ??1U2OpStatus2Log@U2@@UAE@XZ 10039eca f   U2Core:U2Core.dll
 0001:00038ed0       ??0Plugin@U2@@QAE@ABVQString@@0_NW4PluginState@1@@Z 10039ed0 f   U2Core:U2Core.dll
 0001:00038ed6       ??1Plugin@U2@@UAE@XZ       10039ed6 f   U2Core:U2Core.dll
 0001:00038edc       ?metaObject@TaskStarter@U2@@UBEPBUQMetaObject@@XZ 10039edc f   U2Core:U2Core.dll
 0001:00038ee2       ?qt_metacall@TaskStarter@U2@@UAEHW4Call@QMetaObject@@HPAPAX@Z 10039ee2 f   U2Core:U2Core.dll
 0001:00038ee8       ?qt_metacast@TaskStarter@U2@@UAEPAXPBD@Z 10039ee8 f   U2Core:U2Core.dll
 0001:00038eee       ?hasError@Task@U2@@QBE_NXZ 10039eee f   U2Core:U2Core.dll
 0001:00038ef4       ??1MultipleAlignment@U2@@UAE@XZ 10039ef4 f   U2Core:U2Core.dll
 0001:00038efa       ??0MultipleSequenceAlignment@U2@@QAE@ABVMultipleAlignment@1@@Z 10039efa f   U2Core:U2Core.dll
 0001:00038f00       ??1MultipleSequenceAlignment@U2@@UAE@XZ 10039f00 f   U2Core:U2Core.dll
 0001:00038f06       ?findGObjectByType@Document@U2@@QBE?AV?$QList@PAVGObject@U2@@@@VQString@@W4UnloadedObjectFilter@2@@Z 10039f06 f   U2Core:U2Core.dll
 0001:00038f0c       ?getMultipleAlignment@MultipleAlignmentObject@U2@@QBEABVMultipleAlignment@2@XZ 10039f0c f   U2Core:U2Core.dll
 0001:00038f12       ?treesAreAlike@PhyTreeObject@U2@@SA_NABV?$QSharedDataPointer@VPhyTreeData@U2@@@@0@Z 10039f12 f   U2Core:U2Core.dll
 0001:00038f18       ??0U2DbiRef@U2@@QAE@ABV01@@Z 10039f18 f   U2Core:U2Core.dll
 0001:00038f1e       ??0U2EntityRef@U2@@QAE@ABV01@@Z 10039f1e f   U2Core:U2Core.dll
 0001:00038f24       ??0CmdlineTask@U2@@QAE@ABVQString@@V?$QFlags@W4TaskFlag@U2@@@@@Z 10039f24 f   U2Core:U2Core.dll
 0001:00038f2a       ?report@CmdlineTask@U2@@UAE?AW4ReportResult@Task@2@XZ 10039f2a f   U2Core:U2Core.dll
 0001:00038f30       ??1CmdlineTask@U2@@UAE@XZ  10039f30 f   U2Core:U2Core.dll
 0001:00038f36       ?logOutputObject@CmdlineInOutTaskRunner@U2@@SAXABVQByteArray@@@Z 10039f36 f   U2Core:U2Core.dll
 0001:00038f3c       ??1MultipleAlignmentObject@U2@@UAE@XZ 10039f3c f   U2Core:U2Core.dll
 0001:00038f42       ??0MultipleSequenceAlignment@U2@@QAE@ABVQString@@PBVDNAAlphabet@1@ABV?$QList@VMultipleSequenceAlignmentRow@U2@@@@@Z 10039f42 f   U2Core:U2Core.dll
 0001:00038f48       ??0MultipleSequenceAlignmentObject@U2@@QAE@ABVQString@@ABVU2EntityRef@1@ABV?$QMap@VQString@@VQVariant@@@@ABVMultipleSequenceAlignment@1@@Z 10039f48 f   U2Core:U2Core.dll
 0001:00038f4e       ?createInstance@PhyTreeObject@U2@@SAPAV12@ABV?$QSharedDataPointer@VPhyTreeData@U2@@@@ABVQString@@ABVU2DbiRef@2@AAVU2OpStatus@2@ABV?$QMap@VQString@@VQVariant@@@@@Z 10039f4e f   U2Core:U2Core.dll
 0001:00038f54       ?charAt@MultipleSequenceAlignmentObject@U2@@UBEDH_J@Z 10039f54 f   U2Core:U2Core.dll
 0001:00038f5a       ?clone@MultipleSequenceAlignmentObject@U2@@UBEPAV12@ABVU2DbiRef@2@AAVU2OpStatus@2@ABV?$QMap@VQString@@VQVariant@@@@@Z 10039f5a f   U2Core:U2Core.dll
 0001:00038f60       ?deleteColumnsWithGaps@MultipleSequenceAlignmentObject@U2@@UAEXAAVU2OpStatus@2@H@Z 10039f60 f   U2Core:U2Core.dll
 0001:00038f66       ?getTaskError@CmdlineTask@U2@@MBE?AVQString@@XZ 10039f66 f   U2Core:U2Core.dll
 0001:00038f6c       ?insertGap@MultipleSequenceAlignmentObject@U2@@EAEXABVU2Region@2@HH@Z 10039f6c f   U2Core:U2Core.dll
 0001:00038f72       ?loadAlignment@MultipleSequenceAlignmentObject@U2@@EAEXAAVU2OpStatus@2@@Z 10039f72 f   U2Core:U2Core.dll
 0001:00038f78       ?loadDataCore@MultipleAlignmentObject@U2@@EAEXAAVU2OpStatus@2@@Z 10039f78 f   U2Core:U2Core.dll
 0001:00038f7e       ?metaObject@MultipleSequenceAlignmentObject@U2@@UBEPBUQMetaObject@@XZ 10039f7e f   U2Core:U2Core.dll
 0001:00038f84       ?qt_metacall@MultipleSequenceAlignmentObject@U2@@UAEHW4Call@QMetaObject@@HPAPAX@Z 10039f84 f   U2Core:U2Core.dll
 0001:00038f8a       ?qt_metacast@MultipleSequenceAlignmentObject@U2@@UAEPAXPBD@Z 10039f8a f   U2Core:U2Core.dll
 0001:00038f90       ?removeRegionPrivate@MultipleSequenceAlignmentObject@U2@@EAEXAAVU2OpStatus@2@ABVU2EntityRef@2@ABV?$QList@_J@@HH@Z 10039f90 f   U2Core:U2Core.dll
 0001:00038f96       ?removeRowPrivate@MultipleSequenceAlignmentObject@U2@@EAEXAAVU2OpStatus@2@ABVU2EntityRef@2@_J@Z 10039f96 f   U2Core:U2Core.dll
 0001:00038f9c       ?replaceCharacter@MultipleSequenceAlignmentObject@U2@@UAEXHHD@Z 10039f9c f   U2Core:U2Core.dll
 0001:00038fa2       ?setGObjectName@MultipleAlignmentObject@U2@@UAEXABVQString@@@Z 10039fa2 f   U2Core:U2Core.dll
 0001:00038fa8       ?updateCachedRows@MultipleSequenceAlignmentObject@U2@@EAEXAAVU2OpStatus@2@ABV?$QList@_J@@@Z 10039fa8 f   U2Core:U2Core.dll
 0001:00038fae       ?updateDatabase@MultipleSequenceAlignmentObject@U2@@EAEXAAVU2OpStatus@2@ABVMultipleAlignment@2@@Z 10039fae f   U2Core:U2Core.dll
 0001:00038fb4       ??CMultipleSequenceAlignment@U2@@QAEPAVMultipleSequenceAlignmentData@1@XZ 10039fb4 f   U2Core:U2Core.dll
 0001:00038fba       ??0MultipleSequenceAlignment@U2@@QAE@ABV01@@Z 10039fba f   U2Core:U2Core.dll
 0001:00038fc0       ??4MultipleSequenceAlignment@U2@@QAEAAV01@ABV01@@Z 10039fc0 f   U2Core:U2Core.dll
 0001:00038fc6       ?prepareDirLocation@GUrlUtils@U2@@SA?AVQString@@ABV3@AAVU2OpStatus@2@@Z 10039fc6 f   U2Core:U2Core.dll
 0001:00038fcc       ?addRow@MultipleSequenceAlignmentData@U2@@QAEXABVQString@@ABVQByteArray@@@Z 10039fcc f   U2Core:U2Core.dll
 0001:00038fd2       ?appendChars@MultipleSequenceAlignmentData@U2@@QAEXHPBDH@Z 10039fd2 f   U2Core:U2Core.dll
 0001:00038fd8       ?qt_metacast@Plugin@U2@@UAEPAXPBD@Z 10039fd8 f   U2Core:U2Core.dll
 0001:00038fde       ?qt_metacall@Plugin@U2@@UAEHW4Call@QMetaObject@@HPAPAX@Z 10039fde f   U2Core:U2Core.dll
 0001:00038fe4       ?qt_metacast@CmdlineTask@U2@@UAEPAXPBD@Z 10039fe4 f   U2Core:U2Core.dll
 0001:00038fea       ?qt_metacall@CmdlineTask@U2@@UAEHW4Call@QMetaObject@@HPAPAX@Z 10039fea f   U2Core:U2Core.dll
 0001:00038ff0       ??0PhyTreeGeneratorTask@U2@@QAE@ABVMultipleSequenceAlignment@1@ABVCreatePhyTreeSettings@1@@Z 10039ff0 f   U2Algorithm:U2Algorithm.dll
 0001:00038ff6       ??1PhyTreeGeneratorTask@U2@@UAE@XZ 10039ff6 f   U2Algorithm:U2Algorithm.dll
 0001:00038ffe       ?metaObject@PhyTreeGeneratorTask@U2@@UBEPBUQMetaObject@@XZ 10039ffe f   U2Algorithm:U2Algorithm.dll
 0001:00039004       ?qt_metacall@PhyTreeGeneratorTask@U2@@UAEHW4Call@QMetaObject@@HPAPAX@Z 1003a004 f   U2Algorithm:U2Algorithm.dll
 0001:0003900a       ?qt_metacast@PhyTreeGeneratorTask@U2@@UAEPAXPBD@Z 1003a00a f   U2Algorithm:U2Algorithm.dll
 0001:00039010       ?report@PhyTreeGeneratorTask@U2@@UAE?AW4ReportResult@Task@2@XZ 1003a010 f   U2Algorithm:U2Algorithm.dll
 0001:00039016       ?run@PhyTreeGeneratorTask@U2@@UAEXXZ 1003a016 f   U2Algorithm:U2Algorithm.dll
 0001:0003901c       ??0CreatePhyTreeSettings@U2@@QAE@XZ 1003a01c f   U2Algorithm:U2Algorithm.dll
 0001:00039022       ??1CreatePhyTreeSettings@U2@@QAE@XZ 1003a022 f   U2Algorithm:U2Algorithm.dll
 0001:00039028       ?registerPhyTreeGenerator@PhyTreeGeneratorRegistry@U2@@QAE_NPAVPhyTreeGenerator@2@ABVQString@@@Z 1003a028 f   U2Algorithm:U2Algorithm.dll
 0001:0003902e       ??0PhyTreeGeneratorLauncherTask@U2@@QAE@ABVMultipleSequenceAlignment@1@ABVCreatePhyTreeSettings@1@@Z 1003a02e f   U2Algorithm:U2Algorithm.dll
 0001:00039034       ??1PhyTreeGeneratorLauncherTask@U2@@UAE@XZ 1003a034 f   U2Algorithm:U2Algorithm.dll
 0001:0003903a       ?getResult@PhyTreeGeneratorLauncherTask@U2@@QAE?AV?$QSharedDataPointer@VPhyTreeData@U2@@@@XZ 1003a03a f   U2Algorithm:U2Algorithm.dll
 0001:00039040       ?metaObject@PhyTreeGeneratorLauncherTask@U2@@UBEPBUQMetaObject@@XZ 1003a040 f   U2Algorithm:U2Algorithm.dll
 0001:00039046       ?prepare@PhyTreeGeneratorLauncherTask@U2@@UAEXXZ 1003a046 f   U2Algorithm:U2Algorithm.dll
 0001:0003904c       ?qt_metacall@PhyTreeGeneratorLauncherTask@U2@@UAEHW4Call@QMetaObject@@HPAPAX@Z 1003a04c f   U2Algorithm:U2Algorithm.dll
 0001:00039052       ?qt_metacast@PhyTreeGeneratorLauncherTask@U2@@UAEPAXPBD@Z 1003a052 f   U2Algorithm:U2Algorithm.dll
 0001:00039058       ?report@PhyTreeGeneratorLauncherTask@U2@@UAE?AW4ReportResult@Task@2@XZ 1003a058 f   U2Algorithm:U2Algorithm.dll
 0001:0003905e       ?run@PhyTreeGeneratorLauncherTask@U2@@UAEXXZ 1003a05e f   U2Algorithm:U2Algorithm.dll
 0001:00039064       ??0CreatePhyTreeSettings@U2@@QAE@ABV01@@Z 1003a064 f   U2Algorithm:U2Algorithm.dll
 0001:0003906a       ?getResult@PhyTreeGeneratorTask@U2@@QAE?AV?$QSharedDataPointer@VPhyTreeData@U2@@@@XZ 1003a06a f   U2Algorithm:U2Algorithm.dll
 0001:00039070       ??4CreatePhyTreeSettings@U2@@QAEAAV01@ABV01@@Z 1003a070 f   U2Algorithm:U2Algorithm.dll
 0001:00039076       ??0CreatePhyTreeWidget@U2@@QAE@PAVQWidget@@@Z 1003a076 f   U2View:U2View.dll
 0001:0003907c       ?settingsPath@CreatePhyTreeWidget@U2@@SA?AVQString@@XZ 1003a07c f   U2View:U2View.dll
 0001:00039082       ??1CreatePhyTreeWidget@U2@@UAE@XZ 1003a082 f   U2View:U2View.dll
 0001:00039088       ??0PhyTreeDisplayOptionsWidget@U2@@QAE@PAVQWidget@@@Z 1003a088 f   U2View:U2View.dll
 0001:0003908e       ??1PhyTreeDisplayOptionsWidget@U2@@UAE@XZ 1003a08e f   U2View:U2View.dll
 0001:00039094       ?checkMemoryEstimation@CreatePhyTreeWidget@U2@@UAE_NAAVQString@@ABVMultipleSequenceAlignment@2@ABVCreatePhyTreeSettings@2@@Z 1003a094 f   U2View:U2View.dll
 0001:0003909a       ?checkSettings@CreatePhyTreeWidget@U2@@UAE_NAAVQString@@ABVCreatePhyTreeSettings@2@@Z 1003a09a f   U2View:U2View.dll
 0001:000390a0       ?fillSettings@PhyTreeDisplayOptionsWidget@U2@@UAEXAAVCreatePhyTreeSettings@2@@Z 1003a0a0 f   U2View:U2View.dll
 0001:000390a6       ?insertOutputOptionWidget@CreatePhyTreeWidget@U2@@UAE_NPAVPhyTreeDisplayOptionsWidget@2@@Z 1003a0a6 f   U2View:U2View.dll
 0001:000390ac       ?restoreDefault@PhyTreeDisplayOptionsWidget@U2@@UAEXXZ 1003a0ac f   U2View:U2View.dll
 0001:000390b2       ?storeSettings@PhyTreeDisplayOptionsWidget@U2@@UAEXXZ 1003a0b2 f   U2View:U2View.dll
 0001:000390b8       ?findFormat@GTestFormatRegistry@U2@@QAEPAVGTestFormat@2@ABVQString@@@Z 1003a0b8 f   U2Test:U2Test.dll
 0001:000390be       ?getContext@GTest@U2@@QBEPAVQObject@@ABVQString@@@Z 1003a0be f   U2Test:U2Test.dll
 0001:000390c4       ?failMissingValue@GTest@U2@@IAEXABVQString@@@Z 1003a0c4 f   U2Test:U2Test.dll
 0001:000390ca       ??0XMLTestFactory@U2@@QAE@ABVQString@@@Z 1003a0ca f   U2Test:U2Test.dll
 0001:000390d0       ??1XMLTestFactory@U2@@UAE@XZ 1003a0d0 f   U2Test:U2Test.dll
 0001:000390d6       ??0XmlTest@U2@@QAE@ABVQString@@PAVGTest@1@PBVGTestEnvironment@1@V?$QFlags@W4TaskFlag@U2@@@@ABV?$QList@PAVGTest@U2@@@@@Z 1003a0d6 f   U2Test:U2Test.dll
 0001:000390dc       ??1XmlTest@U2@@UAE@XZ      1003a0dc f   U2Test:U2Test.dll
 0001:000390e2       ?qt_metacast@GTest@U2@@UAEPAXPBD@Z 1003a0e2 f   U2Test:U2Test.dll
 0001:000390e8       ?qt_metacall@GTest@U2@@UAEHW4Call@QMetaObject@@HPAPAX@Z 1003a0e8 f   U2Test:U2Test.dll
 0001:000390ee       ??0QSizePolicy@@QAE@W4Policy@0@0W4ControlType@0@@Z 1003a0ee f   Qt5Widgets:Qt5Widgets.dll
 0001:000390f4       ?setHorizontalStretch@QSizePolicy@@QAEXH@Z 1003a0f4 f   Qt5Widgets:Qt5Widgets.dll
 0001:000390fa       ?setVerticalStretch@QSizePolicy@@QAEXH@Z 1003a0fa f   Qt5Widgets:Qt5Widgets.dll
 0001:00039100       ??0QWidget@@QAE@PAV0@V?$QFlags@W4WindowType@Qt@@@@@Z 1003a100 f   Qt5Widgets:Qt5Widgets.dll
 0001:00039106       ??1QWidget@@UAE@XZ         1003a106 f   Qt5Widgets:Qt5Widgets.dll
 0001:0003910c       ?setEnabled@QWidget@@QAEX_N@Z 1003a10c f   Qt5Widgets:Qt5Widgets.dll
 0001:00039112       ?setMinimumSize@QWidget@@QAEXHH@Z 1003a112 f   Qt5Widgets:Qt5Widgets.dll
 0001:00039118       ?resize@QWidget@@QAEXABVQSize@@@Z 1003a118 f   Qt5Widgets:Qt5Widgets.dll
 0001:0003911e       ?sizePolicy@QWidget@@QBE?AVQSizePolicy@@XZ 1003a11e f   Qt5Widgets:Qt5Widgets.dll
 0001:00039124       ?setSizePolicy@QWidget@@QAEXVQSizePolicy@@@Z 1003a124 f   Qt5Widgets:Qt5Widgets.dll
 0001:0003912a       ?setText@QAbstractButton@@QAEXABVQString@@@Z 1003a12a f   Qt5Widgets:Qt5Widgets.dll
 0001:00039130       ?isChecked@QAbstractButton@@QBE_NXZ 1003a130 f   Qt5Widgets:Qt5Widgets.dll
 0001:00039136       ?setChecked@QAbstractButton@@QAEX_N@Z 1003a136 f   Qt5Widgets:Qt5Widgets.dll
 0001:0003913c       ??0QCheckBox@@QAE@PAVQWidget@@@Z 1003a13c f   Qt5Widgets:Qt5Widgets.dll
 0001:00039142       ??1QCheckBox@@UAE@XZ       1003a142 f   Qt5Widgets:Qt5Widgets.dll
 0001:00039148       ??0QTabWidget@@QAE@PAVQWidget@@@Z 1003a148 f   Qt5Widgets:Qt5Widgets.dll
 0001:0003914e       ??1QTabWidget@@UAE@XZ      1003a14e f   Qt5Widgets:Qt5Widgets.dll
 0001:00039154       ?addTab@QTabWidget@@QAEHPAVQWidget@@ABVQString@@@Z 1003a154 f   Qt5Widgets:Qt5Widgets.dll
 0001:0003915a       ?setTabText@QTabWidget@@QAEXHABVQString@@@Z 1003a15a f   Qt5Widgets:Qt5Widgets.dll
 0001:00039160       ?indexOf@QTabWidget@@QBEHPAVQWidget@@@Z 1003a160 f   Qt5Widgets:Qt5Widgets.dll
 0001:00039166       ?setCurrentIndex@QTabWidget@@QAEXH@Z 1003a166 f   Qt5Widgets:Qt5Widgets.dll
 0001:0003916c       ??0QComboBox@@QAE@PAVQWidget@@@Z 1003a16c f   Qt5Widgets:Qt5Widgets.dll
 0001:00039172       ??1QComboBox@@UAE@XZ       1003a172 f   Qt5Widgets:Qt5Widgets.dll
 0001:00039178       ?count@QComboBox@@QBEHXZ   1003a178 f   Qt5Widgets:Qt5Widgets.dll
 0001:0003917e       ?findData@QComboBox@@QBEHABVQVariant@@HV?$QFlags@W4MatchFlag@Qt@@@@@Z 1003a17e f   Qt5Widgets:Qt5Widgets.dll
 0001:00039184       ?currentText@QComboBox@@QBE?AVQString@@XZ 1003a184 f   Qt5Widgets:Qt5Widgets.dll
 0001:0003918a       ?itemText@QComboBox@@QBE?AVQString@@H@Z 1003a18a f   Qt5Widgets:Qt5Widgets.dll
 0001:00039190       ?insertItems@QComboBox@@QAEXHABVQStringList@@@Z 1003a190 f   Qt5Widgets:Qt5Widgets.dll
 0001:00039196       ?setCurrentIndex@QComboBox@@QAEXH@Z 1003a196 f   Qt5Widgets:Qt5Widgets.dll
 0001:0003919c       ??0QSpinBox@@QAE@PAVQWidget@@@Z 1003a19c f   Qt5Widgets:Qt5Widgets.dll
 0001:000391a2       ??1QSpinBox@@UAE@XZ        1003a1a2 f   Qt5Widgets:Qt5Widgets.dll
 0001:000391a8       ?value@QSpinBox@@QBEHXZ    1003a1a8 f   Qt5Widgets:Qt5Widgets.dll
 0001:000391ae       ?setSingleStep@QSpinBox@@QAEXH@Z 1003a1ae f   Qt5Widgets:Qt5Widgets.dll
 0001:000391b4       ?setMinimum@QSpinBox@@QAEXH@Z 1003a1b4 f   Qt5Widgets:Qt5Widgets.dll
 0001:000391ba       ?setMaximum@QSpinBox@@QAEXH@Z 1003a1ba f   Qt5Widgets:Qt5Widgets.dll
 0001:000391c0       ?setValue@QSpinBox@@QAEXH@Z 1003a1c0 f   Qt5Widgets:Qt5Widgets.dll
 0001:000391c6       ??0QDoubleSpinBox@@QAE@PAVQWidget@@@Z 1003a1c6 f   Qt5Widgets:Qt5Widgets.dll
 0001:000391cc       ??1QDoubleSpinBox@@UAE@XZ  1003a1cc f   Qt5Widgets:Qt5Widgets.dll
 0001:000391d2       ?value@QDoubleSpinBox@@QBENXZ 1003a1d2 f   Qt5Widgets:Qt5Widgets.dll
 0001:000391d8       ?setSingleStep@QDoubleSpinBox@@QAEXN@Z 1003a1d8 f   Qt5Widgets:Qt5Widgets.dll
 0001:000391de       ?setMinimum@QDoubleSpinBox@@QAEXN@Z 1003a1de f   Qt5Widgets:Qt5Widgets.dll
 0001:000391e4       ?setMaximum@QDoubleSpinBox@@QAEXN@Z 1003a1e4 f   Qt5Widgets:Qt5Widgets.dll
 0001:000391ea       ?setDecimals@QDoubleSpinBox@@QAEXH@Z 1003a1ea f   Qt5Widgets:Qt5Widgets.dll
 0001:000391f0       ?setValue@QDoubleSpinBox@@QAEXN@Z 1003a1f0 f   Qt5Widgets:Qt5Widgets.dll
 0001:000391f6       ??0QSpacerItem@@QAE@HHW4Policy@QSizePolicy@@0@Z 1003a1f6 f   Qt5Widgets:Qt5Widgets.dll
 0001:000391fc       ??1QSpacerItem@@UAE@XZ     1003a1fc f   Qt5Widgets:Qt5Widgets.dll
 0001:00039202       ?setContentsMargins@QLayout@@QAEXHHHH@Z 1003a202 f   Qt5Widgets:Qt5Widgets.dll
 0001:00039208       ?setSizeConstraint@QLayout@@QAEXW4SizeConstraint@1@@Z 1003a208 f   Qt5Widgets:Qt5Widgets.dll
 0001:0003920e       ?addWidget@QBoxLayout@@QAEXPAVQWidget@@HV?$QFlags@W4AlignmentFlag@Qt@@@@@Z 1003a20e f   Qt5Widgets:Qt5Widgets.dll
 0001:00039214       ?addLayout@QBoxLayout@@QAEXPAVQLayout@@H@Z 1003a214 f   Qt5Widgets:Qt5Widgets.dll
 0001:0003921a       ?setSpacing@QBoxLayout@@QAEXH@Z 1003a21a f   Qt5Widgets:Qt5Widgets.dll
 0001:00039220       ??0QHBoxLayout@@QAE@XZ     1003a220 f   Qt5Widgets:Qt5Widgets.dll
 0001:00039226       ??1QHBoxLayout@@UAE@XZ     1003a226 f   Qt5Widgets:Qt5Widgets.dll
 0001:0003922c       ??0QVBoxLayout@@QAE@PAVQWidget@@@Z 1003a22c f   Qt5Widgets:Qt5Widgets.dll
 0001:00039232       ??1QVBoxLayout@@UAE@XZ     1003a232 f   Qt5Widgets:Qt5Widgets.dll
 0001:00039238       ??0QGridLayout@@QAE@XZ     1003a238 f   Qt5Widgets:Qt5Widgets.dll
 0001:0003923e       ??1QGridLayout@@UAE@XZ     1003a23e f   Qt5Widgets:Qt5Widgets.dll
 0001:00039244       ?addWidget@QGridLayout@@QAEXPAVQWidget@@HHHHV?$QFlags@W4AlignmentFlag@Qt@@@@@Z 1003a244 f   Qt5Widgets:Qt5Widgets.dll
 0001:0003924a       ??0QLabel@@QAE@PAVQWidget@@V?$QFlags@W4WindowType@Qt@@@@@Z 1003a24a f   Qt5Widgets:Qt5Widgets.dll
 0001:00039250       ??1QLabel@@UAE@XZ          1003a250 f   Qt5Widgets:Qt5Widgets.dll
 0001:00039256       ?setWordWrap@QLabel@@QAEX_N@Z 1003a256 f   Qt5Widgets:Qt5Widgets.dll
 0001:0003925c       ?setText@QLabel@@QAEXABVQString@@@Z 1003a25c f   Qt5Widgets:Qt5Widgets.dll
 0001:00039262       ?actionEvent@QWidget@@MAEXPAVQActionEvent@@@Z 1003a262 f   Qt5Widgets:Qt5Widgets.dll
 0001:00039268       ?addItem@QBoxLayout@@UAEXPAVQLayoutItem@@@Z 1003a268 f   Qt5Widgets:Qt5Widgets.dll
 0001:0003926e       ?addItem@QGridLayout@@MAEXPAVQLayoutItem@@@Z 1003a26e f   Qt5Widgets:Qt5Widgets.dll
 0001:00039274       ?changeEvent@QAbstractButton@@MAEXPAVQEvent@@@Z 1003a274 f   Qt5Widgets:Qt5Widgets.dll
 0001:0003927a       ?changeEvent@QAbstractSpinBox@@MAEXPAVQEvent@@@Z 1003a27a f   Qt5Widgets:Qt5Widgets.dll
 0001:00039280       ?changeEvent@QComboBox@@MAEXPAVQEvent@@@Z 1003a280 f   Qt5Widgets:Qt5Widgets.dll
 0001:00039286       ?changeEvent@QLabel@@MAEXPAVQEvent@@@Z 1003a286 f   Qt5Widgets:Qt5Widgets.dll
 0001:0003928c       ?changeEvent@QTabWidget@@MAEXPAVQEvent@@@Z 1003a28c f   Qt5Widgets:Qt5Widgets.dll
 0001:00039292       ?changeEvent@QWidget@@MAEXPAVQEvent@@@Z 1003a292 f   Qt5Widgets:Qt5Widgets.dll
 0001:00039298       ?checkStateSet@QCheckBox@@MAEXXZ 1003a298 f   Qt5Widgets:Qt5Widgets.dll
 0001:0003929e       ?childEvent@QLayout@@MAEXPAVQChildEvent@@@Z 1003a29e f   Qt5Widgets:Qt5Widgets.dll
 0001:000392a4       ?clear@QAbstractSpinBox@@UAEXXZ 1003a2a4 f   Qt5Widgets:Qt5Widgets.dll
 0001:000392aa       ?closeEvent@QAbstractSpinBox@@MAEXPAVQCloseEvent@@@Z 1003a2aa f   Qt5Widgets:Qt5Widgets.dll
 0001:000392b0       ?closeEvent@QWidget@@MAEXPAVQCloseEvent@@@Z 1003a2b0 f   Qt5Widgets:Qt5Widgets.dll
 0001:000392b6       ?contextMenuEvent@QAbstractSpinBox@@MAEXPAVQContextMenuEvent@@@Z 1003a2b6 f   Qt5Widgets:Qt5Widgets.dll
 0001:000392bc       ?contextMenuEvent@QComboBox@@MAEXPAVQContextMenuEvent@@@Z 1003a2bc f   Qt5Widgets:Qt5Widgets.dll
 0001:000392c2       ?contextMenuEvent@QLabel@@MAEXPAVQContextMenuEvent@@@Z 1003a2c2 f   Qt5Widgets:Qt5Widgets.dll
 0001:000392c8       ?contextMenuEvent@QWidget@@MAEXPAVQContextMenuEvent@@@Z 1003a2c8 f   Qt5Widgets:Qt5Widgets.dll
 0001:000392ce       ?controlTypes@QLayout@@UBE?AV?$QFlags@W4ControlType@QSizePolicy@@@@XZ 1003a2ce f   Qt5Widgets:Qt5Widgets.dll
 0001:000392d4       ?controlTypes@QLayoutItem@@UBE?AV?$QFlags@W4ControlType@QSizePolicy@@@@XZ 1003a2d4 f   Qt5Widgets:Qt5Widgets.dll
 0001:000392da       ?count@QBoxLayout@@UBEHXZ  1003a2da f   Qt5Widgets:Qt5Widgets.dll
 0001:000392e0       ?count@QGridLayout@@UBEHXZ 1003a2e0 f   Qt5Widgets:Qt5Widgets.dll
 0001:000392e6       ?devType@QWidget@@UBEHXZ   1003a2e6 f   Qt5Widgets:Qt5Widgets.dll
 0001:000392ec       ?dragEnterEvent@QWidget@@MAEXPAVQDragEnterEvent@@@Z 1003a2ec f   Qt5Widgets:Qt5Widgets.dll
 0001:000392f2       ?dragLeaveEvent@QWidget@@MAEXPAVQDragLeaveEvent@@@Z 1003a2f2 f   Qt5Widgets:Qt5Widgets.dll
 0001:000392f8       ?dragMoveEvent@QWidget@@MAEXPAVQDragMoveEvent@@@Z 1003a2f8 f   Qt5Widgets:Qt5Widgets.dll
 0001:000392fe       ?dropEvent@QWidget@@MAEXPAVQDropEvent@@@Z 1003a2fe f   Qt5Widgets:Qt5Widgets.dll
 0001:00039304       ?enterEvent@QWidget@@MAEXPAVQEvent@@@Z 1003a304 f   Qt5Widgets:Qt5Widgets.dll
 0001:0003930a       ?event@QAbstractSpinBox@@UAE_NPAVQEvent@@@Z 1003a30a f   Qt5Widgets:Qt5Widgets.dll
 0001:00039310       ?event@QCheckBox@@MAE_NPAVQEvent@@@Z 1003a310 f   Qt5Widgets:Qt5Widgets.dll
 0001:00039316       ?event@QComboBox@@UAE_NPAVQEvent@@@Z 1003a316 f   Qt5Widgets:Qt5Widgets.dll
 0001:0003931c       ?event@QLabel@@MAE_NPAVQEvent@@@Z 1003a31c f   Qt5Widgets:Qt5Widgets.dll
 0001:00039322       ?event@QSpinBox@@MAE_NPAVQEvent@@@Z 1003a322 f   Qt5Widgets:Qt5Widgets.dll
 0001:00039328       ?event@QTabWidget@@MAE_NPAVQEvent@@@Z 1003a328 f   Qt5Widgets:Qt5Widgets.dll
 0001:0003932e       ?event@QWidget@@MAE_NPAVQEvent@@@Z 1003a32e f   Qt5Widgets:Qt5Widgets.dll
 0001:00039334       ?expandingDirections@QBoxLayout@@UBE?AV?$QFlags@W4Orientation@Qt@@@@XZ 1003a334 f   Qt5Widgets:Qt5Widgets.dll
 0001:0003933a       ?expandingDirections@QGridLayout@@UBE?AV?$QFlags@W4Orientation@Qt@@@@XZ 1003a33a f   Qt5Widgets:Qt5Widgets.dll
 0001:00039340       ?expandingDirections@QSpacerItem@@UBE?AV?$QFlags@W4Orientation@Qt@@@@XZ 1003a340 f   Qt5Widgets:Qt5Widgets.dll
 0001:00039346       ?fixup@QDoubleSpinBox@@UBEXAAVQString@@@Z 1003a346 f   Qt5Widgets:Qt5Widgets.dll
 0001:0003934c       ?fixup@QSpinBox@@MBEXAAVQString@@@Z 1003a34c f   Qt5Widgets:Qt5Widgets.dll
 0001:00039352       ?focusInEvent@QAbstractButton@@MAEXPAVQFocusEvent@@@Z 1003a352 f   Qt5Widgets:Qt5Widgets.dll
 0001:00039358       ?focusInEvent@QAbstractSpinBox@@MAEXPAVQFocusEvent@@@Z 1003a358 f   Qt5Widgets:Qt5Widgets.dll
 0001:0003935e       ?focusInEvent@QComboBox@@MAEXPAVQFocusEvent@@@Z 1003a35e f   Qt5Widgets:Qt5Widgets.dll
 0001:00039364       ?focusInEvent@QLabel@@MAEXPAVQFocusEvent@@@Z 1003a364 f   Qt5Widgets:Qt5Widgets.dll
 0001:0003936a       ?focusInEvent@QWidget@@MAEXPAVQFocusEvent@@@Z 1003a36a f   Qt5Widgets:Qt5Widgets.dll
 0001:00039370       ?focusNextPrevChild@QLabel@@MAE_N_N@Z 1003a370 f   Qt5Widgets:Qt5Widgets.dll
 0001:00039376       ?focusNextPrevChild@QWidget@@MAE_N_N@Z 1003a376 f   Qt5Widgets:Qt5Widgets.dll
 0001:0003937c       ?focusOutEvent@QAbstractButton@@MAEXPAVQFocusEvent@@@Z 1003a37c f   Qt5Widgets:Qt5Widgets.dll
 0001:00039382       ?focusOutEvent@QAbstractSpinBox@@MAEXPAVQFocusEvent@@@Z 1003a382 f   Qt5Widgets:Qt5Widgets.dll
 0001:00039388       ?focusOutEvent@QComboBox@@MAEXPAVQFocusEvent@@@Z 1003a388 f   Qt5Widgets:Qt5Widgets.dll
 0001:0003938e       ?focusOutEvent@QLabel@@MAEXPAVQFocusEvent@@@Z 1003a38e f   Qt5Widgets:Qt5Widgets.dll
 0001:00039394       ?focusOutEvent@QWidget@@MAEXPAVQFocusEvent@@@Z 1003a394 f   Qt5Widgets:Qt5Widgets.dll
 0001:0003939a       ?geometry@QLayout@@UBE?AVQRect@@XZ 1003a39a f   Qt5Widgets:Qt5Widgets.dll
 0001:000393a0       ?geometry@QSpacerItem@@UBE?AVQRect@@XZ 1003a3a0 f   Qt5Widgets:Qt5Widgets.dll
 0001:000393a6       ?hasHeightForWidth@QBoxLayout@@UBE_NXZ 1003a3a6 f   Qt5Widgets:Qt5Widgets.dll
 0001:000393ac       ?hasHeightForWidth@QGridLayout@@UBE_NXZ 1003a3ac f   Qt5Widgets:Qt5Widgets.dll
 0001:000393b2       ?hasHeightForWidth@QLayoutItem@@UBE_NXZ 1003a3b2 f   Qt5Widgets:Qt5Widgets.dll
 0001:000393b8       ?hasHeightForWidth@QTabWidget@@UBE_NXZ 1003a3b8 f   Qt5Widgets:Qt5Widgets.dll
 0001:000393be       ?hasHeightForWidth@QWidget@@UBE_NXZ 1003a3be f   Qt5Widgets:Qt5Widgets.dll
 0001:000393c4       ?heightForWidth@QBoxLayout@@UBEHH@Z 1003a3c4 f   Qt5Widgets:Qt5Widgets.dll
 0001:000393ca       ?heightForWidth@QGridLayout@@UBEHH@Z 1003a3ca f   Qt5Widgets:Qt5Widgets.dll
 0001:000393d0       ?heightForWidth@QLabel@@UBEHH@Z 1003a3d0 f   Qt5Widgets:Qt5Widgets.dll
 0001:000393d6       ?heightForWidth@QLayoutItem@@UBEHH@Z 1003a3d6 f   Qt5Widgets:Qt5Widgets.dll
 0001:000393dc       ?heightForWidth@QTabWidget@@UBEHH@Z 1003a3dc f   Qt5Widgets:Qt5Widgets.dll
 0001:000393e2       ?heightForWidth@QWidget@@UBEHH@Z 1003a3e2 f   Qt5Widgets:Qt5Widgets.dll
 0001:000393e8       ?hideEvent@QAbstractSpinBox@@MAEXPAVQHideEvent@@@Z 1003a3e8 f   Qt5Widgets:Qt5Widgets.dll
 0001:000393ee       ?hideEvent@QComboBox@@MAEXPAVQHideEvent@@@Z 1003a3ee f   Qt5Widgets:Qt5Widgets.dll
 0001:000393f4       ?hideEvent@QWidget@@MAEXPAVQHideEvent@@@Z 1003a3f4 f   Qt5Widgets:Qt5Widgets.dll
 0001:000393fa       ?hidePopup@QComboBox@@UAEXXZ 1003a3fa f   Qt5Widgets:Qt5Widgets.dll
 0001:00039400       ?hitButton@QCheckBox@@MBE_NABVQPoint@@@Z 1003a400 f   Qt5Widgets:Qt5Widgets.dll
 0001:00039406       ?indexOf@QLayout@@UBEHPAVQWidget@@@Z 1003a406 f   Qt5Widgets:Qt5Widgets.dll
 0001:0003940c       ?initPainter@QWidget@@MBEXPAVQPainter@@@Z 1003a40c f   Qt5Widgets:Qt5Widgets.dll
 0001:00039412       ?inputMethodEvent@QComboBox@@MAEXPAVQInputMethodEvent@@@Z 1003a412 f   Qt5Widgets:Qt5Widgets.dll
 0001:00039418       ?inputMethodEvent@QWidget@@MAEXPAVQInputMethodEvent@@@Z 1003a418 f   Qt5Widgets:Qt5Widgets.dll
 0001:0003941e       ?inputMethodQuery@QAbstractSpinBox@@UBE?AVQVariant@@W4InputMethodQuery@Qt@@@Z 1003a41e f   Qt5Widgets:Qt5Widgets.dll
 0001:00039424       ?inputMethodQuery@QComboBox@@UBE?AVQVariant@@W4InputMethodQuery@Qt@@@Z 1003a424 f   Qt5Widgets:Qt5Widgets.dll
 0001:0003942a       ?inputMethodQuery@QWidget@@UBE?AVQVariant@@W4InputMethodQuery@Qt@@@Z 1003a42a f   Qt5Widgets:Qt5Widgets.dll
 0001:00039430       ?invalidate@QBoxLayout@@UAEXXZ 1003a430 f   Qt5Widgets:Qt5Widgets.dll
 0001:00039436       ?invalidate@QGridLayout@@UAEXXZ 1003a436 f   Qt5Widgets:Qt5Widgets.dll
 0001:0003943c       ?invalidate@QLayoutItem@@UAEXXZ 1003a43c f   Qt5Widgets:Qt5Widgets.dll
 0001:00039442       ?isEmpty@QLayout@@UBE_NXZ  1003a442 f   Qt5Widgets:Qt5Widgets.dll
 0001:00039448       ?isEmpty@QSpacerItem@@UBE_NXZ 1003a448 f   Qt5Widgets:Qt5Widgets.dll
 0001:0003944e       ?itemAt@QBoxLayout@@UBEPAVQLayoutItem@@H@Z 1003a44e f   Qt5Widgets:Qt5Widgets.dll
 0001:00039454       ?itemAt@QGridLayout@@UBEPAVQLayoutItem@@H@Z 1003a454 f   Qt5Widgets:Qt5Widgets.dll
 0001:0003945a       ?keyPressEvent@QAbstractButton@@MAEXPAVQKeyEvent@@@Z 1003a45a f   Qt5Widgets:Qt5Widgets.dll
 0001:00039460       ?keyPressEvent@QAbstractSpinBox@@MAEXPAVQKeyEvent@@@Z 1003a460 f   Qt5Widgets:Qt5Widgets.dll
 0001:00039466       ?keyPressEvent@QComboBox@@MAEXPAVQKeyEvent@@@Z 1003a466 f   Qt5Widgets:Qt5Widgets.dll
 0001:0003946c       ?keyPressEvent@QLabel@@MAEXPAVQKeyEvent@@@Z 1003a46c f   Qt5Widgets:Qt5Widgets.dll
 0001:00039472       ?keyPressEvent@QTabWidget@@MAEXPAVQKeyEvent@@@Z 1003a472 f   Qt5Widgets:Qt5Widgets.dll
 0001:00039478       ?keyPressEvent@QWidget@@MAEXPAVQKeyEvent@@@Z 1003a478 f   Qt5Widgets:Qt5Widgets.dll
 0001:0003947e       ?keyReleaseEvent@QAbstractButton@@MAEXPAVQKeyEvent@@@Z 1003a47e f   Qt5Widgets:Qt5Widgets.dll
 0001:00039484       ?keyReleaseEvent@QAbstractSpinBox@@MAEXPAVQKeyEvent@@@Z 1003a484 f   Qt5Widgets:Qt5Widgets.dll
 0001:0003948a       ?keyReleaseEvent@QComboBox@@MAEXPAVQKeyEvent@@@Z 1003a48a f   Qt5Widgets:Qt5Widgets.dll
 0001:00039490       ?keyReleaseEvent@QWidget@@MAEXPAVQKeyEvent@@@Z 1003a490 f   Qt5Widgets:Qt5Widgets.dll
 0001:00039496       ?layout@QLayout@@UAEPAV1@XZ 1003a496 f   Qt5Widgets:Qt5Widgets.dll
 0001:0003949c       ?layout@QLayoutItem@@UAEPAVQLayout@@XZ 1003a49c f   Qt5Widgets:Qt5Widgets.dll
 0001:000394a2       ?leaveEvent@QWidget@@MAEXPAVQEvent@@@Z 1003a4a2 f   Qt5Widgets:Qt5Widgets.dll
 0001:000394a8       ?maximumSize@QBoxLayout@@UBE?AVQSize@@XZ 1003a4a8 f   Qt5Widgets:Qt5Widgets.dll
 0001:000394ae       ?maximumSize@QGridLayout@@UBE?AVQSize@@XZ 1003a4ae f   Qt5Widgets:Qt5Widgets.dll
 0001:000394b4       ?maximumSize@QSpacerItem@@UBE?AVQSize@@XZ 1003a4b4 f   Qt5Widgets:Qt5Widgets.dll
 0001:000394ba       ?metaObject@QCheckBox@@UBEPBUQMetaObject@@XZ 1003a4ba f   Qt5Widgets:Qt5Widgets.dll
 0001:000394c0       ?metaObject@QComboBox@@UBEPBUQMetaObject@@XZ 1003a4c0 f   Qt5Widgets:Qt5Widgets.dll
 0001:000394c6       ?metaObject@QDoubleSpinBox@@UBEPBUQMetaObject@@XZ 1003a4c6 f   Qt5Widgets:Qt5Widgets.dll
 0001:000394cc       ?metaObject@QGridLayout@@UBEPBUQMetaObject@@XZ 1003a4cc f   Qt5Widgets:Qt5Widgets.dll
 0001:000394d2       ?metaObject@QHBoxLayout@@UBEPBUQMetaObject@@XZ 1003a4d2 f   Qt5Widgets:Qt5Widgets.dll
 0001:000394d8       ?metaObject@QLabel@@UBEPBUQMetaObject@@XZ 1003a4d8 f   Qt5Widgets:Qt5Widgets.dll
 0001:000394de       ?metaObject@QSpinBox@@UBEPBUQMetaObject@@XZ 1003a4de f   Qt5Widgets:Qt5Widgets.dll
 0001:000394e4       ?metaObject@QTabWidget@@UBEPBUQMetaObject@@XZ 1003a4e4 f   Qt5Widgets:Qt5Widgets.dll
 0001:000394ea       ?metaObject@QVBoxLayout@@UBEPBUQMetaObject@@XZ 1003a4ea f   Qt5Widgets:Qt5Widgets.dll
 0001:000394f0       ?metaObject@QWidget@@UBEPBUQMetaObject@@XZ 1003a4f0 f   Qt5Widgets:Qt5Widgets.dll
 0001:000394f6       ?metric@QWidget@@MBEHW4PaintDeviceMetric@QPaintDevice@@@Z 1003a4f6 f   Qt5Widgets:Qt5Widgets.dll
 0001:000394fc       ?minimumHeightForWidth@QBoxLayout@@UBEHH@Z 1003a4fc f   Qt5Widgets:Qt5Widgets.dll
 0001:00039502       ?minimumHeightForWidth@QGridLayout@@UBEHH@Z 1003a502 f   Qt5Widgets:Qt5Widgets.dll
 0001:00039508       ?minimumHeightForWidth@QLayoutItem@@UBEHH@Z 1003a508 f   Qt5Widgets:Qt5Widgets.dll
 0001:0003950e       ?minimumSize@QBoxLayout@@UBE?AVQSize@@XZ 1003a50e f   Qt5Widgets:Qt5Widgets.dll
 0001:00039514       ?minimumSize@QGridLayout@@UBE?AVQSize@@XZ 1003a514 f   Qt5Widgets:Qt5Widgets.dll
 0001:0003951a       ?minimumSize@QSpacerItem@@UBE?AVQSize@@XZ 1003a51a f   Qt5Widgets:Qt5Widgets.dll
 0001:00039520       ?minimumSizeHint@QAbstractSpinBox@@UBE?AVQSize@@XZ 1003a520 f   Qt5Widgets:Qt5Widgets.dll
 0001:00039526       ?minimumSizeHint@QCheckBox@@UBE?AVQSize@@XZ 1003a526 f   Qt5Widgets:Qt5Widgets.dll
 0001:0003952c       ?minimumSizeHint@QComboBox@@UBE?AVQSize@@XZ 1003a52c f   Qt5Widgets:Qt5Widgets.dll
 0001:00039532       ?minimumSizeHint@QLabel@@UBE?AVQSize@@XZ 1003a532 f   Qt5Widgets:Qt5Widgets.dll
 0001:00039538       ?minimumSizeHint@QTabWidget@@UBE?AVQSize@@XZ 1003a538 f   Qt5Widgets:Qt5Widgets.dll
 0001:0003953e       ?minimumSizeHint@QWidget@@UBE?AVQSize@@XZ 1003a53e f   Qt5Widgets:Qt5Widgets.dll
 0001:00039544       ?mouseDoubleClickEvent@QWidget@@MAEXPAVQMouseEvent@@@Z 1003a544 f   Qt5Widgets:Qt5Widgets.dll
 0001:0003954a       ?mouseMoveEvent@QAbstractSpinBox@@MAEXPAVQMouseEvent@@@Z 1003a54a f   Qt5Widgets:Qt5Widgets.dll
 0001:00039550       ?mouseMoveEvent@QCheckBox@@MAEXPAVQMouseEvent@@@Z 1003a550 f   Qt5Widgets:Qt5Widgets.dll
 0001:00039556       ?mouseMoveEvent@QLabel@@MAEXPAVQMouseEvent@@@Z 1003a556 f   Qt5Widgets:Qt5Widgets.dll
 0001:0003955c       ?mouseMoveEvent@QWidget@@MAEXPAVQMouseEvent@@@Z 1003a55c f   Qt5Widgets:Qt5Widgets.dll
 0001:00039562       ?mousePressEvent@QAbstractButton@@MAEXPAVQMouseEvent@@@Z 1003a562 f   Qt5Widgets:Qt5Widgets.dll
 0001:00039568       ?mousePressEvent@QAbstractSpinBox@@MAEXPAVQMouseEvent@@@Z 1003a568 f   Qt5Widgets:Qt5Widgets.dll
 0001:0003956e       ?mousePressEvent@QComboBox@@MAEXPAVQMouseEvent@@@Z 1003a56e f   Qt5Widgets:Qt5Widgets.dll
 0001:00039574       ?mousePressEvent@QLabel@@MAEXPAVQMouseEvent@@@Z 1003a574 f   Qt5Widgets:Qt5Widgets.dll
 0001:0003957a       ?mousePressEvent@QWidget@@MAEXPAVQMouseEvent@@@Z 1003a57a f   Qt5Widgets:Qt5Widgets.dll
 0001:00039580       ?mouseReleaseEvent@QAbstractButton@@MAEXPAVQMouseEvent@@@Z 1003a580 f   Qt5Widgets:Qt5Widgets.dll
 0001:00039586       ?mouseReleaseEvent@QAbstractSpinBox@@MAEXPAVQMouseEvent@@@Z 1003a586 f   Qt5Widgets:Qt5Widgets.dll
 0001:0003958c       ?mouseReleaseEvent@QComboBox@@MAEXPAVQMouseEvent@@@Z 1003a58c f   Qt5Widgets:Qt5Widgets.dll
 0001:00039592       ?mouseReleaseEvent@QLabel@@MAEXPAVQMouseEvent@@@Z 1003a592 f   Qt5Widgets:Qt5Widgets.dll
 0001:00039598       ?mouseReleaseEvent@QWidget@@MAEXPAVQMouseEvent@@@Z 1003a598 f   Qt5Widgets:Qt5Widgets.dll
 0001:0003959e       ?moveEvent@QWidget@@MAEXPAVQMoveEvent@@@Z 1003a59e f   Qt5Widgets:Qt5Widgets.dll
 0001:000395a4       ?nativeEvent@QWidget@@MAE_NABVQByteArray@@PAXPAJ@Z 1003a5a4 f   Qt5Widgets:Qt5Widgets.dll
 0001:000395aa       ?nextCheckState@QCheckBox@@MAEXXZ 1003a5aa f   Qt5Widgets:Qt5Widgets.dll
 0001:000395b0       ?paintEngine@QWidget@@UBEPAVQPaintEngine@@XZ 1003a5b0 f   Qt5Widgets:Qt5Widgets.dll
 0001:000395b6       ?paintEvent@QAbstractSpinBox@@MAEXPAVQPaintEvent@@@Z 1003a5b6 f   Qt5Widgets:Qt5Widgets.dll
 0001:000395bc       ?paintEvent@QCheckBox@@MAEXPAVQPaintEvent@@@Z 1003a5bc f   Qt5Widgets:Qt5Widgets.dll
 0001:000395c2       ?paintEvent@QComboBox@@MAEXPAVQPaintEvent@@@Z 1003a5c2 f   Qt5Widgets:Qt5Widgets.dll
 0001:000395c8       ?paintEvent@QLabel@@MAEXPAVQPaintEvent@@@Z 1003a5c8 f   Qt5Widgets:Qt5Widgets.dll
 0001:000395ce       ?paintEvent@QTabWidget@@MAEXPAVQPaintEvent@@@Z 1003a5ce f   Qt5Widgets:Qt5Widgets.dll
 0001:000395d4       ?paintEvent@QWidget@@MAEXPAVQPaintEvent@@@Z 1003a5d4 f   Qt5Widgets:Qt5Widgets.dll
 0001:000395da       ?qt_metacall@QCheckBox@@UAEHW4Call@QMetaObject@@HPAPAX@Z 1003a5da f   Qt5Widgets:Qt5Widgets.dll
 0001:000395e0       ?qt_metacall@QComboBox@@UAEHW4Call@QMetaObject@@HPAPAX@Z 1003a5e0 f   Qt5Widgets:Qt5Widgets.dll
 0001:000395e6       ?qt_metacall@QDoubleSpinBox@@UAEHW4Call@QMetaObject@@HPAPAX@Z 1003a5e6 f   Qt5Widgets:Qt5Widgets.dll
 0001:000395ec       ?qt_metacall@QGridLayout@@UAEHW4Call@QMetaObject@@HPAPAX@Z 1003a5ec f   Qt5Widgets:Qt5Widgets.dll
 0001:000395f2       ?qt_metacall@QHBoxLayout@@UAEHW4Call@QMetaObject@@HPAPAX@Z 1003a5f2 f   Qt5Widgets:Qt5Widgets.dll
 0001:000395f8       ?qt_metacall@QLabel@@UAEHW4Call@QMetaObject@@HPAPAX@Z 1003a5f8 f   Qt5Widgets:Qt5Widgets.dll
 0001:000395fe       ?qt_metacall@QSpinBox@@UAEHW4Call@QMetaObject@@HPAPAX@Z 1003a5fe f   Qt5Widgets:Qt5Widgets.dll
 0001:00039604       ?qt_metacall@QTabWidget@@UAEHW4Call@QMetaObject@@HPAPAX@Z 1003a604 f   Qt5Widgets:Qt5Widgets.dll
 0001:0003960a       ?qt_metacall@QVBoxLayout@@UAEHW4Call@QMetaObject@@HPAPAX@Z 1003a60a f   Qt5Widgets:Qt5Widgets.dll
 0001:00039610       ?qt_metacall@QWidget@@UAEHW4Call@QMetaObject@@HPAPAX@Z 1003a610 f   Qt5Widgets:Qt5Widgets.dll
 0001:00039616       ?qt_metacast@QCheckBox@@UAEPAXPBD@Z 1003a616 f   Qt5Widgets:Qt5Widgets.dll
 0001:0003961c       ?qt_metacast@QComboBox@@UAEPAXPBD@Z 1003a61c f   Qt5Widgets:Qt5Widgets.dll
 0001:00039622       ?qt_metacast@QDoubleSpinBox@@UAEPAXPBD@Z 1003a622 f   Qt5Widgets:Qt5Widgets.dll
 0001:00039628       ?qt_metacast@QGridLayout@@UAEPAXPBD@Z 1003a628 f   Qt5Widgets:Qt5Widgets.dll
 0001:0003962e       ?qt_metacast@QHBoxLayout@@UAEPAXPBD@Z 1003a62e f   Qt5Widgets:Qt5Widgets.dll
 0001:00039634       ?qt_metacast@QLabel@@UAEPAXPBD@Z 1003a634 f   Qt5Widgets:Qt5Widgets.dll
 0001:0003963a       ?qt_metacast@QSpinBox@@UAEPAXPBD@Z 1003a63a f   Qt5Widgets:Qt5Widgets.dll
 0001:00039640       ?qt_metacast@QTabWidget@@UAEPAXPBD@Z 1003a640 f   Qt5Widgets:Qt5Widgets.dll
 0001:00039646       ?qt_metacast@QVBoxLayout@@UAEPAXPBD@Z 1003a646 f   Qt5Widgets:Qt5Widgets.dll
 0001:0003964c       ?qt_metacast@QWidget@@UAEPAXPBD@Z 1003a64c f   Qt5Widgets:Qt5Widgets.dll
 0001:00039652       ?redirected@QWidget@@MBEPAVQPaintDevice@@PAVQPoint@@@Z 1003a652 f   Qt5Widgets:Qt5Widgets.dll
 0001:00039658       ?resizeEvent@QAbstractSpinBox@@MAEXPAVQResizeEvent@@@Z 1003a658 f   Qt5Widgets:Qt5Widgets.dll
 0001:0003965e       ?resizeEvent@QComboBox@@MAEXPAVQResizeEvent@@@Z 1003a65e f   Qt5Widgets:Qt5Widgets.dll
 0001:00039664       ?resizeEvent@QTabWidget@@MAEXPAVQResizeEvent@@@Z 1003a664 f   Qt5Widgets:Qt5Widgets.dll
 0001:0003966a       ?resizeEvent@QWidget@@MAEXPAVQResizeEvent@@@Z 1003a66a f   Qt5Widgets:Qt5Widgets.dll
 0001:00039670       ?setGeometry@QBoxLayout@@UAEXABVQRect@@@Z 1003a670 f   Qt5Widgets:Qt5Widgets.dll
 0001:00039676       ?setGeometry@QGridLayout@@UAEXABVQRect@@@Z 1003a676 f   Qt5Widgets:Qt5Widgets.dll
 0001:0003967c       ?setGeometry@QSpacerItem@@UAEXABVQRect@@@Z 1003a67c f   Qt5Widgets:Qt5Widgets.dll
 0001:00039682       ?setVisible@QWidget@@UAEX_N@Z 1003a682 f   Qt5Widgets:Qt5Widgets.dll
 0001:00039688       ?sharedPainter@QWidget@@MBEPAVQPainter@@XZ 1003a688 f   Qt5Widgets:Qt5Widgets.dll
 0001:0003968e       ?showEvent@QAbstractSpinBox@@MAEXPAVQShowEvent@@@Z 1003a68e f   Qt5Widgets:Qt5Widgets.dll
 0001:00039694       ?showEvent@QComboBox@@MAEXPAVQShowEvent@@@Z 1003a694 f   Qt5Widgets:Qt5Widgets.dll
 0001:0003969a       ?showEvent@QTabWidget@@MAEXPAVQShowEvent@@@Z 1003a69a f   Qt5Widgets:Qt5Widgets.dll
 0001:000396a0       ?showEvent@QWidget@@MAEXPAVQShowEvent@@@Z 1003a6a0 f   Qt5Widgets:Qt5Widgets.dll
 0001:000396a6       ?showPopup@QComboBox@@UAEXXZ 1003a6a6 f   Qt5Widgets:Qt5Widgets.dll
 0001:000396ac       ?sizeHint@QAbstractSpinBox@@UBE?AVQSize@@XZ 1003a6ac f   Qt5Widgets:Qt5Widgets.dll
 0001:000396b2       ?sizeHint@QBoxLayout@@UBE?AVQSize@@XZ 1003a6b2 f   Qt5Widgets:Qt5Widgets.dll
 0001:000396b8       ?sizeHint@QCheckBox@@UBE?AVQSize@@XZ 1003a6b8 f   Qt5Widgets:Qt5Widgets.dll
 0001:000396be       ?sizeHint@QComboBox@@UBE?AVQSize@@XZ 1003a6be f   Qt5Widgets:Qt5Widgets.dll
 0001:000396c4       ?sizeHint@QGridLayout@@UBE?AVQSize@@XZ 1003a6c4 f   Qt5Widgets:Qt5Widgets.dll
 0001:000396ca       ?sizeHint@QLabel@@UBE?AVQSize@@XZ 1003a6ca f   Qt5Widgets:Qt5Widgets.dll
 0001:000396d0       ?sizeHint@QSpacerItem@@UBE?AVQSize@@XZ 1003a6d0 f   Qt5Widgets:Qt5Widgets.dll
 0001:000396d6       ?sizeHint@QTabWidget@@UBE?AVQSize@@XZ 1003a6d6 f   Qt5Widgets:Qt5Widgets.dll
 0001:000396dc       ?sizeHint@QWidget@@UBE?AVQSize@@XZ 1003a6dc f   Qt5Widgets:Qt5Widgets.dll
 0001:000396e2       ?spacerItem@QLayoutItem@@UAEPAVQSpacerItem@@XZ 1003a6e2 f   Qt5Widgets:Qt5Widgets.dll
 0001:000396e8       ?spacerItem@QSpacerItem@@UAEPAV1@XZ 1003a6e8 f   Qt5Widgets:Qt5Widgets.dll
 0001:000396ee       ?stepBy@QAbstractSpinBox@@UAEXH@Z 1003a6ee f   Qt5Widgets:Qt5Widgets.dll
 0001:000396f4       ?stepEnabled@QAbstractSpinBox@@MBE?AV?$QFlags@W4StepEnabledFlag@QAbstractSpinBox@@@@XZ 1003a6f4 f   Qt5Widgets:Qt5Widgets.dll
 0001:000396fa       ?tabInserted@QTabWidget@@MAEXH@Z 1003a6fa f   Qt5Widgets:Qt5Widgets.dll
 0001:00039700       ?tabRemoved@QTabWidget@@MAEXH@Z 1003a700 f   Qt5Widgets:Qt5Widgets.dll
 0001:00039706       ?tabletEvent@QWidget@@MAEXPAVQTabletEvent@@@Z 1003a706 f   Qt5Widgets:Qt5Widgets.dll
 0001:0003970c       ?takeAt@QBoxLayout@@UAEPAVQLayoutItem@@H@Z 1003a70c f   Qt5Widgets:Qt5Widgets.dll
 0001:00039712       ?takeAt@QGridLayout@@UAEPAVQLayoutItem@@H@Z 1003a712 f   Qt5Widgets:Qt5Widgets.dll
 0001:00039718       ?textFromValue@QDoubleSpinBox@@UBE?AVQString@@N@Z 1003a718 f   Qt5Widgets:Qt5Widgets.dll
 0001:0003971e       ?textFromValue@QSpinBox@@MBE?AVQString@@H@Z 1003a71e f   Qt5Widgets:Qt5Widgets.dll
 0001:00039724       ?timerEvent@QAbstractButton@@MAEXPAVQTimerEvent@@@Z 1003a724 f   Qt5Widgets:Qt5Widgets.dll
 0001:0003972a       ?timerEvent@QAbstractSpinBox@@MAEXPAVQTimerEvent@@@Z 1003a72a f   Qt5Widgets:Qt5Widgets.dll
 0001:00039730       ?validate@QDoubleSpinBox@@UBE?AW4State@QValidator@@AAVQString@@AAH@Z 1003a730 f   Qt5Widgets:Qt5Widgets.dll
 0001:00039736       ?validate@QSpinBox@@MBE?AW4State@QValidator@@AAVQString@@AAH@Z 1003a736 f   Qt5Widgets:Qt5Widgets.dll
 0001:0003973c       ?valueFromText@QDoubleSpinBox@@UBENABVQString@@@Z 1003a73c f   Qt5Widgets:Qt5Widgets.dll
 0001:00039742       ?valueFromText@QSpinBox@@MBEHABVQString@@@Z 1003a742 f   Qt5Widgets:Qt5Widgets.dll
 0001:00039748       ?wheelEvent@QAbstractSpinBox@@MAEXPAVQWheelEvent@@@Z 1003a748 f   Qt5Widgets:Qt5Widgets.dll
 0001:0003974e       ?wheelEvent@QComboBox@@MAEXPAVQWheelEvent@@@Z 1003a74e f   Qt5Widgets:Qt5Widgets.dll
 0001:00039754       ?wheelEvent@QWidget@@MAEXPAVQWheelEvent@@@Z 1003a754 f   Qt5Widgets:Qt5Widgets.dll
 0001:0003975a       ?widget@QLayoutItem@@UAEPAVQWidget@@XZ 1003a75a f   Qt5Widgets:Qt5Widgets.dll
 0001:00039760       ?attribute@QDomElement@@QBE?AVQString@@ABV2@0@Z 1003a760 f   Qt5Xml:Qt5Xml.dll
 0001:00039766       ?qBadAlloc@@YAXXZ          1003a766 f   Qt5Core:Qt5Core.dll
 0001:0003976c       ?data@QArrayData@@QAEPAXXZ 1003a76c f   Qt5Core:Qt5Core.dll
 0001:00039772       ?allocate@QArrayData@@SAPAU1@IIIV?$QFlags@W4AllocationOption@QArrayData@@@@@Z 1003a772 f   Qt5Core:Qt5Core.dll
 0001:00039778       ?deallocate@QArrayData@@SAXPAU1@II@Z 1003a778 f   Qt5Core:Qt5Core.dll
 0001:0003977e       ?detach@QListData@@QAEPAUData@1@H@Z 1003a77e f   Qt5Core:Qt5Core.dll
 0001:00039784       ?detach_grow@QListData@@QAEPAUData@1@PAHH@Z 1003a784 f   Qt5Core:Qt5Core.dll
 0001:0003978a       ?realloc@QListData@@QAEXH@Z 1003a78a f   Qt5Core:Qt5Core.dll
 0001:00039790       ?dispose@QListData@@SAXPAUData@1@@Z 1003a790 f   Qt5Core:Qt5Core.dll
 0001:00039796       ?append@QListData@@QAEPAPAXXZ 1003a796 f   Qt5Core:Qt5Core.dll
 0001:0003979c       ??1QByteArray@@QAE@XZ      1003a79c f   Qt5Core:Qt5Core.dll
 0001:000397a2       ?constData@QByteArray@@QBEPBDXZ 1003a7a2 f   Qt5Core:Qt5Core.dll
 0001:000397a8       ?nextNode@QMapNodeBase@@QBEPBU1@XZ 1003a7a8 f   Qt5Core:Qt5Core.dll
 0001:000397ae       ?freeNodeAndRebalance@QMapDataBase@@QAEXPAUQMapNodeBase@@@Z 1003a7ae f   Qt5Core:Qt5Core.dll
 0001:000397b4       ?recalcMostLeftNode@QMapDataBase@@QAEXXZ 1003a7b4 f   Qt5Core:Qt5Core.dll
 0001:000397ba       ?createNode@QMapDataBase@@QAEPAUQMapNodeBase@@HHPAU2@_N@Z 1003a7ba f   Qt5Core:Qt5Core.dll
 0001:000397c0       ?freeTree@QMapDataBase@@QAEXPAUQMapNodeBase@@H@Z 1003a7c0 f   Qt5Core:Qt5Core.dll
 0001:000397c6       ?createData@QMapDataBase@@SAPAU1@XZ 1003a7c6 f   Qt5Core:Qt5Core.dll
 0001:000397cc       ?freeData@QMapDataBase@@SAXPAU1@@Z 1003a7cc f   Qt5Core:Qt5Core.dll
 0001:000397d2       ??0QChar@@QAE@UQLatin1Char@@@Z 1003a7d2 f   Qt5Core:Qt5Core.dll
 0001:000397d8       ??0QString@@QAE@XZ         1003a7d8 f   Qt5Core:Qt5Core.dll
 0001:000397de       ??0QString@@QAE@ABV0@@Z    1003a7de f   Qt5Core:Qt5Core.dll
 0001:000397e4       ??1QString@@QAE@XZ         1003a7e4 f   Qt5Core:Qt5Core.dll
 0001:000397ea       ??4QString@@QAEAAV0@ABV0@@Z 1003a7ea f   Qt5Core:Qt5Core.dll
 0001:000397f0       ??4QString@@QAEAAV0@$$QAV0@@Z 1003a7f0 f   Qt5Core:Qt5Core.dll
 0001:000397f6       ?arg@QString@@QBE?AV1@HHHVQChar@@@Z 1003a7f6 f   Qt5Core:Qt5Core.dll
 0001:000397fc       ?arg@QString@@QBE?AV1@ABV1@HVQChar@@@Z 1003a7fc f   Qt5Core:Qt5Core.dll
 0001:00039802       ?startsWith@QString@@QBE_NABV1@W4CaseSensitivity@Qt@@@Z 1003a802 f   Qt5Core:Qt5Core.dll
 0001:00039808       ?append@QString@@QAEAAV1@ABV1@@Z 1003a808 f   Qt5Core:Qt5Core.dll
 0001:0003980e       ?toLatin1@QString@@QBE?AVQByteArray@@XZ 1003a80e f   Qt5Core:Qt5Core.dll
 0001:00039814       ??8@YA_NABVQString@@0@Z    1003a814 f   Qt5Core:Qt5Core.dll
 0001:0003981a       ??M@YA_NABVQString@@0@Z    1003a81a f   Qt5Core:Qt5Core.dll
 0001:00039820       ?append@QString@@QAEAAV1@PBD@Z 1003a820 f   Qt5Core:Qt5Core.dll
 0001:00039826       ??9QString@@QBE_NPBD@Z     1003a826 f   Qt5Core:Qt5Core.dll
 0001:0003982c       ?fromAscii_helper@QString@@CAPAU?$QTypedArrayData@G@@PBDH@Z 1003a82c f   Qt5Core:Qt5Core.dll
 0001:00039832       ??0QMutex@@QAE@W4RecursionMode@0@@Z 1003a832 f   Qt5Core:Qt5Core.dll
 0001:00039838       ??1QMutex@@QAE@XZ          1003a838 f   Qt5Core:Qt5Core.dll
 0001:0003983e       ??0QMutexLocker@@QAE@PAVQBasicMutex@@@Z 1003a83e f   Qt5Core:Qt5Core.dll
 0001:00039844       ??1QMutexLocker@@QAE@XZ    1003a844 f   Qt5Core:Qt5Core.dll
 0001:0003984a       ?unlock@QMutexLocker@@QAEXXZ 1003a84a f   Qt5Core:Qt5Core.dll
 0001:00039850       ?qstrncpy@@YAPADPADPBDI@Z  1003a850 f   Qt5Core:Qt5Core.dll
 0001:00039856       ?replace@QByteArray@@QAEAAV1@DD@Z 1003a856 f   Qt5Core:Qt5Core.dll
 0001:0003985c       ?fromLatin1@QString@@SA?AV1@PBDH@Z 1003a85c f   Qt5Core:Qt5Core.dll
 0001:00039862       ?toStdString@QString@@QBE?AV?$basic_string@DU?$char_traits@D@std@@V?$allocator@D@2@@std@@XZ 1003a862 f   Qt5Core:Qt5Core.dll
 0001:00039868       ??0QTemporaryFile@@QAE@XZ  1003a868 f   Qt5Core:Qt5Core.dll
 0001:0003986e       ??1QTemporaryFile@@UAE@XZ  1003a86e f   Qt5Core:Qt5Core.dll
 0001:00039874       ?open@QTemporaryFile@@QAE_NXZ 1003a874 f   Qt5Core:Qt5Core.dll
 0001:0003987a       ?fileName@QTemporaryFile@@UBE?AVQString@@XZ 1003a87a f   Qt5Core:Qt5Core.dll
 0001:00039880       ?setFileTemplate@QTemporaryFile@@QAEXABVQString@@@Z 1003a880 f   Qt5Core:Qt5Core.dll
 0001:00039886       ?childEvent@QObject@@MAEXPAVQChildEvent@@@Z 1003a886 f   Qt5Core:Qt5Core.dll
 0001:0003988c       ?connectNotify@QObject@@MAEXABVQMetaMethod@@@Z 1003a88c f   Qt5Core:Qt5Core.dll
 0001:00039892       ?customEvent@QObject@@MAEXPAVQEvent@@@Z 1003a892 f   Qt5Core:Qt5Core.dll
 0001:00039898       ?disconnectNotify@QObject@@MAEXABVQMetaMethod@@@Z 1003a898 f   Qt5Core:Qt5Core.dll
 0001:0003989e       ?event@QObject@@UAE_NPAVQEvent@@@Z 1003a89e f   Qt5Core:Qt5Core.dll
 0001:000398a4       ?eventFilter@QObject@@UAE_NPAV1@PAVQEvent@@@Z 1003a8a4 f   Qt5Core:Qt5Core.dll
 0001:000398aa       ?timerEvent@QObject@@MAEXPAVQTimerEvent@@@Z 1003a8aa f   Qt5Core:Qt5Core.dll
 0001:000398b0       ?qsrand@@YAXI@Z            1003a8b0 f   Qt5Core:Qt5Core.dll
 0001:000398b6       ?qrand@@YAHXZ              1003a8b6 f   Qt5Core:Qt5Core.dll
 0001:000398bc       ?tr@QMetaObject@@QBE?AVQString@@PBD0H@Z 1003a8bc f   Qt5Core:Qt5Core.dll
 0001:000398c2       ?connectSlotsByName@QMetaObject@@SAXPAVQObject@@@Z 1003a8c2 f   Qt5Core:Qt5Core.dll
 0001:000398c8       ??1Connection@QMetaObject@@QAE@XZ 1003a8c8 f   Qt5Core:Qt5Core.dll
 0001:000398ce       ?arg@QString@@QBE?AV1@_JHHVQChar@@@Z 1003a8ce f   Qt5Core:Qt5Core.dll
 0001:000398d4       ?fromUtf8@QString@@SA?AV1@PBDH@Z 1003a8d4 f   Qt5Core:Qt5Core.dll
 0001:000398da       ?objectName@QObject@@QBE?AVQString@@XZ 1003a8da f   Qt5Core:Qt5Core.dll
 0001:000398e0       ?setObjectName@QObject@@QAEXABVQString@@@Z 1003a8e0 f   Qt5Core:Qt5Core.dll
 0001:000398e6       ?connect@QObject@@SA?AVConnection@QMetaObject@@PBV1@PBD01W4ConnectionType@Qt@@@Z 1003a8e6 f   Qt5Core:Qt5Core.dll
 0001:000398ec       ?connect@QObject@@QBE?AVConnection@QMetaObject@@PBV1@PBD1W4ConnectionType@Qt@@@Z 1003a8ec f   Qt5Core:Qt5Core.dll
 0001:000398f2       ??1QVariant@@QAE@XZ        1003a8f2 f   Qt5Core:Qt5Core.dll
 0001:000398f8       ??0QVariant@@QAE@H@Z       1003a8f8 f   Qt5Core:Qt5Core.dll
 0001:000398fe       ??0QVariant@@QAE@_N@Z      1003a8fe f   Qt5Core:Qt5Core.dll
 0001:00039904       ??0QVariant@@QAE@N@Z       1003a904 f   Qt5Core:Qt5Core.dll
 0001:0003990a       ??0QVariant@@QAE@ABVQString@@@Z 1003a90a f   Qt5Core:Qt5Core.dll
 0001:00039910       ?toInt@QVariant@@QBEHPA_N@Z 1003a910 f   Qt5Core:Qt5Core.dll
 0001:00039916       ?toBool@QVariant@@QBE_NXZ  1003a916 f   Qt5Core:Qt5Core.dll
 0001:0003991c       ?toDouble@QVariant@@QBENPA_N@Z 1003a91c f   Qt5Core:Qt5Core.dll
 0001:00039922       ?toString@QVariant@@QBE?AVQString@@XZ 1003a922 f   Qt5Core:Qt5Core.dll
 0001:00039928       ??0QTime@@QAE@HHHH@Z       1003a928 f   Qt5Core:Qt5Core.dll
 0001:0003992e       ?secsTo@QTime@@QBEHABV1@@Z 1003a92e f   Qt5Core:Qt5Core.dll
 0001:00039934       ?currentTime@QTime@@SA?AV1@XZ 1003a934 f   Qt5Core:Qt5Core.dll
 0001:0003993a       ?translate@QCoreApplication@@SA?AVQString@@PBD00H@Z 1003a93a f   Qt5Core:Qt5Core.dll
 0001:00039940       ??0QByteArray@@QAE@ABV0@@Z 1003a940 f   Qt5Core:Qt5Core.dll
 0001:00039946       ?arg@QString@@QBE?AV1@NHDHVQChar@@@Z 1003a946 f   Qt5Core:Qt5Core.dll
 0001:0003994c       ??4QString@@QAEAAV0@PBD@Z  1003a94c f   Qt5Core:Qt5Core.dll
 0001:00039952       ?setParent@QObject@@QAEXPAV1@@Z 1003a952 f   Qt5Core:Qt5Core.dll
 0001:00039958       ?remove@QFile@@SA_NABVQString@@@Z 1003a958 f   Qt5Core:Qt5Core.dll
 0001:0003995e       ?qHash@@YAIABVQString@@I@Z 1003a95e f   Qt5Core:Qt5Core.dll
 0001:00039964       ?allocateNode@QHashData@@QAEPAXH@Z 1003a964 f   Qt5Core:Qt5Core.dll
 0001:0003996a       ?detach_helper@QHashData@@QAEPAU1@P6AXPAUNode@1@PAX@ZP6AX0@ZHH@Z 1003a96a f   Qt5Core:Qt5Core.dll
 0001:00039970       ?rehash@QHashData@@QAEXH@Z 1003a970 f   Qt5Core:Qt5Core.dll
 0001:00039976       ?free_helper@QHashData@@QAEXP6AXPAUNode@1@@Z@Z 1003a976 f   Qt5Core:Qt5Core.dll
 0001:0003997c       ?cast@QMetaObject@@QBEPAVQObject@@PAV2@@Z 1003a97c f   Qt5Core:Qt5Core.dll
 0001:00039982       ?toInt@QString@@QBEHPA_NH@Z 1003a982 f   Qt5Core:Qt5Core.dll
 0001:00039988       ?toDouble@QString@@QBENPA_N@Z 1003a988 f   Qt5Core:Qt5Core.dll
 0001:0003998e       ??0QObject@@QAE@PAV0@@Z    1003a98e f   Qt5Core:Qt5Core.dll
 0001:00039994       ??1QObject@@UAE@XZ         1003a994 f   Qt5Core:Qt5Core.dll
 0001:0003999a       ?metaObject@QObject@@UBEPBUQMetaObject@@XZ 1003a99a f   Qt5Core:Qt5Core.dll
 0001:000399a0       ?qt_metacall@QObject@@UAEHW4Call@QMetaObject@@HPAPAX@Z 1003a9a0 f   Qt5Core:Qt5Core.dll
 0001:000399a6       ?qt_metacast@QObject@@UAEPAXPBD@Z 1003a9a6 f   Qt5Core:Qt5Core.dll
 0001:000399ac       ??8QString@@QBE_NPBD@Z     1003a9ac f   Qt5Core:Qt5Core.dll
 0001:000399b2       ??0QByteArray@@QAE@XZ      1003a9b2 f   Qt5Core:Qt5Core.dll
 0001:000399b8       ??0QByteArray@@QAE@$$QAV0@@Z 1003a9b8 f   Qt5Core:Qt5Core.dll
 0001:000399be       ??0QString@@QAE@$$QAV0@@Z  1003a9be f   Qt5Core:Qt5Core.dll
 0001:000399c4       ??YQString@@QAEAAV0@PBD@Z  1003a9c4 f   Qt5Core:Qt5Core.dll
 0001:000399ca       ?data@QByteArray@@QAEPADXZ 1003a9ca f   Qt5Core:Qt5Core.dll
 0001:000399d0       ?append@QByteArray@@QAEAAV1@D@Z 1003a9d0 f   Qt5Core:Qt5Core.dll
 0001:000399d6       ?dynamicMetaObject@QObjectData@@QBEPAUQMetaObject@@XZ 1003a9d6 f   Qt5Core:Qt5Core.dll
 0001:000399dc       _GetStdHandle@4            1003a9dc f   kernel32:KERNEL32.dll
 0001:000399e2       _FillConsoleOutputCharacterW@20 1003a9e2 f   kernel32:KERNEL32.dll
 0001:000399e8       _FillConsoleOutputAttribute@20 1003a9e8 f   kernel32:KERNEL32.dll
 0001:000399ee       _GetConsoleScreenBufferInfo@8 1003a9ee f   kernel32:KERNEL32.dll
 0001:000399f4       _SetConsoleCursorPosition@8 1003a9f4 f   kernel32:KERNEL32.dll
 0001:000399fa       _SetConsoleTextAttribute@8 1003a9fa f   kernel32:KERNEL32.dll
 0001:00039a00       ?uncaught_exception@std@@YA_NXZ 1003aa00 f   msvcprt:MSVCP120.dll
 0001:00039a06       ?_Xbad_alloc@std@@YAXXZ    1003aa06 f   msvcprt:MSVCP120.dll
 0001:00039a0c       ?_Xlength_error@std@@YAXPBD@Z 1003aa0c f   msvcprt:MSVCP120.dll
 0001:00039a12       ?_Xout_of_range@std@@YAXPBD@Z 1003aa12 f   msvcprt:MSVCP120.dll
 0001:00039a18       ?_Syserror_map@std@@YAPBDH@Z 1003aa18 f   msvcprt:MSVCP120.dll
 0001:00039a1e       ?_Winerror_map@std@@YAPBDH@Z 1003aa1e f   msvcprt:MSVCP120.dll
 0001:00039a24       ?sputc@?$basic_streambuf@DU?$char_traits@D@std@@@std@@QAEHD@Z 1003aa24 f   msvcprt:MSVCP120.dll
 0001:00039a2a       ?sputn@?$basic_streambuf@DU?$char_traits@D@std@@@std@@QAE_JPBD_J@Z 1003aa2a f   msvcprt:MSVCP120.dll
 0001:00039a30       ?setstate@?$basic_ios@DU?$char_traits@D@std@@@std@@QAEXH_N@Z 1003aa30 f   msvcprt:MSVCP120.dll
 0001:00039a36       ?widen@?$basic_ios@DU?$char_traits@D@std@@@std@@QBEDD@Z 1003aa36 f   msvcprt:MSVCP120.dll
 0001:00039a3c       ?_Osfx@?$basic_ostream@DU?$char_traits@D@std@@@std@@QAEXXZ 1003aa3c f   msvcprt:MSVCP120.dll
 0001:00039a42       ??6?$basic_ostream@DU?$char_traits@D@std@@@std@@QAEAAV01@P6AAAV01@AAV01@@Z@Z 1003aa42 f   msvcprt:MSVCP120.dll
 0001:00039a48       ??6?$basic_ostream@DU?$char_traits@D@std@@@std@@QAEAAV01@H@Z 1003aa48 f   msvcprt:MSVCP120.dll
 0001:00039a4e       ??6?$basic_ostream@DU?$char_traits@D@std@@@std@@QAEAAV01@M@Z 1003aa4e f   msvcprt:MSVCP120.dll
 0001:00039a54       ?put@?$basic_ostream@DU?$char_traits@D@std@@@std@@QAEAAV12@D@Z 1003aa54 f   msvcprt:MSVCP120.dll
 0001:00039a5a       ?flush@?$basic_ostream@DU?$char_traits@D@std@@@std@@QAEAAV12@XZ 1003aa5a f   msvcprt:MSVCP120.dll
 0001:00039a60       __purecall                 1003aa60 f   MSVCRT:MSVCR120.dll
 0001:00039a66       ??2@YAPAXI@Z               1003aa66 f   MSVCRT:MSVCR120.dll
 0001:00039a6c       ??3@YAXPAX@Z               1003aa6c f   MSVCRT:MSVCR120.dll
 0001:00039a72       ___atonexitinit            1003aa72 f   MSVCRT:atonexit.obj
 0001:00039aae       __onexit                   1003aaae f   MSVCRT:atonexit.obj
 0001:00039b57       _atexit                    1003ab57 f   MSVCRT:atonexit.obj
 0001:00039b6c       _free                      1003ab6c f   MSVCRT:MSVCR120.dll
 0001:00039b72       _memmove                   1003ab72 f   MSVCRT:MSVCR120.dll
 0001:00039b78       __hypot                    1003ab78 f   MSVCRT:MSVCR120.dll
 0001:00039b7e       @__security_check_cookie@4 1003ab7e f   MSVCRT:secchk.obj
 0001:00039b8e       __CxxThrowException@8      1003ab8e f   MSVCRT:MSVCR120.dll
 0001:00039b94       ___CxxFrameHandler3        1003ab94 f   MSVCRT:MSVCR120.dll
 0001:00039ba0       __alldiv                   1003aba0 f   MSVCRT:lldiv.obj
 0001:00039c4a       _memcpy                    1003ac4a f   MSVCRT:MSVCR120.dll
 0001:00039c50       _memset                    1003ac50 f   MSVCRT:MSVCR120.dll
 0001:00039c56       ??0type_info@@AAE@ABV0@@Z  1003ac56 f   MSVCRT:ti_inst.obj
 0001:00039c61       ??4type_info@@AAEAAV0@ABV0@@Z 1003ac61 f   MSVCRT:ti_inst.obj
 0001:00039c66       ??_Etype_info@@UAEPAXI@Z   1003ac66 f i MSVCRT:ti_inst.obj
 0001:00039cb0       __allmul                   1003acb0 f   MSVCRT:llmul.obj
 0001:00039ce4       _fclose                    1003ace4 f   MSVCRT:MSVCR120.dll
 0001:00039cea       _fopen                     1003acea f   MSVCRT:MSVCR120.dll
 0001:00039cf0       _fprintf                   1003acf0 f   MSVCRT:MSVCR120.dll
 0001:00039cf6       _fscanf                    1003acf6 f   MSVCRT:MSVCR120.dll
 0001:00039cfc       _fseek                     1003acfc f   MSVCRT:MSVCR120.dll
 0001:00039d02       _ftell                     1003ad02 f   MSVCRT:MSVCR120.dll
 0001:00039d08       _printf                    1003ad08 f   MSVCRT:MSVCR120.dll
 0001:00039d0e       _putc                      1003ad0e f   MSVCRT:MSVCR120.dll
 0001:00039d14       _putchar                   1003ad14 f   MSVCRT:MSVCR120.dll
 0001:00039d1a       _puts                      1003ad1a f   MSVCRT:MSVCR120.dll
 0001:00039d20       _ungetc                    1003ad20 f   MSVCRT:MSVCR120.dll
 0001:00039d26       _strncmp                   1003ad26 f   MSVCRT:MSVCR120.dll
 0001:00039d2c       _strncpy                   1003ad2c f   MSVCRT:MSVCR120.dll
 0001:00039d32       __libm_sse2_sqrt_precise   1003ad32 f   MSVCRT:MSVCR120.dll
 0001:00039d38       _ceil                      1003ad38 f   MSVCRT:MSVCR120.dll
 0001:00039d3e       _floor                     1003ad3e f   MSVCRT:MSVCR120.dll
 0001:00039d44       __libm_sse2_log_precise    1003ad44 f   MSVCRT:MSVCR120.dll
 0001:00039d4a       ___iob_func                1003ad4a f   MSVCRT:MSVCR120.dll
 0001:00039d50       _fflush                    1003ad50 f   MSVCRT:MSVCR120.dll
 0001:00039d56       _strchr                    1003ad56 f   MSVCRT:MSVCR120.dll
 0001:00039d5c       __libm_sse2_exp_precise    1003ad5c f   MSVCRT:MSVCR120.dll
 0001:00039d62       ___raise_securityfailure   1003ad62 f   MSVCRT:gs_report.obj
 0001:00039d9f       ___report_gsfailure        1003ad9f f   MSVCRT:gs_report.obj
 0001:00039e9a       ___report_rangecheckfailure 1003ae9a f   MSVCRT:gs_report.obj
 0001:00039ea6       ___report_securityfailure  1003aea6 f   MSVCRT:gs_report.obj
 0001:00039f76       ___report_securityfailureEx 1003af76 f   MSVCRT:gs_report.obj
 0001:0003a08c       _feof                      1003b08c f   MSVCRT:MSVCR120.dll
 0001:0003a092       _fgetc                     1003b092 f   MSVCRT:MSVCR120.dll
 0001:0003a098       _fgetpos                   1003b098 f   MSVCRT:MSVCR120.dll
 0001:0003a09e       _fgets                     1003b09e f   MSVCRT:MSVCR120.dll
 0001:0003a0a4       _fputs                     1003b0a4 f   MSVCRT:MSVCR120.dll
 0001:0003a0aa       _fsetpos                   1003b0aa f   MSVCRT:MSVCR120.dll
 0001:0003a0b0       _getc                      1003b0b0 f   MSVCRT:MSVCR120.dll
 0001:0003a0b6       _getchar                   1003b0b6 f   MSVCRT:MSVCR120.dll
 0001:0003a0bc       _rewind                    1003b0bc f   MSVCRT:MSVCR120.dll
 0001:0003a0c2       _scanf                     1003b0c2 f   MSVCRT:MSVCR120.dll
 0001:0003a0c8       _sscanf                    1003b0c8 f   MSVCRT:MSVCR120.dll
 0001:0003a0ce       _sprintf                   1003b0ce f   MSVCRT:MSVCR120.dll
 0001:0003a0d4       _signal                    1003b0d4 f   MSVCRT:MSVCR120.dll
 0001:0003a0da       _exit                      1003b0da f   MSVCRT:MSVCR120.dll
 0001:0003a0e0       _abort                     1003b0e0 f   MSVCRT:MSVCR120.dll
 0001:0003a0e6       _calloc                    1003b0e6 f   MSVCRT:MSVCR120.dll
 0001:0003a0ec       _isalpha                   1003b0ec f   MSVCRT:MSVCR120.dll
 0001:0003a0f2       _islower                   1003b0f2 f   MSVCRT:MSVCR120.dll
 0001:0003a0f8       _isdigit                   1003b0f8 f   MSVCRT:MSVCR120.dll
 0001:0003a0fe       _toupper                   1003b0fe f   MSVCRT:MSVCR120.dll
 0001:0003a104       _strpbrk                   1003b104 f   MSVCRT:MSVCR120.dll
 0001:0003a10a       _strrchr                   1003b10a f   MSVCRT:MSVCR120.dll
 0001:0003a110       __libm_sse2_pow_precise    1003b110 f   MSVCRT:MSVCR120.dll
 0001:0003a116       ___isa_available_init      1003b116 f   MSVCRT:cpu_disp.obj
 0001:0003a290       _isupper                   1003b290 f   MSVCRT:MSVCR120.dll
 0001:0003a2a0       __ftoui3                   1003b2a0 f   MSVCRT:ftol3.obj
 0001:0003a2af       __ftoul3                   1003b2af f   MSVCRT:ftol3.obj
 0001:0003a2be       __ftol3                    1003b2be f   MSVCRT:ftol3.obj
 0001:0003a2cb       __ftol3_NaN                1003b2cb f   MSVCRT:ftol3.obj
 0001:0003a2e3       __ftol3_work               1003b2e3 f   MSVCRT:ftol3.obj
 0001:0003a369       __ftol3_common             1003b369 f   MSVCRT:ftol3.obj
 0001:0003a42b       __ftol3_arg_error          1003b42b f   MSVCRT:ftol3.obj
 0001:0003a43d       __ftol3_except             1003b43d f   MSVCRT:ftol3.obj
 0001:0003a481       __dtoui3                   1003b481 f   MSVCRT:ftol3.obj
 0001:0003a490       __dtoul3                   1003b490 f   MSVCRT:ftol3.obj
 0001:0003a49f       __dtol3                    1003b49f f   MSVCRT:ftol3.obj
 0001:0003a4ac       __dtol3_NaN                1003b4ac f   MSVCRT:ftol3.obj
 0001:0003a4c9       __dtol3_work               1003b4c9 f   MSVCRT:ftol3.obj
 0001:0003a5ae       __ultod3                   1003b5ae f   MSVCRT:ftol3.obj
 0001:0003a63f       __ltod3                    1003b63f f   MSVCRT:ftol3.obj
 0001:0003a6b9       _NtCurrentTeb              1003b6b9 f i MSVCRT:crtdll.obj
 0001:0003a6c0       __CRT_INIT@12              1003b6c0 f   MSVCRT:crtdll.obj
 0001:0003a8b7       __DllMainCRTStartup@12     1003b8b7 f   MSVCRT:crtdll.obj
 0001:0003aa0e       __lock                     1003ba0e f   MSVCRT:MSVCR120.dll
 0001:0003aa14       __unlock                   1003ba14 f   MSVCRT:MSVCR120.dll
 0001:0003aa1a       __calloc_crt               1003ba1a f   MSVCRT:MSVCR120.dll
 0001:0003aa20       ___dllonexit               1003ba20 f   MSVCRT:MSVCR120.dll
 0001:0003aa30       __SEH_prolog4              1003ba30 f   MSVCRT:sehprolg4.obj
 0001:0003aa75       __SEH_epilog4              1003ba75 f   MSVCRT:sehprolg4.obj
 0001:0003aa89       __except_handler4          1003ba89 f   MSVCRT:chandler4gs.obj
 0001:0003aaac       ??_M@YGXPAXIHP6EX0@Z@Z     1003baac f   MSVCRT:ehvecdtr.obj
 0001:0003ab34       ?__ArrayUnwind@@YGXPAXIHP6EX0@Z@Z 1003bb34 f   MSVCRT:ehvecdtr.obj
 0001:0003ab92       ??1type_info@@UAE@XZ       1003bb92 f   MSVCRT:MSVCR120.dll
 0001:0003ab98       __crt_debugger_hook        1003bb98 f   MSVCRT:MSVCR120.dll
 0001:0003ab9e       ___crtUnhandledException   1003bb9e f   MSVCRT:MSVCR120.dll
 0001:0003aba4       ___crtTerminateProcess     1003bba4 f   MSVCRT:MSVCR120.dll
 0001:0003abaa       __except1                  1003bbaa f   MSVCRT:MSVCR120.dll
 0001:0003abb0       ___CppXcptFilter           1003bbb0 f   MSVCRT:MSVCR120.dll
 0001:0003abb6       __amsg_exit                1003bbb6 f   MSVCRT:MSVCR120.dll
 0001:0003abc0       __FindPESection            1003bbc0 f   MSVCRT:pesect.obj
 0001:0003ac10       __IsNonwritableInCurrentImage 1003bc10 f   MSVCRT:pesect.obj
 0001:0003acd0       __ValidateImageBase        1003bcd0 f   MSVCRT:pesect.obj
 0001:0003ad01       ___security_init_cookie    1003bd01 f   MSVCRT:gs_support.obj
 0001:0003ad9d       _DllMain@12                1003bd9d f   MSVCRT:dllmain.obj
 0001:0003adc0       __malloc_crt               1003bdc0 f   MSVCRT:MSVCR120.dll
 0001:0003adc6       __RTC_Initialize           1003bdc6 f   MSVCRT:initsect.obj
 0001:0003ade6       __RTC_Terminate            1003bde6 f   MSVCRT:initsect.obj
 0001:0003ae06       __initterm                 1003be06 f   MSVCRT:MSVCR120.dll
 0001:0003ae0c       __initterm_e               1003be0c f   MSVCRT:MSVCR120.dll
 0001:0003ae12       ___clean_type_info_names   1003be12 f   MSVCRT:tncleanup.obj
 0001:0003ae1e       __except_handler4_common   1003be1e f   MSVCRT:MSVCR120.dll
 0001:0003ae24       ?terminate@@YAXXZ          1003be24 f   MSVCRT:MSVCR120.dll
 0001:0003ae2a       ___clean_type_info_names_internal 1003be2a f   MSVCRT:MSVCR120.dll
 0001:0003ae30       _EncodePointer@4           1003be30 f   kernel32:KERNEL32.dll
 0001:0003ae36       _DecodePointer@4           1003be36 f   kernel32:KERNEL32.dll
 0001:0003ae3c       _IsDebuggerPresent@0       1003be3c f   kernel32:KERNEL32.dll
 0001:0003ae42       _IsProcessorFeaturePresent@4 1003be42 f   kernel32:KERNEL32.dll
 0001:0003ae48       _QueryPerformanceCounter@4 1003be48 f   kernel32:KERNEL32.dll
 0001:0003ae4e       _GetCurrentProcessId@0     1003be4e f   kernel32:KERNEL32.dll
 0001:0003ae54       _GetCurrentThreadId@0      1003be54 f   kernel32:KERNEL32.dll
 0001:0003ae5a       _GetSystemTimeAsFileTime@4 1003be5a f   kernel32:KERNEL32.dll
 0001:0003ae60       _DisableThreadLibraryCalls@4 1003be60 f   kernel32:KERNEL32.dll
 0002:00000000       __imp__DisableThreadLibraryCalls@4 10042000     kernel32:KERNEL32.dll
 0002:00000004       __imp__GetSystemTimeAsFileTime@4 10042004     kernel32:KERNEL32.dll
 0002:00000008       __imp__GetCurrentThreadId@0 10042008     kernel32:KERNEL32.dll
 0002:0000000c       __imp__GetCurrentProcessId@0 1004200c     kernel32:KERNEL32.dll
 0002:00000010       __imp__QueryPerformanceCounter@4 10042010     kernel32:KERNEL32.dll
 0002:00000014       __imp__IsProcessorFeaturePresent@4 10042014     kernel32:KERNEL32.dll
 0002:00000018       __imp__IsDebuggerPresent@0 10042018     kernel32:KERNEL32.dll
 0002:0000001c       __imp__DecodePointer@4     1004201c     kernel32:KERNEL32.dll
 0002:00000020       __imp__EncodePointer@4     10042020     kernel32:KERNEL32.dll
 0002:00000024       __imp__FillConsoleOutputCharacterW@20 10042024     kernel32:KERNEL32.dll
 0002:00000028       __imp__FillConsoleOutputAttribute@20 10042028     kernel32:KERNEL32.dll
 0002:0000002c       __imp__GetConsoleScreenBufferInfo@8 1004202c     kernel32:KERNEL32.dll
 0002:00000030       __imp__SetConsoleCursorPosition@8 10042030     kernel32:KERNEL32.dll
 0002:00000034       __imp__SetConsoleTextAttribute@8 10042034     kernel32:KERNEL32.dll
 0002:00000038       __imp__GetStdHandle@4      10042038     kernel32:KERNEL32.dll
 0002:0000003c       \177KERNEL32_NULL_THUNK_DATA 1004203c     kernel32:KERNEL32.dll
 0002:00000040       __imp_?uncaught_exception@std@@YA_NXZ 10042040     msvcprt:MSVCP120.dll
 0002:00000044       __imp_?_Xlength_error@std@@YAXPBD@Z 10042044     msvcprt:MSVCP120.dll
 0002:00000048       __imp_?_Xout_of_range@std@@YAXPBD@Z 10042048     msvcprt:MSVCP120.dll
 0002:0000004c       __imp_?_Syserror_map@std@@YAPBDH@Z 1004204c     msvcprt:MSVCP120.dll
 0002:00000050       __imp_?_Winerror_map@std@@YAPBDH@Z 10042050     msvcprt:MSVCP120.dll
 0002:00000054       __imp_?sputc@?$basic_streambuf@DU?$char_traits@D@std@@@std@@QAEHD@Z 10042054     msvcprt:MSVCP120.dll
 0002:00000058       __imp_?sputn@?$basic_streambuf@DU?$char_traits@D@std@@@std@@QAE_JPBD_J@Z 10042058     msvcprt:MSVCP120.dll
 0002:0000005c       __imp_?setstate@?$basic_ios@DU?$char_traits@D@std@@@std@@QAEXH_N@Z 1004205c     msvcprt:MSVCP120.dll
 0002:00000060       __imp_?widen@?$basic_ios@DU?$char_traits@D@std@@@std@@QBEDD@Z 10042060     msvcprt:MSVCP120.dll
 0002:00000064       __imp_?_Osfx@?$basic_ostream@DU?$char_traits@D@std@@@std@@QAEXXZ 10042064     msvcprt:MSVCP120.dll
 0002:00000068       __imp_??6?$basic_ostream@DU?$char_traits@D@std@@@std@@QAEAAV01@P6AAAV01@AAV01@@Z@Z 10042068     msvcprt:MSVCP120.dll
 0002:0000006c       __imp_??6?$basic_ostream@DU?$char_traits@D@std@@@std@@QAEAAV01@H@Z 1004206c     msvcprt:MSVCP120.dll
 0002:00000070       __imp_??6?$basic_ostream@DU?$char_traits@D@std@@@std@@QAEAAV01@M@Z 10042070     msvcprt:MSVCP120.dll
 0002:00000074       __imp_?put@?$basic_ostream@DU?$char_traits@D@std@@@std@@QAEAAV12@D@Z 10042074     msvcprt:MSVCP120.dll
 0002:00000078       __imp_?flush@?$basic_ostream@DU?$char_traits@D@std@@@std@@QAEAAV12@XZ 10042078     msvcprt:MSVCP120.dll
 0002:0000007c       __imp_?cout@std@@3V?$basic_ostream@DU?$char_traits@D@std@@@1@A 1004207c     msvcprt:MSVCP120.dll
 0002:00000080       __imp_?_Xbad_alloc@std@@YAXXZ 10042080     msvcprt:MSVCP120.dll
 0002:00000084       \177MSVCP120_NULL_THUNK_DATA 10042084     msvcprt:MSVCP120.dll
 0002:00000088       __imp__islower             10042088     MSVCRT:MSVCR120.dll
 0002:0000008c       __imp__isalpha             1004208c     MSVCRT:MSVCR120.dll
 0002:00000090       __imp__calloc              10042090     MSVCRT:MSVCR120.dll
 0002:00000094       __imp__abort               10042094     MSVCRT:MSVCR120.dll
 0002:00000098       __imp__exit                10042098     MSVCRT:MSVCR120.dll
 0002:0000009c       __imp__signal              1004209c     MSVCRT:MSVCR120.dll
 0002:000000a0       __imp__sprintf             100420a0     MSVCRT:MSVCR120.dll
 0002:000000a4       __imp__sscanf              100420a4     MSVCRT:MSVCR120.dll
 0002:000000a8       __imp__scanf               100420a8     MSVCRT:MSVCR120.dll
 0002:000000ac       __imp__rewind              100420ac     MSVCRT:MSVCR120.dll
 0002:000000b0       __imp__getchar             100420b0     MSVCRT:MSVCR120.dll
 0002:000000b4       __imp__getc                100420b4     MSVCRT:MSVCR120.dll
 0002:000000b8       __imp__fsetpos             100420b8     MSVCRT:MSVCR120.dll
 0002:000000bc       __imp__fputs               100420bc     MSVCRT:MSVCR120.dll
 0002:000000c0       __imp__fgets               100420c0     MSVCRT:MSVCR120.dll
 0002:000000c4       __imp__fgetpos             100420c4     MSVCRT:MSVCR120.dll
 0002:000000c8       __imp__fgetc               100420c8     MSVCRT:MSVCR120.dll
 0002:000000cc       __imp__feof                100420cc     MSVCRT:MSVCR120.dll
 0002:000000d0       __imp___libm_sse2_exp_precise 100420d0     MSVCRT:MSVCR120.dll
 0002:000000d4       __imp__strchr              100420d4     MSVCRT:MSVCR120.dll
 0002:000000d8       __imp___malloc_crt         100420d8     MSVCRT:MSVCR120.dll
 0002:000000dc       __imp____iob_func          100420dc     MSVCRT:MSVCR120.dll
 0002:000000e0       __imp___libm_sse2_log_precise 100420e0     MSVCRT:MSVCR120.dll
 0002:000000e4       __imp__floor               100420e4     MSVCRT:MSVCR120.dll
 0002:000000e8       __imp__isdigit             100420e8     MSVCRT:MSVCR120.dll
 0002:000000ec       __imp___libm_sse2_sqrt_precise 100420ec     MSVCRT:MSVCR120.dll
 0002:000000f0       __imp__strncpy             100420f0     MSVCRT:MSVCR120.dll
 0002:000000f4       __imp__strncmp             100420f4     MSVCRT:MSVCR120.dll
 0002:000000f8       __imp__ungetc              100420f8     MSVCRT:MSVCR120.dll
 0002:000000fc       __imp__puts                100420fc     MSVCRT:MSVCR120.dll
 0002:00000100       __imp__putchar             10042100     MSVCRT:MSVCR120.dll
 0002:00000104       __imp__putc                10042104     MSVCRT:MSVCR120.dll
 0002:00000108       __imp__printf              10042108     MSVCRT:MSVCR120.dll
 0002:0000010c       __imp__ftell               1004210c     MSVCRT:MSVCR120.dll
 0002:00000110       __imp__fseek               10042110     MSVCRT:MSVCR120.dll
 0002:00000114       __imp__fscanf              10042114     MSVCRT:MSVCR120.dll
 0002:00000118       __imp__fprintf             10042118     MSVCRT:MSVCR120.dll
 0002:0000011c       __imp__fopen               1004211c     MSVCRT:MSVCR120.dll
 0002:00000120       __imp__fclose              10042120     MSVCRT:MSVCR120.dll
 0002:00000124       __imp__memset              10042124     MSVCRT:MSVCR120.dll
 0002:00000128       __imp__memcpy              10042128     MSVCRT:MSVCR120.dll
 0002:0000012c       __imp____CxxFrameHandler3  1004212c     MSVCRT:MSVCR120.dll
 0002:00000130       __imp___CxxThrowException@8 10042130     MSVCRT:MSVCR120.dll
 0002:00000134       __imp___hypot              10042134     MSVCRT:MSVCR120.dll
 0002:00000138       __imp__memmove             10042138     MSVCRT:MSVCR120.dll
 0002:0000013c       __imp__free                1004213c     MSVCRT:MSVCR120.dll
 0002:00000140       __imp_??3@YAXPAX@Z         10042140     MSVCRT:MSVCR120.dll
 0002:00000144       __imp_??2@YAPAXI@Z         10042144     MSVCRT:MSVCR120.dll
 0002:00000148       __imp___purecall           10042148     MSVCRT:MSVCR120.dll
 0002:0000014c       __imp__toupper             1004214c     MSVCRT:MSVCR120.dll
 0002:00000150       __imp__strpbrk             10042150     MSVCRT:MSVCR120.dll
 0002:00000154       __imp__strrchr             10042154     MSVCRT:MSVCR120.dll
 0002:00000158       __imp___libm_sse2_pow_precise 10042158     MSVCRT:MSVCR120.dll
 0002:0000015c       __imp__isupper             1004215c     MSVCRT:MSVCR120.dll
 0002:00000160       __imp___lock               10042160     MSVCRT:MSVCR120.dll
 0002:00000164       __imp___unlock             10042164     MSVCRT:MSVCR120.dll
 0002:00000168       __imp___calloc_crt         10042168     MSVCRT:MSVCR120.dll
 0002:0000016c       __imp____dllonexit         1004216c     MSVCRT:MSVCR120.dll
 0002:00000170       __imp___onexit             10042170     MSVCRT:MSVCR120.dll
 0002:00000174       __imp_??1type_info@@UAE@XZ 10042174     MSVCRT:MSVCR120.dll
 0002:00000178       __imp___crt_debugger_hook  10042178     MSVCRT:MSVCR120.dll
 0002:0000017c       __imp____crtUnhandledException 1004217c     MSVCRT:MSVCR120.dll
 0002:00000180       __imp____crtTerminateProcess 10042180     MSVCRT:MSVCR120.dll
 0002:00000184       __imp___except1            10042184     MSVCRT:MSVCR120.dll
 0002:00000188       __imp____CppXcptFilter     10042188     MSVCRT:MSVCR120.dll
 0002:0000018c       __imp__ceil                1004218c     MSVCRT:MSVCR120.dll
 0002:00000190       __imp___amsg_exit          10042190     MSVCRT:MSVCR120.dll
 0002:00000194       __imp___initterm           10042194     MSVCRT:MSVCR120.dll
 0002:00000198       __imp___initterm_e         10042198     MSVCRT:MSVCR120.dll
 0002:0000019c       __imp___except_handler4_common 1004219c     MSVCRT:MSVCR120.dll
 0002:000001a0       __imp_?terminate@@YAXXZ    100421a0     MSVCRT:MSVCR120.dll
 0002:000001a4       __imp____clean_type_info_names_internal 100421a4     MSVCRT:MSVCR120.dll
 0002:000001a8       __imp__fflush              100421a8     MSVCRT:MSVCR120.dll
 0002:000001ac       \177MSVCR120_NULL_THUNK_DATA 100421ac     MSVCRT:MSVCR120.dll
 0002:000001b0       __imp_?dynamicMetaObject@QObjectData@@QBEPAUQMetaObject@@XZ 100421b0     Qt5Core:Qt5Core.dll
 0002:000001b4       __imp_?append@QByteArray@@QAEAAV1@D@Z 100421b4     Qt5Core:Qt5Core.dll
 0002:000001b8       __imp_?data@QByteArray@@QAEPADXZ 100421b8     Qt5Core:Qt5Core.dll
 0002:000001bc       __imp_??YQString@@QAEAAV0@PBD@Z 100421bc     Qt5Core:Qt5Core.dll
 0002:000001c0       __imp_??0QString@@QAE@$$QAV0@@Z 100421c0     Qt5Core:Qt5Core.dll
 0002:000001c4       __imp_??0QByteArray@@QAE@$$QAV0@@Z 100421c4     Qt5Core:Qt5Core.dll
 0002:000001c8       __imp_??0QByteArray@@QAE@XZ 100421c8     Qt5Core:Qt5Core.dll
 0002:000001cc       __imp_??8QString@@QBE_NPBD@Z 100421cc     Qt5Core:Qt5Core.dll
 0002:000001d0       __imp_?qt_metacast@QObject@@UAEPAXPBD@Z 100421d0     Qt5Core:Qt5Core.dll
 0002:000001d4       __imp_?qt_metacall@QObject@@UAEHW4Call@QMetaObject@@HPAPAX@Z 100421d4     Qt5Core:Qt5Core.dll
 0002:000001d8       __imp_?metaObject@QObject@@UBEPBUQMetaObject@@XZ 100421d8     Qt5Core:Qt5Core.dll
 0002:000001dc       __imp_??1QObject@@UAE@XZ   100421dc     Qt5Core:Qt5Core.dll
 0002:000001e0       __imp_??0QObject@@QAE@PAV0@@Z 100421e0     Qt5Core:Qt5Core.dll
 0002:000001e4       __imp_?toDouble@QString@@QBENPA_N@Z 100421e4     Qt5Core:Qt5Core.dll
 0002:000001e8       __imp_?toInt@QString@@QBEHPA_NH@Z 100421e8     Qt5Core:Qt5Core.dll
 0002:000001ec       __imp_?cast@QMetaObject@@QBEPAVQObject@@PAV2@@Z 100421ec     Qt5Core:Qt5Core.dll
 0002:000001f0       __imp_?shared_null@QHashData@@2U1@B 100421f0     Qt5Core:Qt5Core.dll
 0002:000001f4       __imp_?free_helper@QHashData@@QAEXP6AXPAUNode@1@@Z@Z 100421f4     Qt5Core:Qt5Core.dll
 0002:000001f8       __imp_?rehash@QHashData@@QAEXH@Z 100421f8     Qt5Core:Qt5Core.dll
 0002:000001fc       __imp_?detach_helper@QHashData@@QAEPAU1@P6AXPAUNode@1@PAX@ZP6AX0@ZHH@Z 100421fc     Qt5Core:Qt5Core.dll
 0002:00000200       __imp_?allocateNode@QHashData@@QAEPAXH@Z 10042200     Qt5Core:Qt5Core.dll
 0002:00000204       __imp_?qHash@@YAIABVQString@@I@Z 10042204     Qt5Core:Qt5Core.dll
 0002:00000208       __imp_?remove@QFile@@SA_NABVQString@@@Z 10042208     Qt5Core:Qt5Core.dll
 0002:0000020c       __imp_?setParent@QObject@@QAEXPAV1@@Z 1004220c     Qt5Core:Qt5Core.dll
 0002:00000210       __imp_??4QString@@QAEAAV0@PBD@Z 10042210     Qt5Core:Qt5Core.dll
 0002:00000214       __imp_?arg@QString@@QBE?AV1@NHDHVQChar@@@Z 10042214     Qt5Core:Qt5Core.dll
 0002:00000218       __imp_??0QByteArray@@QAE@ABV0@@Z 10042218     Qt5Core:Qt5Core.dll
 0002:0000021c       __imp_?translate@QCoreApplication@@SA?AVQString@@PBD00H@Z 1004221c     Qt5Core:Qt5Core.dll
 0002:00000220       __imp_?currentTime@QTime@@SA?AV1@XZ 10042220     Qt5Core:Qt5Core.dll
 0002:00000224       __imp_?secsTo@QTime@@QBEHABV1@@Z 10042224     Qt5Core:Qt5Core.dll
 0002:00000228       __imp_??0QTime@@QAE@HHHH@Z 10042228     Qt5Core:Qt5Core.dll
 0002:0000022c       __imp_?toString@QVariant@@QBE?AVQString@@XZ 1004222c     Qt5Core:Qt5Core.dll
 0002:00000230       __imp_?toDouble@QVariant@@QBENPA_N@Z 10042230     Qt5Core:Qt5Core.dll
 0002:00000234       __imp_?toBool@QVariant@@QBE_NXZ 10042234     Qt5Core:Qt5Core.dll
 0002:00000238       __imp_?toInt@QVariant@@QBEHPA_N@Z 10042238     Qt5Core:Qt5Core.dll
 0002:0000023c       __imp_??0QVariant@@QAE@ABVQString@@@Z 1004223c     Qt5Core:Qt5Core.dll
 0002:00000240       __imp_??0QVariant@@QAE@N@Z 10042240     Qt5Core:Qt5Core.dll
 0002:00000244       __imp_??0QVariant@@QAE@_N@Z 10042244     Qt5Core:Qt5Core.dll
 0002:00000248       __imp_??0QVariant@@QAE@H@Z 10042248     Qt5Core:Qt5Core.dll
 0002:0000024c       __imp_??1QVariant@@QAE@XZ  1004224c     Qt5Core:Qt5Core.dll
 0002:00000250       __imp_?connect@QObject@@QBE?AVConnection@QMetaObject@@PBV1@PBD1W4ConnectionType@Qt@@@Z 10042250     Qt5Core:Qt5Core.dll
 0002:00000254       __imp_?connect@QObject@@SA?AVConnection@QMetaObject@@PBV1@PBD01W4ConnectionType@Qt@@@Z 10042254     Qt5Core:Qt5Core.dll
 0002:00000258       __imp_?setObjectName@QObject@@QAEXABVQString@@@Z 10042258     Qt5Core:Qt5Core.dll
 0002:0000025c       __imp_?objectName@QObject@@QBE?AVQString@@XZ 1004225c     Qt5Core:Qt5Core.dll
 0002:00000260       __imp_?fromUtf8@QString@@SA?AV1@PBDH@Z 10042260     Qt5Core:Qt5Core.dll
 0002:00000264       __imp_?arg@QString@@QBE?AV1@_JHHVQChar@@@Z 10042264     Qt5Core:Qt5Core.dll
 0002:00000268       __imp_??1Connection@QMetaObject@@QAE@XZ 10042268     Qt5Core:Qt5Core.dll
 0002:0000026c       __imp_?connectSlotsByName@QMetaObject@@SAXPAVQObject@@@Z 1004226c     Qt5Core:Qt5Core.dll
 0002:00000270       __imp_?tr@QMetaObject@@QBE?AVQString@@PBD0H@Z 10042270     Qt5Core:Qt5Core.dll
 0002:00000274       __imp_?qrand@@YAHXZ        10042274     Qt5Core:Qt5Core.dll
 0002:00000278       __imp_?qsrand@@YAXI@Z      10042278     Qt5Core:Qt5Core.dll
 0002:0000027c       __imp_?timerEvent@QObject@@MAEXPAVQTimerEvent@@@Z 1004227c     Qt5Core:Qt5Core.dll
 0002:00000280       __imp_?eventFilter@QObject@@UAE_NPAV1@PAVQEvent@@@Z 10042280     Qt5Core:Qt5Core.dll
 0002:00000284       __imp_?event@QObject@@UAE_NPAVQEvent@@@Z 10042284     Qt5Core:Qt5Core.dll
 0002:00000288       __imp_?disconnectNotify@QObject@@MAEXABVQMetaMethod@@@Z 10042288     Qt5Core:Qt5Core.dll
 0002:0000028c       __imp_?customEvent@QObject@@MAEXPAVQEvent@@@Z 1004228c     Qt5Core:Qt5Core.dll
 0002:00000290       __imp_?connectNotify@QObject@@MAEXABVQMetaMethod@@@Z 10042290     Qt5Core:Qt5Core.dll
 0002:00000294       __imp_?childEvent@QObject@@MAEXPAVQChildEvent@@@Z 10042294     Qt5Core:Qt5Core.dll
 0002:00000298       __imp_?setFileTemplate@QTemporaryFile@@QAEXABVQString@@@Z 10042298     Qt5Core:Qt5Core.dll
 0002:0000029c       __imp_?fileName@QTemporaryFile@@UBE?AVQString@@XZ 1004229c     Qt5Core:Qt5Core.dll
 0002:000002a0       __imp_?open@QTemporaryFile@@QAE_NXZ 100422a0     Qt5Core:Qt5Core.dll
 0002:000002a4       __imp_??1QTemporaryFile@@UAE@XZ 100422a4     Qt5Core:Qt5Core.dll
 0002:000002a8       __imp_??0QTemporaryFile@@QAE@XZ 100422a8     Qt5Core:Qt5Core.dll
 0002:000002ac       __imp_?toStdString@QString@@QBE?AV?$basic_string@DU?$char_traits@D@std@@V?$allocator@D@2@@std@@XZ 100422ac     Qt5Core:Qt5Core.dll
 0002:000002b0       __imp_?fromLatin1@QString@@SA?AV1@PBDH@Z 100422b0     Qt5Core:Qt5Core.dll
 0002:000002b4       __imp_?replace@QByteArray@@QAEAAV1@DD@Z 100422b4     Qt5Core:Qt5Core.dll
 0002:000002b8       __imp_?qstrncpy@@YAPADPADPBDI@Z 100422b8     Qt5Core:Qt5Core.dll
 0002:000002bc       __imp_?unlock@QMutexLocker@@QAEXXZ 100422bc     Qt5Core:Qt5Core.dll
 0002:000002c0       __imp_??1QMutexLocker@@QAE@XZ 100422c0     Qt5Core:Qt5Core.dll
 0002:000002c4       __imp_??0QMutexLocker@@QAE@PAVQBasicMutex@@@Z 100422c4     Qt5Core:Qt5Core.dll
 0002:000002c8       __imp_??1QMutex@@QAE@XZ    100422c8     Qt5Core:Qt5Core.dll
 0002:000002cc       __imp_??0QMutex@@QAE@W4RecursionMode@0@@Z 100422cc     Qt5Core:Qt5Core.dll
 0002:000002d0       __imp_?shared_null@QMapDataBase@@2U1@B 100422d0     Qt5Core:Qt5Core.dll
 0002:000002d4       __imp_?shared_null@QListData@@2UData@1@B 100422d4     Qt5Core:Qt5Core.dll
 0002:000002d8       __imp_?shared_null@QArrayData@@2QBU1@B 100422d8     Qt5Core:Qt5Core.dll
 0002:000002dc       __imp_?fromAscii_helper@QString@@CAPAU?$QTypedArrayData@G@@PBDH@Z 100422dc     Qt5Core:Qt5Core.dll
 0002:000002e0       __imp_??9QString@@QBE_NPBD@Z 100422e0     Qt5Core:Qt5Core.dll
 0002:000002e4       __imp_?append@QString@@QAEAAV1@PBD@Z 100422e4     Qt5Core:Qt5Core.dll
 0002:000002e8       __imp_??M@YA_NABVQString@@0@Z 100422e8     Qt5Core:Qt5Core.dll
 0002:000002ec       __imp_??8@YA_NABVQString@@0@Z 100422ec     Qt5Core:Qt5Core.dll
 0002:000002f0       __imp_?toLatin1@QString@@QBE?AVQByteArray@@XZ 100422f0     Qt5Core:Qt5Core.dll
 0002:000002f4       __imp_?append@QString@@QAEAAV1@ABV1@@Z 100422f4     Qt5Core:Qt5Core.dll
 0002:000002f8       __imp_?startsWith@QString@@QBE_NABV1@W4CaseSensitivity@Qt@@@Z 100422f8     Qt5Core:Qt5Core.dll
 0002:000002fc       __imp_?arg@QString@@QBE?AV1@ABV1@HVQChar@@@Z 100422fc     Qt5Core:Qt5Core.dll
 0002:00000300       __imp_?arg@QString@@QBE?AV1@HHHVQChar@@@Z 10042300     Qt5Core:Qt5Core.dll
 0002:00000304       __imp_??4QString@@QAEAAV0@$$QAV0@@Z 10042304     Qt5Core:Qt5Core.dll
 0002:00000308       __imp_??4QString@@QAEAAV0@ABV0@@Z 10042308     Qt5Core:Qt5Core.dll
 0002:0000030c       __imp_??1QString@@QAE@XZ   1004230c     Qt5Core:Qt5Core.dll
 0002:00000310       __imp_??0QString@@QAE@ABV0@@Z 10042310     Qt5Core:Qt5Core.dll
 0002:00000314       __imp_??0QString@@QAE@XZ   10042314     Qt5Core:Qt5Core.dll
 0002:00000318       __imp_??0QChar@@QAE@UQLatin1Char@@@Z 10042318     Qt5Core:Qt5Core.dll
 0002:0000031c       __imp_?freeData@QMapDataBase@@SAXPAU1@@Z 1004231c     Qt5Core:Qt5Core.dll
 0002:00000320       __imp_?createData@QMapDataBase@@SAPAU1@XZ 10042320     Qt5Core:Qt5Core.dll
 0002:00000324       __imp_?freeTree@QMapDataBase@@QAEXPAUQMapNodeBase@@H@Z 10042324     Qt5Core:Qt5Core.dll
 0002:00000328       __imp_?createNode@QMapDataBase@@QAEPAUQMapNodeBase@@HHPAU2@_N@Z 10042328     Qt5Core:Qt5Core.dll
 0002:0000032c       __imp_?recalcMostLeftNode@QMapDataBase@@QAEXXZ 1004232c     Qt5Core:Qt5Core.dll
 0002:00000330       __imp_?freeNodeAndRebalance@QMapDataBase@@QAEXPAUQMapNodeBase@@@Z 10042330     Qt5Core:Qt5Core.dll
 0002:00000334       __imp_?nextNode@QMapNodeBase@@QBEPBU1@XZ 10042334     Qt5Core:Qt5Core.dll
 0002:00000338       __imp_?constData@QByteArray@@QBEPBDXZ 10042338     Qt5Core:Qt5Core.dll
 0002:0000033c       __imp_??1QByteArray@@QAE@XZ 1004233c     Qt5Core:Qt5Core.dll
 0002:00000340       __imp_?append@QListData@@QAEPAPAXXZ 10042340     Qt5Core:Qt5Core.dll
 0002:00000344       __imp_?dispose@QListData@@SAXPAUData@1@@Z 10042344     Qt5Core:Qt5Core.dll
 0002:00000348       __imp_?realloc@QListData@@QAEXH@Z 10042348     Qt5Core:Qt5Core.dll
 0002:0000034c       __imp_?detach_grow@QListData@@QAEPAUData@1@PAHH@Z 1004234c     Qt5Core:Qt5Core.dll
 0002:00000350       __imp_?detach@QListData@@QAEPAUData@1@H@Z 10042350     Qt5Core:Qt5Core.dll
 0002:00000354       __imp_?deallocate@QArrayData@@SAXPAU1@II@Z 10042354     Qt5Core:Qt5Core.dll
 0002:00000358       __imp_?allocate@QArrayData@@SAPAU1@IIIV?$QFlags@W4AllocationOption@QArrayData@@@@@Z 10042358     Qt5Core:Qt5Core.dll
 0002:0000035c       __imp_?data@QArrayData@@QAEPAXXZ 1004235c     Qt5Core:Qt5Core.dll
 0002:00000360       __imp_?qBadAlloc@@YAXXZ    10042360     Qt5Core:Qt5Core.dll
 0002:00000364       \177Qt5Core_NULL_THUNK_DATA 10042364     Qt5Core:Qt5Core.dll
 0002:00000368       __imp_?staticMetaObject@QWidget@@2UQMetaObject@@B 10042368     Qt5Widgets:Qt5Widgets.dll
 0002:0000036c       __imp_?widget@QLayoutItem@@UAEPAVQWidget@@XZ 1004236c     Qt5Widgets:Qt5Widgets.dll
 0002:00000370       __imp_?wheelEvent@QWidget@@MAEXPAVQWheelEvent@@@Z 10042370     Qt5Widgets:Qt5Widgets.dll
 0002:00000374       __imp_?wheelEvent@QComboBox@@MAEXPAVQWheelEvent@@@Z 10042374     Qt5Widgets:Qt5Widgets.dll
 0002:00000378       __imp_?wheelEvent@QAbstractSpinBox@@MAEXPAVQWheelEvent@@@Z 10042378     Qt5Widgets:Qt5Widgets.dll
 0002:0000037c       __imp_?valueFromText@QSpinBox@@MBEHABVQString@@@Z 1004237c     Qt5Widgets:Qt5Widgets.dll
 0002:00000380       __imp_?valueFromText@QDoubleSpinBox@@UBENABVQString@@@Z 10042380     Qt5Widgets:Qt5Widgets.dll
 0002:00000384       __imp_?validate@QSpinBox@@MBE?AW4State@QValidator@@AAVQString@@AAH@Z 10042384     Qt5Widgets:Qt5Widgets.dll
 0002:00000388       __imp_??0QSizePolicy@@QAE@W4Policy@0@0W4ControlType@0@@Z 10042388     Qt5Widgets:Qt5Widgets.dll
 0002:0000038c       __imp_?setHorizontalStretch@QSizePolicy@@QAEXH@Z 1004238c     Qt5Widgets:Qt5Widgets.dll
 0002:00000390       __imp_?setVerticalStretch@QSizePolicy@@QAEXH@Z 10042390     Qt5Widgets:Qt5Widgets.dll
 0002:00000394       __imp_??0QWidget@@QAE@PAV0@V?$QFlags@W4WindowType@Qt@@@@@Z 10042394     Qt5Widgets:Qt5Widgets.dll
 0002:00000398       __imp_??1QWidget@@UAE@XZ   10042398     Qt5Widgets:Qt5Widgets.dll
 0002:0000039c       __imp_?setEnabled@QWidget@@QAEX_N@Z 1004239c     Qt5Widgets:Qt5Widgets.dll
 0002:000003a0       __imp_?setMinimumSize@QWidget@@QAEXHH@Z 100423a0     Qt5Widgets:Qt5Widgets.dll
 0002:000003a4       __imp_?resize@QWidget@@QAEXABVQSize@@@Z 100423a4     Qt5Widgets:Qt5Widgets.dll
 0002:000003a8       __imp_?sizePolicy@QWidget@@QBE?AVQSizePolicy@@XZ 100423a8     Qt5Widgets:Qt5Widgets.dll
 0002:000003ac       __imp_?setSizePolicy@QWidget@@QAEXVQSizePolicy@@@Z 100423ac     Qt5Widgets:Qt5Widgets.dll
 0002:000003b0       __imp_?setText@QAbstractButton@@QAEXABVQString@@@Z 100423b0     Qt5Widgets:Qt5Widgets.dll
 0002:000003b4       __imp_?isChecked@QAbstractButton@@QBE_NXZ 100423b4     Qt5Widgets:Qt5Widgets.dll
 0002:000003b8       __imp_?setChecked@QAbstractButton@@QAEX_N@Z 100423b8     Qt5Widgets:Qt5Widgets.dll
 0002:000003bc       __imp_??0QCheckBox@@QAE@PAVQWidget@@@Z 100423bc     Qt5Widgets:Qt5Widgets.dll
 0002:000003c0       __imp_??1QCheckBox@@UAE@XZ 100423c0     Qt5Widgets:Qt5Widgets.dll
 0002:000003c4       __imp_??0QTabWidget@@QAE@PAVQWidget@@@Z 100423c4     Qt5Widgets:Qt5Widgets.dll
 0002:000003c8       __imp_??1QTabWidget@@UAE@XZ 100423c8     Qt5Widgets:Qt5Widgets.dll
 0002:000003cc       __imp_?addTab@QTabWidget@@QAEHPAVQWidget@@ABVQString@@@Z 100423cc     Qt5Widgets:Qt5Widgets.dll
 0002:000003d0       __imp_?setTabText@QTabWidget@@QAEXHABVQString@@@Z 100423d0     Qt5Widgets:Qt5Widgets.dll
 0002:000003d4       __imp_?indexOf@QTabWidget@@QBEHPAVQWidget@@@Z 100423d4     Qt5Widgets:Qt5Widgets.dll
 0002:000003d8       __imp_?setCurrentIndex@QTabWidget@@QAEXH@Z 100423d8     Qt5Widgets:Qt5Widgets.dll
 0002:000003dc       __imp_??0QComboBox@@QAE@PAVQWidget@@@Z 100423dc     Qt5Widgets:Qt5Widgets.dll
 0002:000003e0       __imp_??1QComboBox@@UAE@XZ 100423e0     Qt5Widgets:Qt5Widgets.dll
 0002:000003e4       __imp_?count@QComboBox@@QBEHXZ 100423e4     Qt5Widgets:Qt5Widgets.dll
 0002:000003e8       __imp_?findData@QComboBox@@QBEHABVQVariant@@HV?$QFlags@W4MatchFlag@Qt@@@@@Z 100423e8     Qt5Widgets:Qt5Widgets.dll
 0002:000003ec       __imp_?currentText@QComboBox@@QBE?AVQString@@XZ 100423ec     Qt5Widgets:Qt5Widgets.dll
 0002:000003f0       __imp_?itemText@QComboBox@@QBE?AVQString@@H@Z 100423f0     Qt5Widgets:Qt5Widgets.dll
 0002:000003f4       __imp_?insertItems@QComboBox@@QAEXHABVQStringList@@@Z 100423f4     Qt5Widgets:Qt5Widgets.dll
 0002:000003f8       __imp_?setCurrentIndex@QComboBox@@QAEXH@Z 100423f8     Qt5Widgets:Qt5Widgets.dll
 0002:000003fc       __imp_??0QSpinBox@@QAE@PAVQWidget@@@Z 100423fc     Qt5Widgets:Qt5Widgets.dll
 0002:00000400       __imp_??1QSpinBox@@UAE@XZ  10042400     Qt5Widgets:Qt5Widgets.dll
 0002:00000404       __imp_?value@QSpinBox@@QBEHXZ 10042404     Qt5Widgets:Qt5Widgets.dll
 0002:00000408       __imp_?setSingleStep@QSpinBox@@QAEXH@Z 10042408     Qt5Widgets:Qt5Widgets.dll
 0002:0000040c       __imp_?setMinimum@QSpinBox@@QAEXH@Z 1004240c     Qt5Widgets:Qt5Widgets.dll
 0002:00000410       __imp_?setMaximum@QSpinBox@@QAEXH@Z 10042410     Qt5Widgets:Qt5Widgets.dll
 0002:00000414       __imp_?setValue@QSpinBox@@QAEXH@Z 10042414     Qt5Widgets:Qt5Widgets.dll
 0002:00000418       __imp_??0QDoubleSpinBox@@QAE@PAVQWidget@@@Z 10042418     Qt5Widgets:Qt5Widgets.dll
 0002:0000041c       __imp_??1QDoubleSpinBox@@UAE@XZ 1004241c     Qt5Widgets:Qt5Widgets.dll
 0002:00000420       __imp_?value@QDoubleSpinBox@@QBENXZ 10042420     Qt5Widgets:Qt5Widgets.dll
 0002:00000424       __imp_?setSingleStep@QDoubleSpinBox@@QAEXN@Z 10042424     Qt5Widgets:Qt5Widgets.dll
 0002:00000428       __imp_?setMinimum@QDoubleSpinBox@@QAEXN@Z 10042428     Qt5Widgets:Qt5Widgets.dll
 0002:0000042c       __imp_?setMaximum@QDoubleSpinBox@@QAEXN@Z 1004242c     Qt5Widgets:Qt5Widgets.dll
 0002:00000430       __imp_?setDecimals@QDoubleSpinBox@@QAEXH@Z 10042430     Qt5Widgets:Qt5Widgets.dll
 0002:00000434       __imp_?setValue@QDoubleSpinBox@@QAEXN@Z 10042434     Qt5Widgets:Qt5Widgets.dll
 0002:00000438       __imp_??0QSpacerItem@@QAE@HHW4Policy@QSizePolicy@@0@Z 10042438     Qt5Widgets:Qt5Widgets.dll
 0002:0000043c       __imp_??1QSpacerItem@@UAE@XZ 1004243c     Qt5Widgets:Qt5Widgets.dll
 0002:00000440       __imp_?setContentsMargins@QLayout@@QAEXHHHH@Z 10042440     Qt5Widgets:Qt5Widgets.dll
 0002:00000444       __imp_?setSizeConstraint@QLayout@@QAEXW4SizeConstraint@1@@Z 10042444     Qt5Widgets:Qt5Widgets.dll
 0002:00000448       __imp_?addWidget@QBoxLayout@@QAEXPAVQWidget@@HV?$QFlags@W4AlignmentFlag@Qt@@@@@Z 10042448     Qt5Widgets:Qt5Widgets.dll
 0002:0000044c       __imp_?addLayout@QBoxLayout@@QAEXPAVQLayout@@H@Z 1004244c     Qt5Widgets:Qt5Widgets.dll
 0002:00000450       __imp_?setSpacing@QBoxLayout@@QAEXH@Z 10042450     Qt5Widgets:Qt5Widgets.dll
 0002:00000454       __imp_??0QHBoxLayout@@QAE@XZ 10042454     Qt5Widgets:Qt5Widgets.dll
 0002:00000458       __imp_??1QHBoxLayout@@UAE@XZ 10042458     Qt5Widgets:Qt5Widgets.dll
 0002:0000045c       __imp_??0QVBoxLayout@@QAE@PAVQWidget@@@Z 1004245c     Qt5Widgets:Qt5Widgets.dll
 0002:00000460       __imp_??1QVBoxLayout@@UAE@XZ 10042460     Qt5Widgets:Qt5Widgets.dll
 0002:00000464       __imp_??0QGridLayout@@QAE@XZ 10042464     Qt5Widgets:Qt5Widgets.dll
 0002:00000468       __imp_??1QGridLayout@@UAE@XZ 10042468     Qt5Widgets:Qt5Widgets.dll
 0002:0000046c       __imp_?addWidget@QGridLayout@@QAEXPAVQWidget@@HHHHV?$QFlags@W4AlignmentFlag@Qt@@@@@Z 1004246c     Qt5Widgets:Qt5Widgets.dll
 0002:00000470       __imp_??0QLabel@@QAE@PAVQWidget@@V?$QFlags@W4WindowType@Qt@@@@@Z 10042470     Qt5Widgets:Qt5Widgets.dll
 0002:00000474       __imp_??1QLabel@@UAE@XZ    10042474     Qt5Widgets:Qt5Widgets.dll
 0002:00000478       __imp_?setWordWrap@QLabel@@QAEX_N@Z 10042478     Qt5Widgets:Qt5Widgets.dll
 0002:0000047c       __imp_?setText@QLabel@@QAEXABVQString@@@Z 1004247c     Qt5Widgets:Qt5Widgets.dll
 0002:00000480       __imp_?actionEvent@QWidget@@MAEXPAVQActionEvent@@@Z 10042480     Qt5Widgets:Qt5Widgets.dll
 0002:00000484       __imp_?addItem@QBoxLayout@@UAEXPAVQLayoutItem@@@Z 10042484     Qt5Widgets:Qt5Widgets.dll
 0002:00000488       __imp_?addItem@QGridLayout@@MAEXPAVQLayoutItem@@@Z 10042488     Qt5Widgets:Qt5Widgets.dll
 0002:0000048c       __imp_?changeEvent@QAbstractButton@@MAEXPAVQEvent@@@Z 1004248c     Qt5Widgets:Qt5Widgets.dll
 0002:00000490       __imp_?changeEvent@QAbstractSpinBox@@MAEXPAVQEvent@@@Z 10042490     Qt5Widgets:Qt5Widgets.dll
 0002:00000494       __imp_?changeEvent@QComboBox@@MAEXPAVQEvent@@@Z 10042494     Qt5Widgets:Qt5Widgets.dll
 0002:00000498       __imp_?changeEvent@QLabel@@MAEXPAVQEvent@@@Z 10042498     Qt5Widgets:Qt5Widgets.dll
 0002:0000049c       __imp_?changeEvent@QTabWidget@@MAEXPAVQEvent@@@Z 1004249c     Qt5Widgets:Qt5Widgets.dll
 0002:000004a0       __imp_?changeEvent@QWidget@@MAEXPAVQEvent@@@Z 100424a0     Qt5Widgets:Qt5Widgets.dll
 0002:000004a4       __imp_?checkStateSet@QCheckBox@@MAEXXZ 100424a4     Qt5Widgets:Qt5Widgets.dll
 0002:000004a8       __imp_?childEvent@QLayout@@MAEXPAVQChildEvent@@@Z 100424a8     Qt5Widgets:Qt5Widgets.dll
 0002:000004ac       __imp_?clear@QAbstractSpinBox@@UAEXXZ 100424ac     Qt5Widgets:Qt5Widgets.dll
 0002:000004b0       __imp_?closeEvent@QAbstractSpinBox@@MAEXPAVQCloseEvent@@@Z 100424b0     Qt5Widgets:Qt5Widgets.dll
 0002:000004b4       __imp_?closeEvent@QWidget@@MAEXPAVQCloseEvent@@@Z 100424b4     Qt5Widgets:Qt5Widgets.dll
 0002:000004b8       __imp_?contextMenuEvent@QAbstractSpinBox@@MAEXPAVQContextMenuEvent@@@Z 100424b8     Qt5Widgets:Qt5Widgets.dll
 0002:000004bc       __imp_?contextMenuEvent@QComboBox@@MAEXPAVQContextMenuEvent@@@Z 100424bc     Qt5Widgets:Qt5Widgets.dll
 0002:000004c0       __imp_?contextMenuEvent@QLabel@@MAEXPAVQContextMenuEvent@@@Z 100424c0     Qt5Widgets:Qt5Widgets.dll
 0002:000004c4       __imp_?contextMenuEvent@QWidget@@MAEXPAVQContextMenuEvent@@@Z 100424c4     Qt5Widgets:Qt5Widgets.dll
 0002:000004c8       __imp_?controlTypes@QLayout@@UBE?AV?$QFlags@W4ControlType@QSizePolicy@@@@XZ 100424c8     Qt5Widgets:Qt5Widgets.dll
 0002:000004cc       __imp_?controlTypes@QLayoutItem@@UBE?AV?$QFlags@W4ControlType@QSizePolicy@@@@XZ 100424cc     Qt5Widgets:Qt5Widgets.dll
 0002:000004d0       __imp_?count@QBoxLayout@@UBEHXZ 100424d0     Qt5Widgets:Qt5Widgets.dll
 0002:000004d4       __imp_?count@QGridLayout@@UBEHXZ 100424d4     Qt5Widgets:Qt5Widgets.dll
 0002:000004d8       __imp_?devType@QWidget@@UBEHXZ 100424d8     Qt5Widgets:Qt5Widgets.dll
 0002:000004dc       __imp_?dragEnterEvent@QWidget@@MAEXPAVQDragEnterEvent@@@Z 100424dc     Qt5Widgets:Qt5Widgets.dll
 0002:000004e0       __imp_?dragLeaveEvent@QWidget@@MAEXPAVQDragLeaveEvent@@@Z 100424e0     Qt5Widgets:Qt5Widgets.dll
 0002:000004e4       __imp_?dragMoveEvent@QWidget@@MAEXPAVQDragMoveEvent@@@Z 100424e4     Qt5Widgets:Qt5Widgets.dll
 0002:000004e8       __imp_?dropEvent@QWidget@@MAEXPAVQDropEvent@@@Z 100424e8     Qt5Widgets:Qt5Widgets.dll
 0002:000004ec       __imp_?enterEvent@QWidget@@MAEXPAVQEvent@@@Z 100424ec     Qt5Widgets:Qt5Widgets.dll
 0002:000004f0       __imp_?event@QAbstractSpinBox@@UAE_NPAVQEvent@@@Z 100424f0     Qt5Widgets:Qt5Widgets.dll
 0002:000004f4       __imp_?event@QCheckBox@@MAE_NPAVQEvent@@@Z 100424f4     Qt5Widgets:Qt5Widgets.dll
 0002:000004f8       __imp_?event@QComboBox@@UAE_NPAVQEvent@@@Z 100424f8     Qt5Widgets:Qt5Widgets.dll
 0002:000004fc       __imp_?event@QLabel@@MAE_NPAVQEvent@@@Z 100424fc     Qt5Widgets:Qt5Widgets.dll
 0002:00000500       __imp_?event@QSpinBox@@MAE_NPAVQEvent@@@Z 10042500     Qt5Widgets:Qt5Widgets.dll
 0002:00000504       __imp_?event@QTabWidget@@MAE_NPAVQEvent@@@Z 10042504     Qt5Widgets:Qt5Widgets.dll
 0002:00000508       __imp_?event@QWidget@@MAE_NPAVQEvent@@@Z 10042508     Qt5Widgets:Qt5Widgets.dll
 0002:0000050c       __imp_?expandingDirections@QBoxLayout@@UBE?AV?$QFlags@W4Orientation@Qt@@@@XZ 1004250c     Qt5Widgets:Qt5Widgets.dll
 0002:00000510       __imp_?expandingDirections@QGridLayout@@UBE?AV?$QFlags@W4Orientation@Qt@@@@XZ 10042510     Qt5Widgets:Qt5Widgets.dll
 0002:00000514       __imp_?expandingDirections@QSpacerItem@@UBE?AV?$QFlags@W4Orientation@Qt@@@@XZ 10042514     Qt5Widgets:Qt5Widgets.dll
 0002:00000518       __imp_?fixup@QDoubleSpinBox@@UBEXAAVQString@@@Z 10042518     Qt5Widgets:Qt5Widgets.dll
 0002:0000051c       __imp_?fixup@QSpinBox@@MBEXAAVQString@@@Z 1004251c     Qt5Widgets:Qt5Widgets.dll
 0002:00000520       __imp_?focusInEvent@QAbstractButton@@MAEXPAVQFocusEvent@@@Z 10042520     Qt5Widgets:Qt5Widgets.dll
 0002:00000524       __imp_?focusInEvent@QAbstractSpinBox@@MAEXPAVQFocusEvent@@@Z 10042524     Qt5Widgets:Qt5Widgets.dll
 0002:00000528       __imp_?focusInEvent@QComboBox@@MAEXPAVQFocusEvent@@@Z 10042528     Qt5Widgets:Qt5Widgets.dll
 0002:0000052c       __imp_?focusInEvent@QLabel@@MAEXPAVQFocusEvent@@@Z 1004252c     Qt5Widgets:Qt5Widgets.dll
 0002:00000530       __imp_?focusInEvent@QWidget@@MAEXPAVQFocusEvent@@@Z 10042530     Qt5Widgets:Qt5Widgets.dll
 0002:00000534       __imp_?focusNextPrevChild@QLabel@@MAE_N_N@Z 10042534     Qt5Widgets:Qt5Widgets.dll
 0002:00000538       __imp_?focusNextPrevChild@QWidget@@MAE_N_N@Z 10042538     Qt5Widgets:Qt5Widgets.dll
 0002:0000053c       __imp_?focusOutEvent@QAbstractButton@@MAEXPAVQFocusEvent@@@Z 1004253c     Qt5Widgets:Qt5Widgets.dll
 0002:00000540       __imp_?focusOutEvent@QAbstractSpinBox@@MAEXPAVQFocusEvent@@@Z 10042540     Qt5Widgets:Qt5Widgets.dll
 0002:00000544       __imp_?focusOutEvent@QComboBox@@MAEXPAVQFocusEvent@@@Z 10042544     Qt5Widgets:Qt5Widgets.dll
 0002:00000548       __imp_?focusOutEvent@QLabel@@MAEXPAVQFocusEvent@@@Z 10042548     Qt5Widgets:Qt5Widgets.dll
 0002:0000054c       __imp_?focusOutEvent@QWidget@@MAEXPAVQFocusEvent@@@Z 1004254c     Qt5Widgets:Qt5Widgets.dll
 0002:00000550       __imp_?geometry@QLayout@@UBE?AVQRect@@XZ 10042550     Qt5Widgets:Qt5Widgets.dll
 0002:00000554       __imp_?geometry@QSpacerItem@@UBE?AVQRect@@XZ 10042554     Qt5Widgets:Qt5Widgets.dll
 0002:00000558       __imp_?hasHeightForWidth@QBoxLayout@@UBE_NXZ 10042558     Qt5Widgets:Qt5Widgets.dll
 0002:0000055c       __imp_?hasHeightForWidth@QGridLayout@@UBE_NXZ 1004255c     Qt5Widgets:Qt5Widgets.dll
 0002:00000560       __imp_?hasHeightForWidth@QLayoutItem@@UBE_NXZ 10042560     Qt5Widgets:Qt5Widgets.dll
 0002:00000564       __imp_?hasHeightForWidth@QTabWidget@@UBE_NXZ 10042564     Qt5Widgets:Qt5Widgets.dll
 0002:00000568       __imp_?hasHeightForWidth@QWidget@@UBE_NXZ 10042568     Qt5Widgets:Qt5Widgets.dll
 0002:0000056c       __imp_?heightForWidth@QBoxLayout@@UBEHH@Z 1004256c     Qt5Widgets:Qt5Widgets.dll
 0002:00000570       __imp_?heightForWidth@QGridLayout@@UBEHH@Z 10042570     Qt5Widgets:Qt5Widgets.dll
 0002:00000574       __imp_?heightForWidth@QLabel@@UBEHH@Z 10042574     Qt5Widgets:Qt5Widgets.dll
 0002:00000578       __imp_?heightForWidth@QLayoutItem@@UBEHH@Z 10042578     Qt5Widgets:Qt5Widgets.dll
 0002:0000057c       __imp_?heightForWidth@QTabWidget@@UBEHH@Z 1004257c     Qt5Widgets:Qt5Widgets.dll
 0002:00000580       __imp_?heightForWidth@QWidget@@UBEHH@Z 10042580     Qt5Widgets:Qt5Widgets.dll
 0002:00000584       __imp_?hideEvent@QAbstractSpinBox@@MAEXPAVQHideEvent@@@Z 10042584     Qt5Widgets:Qt5Widgets.dll
 0002:00000588       __imp_?hideEvent@QComboBox@@MAEXPAVQHideEvent@@@Z 10042588     Qt5Widgets:Qt5Widgets.dll
 0002:0000058c       __imp_?hideEvent@QWidget@@MAEXPAVQHideEvent@@@Z 1004258c     Qt5Widgets:Qt5Widgets.dll
 0002:00000590       __imp_?hidePopup@QComboBox@@UAEXXZ 10042590     Qt5Widgets:Qt5Widgets.dll
 0002:00000594       __imp_?hitButton@QCheckBox@@MBE_NABVQPoint@@@Z 10042594     Qt5Widgets:Qt5Widgets.dll
 0002:00000598       __imp_?indexOf@QLayout@@UBEHPAVQWidget@@@Z 10042598     Qt5Widgets:Qt5Widgets.dll
 0002:0000059c       __imp_?initPainter@QWidget@@MBEXPAVQPainter@@@Z 1004259c     Qt5Widgets:Qt5Widgets.dll
 0002:000005a0       __imp_?inputMethodEvent@QComboBox@@MAEXPAVQInputMethodEvent@@@Z 100425a0     Qt5Widgets:Qt5Widgets.dll
 0002:000005a4       __imp_?inputMethodEvent@QWidget@@MAEXPAVQInputMethodEvent@@@Z 100425a4     Qt5Widgets:Qt5Widgets.dll
 0002:000005a8       __imp_?inputMethodQuery@QAbstractSpinBox@@UBE?AVQVariant@@W4InputMethodQuery@Qt@@@Z 100425a8     Qt5Widgets:Qt5Widgets.dll
 0002:000005ac       __imp_?inputMethodQuery@QComboBox@@UBE?AVQVariant@@W4InputMethodQuery@Qt@@@Z 100425ac     Qt5Widgets:Qt5Widgets.dll
 0002:000005b0       __imp_?inputMethodQuery@QWidget@@UBE?AVQVariant@@W4InputMethodQuery@Qt@@@Z 100425b0     Qt5Widgets:Qt5Widgets.dll
 0002:000005b4       __imp_?invalidate@QBoxLayout@@UAEXXZ 100425b4     Qt5Widgets:Qt5Widgets.dll
 0002:000005b8       __imp_?invalidate@QGridLayout@@UAEXXZ 100425b8     Qt5Widgets:Qt5Widgets.dll
 0002:000005bc       __imp_?invalidate@QLayoutItem@@UAEXXZ 100425bc     Qt5Widgets:Qt5Widgets.dll
 0002:000005c0       __imp_?isEmpty@QLayout@@UBE_NXZ 100425c0     Qt5Widgets:Qt5Widgets.dll
 0002:000005c4       __imp_?isEmpty@QSpacerItem@@UBE_NXZ 100425c4     Qt5Widgets:Qt5Widgets.dll
 0002:000005c8       __imp_?itemAt@QBoxLayout@@UBEPAVQLayoutItem@@H@Z 100425c8     Qt5Widgets:Qt5Widgets.dll
 0002:000005cc       __imp_?itemAt@QGridLayout@@UBEPAVQLayoutItem@@H@Z 100425cc     Qt5Widgets:Qt5Widgets.dll
 0002:000005d0       __imp_?keyPressEvent@QAbstractButton@@MAEXPAVQKeyEvent@@@Z 100425d0     Qt5Widgets:Qt5Widgets.dll
 0002:000005d4       __imp_?keyPressEvent@QAbstractSpinBox@@MAEXPAVQKeyEvent@@@Z 100425d4     Qt5Widgets:Qt5Widgets.dll
 0002:000005d8       __imp_?keyPressEvent@QComboBox@@MAEXPAVQKeyEvent@@@Z 100425d8     Qt5Widgets:Qt5Widgets.dll
 0002:000005dc       __imp_?keyPressEvent@QLabel@@MAEXPAVQKeyEvent@@@Z 100425dc     Qt5Widgets:Qt5Widgets.dll
 0002:000005e0       __imp_?keyPressEvent@QTabWidget@@MAEXPAVQKeyEvent@@@Z 100425e0     Qt5Widgets:Qt5Widgets.dll
 0002:000005e4       __imp_?keyPressEvent@QWidget@@MAEXPAVQKeyEvent@@@Z 100425e4     Qt5Widgets:Qt5Widgets.dll
 0002:000005e8       __imp_?keyReleaseEvent@QAbstractButton@@MAEXPAVQKeyEvent@@@Z 100425e8     Qt5Widgets:Qt5Widgets.dll
 0002:000005ec       __imp_?keyReleaseEvent@QAbstractSpinBox@@MAEXPAVQKeyEvent@@@Z 100425ec     Qt5Widgets:Qt5Widgets.dll
 0002:000005f0       __imp_?keyReleaseEvent@QComboBox@@MAEXPAVQKeyEvent@@@Z 100425f0     Qt5Widgets:Qt5Widgets.dll
 0002:000005f4       __imp_?keyReleaseEvent@QWidget@@MAEXPAVQKeyEvent@@@Z 100425f4     Qt5Widgets:Qt5Widgets.dll
 0002:000005f8       __imp_?layout@QLayout@@UAEPAV1@XZ 100425f8     Qt5Widgets:Qt5Widgets.dll
 0002:000005fc       __imp_?layout@QLayoutItem@@UAEPAVQLayout@@XZ 100425fc     Qt5Widgets:Qt5Widgets.dll
 0002:00000600       __imp_?leaveEvent@QWidget@@MAEXPAVQEvent@@@Z 10042600     Qt5Widgets:Qt5Widgets.dll
 0002:00000604       __imp_?maximumSize@QBoxLayout@@UBE?AVQSize@@XZ 10042604     Qt5Widgets:Qt5Widgets.dll
 0002:00000608       __imp_?maximumSize@QGridLayout@@UBE?AVQSize@@XZ 10042608     Qt5Widgets:Qt5Widgets.dll
 0002:0000060c       __imp_?maximumSize@QSpacerItem@@UBE?AVQSize@@XZ 1004260c     Qt5Widgets:Qt5Widgets.dll
 0002:00000610       __imp_?metaObject@QCheckBox@@UBEPBUQMetaObject@@XZ 10042610     Qt5Widgets:Qt5Widgets.dll
 0002:00000614       __imp_?metaObject@QComboBox@@UBEPBUQMetaObject@@XZ 10042614     Qt5Widgets:Qt5Widgets.dll
 0002:00000618       __imp_?metaObject@QDoubleSpinBox@@UBEPBUQMetaObject@@XZ 10042618     Qt5Widgets:Qt5Widgets.dll
 0002:0000061c       __imp_?metaObject@QGridLayout@@UBEPBUQMetaObject@@XZ 1004261c     Qt5Widgets:Qt5Widgets.dll
 0002:00000620       __imp_?metaObject@QHBoxLayout@@UBEPBUQMetaObject@@XZ 10042620     Qt5Widgets:Qt5Widgets.dll
 0002:00000624       __imp_?metaObject@QLabel@@UBEPBUQMetaObject@@XZ 10042624     Qt5Widgets:Qt5Widgets.dll
 0002:00000628       __imp_?metaObject@QSpinBox@@UBEPBUQMetaObject@@XZ 10042628     Qt5Widgets:Qt5Widgets.dll
 0002:0000062c       __imp_?metaObject@QTabWidget@@UBEPBUQMetaObject@@XZ 1004262c     Qt5Widgets:Qt5Widgets.dll
 0002:00000630       __imp_?metaObject@QVBoxLayout@@UBEPBUQMetaObject@@XZ 10042630     Qt5Widgets:Qt5Widgets.dll
 0002:00000634       __imp_?metaObject@QWidget@@UBEPBUQMetaObject@@XZ 10042634     Qt5Widgets:Qt5Widgets.dll
 0002:00000638       __imp_?metric@QWidget@@MBEHW4PaintDeviceMetric@QPaintDevice@@@Z 10042638     Qt5Widgets:Qt5Widgets.dll
 0002:0000063c       __imp_?minimumHeightForWidth@QBoxLayout@@UBEHH@Z 1004263c     Qt5Widgets:Qt5Widgets.dll
 0002:00000640       __imp_?minimumHeightForWidth@QGridLayout@@UBEHH@Z 10042640     Qt5Widgets:Qt5Widgets.dll
 0002:00000644       __imp_?minimumHeightForWidth@QLayoutItem@@UBEHH@Z 10042644     Qt5Widgets:Qt5Widgets.dll
 0002:00000648       __imp_?minimumSize@QBoxLayout@@UBE?AVQSize@@XZ 10042648     Qt5Widgets:Qt5Widgets.dll
 0002:0000064c       __imp_?minimumSize@QGridLayout@@UBE?AVQSize@@XZ 1004264c     Qt5Widgets:Qt5Widgets.dll
 0002:00000650       __imp_?minimumSize@QSpacerItem@@UBE?AVQSize@@XZ 10042650     Qt5Widgets:Qt5Widgets.dll
 0002:00000654       __imp_?minimumSizeHint@QAbstractSpinBox@@UBE?AVQSize@@XZ 10042654     Qt5Widgets:Qt5Widgets.dll
 0002:00000658       __imp_?minimumSizeHint@QCheckBox@@UBE?AVQSize@@XZ 10042658     Qt5Widgets:Qt5Widgets.dll
 0002:0000065c       __imp_?minimumSizeHint@QComboBox@@UBE?AVQSize@@XZ 1004265c     Qt5Widgets:Qt5Widgets.dll
 0002:00000660       __imp_?minimumSizeHint@QLabel@@UBE?AVQSize@@XZ 10042660     Qt5Widgets:Qt5Widgets.dll
 0002:00000664       __imp_?minimumSizeHint@QTabWidget@@UBE?AVQSize@@XZ 10042664     Qt5Widgets:Qt5Widgets.dll
 0002:00000668       __imp_?minimumSizeHint@QWidget@@UBE?AVQSize@@XZ 10042668     Qt5Widgets:Qt5Widgets.dll
 0002:0000066c       __imp_?mouseDoubleClickEvent@QWidget@@MAEXPAVQMouseEvent@@@Z 1004266c     Qt5Widgets:Qt5Widgets.dll
 0002:00000670       __imp_?mouseMoveEvent@QAbstractSpinBox@@MAEXPAVQMouseEvent@@@Z 10042670     Qt5Widgets:Qt5Widgets.dll
 0002:00000674       __imp_?mouseMoveEvent@QCheckBox@@MAEXPAVQMouseEvent@@@Z 10042674     Qt5Widgets:Qt5Widgets.dll
 0002:00000678       __imp_?mouseMoveEvent@QLabel@@MAEXPAVQMouseEvent@@@Z 10042678     Qt5Widgets:Qt5Widgets.dll
 0002:0000067c       __imp_?mouseMoveEvent@QWidget@@MAEXPAVQMouseEvent@@@Z 1004267c     Qt5Widgets:Qt5Widgets.dll
 0002:00000680       __imp_?mousePressEvent@QAbstractButton@@MAEXPAVQMouseEvent@@@Z 10042680     Qt5Widgets:Qt5Widgets.dll
 0002:00000684       __imp_?mousePressEvent@QAbstractSpinBox@@MAEXPAVQMouseEvent@@@Z 10042684     Qt5Widgets:Qt5Widgets.dll
 0002:00000688       __imp_?mousePressEvent@QComboBox@@MAEXPAVQMouseEvent@@@Z 10042688     Qt5Widgets:Qt5Widgets.dll
 0002:0000068c       __imp_?mousePressEvent@QLabel@@MAEXPAVQMouseEvent@@@Z 1004268c     Qt5Widgets:Qt5Widgets.dll
 0002:00000690       __imp_?mousePressEvent@QWidget@@MAEXPAVQMouseEvent@@@Z 10042690     Qt5Widgets:Qt5Widgets.dll
 0002:00000694       __imp_?mouseReleaseEvent@QAbstractButton@@MAEXPAVQMouseEvent@@@Z 10042694     Qt5Widgets:Qt5Widgets.dll
 0002:00000698       __imp_?mouseReleaseEvent@QAbstractSpinBox@@MAEXPAVQMouseEvent@@@Z 10042698     Qt5Widgets:Qt5Widgets.dll
 0002:0000069c       __imp_?mouseReleaseEvent@QComboBox@@MAEXPAVQMouseEvent@@@Z 1004269c     Qt5Widgets:Qt5Widgets.dll
 0002:000006a0       __imp_?mouseReleaseEvent@QLabel@@MAEXPAVQMouseEvent@@@Z 100426a0     Qt5Widgets:Qt5Widgets.dll
 0002:000006a4       __imp_?mouseReleaseEvent@QWidget@@MAEXPAVQMouseEvent@@@Z 100426a4     Qt5Widgets:Qt5Widgets.dll
 0002:000006a8       __imp_?moveEvent@QWidget@@MAEXPAVQMoveEvent@@@Z 100426a8     Qt5Widgets:Qt5Widgets.dll
 0002:000006ac       __imp_?nativeEvent@QWidget@@MAE_NABVQByteArray@@PAXPAJ@Z 100426ac     Qt5Widgets:Qt5Widgets.dll
 0002:000006b0       __imp_?nextCheckState@QCheckBox@@MAEXXZ 100426b0     Qt5Widgets:Qt5Widgets.dll
 0002:000006b4       __imp_?paintEngine@QWidget@@UBEPAVQPaintEngine@@XZ 100426b4     Qt5Widgets:Qt5Widgets.dll
 0002:000006b8       __imp_?paintEvent@QAbstractSpinBox@@MAEXPAVQPaintEvent@@@Z 100426b8     Qt5Widgets:Qt5Widgets.dll
 0002:000006bc       __imp_?paintEvent@QCheckBox@@MAEXPAVQPaintEvent@@@Z 100426bc     Qt5Widgets:Qt5Widgets.dll
 0002:000006c0       __imp_?paintEvent@QComboBox@@MAEXPAVQPaintEvent@@@Z 100426c0     Qt5Widgets:Qt5Widgets.dll
 0002:000006c4       __imp_?paintEvent@QLabel@@MAEXPAVQPaintEvent@@@Z 100426c4     Qt5Widgets:Qt5Widgets.dll
 0002:000006c8       __imp_?paintEvent@QTabWidget@@MAEXPAVQPaintEvent@@@Z 100426c8     Qt5Widgets:Qt5Widgets.dll
 0002:000006cc       __imp_?paintEvent@QWidget@@MAEXPAVQPaintEvent@@@Z 100426cc     Qt5Widgets:Qt5Widgets.dll
 0002:000006d0       __imp_?qt_metacall@QCheckBox@@UAEHW4Call@QMetaObject@@HPAPAX@Z 100426d0     Qt5Widgets:Qt5Widgets.dll
 0002:000006d4       __imp_?qt_metacall@QComboBox@@UAEHW4Call@QMetaObject@@HPAPAX@Z 100426d4     Qt5Widgets:Qt5Widgets.dll
 0002:000006d8       __imp_?qt_metacall@QDoubleSpinBox@@UAEHW4Call@QMetaObject@@HPAPAX@Z 100426d8     Qt5Widgets:Qt5Widgets.dll
 0002:000006dc       __imp_?qt_metacall@QGridLayout@@UAEHW4Call@QMetaObject@@HPAPAX@Z 100426dc     Qt5Widgets:Qt5Widgets.dll
 0002:000006e0       __imp_?qt_metacall@QHBoxLayout@@UAEHW4Call@QMetaObject@@HPAPAX@Z 100426e0     Qt5Widgets:Qt5Widgets.dll
 0002:000006e4       __imp_?qt_metacall@QLabel@@UAEHW4Call@QMetaObject@@HPAPAX@Z 100426e4     Qt5Widgets:Qt5Widgets.dll
 0002:000006e8       __imp_?qt_metacall@QSpinBox@@UAEHW4Call@QMetaObject@@HPAPAX@Z 100426e8     Qt5Widgets:Qt5Widgets.dll
 0002:000006ec       __imp_?qt_metacall@QTabWidget@@UAEHW4Call@QMetaObject@@HPAPAX@Z 100426ec     Qt5Widgets:Qt5Widgets.dll
 0002:000006f0       __imp_?qt_metacall@QVBoxLayout@@UAEHW4Call@QMetaObject@@HPAPAX@Z 100426f0     Qt5Widgets:Qt5Widgets.dll
 0002:000006f4       __imp_?qt_metacall@QWidget@@UAEHW4Call@QMetaObject@@HPAPAX@Z 100426f4     Qt5Widgets:Qt5Widgets.dll
 0002:000006f8       __imp_?qt_metacast@QCheckBox@@UAEPAXPBD@Z 100426f8     Qt5Widgets:Qt5Widgets.dll
 0002:000006fc       __imp_?qt_metacast@QComboBox@@UAEPAXPBD@Z 100426fc     Qt5Widgets:Qt5Widgets.dll
 0002:00000700       __imp_?qt_metacast@QDoubleSpinBox@@UAEPAXPBD@Z 10042700     Qt5Widgets:Qt5Widgets.dll
 0002:00000704       __imp_?qt_metacast@QGridLayout@@UAEPAXPBD@Z 10042704     Qt5Widgets:Qt5Widgets.dll
 0002:00000708       __imp_?qt_metacast@QHBoxLayout@@UAEPAXPBD@Z 10042708     Qt5Widgets:Qt5Widgets.dll
 0002:0000070c       __imp_?qt_metacast@QLabel@@UAEPAXPBD@Z 1004270c     Qt5Widgets:Qt5Widgets.dll
 0002:00000710       __imp_?qt_metacast@QSpinBox@@UAEPAXPBD@Z 10042710     Qt5Widgets:Qt5Widgets.dll
 0002:00000714       __imp_?qt_metacast@QTabWidget@@UAEPAXPBD@Z 10042714     Qt5Widgets:Qt5Widgets.dll
 0002:00000718       __imp_?qt_metacast@QVBoxLayout@@UAEPAXPBD@Z 10042718     Qt5Widgets:Qt5Widgets.dll
 0002:0000071c       __imp_?qt_metacast@QWidget@@UAEPAXPBD@Z 1004271c     Qt5Widgets:Qt5Widgets.dll
 0002:00000720       __imp_?redirected@QWidget@@MBEPAVQPaintDevice@@PAVQPoint@@@Z 10042720     Qt5Widgets:Qt5Widgets.dll
 0002:00000724       __imp_?resizeEvent@QAbstractSpinBox@@MAEXPAVQResizeEvent@@@Z 10042724     Qt5Widgets:Qt5Widgets.dll
 0002:00000728       __imp_?resizeEvent@QComboBox@@MAEXPAVQResizeEvent@@@Z 10042728     Qt5Widgets:Qt5Widgets.dll
 0002:0000072c       __imp_?resizeEvent@QTabWidget@@MAEXPAVQResizeEvent@@@Z 1004272c     Qt5Widgets:Qt5Widgets.dll
 0002:00000730       __imp_?resizeEvent@QWidget@@MAEXPAVQResizeEvent@@@Z 10042730     Qt5Widgets:Qt5Widgets.dll
 0002:00000734       __imp_?setGeometry@QBoxLayout@@UAEXABVQRect@@@Z 10042734     Qt5Widgets:Qt5Widgets.dll
 0002:00000738       __imp_?setGeometry@QGridLayout@@UAEXABVQRect@@@Z 10042738     Qt5Widgets:Qt5Widgets.dll
 0002:0000073c       __imp_?setGeometry@QSpacerItem@@UAEXABVQRect@@@Z 1004273c     Qt5Widgets:Qt5Widgets.dll
 0002:00000740       __imp_?setVisible@QWidget@@UAEX_N@Z 10042740     Qt5Widgets:Qt5Widgets.dll
 0002:00000744       __imp_?sharedPainter@QWidget@@MBEPAVQPainter@@XZ 10042744     Qt5Widgets:Qt5Widgets.dll
 0002:00000748       __imp_?showEvent@QAbstractSpinBox@@MAEXPAVQShowEvent@@@Z 10042748     Qt5Widgets:Qt5Widgets.dll
 0002:0000074c       __imp_?showEvent@QComboBox@@MAEXPAVQShowEvent@@@Z 1004274c     Qt5Widgets:Qt5Widgets.dll
 0002:00000750       __imp_?showEvent@QTabWidget@@MAEXPAVQShowEvent@@@Z 10042750     Qt5Widgets:Qt5Widgets.dll
 0002:00000754       __imp_?showEvent@QWidget@@MAEXPAVQShowEvent@@@Z 10042754     Qt5Widgets:Qt5Widgets.dll
 0002:00000758       __imp_?showPopup@QComboBox@@UAEXXZ 10042758     Qt5Widgets:Qt5Widgets.dll
 0002:0000075c       __imp_?sizeHint@QAbstractSpinBox@@UBE?AVQSize@@XZ 1004275c     Qt5Widgets:Qt5Widgets.dll
 0002:00000760       __imp_?sizeHint@QBoxLayout@@UBE?AVQSize@@XZ 10042760     Qt5Widgets:Qt5Widgets.dll
 0002:00000764       __imp_?sizeHint@QCheckBox@@UBE?AVQSize@@XZ 10042764     Qt5Widgets:Qt5Widgets.dll
 0002:00000768       __imp_?sizeHint@QComboBox@@UBE?AVQSize@@XZ 10042768     Qt5Widgets:Qt5Widgets.dll
 0002:0000076c       __imp_?sizeHint@QGridLayout@@UBE?AVQSize@@XZ 1004276c     Qt5Widgets:Qt5Widgets.dll
 0002:00000770       __imp_?sizeHint@QLabel@@UBE?AVQSize@@XZ 10042770     Qt5Widgets:Qt5Widgets.dll
 0002:00000774       __imp_?sizeHint@QSpacerItem@@UBE?AVQSize@@XZ 10042774     Qt5Widgets:Qt5Widgets.dll
 0002:00000778       __imp_?sizeHint@QTabWidget@@UBE?AVQSize@@XZ 10042778     Qt5Widgets:Qt5Widgets.dll
 0002:0000077c       __imp_?sizeHint@QWidget@@UBE?AVQSize@@XZ 1004277c     Qt5Widgets:Qt5Widgets.dll
 0002:00000780       __imp_?spacerItem@QLayoutItem@@UAEPAVQSpacerItem@@XZ 10042780     Qt5Widgets:Qt5Widgets.dll
 0002:00000784       __imp_?spacerItem@QSpacerItem@@UAEPAV1@XZ 10042784     Qt5Widgets:Qt5Widgets.dll
 0002:00000788       __imp_?stepBy@QAbstractSpinBox@@UAEXH@Z 10042788     Qt5Widgets:Qt5Widgets.dll
 0002:0000078c       __imp_?stepEnabled@QAbstractSpinBox@@MBE?AV?$QFlags@W4StepEnabledFlag@QAbstractSpinBox@@@@XZ 1004278c     Qt5Widgets:Qt5Widgets.dll
 0002:00000790       __imp_?tabInserted@QTabWidget@@MAEXH@Z 10042790     Qt5Widgets:Qt5Widgets.dll
 0002:00000794       __imp_?tabRemoved@QTabWidget@@MAEXH@Z 10042794     Qt5Widgets:Qt5Widgets.dll
 0002:00000798       __imp_?tabletEvent@QWidget@@MAEXPAVQTabletEvent@@@Z 10042798     Qt5Widgets:Qt5Widgets.dll
 0002:0000079c       __imp_?takeAt@QBoxLayout@@UAEPAVQLayoutItem@@H@Z 1004279c     Qt5Widgets:Qt5Widgets.dll
 0002:000007a0       __imp_?takeAt@QGridLayout@@UAEPAVQLayoutItem@@H@Z 100427a0     Qt5Widgets:Qt5Widgets.dll
 0002:000007a4       __imp_?textFromValue@QDoubleSpinBox@@UBE?AVQString@@N@Z 100427a4     Qt5Widgets:Qt5Widgets.dll
 0002:000007a8       __imp_?textFromValue@QSpinBox@@MBE?AVQString@@H@Z 100427a8     Qt5Widgets:Qt5Widgets.dll
 0002:000007ac       __imp_?timerEvent@QAbstractButton@@MAEXPAVQTimerEvent@@@Z 100427ac     Qt5Widgets:Qt5Widgets.dll
 0002:000007b0       __imp_?timerEvent@QAbstractSpinBox@@MAEXPAVQTimerEvent@@@Z 100427b0     Qt5Widgets:Qt5Widgets.dll
 0002:000007b4       __imp_?validate@QDoubleSpinBox@@UBE?AW4State@QValidator@@AAVQString@@AAH@Z 100427b4     Qt5Widgets:Qt5Widgets.dll
 0002:000007b8       \177Qt5Widgets_NULL_THUNK_DATA 100427b8     Qt5Widgets:Qt5Widgets.dll
 0002:000007bc       __imp_?attribute@QDomElement@@QBE?AVQString@@ABV2@0@Z 100427bc     Qt5Xml:Qt5Xml.dll
 0002:000007c0       \177Qt5Xml_NULL_THUNK_DATA 100427c0     Qt5Xml:Qt5Xml.dll
 0002:000007c4       __imp_?qt_metacast@PhyTreeGeneratorTask@U2@@UAEPAXPBD@Z 100427c4     U2Algorithm:U2Algorithm.dll
 0002:000007c8       __imp_?report@PhyTreeGeneratorTask@U2@@UAE?AW4ReportResult@Task@2@XZ 100427c8     U2Algorithm:U2Algorithm.dll
 0002:000007cc       __imp_?metaObject@PhyTreeGeneratorTask@U2@@UBEPBUQMetaObject@@XZ 100427cc     U2Algorithm:U2Algorithm.dll
 0002:000007d0       __imp_??0CreatePhyTreeSettings@U2@@QAE@XZ 100427d0     U2Algorithm:U2Algorithm.dll
 0002:000007d4       __imp_??1CreatePhyTreeSettings@U2@@QAE@XZ 100427d4     U2Algorithm:U2Algorithm.dll
 0002:000007d8       __imp_?registerPhyTreeGenerator@PhyTreeGeneratorRegistry@U2@@QAE_NPAVPhyTreeGenerator@2@ABVQString@@@Z 100427d8     U2Algorithm:U2Algorithm.dll
 0002:000007dc       __imp_?run@PhyTreeGeneratorTask@U2@@UAEXXZ 100427dc     U2Algorithm:U2Algorithm.dll
 0002:000007e0       __imp_?qt_metacall@PhyTreeGeneratorTask@U2@@UAEHW4Call@QMetaObject@@HPAPAX@Z 100427e0     U2Algorithm:U2Algorithm.dll
 0002:000007e4       __imp_??0PhyTreeGeneratorTask@U2@@QAE@ABVMultipleSequenceAlignment@1@ABVCreatePhyTreeSettings@1@@Z 100427e4     U2Algorithm:U2Algorithm.dll
 0002:000007e8       __imp_??_7PhyTreeGenerator@U2@@6B@ 100427e8     U2Algorithm:U2Algorithm.dll
 0002:000007ec       __imp_??0PhyTreeGeneratorLauncherTask@U2@@QAE@ABVMultipleSequenceAlignment@1@ABVCreatePhyTreeSettings@1@@Z 100427ec     U2Algorithm:U2Algorithm.dll
 0002:000007f0       __imp_??1PhyTreeGeneratorLauncherTask@U2@@UAE@XZ 100427f0     U2Algorithm:U2Algorithm.dll
 0002:000007f4       __imp_?getResult@PhyTreeGeneratorLauncherTask@U2@@QAE?AV?$QSharedDataPointer@VPhyTreeData@U2@@@@XZ 100427f4     U2Algorithm:U2Algorithm.dll
 0002:000007f8       __imp_?metaObject@PhyTreeGeneratorLauncherTask@U2@@UBEPBUQMetaObject@@XZ 100427f8     U2Algorithm:U2Algorithm.dll
 0002:000007fc       __imp_?prepare@PhyTreeGeneratorLauncherTask@U2@@UAEXXZ 100427fc     U2Algorithm:U2Algorithm.dll
 0002:00000800       __imp_?qt_metacall@PhyTreeGeneratorLauncherTask@U2@@UAEHW4Call@QMetaObject@@HPAPAX@Z 10042800     U2Algorithm:U2Algorithm.dll
 0002:00000804       __imp_?qt_metacast@PhyTreeGeneratorLauncherTask@U2@@UAEPAXPBD@Z 10042804     U2Algorithm:U2Algorithm.dll
 0002:00000808       __imp_?report@PhyTreeGeneratorLauncherTask@U2@@UAE?AW4ReportResult@Task@2@XZ 10042808     U2Algorithm:U2Algorithm.dll
 0002:0000080c       __imp_?run@PhyTreeGeneratorLauncherTask@U2@@UAEXXZ 1004280c     U2Algorithm:U2Algorithm.dll
 0002:00000810       __imp_??0CreatePhyTreeSettings@U2@@QAE@ABV01@@Z 10042810     U2Algorithm:U2Algorithm.dll
 0002:00000814       __imp_?getResult@PhyTreeGeneratorTask@U2@@QAE?AV?$QSharedDataPointer@VPhyTreeData@U2@@@@XZ 10042814     U2Algorithm:U2Algorithm.dll
 0002:00000818       __imp_??4CreatePhyTreeSettings@U2@@QAEAAV01@ABV01@@Z 10042818     U2Algorithm:U2Algorithm.dll
 0002:0000081c       __imp_?staticMetaObject@PhyTreeGeneratorTask@U2@@2UQMetaObject@@B 1004281c     U2Algorithm:U2Algorithm.dll
 0002:00000820       __imp_??1PhyTreeGeneratorTask@U2@@UAE@XZ 10042820     U2Algorithm:U2Algorithm.dll
 0002:00000824       \177U2Algorithm_NULL_THUNK_DATA 10042824     U2Algorithm:U2Algorithm.dll
 0002:00000828       __imp_?getBranchesDistance@PhyNode@U2@@QBENH@Z 10042828     U2Core:U2Core.dll
 0002:0000082c       __imp_?branchCount@PhyNode@U2@@QBEHXZ 1004282c     U2Core:U2Core.dll
 0002:00000830       __imp_??0PhyNode@U2@@QAE@XZ 10042830     U2Core:U2Core.dll
 0002:00000834       __imp_?removeBranch@PhyTreeData@U2@@SAXPAVPhyNode@2@0@Z 10042834     U2Core:U2Core.dll
 0002:00000838       __imp_?addBranch@PhyTreeData@U2@@SAPAVPhyBranch@2@PAVPhyNode@2@0N@Z 10042838     U2Core:U2Core.dll
 0002:0000083c       __imp_?print@PhyTreeData@U2@@QBEXXZ 1004283c     U2Core:U2Core.dll
 0002:00000840       __imp_??1PhyTreeData@U2@@QAE@XZ 10042840     U2Core:U2Core.dll
 0002:00000844       __imp_??0PhyTreeData@U2@@QAE@ABV01@@Z 10042844     U2Core:U2Core.dll
 0002:00000848       __imp_?getMsaRows@MultipleSequenceAlignmentData@U2@@QBE?BV?$QList@VMultipleSequenceAlignmentRow@U2@@@@XZ 10042848     U2Core:U2Core.dll
 0002:0000084c       __imp_?getMsaRow@MultipleSequenceAlignmentData@U2@@QBE?BVMultipleSequenceAlignmentRow@2@H@Z 1004284c     U2Core:U2Core.dll
 0002:00000850       __imp_?getNumRows@MultipleSequenceAlignmentData@U2@@QBEHXZ 10042850     U2Core:U2Core.dll
 0002:00000854       __imp_??CMultipleSequenceAlignment@U2@@QBEPBVMultipleSequenceAlignmentData@1@XZ 10042854     U2Core:U2Core.dll
 0002:00000858       __imp_??0MultipleSequenceAlignmentRow@U2@@QAE@ABV01@@Z 10042858     U2Core:U2Core.dll
 0002:0000085c       __imp_??1MultipleSequenceAlignmentRow@U2@@UAE@XZ 1004285c     U2Core:U2Core.dll
 0002:00000860       __imp_??CMultipleSequenceAlignmentRow@U2@@QBEPBVMultipleSequenceAlignmentRowData@1@XZ 10042860     U2Core:U2Core.dll
 0002:00000864       __imp_?getLength@MultipleAlignmentData@U2@@QBEHXZ 10042864     U2Core:U2Core.dll
 0002:00000868       __imp_?getAlphabet@MultipleAlignmentData@U2@@QBEPBVDNAAlphabet@2@XZ 10042868     U2Core:U2Core.dll
 0002:0000086c       __imp_?getName@MultipleAlignmentData@U2@@QBE?AVQString@@XZ 1004286c     U2Core:U2Core.dll
 0002:00000870       __imp_??1MultipleAlignmentRow@U2@@UAE@XZ 10042870     U2Core:U2Core.dll
 0002:00000874       __imp_?instance@AppResourcePool@U2@@SAPAV12@XZ 10042874     U2Core:U2Core.dll
 0002:00000878       __imp_?getResource@AppResourcePool@U2@@QBEPAVAppResource@2@H@Z 10042878     U2Core:U2Core.dll
 0002:0000087c       __imp_??1Logger@U2@@UAE@XZ 1004287c     U2Core:U2Core.dll
 0002:00000880       __imp_?isConnected@PhyNode@U2@@QBE_NPBV12@@Z 10042880     U2Core:U2Core.dll
 0002:00000884       __imp_?getParameterValue@CMDLineRegistry@U2@@QBE?AVQString@@ABV3@H@Z 10042884     U2Core:U2Core.dll
 0002:00000888       __imp_?staticMetaObject@CmdlineTask@U2@@2UQMetaObject@@B 10042888     U2Core:U2Core.dll
 0002:0000088c       __imp_?qt_metacall@CmdlineTask@U2@@UAEHW4Call@QMetaObject@@HPAPAX@Z 1004288c     U2Core:U2Core.dll
 0002:00000890       __imp_?qt_metacast@CmdlineTask@U2@@UAEPAXPBD@Z 10042890     U2Core:U2Core.dll
 0002:00000894       __imp_?staticMetaObject@Plugin@U2@@2UQMetaObject@@B 10042894     U2Core:U2Core.dll
 0002:00000898       __imp_?qt_metacall@Plugin@U2@@UAEHW4Call@QMetaObject@@HPAPAX@Z 10042898     U2Core:U2Core.dll
 0002:0000089c       __imp_?qt_metacast@Plugin@U2@@UAEPAXPBD@Z 1004289c     U2Core:U2Core.dll
 0002:000008a0       __imp_?appendChars@MultipleSequenceAlignmentData@U2@@QAEXHPBDH@Z 100428a0     U2Core:U2Core.dll
 0002:000008a4       __imp_?addRow@MultipleSequenceAlignmentData@U2@@QAEXABVQString@@ABVQByteArray@@@Z 100428a4     U2Core:U2Core.dll
 0002:000008a8       __imp_?prepareDirLocation@GUrlUtils@U2@@SA?AVQString@@ABV3@AAVU2OpStatus@2@@Z 100428a8     U2Core:U2Core.dll
 0002:000008ac       __imp_??4MultipleSequenceAlignment@U2@@QAEAAV01@ABV01@@Z 100428ac     U2Core:U2Core.dll
 0002:000008b0       __imp_??0MultipleSequenceAlignment@U2@@QAE@ABV01@@Z 100428b0     U2Core:U2Core.dll
 0002:000008b4       __imp_??CMultipleSequenceAlignment@U2@@QAEPAVMultipleSequenceAlignmentData@1@XZ 100428b4     U2Core:U2Core.dll
 0002:000008b8       __imp_?updateDatabase@MultipleSequenceAlignmentObject@U2@@EAEXAAVU2OpStatus@2@ABVMultipleAlignment@2@@Z 100428b8     U2Core:U2Core.dll
 0002:000008bc       __imp_?updateCachedRows@MultipleSequenceAlignmentObject@U2@@EAEXAAVU2OpStatus@2@ABV?$QList@_J@@@Z 100428bc     U2Core:U2Core.dll
 0002:000008c0       __imp_?setGObjectName@MultipleAlignmentObject@U2@@UAEXABVQString@@@Z 100428c0     U2Core:U2Core.dll
 0002:000008c4       __imp_?replaceCharacter@MultipleSequenceAlignmentObject@U2@@UAEXHHD@Z 100428c4     U2Core:U2Core.dll
 0002:000008c8       __imp_?removeRowPrivate@MultipleSequenceAlignmentObject@U2@@EAEXAAVU2OpStatus@2@ABVU2EntityRef@2@_J@Z 100428c8     U2Core:U2Core.dll
 0002:000008cc       __imp_?removeRegionPrivate@MultipleSequenceAlignmentObject@U2@@EAEXAAVU2OpStatus@2@ABVU2EntityRef@2@ABV?$QList@_J@@HH@Z 100428cc     U2Core:U2Core.dll
 0002:000008d0       __imp_?qt_metacast@MultipleSequenceAlignmentObject@U2@@UAEPAXPBD@Z 100428d0     U2Core:U2Core.dll
 0002:000008d4       __imp_?qt_metacall@MultipleSequenceAlignmentObject@U2@@UAEHW4Call@QMetaObject@@HPAPAX@Z 100428d4     U2Core:U2Core.dll
 0002:000008d8       __imp_?metaObject@MultipleSequenceAlignmentObject@U2@@UBEPBUQMetaObject@@XZ 100428d8     U2Core:U2Core.dll
 0002:000008dc       __imp_?loadDataCore@MultipleAlignmentObject@U2@@EAEXAAVU2OpStatus@2@@Z 100428dc     U2Core:U2Core.dll
 0002:000008e0       __imp_?loadAlignment@MultipleSequenceAlignmentObject@U2@@EAEXAAVU2OpStatus@2@@Z 100428e0     U2Core:U2Core.dll
 0002:000008e4       __imp_?insertGap@MultipleSequenceAlignmentObject@U2@@EAEXABVU2Region@2@HH@Z 100428e4     U2Core:U2Core.dll
 0002:000008e8       __imp_?getTaskError@CmdlineTask@U2@@MBE?AVQString@@XZ 100428e8     U2Core:U2Core.dll
 0002:000008ec       __imp_?deleteColumnsWithGaps@MultipleSequenceAlignmentObject@U2@@UAEXAAVU2OpStatus@2@H@Z 100428ec     U2Core:U2Core.dll
 0002:000008f0       __imp_?clone@MultipleSequenceAlignmentObject@U2@@UBEPAV12@ABVU2DbiRef@2@AAVU2OpStatus@2@ABV?$QMap@VQString@@VQVariant@@@@@Z 100428f0     U2Core:U2Core.dll
 0002:000008f4       __imp_?charAt@MultipleSequenceAlignmentObject@U2@@UBEDH_J@Z 100428f4     U2Core:U2Core.dll
 0002:000008f8       __imp_?createInstance@PhyTreeObject@U2@@SAPAV12@ABV?$QSharedDataPointer@VPhyTreeData@U2@@@@ABVQString@@ABVU2DbiRef@2@AAVU2OpStatus@2@ABV?$QMap@VQString@@VQVariant@@@@@Z 100428f8     U2Core:U2Core.dll
 0002:000008fc       __imp_??0MultipleSequenceAlignmentObject@U2@@QAE@ABVQString@@ABVU2EntityRef@1@ABV?$QMap@VQString@@VQVariant@@@@ABVMultipleSequenceAlignment@1@@Z 100428fc     U2Core:U2Core.dll
 0002:00000900       __imp_??0MultipleSequenceAlignment@U2@@QAE@ABVQString@@PBVDNAAlphabet@1@ABV?$QList@VMultipleSequenceAlignmentRow@U2@@@@@Z 10042900     U2Core:U2Core.dll
 0002:00000904       __imp_??1MultipleAlignmentObject@U2@@UAE@XZ 10042904     U2Core:U2Core.dll
 0002:00000908       __imp_?logOutputObject@CmdlineInOutTaskRunner@U2@@SAXABVQByteArray@@@Z 10042908     U2Core:U2Core.dll
 0002:0000090c       __imp_??1CmdlineTask@U2@@UAE@XZ 1004290c     U2Core:U2Core.dll
 0002:00000910       __imp_?report@CmdlineTask@U2@@UAE?AW4ReportResult@Task@2@XZ 10042910     U2Core:U2Core.dll
 0002:00000914       __imp_??0CmdlineTask@U2@@QAE@ABVQString@@V?$QFlags@W4TaskFlag@U2@@@@@Z 10042914     U2Core:U2Core.dll
 0002:00000918       __imp_??0U2EntityRef@U2@@QAE@ABV01@@Z 10042918     U2Core:U2Core.dll
 0002:0000091c       __imp_??0U2DbiRef@U2@@QAE@ABV01@@Z 1004291c     U2Core:U2Core.dll
 0002:00000920       __imp_?staticMetaObject@PhyTreeObject@U2@@2UQMetaObject@@B 10042920     U2Core:U2Core.dll
 0002:00000924       __imp_?staticMetaObject@MultipleSequenceAlignmentObject@U2@@2UQMetaObject@@B 10042924     U2Core:U2Core.dll
 0002:00000928       __imp_?staticMetaObject@Document@U2@@2UQMetaObject@@B 10042928     U2Core:U2Core.dll
 0002:0000092c       __imp_?PHYLOGENETIC_TREE@GObjectTypes@U2@@2VQString@@B 1004292c     U2Core:U2Core.dll
 0002:00000930       __imp_?MULTIPLE_SEQUENCE_ALIGNMENT@GObjectTypes@U2@@2VQString@@B 10042930     U2Core:U2Core.dll
 0002:00000934       __imp_?treesAreAlike@PhyTreeObject@U2@@SA_NABV?$QSharedDataPointer@VPhyTreeData@U2@@@@0@Z 10042934     U2Core:U2Core.dll
 0002:00000938       __imp_?getMultipleAlignment@MultipleAlignmentObject@U2@@QBEABVMultipleAlignment@2@XZ 10042938     U2Core:U2Core.dll
 0002:0000093c       __imp_?findGObjectByType@Document@U2@@QBE?AV?$QList@PAVGObject@U2@@@@VQString@@W4UnloadedObjectFilter@2@@Z 1004293c     U2Core:U2Core.dll
 0002:00000940       __imp_??1MultipleSequenceAlignment@U2@@UAE@XZ 10042940     U2Core:U2Core.dll
 0002:00000944       __imp_??0MultipleSequenceAlignment@U2@@QAE@ABVMultipleAlignment@1@@Z 10042944     U2Core:U2Core.dll
 0002:00000948       __imp_??1MultipleAlignment@U2@@UAE@XZ 10042948     U2Core:U2Core.dll
 0002:0000094c       __imp_?hasError@Task@U2@@QBE_NXZ 1004294c     U2Core:U2Core.dll
 0002:00000950       __imp_?OUT_DB_ARG@CmdlineInOutTaskRunner@U2@@2VQString@@B 10042950     U2Core:U2Core.dll
 0002:00000954       __imp_?IN_ID_ARG@CmdlineInOutTaskRunner@U2@@2VQString@@B 10042954     U2Core:U2Core.dll
 0002:00000958       __imp_?IN_DB_ARG@CmdlineInOutTaskRunner@U2@@2VQString@@B 10042958     U2Core:U2Core.dll
 0002:0000095c       __imp_?qt_metacast@TaskStarter@U2@@UAEPAXPBD@Z 1004295c     U2Core:U2Core.dll
 0002:00000960       __imp_?qt_metacall@TaskStarter@U2@@UAEHW4Call@QMetaObject@@HPAPAX@Z 10042960     U2Core:U2Core.dll
 0002:00000964       __imp_?metaObject@TaskStarter@U2@@UBEPBUQMetaObject@@XZ 10042964     U2Core:U2Core.dll
 0002:00000968       __imp_??1Plugin@U2@@UAE@XZ 10042968     U2Core:U2Core.dll
 0002:0000096c       __imp_??0Plugin@U2@@QAE@ABVQString@@0_NW4PluginState@1@@Z 1004296c     U2Core:U2Core.dll
 0002:00000970       __imp_??1U2OpStatus2Log@U2@@UAE@XZ 10042970     U2Core:U2Core.dll
 0002:00000974       __imp_??0U2OpStatus2Log@U2@@QAE@W4LogLevel@1@@Z 10042974     U2Core:U2Core.dll
 0002:00000978       __imp_?parseDataId@CmdlineInOutTaskRunner@U2@@SA?AVQByteArray@@ABVQString@@ABVU2DbiRef@2@AAVU2OpStatus@2@@Z 10042978     U2Core:U2Core.dll
 0002:0000097c       __imp_?parseDbiRef@CmdlineInOutTaskRunner@U2@@SA?AVU2DbiRef@2@ABVQString@@AAVU2OpStatus@2@@Z 1004297c     U2Core:U2Core.dll
 0002:00000980       __imp_??0Logger@U2@@QAE@ABVQString@@@Z 10042980     U2Core:U2Core.dll
 0002:00000984       __imp_?hasParameter@CMDLineRegistry@U2@@QBE_NABVQString@@H@Z 10042984     U2Core:U2Core.dll
 0002:00000988       __imp_?getCMDLineRegistry@AppContext@U2@@SAPAVCMDLineRegistry@2@XZ 10042988     U2Core:U2Core.dll
 0002:0000098c       __imp_?getPhyTreeGeneratorRegistry@AppContext@U2@@SAPAVPhyTreeGeneratorRegistry@2@XZ 1004298c     U2Core:U2Core.dll
 0002:00000990       __imp_?getTestFramework@AppContext@U2@@SAPAVTestFramework@2@XZ 10042990     U2Core:U2Core.dll
 0002:00000994       __imp_?getPluginSupport@AppContext@U2@@SAPAVPluginSupport@2@XZ 10042994     U2Core:U2Core.dll
 0002:00000998       __imp_?isCoR@U2OpStatus@U2@@UBE_NXZ 10042998     U2Core:U2Core.dll
 0002:0000099c       __imp_?U2_DBI_LOCKING_MODE@U2DbiOptions@U2@@2VQString@@B 1004299c     U2Core:U2Core.dll
 0002:000009a0       __imp_?unlockState@StateLockableTreeItem@U2@@UAEXPAVStateLock@2@@Z 100429a0     U2Core:U2Core.dll
 0002:000009a4       __imp_?setParentStateLockItem@GObject@U2@@EAEXPAVStateLockableTreeItem@2@@Z 100429a4     U2Core:U2Core.dll
 0002:000009a8       __imp_?setModified@StateLockableTreeItem@U2@@UAEX_NABVQString@@@Z 100429a8     U2Core:U2Core.dll
 0002:000009ac       __imp_?setModificationTrack@StateLockableTreeItem@U2@@UAEX_N@Z 100429ac     U2Core:U2Core.dll
 0002:000009b0       __imp_?setMainThreadModificationOnly@StateLockableItem@U2@@UAEX_N@Z 100429b0     U2Core:U2Core.dll
 0002:000009b4       __imp_?setGObjectName@GObject@U2@@UAEXABVQString@@@Z 100429b4     U2Core:U2Core.dll
 0002:000009b8       __imp_?run@Task@U2@@UAEXXZ 100429b8     U2Core:U2Core.dll
 0002:000009bc       __imp_?report@CmdlineInOutTaskRunner@U2@@UAE?AW4ReportResult@Task@2@XZ 100429bc     U2Core:U2Core.dll
 0002:000009c0       __imp_?qt_metacast@PhyTreeObject@U2@@UAEPAXPBD@Z 100429c0     U2Core:U2Core.dll
 0002:000009c4       __imp_?qt_metacast@CmdlineInOutTaskRunner@U2@@UAEPAXPBD@Z 100429c4     U2Core:U2Core.dll
 0002:000009c8       __imp_?qt_metacall@PhyTreeObject@U2@@UAEHW4Call@QMetaObject@@HPAPAX@Z 100429c8     U2Core:U2Core.dll
 0002:000009cc       __imp_?qt_metacall@CmdlineInOutTaskRunner@U2@@UAEHW4Call@QMetaObject@@HPAPAX@Z 100429cc     U2Core:U2Core.dll
 0002:000009d0       __imp_?prepare@CmdlineTaskRunner@U2@@UAEXXZ 100429d0     U2Core:U2Core.dll
 0002:000009d4       __imp_?parseCommandLogWord@CmdlineInOutTaskRunner@U2@@EAE_NABVQString@@@Z 100429d4     U2Core:U2Core.dll
 0002:000009d8       __imp_?metaObject@PhyTreeObject@U2@@UBEPBUQMetaObject@@XZ 100429d8     U2Core:U2Core.dll
 0002:000009dc       __imp_?metaObject@CmdlineInOutTaskRunner@U2@@UBEPBUQMetaObject@@XZ 100429dc     U2Core:U2Core.dll
 0002:000009e0       __imp_?lockState@StateLockableTreeItem@U2@@UAEXPAVStateLock@2@@Z 100429e0     U2Core:U2Core.dll
 0002:000009e4       __imp_?loadDataCore@PhyTreeObject@U2@@MAEXAAVU2OpStatus@2@@Z 100429e4     U2Core:U2Core.dll
 0002:000009e8       __imp_?isTreeItemModified@StateLockableTreeItem@U2@@UBE_NXZ 100429e8     U2Core:U2Core.dll
 0002:000009ec       __imp_?isStateLocked@StateLockableTreeItem@U2@@UBE_NXZ 100429ec     U2Core:U2Core.dll
 0002:000009f0       __imp_?isModificationTracked@StateLockableItem@U2@@UBE_NXZ 100429f0     U2Core:U2Core.dll
 0002:000009f4       __imp_?isModificationAllowed@StateLockableItem@U2@@UAE_NABVQString@@@Z 100429f4     U2Core:U2Core.dll
 0002:000009f8       __imp_?isMainThreadObject@StateLockableItem@U2@@UBE_NXZ 100429f8     U2Core:U2Core.dll
 0002:000009fc       __imp_?isMainThreadModificationOnly@StateLockableTreeItem@U2@@UBE_NXZ 100429fc     U2Core:U2Core.dll
 0002:00000a00       __imp_?isItemModified@StateLockableItem@U2@@UBE_NXZ 10042a00     U2Core:U2Core.dll
 0002:00000a04       __imp_?isCommandLogLine@CmdlineInOutTaskRunner@U2@@EBE_NABVQString@@@Z 10042a04     U2Core:U2Core.dll
 0002:00000a08       __imp_?hasModifiedChildren@StateLockableTreeItem@U2@@UBE_NXZ 10042a08     U2Core:U2Core.dll
 0002:00000a0c       __imp_?getTree@PhyTreeObject@U2@@UBEABV?$QSharedDataPointer@VPhyTreeData@U2@@@@XZ 10042a0c     U2Core:U2Core.dll
 0002:00000a10       __imp_?getModificationVersion@StateLockableItem@U2@@UBEHXZ 10042a10     U2Core:U2Core.dll
 0002:00000a14       __imp_?getDocument@GObject@U2@@UBEPAVDocument@2@XZ 10042a14     U2Core:U2Core.dll
 0002:00000a18       __imp_?clone@PhyTreeObject@U2@@UBEPAVGObject@2@ABVU2DbiRef@2@AAVU2OpStatus@2@ABV?$QMap@VQString@@VQVariant@@@@@Z 10042a18     U2Core:U2Core.dll
 0002:00000a1c       __imp_?checkConstraints@GObject@U2@@UBE_NPBVGObjectConstraints@2@@Z 10042a1c     U2Core:U2Core.dll
 0002:00000a20       __imp_?getCurrentProcessTemporaryDirPath@UserAppsSettings@U2@@QBE?AVQString@@ABV3@@Z 10042a20     U2Core:U2Core.dll
 0002:00000a24       __imp_??1DbiConnection@U2@@QAE@XZ 10042a24     U2Core:U2Core.dll
 0002:00000a28       __imp_??0DbiConnection@U2@@QAE@ABVU2DbiRef@1@_NAAVU2OpStatus@1@ABV?$QHash@VQString@@V1@@@@Z 10042a28     U2Core:U2Core.dll
 0002:00000a2c       __imp_??1PhyTreeObject@U2@@UAE@XZ 10042a2c     U2Core:U2Core.dll
 0002:00000a30       __imp_??0PhyTreeObject@U2@@QAE@ABVQString@@ABVU2EntityRef@1@ABV?$QMap@VQString@@VQVariant@@@@@Z 10042a30     U2Core:U2Core.dll
 0002:00000a34       __imp_?createAlignment@MultipleSequenceAlignmentImporter@U2@@SAPAVMultipleSequenceAlignmentObject@2@ABVU2DbiRef@2@AAVMultipleSequenceAlignment@2@AAVU2OpStatus@2@@Z 10042a34     U2Core:U2Core.dll
 0002:00000a38       __imp_?prepareTmpFileLocation@GUrlUtils@U2@@SA?AVQString@@ABV3@00AAVU2OpStatus@2@@Z 10042a38     U2Core:U2Core.dll
 0002:00000a3c       __imp_??1CmdlineInOutTaskRunner@U2@@UAE@XZ 10042a3c     U2Core:U2Core.dll
 0002:00000a40       __imp_?getOutputObjects@CmdlineInOutTaskRunner@U2@@QBEABV?$QList@VQByteArray@@@@XZ 10042a40     U2Core:U2Core.dll
 0002:00000a44       __imp_??0CmdlineInOutTaskRunner@U2@@QAE@ABVCmdlineInOutTaskConfig@1@@Z 10042a44     U2Core:U2Core.dll
 0002:00000a48       __imp_??1CmdlineInOutTaskConfig@U2@@QAE@XZ 10042a48     U2Core:U2Core.dll
 0002:00000a4c       __imp_??0CmdlineInOutTaskConfig@U2@@QAE@XZ 10042a4c     U2Core:U2Core.dll
 0002:00000a50       __imp_?addSubTask@Task@U2@@QAEXPAV12@@Z 10042a50     U2Core:U2Core.dll
 0002:00000a54       __imp_??1U2EntityRef@U2@@QAE@XZ 10042a54     U2Core:U2Core.dll
 0002:00000a58       __imp_??0U2EntityRef@U2@@QAE@ABVU2DbiRef@1@ABVQByteArray@@@Z 10042a58     U2Core:U2Core.dll
 0002:00000a5c       __imp_??1U2DbiRef@U2@@QAE@XZ 10042a5c     U2Core:U2Core.dll
 0002:00000a60       __imp_??0U2DbiRef@U2@@QAE@ABVQString@@0@Z 10042a60     U2Core:U2Core.dll
 0002:00000a64       __imp_?getAppSettings@AppContext@U2@@SAPAVAppSettings@2@XZ 10042a64     U2Core:U2Core.dll
 0002:00000a68       __imp_?getSettings@AppContext@U2@@SAPAVSettings@2@XZ 10042a68     U2Core:U2Core.dll
 0002:00000a6c       __imp_??_7SimpleEventCounter@U2@@6B@ 10042a6c     U2Core:U2Core.dll
 0002:00000a70       __imp_?setReportingSupported@Task@U2@@UAEX_N@Z 10042a70     U2Core:U2Core.dll
 0002:00000a74       __imp_?setReportingEnabled@Task@U2@@UAEX_N@Z 10042a74     U2Core:U2Core.dll
 0002:00000a78       __imp_?setNotificationReport@Task@U2@@UAEX_N@Z 10042a78     U2Core:U2Core.dll
 0002:00000a7c       __imp_?setNoAutoDelete@Task@U2@@UAEX_N@Z 10042a7c     U2Core:U2Core.dll
 0002:00000a80       __imp_?setCollectChildrensWarningsFlag@Task@U2@@UAEX_N@Z 10042a80     U2Core:U2Core.dll
 0002:00000a84       __imp_?propagateSubtaskError@Task@U2@@UAE_NXZ 10042a84     U2Core:U2Core.dll
 0002:00000a88       __imp_?prepare@Task@U2@@UAEXXZ 10042a88     U2Core:U2Core.dll
 0002:00000a8c       __imp_?onSubTaskFinished@Task@U2@@MAE?AV?$QList@PAVTask@U2@@@@PAV12@@Z 10042a8c     U2Core:U2Core.dll
 0002:00000a90       __imp_?isTopLevelTask@Task@U2@@UBE_NXZ 10042a90     U2Core:U2Core.dll
 0002:00000a94       __imp_?isReportingSupported@Task@U2@@UBE_NXZ 10042a94     U2Core:U2Core.dll
 0002:00000a98       __imp_?isReportingEnabled@Task@U2@@UBE_NXZ 10042a98     U2Core:U2Core.dll
 0002:00000a9c       __imp_?isNotificationReport@Task@U2@@UBE_NXZ 10042a9c     U2Core:U2Core.dll
 0002:00000aa0       __imp_?hasWarning@Task@U2@@UBE_NXZ 10042aa0     U2Core:U2Core.dll
 0002:00000aa4       __imp_?hasSubtasksWithErrors@Task@U2@@UBE_NXZ 10042aa4     U2Core:U2Core.dll
 0002:00000aa8       __imp_?getWarnings@Task@U2@@UBE?AVQStringList@@XZ 10042aa8     U2Core:U2Core.dll
 0002:00000aac       __imp_?getTopLevelParentTask@Task@U2@@UAEPAV12@XZ 10042aac     U2Core:U2Core.dll
 0002:00000ab0       __imp_?getTaskId@Task@U2@@UBE_JXZ 10042ab0     U2Core:U2Core.dll
 0002:00000ab4       __imp_?getSubtaskWithErrors@Task@U2@@UBEPAV12@XZ 10042ab4     U2Core:U2Core.dll
 0002:00000ab8       __imp_?getParentTask@Task@U2@@UBEPAV12@XZ 10042ab8     U2Core:U2Core.dll
 0002:00000abc       __imp_?getNumParallelSubtasks@Task@U2@@UBEHXZ 10042abc     U2Core:U2Core.dll
 0002:00000ac0       __imp_?generateReport@Task@U2@@UBE?AVQString@@XZ 10042ac0     U2Core:U2Core.dll
 0002:00000ac4       __imp_?cleanup@Task@U2@@UAEXXZ 10042ac4     U2Core:U2Core.dll
 0002:00000ac8       __imp_??0PhyTreeData@U2@@QAE@XZ 10042ac8     U2Core:U2Core.dll
 0002:00000acc       __imp_?setTaskName@Task@U2@@IAEXABVQString@@@Z 10042acc     U2Core:U2Core.dll
 0002:00000ad0       __imp_?setError@Task@U2@@QAEXABVQString@@@Z 10042ad0     U2Core:U2Core.dll
 0002:00000ad4       __imp_??1SimpleEventCounter@U2@@UAE@XZ 10042ad4     U2Core:U2Core.dll
 0002:00000ad8       __imp_??0GReportableCounter@U2@@QAE@ABVQString@@0N@Z 10042ad8     U2Core:U2Core.dll
 0002:00000adc       __imp_??1GCounter@U2@@UAE@XZ 10042adc     U2Core:U2Core.dll
 0002:00000ae0       __imp_?setBranchesDistance@PhyNode@U2@@QAEXHN@Z 10042ae0     U2Core:U2Core.dll
 0002:00000ae4       __imp_?getParentNode@PhyNode@U2@@QAEPAV12@XZ 10042ae4     U2Core:U2Core.dll
 0002:00000ae8       __imp_?getBranch@PhyNode@U2@@QBEPAVPhyBranch@2@H@Z 10042ae8     U2Core:U2Core.dll
 0002:00000aec       \177U2Core_NULL_THUNK_DATA 10042aec     U2Core:U2Core.dll
 0002:00000af0       __imp_?findFormat@GTestFormatRegistry@U2@@QAEPAVGTestFormat@2@ABVQString@@@Z 10042af0     U2Test:U2Test.dll
 0002:00000af4       __imp_?staticMetaObject@GTest@U2@@2UQMetaObject@@B 10042af4     U2Test:U2Test.dll
 0002:00000af8       __imp_?qt_metacall@GTest@U2@@UAEHW4Call@QMetaObject@@HPAPAX@Z 10042af8     U2Test:U2Test.dll
 0002:00000afc       __imp_?qt_metacast@GTest@U2@@UAEPAXPBD@Z 10042afc     U2Test:U2Test.dll
 0002:00000b00       __imp_??1XmlTest@U2@@UAE@XZ 10042b00     U2Test:U2Test.dll
 0002:00000b04       __imp_??0XmlTest@U2@@QAE@ABVQString@@PAVGTest@1@PBVGTestEnvironment@1@V?$QFlags@W4TaskFlag@U2@@@@ABV?$QList@PAVGTest@U2@@@@@Z 10042b04     U2Test:U2Test.dll
 0002:00000b08       __imp_??1XMLTestFactory@U2@@UAE@XZ 10042b08     U2Test:U2Test.dll
 0002:00000b0c       __imp_??0XMLTestFactory@U2@@QAE@ABVQString@@@Z 10042b0c     U2Test:U2Test.dll
 0002:00000b10       __imp_?failMissingValue@GTest@U2@@IAEXABVQString@@@Z 10042b10     U2Test:U2Test.dll
 0002:00000b14       __imp_?getContext@GTest@U2@@QBEPAVQObject@@ABVQString@@@Z 10042b14     U2Test:U2Test.dll
 0002:00000b18       __imp_?staticMetaObject@XMLTestFormat@U2@@2UQMetaObject@@B 10042b18     U2Test:U2Test.dll
 0002:00000b1c       \177U2Test_NULL_THUNK_DATA 10042b1c     U2Test:U2Test.dll
 0002:00000b20       __imp_?storeSettings@PhyTreeDisplayOptionsWidget@U2@@UAEXXZ 10042b20     U2View:U2View.dll
 0002:00000b24       __imp_?restoreDefault@PhyTreeDisplayOptionsWidget@U2@@UAEXXZ 10042b24     U2View:U2View.dll
 0002:00000b28       __imp_?insertOutputOptionWidget@CreatePhyTreeWidget@U2@@UAE_NPAVPhyTreeDisplayOptionsWidget@2@@Z 10042b28     U2View:U2View.dll
 0002:00000b2c       __imp_?fillSettings@PhyTreeDisplayOptionsWidget@U2@@UAEXAAVCreatePhyTreeSettings@2@@Z 10042b2c     U2View:U2View.dll
 0002:00000b30       __imp_?checkSettings@CreatePhyTreeWidget@U2@@UAE_NAAVQString@@ABVCreatePhyTreeSettings@2@@Z 10042b30     U2View:U2View.dll
 0002:00000b34       __imp_?checkMemoryEstimation@CreatePhyTreeWidget@U2@@UAE_NAAVQString@@ABVMultipleSequenceAlignment@2@ABVCreatePhyTreeSettings@2@@Z 10042b34     U2View:U2View.dll
 0002:00000b38       __imp_??1PhyTreeDisplayOptionsWidget@U2@@UAE@XZ 10042b38     U2View:U2View.dll
 0002:00000b3c       __imp_??0PhyTreeDisplayOptionsWidget@U2@@QAE@PAVQWidget@@@Z 10042b3c     U2View:U2View.dll
 0002:00000b40       __imp_??1CreatePhyTreeWidget@U2@@UAE@XZ 10042b40     U2View:U2View.dll
 0002:00000b44       __imp_?settingsPath@CreatePhyTreeWidget@U2@@SA?AVQString@@XZ 10042b44     U2View:U2View.dll
 0002:00000b48       __imp_??0CreatePhyTreeWidget@U2@@QAE@PAVQWidget@@@Z 10042b48     U2View:U2View.dll
 0002:00000b4c       \177U2View_NULL_THUNK_DATA 10042b4c     U2View:U2View.dll
 0002:00000b50       ___xc_a                    10042b50     MSVCRT:cinitexe.obj
 0002:00000efc       ___xc_z                    10042efc     MSVCRT:cinitexe.obj
 0002:00000f00       ___xi_a                    10042f00     MSVCRT:cinitexe.obj
 0002:00000f10       ___xi_z                    10042f10     MSVCRT:cinitexe.obj
 0002:00000f58       ??_C@_00CNPNBAHC@?$AA@     10042f58     DistanceMatrix.obj
 0002:00000f60       ??_7error_category@std@@6B@ 10042f60     DistanceMatrix.obj
 0002:00000f7c       ??_7_Generic_error_category@std@@6B@ 10042f7c     DistanceMatrix.obj
 0002:00000f94       ??_C@_07DCLBNMLN@generic?$AA@ 10042f94     DistanceMatrix.obj
 0002:00000f9c       ??_C@_0O@BFJCFAAK@unknown?5error?$AA@ 10042f9c     DistanceMatrix.obj
 0002:00000fb0       ??_7_Iostream_error_category@std@@6B@ 10042fb0     DistanceMatrix.obj
 0002:00000fc8       ??_C@_08LLGCOLLL@iostream?$AA@ 10042fc8     DistanceMatrix.obj
 0002:00000fd4       ??_C@_0BG@PADBLCHM@iostream?5stream?5error?$AA@ 10042fd4     DistanceMatrix.obj
 0002:00000ff0       ??_7_System_error_category@std@@6B@ 10042ff0     DistanceMatrix.obj
 0002:00001008       ??_C@_06FHFOAHML@system?$AA@ 10043008     DistanceMatrix.obj
 0002:00001010       ??_C@_0L@JLHNEGIN@Algorithms?$AA@ 10043010     DistanceMatrix.obj
 0002:0000101c       ??_C@_07PGLPGHFC@Console?$AA@ 1004301c     DistanceMatrix.obj
 0002:00001024       ??_C@_0O@BOFHOPCF@Core?5Services?$AA@ 10043024     DistanceMatrix.obj
 0002:00001034       ??_C@_0N@PPADAKBM@Input?1Output?$AA@ 10043034     DistanceMatrix.obj
 0002:00001044       ??_C@_0M@KPPBKPKK@Performance?$AA@ 10043044     DistanceMatrix.obj
 0002:00001050       ??_C@_07BFDHHBBI@Scripts?$AA@ 10043050     DistanceMatrix.obj
 0002:00001058       ??_C@_05EEGKELMG@Tasks?$AA@ 10043058     DistanceMatrix.obj
 0002:00001060       ??_C@_0P@NIIOBHGA@User?5Interface?$AA@ 10043060     DistanceMatrix.obj
 0002:00001070       ??_C@_0N@JINCGGMN@User?5Actions?$AA@ 10043070     DistanceMatrix.obj
 0002:00001084       ??_7MemoryLocker@U2@@6B@   10043084     DistanceMatrix.obj
 0002:00001088       ??_C@_0BO@FLJHDJNA@MemoryLocker?5?9?5Resource?5error?$AA@ 10043088     DistanceMatrix.obj
 0002:000010a8       ??_C@_0EC@PGPNOHNG@MemoryLocker?5?9?5Not?5enough?5memory@ 100430a8     DistanceMatrix.obj
 0002:000010f0       ??_SMultipleSequenceAlignmentRow@U2@@6B@ 100430f0     DistanceMatrix.obj
 0002:000010f8       ??_C@_0EC@BCFJDHH@Not?5enough?5memory?5to?5calculate?5d@ 100430f8     DistanceMatrix.obj
 0002:0000113c       ??_C@_0BB@HDDJILBO@Distance?5Matrix?5?$AA@ 1004313c     DistanceMatrix.obj
 0002:00001150       ??_C@_01CLKCMJKC@?5?$AA@   10043150     DistanceMatrix.obj
 0002:00001154       ??_C@_09MNOCDBIK@Q?5Matrix?5?$AA@ 10043154     DistanceMatrix.obj
 0002:00001160       ??_C@_03BHBGBHAB@___?$AA@  10043160     DistanceMatrix.obj
 0002:00001164       ??_C@_04BNGIIOIP@ROOT?$AA@ 10043164     DistanceMatrix.obj
 0002:0000116c       ??_C@_06KLJADLOP@name?3?5?$AA@ 1004316c     DistanceMatrix.obj
 0002:00001174       ??_C@_06PMEKPMOJ@?5Keys?3?$AA@ 10043174     DistanceMatrix.obj
 0002:0000117c       ??_C@_07HLENKCLA@Value?5?3?$AA@ 1004317c     DistanceMatrix.obj
 0002:00001184       ??_C@_0BA@JFNIOLAK@string?5too?5long?$AA@ 10043184     DistanceMatrix.obj
 0002:00001194       ??_C@_0BI@CFPLBAOH@invalid?5string?5position?$AA@ 10043194     DistanceMatrix.obj
 0002:000011ac       __real@3f000000            100431ac     DistanceMatrix.obj
 0002:000011b0       __real@3ff0000000000000    100431b0     DistanceMatrix.obj
 0002:000011b8       __real@7fefffffffffffff    100431b8     DistanceMatrix.obj
 0002:000011c0       __real@ffefffffffffffff    100431c0     DistanceMatrix.obj
 0002:000011d0       __xmm@7fffffffffffffff7fffffffffffffff 100431d0     DistanceMatrix.obj
 0002:000011e4       ??_7NeighborJoinCalculateTreeTask@U2@@6B@ 100431e4     NeighborJoinAdapter.obj
 0002:00001270       ??_C@_07LIBMDHOF@node?5?$CF1?$AA@ 10043270     NeighborJoinAdapter.obj
 0002:00001280       ??_C@_0BH@CMOIIDEL@NeighborJoin?5algorithm?$AA@ 10043280     NeighborJoinAdapter.obj
 0002:00001298       ??_C@_0BC@INBDOCAP@PhylipNeigborJoin?$AA@ 10043298     NeighborJoinAdapter.obj
 0002:000012ac       ??_C@_0DD@MOCIKLCI@Neighbor?9Joining?5runs?5must?5have?5@ 100432ac     NeighborJoinAdapter.obj
 0002:000012e0       ??_C@_0BF@LEHMBNFM@Generating?5sequences?$AA@ 100432e0     NeighborJoinAdapter.obj
 0002:000012f8       ??_C@_0BM@KEGJNKHI@Can?8t?5create?5temporary?5file?$AA@ 100432f8     NeighborJoinAdapter.obj
 0002:00001314       ??_C@_0BC@PJCPCLG@Calculating?5trees?$AA@ 10043314     NeighborJoinAdapter.obj
 0002:00001328       ??_C@_0CG@LCFCFFEG@Calculated?5distance?5matrix?5is?5in@ 10043328     NeighborJoinAdapter.obj
 0002:00001350       ??_C@_0BL@OANLHJCD@Calculating?5consensus?5tree?$AA@ 10043350     NeighborJoinAdapter.obj
 0002:0000136c       ??_C@_0DH@HCFGKCJA@Not?5enough?5memory?5to?5calculate?5t@ 1004336c     NeighborJoinAdapter.obj
 0002:000013a4       ??_C@_0BA@CDHBGMBD@Phylip?5error?5?$CF1?$AA@ 100433a4     NeighborJoinAdapter.obj
 0002:000013b8       __real@0000000000000000    100433b8     NeighborJoinAdapter.obj
 0002:000013c0       __real@3fdbcb7b157df63a    100433c0     NeighborJoinAdapter.obj
 0002:000013c8       __real@42c80000            100433c8     NeighborJoinAdapter.obj
 0002:000013d4       ??_SQWidget@@6BQObject@@@  100433d4     NeighborJoinWidget.obj
 0002:0000148c       ??_SQWidget@@6BQPaintDevice@@@ 1004348c     NeighborJoinWidget.obj
 0002:000014ac       ??_SQCheckBox@@6BQObject@@@ 100434ac     NeighborJoinWidget.obj
 0002:00001570       ??_SQCheckBox@@6BQPaintDevice@@@ 10043570     NeighborJoinWidget.obj
 0002:00001594       ??_SQTabWidget@@6BQObject@@@ 10043594     NeighborJoinWidget.obj
 0002:00001654       ??_SQTabWidget@@6BQPaintDevice@@@ 10043654     NeighborJoinWidget.obj
 0002:00001674       ??_SQComboBox@@6BQObject@@@ 10043674     NeighborJoinWidget.obj
 0002:00001734       ??_SQComboBox@@6BQPaintDevice@@@ 10043734     NeighborJoinWidget.obj
 0002:00001754       ??_SQSpinBox@@6BQObject@@@ 10043754     NeighborJoinWidget.obj
 0002:00001828       ??_SQSpinBox@@6BQPaintDevice@@@ 10043828     NeighborJoinWidget.obj
 0002:0000184c       ??_SQDoubleSpinBox@@6BQObject@@@ 1004384c     NeighborJoinWidget.obj
 0002:00001920       ??_SQDoubleSpinBox@@6BQPaintDevice@@@ 10043920     NeighborJoinWidget.obj
 0002:00001944       ??_SQSpacerItem@@6B@       10043944     NeighborJoinWidget.obj
 0002:0000198c       ??_SQHBoxLayout@@6BQObject@@@ 1004398c     NeighborJoinWidget.obj
 0002:000019d4       ??_SQHBoxLayout@@6BQLayoutItem@@@ 100439d4     NeighborJoinWidget.obj
 0002:00001a1c       ??_SQVBoxLayout@@6BQObject@@@ 10043a1c     NeighborJoinWidget.obj
 0002:00001a64       ??_SQVBoxLayout@@6BQLayoutItem@@@ 10043a64     NeighborJoinWidget.obj
 0002:00001aac       ??_SQGridLayout@@6BQObject@@@ 10043aac     NeighborJoinWidget.obj
 0002:00001af4       ??_SQGridLayout@@6BQLayoutItem@@@ 10043af4     NeighborJoinWidget.obj
 0002:00001b3c       ??_SQLabel@@6BQObject@@@   10043b3c     NeighborJoinWidget.obj
 0002:00001bf4       ??_SQLabel@@6BQPaintDevice@@@ 10043bf4     NeighborJoinWidget.obj
 0002:00001c14       ??_SPhyTreeDisplayOptionsWidget@U2@@6BQObject@@@ 10043c14     NeighborJoinWidget.obj
 0002:00001ce4       ??_SPhyTreeDisplayOptionsWidget@U2@@6BQPaintDevice@@@ 10043ce4     NeighborJoinWidget.obj
 0002:00001d00       ??_C@_0BC@DLEJKFKG@1setEnabled?$CIbool?$CJ?$AA@ 10043d00     NeighborJoinWidget.obj
 0002:00001d14       ??_C@_0P@POCECEMJ@2toggled?$CIbool?$CJ?$AA@ 10043d14     NeighborJoinWidget.obj
 0002:00001d24       ??_C@_0BG@OFEGBGCK@Distance?5matrix?5model?$AA@ 10043d24     NeighborJoinWidget.obj
 0002:00001d3c       ??_C@_0BD@PIBKIBN@NeighborJoinWidget?$AA@ 10043d3c     NeighborJoinWidget.obj
 0002:00001d50       ??_C@_0DK@LMBHFKGK@Coefficient?5of?5variation?5of?5subs@ 10043d50     NeighborJoinWidget.obj
 0002:00001d8c       ??_C@_0CF@BIPAIMFI@Gamma?5distributed?5rates?5across?5s@ 10043d8c     NeighborJoinWidget.obj
 0002:00001db4       ??_C@_0BO@DJOLOABM@Transition?1transversion?5ratio?$AA@ 10043db4     NeighborJoinWidget.obj
 0002:00001dd4       ??_C@_0BA@NOPDLNEP@Distance?5Matrix?$AA@ 10043dd4     NeighborJoinWidget.obj
 0002:00001de4       ??_C@_0BF@HNDHAGOJ@Enable?5bootstrapping?$AA@ 10043de4     NeighborJoinWidget.obj
 0002:00001dfc       ??_C@_0BF@IECLMDCN@Number?5of?5replicates?$AA@ 10043dfc     NeighborJoinWidget.obj
 0002:00001e14       ??_C@_0BD@MAOOIOEE@Seed?5?$CImust?5be?5odd?$CJ?$AA@ 10043e14     NeighborJoinWidget.obj
 0002:00001e28       ??_C@_0P@MBCDKMFP@Consensus?5type?$AA@ 10043e28     NeighborJoinWidget.obj
 0002:00001e38       ??_C@_08LCDAJCG@Fraction?$AA@ 10043e38     NeighborJoinWidget.obj
 0002:00001e44       ??_C@_0CB@LHMAGAAD@Bootstrapping?5and?5Consensus?5Tree@ 10043e44     NeighborJoinWidget.obj
 0002:00001e68       ??_C@_0BA@PIEIIDAK@Display?5Options?$AA@ 10043e68     NeighborJoinWidget.obj
 0002:00002508       ??_7NeighborJoinWidget@U2@@6BQObject@@@ 10044508     NeighborJoinWidget.obj
 0002:000025d8       ??_7NeighborJoinWidget@U2@@6BQPaintDevice@@@ 100445d8     NeighborJoinWidget.obj
 0002:000025f4       ??_C@_02LOKBDPMM@M1?$AA@   100445f4     NeighborJoinWidget.obj
 0002:000025f8       ??_C@_06CEODFONB@Strict?$AA@ 100445f8     NeighborJoinWidget.obj
 0002:00002600       ??_C@_0BJ@FICOEHIJ@Majority?5Rule?5?$CIextended?$CJ?$AA@ 10044600     NeighborJoinWidget.obj
 0002:0000261c       ??_C@_0O@BJGEOIID@Majority?5Rule?$AA@ 1004461c     NeighborJoinWidget.obj
 0002:0000262c       ??_C@_06MHHONINI@?1model?$AA@ 1004462c     NeighborJoinWidget.obj
 0002:00002634       ??_C@_0N@NJMALHHA@?1gamma_distr?$AA@ 10044634     NeighborJoinWidget.obj
 0002:00002644       ??_C@_0N@NJNIALIA@?1alfa_factor?$AA@ 10044644     NeighborJoinWidget.obj
 0002:00002654       ??_C@_08NHAFIPEK@?1ttratio?$AA@ 10044654     NeighborJoinWidget.obj
 0002:00002660       ??_C@_08GJAFBCOD@?1bootstr?$AA@ 10044660     NeighborJoinWidget.obj
 0002:0000266c       ??_C@_0M@JCKHBBDE@?1replicates?$AA@ 1004466c     NeighborJoinWidget.obj
 0002:00002678       ??_C@_0P@GCOBEGMC@?1seq_boot_seed?$AA@ 10044678     NeighborJoinWidget.obj
 0002:00002688       ??_C@_09DCAHKPAA@?1fraction?$AA@ 10044688     NeighborJoinWidget.obj
 0002:00002694       ??_C@_0N@JDLHIKOD@?1consensusID?$AA@ 10044694     NeighborJoinWidget.obj
 0002:000026a8       ??_C@_0MB@CDGFLDKF@Probably?0?5for?5that?5alignment?5the@ 100446a8     NeighborJoinWidget.obj
 0002:0000276c       ??_C@_0BB@ODCHNCBJ@Seed?5must?5be?5odd?$AA@ 1004476c     NeighborJoinWidget.obj
 0002:00002780       ??_C@_0CK@DJIIDDDK@1sl_onMatrixModelChanged?$CIconst?5Q@ 10044780     NeighborJoinWidget.obj
 0002:000027ac       ??_C@_0CG@DDDJCHLP@2currentIndexChanged?$CIconst?5QStri@ 100447ac     NeighborJoinWidget.obj
 0002:000027d4       ??_C@_0CM@LPKOJCNM@1sl_onConsensusTypeChanged?$CIconst@ 100447d4     NeighborJoinWidget.obj
 0002:00002800       __real@3f847ae147ae147b    10044800     NeighborJoinWidget.obj
 0002:00002808       __real@3fb999999999999a    10044808     NeighborJoinWidget.obj
 0002:00002810       __real@3fe0000000000000    10044810     NeighborJoinWidget.obj
 0002:00002818       __real@4000000000000000    10044818     NeighborJoinWidget.obj
 0002:00002820       __real@4069000000000000    10044820     NeighborJoinWidget.obj
 0002:0000282c       ??_SCmdlineInOutTaskRunner@U2@@6B@ 1004482c     PhylipCmdlineTask.obj
 0002:000028c4       ??_SPhyTreeObject@U2@@6B@  100448c4     PhylipCmdlineTask.obj
 0002:00002948       ??_7PhylipCmdlineTask@U2@@6B@ 10044948     PhylipCmdlineTask.obj
 0002:000029d4       ??_C@_06IHFHDOMB@phylip?$AA@ 100449d4     PhylipCmdlineTask.obj
 0002:000029dc       ??_C@_06CGNOPMBC@matrix?$AA@ 100449dc     PhylipCmdlineTask.obj
 0002:000029e4       ??_C@_05KDLBCAI@gamma?$AA@ 100449e4     PhylipCmdlineTask.obj
 0002:000029ec       ??_C@_0N@FEEMGHCH@alpha?9factor?$AA@ 100449ec     PhylipCmdlineTask.obj
 0002:000029fc       ??_C@_08JBEPPMIF@tt?9ratio?$AA@ 100449fc     PhylipCmdlineTask.obj
 0002:00002a08       ??_C@_09HNKJMCAI@bootstrap?$AA@ 10044a08     PhylipCmdlineTask.obj
 0002:00002a14       ??_C@_0L@OIFACCDO@replicates?$AA@ 10044a14     PhylipCmdlineTask.obj
 0002:00002a20       ??_C@_04MENKDCKE@seed?$AA@ 10044a20     PhylipCmdlineTask.obj
 0002:00002a28       ??_C@_08IJNCILIF@fraction?$AA@ 10044a28     PhylipCmdlineTask.obj
 0002:00002a34       ??_C@_09OMAHMGIJ@consensus?$AA@ 10044a34     PhylipCmdlineTask.obj
 0002:00002a40       ??_C@_0CB@MACOHMJP@PHYLIP?5command?5line?5wrapper?5task@ 10044a40     PhylipCmdlineTask.obj
 0002:00002a64       ??_C@_0BH@DEDHGCKN@No?5tree?5objects?5found?4?$AA@ 10044a64     PhylipCmdlineTask.obj
 0002:00002a7c       ??_C@_04KCCPLAND@tree?$AA@ 10044a7c     PhylipCmdlineTask.obj
 0002:00002a84       ??_C@_02BAABKJLB@?9?9?$AA@ 10044a84     PhylipCmdlineTask.obj
 0002:00002a88       ??_C@_09HOLOPIAM@?9?9?$CF1?$DN?$CC?$CF2?$CC?$AA@ 10044a88     PhylipCmdlineTask.obj
 0002:00002a94       ??_C@_07FKKKPHCE@ugenedb?$AA@ 10044a94     PhylipCmdlineTask.obj
 0002:00002a9c       ??_C@_09GBBIJGED@SQLiteDbi?$AA@ 10044a9c     PhylipCmdlineTask.obj
 0002:00002aa8       ??_C@_06IKLLLDHL@normal?$AA@ 10044aa8     PhylipCmdlineTask.obj
 0002:00002ab4       ??_7?$AbstractId@H@U2@@6B@ 10044ab4     PhylipPlugin.obj
 0002:00002ac0       ??_7AbstractInt32Id@U2@@6B@ 10044ac0     PhylipPlugin.obj
 0002:00002acc       ??_7ServiceType@U2@@6B@    10044acc     PhylipPlugin.obj
 0002:00002ad8       ??_STaskStarter@U2@@6B@    10044ad8     PhylipPlugin.obj
 0002:00002b08       ??_7NeighborJoinAdapter@U2@@6B@ 10044b08     PhylipPlugin.obj
 0002:00002b18       ??_7PhylipPlugin@U2@@6B@   10044b18     PhylipPlugin.obj
 0002:00002b44       ??_C@_0BI@IDNFIBFF@PHYLIP?5Neighbor?5Joining?$AA@ 10044b44     PhylipPlugin.obj
 0002:00002b60       ??_C@_0LM@KABOLGED@PHYLIP?5?$CIthe?5PHYLogeny?5Inference?5@ 10044b60     PhylipPlugin.obj
 0002:00002c1c       ??_C@_06IDHMOABD@PHYLIP?$AA@ 10044c1c     PhylipPlugin.obj
 0002:00002c24       ??_C@_03PEIMBJDE@XML?$AA@  10044c24     PhylipPlugin.obj
 0002:00002c2c       ??_7?$GAutoDeleteList@VXMLTestFactory@U2@@@U2@@6B@ 10044c2c     PhylipPlugin.obj
 0002:00002c58       ??_C@_0BA@HIHHFANN@1registerTask?$CI?$CJ?$AA@ 10044c58     PhylipPlugin.obj
 0002:00002c68       ??_C@_0BO@OEDOLCDP@2si_allStartUpPluginsLoaded?$CI?$CJ?$AA@ 10044c68     PhylipPlugin.obj
 0002:00002c8c       ??_SPhyTreeGeneratorLauncherTask@U2@@6B@ 10044c8c     PhylipPluginTests.obj
 0002:00002d1c       ??_7GTest_NeighborJoinFactory@GTest_NeighborJoin@U2@@6B@ 10044d1c     PhylipPluginTests.obj
 0002:00002d28       ??_7GTest_NeighborJoin@U2@@6B@ 10044d28     PhylipPluginTests.obj
 0002:00002db4       ??_C@_0BD@BCEIMFKK@test?9neighbor?9join?$AA@ 10044db4     PhylipPluginTests.obj
 0002:00002dc8       ??_C@_02LMMGJAGL@in?$AA@   10044dc8     PhylipPluginTests.obj
 0002:00002dcc       ??_C@_06CPGBIIAO@sample?$AA@ 10044dcc     PhylipPluginTests.obj
 0002:00002dd4       ??_C@_0O@DKCIHFKC@bootstrapSeed?$AA@ 10044dd4     PhylipPluginTests.obj
 0002:00002de4       ??_C@_0BF@JDCOOOAG@context?5not?5found?5?$CF1?$AA@ 10044de4     PhylipPluginTests.obj
 0002:00002dfc       ??_C@_0CM@JHIEDKIP@container?5of?5object?5with?5type?5?$CC?$CF@ 10044dfc     PhylipPluginTests.obj
 0002:00002e28       ??_C@_0CA@IPABBKDH@object?5with?5type?5?$CC?$CF1?$CC?5not?5found?$AA@ 10044e28     PhylipPluginTests.obj
 0002:00002e48       ??_C@_0DE@OHFHLOPG@error?5can?8t?5cast?5to?5multiple?5ali@ 10044e48     PhylipPluginTests.obj
 0002:00002e7c       ??_C@_0DD@DDFOGEHA@error?5can?8t?5cast?5to?5phylogenetic@ 10044e7c     PhylipPluginTests.obj
 0002:00002eb0       ??_C@_0BE@NLFLJLFH@Result?5tree?5is?5NULL?$AA@ 10044eb0     PhylipPluginTests.obj
 0002:00002ec4       ??_C@_0BE@ILOBGFAE@Trees?5are?5not?5equal?$AA@ 10044ec4     PhylipPluginTests.obj
 0002:00002edc       ??_SMultipleSequenceAlignmentObject@U2@@6B@ 10044edc     PhylipTask.obj
 0002:00002f80       ??_7PhylipTask@U2@@6B@     10044f80     PhylipTask.obj
 0002:00003010       ??_C@_0M@OEKAEBOM@PHYLIP?5task?$AA@ 10045010     PhylipTask.obj
 0002:0000301c       ??_C@_03DNKGIDNC@msa?$AA@  1004501c     PhylipTask.obj
 0002:00003020       ??_C@_04GDOOJPNH@Tree?$AA@ 10045020     PhylipTask.obj
 0002:0000302c       ??_SMultipleSequenceAlignment@U2@@6B@ 1004502c     SeqBootAdapter.obj
 0002:00003030       ??_C@_0P@BMNIILAK@?1bootstrXXXXXX?$AA@ 10045030     SeqBootAdapter.obj
 0002:00003040       ??_C@_0N@DMNDMC@bootstrap?5?$CF1?$AA@ 10045040     SeqBootAdapter.obj
 0002:00003050       ??_C@_0CN@KHCEOAFG@?6?6ERROR?5in?5user?5tree?3?5duplicate?5@ 10045050     cons.obj
 0002:00003080       ??_C@_02PHMGELLB@?6?6?$AA@ 10045080     cons.obj
 0002:00003084       ??_C@_0CL@KPOBLNKP@?6?6ERROR?5in?5user?5tree?3?5name?5?$CFs?5no@ 10045084     cons.obj
 0002:000030b0       ??_C@_02JDPG@rb?$AA@       100450b0     cons.obj
 0002:000030b4       ??_C@_01EEMJAFIK@?6?$AA@   100450b4     cons.obj
 0002:000030b8       ??_C@_07JOENPDML@Done?4?6?6?$AA@ 100450b8     cons.obj
 0002:000030c0       ??_C@_03DLDNIBIK@?$CFlf?$AA@ 100450c0     cons.obj
 0002:000030c4       ??_C@_0CI@DMADLMMA@?6?6ERROR?3?5Missing?5right?5square?5br@ 100450c4     cons.obj
 0002:000030ec       ??_C@_0DD@FEDALPN@?6?6ERROR?3?5Missing?5semicolon?5after@ 100450ec     cons.obj
 0002:00003120       ??_C@_0DH@NKPKFNOJ@?6?6ERROR?3?5Expecting?5tree?5weight?5i@ 10045120     cons.obj
 0002:00003158       ??_C@_0CB@PEJCLGME@WARNING?3?5Tree?5weight?5set?5to?51?40?6@ 10045158     cons.obj
 0002:0000317c       ??_C@_0BL@LLDAJBDN@?6Set?5?$CIspecies?5in?5order?$CJ?5?5?5?$AA@ 1004517c     cons.obj
 0002:00003198       ??_C@_0CA@OLPECBOJ@?5?5How?5many?5times?5out?5of?5?$CF7?42f?6?6?$AA@ 10045198     cons.obj
 0002:000031b8       ??_C@_0L@HNGKFMJD@?5?5?5?5?$CF5?42f?6?$AA@ 100451b8     cons.obj
 0002:000031c4       ??_C@_06LFKKDFDG@?5NONE?6?$AA@ 100451c4     cons.obj
 0002:000031cc       ??_C@_02KNHHEEKP@?5?5?$AA@ 100451cc     cons.obj
 0002:000031d0       ??_C@_08MFHFMIIJ@?9?9?9?9?9?9?9?$HM?$AA@ 100451d0     cons.obj
 0002:000031dc       ??_C@_08BAFAPPDE@?9?$CF5?40f?9?$HM?$AA@ 100451dc     cons.obj
 0002:000031e8       ??_C@_09JAHAADI@?9?9?$CF4?40f?9?$HM?$AA@ 100451e8     cons.obj
 0002:000031f4       ??_C@_08CNDANGIE@?9?$CF5?41f?9?$HM?$AA@ 100451f4     cons.obj
 0002:00003200       ??_C@_09DEGHCJII@?9?9?$CF4?41f?9?$HM?$AA@ 10045200     cons.obj
 0002:0000320c       ??_C@_09HDMHFDFI@?9?9?$CF4?42f?9?$HM?$AA@ 1004520c     cons.obj
 0002:00003218       ??_C@_0BC@FEOFOLPL@?6CONSENSUS?5TREE?3?6?$AA@ 10045218     cons.obj
 0002:0000322c       ??_C@_0DB@BKNKEEID@the?5numbers?5on?5the?5branches?5indi@ 1004522c     cons.obj
 0002:00003260       ??_C@_0DJ@LJHILGGO@of?5times?5the?5partition?5of?5the?5sp@ 10045260     cons.obj
 0002:0000329c       ??_C@_0CN@JGFANDJH@which?5are?5separated?5by?5that?5bran@ 1004529c     cons.obj
 0002:000032cc       ??_C@_0CH@NHAJEHDP@the?5numbers?5forks?5indicate?5the?5n@ 100452cc     cons.obj
 0002:000032f4       ??_C@_0CO@OBJNPCAH@of?5times?5the?5group?5consisting?5of@ 100452f4     cons.obj
 0002:00003324       ??_C@_0CO@OFHAFCPJ@which?5are?5to?5the?5right?5of?5that?5f@ 10045324     cons.obj
 0002:00003354       ??_C@_0CF@IAAECBJM@among?5the?5trees?0?5out?5of?5?$CF6?42f?5tr@ 10045354     cons.obj
 0002:0000337c       ??_C@_0CA@HCAIJFGC@?$CItrees?5had?5fractional?5weights?$CJ?6?$AA@ 1004537c     cons.obj
 0002:0000339c       ??_C@_0N@LONJBMN@?6?5?5remember?3?$AA@ 1004539c     cons.obj
 0002:000033ac       ??_C@_0BP@HKLMNBFP@?5?$CIthough?5rerooted?5by?5outgroup?$CJ?$AA@ 100453ac     cons.obj
 0002:000033cc       ??_C@_0BM@PDLDMKDM@?5this?5is?5an?5unrooted?5tree?$CB?6?$AA@ 100453cc     cons.obj
 0002:000033e8       ??_C@_0CG@LEGIOKKC@?6Sets?5included?5in?5the?5consensus?5@ 100453e8     cons.obj
 0002:00003410       ??_C@_0CH@DGBKHIPD@?6?6Sets?5NOT?5included?5in?5consensus@ 10045410     cons.obj
 0002:00003438       ??_C@_0BI@LIEMNODC@?6Strict?5consensus?5tree?6?$AA@ 10045438     cons.obj
 0002:00003450       ??_C@_0CI@GABJMFNG@?6Extended?5majority?5rule?5consensu@ 10045450     cons.obj
 0002:00003478       ??_C@_0CA@LEGABDOP@?6M?5?5consensus?5tree?5?$CIl?5?$DN?5?$CF4?42f?$CJ?6?$AA@ 10045478     cons.obj
 0002:00003498       ??_C@_03MFKLFFBD@?5l?6?$AA@ 10045498     cons.obj
 0002:0000349c       ??_C@_0BP@LPOGEAPM@?6Majority?5rule?5consensus?5tree?6?$AA@ 1004549c     cons.obj
 0002:000034bc       ??_C@_0DJ@KOFICJFN@?6?6ERROR?5in?5user?5tree?3?5name?5?$CFs?5no@ 100454bc     cons.obj
 0002:000034f8       __real@3ff004189374bc6a    100454f8     cons.obj
 0002:00003500       __real@4014000000000000    10045500     cons.obj
 0002:00003508       __real@4024000000000000    10045508     cons.obj
 0002:00003510       __real@403f000000000000    10045510     cons.obj
 0002:00003518       __real@4059000000000000    10045518     cons.obj
 0002:00003520       __real@408f400000000000    10045520     cons.obj
 0002:00003528       __real@40c3880000000000    10045528     cons.obj
 0002:00003530       __real@bff0000000000000    10045530     cons.obj
 0002:00003538       ??_C@_03JALODAI@?$CFld?$AA@ 10045538     dist.obj
 0002:0000353c       ??_C@_0DG@DPIMKJJF@Species?5name?5may?5not?5contain?5cha@ 1004553c     dist.obj
 0002:00003574       ??_C@_0DI@ONKKLJKN@?6ERROR?3?5diagonal?5element?5of?5row?5@ 10045574     dist.obj
 0002:000035ac       ??_C@_0O@FNPNOJLJ@is?5not?5zero?4?6?$AA@ 100455ac     dist.obj
 0002:000035bc       ??_C@_0CC@PCIBNHCL@?5?5?5?5?5?5?5Is?5it?5a?5distance?5matrix?$DP?6@ 100455bc     dist.obj
 0002:000035e0       ??_C@_0CK@JNPHGJOI@ERROR?3?5distance?5matrix?5is?5not?5sy@ 100455e0     dist.obj
 0002:0000360c       ??_C@_0DN@FDAJLDBB@?5?5?5?5?5?5?5?$CI?$CFld?0?$CFld?$CJ?5element?5and?5?$CI?$CFl@ 1004560c     dist.obj
 0002:0000364c       ??_C@_0DC@OPIFJKII@?5?5?5?5?5?5?5They?5are?5?$CF10?46f?5and?5?$CF10?46@ 1004564c     dist.obj
 0002:00003680       ??_C@_0CB@DGDOKKPK@The?5infile?5is?5of?5the?5wrong?5type?6@ 10045680     dist.obj
 0002:000036a4       ??_C@_06MAPLGJGD@?$CF10?45f?$AA@ 100456a4     dist.obj
 0002:000036ac       ??_C@_07FEHBNHEE@?5?$CI?$CF3ld?$CJ?$AA@ 100456ac     dist.obj
 0002:000036b4       ??_C@_01JOAMLHOP@?9?$AA@   100456b4     dist.obj
 0002:000036b8       ??_C@_04CKICAEFL@?$CF2ld?$AA@ 100456b8     dist.obj
 0002:000036c0       ??_C@_04NHDMCALM@?9?$CFld?$AA@ 100456c0     dist.obj
 0002:000036c8       ??_C@_02NCGPMEBG@?$DL?6?$AA@ 100456c8     dist.obj
 0002:000036cc       ??_C@_02PIGFKFFE@?$CF1?$AA@ 100456cc     dist.obj
 0002:000036d0       ??_C@_03HLLJJGBI@?3?$CFs?$AA@ 100456d0     dist.obj
 0002:000036d8       __real@3e112e0be826d695    100456d8     dist.obj
 0002:000036e0       __real@404e000000000000    100456e0     dist.obj
 0002:000036e8       __real@bfdbcb7b157df63a    100456e8     dist.obj
 0002:000036f0       __xmm@80000000000000008000000000000000 100456f0     dist.obj
 0002:00003700       ??_C@_03PBJGGANN@F84?$AA@  10045700     dnadist.obj
 0002:00003704       ??_C@_06BNLEFKBK@Kimura?$AA@ 10045704     dnadist.obj
 0002:0000370c       ??_C@_0N@OEADEFO@Jukes?9Cantor?$AA@ 1004570c     dnadist.obj
 0002:0000371c       ??_C@_06CCLBFDAN@LogDet?$AA@ 1004571c     dnadist.obj
 0002:00003724       ??_C@_0BL@DLKEJFIP@?$CF2ld?5species?0?5?$CF3ld?5?5sites?6?$AA@ 10045724     dnadist.obj
 0002:00003740       ??_C@_0BC@IJMJLEGB@Rate?5categories?6?6?$AA@ 10045740     dnadist.obj
 0002:00003754       ??_C@_0BJ@NLAKNFDO@?5?5Jukes?9Cantor?5Distance?6?$AA@ 10045754     dnadist.obj
 0002:00003770       ??_C@_0BP@IMOFDPIJ@?5?5Kimura?52?9parameter?5Distance?6?$AA@ 10045770     dnadist.obj
 0002:00003790       ??_C@_0BA@NMKPKPPB@?5?5F84?5Distance?6?$AA@ 10045790     dnadist.obj
 0002:000037a0       ??_C@_0CM@EJBMBNON@?5?5?6?5?5Table?5of?5similarity?5between@ 100457a0     dnadist.obj
 0002:000037cc       ??_C@_0CJ@HKDOJHKK@?6Transition?1transversion?5ratio?5?$DN@ 100457cc     dnadist.obj
 0002:000037f8       ??_C@_07NJJCCLDN@DnaDist?$AA@ 100457f8     dnadist.obj
 0002:00003800       ??_C@_0BA@MEGBFABG@Site?5categories?$AA@ 10045800     dnadist.obj
 0002:00003810       ??_C@_0CC@BKKMDIKG@?6Site?5category?5?5?5Rate?5of?5change?6@ 10045810     dnadist.obj
 0002:00003834       ??_C@_0N@HMLCNDJO@?$CF12ld?$CF13?43f?6?$AA@ 10045834     dnadist.obj
 0002:00003844       ??_C@_0DA@PPNMHOFA@?5WARNING?3?5CANNOT?5USE?5EMPIRICAL?5B@ 10045844     dnadist.obj
 0002:00003874       ??_C@_0DJ@EFGBLJDO@?5WITH?5JUKES?9CANTOR?0?5KIMURA?0?5JIN?1@ 10045874     dnadist.obj
 0002:000038b0       ??_C@_05POFGCFAM@Sites?$AA@ 100458b0     dnadist.obj
 0002:000038b8       ??_C@_05IAKIMJKP@NX?$DPO?9?$AA@ 100458b8     dnadist.obj
 0002:000038c0       ??_C@_0EG@KNICEFA@?6WARNING?3?5NO?5OVERLAP?5BETWEEN?5SEQ@ 100458c0     dnadist.obj
 0002:00003908       ??_C@_0CM@PBAAEOPH@?5WARNING?3?5CANNOT?5CALCULATE?5LOGDE@ 10045908     dnadist.obj
 0002:00003934       ??_C@_0DL@POEJOOPL@?5?5WITH?5PRESENT?5PROGRAM?5IF?5PARTIA@ 10045934     dnadist.obj
 0002:00003970       ??_C@_0BE@DNKFFIOF@?5?5?91?40?5WAS?5WRITTEN?6?$AA@ 10045970     dnadist.obj
 0002:00003984       ??_C@_0CF@NHJKNKAG@?6WARNING?3?5INFINITE?5DISTANCE?5BETW@ 10045984     dnadist.obj
 0002:000039ac       ??_C@_0BI@LGAGBBIJ@?5SPECIES?5?$CF3ld?5AND?5?$CF3ld?6?$AA@ 100459ac     dnadist.obj
 0002:000039c4       ??_C@_0DD@FJCKEMLB@?6WARNING?3?5DIFFERENCE?5BETWEEN?5SPE@ 100459c4     dnadist.obj
 0002:000039f8       ??_C@_0CB@PPONBNBM@?5TOO?5LARGE?5FOR?5INVARIABLE?5SITES?6@ 100459f8     dnadist.obj
 0002:00003a1c       ??_C@_0CB@BHDNNGME@?5TOO?5LARGE?5TO?5ESTIMATE?5DISTANCE?6@ 10045a1c     dnadist.obj
 0002:00003a40       ??_C@_0DL@COMFGMBN@?6Negative?5or?5zero?5determinant?5fo@ 10045a40     dnadist.obj
 0002:00003a7c       ??_C@_0O@PELFOIPC@?5?$CFld?5and?5?$CFld?6?$AA@ 10045a7c     dnadist.obj
 0002:00003a8c       ??_C@_0DD@GCFEADBL@?6WARNING?3?5SPECIES?5?$CF3ld?5AND?5?$CF3ld?5@ 10045a8c     dnadist.obj
 0002:00003ac0       ??_C@_0BC@BAIDMPJL@?5CAN?5BE?5COMPARED?6?$AA@ 10045ac0     dnadist.obj
 0002:00003ad4       ??_C@_0CC@CACGNCAO@Distances?5calculated?5for?5species@ 10045ad4     dnadist.obj
 0002:00003af8       ??_C@_04PFOHOKJK@?5?5?5?5?$AA@ 10045af8     dnadist.obj
 0002:00003b00       ??_C@_03NDEAONJP@?5?5?5?$AA@ 10045b00     dnadist.obj
 0002:00003b04       ??_C@_0P@CAMMPPGD@Task?5canceled?$CB?$AA@ 10045b04     dnadist.obj
 0002:00003b14       ??_C@_0CC@MKKNAIEO@?6Distances?5written?5to?5file?5?$CC?$CFs?$CC?6@ 10045b14     dnadist.obj
 0002:00003b38       __real@3e45798ee2308c3a    10045b38     dnadist.obj
 0002:00003b40       __real@3e8ad7f29abcaf48    10045b40     dnadist.obj
 0002:00003b48       __real@3eb0c6f7a0b5ed8d    10045b48     dnadist.obj
 0002:00003b50       __real@3f800000            10045b50     dnadist.obj
 0002:00003b58       __real@3fd0000000000000    10045b58     dnadist.obj
 0002:00003b60       __real@3fe0000035afe535    10045b60     dnadist.obj
 0002:00003b68       __real@3fe8000000000000    10045b68     dnadist.obj
 0002:00003b70       __real@3feffffde7210be9    10045b70     dnadist.obj
 0002:00003b78       __real@4008000000000000    10045b78     dnadist.obj
 0002:00003b80       __real@4010000000000000    10045b80     dnadist.obj
 0002:00003b88       __real@4058c00000000000    10045b88     dnadist.obj
 0002:00003b90       __real@bfd0000000000000    10045b90     dnadist.obj
 0002:00003b98       __real@bfe0000000000000    10045b98     dnadist.obj
 0002:00003ba0       __real@bfe8000000000000    10045ba0     dnadist.obj
 0002:00003ba8       ??_C@_05NMNPGDGM@3?4697?$AA@ 10045ba8     neighbor.obj
 0002:00003bb0       ??_C@_0CM@OBCKLEBA@?6Neighbor?9Joining?1UPGMA?5method?5v@ 10045bb0     neighbor.obj
 0002:00003bdc       ??_C@_0BJ@GMAGHECB@Neighbor?9joining?5method?6?$AA@ 10045bdc     neighbor.obj
 0002:00003bf8       ??_C@_0P@CIGEDBFA@?$CF4ld?5?5?5?5?5?5?5?5?5?5?$AA@ 10045bf8     neighbor.obj
 0002:00003c08       ??_C@_09PFPHPEIP@?$CF4ld?5?5?5?5?5?$AA@ 10045c08     neighbor.obj
 0002:00003c14       ??_C@_0M@KLACCFDE@?$CF4ld?5?5?5?5?5?5?5?$AA@ 10045c14     neighbor.obj
 0002:00003c20       ??_C@_07GDFMICAK@?$CF12?45f?6?$AA@ 10045c20     neighbor.obj
 0002:00003c28       ??_C@_0BE@ENMNOLGG@?$CF10?45f?5?5?5?5?5?5?$CF10?45f?6?$AA@ 10045c28     neighbor.obj
 0002:00003c3c       ??_C@_09EDOBINDA@remember?3?$AA@ 10045c3c     neighbor.obj
 0002:00003c48       ??_C@_0BP@IOEBMAIN@?5?$CIalthough?5rooted?5by?5outgroup?$CJ?$AA@ 10045c48     neighbor.obj
 0002:00003c68       ??_C@_0CH@OBEAAHPB@?6Between?5?5?5?5?5?5?5?5And?5?5?5?5?5?5?5?5?5?5?5?5L@ 10045c68     neighbor.obj
 0002:00003c90       ??_C@_0CG@KIGMEDKF@?9?9?9?9?9?9?9?5?5?5?5?5?5?5?5?9?9?9?5?5?5?5?5?5?5?5?5?5?5?5?9?9@ 10045c90     neighbor.obj
 0002:00003cb8       ??_C@_0CP@LHNLHPLH@From?5?5?5?5?5To?5?5?5?5?5?5?5?5?5?5?5?5Length?5?5?5@ 10045cb8     neighbor.obj
 0002:00003ce8       ??_C@_0CP@PMAKMBCM@?9?9?9?9?5?5?5?5?5?9?9?5?5?5?5?5?5?5?5?5?5?5?5?9?9?9?9?9?9?5?5?5@ 10045ce8     neighbor.obj
 0002:00003d18       ??_C@_04CLMONKIF@node?$AA@ 10045d18     neighbor.obj
 0002:00003d20       ??_C@_07NOOBGOMN@species?$AA@ 10045d20     neighbor.obj
 0002:00003d28       ??_C@_0N@OPNFJAMD@Cycle?5?$CF3ld?3?5?$AA@ 10045d28     neighbor.obj
 0002:00003d38       ??_C@_0BF@EGGCBACH@?5?$CFld?5?$CI?$CF10?45f?$CJ?5joins?5?$AA@ 10045d38     neighbor.obj
 0002:00003d50       ??_C@_0P@CCBOHDMF@?5?$CFld?5?$CI?$CF10?45f?$CJ?6?$AA@ 10045d50     neighbor.obj
 0002:00003d60       ??_C@_0N@OHHLDDOJ@last?5cycle?3?6?$AA@ 10045d60     neighbor.obj
 0002:00003d70       ??_C@_0BG@NPDDIGKL@?5?$CFld?5?5?$CI?$CF10?45f?$CJ?5joins?5?$AA@ 10045d70     neighbor.obj
 0002:00003d88       ??_C@_0BA@LLEHKJNC@?5?$CFld?5?5?$CI?$CF10?45f?$CJ?6?$AA@ 10045d88     neighbor.obj
 0002:00003d98       ??_C@_0DN@GFNECHND@?6ERROR?3?5Neighbor?9Joining?5runs?5mu@ 10045d98     neighbor.obj
 0002:00003dd8       ??_C@_0BP@DLDIFOOF@?6Output?5written?5on?5file?5?$CC?$CFs?$CC?6?6?$AA@ 10045dd8     neighbor.obj
 0002:00003df8       ??_C@_0BM@IDLNDOLA@Tree?5written?5on?5file?5?$CC?$CFs?$CC?6?6?$AA@ 10045df8     neighbor.obj
 0002:00003e14       ??_C@_01MCMALHOG@a?$AA@    10045e14     neighbor.obj
 0002:00003e18       ??_C@_0BB@HKEPLOEN@Data?5set?5?$CD?5?$CFld?3?6?$AA@ 10045e18     neighbor.obj
 0002:00003e2c       ??_C@_08KADIPPKJ@ERROR?3?5?5?$AA@ 10045e2c     phylip.obj
 0002:00003e38       ??_C@_0CO@OMKCPIKI@This?5program?5has?5caused?5a?5Segmen@ 10045e38     phylip.obj
 0002:00003e68       ??_C@_0DD@FOIIIFKE@This?5program?5has?5caused?5a?5Floati@ 10045e68     phylip.obj
 0002:00003e9c       ??_C@_0DC@DDKKKPNH@This?5program?5has?5attempted?5an?5il@ 10045e9c     phylip.obj
 0002:00003ed0       ??_C@_0EI@LPDAGIFD@?5?5?5?5?5?5?5This?5may?5have?5been?5caused@ 10045ed0     phylip.obj
 0002:00003f18       ??_C@_0EE@NLEJOIGI@?5?5?5?5?5?5?5or?5input?5tree?5file?4?5?5You?5@ 10045f18     phylip.obj
 0002:00003f60       ??_C@_0EE@DMKDCAOO@?5?5?5?5?5?5?5If?5this?5seems?5to?5be?5a?5bug@ 10045f60     phylip.obj
 0002:00003fa4       ??_C@_0DP@NHFDKHHM@?5?5?5?5?5?5?5Most?5likely?0?5you?5have?5enc@ 10045fa4     phylip.obj
 0002:00003fe8       ??_C@_0EH@DADNGLOJ@?5?5?5?5?5?5?5Since?5this?5seems?5to?5be?5a?5@ 10045fe8     phylip.obj
 0002:00004030       ??_C@_0EA@FMHDJFJJ@?5?5?5?5?5?5?5with?5the?5name?5of?5the?5prog@ 10046030     phylip.obj
 0002:00004070       ??_C@_0EI@PHGKLKPB@?5?5?5?5?5?5?5a?5full?5description?5of?5the@ 10046070     phylip.obj
 0002:000040b8       ??_C@_0EL@FDNGMFCE@?5?5?5?5?5?5?5?$CIwhich?5should?5be?5in?5the?5b@ 100460b8     phylip.obj
 0002:00004104       ??_C@_01KDCPPGHE@r?$AA@    10046104     phylip.obj
 0002:00004108       ??_C@_0CC@JILFGELM@?6?6ERROR?3?5Unexpected?5end?9of?9file?4@ 10046108     phylip.obj
 0002:0000412c       ??_C@_02LIIHNNHG@?6?$AN?$AA@ 1004612c     phylip.obj
 0002:00004130       ??_C@_0EA@OLLJNIAP@?6ERROR?3?5Made?5?$CFld?5attempts?5to?5rea@ 10046130     phylip.obj
 0002:00004170       ??_C@_0CH@HKMPNMPP@?6?$CFs?3?5the?5file?5?$CC?$CFs?$CC?5that?5you?5want@ 10046170     phylip.obj
 0002:00004198       ??_C@_0CA@PKIOAILJ@?5?5?5?5?5use?5as?5?$CFs?5already?5exists?4?6?$AA@ 10046198     phylip.obj
 0002:000041b8       ??_C@_0CP@HBJICJPO@?5?5?5?5?5Do?5you?5want?5to?5Replace?5it?0?5@ 100461b8     phylip.obj
 0002:000041e8       ??_C@_0CE@KNCGEFEP@?5?5?5?5?5write?5to?5a?5new?5File?0?5or?5Qui@ 100461e8     phylip.obj
 0002:0000420c       ??_C@_0CD@BOCPGMMC@?5?5?5?5?5?$CIplease?5type?5R?0?5A?0?5F?0?5or?5Q?$CJ@ 1004620c     phylip.obj
 0002:00004230       ??_C@_0BP@JIHKKBDK@Please?5enter?5a?5new?5file?5name?$DO?5?$AA@ 10046230     phylip.obj
 0002:00004250       ??_C@_0BI@BJOBCOGM@?$CFs?3?5can?8t?5find?5?$CFs?5?$CC?$CFs?$CC?6?$AA@ 10046250     phylip.obj
 0002:00004268       ??_C@_0BJ@PIHLFKAA@?$CFs?3?5can?8t?5write?5?$CFs?5?$CC?$CFs?$CC?6?$AA@ 10046268     phylip.obj
 0002:00004284       ??_C@_0DM@EFDAKJPG@There?5is?5some?5error?5in?5the?5call?5@ 10046284     phylip.obj
 0002:000042c0       ??_C@_02DKCKIIND@?$CFs?$AA@ 100462c0     phylip.obj
 0002:000042c4       ??_C@_0CE@LHMHCLBK@?6Random?5number?5seed?5?$CImust?5be?5odd@ 100462c4     phylip.obj
 0002:000042e8       ??_C@_09GNGJDAD@?$CFld?$CF?$CK?$FL?$FO?6?$FN?$AA@ 100462e8     phylip.obj
 0002:000042f4       ??_C@_0BM@PEBGIFKG@Number?5of?5times?5to?5jumble?$DP?6?$AA@ 100462f4     phylip.obj
 0002:00004310       ??_C@_0BO@CIIEAAEG@Type?5number?5of?5the?5outgroup?3?6?$AA@ 10046310     phylip.obj
 0002:00004330       ??_C@_0BK@LALHOPOC@BAD?5OUTGROUP?5NUMBER?3?5?$CFld?6?$AA@ 10046330     phylip.obj
 0002:0000434c       ??_C@_0BM@JHKCIBLF@?5?5Must?5be?5in?5range?51?5?9?5?$CFld?6?$AA@ 1004634c     phylip.obj
 0002:00004368       ??_C@_0CD@KIHFOJCN@What?5will?5be?5the?5threshold?5value@ 10046368     phylip.obj
 0002:0000438c       ??_C@_09EEPDJEHO@?$CFlf?$CF?$CK?$FL?$FO?6?$FN?$AA@ 1004638c     phylip.obj
 0002:00004398       ??_C@_0DB@IGNCHDFO@BAD?5THRESHOLD?5VALUE?3?5?5it?5must?5be@ 10046398     phylip.obj
 0002:000043cc       ??_C@_0BO@OHBMJHMB@Number?5of?5categories?5?$CI1?9?$CFd?$CJ?$DP?6?$AA@ 100463cc     phylip.obj
 0002:000043ec       ??_C@_0DD@GOCHJLKP@Rate?5for?5each?5category?$DP?5?$CIuse?5a?5s@ 100463ec     phylip.obj
 0002:00004420       ??_C@_09OHJNAJAM@?$CFlf?5?$CF?$FL?$FO?6?$FN?$AA@ 10046420     phylip.obj
 0002:0000442c       ??_C@_0CC@BDPDIOPM@Please?5enter?5exactly?5?$CFld?5values?4@ 1004642c     phylip.obj
 0002:00004450       ??_C@_0BP@DJFKGKHN@Probability?5for?5each?5category?$DP?$AA@ 10046450     phylip.obj
 0002:00004470       ??_C@_0BM@HNAOECDD@?5?$CIuse?5a?5space?5to?5separate?$CJ?6?$AA@ 10046470     phylip.obj
 0002:0000448c       ??_C@_0BN@CMOGBDAL@Probabilities?5must?5add?5up?5to?$AA@ 1004648c     phylip.obj
 0002:000044ac       ??_C@_0BM@GLJDJCHL@?51?40?0?5plus?5or?5minus?50?4001?4?6?$AA@ 100464ac     phylip.obj
 0002:000044c8       ??_C@_0CA@DEAFGGCG@How?5many?5cycles?5of?5?$CF4ld?5trees?$DP?6?$AA@ 100464c8     phylip.obj
 0002:000044e8       ??_C@_0BL@HEIEFCOA@How?5many?5trees?5per?5cycle?$DP?6?$AA@ 100464e8     phylip.obj
 0002:00004508       ??_C@_0ED@INOMEIOO@Mean?5block?5length?5of?5sites?5havin@ 10046508     phylip.obj
 0002:0000454c       ??_C@_0DN@EOAEKBPE@Base?5frequencies?5for?5A?0?5C?0?5G?0?5T?1@ 1004654c     phylip.obj
 0002:0000458c       ??_C@_0BD@GPEGJEHC@?$CFlf?$CFlf?$CFlf?$CFlf?$CF?$CK?$FL?$FO?6?$FN?$AA@ 1004658c     phylip.obj
 0002:000045a0       ??_C@_0CA@IMHPKBM@Please?5enter?5exactly?54?5values?4?6?$AA@ 100465a0     phylip.obj
 0002:000045c0       ??_C@_0CA@JDKFMMOJ@Transition?1transversion?5ratio?$DP?6?$AA@ 100465c0     phylip.obj
 0002:000045e0       ??_C@_0DD@PHEEDGII@Transition?1transversion?5ratio?5ca@ 100465e0     phylip.obj
 0002:00004614       ??_C@_0M@GICKDBKO@New?5power?$DP?6?$AA@ 10046614     phylip.obj
 0002:00004620       ??_C@_0BF@CPMGEFDH@How?5many?5data?5sets?$DP?6?$AA@ 10046620     phylip.obj
 0002:00004638       ??_C@_0DC@GFKNLDPA@Bad?5data?5sets?5number?3?5?5it?5must?5b@ 10046638     phylip.obj
 0002:0000466c       ??_C@_0BL@JCDLFMPN@How?5many?5sets?5of?5weights?$DP?6?$AA@ 1004666c     phylip.obj
 0002:00004688       ??_C@_0CI@NEEDNEPO@BAD?5NUMBER?3?5?5it?5must?5be?5greater?5@ 10046688     phylip.obj
 0002:000046b0       ??_C@_0BM@LEBNKABL@Number?5of?5lines?5on?5screen?$DP?6?$AA@ 100466b0     phylip.obj
 0002:000046cc       ??_C@_06DLCCOLPN@?$CFld?$CFld?$AA@ 100466cc     phylip.obj
 0002:000046d8       ??_C@_0EH@PKOAAFLL@ERROR?3?5Unable?5to?5read?5the?5number@ 100466d8     phylip.obj
 0002:00004720       ??_C@_0ED@NGFECBJM@The?5input?5file?5is?5incorrect?5?$CIper@ 10046720     phylip.obj
 0002:00004764       ??_C@_0DJ@PMBOJNCI@ERROR?3?5Unable?5to?5read?5the?5number@ 10046764     phylip.obj
 0002:000047a0       ??_C@_0BD@HAOGIAFL@?6?$CF4ld?5Populations?6?$AA@ 100467a0     phylip.obj
 0002:000047b4       ??_C@_0DK@NGCKPFGL@?6?6ERROR?3?5Inconsistent?5number?5of?5@ 100467b4     phylip.obj
 0002:000047f0       ??_C@_0DP@KFLLFMOF@Unable?5to?5read?5number?5of?5species@ 100467f0     phylip.obj
 0002:00004830       ??_C@_0DL@DECKFLJA@?6?6ERROR?3?5Unable?5to?5read?5number?5o@ 10046830     phylip.obj
 0002:0000486c       ??_C@_0BK@PGLBCKLJ@BAD?5OPTION?5CHARACTER?3?5?$CFc?6?$AA@ 1004686c     phylip.obj
 0002:00004888       ??_C@_0CI@KCDMJDOE@ERROR?3?5Incorrect?5auxiliary?5optio@ 10046888     phylip.obj
 0002:000048b0       ??_C@_0BH@HJFFDFMG@?5which?5starts?5with?5?$CFc?6?$AA@ 100468b0     phylip.obj
 0002:000048c8       ??_C@_0CE@LKCKFJD@?6?6ERROR?3?5Bad?5weight?5character?3?5?$CF@ 100468c8     phylip.obj
 0002:000048ec       ??_C@_0CG@OPFFNECP@?6?6ERROR?3?5Bad?5weight?5character?3?5?$CF@ 100468ec     phylip.obj
 0002:00004914       ??_C@_0BO@NHDGOMLN@weights?5in?5?$CFs?5must?5be?50?5or?51?6?$AA@ 10046914     phylip.obj
 0002:00004934       ??_C@_0CB@CIJMBFPE@?6?5?5?5?5?$CFs?5are?5weighted?5as?5follows?3@ 10046934     phylip.obj
 0002:00004958       ??_C@_0BJ@NBINBLNN@?5?$CIA?5?$DN?510?0?5B?5?$DN?511?0?5etc?4?$CJ?6?$AA@ 10046958     phylip.obj
 0002:00004974       ??_C@_02HAOIJKIC@?$CFc?$AA@ 10046974     phylip.obj
 0002:00004978       ??_C@_0CE@GKKICOCL@?6?6ERROR?3?5Bad?5category?5character?3@ 10046978     phylip.obj
 0002:0000499c       ??_C@_0CK@OONKFEKJ@?5?9?9?5categories?5in?5?$CFs?5are?5current@ 1004699c     phylip.obj
 0002:000049c8       ??_C@_0O@CEKIMIAH@?6?5?5?5?5?$CFs?5are?3?6?$AA@ 100469c8     phylip.obj
 0002:000049d8       ??_C@_0N@FJFCGLJK@Factors?$CFs?3?6?6?$AA@ 100469d8     phylip.obj
 0002:000049e8       ??_C@_04FABLJDN@Name?$AA@  100469e8     phylip.obj
 0002:000049f0       ??_C@_03OFAPEBGM@?$CFs?6?$AA@ 100469f0     phylip.obj
 0002:000049f4       ??_C@_04ECGLBLOI@?9?9?9?9?$AA@ 100469f4     phylip.obj
 0002:000049fc       ??_C@_04LOAOMKLI@?$CFs?6?6?$AA@ 100469fc     phylip.obj
 0002:00004a04       ??_C@_0CE@HIOPDILM@?6?6ERROR?3?5end?9of?9line?5or?5end?9of?9f@ 10046a04     phylip.obj
 0002:00004a28       ??_C@_0DB@OHGBKCMM@?5in?5the?5middle?5of?5species?5name?5f@ 10046a28     phylip.obj
 0002:00004a60       ??_C@_0EA@FGPNPHMP@?6ERROR?3?5Species?5name?5may?5not?5con@ 10046a60     phylip.obj
 0002:00004aa0       ??_C@_0DN@JGNONKHC@?5?5?5?5?5?5?5In?5name?5of?5species?5number@ 10046aa0     phylip.obj
 0002:00004ae0       ??_C@_0ED@NGNPODD@?6?6ERROR?5in?5user?5tree?5?$CFld?3?5unmatc@ 10046ae0     phylip.obj
 0002:00004b24       ??_C@_0BL@ICMFJFAL@?6?6ERROR?5in?5user?5tree?5?$CFld?3?5?$AA@ 10046b24     phylip.obj
 0002:00004b40       ??_C@_0CP@HOAOOEPD@unmatched?5parenthesis?5or?5non?9bif@ 10046b40     phylip.obj
 0002:00004b70       ??_C@_0CN@KJGFOJNI@unmatched?5parenthesis?5or?5missing@ 10046b70     phylip.obj
 0002:00004ba0       ??_C@_0BH@MKGGKFJK@?6?6ERROR?5in?5user?5tree?3?5?$AA@ 10046ba0     phylip.obj
 0002:00004bb8       ??_C@_0CF@GKHKIKHM@unmatched?5parenthesis?0?5missing?5c@ 10046bb8     phylip.obj
 0002:00004be0       ??_C@_0BL@MKEDCDGA@?5or?5non?9trifurcated?5base?6?6?$AA@ 10046be0     phylip.obj
 0002:00004c00       ??_C@_0EF@EIBCPLAB@?6?6ERROR?5in?5user?5tree?3?5unmatched?5@ 10046c00     phylip.obj
 0002:00004c48       ??_C@_0DN@EBNHEKHE@?6?6ERROR?3?5Branch?5length?5found?5wit@ 10046c48     phylip.obj
 0002:00004c88       ??_C@_0EA@FAJDBLOJ@?6?6ERROR?3?5Branch?5length?5found?5wit@ 10046c88     phylip.obj
 0002:00004cc8       ??_C@_0EA@MBPCMLHA@?6?6ERROR?3?5Branch?5length?5found?5wit@ 10046cc8     phylip.obj
 0002:00004d08       ??_C@_0DN@BIBHICHC@?6?6ERROR?3?5Branch?5length?5found?5wit@ 10046d08     phylip.obj
 0002:00004d48       ??_C@_07DDBBJEKI@?5?$CF3ld?4?5?$AA@ 10046d48     phylip.obj
 0002:00004d50       ??_C@_0BI@OOBIPLKB@Error?5allocating?5memory?$AA@ 10046d50     phylip.obj
 0002:00004d68       ??_C@_0DO@NELOCBHN@ERROR?3?5a?5function?5asked?5for?5an?5i@ 10046d68     phylip.obj
 0002:00004da8       ??_C@_0EB@MKAHKHBL@Error?3?5the?5function?5count_sibs?5c@ 10046da8     phylip.obj
 0002:00004dec       ??_C@_0CI@OGGAAFFN@Error?3?5a?5loop?5of?5nodes?5was?5not?5c@ 10046dec     phylip.obj
 0002:00004e14       ??_C@_0CG@FHABMLPG@?6?6ERROR?3?5Unmatched?5comment?5brack@ 10046e14     phylip.obj
 0002:00004e3c       ??_C@_0CJ@LCCFCHDO@?6?6ERROR?3?5Could?5not?5save?5file?5pos@ 10046e3c     phylip.obj
 0002:00004e68       ??_C@_0CO@IOIJPAEF@Error?5reading?5number?5of?5trees?5in@ 10046e68     phylip.obj
 0002:00004e98       ??_C@_0BG@OPGLMEDM@Error?5in?5Link_Trees?$CI?$CJ?$AA@ 10046e98     phylip.obj
 0002:00004eb0       ??_C@_05GOIMHGEP@?3?0?$CJ?$FL?$DL?$AA@ 10046eb0     phylip.obj
 0002:00004eb8       ??_C@_0BP@KANBLONM@?6?6ERROR?3?5Cannot?5find?5species?3?5?$AA@ 10046eb8     phylip.obj
 0002:00004ed8       ??_C@_0BA@FDBCBHLH@?5in?5data?5file?6?6?$AA@ 10046ed8     phylip.obj
 0002:00004ee8       ??_C@_0DG@GMDFKNJB@ERROR?5in?5input?5tree?5file?3?5Attemp@ 10046ee8     phylip.obj
 0002:00004f20       ??_C@_0DH@LFGJMNE@many?5nodes?4?5This?5is?5usually?5caus@ 10046f20     phylip.obj
 0002:00004f58       ??_C@_0DI@GGFNEOEB@To?5use?5this?5tree?5with?5this?5progr@ 10046f58     phylip.obj
 0002:00004f90       ??_C@_0BG@KFFKJPDJ@and?5write?5this?5tree?4?6?$AA@ 10046f90     phylip.obj
 0002:00004fa8       ??_C@_0DK@LLMMCCPG@ERROR?5in?5input?5tree?5file?3?5A?5Unif@ 10046fa8     phylip.obj
 0002:00004fe4       ??_C@_0DK@GDJGHHAP@To?5use?5this?5tree?5with?5this?5progr@ 10046fe4     phylip.obj
 0002:00005020       ??_C@_0BC@CPODJHEK@?5write?5this?5tree?6?$AA@ 10047020     phylip.obj
 0002:00005034       ??_C@_0CO@LICJHEHG@?6?6ERROR?5in?5tree?5file?3?5unmatched?5@ 10047034     phylip.obj
 0002:00005064       ??_C@_0DN@GAGBCMIB@ERROR?5in?5intree?5file?3?5Attempting@ 10047064     phylip.obj
 0002:000050a4       ??_C@_0DI@BIOGIJKN@This?5is?5usually?5caused?5by?5a?5unif@ 100470a4     phylip.obj
 0002:000050dc       ??_C@_0DI@JGMCGNBL@intree?5with?5this?5program?5?5use?5re@ 100470dc     phylip.obj
 0002:00005114       ??_C@_0M@JPAAGCAE@this?5tree?4?6?$AA@ 10047114     phylip.obj
 0002:00005120       ??_C@_0DE@IJGCMGNM@ERROR?5in?5intree?5file?3?5A?5Unifurca@ 10047120     phylip.obj
 0002:00005154       ??_C@_0DM@DLNJLKND@To?5use?5this?5intree?5with?5this?5pro@ 10047154     phylip.obj
 0002:00005190       ??_C@_0DI@MLDHAGC@?6?6ERROR?3?5Expecting?5tree?5weight?5i@ 10047190     phylip.obj
 0002:000051c8       ??_C@_0CB@KEEEILO@WARNING?3?5tree?5weight?5set?5to?51?40?6@ 100471c8     phylip.obj
 0002:000051ec       ??_C@_0CP@JFJBKIFN@?6?6ERROR?5in?5tree?5file?3?5?5unmatched@ 100471ec     phylip.obj
 0002:0000521c       ??_C@_0BG@EECHAHHP@Press?5enter?5to?5quit?4?6?$AA@ 1004721c     phylip.obj
 0002:00005234       ??_C@_06CAPHAKMM@?$CF?$CF?4?$CFuf?$AA@ 10047234     phylip.obj
 0002:0000523c       ??_C@_05KJLIPHKF@?$CF5lu?6?$AA@ 1004723c     phylip.obj
 0002:00005244       ??_C@_05MBIBHAHC@?$CF?$CK?46f?$AA@ 10047244     phylip.obj
 0002:00005250       __real@3ee4f8b588e368f1    10047250     phylip.obj
 0002:00005258       __real@3f50624dd2f1a9fc    10047258     phylip.obj
 0002:00005260       __real@3f90000000000000    10047260     phylip.obj
 0002:00005268       __real@3fe62e42fefa3857    10047268     phylip.obj
 0002:00005270       __real@3fe62e42fefa39ef    10047270     phylip.obj
 0002:00005278       __real@3ff6a09e667f3bcd    10047278     phylip.obj
 0002:00005280       __real@3ffcab0bfa2a2002    10047280     phylip.obj
 0002:00005288       __real@40096ca77c922cf9    10047288     phylip.obj
 0002:00005290       __real@401326643c4479c9    10047290     phylip.obj
 0002:00005298       __real@4018000000000000    10047298     phylip.obj
 0002:000052a0       __real@401a51273acf01ca    100472a0     phylip.obj
 0002:000052a8       __real@40210ce1f32dcc30    100472a8     phylip.obj
 0002:000052b0       __real@4025358e82fcb70d    100472b0     phylip.obj
 0002:000052b8       __real@40299a8921a7f7cf    100472b8     phylip.obj
 0002:000052c0       __real@402e357590954d15    100472c0     phylip.obj
 0002:000052c8       __real@403180973f3a8d74    100472c8     phylip.obj
 0002:000052d0       __real@4033fcba16d50143    100472d0     phylip.obj
 0002:000052d8       __real@40f86a0000000000    100472d8     phylip.obj
 0002:000052e0       __xmm@0000000600000016000000180000000d 100472e0     phylip.obj
 0002:000052f0       __xmm@3ff00000000000003ff0000000000000 100472f0     phylip.obj
 0002:00005300       ??_C@_0BG@EFEGLLGD@Jones?9Taylor?9Thornton?$AA@ 10047300     protdist.obj
 0002:00005318       ??_C@_0BF@PPCHFICL@Henikoff?1Tillier?5PMB?$AA@ 10047318     protdist.obj
 0002:00005330       ??_C@_0M@MKLBKAJP@Dayhoff?5PAM?$AA@ 10047330     protdist.obj
 0002:0000533c       ??_C@_0CA@CBOBJFGD@?$CF2ld?5species?0?5?$CF3ld?5?5positions?6?6?$AA@ 1004733c     protdist.obj
 0002:0000535c       ??_C@_0CK@CLJKOOEK@?6Protein?5distance?5algorithm?0?5ver@ 1004735c     protdist.obj
 0002:00005388       ??_C@_0DG@FJCKIBAP@THIS?5TRANSITION?9TRANSVERSION?5RAT@ 10047388     protdist.obj
 0002:000053c0       ??_C@_0BJ@MLFLADFJ@?5THESE?5BASE?5FREQUENCIES?6?$AA@ 100473c0     protdist.obj
 0002:000053dc       ??_C@_0CI@DOMKEIDH@?5?5Jones?9Taylor?9Thornton?5model?5di@ 100473dc     protdist.obj
 0002:00005404       ??_C@_0CH@KFGAPCIC@?5?5Henikoff?1Tillier?5PMB?5model?5dis@ 10047404     protdist.obj
 0002:0000542c       ??_C@_0BO@JIKFCOGG@?5?5Dayhoff?5PAM?5model?5distance?6?$AA@ 1004742c     protdist.obj
 0002:0000544c       ??_C@_0BL@INNKLMNL@?5?5Kimura?5protein?5distance?6?$AA@ 1004744c     protdist.obj
 0002:00005468       ??_C@_0BN@PMFMMIOD@?5?5Categories?5model?5distance?6?$AA@ 10047468     protdist.obj
 0002:00005488       ??_C@_08JOCFGDOK@ProtDist?$AA@ 10047488     protdist.obj
 0002:00005494       ??_C@_0BE@MPBKCGNM@Position?5categories?$AA@ 10047494     protdist.obj
 0002:000054a8       ??_C@_09DLMFLBFA@Positions?$AA@ 100474a8     protdist.obj
 0002:000054b4       ??_C@_05NDHKMMOF@?6Name?$AA@ 100474b4     protdist.obj
 0002:000054bc       ??_C@_0L@NEMAELCH@Sequences?6?$AA@ 100474bc     protdist.obj
 0002:000054c8       ??_C@_0M@GNPLAEPL@?9?9?9?9?9?9?9?9?9?6?6?$AA@ 100474c8     protdist.obj
 0002:000054d4       ??_C@_0DN@NGPNLHFN@ERROR?5?9?9?5bad?5amino?5acid?3?5?$CFc?5at?5p@ 100474d4     protdist.obj
 0002:00005514       ??_C@_0DJ@PNHGBFDG@?5?5?5?5?5?5?5?5?5Periods?5?$CI?4?$CJ?5may?5not?5be?5@ 10047514     protdist.obj
 0002:00005550       ??_C@_0CL@FHEEFNFH@?5?5?5?5?5?5?5?5?5The?5correct?5gap?5charact@ 10047550     protdist.obj
 0002:0000557c       ??_C@_0CD@GJFMOCNL@ERROR?3?5SEQUENCES?5OUT?5OF?5ALIGNMEN@ 1004757c     protdist.obj
 0002:000055a0       ??_C@_0EL@JLMIOJOJ@?6WARNING?3?5INFINITE?5DISTANCE?5BETW@ 100475a0     protdist.obj
 0002:000055f0       ??_C@_0EL@FAJDBEFE@?6DISTANCE?5BETWEEN?5SEQUENCES?5?$CF3ld@ 100475f0     protdist.obj
 0002:00005640       __real@3fc999999999999a    10047640     protdist.obj
 0002:00005648       __real@3fdd3f7ced916873    10047648     protdist.obj
 0002:00005650       __real@bf1a36e2eb1c432d    10047650     protdist.obj
 0002:00005660       __xmm@00000001000000010000000100000001 10047660     protdist.obj
 0002:00005670       __xmm@00000001000000010000001900000019 10047670     protdist.obj
 0002:00005680       __xmm@00000005000000050000000800000008 10047680     protdist.obj
 0002:00005690       __xmm@00000006000000060000000300000003 10047690     protdist.obj
 0002:000056a0       __xmm@00000007000000070000000700000007 100476a0     protdist.obj
 0002:000056b0       __xmm@0000000a0000000a0000000a0000000a 100476b0     protdist.obj
 0002:000056c0       __xmm@0000000a0000000a0000000d0000000d 100476c0     protdist.obj
 0002:000056d0       __xmm@0000000b0000000b0000000200000002 100476d0     protdist.obj
 0002:000056e0       __xmm@0000000c000000090000000900000009 100476e0     protdist.obj
 0002:000056f0       __xmm@0000000e0000000e0000000e0000000e 100476f0     protdist.obj
 0002:00005700       __xmm@00000011000000110000001100000011 10047700     protdist.obj
 0002:00005710       __xmm@00000012000000160000000400000004 10047710     protdist.obj
 0002:00005720       __xmm@00000014000000140000001400000014 10047720     protdist.obj
 0002:00005730       __xmm@00000016000000160000001300000013 10047730     protdist.obj
 0002:00005740       __xmm@00000019000000190000001900000019 10047740     protdist.obj
 0002:00005750       ??_C@_09NJPFFACE@?9?9?9?9?9?9?9?9?9?$AA@ 10047750     seq.obj
 0002:0000575c       ??_C@_09JLKOCMHN@Sequences?$AA@ 1004775c     seq.obj
 0002:00005768       ??_C@_0BF@BKHEHHFO@ABCDGHKMNRSTUVWXY?$DPO?9?$AA@ 10047768     seq.obj
 0002:00005780       ??_C@_0DC@FLJJIDGI@ERROR?3?5bad?5base?3?5?$CFc?5at?5site?5?$CF5ld@ 10047780     seq.obj
 0002:000057b4       ??_C@_0DH@JGGEDPAL@?5?5?5?5?5?5?5Periods?5?$CI?4?$CJ?5may?5not?5be?5us@ 100477b4     seq.obj
 0002:000057ec       ??_C@_0CJ@GIGPFGDN@?5?5?5?5?5?5?5The?5correct?5gap?5character@ 100477ec     seq.obj
 0002:00005818       ??_C@_0DD@KBBBPGLL@?6ERROR?3?5sequences?5out?5of?5alignme@ 10047818     seq.obj
 0002:0000584c       ??_C@_0BC@FJBGHAOA@?5of?5species?5?$CFld?6?6?$AA@ 1004784c     seq.obj
 0002:00005860       ??_C@_0L@PFDEBILG@Empirical?5?$AA@ 10047860     seq.obj
 0002:0000586c       ??_C@_0BE@KNCOOJFK@Base?5Frequencies?3?6?6?$AA@ 1004786c     seq.obj
 0002:00005880       ??_C@_0BA@MGIJBHHE@?5?5?5A?5?5?5?5?$CF10?45f?6?$AA@ 10047880     seq.obj
 0002:00005890       ??_C@_0BA@KGNFKCDP@?5?5?5C?5?5?5?5?$CF10?45f?6?$AA@ 10047890     seq.obj
 0002:000058a0       ??_C@_0BA@GGGMMIKJ@?5?5?5G?5?5?5?5?$CF10?45f?6?$AA@ 100478a0     seq.obj
 0002:000058b0       ??_C@_0BA@HLIIDDPN@?5?5T?$CIU?$CJ?5?5?$CF10?45f?6?$AA@ 100478b0     seq.obj
 0002:000058c0       ??_C@_0CP@OMLKAHJG@?6?5WARNING?3?5This?5transition?1trans@ 100478c0     seq.obj
 0002:000058f0       ??_C@_0CN@IPAFLGHK@?5is?5impossible?5with?5these?5base?5f@ 100478f0     seq.obj
 0002:00005920       ??_C@_0CK@GOBGAPED@?5Transition?1transversion?5paramet@ 10047920     seq.obj
 0002:0000594c       ??_C@_0CP@IMJDJJNA@?5?5so?5transition?1transversion?5rat@ 1004794c     seq.obj
 0002:0000597c       ??_C@_07GHIAJMBC@?5?5?5?5?5?5?5?$AA@ 1004797c     seq.obj
 0002:00005984       ??_C@_07PBFNLMIL@root?5?5?5?$AA@ 10047984     seq.obj
 0002:0000598c       ??_C@_07GJBIBODF@?$CF4ld?5?5?5?$AA@ 1004798c     seq.obj
 0002:00005994       ??_C@_0L@OIHGENOH@?$CF4ld?5?5?5?5?5?5?$AA@ 10047994     seq.obj
 0002:000059a0       ??_C@_0L@CCBFPMDD@?5?5?5?5?5?5?5?5?5?5?$AA@ 100479a0     seq.obj
 0002:000059ac       ??_C@_0L@PEFFDEFJ@?5?5?5yes?5?5?5?5?$AA@ 100479ac     seq.obj
 0002:000059b8       ??_C@_0L@IMDBAKCK@?5?5maybe?5?5?5?$AA@ 100479b8     seq.obj
 0002:000059c4       ??_C@_0L@KMEBCJHM@?5?5?5no?5?5?5?5?5?$AA@ 100479c4     seq.obj
 0002:000059d0       ??_C@_0DD@HGMNKPEM@?6From?5?5?5?5To?5?5?5?5?5Any?5Steps?$DP?5?5?5?5St@ 100479d0     seq.obj
 0002:00005a04       ??_C@_0BN@HEKDNLMP@?5?5?5?5?5?5?5?5?5?5?5?5?5?5?5?5?5?5?5?5?5?5?5?5?5?5?5?5?$AA@ 10047a04     seq.obj
 0002:00005a24       ??_C@_0DC@INGNMJCB@?5?$CI?5?4?5means?5same?5as?5in?5the?5node?5b@ 10047a24     seq.obj
 0002:00005a58       ??_C@_0L@OMIDJNNK@?$CF6ld?5?5?5?5?5?5?$AA@ 10047a58     seq.obj
 0002:00005a64       ??_C@_08IBHLPPOC@?$CF6ld?5?5?5?5?$AA@ 10047a64     seq.obj
 0002:00005a70       ??_C@_06EKBKDDDL@?5?5?5?$CFf?6?$AA@ 10047a70     seq.obj
 0002:00005a78       ??_C@_05FKMOFHND@?5?$CF2ld?$AA@ 10047a78     seq.obj
 0002:00005a80       ??_C@_05FPOALHIF@?5?5?$CFld?$AA@ 10047a80     seq.obj
 0002:00005a88       ??_C@_0BN@NFHDCHMH@?5this?5is?5an?5unrooted?5tree?$CB?6?6?$AA@ 10047a88     seq.obj
 0002:00005aa8       ??_C@_09KBPGIPCP@weighted?5?$AA@ 10047aa8     seq.obj
 0002:00005ab4       ??_C@_0BF@DEHICNAI@steps?5in?5each?5site?3?6?$AA@ 10047ab4     seq.obj
 0002:00005acc       ??_C@_06GGLIPOFD@?5?5?5?5?5?5?$AA@ 10047acc     seq.obj
 0002:00005ad4       ??_C@_04POJFLIH@?$CF4ld?$AA@ 10047ad4     seq.obj
 0002:00005adc       ??_C@_0CM@OGHCGHIO@?6?5?5?5?5?5?$CK?9?9?9?9?9?9?9?9?9?9?9?9?9?9?9?9?9?9?9?9?9?9?9?9?9@ 10047adc     seq.obj
 0002:00005b08       ??_C@_06NGLIMPFK@?9?9?9?9?9?6?$AA@ 10047b08     seq.obj
 0002:00005b10       ??_C@_04LHFFDMOC@?$CF5ld?$AA@ 10047b10     seq.obj
 0002:00005b18       ??_C@_04LPCFPIML@?5?5?50?$AA@ 10047b18     seq.obj
 0002:00005b20       ??_C@_09CLOIMHDD@?$FL?$CF6?44f?$FN?$DL?6?$AA@ 10047b20     seq.obj
 0002:00005b2c       ??_C@_06ODHKEKOK@?3?$CF?$CK?45f?$AA@ 10047b2c     seq.obj
 0002:00005b34       ??_C@_0CC@KDAHFODD@Kishino?9Hasegawa?9Templeton?5test?6@ 10047b34     seq.obj
 0002:00005b58       ??_C@_0CG@HFMAFGEG@Tree?5?5?5?5Steps?5?5?5Diff?5Steps?5?5?5Its@ 10047b58     seq.obj
 0002:00005b80       ??_C@_0BK@CJEHBLKJ@?5?5?5Significantly?5worse?$DP?6?6?$AA@ 10047b80     seq.obj
 0002:00005b9c       ??_C@_0L@KLOAGJHC@?$CF3ld?$CF10?41f?$AA@ 10047b9c     seq.obj
 0002:00005ba8       ??_C@_0BA@JCPJMFAK@?5?5?$DM?9?9?9?9?9?9?5best?6?$AA@ 10047ba8     seq.obj
 0002:00005bb8       ??_C@_0N@FOAMEOJH@?$CF10?41f?$CF12?44f?$AA@ 10047bb8     seq.obj
 0002:00005bc8       ??_C@_0BA@FGBNNMM@?5?5?5?5?5?5?5?5?5?5?5Yes?6?$AA@ 10047bc8     seq.obj
 0002:00005bd8       ??_C@_0P@LPPLBOJG@?5?5?5?5?5?5?5?5?5?5?5No?6?$AA@ 10047bd8     seq.obj
 0002:00005be8       ??_C@_0DE@MHBOCCI@Shimodaira?9Hasegawa?5test?5on?5firs@ 10047be8     seq.obj
 0002:00005c1c       ??_C@_0BL@NPFDKIL@Shimodaira?9Hasegawa?5test?6?6?$AA@ 10047c1c     seq.obj
 0002:00005c38       ??_C@_0CF@LDCNOMKG@Tree?5?5?5?5Steps?5?5?5Diff?5Steps?5?5?5P?5v@ 10047c38     seq.obj
 0002:00005c60       ??_C@_0P@HALNAOFM@?5?$CF9?41f?5?5?$CF10?43f?$AA@ 10047c60     seq.obj
 0002:00005c70       ??_C@_0CG@OEDPFPNN@Tree?5?5?5?5logL?5?5?5?5Diff?5logL?5?5?5?5Its@ 10047c70     seq.obj
 0002:00005c98       ??_C@_0L@GMIPGECJ@?$CF3ld?5?$CF9?41f?$AA@ 10047c98     seq.obj
 0002:00005ca4       ??_C@_0O@LCFLEPOJ@?$CF10?41f?5?$CF11?44f?$AA@ 10047ca4     seq.obj
 0002:00005cb4       ??_C@_0CF@CIEIOAOI@Tree?5?5?5?5logL?5?5?5?5Diff?5logL?5?5?5?5P?5v@ 10047cb4     seq.obj
 0002:00005cdc       ??_C@_0BK@BHJEINFC@Collapsing?5best?5trees?6?5?5?5?$AA@ 10047cdc     seq.obj
 0002:00005cf8       __real@3d719799812dea11    10047cf8     seq.obj
 0002:00005d00       __real@3fa999999999999a    10047d00     seq.obj
 0002:00005d08       __real@3ff8000000000000    10047d08     seq.obj
 0002:00005d10       __real@3fff5bff04577d95    10047d10     seq.obj
 0002:00005d18       __real@c12e847e00000000    10047d18     seq.obj
 0002:00005d20       ??_C@_07CJJNPIFE@seqboot?$AA@ 10047d20     seqboot.obj
 0002:00005d28       ??_C@_0BL@DJBGLKEM@?5?$CIleast?5significant?5digit?$CJ?$AA@ 10047d28     seqboot.obj
 0002:00005d44       ??_C@_0CI@JCLMMHKN@?6Bootstrapping?5algorithm?0?5versio@ 10047d44     seqboot.obj
 0002:00005d6c       ??_C@_0CG@CHOFJOCB@Block?9bootstrap?5with?5block?5size?5@ 10047d6c     seqboot.obj
 0002:00005d94       ??_C@_0DI@JBFAIGIO@Partial?5?$CI?$CF2?40f?$CF?$CF?$CJ?5block?9bootstra@ 10047d94     seqboot.obj
 0002:00005dcc       ??_C@_0M@FCPKOCJJ@Bootstrap?6?6?$AA@ 10047dcc     seqboot.obj
 0002:00005dd8       ??_C@_0BO@MGNLKEOK@Partial?5?$CI?$CF2?40f?$CF?$CF?$CJ?5bootstrap?6?6?$AA@ 10047dd8     seqboot.obj
 0002:00005df8       ??_C@_0BI@EFIGNICB@Delete?9half?5Jackknife?6?6?$AA@ 10047df8     seqboot.obj
 0002:00005e10       ??_C@_0BL@GBGCNOPG@Delete?9?$CF2?40f?$CF?$CF?5Jackknife?6?6?$AA@ 10047e10     seqboot.obj
 0002:00005e2c       ??_C@_0CL@FOPMFGGG@Species?5order?5permuted?5separatel@ 10047e2c     seqboot.obj
 0002:00005e58       ??_C@_08FABNJAGP@?5locus?6?6?$AA@ 10047e58     seqboot.obj
 0002:00005e64       ??_C@_07GGACPKIG@?5site?6?6?$AA@ 10047e64     seqboot.obj
 0002:00005e6c       ??_C@_0N@EHGOPLOM@?5character?6?6?$AA@ 10047e6c     seqboot.obj
 0002:00005e7c       ??_C@_05FCHOKMLE@Locus?$AA@ 10047e7c     seqboot.obj
 0002:00005e84       ??_C@_04ELDCFKBO@Site?$AA@ 10047e84     seqboot.obj
 0002:00005e8c       ??_C@_09EDIHJNKH@Character?$AA@ 10047e8c     seqboot.obj
 0002:00005e98       ??_C@_0BC@EKPMCPEA@?5order?5permuted?6?6?$AA@ 10047e98     seqboot.obj
 0002:00005eac       ??_C@_0CO@GNBIOMCO@?5order?5permuted?5separately?5for?5e@ 10047eac     seqboot.obj
 0002:00005edc       ??_C@_0BL@FIEAJLNH@?$CF3ld?5species?0?5?$CF3ld?5?5loci?6?6?$AA@ 10047edc     seqboot.obj
 0002:00005ef8       ??_C@_0P@BBKAJBHF@?$CF3ld?5species?0?5?$AA@ 10047ef8     seqboot.obj
 0002:00005f08       ??_C@_0O@KOKLBOKN@?$CF3ld?5?5sites?6?6?$AA@ 10047f08     seqboot.obj
 0002:00005f18       ??_C@_0BD@EMLFHFLJ@?$CF3ld?5?5characters?6?6?$AA@ 10047f18     seqboot.obj
 0002:00005f2c       ??_C@_05CJABDGIN@Data?6?$AA@ 10047f2c     seqboot.obj
 0002:00005f34       ??_C@_06OLLKJPDP@?9?9?9?9?6?6?$AA@ 10047f34     seqboot.obj
 0002:00005f3c       ??_C@_0DD@GNGHMMPA@ERROR?3?5Invalid?5value?5for?5locus?5?$CF@ 10047f3c     seqboot.obj
 0002:00005f70       ??_C@_0CI@KDNGNPPB@GENE?5FREQ?5OUTSIDE?5?$FL0?01?$FN?5in?5speci@ 10047f70     seqboot.obj
 0002:00005f98       ??_C@_0DA@CHCFNEIN@?6?6ERROR?3?5sequences?5out?5of?5alignm@ 10047f98     seqboot.obj
 0002:00005fc8       ??_C@_05NJOHAKMJ@?$CF8?45f?$AA@ 10047fc8     seqboot.obj
 0002:00005fd0       ??_C@_0BC@GONCKDBG@input?5weight?5file?$AA@ 10047fd0     seqboot.obj
 0002:00005fe4       ??_C@_07EIFHBLMH@weights?$AA@ 10047fe4     seqboot.obj
 0002:00005fec       ??_C@_0N@DEJECCFB@mixture?5file?$AA@ 10047fec     seqboot.obj
 0002:00005ffc       ??_C@_07DHCACGBL@mixture?$AA@ 10047ffc     seqboot.obj
 0002:00006004       ??_C@_01NOFIACDB@w?$AA@    10048004     seqboot.obj
 0002:00006008       ??_C@_0BF@GFDMCHJK@output?5mixtures?5file?$AA@ 10048008     seqboot.obj
 0002:00006020       ??_C@_0L@EHIGPGGF@outmixture?$AA@ 10048020     seqboot.obj
 0002:0000602c       ??_C@_0O@HJHGPHKI@ancestor?5file?$AA@ 1004802c     seqboot.obj
 0002:0000603c       ??_C@_09IANNCONF@ancestors?$AA@ 1004803c     seqboot.obj
 0002:00006048       ??_C@_0BG@CBDCBEGC@output?5ancestors?5file?$AA@ 10048048     seqboot.obj
 0002:00006060       ??_C@_0N@LHLCNINP@outancestors?$AA@ 10048060     seqboot.obj
 0002:00006070       ??_C@_0BE@OEGGLMD@input?5category?5file?$AA@ 10048070     seqboot.obj
 0002:00006084       ??_C@_0L@GOKOAKFO@categories?$AA@ 10048084     seqboot.obj
 0002:00006090       ??_C@_0BF@DCAMGEHC@output?5category?5file?$AA@ 10048090     seqboot.obj
 0002:000060a8       ??_C@_0O@IOEMIMLG@outcategories?$AA@ 100480a8     seqboot.obj
 0002:000060b8       ??_C@_07BBCKLFAG@SeqBoot?$AA@ 100480b8     seqboot.obj
 0002:000060c0       ??_C@_0N@GFGGMJJI@factors?5file?$AA@ 100480c0     seqboot.obj
 0002:000060d0       ??_C@_07BDIIIEFO@factors?$AA@ 100480d0     seqboot.obj
 0002:000060d8       ??_C@_0BE@DCBHJMAC@output?5factors?5file?$AA@ 100480d8     seqboot.obj
 0002:000060ec       ??_C@_0L@GDCOFECA@outfactors?$AA@ 100480ec     seqboot.obj
 0002:000060f8       ??_C@_0BD@OMPFMKPA@output?5weight?5file?$AA@ 100480f8     seqboot.obj
 0002:0000610c       ??_C@_0L@DIPBMLLJ@outweights?$AA@ 1004810c     seqboot.obj
 0002:00006118       ??_C@_0BB@NOHEIJPF@output?5data?5file?$AA@ 10048118     seqboot.obj
 0002:0000612c       ??_C@_07LEOOLFBI@outfile?$AA@ 1004812c     seqboot.obj
 0002:00006134       ??_C@_0DL@FFALOFMI@ERROR?3?5sampling?5frequency?5or?5num@ 10048134     seqboot.obj
 0002:00006170       ??_C@_0BA@GMPPAADB@?$CF5ld?5?$CF5ld?$CF?54ld?6?$AA@ 10048170     seqboot.obj
 0002:00006180       ??_C@_0L@DGEDKBCJ@?$CF5ld?5?$CF5ld?6?$AA@ 10048180     seqboot.obj
 0002:0000618c       ??_C@_0N@PAPNNFFE@?$DMalignment?$DO?6?$AA@ 1004818c     seqboot.obj
 0002:0000619c       ??_C@_07MGCANDCB@?$CDNEXUS?6?$AA@ 1004819c     seqboot.obj
 0002:000061a4       ??_C@_0N@LPMKPLLD@BEGIN?5DATA?$DL?6?$AA@ 100481a4     seqboot.obj
 0002:000061b4       ??_C@_0CC@FIEEBBPN@?5?5DIMENSIONS?5NTAX?$DN?$CFld?5NCHAR?$DN?$CFld?$DL@ 100481b4     seqboot.obj
 0002:000061d8       ??_C@_08DPIGJALC@?5?5FORMAT?$AA@ 100481d8     seqboot.obj
 0002:000061e4       ??_C@_0BA@IOEOKNN@?5interleave?$DNyes?$AA@ 100481e4     seqboot.obj
 0002:000061f4       ??_C@_0P@KDFNINLE@?5interleave?$DNno?$AA@ 100481f4     seqboot.obj
 0002:00006204       ??_C@_0L@KOEBNMH@?5DATATYPE?$DN?$AA@ 10048204     seqboot.obj
 0002:00006210       ??_C@_0BE@MCPCONLJ@DNA?5missing?$DNN?5gap?$DN?9?$AA@ 10048210     seqboot.obj
 0002:00006224       ??_C@_0BE@KGBHNLEJ@RNA?5missing?$DNN?5gap?$DN?9?$AA@ 10048224     seqboot.obj
 0002:00006238       ??_C@_0BI@FONBELJF@protein?5missing?$DN?$DP?5gap?$DN?9?$AA@ 10048238     seqboot.obj
 0002:00006250       ??_C@_08CBJNMPAB@STANDARD?$AA@ 10048250     seqboot.obj
 0002:0000625c       ??_C@_0M@DFOGINOD@?$DL?6?5?5MATRIX?6?$AA@ 1004825c     seqboot.obj
 0002:00006268       ??_C@_05OCHCDALG@?5?$CF3ld?$AA@ 10048268     seqboot.obj
 0002:00006270       ??_C@_0N@DHHCEAKF@?5?5?5?$DMsequence?$AA@ 10048270     seqboot.obj
 0002:00006280       ??_C@_0M@GKCINGGE@?5type?$DN?$CCdna?$CC?$AA@ 10048280     seqboot.obj
 0002:0000628c       ??_C@_0M@IFIILEEG@?5type?$DN?$CCrna?$CC?$AA@ 1004828c     seqboot.obj
 0002:00006298       ??_C@_0BA@GPKNEICK@?5type?$DN?$CCprotein?$CC?$AA@ 10048298     seqboot.obj
 0002:000062a8       ??_C@_02NEKEAGPN@?$DO?6?$AA@ 100482a8     seqboot.obj
 0002:000062ac       ??_C@_0N@NGHIIHBL@?5?5?5?5?5?5?$DMname?$DO?$AA@ 100482ac     seqboot.obj
 0002:000062bc       ??_C@_0BF@LIAHLIMH@?$DM?1name?$DO?6?5?5?5?5?5?5?$DMdata?$DO?$AA@ 100482bc     seqboot.obj
 0002:000062d4       ??_C@_0BA@LPHEGKON@?6?5?5?5?5?5?5?5?5?5?5?5?5?5?5?$AA@ 100482d4     seqboot.obj
 0002:000062e4       ??_C@_0O@OBFBHOIO@?6?5?5?5?5?5?5?5?5?5?5?5?5?$AA@ 100482e4     seqboot.obj
 0002:000062f4       ??_C@_0N@GEIILGID@?6?5?5?5?5?5?5?5?5?5?5?5?$AA@ 100482f4     seqboot.obj
 0002:00006304       ??_C@_0BI@IONFDCDB@?$DM?1data?$DO?6?5?5?5?$DM?1sequence?$DO?6?$AA@ 10048304     seqboot.obj
 0002:0000631c       ??_C@_0O@KGNMPFJM@?$DM?1alignment?$DO?6?$AA@ 1004831c     seqboot.obj
 0002:0000632c       ??_C@_09NDPPFGPJ@?5?5?$DL?6END?$DL?6?$AA@ 1004832c     seqboot.obj
 0002:00006338       ??_C@_01GBGANLPD@0?$AA@    10048338     seqboot.obj
 0002:0000633c       ??_C@_02JIKNIHJJ@?6?5?$AA@ 1004833c     seqboot.obj
 0002:00006340       ??_C@_0CB@CHKJDBFO@completed?5replicate?5number?5?$CF4ld?6@ 10048340     seqboot.obj
 0002:00006370       __xmm@41f00000000000000000000000000000 10048370     seqboot.obj
 0002:000064cc       ??_C@_0BG@CFDANHAH@Ui_NeighborJoinWidget?$AA@ 100484cc     moc_NeighborJoinWidget.obj
 0002:00006668       ?value@?$integral_constant@_N$0A@@std@@2_NB 10048668     MSVCRT:ti_inst.obj
 0002:00006669       ?value@?$integral_constant@_N$00@std@@2_NB 10048669     MSVCRT:ti_inst.obj
 0002:00006670       ??_7type_info@@6B@         10048670     MSVCRT:ti_inst.obj
 0002:00006704       __pDefaultRawDllMain       10048704     MSVCRT:crtdll.obj
 0002:00006704       __pRawDllMain              10048704     MSVCRT:crtdll.obj
 0002:00006708       ?ProcessDetach@NativeDll@<CrtImplementationDetails>@@0IB 10048708     MSVCRT:initsect.obj
 0002:0000670c       ?ProcessAttach@NativeDll@<CrtImplementationDetails>@@0IB 1004870c     MSVCRT:initsect.obj
 0002:00006710       ?ThreadAttach@NativeDll@<CrtImplementationDetails>@@0IB 10048710     MSVCRT:initsect.obj
 0002:00006714       ?ThreadDetach@NativeDll@<CrtImplementationDetails>@@0IB 10048714     MSVCRT:initsect.obj
 0002:00006718       ?ProcessVerifier@NativeDll@<CrtImplementationDetails>@@0IB 10048718     MSVCRT:initsect.obj
 0002:00006720       __load_config_used         10048720     MSVCRT:loadcfg.obj
 0002:000067d4       ??_R4error_category@std@@6B@ 100487d4     DistanceMatrix.obj
 0002:000067e8       ??_R3error_category@std@@8 100487e8     DistanceMatrix.obj
 0002:000067f8       ??_R2error_category@std@@8 100487f8     DistanceMatrix.obj
 0002:00006800       ??_R1A@?0A@EA@error_category@std@@8 10048800     DistanceMatrix.obj
 0002:0000681c       ??_R4_Generic_error_category@std@@6B@ 1004881c     DistanceMatrix.obj
 0002:00006830       ??_R3_Generic_error_category@std@@8 10048830     DistanceMatrix.obj
 0002:00006840       ??_R2_Generic_error_category@std@@8 10048840     DistanceMatrix.obj
 0002:0000684c       ??_R1A@?0A@EA@_Generic_error_category@std@@8 1004884c     DistanceMatrix.obj
 0002:00006868       ??_R4_Iostream_error_category@std@@6B@ 10048868     DistanceMatrix.obj
 0002:0000687c       ??_R3_Iostream_error_category@std@@8 1004887c     DistanceMatrix.obj
 0002:0000688c       ??_R2_Iostream_error_category@std@@8 1004888c     DistanceMatrix.obj
 0002:0000689c       ??_R1A@?0A@EA@_Iostream_error_category@std@@8 1004889c     DistanceMatrix.obj
 0002:000068b8       ??_R4_System_error_category@std@@6B@ 100488b8     DistanceMatrix.obj
 0002:000068cc       ??_R3_System_error_category@std@@8 100488cc     DistanceMatrix.obj
 0002:000068dc       ??_R2_System_error_category@std@@8 100488dc     DistanceMatrix.obj
 0002:000068ec       ??_R1A@?0A@EA@_System_error_category@std@@8 100488ec     DistanceMatrix.obj
 0002:00006908       ??_R4MemoryLocker@U2@@6B@  10048908     DistanceMatrix.obj
 0002:0000691c       ??_R3MemoryLocker@U2@@8    1004891c     DistanceMatrix.obj
 0002:0000692c       ??_R2MemoryLocker@U2@@8    1004892c     DistanceMatrix.obj
 0002:00006934       ??_R1A@?0A@EA@MemoryLocker@U2@@8 10048934     DistanceMatrix.obj
 0002:00006950       ??_R4MultipleSequenceAlignmentRow@U2@@6B@ 10048950     DistanceMatrix.obj
 0002:00006964       ??_R3MultipleSequenceAlignmentRow@U2@@8 10048964     DistanceMatrix.obj
 0002:00006974       ??_R2MultipleSequenceAlignmentRow@U2@@8 10048974     DistanceMatrix.obj
 0002:00006980       ??_R1A@?0A@EA@MultipleSequenceAlignmentRow@U2@@8 10048980     DistanceMatrix.obj
 0002:0000699c       ??_R1A@?0A@EA@MultipleAlignmentRow@U2@@8 1004899c     DistanceMatrix.obj
 0002:000069b8       ??_R3MultipleAlignmentRow@U2@@8 100489b8     DistanceMatrix.obj
 0002:000069c8       ??_R2MultipleAlignmentRow@U2@@8 100489c8     DistanceMatrix.obj
 0002:000069d0       ??_R1A@?0A@EA@QObject@@8   100489d0     NeighborJoinAdapter.obj
 0002:000069ec       ??_R3QObject@@8            100489ec     NeighborJoinAdapter.obj
 0002:000069fc       ??_R2QObject@@8            100489fc     NeighborJoinAdapter.obj
 0002:00006a04       ??_R4NeighborJoinCalculateTreeTask@U2@@6B@ 10048a04     NeighborJoinAdapter.obj
 0002:00006a18       ??_R3NeighborJoinCalculateTreeTask@U2@@8 10048a18     NeighborJoinAdapter.obj
 0002:00006a28       ??_R2NeighborJoinCalculateTreeTask@U2@@8 10048a28     NeighborJoinAdapter.obj
 0002:00006a3c       ??_R1A@?0A@EA@NeighborJoinCalculateTreeTask@U2@@8 10048a3c     NeighborJoinAdapter.obj
 0002:00006a58       ??_R1A@?0A@EA@PhyTreeGeneratorTask@U2@@8 10048a58     NeighborJoinAdapter.obj
 0002:00006a74       ??_R3PhyTreeGeneratorTask@U2@@8 10048a74     NeighborJoinAdapter.obj
 0002:00006a84       ??_R2PhyTreeGeneratorTask@U2@@8 10048a84     NeighborJoinAdapter.obj
 0002:00006a94       ??_R1A@?0A@EA@Task@U2@@8   10048a94     NeighborJoinAdapter.obj
 0002:00006ab0       ??_R3Task@U2@@8            10048ab0     NeighborJoinAdapter.obj
 0002:00006ac0       ??_R2Task@U2@@8            10048ac0     NeighborJoinAdapter.obj
 0002:00006acc       ??_R4QWidget@@6BQObject@@@ 10048acc     NeighborJoinWidget.obj
 0002:00006ae0       ??_R3QWidget@@8            10048ae0     NeighborJoinWidget.obj
 0002:00006af0       ??_R2QWidget@@8            10048af0     NeighborJoinWidget.obj
 0002:00006b00       ??_R1A@?0A@EA@QWidget@@8   10048b00     NeighborJoinWidget.obj
 0002:00006b1c       ??_R17?0A@EA@QPaintDevice@@8 10048b1c     NeighborJoinWidget.obj
 0002:00006b38       ??_R3QPaintDevice@@8       10048b38     NeighborJoinWidget.obj
 0002:00006b48       ??_R2QPaintDevice@@8       10048b48     NeighborJoinWidget.obj
 0002:00006b50       ??_R1A@?0A@EA@QPaintDevice@@8 10048b50     NeighborJoinWidget.obj
 0002:00006b6c       ??_R4QWidget@@6BQPaintDevice@@@ 10048b6c     NeighborJoinWidget.obj
 0002:00006b80       ??_R4PhyTreeDisplayOptionsWidget@U2@@6BQObject@@@ 10048b80     NeighborJoinWidget.obj
 0002:00006b94       ??_R3PhyTreeDisplayOptionsWidget@U2@@8 10048b94     NeighborJoinWidget.obj
 0002:00006ba4       ??_R2PhyTreeDisplayOptionsWidget@U2@@8 10048ba4     NeighborJoinWidget.obj
 0002:00006bbc       ??_R1A@?0A@EA@PhyTreeDisplayOptionsWidget@U2@@8 10048bbc     NeighborJoinWidget.obj
 0002:00006bd8       ??_R1A@?0A@EA@CreatePhyTreeWidget@U2@@8 10048bd8     NeighborJoinWidget.obj
 0002:00006bf4       ??_R3CreatePhyTreeWidget@U2@@8 10048bf4     NeighborJoinWidget.obj
 0002:00006c04       ??_R2CreatePhyTreeWidget@U2@@8 10048c04     NeighborJoinWidget.obj
 0002:00006c18       ??_R4PhyTreeDisplayOptionsWidget@U2@@6BQPaintDevice@@@ 10048c18     NeighborJoinWidget.obj
 0002:00006c2c       ??_R4QCheckBox@@6BQObject@@@ 10048c2c     NeighborJoinWidget.obj
 0002:00006c40       ??_R3QCheckBox@@8          10048c40     NeighborJoinWidget.obj
 0002:00006c50       ??_R2QCheckBox@@8          10048c50     NeighborJoinWidget.obj
 0002:00006c68       ??_R1A@?0A@EA@QCheckBox@@8 10048c68     NeighborJoinWidget.obj
 0002:00006c84       ??_R1A@?0A@EA@QAbstractButton@@8 10048c84     NeighborJoinWidget.obj
 0002:00006ca0       ??_R3QAbstractButton@@8    10048ca0     NeighborJoinWidget.obj
 0002:00006cb0       ??_R2QAbstractButton@@8    10048cb0     NeighborJoinWidget.obj
 0002:00006cc4       ??_R4QCheckBox@@6BQPaintDevice@@@ 10048cc4     NeighborJoinWidget.obj
 0002:00006cd8       ??_R4QTabWidget@@6BQObject@@@ 10048cd8     NeighborJoinWidget.obj
 0002:00006cec       ??_R3QTabWidget@@8         10048cec     NeighborJoinWidget.obj
 0002:00006cfc       ??_R2QTabWidget@@8         10048cfc     NeighborJoinWidget.obj
 0002:00006d10       ??_R1A@?0A@EA@QTabWidget@@8 10048d10     NeighborJoinWidget.obj
 0002:00006d2c       ??_R4QTabWidget@@6BQPaintDevice@@@ 10048d2c     NeighborJoinWidget.obj
 0002:00006d40       ??_R4QComboBox@@6BQObject@@@ 10048d40     NeighborJoinWidget.obj
 0002:00006d54       ??_R3QComboBox@@8          10048d54     NeighborJoinWidget.obj
 0002:00006d64       ??_R2QComboBox@@8          10048d64     NeighborJoinWidget.obj
 0002:00006d78       ??_R1A@?0A@EA@QComboBox@@8 10048d78     NeighborJoinWidget.obj
 0002:00006d94       ??_R4QComboBox@@6BQPaintDevice@@@ 10048d94     NeighborJoinWidget.obj
 0002:00006da8       ??_R4QSpinBox@@6BQObject@@@ 10048da8     NeighborJoinWidget.obj
 0002:00006dbc       ??_R3QSpinBox@@8           10048dbc     NeighborJoinWidget.obj
 0002:00006dcc       ??_R2QSpinBox@@8           10048dcc     NeighborJoinWidget.obj
 0002:00006de4       ??_R1A@?0A@EA@QSpinBox@@8  10048de4     NeighborJoinWidget.obj
 0002:00006e00       ??_R1A@?0A@EA@QAbstractSpinBox@@8 10048e00     NeighborJoinWidget.obj
 0002:00006e1c       ??_R3QAbstractSpinBox@@8   10048e1c     NeighborJoinWidget.obj
 0002:00006e2c       ??_R2QAbstractSpinBox@@8   10048e2c     NeighborJoinWidget.obj
 0002:00006e40       ??_R4QSpinBox@@6BQPaintDevice@@@ 10048e40     NeighborJoinWidget.obj
 0002:00006e54       ??_R4QDoubleSpinBox@@6BQObject@@@ 10048e54     NeighborJoinWidget.obj
 0002:00006e68       ??_R3QDoubleSpinBox@@8     10048e68     NeighborJoinWidget.obj
 0002:00006e78       ??_R2QDoubleSpinBox@@8     10048e78     NeighborJoinWidget.obj
 0002:00006e90       ??_R1A@?0A@EA@QDoubleSpinBox@@8 10048e90     NeighborJoinWidget.obj
 0002:00006eac       ??_R4QDoubleSpinBox@@6BQPaintDevice@@@ 10048eac     NeighborJoinWidget.obj
 0002:00006ec0       ??_R4QSpacerItem@@6B@      10048ec0     NeighborJoinWidget.obj
 0002:00006ed4       ??_R3QSpacerItem@@8        10048ed4     NeighborJoinWidget.obj
 0002:00006ee4       ??_R2QSpacerItem@@8        10048ee4     NeighborJoinWidget.obj
 0002:00006ef0       ??_R1A@?0A@EA@QSpacerItem@@8 10048ef0     NeighborJoinWidget.obj
 0002:00006f0c       ??_R1A@?0A@EA@QLayoutItem@@8 10048f0c     NeighborJoinWidget.obj
 0002:00006f28       ??_R3QLayoutItem@@8        10048f28     NeighborJoinWidget.obj
 0002:00006f38       ??_R2QLayoutItem@@8        10048f38     NeighborJoinWidget.obj
 0002:00006f40       ??_R4QHBoxLayout@@6BQObject@@@ 10048f40     NeighborJoinWidget.obj
 0002:00006f54       ??_R3QHBoxLayout@@8        10048f54     NeighborJoinWidget.obj
 0002:00006f64       ??_R2QHBoxLayout@@8        10048f64     NeighborJoinWidget.obj
 0002:00006f7c       ??_R1A@?0A@EA@QHBoxLayout@@8 10048f7c     NeighborJoinWidget.obj
 0002:00006f98       ??_R1A@?0A@EA@QBoxLayout@@8 10048f98     NeighborJoinWidget.obj
 0002:00006fb4       ??_R3QBoxLayout@@8         10048fb4     NeighborJoinWidget.obj
 0002:00006fc4       ??_R2QBoxLayout@@8         10048fc4     NeighborJoinWidget.obj
 0002:00006fd8       ??_R1A@?0A@EA@QLayout@@8   10048fd8     NeighborJoinWidget.obj
 0002:00006ff4       ??_R3QLayout@@8            10048ff4     NeighborJoinWidget.obj
 0002:00007004       ??_R2QLayout@@8            10049004     NeighborJoinWidget.obj
 0002:00007014       ??_R17?0A@EA@QLayoutItem@@8 10049014     NeighborJoinWidget.obj
 0002:00007030       ??_R4QHBoxLayout@@6BQLayoutItem@@@ 10049030     NeighborJoinWidget.obj
 0002:00007044       ??_R4QVBoxLayout@@6BQObject@@@ 10049044     NeighborJoinWidget.obj
 0002:00007058       ??_R3QVBoxLayout@@8        10049058     NeighborJoinWidget.obj
 0002:00007068       ??_R2QVBoxLayout@@8        10049068     NeighborJoinWidget.obj
 0002:00007080       ??_R1A@?0A@EA@QVBoxLayout@@8 10049080     NeighborJoinWidget.obj
 0002:0000709c       ??_R4QVBoxLayout@@6BQLayoutItem@@@ 1004909c     NeighborJoinWidget.obj
 0002:000070b0       ??_R4QGridLayout@@6BQObject@@@ 100490b0     NeighborJoinWidget.obj
 0002:000070c4       ??_R3QGridLayout@@8        100490c4     NeighborJoinWidget.obj
 0002:000070d4       ??_R2QGridLayout@@8        100490d4     NeighborJoinWidget.obj
 0002:000070e8       ??_R1A@?0A@EA@QGridLayout@@8 100490e8     NeighborJoinWidget.obj
 0002:00007104       ??_R4QGridLayout@@6BQLayoutItem@@@ 10049104     NeighborJoinWidget.obj
 0002:00007118       ??_R4QLabel@@6BQObject@@@  10049118     NeighborJoinWidget.obj
 0002:0000712c       ??_R3QLabel@@8             1004912c     NeighborJoinWidget.obj
 0002:0000713c       ??_R2QLabel@@8             1004913c     NeighborJoinWidget.obj
 0002:00007154       ??_R1A@?0A@EA@QLabel@@8    10049154     NeighborJoinWidget.obj
 0002:00007170       ??_R1A@?0A@EA@QFrame@@8    10049170     NeighborJoinWidget.obj
 0002:0000718c       ??_R3QFrame@@8             1004918c     NeighborJoinWidget.obj
 0002:0000719c       ??_R2QFrame@@8             1004919c     NeighborJoinWidget.obj
 0002:000071b0       ??_R4QLabel@@6BQPaintDevice@@@ 100491b0     NeighborJoinWidget.obj
 0002:000071c4       ??_R4NeighborJoinWidget@U2@@6BQObject@@@ 100491c4     NeighborJoinWidget.obj
 0002:000071d8       ??_R3NeighborJoinWidget@U2@@8 100491d8     NeighborJoinWidget.obj
 0002:000071e8       ??_R2NeighborJoinWidget@U2@@8 100491e8     NeighborJoinWidget.obj
 0002:00007204       ??_R1A@?0A@EA@NeighborJoinWidget@U2@@8 10049204     NeighborJoinWidget.obj
 0002:00007220       ??_R1BI@?0A@EA@Ui_NeighborJoinWidget@@8 10049220     NeighborJoinWidget.obj
 0002:0000723c       ??_R3Ui_NeighborJoinWidget@@8 1004923c     NeighborJoinWidget.obj
 0002:0000724c       ??_R2Ui_NeighborJoinWidget@@8 1004924c     NeighborJoinWidget.obj
 0002:00007254       ??_R1A@?0A@EA@Ui_NeighborJoinWidget@@8 10049254     NeighborJoinWidget.obj
 0002:00007270       ??_R4NeighborJoinWidget@U2@@6BQPaintDevice@@@ 10049270     NeighborJoinWidget.obj
 0002:00007284       ??_R4CmdlineInOutTaskRunner@U2@@6B@ 10049284     PhylipCmdlineTask.obj
 0002:00007298       ??_R3CmdlineInOutTaskRunner@U2@@8 10049298     PhylipCmdlineTask.obj
 0002:000072a8       ??_R2CmdlineInOutTaskRunner@U2@@8 100492a8     PhylipCmdlineTask.obj
 0002:000072bc       ??_R1A@?0A@EA@CmdlineInOutTaskRunner@U2@@8 100492bc     PhylipCmdlineTask.obj
 0002:000072d8       ??_R1A@?0A@EA@CmdlineTaskRunner@U2@@8 100492d8     PhylipCmdlineTask.obj
 0002:000072f4       ??_R3CmdlineTaskRunner@U2@@8 100492f4     PhylipCmdlineTask.obj
 0002:00007304       ??_R2CmdlineTaskRunner@U2@@8 10049304     PhylipCmdlineTask.obj
 0002:00007314       ??_R4PhyTreeObject@U2@@6B@ 10049314     PhylipCmdlineTask.obj
 0002:00007328       ??_R3PhyTreeObject@U2@@8   10049328     PhylipCmdlineTask.obj
 0002:00007338       ??_R2PhyTreeObject@U2@@8   10049338     PhylipCmdlineTask.obj
 0002:00007350       ??_R1A@?0A@EA@PhyTreeObject@U2@@8 10049350     PhylipCmdlineTask.obj
 0002:0000736c       ??_R1A@?0A@EA@GObject@U2@@8 1004936c     PhylipCmdlineTask.obj
 0002:00007388       ??_R3GObject@U2@@8         10049388     PhylipCmdlineTask.obj
 0002:00007398       ??_R2GObject@U2@@8         10049398     PhylipCmdlineTask.obj
 0002:000073ac       ??_R1A@?0A@EA@StateLockableTreeItem@U2@@8 100493ac     PhylipCmdlineTask.obj
 0002:000073c8       ??_R3StateLockableTreeItem@U2@@8 100493c8     PhylipCmdlineTask.obj
 0002:000073d8       ??_R2StateLockableTreeItem@U2@@8 100493d8     PhylipCmdlineTask.obj
 0002:000073e8       ??_R1A@?0A@EA@StateLockableItem@U2@@8 100493e8     PhylipCmdlineTask.obj
 0002:00007404       ??_R3StateLockableItem@U2@@8 10049404     PhylipCmdlineTask.obj
 0002:00007414       ??_R2StateLockableItem@U2@@8 10049414     PhylipCmdlineTask.obj
 0002:00007420       ??_R4PhylipCmdlineTask@U2@@6B@ 10049420     PhylipCmdlineTask.obj
 0002:00007434       ??_R3PhylipCmdlineTask@U2@@8 10049434     PhylipCmdlineTask.obj
 0002:00007444       ??_R2PhylipCmdlineTask@U2@@8 10049444     PhylipCmdlineTask.obj
 0002:00007458       ??_R1A@?0A@EA@PhylipCmdlineTask@U2@@8 10049458     PhylipCmdlineTask.obj
 0002:00007474       ??_R4AbstractInt32Id@U2@@6B@ 10049474     PhylipPlugin.obj
 0002:00007488       ??_R3AbstractInt32Id@U2@@8 10049488     PhylipPlugin.obj
 0002:00007498       ??_R2AbstractInt32Id@U2@@8 10049498     PhylipPlugin.obj
 0002:000074a4       ??_R1A@?0A@EA@AbstractInt32Id@U2@@8 100494a4     PhylipPlugin.obj
 0002:000074c0       ??_R1A@?0A@EA@?$AbstractId@H@U2@@8 100494c0     PhylipPlugin.obj
 0002:000074dc       ??_R3?$AbstractId@H@U2@@8  100494dc     PhylipPlugin.obj
 0002:000074ec       ??_R2?$AbstractId@H@U2@@8  100494ec     PhylipPlugin.obj
 0002:000074f4       ??_R4?$AbstractId@H@U2@@6B@ 100494f4     PhylipPlugin.obj
 0002:00007508       ??_R4ServiceType@U2@@6B@   10049508     PhylipPlugin.obj
 0002:0000751c       ??_R3ServiceType@U2@@8     1004951c     PhylipPlugin.obj
 0002:0000752c       ??_R2ServiceType@U2@@8     1004952c     PhylipPlugin.obj
 0002:0000753c       ??_R1A@?0A@EA@ServiceType@U2@@8 1004953c     PhylipPlugin.obj
 0002:00007558       ??_R4TaskStarter@U2@@6B@   10049558     PhylipPlugin.obj
 0002:0000756c       ??_R3TaskStarter@U2@@8     1004956c     PhylipPlugin.obj
 0002:0000757c       ??_R2TaskStarter@U2@@8     1004957c     PhylipPlugin.obj
 0002:00007588       ??_R1A@?0A@EA@TaskStarter@U2@@8 10049588     PhylipPlugin.obj
 0002:000075a4       ??_R4NeighborJoinAdapter@U2@@6B@ 100495a4     PhylipPlugin.obj
 0002:000075b8       ??_R3NeighborJoinAdapter@U2@@8 100495b8     PhylipPlugin.obj
 0002:000075c8       ??_R2NeighborJoinAdapter@U2@@8 100495c8     PhylipPlugin.obj
 0002:000075d4       ??_R1A@?0A@EA@NeighborJoinAdapter@U2@@8 100495d4     PhylipPlugin.obj
 0002:000075f0       ??_R1A@?0A@EA@PhyTreeGenerator@U2@@8 100495f0     PhylipPlugin.obj
 0002:0000760c       ??_R3PhyTreeGenerator@U2@@8 1004960c     PhylipPlugin.obj
 0002:0000761c       ??_R2PhyTreeGenerator@U2@@8 1004961c     PhylipPlugin.obj
 0002:00007624       ??_R4PhylipPlugin@U2@@6B@  10049624     PhylipPlugin.obj
 0002:00007638       ??_R3PhylipPlugin@U2@@8    10049638     PhylipPlugin.obj
 0002:00007648       ??_R2PhylipPlugin@U2@@8    10049648     PhylipPlugin.obj
 0002:00007658       ??_R1A@?0A@EA@PhylipPlugin@U2@@8 10049658     PhylipPlugin.obj
 0002:00007674       ??_R1A@?0A@EA@Plugin@U2@@8 10049674     PhylipPlugin.obj
 0002:00007690       ??_R3Plugin@U2@@8          10049690     PhylipPlugin.obj
 0002:000076a0       ??_R2Plugin@U2@@8          100496a0     PhylipPlugin.obj
 0002:000076ac       ??_R4?$GAutoDeleteList@VXMLTestFactory@U2@@@U2@@6B@ 100496ac     PhylipPlugin.obj
 0002:000076c0       ??_R3?$GAutoDeleteList@VXMLTestFactory@U2@@@U2@@8 100496c0     PhylipPlugin.obj
 0002:000076d0       ??_R2?$GAutoDeleteList@VXMLTestFactory@U2@@@U2@@8 100496d0     PhylipPlugin.obj
 0002:000076dc       ??_R1A@?0A@EA@?$GAutoDeleteList@VXMLTestFactory@U2@@@U2@@8 100496dc     PhylipPlugin.obj
 0002:000076f8       ??_R1A@?0A@EA@XmlTest@U2@@8 100496f8     PhylipPluginTests.obj
 0002:00007714       ??_R3XmlTest@U2@@8         10049714     PhylipPluginTests.obj
 0002:00007724       ??_R2XmlTest@U2@@8         10049724     PhylipPluginTests.obj
 0002:00007738       ??_R1A@?0A@EA@GTest@U2@@8  10049738     PhylipPluginTests.obj
 0002:00007754       ??_R3GTest@U2@@8           10049754     PhylipPluginTests.obj
 0002:00007764       ??_R2GTest@U2@@8           10049764     PhylipPluginTests.obj
 0002:00007774       ??_R1A@?0A@EA@XMLTestFactory@U2@@8 10049774     PhylipPluginTests.obj
 0002:00007790       ??_R3XMLTestFactory@U2@@8  10049790     PhylipPluginTests.obj
 0002:000077a0       ??_R2XMLTestFactory@U2@@8  100497a0     PhylipPluginTests.obj
 0002:000077a8       ??_R4PhyTreeGeneratorLauncherTask@U2@@6B@ 100497a8     PhylipPluginTests.obj
 0002:000077bc       ??_R3PhyTreeGeneratorLauncherTask@U2@@8 100497bc     PhylipPluginTests.obj
 0002:000077cc       ??_R2PhyTreeGeneratorLauncherTask@U2@@8 100497cc     PhylipPluginTests.obj
 0002:000077dc       ??_R1A@?0A@EA@PhyTreeGeneratorLauncherTask@U2@@8 100497dc     PhylipPluginTests.obj
 0002:000077f8       ??_R4GTest_NeighborJoin@U2@@6B@ 100497f8     PhylipPluginTests.obj
 0002:0000780c       ??_R3GTest_NeighborJoin@U2@@8 1004980c     PhylipPluginTests.obj
 0002:0000781c       ??_R2GTest_NeighborJoin@U2@@8 1004981c     PhylipPluginTests.obj
 0002:00007834       ??_R1A@?0A@EA@GTest_NeighborJoin@U2@@8 10049834     PhylipPluginTests.obj
 0002:00007850       ??_R4GTest_NeighborJoinFactory@GTest_NeighborJoin@U2@@6B@ 10049850     PhylipPluginTests.obj
 0002:00007864       ??_R3GTest_NeighborJoinFactory@GTest_NeighborJoin@U2@@8 10049864     PhylipPluginTests.obj
 0002:00007874       ??_R2GTest_NeighborJoinFactory@GTest_NeighborJoin@U2@@8 10049874     PhylipPluginTests.obj
 0002:00007880       ??_R1A@?0A@EA@GTest_NeighborJoinFactory@GTest_NeighborJoin@U2@@8 10049880     PhylipPluginTests.obj
 0002:0000789c       ??_R4MultipleSequenceAlignmentObject@U2@@6B@ 1004989c     PhylipTask.obj
 0002:000078b0       ??_R3MultipleSequenceAlignmentObject@U2@@8 100498b0     PhylipTask.obj
 0002:000078c0       ??_R2MultipleSequenceAlignmentObject@U2@@8 100498c0     PhylipTask.obj
 0002:000078dc       ??_R1A@?0A@EA@MultipleSequenceAlignmentObject@U2@@8 100498dc     PhylipTask.obj
 0002:000078f8       ??_R1A@?0A@EA@MultipleAlignmentObject@U2@@8 100498f8     PhylipTask.obj
 0002:00007914       ??_R3MultipleAlignmentObject@U2@@8 10049914     PhylipTask.obj
 0002:00007924       ??_R2MultipleAlignmentObject@U2@@8 10049924     PhylipTask.obj
 0002:0000793c       ??_R4PhylipTask@U2@@6B@    1004993c     PhylipTask.obj
 0002:00007950       ??_R3PhylipTask@U2@@8      10049950     PhylipTask.obj
 0002:00007960       ??_R2PhylipTask@U2@@8      10049960     PhylipTask.obj
 0002:00007974       ??_R1A@?0A@EA@PhylipTask@U2@@8 10049974     PhylipTask.obj
 0002:00007990       ??_R1A@?0A@EA@CmdlineTask@U2@@8 10049990     PhylipTask.obj
 0002:000079ac       ??_R3CmdlineTask@U2@@8     100499ac     PhylipTask.obj
 0002:000079bc       ??_R2CmdlineTask@U2@@8     100499bc     PhylipTask.obj
 0002:000079cc       ??_R4MultipleSequenceAlignment@U2@@6B@ 100499cc     SeqBootAdapter.obj
 0002:000079e0       ??_R3MultipleSequenceAlignment@U2@@8 100499e0     SeqBootAdapter.obj
 0002:000079f0       ??_R2MultipleSequenceAlignment@U2@@8 100499f0     SeqBootAdapter.obj
 0002:000079fc       ??_R1A@?0A@EA@MultipleSequenceAlignment@U2@@8 100499fc     SeqBootAdapter.obj
 0002:00007a18       ??_R1A@?0A@EA@MultipleAlignment@U2@@8 10049a18     SeqBootAdapter.obj
 0002:00007a34       ??_R3MultipleAlignment@U2@@8 10049a34     SeqBootAdapter.obj
 0002:00007a44       ??_R2MultipleAlignment@U2@@8 10049a44     SeqBootAdapter.obj
 0002:00007a4c       ??_R4type_info@@6B@        10049a4c     MSVCRT:ti_inst.obj
 0002:00007a60       ??_R3type_info@@8          10049a60     MSVCRT:ti_inst.obj
 0002:00007a70       ??_R2type_info@@8          10049a70     MSVCRT:ti_inst.obj
 0002:00007a78       ??_R1A@?0A@EA@type_info@@8 10049a78     MSVCRT:ti_inst.obj
 0002:00007aa0       ___safe_se_handler_table   10049aa0     <linker-defined>
 0002:00007f14       ___rtc_iaa                 10049f14     MSVCRT:initsect.obj
 0002:00007f18       ___rtc_izz                 10049f18     MSVCRT:initsect.obj
 0002:00007f1c       ___rtc_taa                 10049f1c     MSVCRT:initsect.obj
 0002:00007f20       ___rtc_tzz                 10049f20     MSVCRT:initsect.obj
 0002:0000bdd8       __TI2CPAD                  1004ddd8     phylip.obj
 0002:0000bde8       __CTA2PAD                  1004dde8     phylip.obj
 0002:0000bdf4       __CT??_R0PAD@84            1004ddf4     phylip.obj
 0002:0000be10       __CT??_R0PAX@84            1004de10     phylip.obj
 0002:0000c8b0       __IMPORT_DESCRIPTOR_U2Core 1004e8b0     U2Core:U2Core.dll
 0002:0000c8c4       __IMPORT_DESCRIPTOR_U2Algorithm 1004e8c4     U2Algorithm:U2Algorithm.dll
 0002:0000c8d8       __IMPORT_DESCRIPTOR_U2View 1004e8d8     U2View:U2View.dll
 0002:0000c8ec       __IMPORT_DESCRIPTOR_U2Test 1004e8ec     U2Test:U2Test.dll
 0002:0000c900       __IMPORT_DESCRIPTOR_Qt5Widgets 1004e900     Qt5Widgets:Qt5Widgets.dll
 0002:0000c914       __IMPORT_DESCRIPTOR_Qt5Xml 1004e914     Qt5Xml:Qt5Xml.dll
 0002:0000c928       __IMPORT_DESCRIPTOR_Qt5Core 1004e928     Qt5Core:Qt5Core.dll
 0002:0000c93c       __IMPORT_DESCRIPTOR_KERNEL32 1004e93c     kernel32:KERNEL32.dll
 0002:0000c950       __IMPORT_DESCRIPTOR_MSVCP120 1004e950     msvcprt:MSVCP120.dll
 0002:0000c964       __IMPORT_DESCRIPTOR_MSVCR120 1004e964     MSVCRT:MSVCR120.dll
 0002:0000c978       __NULL_IMPORT_DESCRIPTOR   1004e978     U2Core:U2Core.dll
 0003:00002760       ?_Generic_object@?$_Error_objects@H@std@@2V_Generic_error_category@2@A 1005a760     DistanceMatrix.obj
 0003:00002764       ?_Iostream_object@?$_Error_objects@H@std@@2V_Iostream_error_category@2@A 1005a764     DistanceMatrix.obj
 0003:00002768       ?_System_object@?$_Error_objects@H@std@@2V_System_error_category@2@A 1005a768     DistanceMatrix.obj
 0003:00009e98       ?staticMetaObject@NeighborJoinWidget@U2@@2UQMetaObject@@B 10061e98     moc_NeighborJoinWidget.obj
 0003:00009eb0       ?staticMetaObject@PhylipCmdlineTask@U2@@2UQMetaObject@@B 10061eb0     moc_PhylipCmdlineTask.obj
 0003:00009f30       ?staticMetaObject@PhylipPlugin@U2@@2UQMetaObject@@B 10061f30     moc_PhylipPlugin.obj
 0003:00009f48       ?staticMetaObject@GTest_NeighborJoin@U2@@2UQMetaObject@@B 10061f48     moc_PhylipPluginTests.obj
 0003:00009f60       ?staticMetaObject@PhylipTask@U2@@2UQMetaObject@@B 10061f60     moc_PhylipTask.obj
 0003:00009f80       ___security_cookie         10061f80     MSVCRT:gs_cookie.obj
 0003:00009f84       ___security_cookie_complement 10061f84     MSVCRT:gs_cookie.obj
 0003:00009f90       ___isa_enabled             10061f90     MSVCRT:cpu_disp.obj
 0003:00009fa0       ___native_dllmain_reason   10061fa0     MSVCRT:natstart.obj
 0003:00009fa4       ??_R0?AVbad_alloc@std@@@8  10061fa4     DistanceMatrix.obj
 0003:00009fc0       ??_R0?AVerror_category@std@@@8 10061fc0     DistanceMatrix.obj
 0003:00009fe4       ??_R0?AV_Generic_error_category@std@@@8 10061fe4     DistanceMatrix.obj
 0003:0000a010       ??_R0?AV_Iostream_error_category@std@@@8 10062010     DistanceMatrix.obj
 0003:0000a03c       ??_R0?AV_System_error_category@std@@@8 1006203c     DistanceMatrix.obj
 0003:0000a068       ??_R0?AVMemoryLocker@U2@@@8 10062068     DistanceMatrix.obj
 0003:0000a088       ??_R0?AVMultipleSequenceAlignmentRow@U2@@@8 10062088     DistanceMatrix.obj
 0003:0000a0b8       ??_R0?AVMultipleAlignmentRow@U2@@@8 100620b8     DistanceMatrix.obj
 0003:0000a0e0       ??_R0PAD@8                 100620e0     NeighborJoinAdapter.obj
 0003:0000a0f0       ??_R0?AVQObject@@@8        100620f0     NeighborJoinAdapter.obj
 0003:0000a108       ??_R0?AVNeighborJoinCalculateTreeTask@U2@@@8 10062108     NeighborJoinAdapter.obj
 0003:0000a138       ??_R0?AVPhyTreeGeneratorTask@U2@@@8 10062138     NeighborJoinAdapter.obj
 0003:0000a160       ??_R0?AVTask@U2@@@8        10062160     NeighborJoinAdapter.obj
 0003:0000a178       ??_R0?AVQWidget@@@8        10062178     NeighborJoinWidget.obj
 0003:0000a190       ??_R0?AVQPaintDevice@@@8   10062190     NeighborJoinWidget.obj
 0003:0000a1ac       ??_R0?AVPhyTreeDisplayOptionsWidget@U2@@@8 100621ac     NeighborJoinWidget.obj
 0003:0000a1dc       ??_R0?AVCreatePhyTreeWidget@U2@@@8 100621dc     NeighborJoinWidget.obj
 0003:0000a204       ??_R0?AVQCheckBox@@@8      10062204     NeighborJoinWidget.obj
 0003:0000a21c       ??_R0?AVQAbstractButton@@@8 1006221c     NeighborJoinWidget.obj
 0003:0000a23c       ??_R0?AVQTabWidget@@@8     1006223c     NeighborJoinWidget.obj
 0003:0000a258       ??_R0?AVQComboBox@@@8      10062258     NeighborJoinWidget.obj
 0003:0000a270       ??_R0?AVQSpinBox@@@8       10062270     NeighborJoinWidget.obj
 0003:0000a288       ??_R0?AVQAbstractSpinBox@@@8 10062288     NeighborJoinWidget.obj
 0003:0000a2a8       ??_R0?AVQDoubleSpinBox@@@8 100622a8     NeighborJoinWidget.obj
 0003:0000a2c8       ??_R0?AVQSpacerItem@@@8    100622c8     NeighborJoinWidget.obj
 0003:0000a2e4       ??_R0?AVQLayoutItem@@@8    100622e4     NeighborJoinWidget.obj
 0003:0000a300       ??_R0?AVQHBoxLayout@@@8    10062300     NeighborJoinWidget.obj
 0003:0000a31c       ??_R0?AVQBoxLayout@@@8     1006231c     NeighborJoinWidget.obj
 0003:0000a338       ??_R0?AVQLayout@@@8        10062338     NeighborJoinWidget.obj
 0003:0000a350       ??_R0?AVQVBoxLayout@@@8    10062350     NeighborJoinWidget.obj
 0003:0000a36c       ??_R0?AVQGridLayout@@@8    1006236c     NeighborJoinWidget.obj
 0003:0000a388       ??_R0?AVQLabel@@@8         10062388     NeighborJoinWidget.obj
 0003:0000a3a0       ??_R0?AVQFrame@@@8         100623a0     NeighborJoinWidget.obj
 0003:0000a3b8       ??_R0?AVNeighborJoinWidget@U2@@@8 100623b8     NeighborJoinWidget.obj
 0003:0000a3dc       ??_R0?AVUi_NeighborJoinWidget@@@8 100623dc     NeighborJoinWidget.obj
 0003:0000a400       ??_R0?AVCmdlineInOutTaskRunner@U2@@@8 10062400     PhylipCmdlineTask.obj
 0003:0000a428       ??_R0?AVCmdlineTaskRunner@U2@@@8 10062428     PhylipCmdlineTask.obj
 0003:0000a44c       ??_R0?AVPhyTreeObject@U2@@@8 1006244c     PhylipCmdlineTask.obj
 0003:0000a46c       ??_R0?AVGObject@U2@@@8     1006246c     PhylipCmdlineTask.obj
 0003:0000a488       ??_R0?AVStateLockableTreeItem@U2@@@8 10062488     PhylipCmdlineTask.obj
 0003:0000a4b0       ??_R0?AVStateLockableItem@U2@@@8 100624b0     PhylipCmdlineTask.obj
 0003:0000a4d4       ??_R0?AVPhylipCmdlineTask@U2@@@8 100624d4     PhylipCmdlineTask.obj
 0003:0000a4f8       ??_R0?AVAbstractInt32Id@U2@@@8 100624f8     PhylipPlugin.obj
 0003:0000a51c       ??_R0?AV?$AbstractId@H@U2@@@8 1006251c     PhylipPlugin.obj
 0003:0000a53c       ??_R0?AVServiceType@U2@@@8 1006253c     PhylipPlugin.obj
 0003:0000a55c       ??_R0?AVTaskStarter@U2@@@8 1006255c     PhylipPlugin.obj
 0003:0000a57c       ??_R0?AVNeighborJoinAdapter@U2@@@8 1006257c     PhylipPlugin.obj
 0003:0000a5a4       ??_R0?AVPhyTreeGenerator@U2@@@8 100625a4     PhylipPlugin.obj
 0003:0000a5c8       ??_R0?AVPhylipPlugin@U2@@@8 100625c8     PhylipPlugin.obj
 0003:0000a5e8       ??_R0?AVPlugin@U2@@@8      100625e8     PhylipPlugin.obj
 0003:0000a600       ??_R0?AV?$GAutoDeleteList@VXMLTestFactory@U2@@@U2@@@8 10062600     PhylipPlugin.obj
 0003:0000a638       ??_R0?AVXmlTest@U2@@@8     10062638     PhylipPluginTests.obj
 0003:0000a654       ??_R0?AVGTest@U2@@@8       10062654     PhylipPluginTests.obj
 0003:0000a66c       ??_R0?AVXMLTestFactory@U2@@@8 1006266c     PhylipPluginTests.obj
 0003:0000a68c       ??_R0?AVPhyTreeGeneratorLauncherTask@U2@@@8 1006268c     PhylipPluginTests.obj
 0003:0000a6bc       ??_R0?AVGTest_NeighborJoin@U2@@@8 100626bc     PhylipPluginTests.obj
 0003:0000a6e0       ??_R0?AVGTest_NeighborJoinFactory@GTest_NeighborJoin@U2@@@8 100626e0     PhylipPluginTests.obj
 0003:0000a720       ??_R0?AVMultipleSequenceAlignmentObject@U2@@@8 10062720     PhylipTask.obj
 0003:0000a754       ??_R0?AVMultipleAlignmentObject@U2@@@8 10062754     PhylipTask.obj
 0003:0000a780       ??_R0?AVPhylipTask@U2@@@8  10062780     PhylipTask.obj
 0003:0000a79c       ??_R0?AVCmdlineTask@U2@@@8 1006279c     PhylipTask.obj
 0003:0000a7bc       ??_R0?AVMultipleSequenceAlignment@U2@@@8 100627bc     SeqBootAdapter.obj
 0003:0000a7e8       ??_R0?AVMultipleAlignment@U2@@@8 100627e8     SeqBootAdapter.obj
 0003:0000a80c       ??_R0PAX@8                 1006280c     phylip.obj
 0003:0000a81c       ??_R0?AVtype_info@@@8      1006281c     MSVCRT:ti_inst.obj
 0003:0000a884       ?id@?$num_put@DV?$back_insert_iterator@V?$basic_string@DU?$char_traits@D@std@@V?$allocator@D@2@@std@@@std@@@std@@2V0locale@2@A 10062884     DistanceMatrix.obj
 0003:0000a888       ?id@?$num_put@_WV?$back_insert_iterator@V?$basic_string@_WU?$char_traits@_W@std@@V?$allocator@_W@2@@std@@@std@@@std@@2V0locale@2@A 10062888     DistanceMatrix.obj
 0003:0000a8d4       ?runLock@NeighborJoinCalculateTreeTask@U2@@0VQMutex@@A 100628d4     NeighborJoinAdapter.obj
 0003:0000a948       ?MajorityRuleExt@ConsensusModelTypes@U2@@2VQString@@A 10062948     NeighborJoinWidget.obj
 0003:0000a96c       ?MajorityRule@ConsensusModelTypes@U2@@2VQString@@A 1006296c     NeighborJoinWidget.obj
 0003:0000a970       ?M1@ConsensusModelTypes@U2@@2VQString@@A 10062970     NeighborJoinWidget.obj
 0003:0000a974       ?Strict@ConsensusModelTypes@U2@@2VQString@@A 10062974     NeighborJoinWidget.obj
 0003:0000a994       ?FRACTION_ARG@PhylipCmdlineTask@U2@@2VQString@@B 10062994     PhylipCmdlineTask.obj
 0003:0000a9a8       ?TT_RATIO_ARG@PhylipCmdlineTask@U2@@2VQString@@B 100629a8     PhylipCmdlineTask.obj
 0003:0000a9ac       ?REPLICATES_ARG@PhylipCmdlineTask@U2@@2VQString@@B 100629ac     PhylipCmdlineTask.obj
 0003:0000a9b8       ?CONSENSUS_ARG@PhylipCmdlineTask@U2@@2VQString@@B 100629b8     PhylipCmdlineTask.obj
 0003:0000a9bc       ?GAMMA_ARG@PhylipCmdlineTask@U2@@2VQString@@B 100629bc     PhylipCmdlineTask.obj
 0003:0000a9e0       ?PHYLIP_CMDLINE@PhylipCmdlineTask@U2@@2VQString@@B 100629e0     PhylipCmdlineTask.obj
 0003:0000a9e4       ?SEED_ARG@PhylipCmdlineTask@U2@@2VQString@@B 100629e4     PhylipCmdlineTask.obj
 0003:0000a9e8       ?MATRIX_ARG@PhylipCmdlineTask@U2@@2VQString@@B 100629e8     PhylipCmdlineTask.obj
 0003:0000a9ec       ?BOOTSTRAP_ARG@PhylipCmdlineTask@U2@@2VQString@@B 100629ec     PhylipCmdlineTask.obj
 0003:0000a9f0       ?ALPHA_ARG@PhylipCmdlineTask@U2@@2VQString@@B 100629f0     PhylipCmdlineTask.obj
 0003:0000aa38       ?PHYLIP_NEIGHBOUR_JOIN@PhylipPlugin@U2@@2VQString@@B 10062a38     PhylipPlugin.obj
 0003:0000ab38       ?tree_pairing@@3HA         10062b38     cons.obj
 0003:0000ab3c       ?root@@3PAUnode@@A         10062b3c     cons.obj
 0003:0000ab40       ?numopts@@3JA              10062b40     cons.obj
 0003:0000ab44       ?outgrno_cons@@3JA         10062b44     cons.obj
 0003:0000ab48       ?col@@3JA                  10062b48     cons.obj
 0003:0000ab4c       ?setsz@@3JA                10062b4c     cons.obj
 0003:0000ab50       ?maxgrp@@3JA               10062b50     cons.obj
 0003:0000ab54       ?trout@@3EA                10062b54     cons.obj
 0003:0000ab55       ?firsttree@@3EA            10062b55     cons.obj
 0003:0000ab56       ?noroot@@3EA               10062b56     cons.obj
 0003:0000ab57       ?outgropt_cons@@3EA        10062b57     cons.obj
 0003:0000ab58       ?didreroot@@3EA            10062b58     cons.obj
 0003:0000ab59       ?prntsets@@3EA             10062b59     cons.obj
 0003:0000ab5a       ?treeprint_cons@@3EA       10062b5a     cons.obj
 0003:0000ab5b       ?goteof@@3EA               10062b5b     cons.obj
 0003:0000ab5c       ?strict@@3EA               10062b5c     cons.obj
 0003:0000ab5d       ?mr@@3EA                   10062b5d     cons.obj
 0003:0000ab5e       ?mre@@3EA                  10062b5e     cons.obj
 0003:0000ab5f       ?ml@@3EA                   10062b5f     cons.obj
 0003:0000ab60       ?nodep_cons@@3PAPAUnode@@A 10062b60     cons.obj
 0003:0000ab64       ?treenode@@3PAPAUnode@@A   10062b64     cons.obj
 0003:0000ab68       ?grouping@@3PAPAHA         10062b68     cons.obj
 0003:0000ab6c       ?grping2@@3PAPAHA          10062b6c     cons.obj
 0003:0000ab70       ?group2@@3PAPAHA           10062b70     cons.obj
 0003:0000ab74       ?lengths@@3PANA            10062b74     cons.obj
 0003:0000ab78       ?lengths2@@3PANA           10062b78     cons.obj
 0003:0000ab7c       ?order@@3PAPAJA            10062b7c     cons.obj
 0003:0000ab80       ?order2@@3PAPAJA           10062b80     cons.obj
 0003:0000ab84       ?lasti@@3JA                10062b84     cons.obj
 0003:0000ab88       ?fullset@@3PAHA            10062b88     cons.obj
 0003:0000ab8c       ?grbg@@3PAUnode@@A         10062b8c     cons.obj
 0003:0000ab90       ?tipy@@3JA                 10062b90     cons.obj
 0003:0000ab94       ?timesseen@@3PAPANA        10062b94     cons.obj
 0003:0000ab98       ?tmseen2@@3PAPANA          10062b98     cons.obj
 0003:0000ab9c       ?times2@@3PAPANA           10062b9c     cons.obj
 0003:0000aba0       ?tchange2@@3PANA           10062ba0     cons.obj
 0003:0000aba4       ?hashp@@3PAPAUnamenode@@A  10062ba4     cons.obj
 0003:0000aba8       ?trweight@@3NA             10062ba8     cons.obj
 0003:0000abb0       ?ntrees@@3NA               10062bb0     cons.obj
 0003:0000abb8       ?mlfrac@@3NA               10062bb8     cons.obj
 0003:0000ac10       ?infilename@@3PADA         10062c10     dnadist.obj
 0003:0000acd8       ?outfilename@@3PADA        10062cd8     dnadist.obj
 0003:0000ada0       ?catfilename@@3PADA        10062da0     dnadist.obj
 0003:0000ae68       ?weightfilename@@3PADA     10062e68     dnadist.obj
 0003:0000af30       ?sites@@3JA                10062f30     dnadist.obj
 0003:0000af34       ?categs@@3JA               10062f34     dnadist.obj
 0003:0000af38       ?weightsum@@3JA            10062f38     dnadist.obj
 0003:0000af3c       ?datasets@@3JA             10062f3c     dnadist.obj
 0003:0000af40       ?ith@@3JA                  10062f40     dnadist.obj
 0003:0000af44       ?rcategs@@3JA              10062f44     dnadist.obj
 0003:0000af48       ?freqsfrom@@3EA            10062f48     dnadist.obj
 0003:0000af49       ?jukes@@3EA                10062f49     dnadist.obj
 0003:0000af4a       ?kimura@@3EA               10062f4a     dnadist.obj
 0003:0000af4b       ?logdet@@3EA               10062f4b     dnadist.obj
 0003:0000af4c       ?gama@@3EA                 10062f4c     dnadist.obj
 0003:0000af4d       ?invar@@3EA                10062f4d     dnadist.obj
 0003:0000af4e       ?similarity@@3EA           10062f4e     dnadist.obj
 0003:0000af4f       ?lower@@3EA                10062f4f     dnadist.obj
 0003:0000af50       ?f84@@3EA                  10062f50     dnadist.obj
 0003:0000af51       ?weights@@3EA              10062f51     dnadist.obj
 0003:0000af52       ?progress@@3EA             10062f52     dnadist.obj
 0003:0000af53       ?ctgry@@3EA                10062f53     dnadist.obj
 0003:0000af54       ?mulsets@@3EA              10062f54     dnadist.obj
 0003:0000af55       ?justwts@@3EA              10062f55     dnadist.obj
 0003:0000af56       ?firstset@@3EA             10062f56     dnadist.obj
 0003:0000af57       ?baddists@@3EA             10062f57     dnadist.obj
 0003:0000af58       ?matrix_flags@@3EA         10062f58     dnadist.obj
 0003:0000af5c       ?nodep@@3PAPAUnode@@A      10062f5c     dnadist.obj
 0003:0000af60       ?xi@@3NA                   10062f60     dnadist.obj
 0003:0000af68       ?xv@@3NA                   10062f68     dnadist.obj
 0003:0000af70       ?ttratio@@3NA              10062f70     dnadist.obj
 0003:0000af78       ?ttratio0@@3NA             10062f78     dnadist.obj
 0003:0000af80       ?freqa@@3NA                10062f80     dnadist.obj
 0003:0000af88       ?freqc@@3NA                10062f88     dnadist.obj
 0003:0000af90       ?freqg@@3NA                10062f90     dnadist.obj
 0003:0000af98       ?freqt@@3NA                10062f98     dnadist.obj
 0003:0000afa0       ?freqr@@3NA                10062fa0     dnadist.obj
 0003:0000afa8       ?freqy@@3NA                10062fa8     dnadist.obj
 0003:0000afb0       ?freqar@@3NA               10062fb0     dnadist.obj
 0003:0000afb8       ?freqcy@@3NA               10062fb8     dnadist.obj
 0003:0000afc0       ?freqgr@@3NA               10062fc0     dnadist.obj
 0003:0000afc8       ?freqty@@3NA               10062fc8     dnadist.obj
 0003:0000afd0       ?cvi@@3NA                  10062fd0     dnadist.obj
 0003:0000afd8       ?invarfrac@@3NA            10062fd8     dnadist.obj
 0003:0000afe0       ?sumrates@@3NA             10062fe0     dnadist.obj
 0003:0000afe8       ?fracchange@@3NA           10062fe8     dnadist.obj
 0003:0000aff0       ?oldweight@@3PAJA          10062ff0     dnadist.obj
 0003:0000aff4       ?d@@3PAPANA                10062ff4     dnadist.obj
 0003:0000aff8       ?rate@@3PANA               10062ff8     dnadist.obj
 0003:0000b040       ?sumweightrat@@3NA         10063040     dnadist.obj
 0003:0000b048       ?weightrat@@3PANA          10063048     dnadist.obj
 0003:0000b050       ?tbl@@3PAUvalrec@@A        10063050     dnadist.obj
 0003:0000b24c       ?Kimura@DNADistModelTypes@@2VQString@@A 1006324c     dnadist.obj
 0003:0000b2e8       ?JukesCantor@DNADistModelTypes@@2VQString@@A 100632e8     dnadist.obj
 0003:0000b2ec       ?LogDet@DNADistModelTypes@@2VQString@@A 100632ec     dnadist.obj
 0003:0000b2f8       ?F84@DNADistModelTypes@@2VQString@@A 100632f8     dnadist.obj
 0003:0000b558       ?infile@@3PAU_iobuf@@A     10063558     phylip.obj
 0003:0000b55c       ?outfile@@3PAU_iobuf@@A    1006355c     phylip.obj
 0003:0000b560       ?intree@@3PAU_iobuf@@A     10063560     phylip.obj
 0003:0000b564       ?intree2@@3PAU_iobuf@@A    10063564     phylip.obj
 0003:0000b568       ?outtree@@3PAU_iobuf@@A    10063568     phylip.obj
 0003:0000b56c       ?weightfile@@3PAU_iobuf@@A 1006356c     phylip.obj
 0003:0000b570       ?catfile@@3PAU_iobuf@@A    10063570     phylip.obj
 0003:0000b574       ?ancfile@@3PAU_iobuf@@A    10063574     phylip.obj
 0003:0000b57d       ?ibmpc@@3EA                1006357d     phylip.obj
 0003:0000b57e       ?ansi@@3EA                 1006357e     phylip.obj
 0003:0000b57f       ?tranvsp@@3EA              1006357f     phylip.obj
 0003:0000b580       ?mixfile@@3PAU_iobuf@@A    10063580     phylip.obj
 0003:0000b584       ?factfile@@3PAU_iobuf@@A   10063584     phylip.obj
 0003:0000b588       ?spp@@3JA                  10063588     phylip.obj
 0003:0000b58c       ?words@@3JA                1006358c     phylip.obj
 0003:0000b590       ?bits@@3JA                 10063590     phylip.obj
 0003:0000b594       ?nayme@@3PAY0BO@DA         10063594     phylip.obj
 0003:0000b598       ?savecsbi@@3U_CONSOLE_SCREEN_BUFFER_INFO@@A 10063598     phylip.obj
 0003:0000b5ae       ?savecsbi_valid@@3EA       100635ae     phylip.obj
 0003:0000b5b0       ?hConsoleOutput@@3PAXA     100635b0     phylip.obj
 0003:0000b600       ___isa_available_default   10063600     phylip.obj
 0003:0000b608       ?chars@@3JA                10063608     protdist.obj
 0003:0000b60c       ?basesequal@@3EA           1006360c     protdist.obj
 0003:0000b60d       ?usepmb@@3EA               1006360d     protdist.obj
 0003:0000b60e       ?usejtt@@3EA               1006360e     protdist.obj
 0003:0000b60f       ?usepam@@3EA               1006360f     protdist.obj
 0003:0000b610       ?ease@@3NA                 10063610     protdist.obj
 0003:0000b618       ?whichcode@@3W4codetype@@A 10063618     protdist.obj
 0003:0000b61c       ?whichcat@@3W4cattype@@A   1006361c     protdist.obj
 0003:0000b620       ?gnode@@3PAPAW4aas@@A      10063620     protdist.obj
 0003:0000b628       ?trans@@3PAY133W4aas@@A    10063628     protdist.obj
 0003:0000b728       ?pie@@3PANA                10063728     protdist.obj
 0003:0000b7c8       ?cat@@3PAJA                100637c8     protdist.obj
 0003:0000b830       ?numaa@@3PAJA              10063830     protdist.obj
 0003:0000b898       ?eig@@3PANA                10063898     protdist.obj
 0003:0000b938       ?prob@@3PAY0BE@NA          10063938     protdist.obj
 0003:0000c5b8       ?eigvecs@@3PAY0BE@NA       100645b8     protdist.obj
 0003:0000d238       ?tt@@3NA                   10065238     protdist.obj
 0003:0000d240       ?p@@3NA                    10065240     protdist.obj
 0003:0000d248       ?dp@@3NA                   10065248     protdist.obj
 0003:0000d250       ?d2p@@3NA                  10065250     protdist.obj
 0003:0000d258       ?q@@3NA                    10065258     protdist.obj
 0003:0000d260       ?elambdat@@3NA             10065260     protdist.obj
 0003:0000d2a4       ?PAM@ProtDistModelTypes@@2VQString@@A 100652a4     protdist.obj
 0003:0000d2b0       ?JTT@ProtDistModelTypes@@2VQString@@A 100652b0     protdist.obj
 0003:0000d2b4       ?PMB@ProtDistModelTypes@@2VQString@@A 100652b4     protdist.obj
 0003:0000d2c0       ?Kimura@ProtDistModelTypes@@2VQString@@A 100652c0     protdist.obj
 0003:0000d2cc       ?nonodes@@3JA              100652cc     seq.obj
 0003:0000d2d0       ?endsite@@3JA              100652d0     seq.obj
 0003:0000d2d4       ?outgrno@@3JA              100652d4     seq.obj
 0003:0000d2d8       ?nextree@@3JA              100652d8     seq.obj
 0003:0000d2dc       ?which@@3JA                100652dc     seq.obj
 0003:0000d2e0       ?interleaved@@3EA          100652e0     seq.obj
 0003:0000d2e1       ?printdata@@3EA            100652e1     seq.obj
 0003:0000d2e2       ?outgropt@@3EA             100652e2     seq.obj
 0003:0000d2e3       ?treeprint@@3EA            100652e3     seq.obj
 0003:0000d2e4       ?dotdiff@@3EA              100652e4     seq.obj
 0003:0000d2e5       ?transvp@@3EA              100652e5     seq.obj
 0003:0000d2e8       ?weight@@3PAJA             100652e8     seq.obj
 0003:0000d2ec       ?category@@3PAJA           100652ec     seq.obj
 0003:0000d2f0       ?alias@@3PAJA              100652f0     seq.obj
 0003:0000d2f4       ?location@@3PAJA           100652f4     seq.obj
 0003:0000d2f8       ?ally@@3PAJA               100652f8     seq.obj
 0003:0000d2fc       ?y@@3PAPADA                100652fc     seq.obj
 0003:0000d308       ?seed_boot@@3PAJA          10065308     seqboot.obj
 0003:0000d320       ?loci@@3JA                 10065320     seqboot.obj
 0003:0000d324       ?maxalleles@@3JA           10065324     seqboot.obj
 0003:0000d328       ?groups@@3JA               10065328     seqboot.obj
 0003:0000d32c       ?nenzymes@@3JA             1006532c     seqboot.obj
 0003:0000d330       ?reps@@3JA                 10065330     seqboot.obj
 0003:0000d334       ?ws@@3JA                   10065334     seqboot.obj
 0003:0000d338       ?blocksize@@3JA            10065338     seqboot.obj
 0003:0000d33c       ?maxnewsites@@3JA          1006533c     seqboot.obj
 0003:0000d340       ?nodep_boot@@3PAPADA       10065340     seqboot.obj
 0003:0000d348       ?factor@@3PADA             10065348     seqboot.obj
 0003:0000d34c       ?factorr@@3PAJA            1006534c     seqboot.obj
 0003:0000d350       ?alleles@@3PAJA            10065350     seqboot.obj
 0003:0000d354       ?newsites@@3JA             10065354     seqboot.obj
 0003:0000d358       ?newgroups@@3JA            10065358     seqboot.obj
 0003:0000d35c       ?newwhere@@3PAJA           1006535c     seqboot.obj
 0003:0000d360       ?newhowmany@@3PAJA         10065360     seqboot.obj
 0003:0000d364       ?newersites@@3JA           10065364     seqboot.obj
 0003:0000d368       ?newergroups@@3JA          10065368     seqboot.obj
 0003:0000d36c       ?newerfactor@@3PAJA        1006536c     seqboot.obj
 0003:0000d370       ?newerwhere@@3PAJA         10065370     seqboot.obj
 0003:0000d374       ?newerhowmany@@3PAJA       10065374     seqboot.obj
 0003:0000d378       ?charorder@@3PAPAJA        10065378     seqboot.obj
 0003:0000d37c       ?sppord@@3PAPAJA           1006537c     seqboot.obj
 0003:0000e100       ___isa_available           10066100     MSVCRT:cpu_disp.obj
 0003:0000e104       ___favor                   10066104     MSVCRT:cpu_disp.obj
 0003:0000e10c       ?__type_info_root_node@@3U__type_info_node@@A 1006610c     MSVCRT:tncleanup.obj
 0003:0000e114       ___native_startup_lock     10066114     <common>
 0003:0000e118       ___native_startup_state    10066118     <common>
 0003:0000e11c       ___dyn_tls_init_callback   1006611c     <common>
 0003:0000e120       ___onexitend               10066120     <common>
 0003:0000e124       ___onexitbegin             10066124     <common>

 entry point at        0001:0003a8b7

 Static symbols

 0001:fffff000       __unwindfunclet$?append@?$QList@VQString@@@@QAEXABVQString@@@Z$7 10000000 f   PhylipCmdlineTask.obj
 0000:fff90000       .debug$S                   10000000     MSVCRT:MSVCR120.dll
 0000:fff90000       .debug$S                   10000000     MSVCRT:MSVCR120.dll
 0000:fff90000       .debug$S                   10000000     MSVCRT:MSVCR120.dll
 0000:fff90000       .debug$S                   10000000     MSVCRT:MSVCR120.dll
 0000:fff90000       .debug$S                   10000000     MSVCRT:MSVCR120.dll
 0000:fff90000       .debug$S                   10000000     MSVCRT:MSVCR120.dll
 0000:fff90000       .debug$S                   10000000     MSVCRT:MSVCR120.dll
 0000:fff90000       .debug$S                   10000000     MSVCRT:MSVCR120.dll
 0000:fff90000       .debug$S                   10000000     MSVCRT:MSVCR120.dll
 0000:fff90000       .debug$S                   10000000     MSVCRT:MSVCR120.dll
 0000:fff90000       .debug$S                   10000000     MSVCRT:MSVCR120.dll
 0000:fff90000       .debug$S                   10000000     MSVCRT:MSVCR120.dll
 0000:fff90000       .debug$S                   10000000     MSVCRT:MSVCR120.dll
 0000:fff90000       .debug$S                   10000000     MSVCRT:MSVCR120.dll
 0000:fff90000       .debug$S                   10000000     MSVCRT:MSVCR120.dll
 0000:fff90000       .debug$S                   10000000     MSVCRT:MSVCR120.dll
 0000:fff90000       .debug$S                   10000000     MSVCRT:MSVCR120.dll
 0000:fff90000       .debug$S                   10000000     MSVCRT:MSVCR120.dll
 0000:fff90000       .debug$S                   10000000     MSVCRT:MSVCR120.dll
 0000:fff90000       .debug$S                   10000000     MSVCRT:MSVCR120.dll
 0000:fff90000       .debug$S                   10000000     MSVCRT:MSVCR120.dll
 0000:fff90000       .debug$S                   10000000     MSVCRT:MSVCR120.dll
 0000:fff90000       .debug$S                   10000000     MSVCRT:MSVCR120.dll
 0000:fff90000       .debug$S                   10000000     MSVCRT:MSVCR120.dll
 0000:fff90000       .debug$S                   10000000     MSVCRT:MSVCR120.dll
 0000:fff90000       .debug$S                   10000000     MSVCRT:MSVCR120.dll
 0000:fff90000       .debug$S                   10000000     MSVCRT:MSVCR120.dll
 0000:fff90000       .debug$S                   10000000     MSVCRT:MSVCR120.dll
 0000:fff90000       .debug$S                   10000000     MSVCRT:MSVCR120.dll
 0000:fff90000       .debug$S                   10000000     MSVCRT:MSVCR120.dll
 0000:fff90000       .debug$S                   10000000     MSVCRT:MSVCR120.dll
 0000:fff90000       .debug$S                   10000000     MSVCRT:MSVCR120.dll
 0000:fff90000       .debug$S                   10000000     MSVCRT:MSVCR120.dll
 0001:fffff000       __ehhandler$?_Copy@?$basic_string@DU?$char_traits@D@std@@V?$allocator@D@2@@std@@QAEXII@Z 10000000 f   moc_PhylipTask.obj
 0000:fff90000       .debug$S                   10000000     MSVCRT:MSVCR120.dll
 0000:fff90000       .debug$S                   10000000     MSVCRT:MSVCR120.dll
 0000:fff90000       .debug$S                   10000000     MSVCRT:MSVCR120.dll
 0000:fff90000       .debug$S                   10000000     MSVCRT:MSVCR120.dll
 0000:fff90000       .debug$S                   10000000     MSVCRT:MSVCR120.dll
 0000:fff90000       .debug$S                   10000000     MSVCRT:MSVCR120.dll
 0000:fff90000       .debug$S                   10000000     MSVCRT:MSVCR120.dll
 0000:fff90000       .debug$S                   10000000     MSVCRT:MSVCR120.dll
 0000:fff90000       .debug$S                   10000000     MSVCRT:MSVCR120.dll
 0000:fff90000       .debug$S                   10000000     MSVCRT:MSVCR120.dll
 0000:fff90000       .debug$S                   10000000     MSVCRT:MSVCR120.dll
 0000:fff90000       .debug$S                   10000000     MSVCRT:MSVCR120.dll
 0000:fff90000       .debug$S                   10000000     MSVCRT:MSVCR120.dll
 0000:fff90000       .debug$S                   10000000     MSVCRT:MSVCR120.dll
 0000:fff90000       .debug$S                   10000000     MSVCRT:MSVCR120.dll
 0000:fff90000       .debug$S                   10000000     MSVCRT:MSVCR120.dll
 0000:fff90000       .debug$S                   10000000     MSVCRT:MSVCR120.dll
 0000:fff90000       .debug$S                   10000000     MSVCRT:MSVCR120.dll
 0000:fff90000       .debug$S                   10000000     MSVCRT:MSVCR120.dll
 0000:fff90000       .debug$S                   10000000     MSVCRT:MSVCR120.dll
 0000:fff90000       .debug$S                   10000000     MSVCRT:MSVCR120.dll
 0000:fff90000       .debug$S                   10000000     MSVCRT:MSVCR120.dll
 0000:fff90000       .debug$S                   10000000     MSVCRT:MSVCR120.dll
 0000:fff90000       .debug$S                   10000000     MSVCRT:MSVCR120.dll
 0002:fffbe000       __catchsym$?_Copy@?$basic_string@DU?$char_traits@D@std@@V?$allocator@D@2@@std@@QAEXII@Z$5 10000000     moc_PhylipTask.obj
 0000:fff90000       .debug$S                   10000000     MSVCRT:MSVCR120.dll
 0000:fff90000       .debug$S                   10000000     MSVCRT:MSVCR120.dll
 0000:fff90000       .debug$S                   10000000     MSVCRT:MSVCR120.dll
 0000:fff90000       .debug$S                   10000000     MSVCRT:MSVCR120.dll
 0000:fff90000       .debug$S                   10000000     MSVCRT:MSVCR120.dll
 0000:fff90000       .debug$S                   10000000     MSVCRT:MSVCR120.dll
 0000:fff90000       .debug$S                   10000000     MSVCRT:MSVCR120.dll
 0000:fff90000       .debug$S                   10000000     MSVCRT:MSVCR120.dll
 0000:fff90000       .debug$S                   10000000     MSVCRT:MSVCR120.dll
 0000:fff90000       .debug$S                   10000000     MSVCRT:MSVCR120.dll
 0000:fff90000       .debug$S                   10000000     MSVCRT:MSVCR120.dll
 0000:fff90000       .debug$S                   10000000     MSVCRT:MSVCR120.dll
 0000:fff90000       .debug$S                   10000000     MSVCRT:MSVCR120.dll
 0000:fff90000       .debug$S                   10000000     MSVCRT:MSVCR120.dll
 0000:fff90000       .debug$S                   10000000     MSVCRT:MSVCR120.dll
 0000:fff90000       .debug$S                   10000000     msvcprt:MSVCP120.dll
 0000:fff90000       .debug$S                   10000000     msvcprt:MSVCP120.dll
 0000:fff90000       .debug$S                   10000000     msvcprt:MSVCP120.dll
 0000:fff90000       .debug$S                   10000000     msvcprt:MSVCP120.dll
 0000:fff90000       .debug$S                   10000000     msvcprt:MSVCP120.dll
 0000:fff90000       .debug$S                   10000000     msvcprt:MSVCP120.dll
 0000:fff90000       .debug$S                   10000000     msvcprt:MSVCP120.dll
 0000:fff90000       .debug$S                   10000000     msvcprt:MSVCP120.dll
 0000:fff90000       .debug$S                   10000000     msvcprt:MSVCP120.dll
 0000:fff90000       .debug$S                   10000000     msvcprt:MSVCP120.dll
 0000:fff90000       .debug$S                   10000000     msvcprt:MSVCP120.dll
 0000:fff90000       .debug$S                   10000000     msvcprt:MSVCP120.dll
 0000:fff90000       .debug$S                   10000000     msvcprt:MSVCP120.dll
 0000:fff90000       .debug$S                   10000000     msvcprt:MSVCP120.dll
 0000:fff90000       .debug$S                   10000000     msvcprt:MSVCP120.dll
 0000:fff90000       .debug$S                   10000000     msvcprt:MSVCP120.dll
 0000:fff90000       .debug$S                   10000000     msvcprt:MSVCP120.dll
 0000:fff90000       .debug$S                   10000000     kernel32:KERNEL32.dll
 0000:fff90000       .debug$S                   10000000     kernel32:KERNEL32.dll
 0000:fff90000       .debug$S                   10000000     kernel32:KERNEL32.dll
 0000:fff90000       .debug$S                   10000000     kernel32:KERNEL32.dll
 0000:fff90000       .debug$S                   10000000     kernel32:KERNEL32.dll
 0000:fff90000       .debug$S                   10000000     kernel32:KERNEL32.dll
 0000:fff90000       .debug$S                   10000000     kernel32:KERNEL32.dll
 0000:fff90000       .debug$S                   10000000     kernel32:KERNEL32.dll
 0000:fff90000       .debug$S                   10000000     kernel32:KERNEL32.dll
 0002:fffbe000       ?_Generic_object$initializer$@?$_Error_objects@H@std@@2P6AXXZA 10000000     moc_PhylipTask.obj
 0002:fffbe000       ?_Iostream_object$initializer$@?$_Error_objects@H@std@@2P6AXXZA 10000000     moc_PhylipTask.obj
 0002:fffbe000       ?_System_object$initializer$@?$_Error_objects@H@std@@2P6AXXZA 10000000     moc_PhylipTask.obj
 0000:fff90000       .debug$S                   10000000     kernel32:KERNEL32.dll
 0000:fff90000       .debug$S                   10000000     kernel32:KERNEL32.dll
 0000:fff90000       .debug$S                   10000000     kernel32:KERNEL32.dll
 0000:fff90000       .debug$S                   10000000     kernel32:KERNEL32.dll
 0000:fff90000       .debug$S                   10000000     kernel32:KERNEL32.dll
 0000:fff90000       .debug$S                   10000000     kernel32:KERNEL32.dll
 0000:fff90000       .debug$S                   10000000     Qt5Core:Qt5Core.dll
 0000:fff90000       .debug$S                   10000000     Qt5Core:Qt5Core.dll
 0000:fff90000       .debug$S                   10000000     Qt5Core:Qt5Core.dll
 0000:fff90000       .debug$S                   10000000     Qt5Core:Qt5Core.dll
 0000:fff90000       .debug$S                   10000000     Qt5Core:Qt5Core.dll
 0000:fff90000       .debug$S                   10000000     Qt5Core:Qt5Core.dll
 0000:fff90000       .debug$S                   10000000     Qt5Core:Qt5Core.dll
 0000:fff90000       .debug$S                   10000000     Qt5Core:Qt5Core.dll
 0000:fff90000       .debug$S                   10000000     Qt5Core:Qt5Core.dll
 0000:fff90000       .debug$S                   10000000     Qt5Core:Qt5Core.dll
 0000:fff90000       .debug$S                   10000000     Qt5Core:Qt5Core.dll
 0000:fff90000       .debug$S                   10000000     Qt5Core:Qt5Core.dll
 0000:fff90000       .debug$S                   10000000     Qt5Core:Qt5Core.dll
 0000:fff90000       .debug$S                   10000000     Qt5Core:Qt5Core.dll
 0000:fff90000       .debug$S                   10000000     Qt5Core:Qt5Core.dll
 0000:fff90000       .debug$S                   10000000     Qt5Core:Qt5Core.dll
 0000:fff90000       .debug$S                   10000000     Qt5Core:Qt5Core.dll
 0000:fff90000       .debug$S                   10000000     Qt5Core:Qt5Core.dll
 0000:fff90000       .debug$S                   10000000     Qt5Core:Qt5Core.dll
 0000:fff90000       .debug$S                   10000000     Qt5Core:Qt5Core.dll
 0000:fff90000       .debug$S                   10000000     Qt5Core:Qt5Core.dll
 0001:fffff000       __ehhandler$?_Copy@?$basic_string@DU?$char_traits@D@std@@V?$allocator@D@2@@std@@QAEXII@Z 10000000 f   moc_PhylipPluginTests.obj
 0000:fff90000       .debug$S                   10000000     Qt5Core:Qt5Core.dll
 0000:fff90000       .debug$S                   10000000     Qt5Core:Qt5Core.dll
 0000:fff90000       .debug$S                   10000000     Qt5Core:Qt5Core.dll
 0000:fff90000       .debug$S                   10000000     Qt5Core:Qt5Core.dll
 0000:fff90000       .debug$S                   10000000     Qt5Core:Qt5Core.dll
 0000:fff90000       .debug$S                   10000000     Qt5Core:Qt5Core.dll
 0000:fff90000       .debug$S                   10000000     Qt5Core:Qt5Core.dll
 0000:fff90000       .debug$S                   10000000     Qt5Core:Qt5Core.dll
 0000:fff90000       .debug$S                   10000000     Qt5Core:Qt5Core.dll
 0000:fff90000       .debug$S                   10000000     Qt5Core:Qt5Core.dll
 0000:fff90000       .debug$S                   10000000     Qt5Core:Qt5Core.dll
 0000:fff90000       .debug$S                   10000000     Qt5Core:Qt5Core.dll
 0000:fff90000       .debug$S                   10000000     Qt5Core:Qt5Core.dll
 0000:fff90000       .debug$S                   10000000     Qt5Core:Qt5Core.dll
 0000:fff90000       .debug$S                   10000000     Qt5Core:Qt5Core.dll
 0000:fff90000       .debug$S                   10000000     Qt5Core:Qt5Core.dll
 0000:fff90000       .debug$S                   10000000     Qt5Core:Qt5Core.dll
 0000:fff90000       .debug$S                   10000000     Qt5Core:Qt5Core.dll
 0000:fff90000       .debug$S                   10000000     Qt5Core:Qt5Core.dll
 0000:fff90000       .debug$S                   10000000     Qt5Core:Qt5Core.dll
 0000:fff90000       .debug$S                   10000000     Qt5Core:Qt5Core.dll
 0000:fff90000       .debug$S                   10000000     Qt5Core:Qt5Core.dll
 0000:fff90000       .debug$S                   10000000     Qt5Core:Qt5Core.dll
 0000:fff90000       .debug$S                   10000000     Qt5Core:Qt5Core.dll
 0002:fffbe000       __catchsym$?_Copy@?$basic_string@DU?$char_traits@D@std@@V?$allocator@D@2@@std@@QAEXII@Z$5 10000000     moc_PhylipPluginTests.obj
 0000:fff90000       .debug$S                   10000000     Qt5Core:Qt5Core.dll
 0000:fff90000       .debug$S                   10000000     Qt5Core:Qt5Core.dll
 0000:fff90000       .debug$S                   10000000     Qt5Core:Qt5Core.dll
 0000:fff90000       .debug$S                   10000000     Qt5Core:Qt5Core.dll
 0000:fff90000       .debug$S                   10000000     Qt5Core:Qt5Core.dll
 0000:fff90000       .debug$S                   10000000     Qt5Core:Qt5Core.dll
 0000:fff90000       .debug$S                   10000000     Qt5Core:Qt5Core.dll
 0000:fff90000       .debug$S                   10000000     Qt5Core:Qt5Core.dll
 0000:fff90000       .debug$S                   10000000     Qt5Core:Qt5Core.dll
 0000:fff90000       .debug$S                   10000000     Qt5Core:Qt5Core.dll
 0000:fff90000       .debug$S                   10000000     Qt5Core:Qt5Core.dll
 0000:fff90000       .debug$S                   10000000     Qt5Core:Qt5Core.dll
 0000:fff90000       .debug$S                   10000000     Qt5Core:Qt5Core.dll
 0000:fff90000       .debug$S                   10000000     Qt5Core:Qt5Core.dll
 0000:fff90000       .debug$S                   10000000     Qt5Core:Qt5Core.dll
 0000:fff90000       .debug$S                   10000000     Qt5Core:Qt5Core.dll
 0000:fff90000       .debug$S                   10000000     Qt5Core:Qt5Core.dll
 0000:fff90000       .debug$S                   10000000     Qt5Core:Qt5Core.dll
 0000:fff90000       .debug$S                   10000000     Qt5Core:Qt5Core.dll
 0000:fff90000       .debug$S                   10000000     Qt5Core:Qt5Core.dll
 0000:fff90000       .debug$S                   10000000     Qt5Core:Qt5Core.dll
 0000:fff90000       .debug$S                   10000000     Qt5Core:Qt5Core.dll
 0000:fff90000       .debug$S                   10000000     Qt5Core:Qt5Core.dll
 0000:fff90000       .debug$S                   10000000     Qt5Core:Qt5Core.dll
 0000:fff90000       .debug$S                   10000000     Qt5Core:Qt5Core.dll
 0000:fff90000       .debug$S                   10000000     Qt5Core:Qt5Core.dll
 0000:fff90000       .debug$S                   10000000     Qt5Core:Qt5Core.dll
 0000:fff90000       .debug$S                   10000000     Qt5Core:Qt5Core.dll
 0000:fff90000       .debug$S                   10000000     Qt5Core:Qt5Core.dll
 0000:fff90000       .debug$S                   10000000     Qt5Core:Qt5Core.dll
 0000:fff90000       .debug$S                   10000000     Qt5Core:Qt5Core.dll
 0000:fff90000       .debug$S                   10000000     Qt5Core:Qt5Core.dll
 0000:fff90000       .debug$S                   10000000     Qt5Core:Qt5Core.dll
 0000:fff90000       .debug$S                   10000000     Qt5Core:Qt5Core.dll
 0000:fff90000       .debug$S                   10000000     Qt5Core:Qt5Core.dll
 0000:fff90000       .debug$S                   10000000     Qt5Core:Qt5Core.dll
 0000:fff90000       .debug$S                   10000000     Qt5Core:Qt5Core.dll
 0000:fff90000       .debug$S                   10000000     Qt5Core:Qt5Core.dll
 0000:fff90000       .debug$S                   10000000     Qt5Core:Qt5Core.dll
 0000:fff90000       .debug$S                   10000000     Qt5Core:Qt5Core.dll
 0000:fff90000       .debug$S                   10000000     Qt5Core:Qt5Core.dll
 0002:fffbe000       ?_Generic_object$initializer$@?$_Error_objects@H@std@@2P6AXXZA 10000000     moc_PhylipPluginTests.obj
 0002:fffbe000       ?_Iostream_object$initializer$@?$_Error_objects@H@std@@2P6AXXZA 10000000     moc_PhylipPluginTests.obj
 0002:fffbe000       ?_System_object$initializer$@?$_Error_objects@H@std@@2P6AXXZA 10000000     moc_PhylipPluginTests.obj
 0000:fff90000       .debug$S                   10000000     Qt5Core:Qt5Core.dll
 0000:fff90000       .debug$S                   10000000     Qt5Core:Qt5Core.dll
 0000:fff90000       .debug$S                   10000000     Qt5Core:Qt5Core.dll
 0000:fff90000       .debug$S                   10000000     Qt5Core:Qt5Core.dll
 0000:fff90000       .debug$S                   10000000     Qt5Core:Qt5Core.dll
 0000:fff90000       .debug$S                   10000000     Qt5Core:Qt5Core.dll
 0000:fff90000       .debug$S                   10000000     Qt5Core:Qt5Core.dll
 0000:fff90000       .debug$S                   10000000     Qt5Core:Qt5Core.dll
 0000:fff90000       .debug$S                   10000000     Qt5Core:Qt5Core.dll
 0000:fff90000       .debug$S                   10000000     Qt5Core:Qt5Core.dll
 0000:fff90000       .debug$S                   10000000     Qt5Core:Qt5Core.dll
 0000:fff90000       .debug$S                   10000000     Qt5Core:Qt5Core.dll
 0000:fff90000       .debug$S                   10000000     Qt5Core:Qt5Core.dll
 0000:fff90000       .debug$S                   10000000     Qt5Core:Qt5Core.dll
 0000:fff90000       .debug$S                   10000000     Qt5Core:Qt5Core.dll
 0000:fff90000       .debug$S                   10000000     Qt5Core:Qt5Core.dll
 0000:fff90000       .debug$S                   10000000     Qt5Core:Qt5Core.dll
 0000:fff90000       .debug$S                   10000000     Qt5Core:Qt5Core.dll
 0000:fff90000       .debug$S                   10000000     Qt5Core:Qt5Core.dll
 0000:fff90000       .debug$S                   10000000     Qt5Core:Qt5Core.dll
 0000:fff90000       .debug$S                   10000000     Qt5Core:Qt5Core.dll
 0000:fff90000       .debug$S                   10000000     Qt5Core:Qt5Core.dll
 0000:fff90000       .debug$S                   10000000     Qt5Core:Qt5Core.dll
 0000:fff90000       .debug$S                   10000000     Qt5Xml:Qt5Xml.dll
 0000:fff90000       .debug$S                   10000000     Qt5Widgets:Qt5Widgets.dll
 0000:fff90000       .debug$S                   10000000     Qt5Widgets:Qt5Widgets.dll
 0000:fff90000       .debug$S                   10000000     Qt5Widgets:Qt5Widgets.dll
 0000:fff90000       .debug$S                   10000000     Qt5Widgets:Qt5Widgets.dll
 0000:fff90000       .debug$S                   10000000     Qt5Widgets:Qt5Widgets.dll
 0000:fff90000       .debug$S                   10000000     Qt5Widgets:Qt5Widgets.dll
 0000:fff90000       .debug$S                   10000000     Qt5Widgets:Qt5Widgets.dll
 0000:fff90000       .debug$S                   10000000     Qt5Widgets:Qt5Widgets.dll
 0000:fff90000       .debug$S                   10000000     Qt5Widgets:Qt5Widgets.dll
 0000:fff90000       .debug$S                   10000000     Qt5Widgets:Qt5Widgets.dll
 0000:fff90000       .debug$S                   10000000     Qt5Widgets:Qt5Widgets.dll
 0001:fffff000       __ehhandler$?_Copy@?$basic_string@DU?$char_traits@D@std@@V?$allocator@D@2@@std@@QAEXII@Z 10000000 f   moc_PhylipPlugin.obj
 0000:fff90000       .debug$S                   10000000     Qt5Widgets:Qt5Widgets.dll
 0000:fff90000       .debug$S                   10000000     Qt5Widgets:Qt5Widgets.dll
 0000:fff90000       .debug$S                   10000000     Qt5Widgets:Qt5Widgets.dll
 0000:fff90000       .debug$S                   10000000     Qt5Widgets:Qt5Widgets.dll
 0000:fff90000       .debug$S                   10000000     Qt5Widgets:Qt5Widgets.dll
 0000:fff90000       .debug$S                   10000000     Qt5Widgets:Qt5Widgets.dll
 0002:fffbe000       __catchsym$?_Copy@?$basic_string@DU?$char_traits@D@std@@V?$allocator@D@2@@std@@QAEXII@Z$5 10000000     moc_PhylipPlugin.obj
 0000:fff90000       .debug$S                   10000000     Qt5Widgets:Qt5Widgets.dll
 0000:fff90000       .debug$S                   10000000     Qt5Widgets:Qt5Widgets.dll
 0000:fff90000       .debug$S                   10000000     Qt5Widgets:Qt5Widgets.dll
 0000:fff90000       .debug$S                   10000000     Qt5Widgets:Qt5Widgets.dll
 0000:fff90000       .debug$S                   10000000     Qt5Widgets:Qt5Widgets.dll
 0000:fff90000       .debug$S                   10000000     Qt5Widgets:Qt5Widgets.dll
 0000:fff90000       .debug$S                   10000000     Qt5Widgets:Qt5Widgets.dll
 0000:fff90000       .debug$S                   10000000     Qt5Widgets:Qt5Widgets.dll
 0000:fff90000       .debug$S                   10000000     Qt5Widgets:Qt5Widgets.dll
 0000:fff90000       .debug$S                   10000000     Qt5Widgets:Qt5Widgets.dll
 0000:fff90000       .debug$S                   10000000     Qt5Widgets:Qt5Widgets.dll
 0000:fff90000       .debug$S                   10000000     Qt5Widgets:Qt5Widgets.dll
 0000:fff90000       .debug$S                   10000000     Qt5Widgets:Qt5Widgets.dll
 0000:fff90000       .debug$S                   10000000     Qt5Widgets:Qt5Widgets.dll
 0000:fff90000       .debug$S                   10000000     Qt5Widgets:Qt5Widgets.dll
 0000:fff90000       .debug$S                   10000000     Qt5Widgets:Qt5Widgets.dll
 0000:fff90000       .debug$S                   10000000     Qt5Widgets:Qt5Widgets.dll
 0000:fff90000       .debug$S                   10000000     Qt5Widgets:Qt5Widgets.dll
 0000:fff90000       .debug$S                   10000000     Qt5Widgets:Qt5Widgets.dll
 0000:fff90000       .debug$S                   10000000     Qt5Widgets:Qt5Widgets.dll
 0000:fff90000       .debug$S                   10000000     Qt5Widgets:Qt5Widgets.dll
 0000:fff90000       .debug$S                   10000000     Qt5Widgets:Qt5Widgets.dll
 0000:fff90000       .debug$S                   10000000     Qt5Widgets:Qt5Widgets.dll
 0000:fff90000       .debug$S                   10000000     Qt5Widgets:Qt5Widgets.dll
 0000:fff90000       .debug$S                   10000000     Qt5Widgets:Qt5Widgets.dll
 0000:fff90000       .debug$S                   10000000     Qt5Widgets:Qt5Widgets.dll
 0000:fff90000       .debug$S                   10000000     Qt5Widgets:Qt5Widgets.dll
 0000:fff90000       .debug$S                   10000000     Qt5Widgets:Qt5Widgets.dll
 0000:fff90000       .debug$S                   10000000     Qt5Widgets:Qt5Widgets.dll
 0000:fff90000       .debug$S                   10000000     Qt5Widgets:Qt5Widgets.dll
 0000:fff90000       .debug$S                   10000000     Qt5Widgets:Qt5Widgets.dll
 0002:fffbe000       ?_Generic_object$initializer$@?$_Error_objects@H@std@@2P6AXXZA 10000000     moc_PhylipPlugin.obj
 0002:fffbe000       ?_Iostream_object$initializer$@?$_Error_objects@H@std@@2P6AXXZA 10000000     moc_PhylipPlugin.obj
 0002:fffbe000       ?_System_object$initializer$@?$_Error_objects@H@std@@2P6AXXZA 10000000     moc_PhylipPlugin.obj
 0000:fff90000       .debug$S                   10000000     Qt5Widgets:Qt5Widgets.dll
 0000:fff90000       .debug$S                   10000000     Qt5Widgets:Qt5Widgets.dll
 0000:fff90000       .debug$S                   10000000     Qt5Widgets:Qt5Widgets.dll
 0000:fff90000       .debug$S                   10000000     Qt5Widgets:Qt5Widgets.dll
 0000:fff90000       .debug$S                   10000000     Qt5Widgets:Qt5Widgets.dll
 0000:fff90000       .debug$S                   10000000     Qt5Widgets:Qt5Widgets.dll
 0000:fff90000       .debug$S                   10000000     Qt5Widgets:Qt5Widgets.dll
 0000:fff90000       .debug$S                   10000000     Qt5Widgets:Qt5Widgets.dll
 0000:fff90000       .debug$S                   10000000     Qt5Widgets:Qt5Widgets.dll
 0000:fff90000       .debug$S                   10000000     Qt5Widgets:Qt5Widgets.dll
 0000:fff90000       .debug$S                   10000000     Qt5Widgets:Qt5Widgets.dll
 0000:fff90000       .debug$S                   10000000     Qt5Widgets:Qt5Widgets.dll
 0000:fff90000       .debug$S                   10000000     Qt5Widgets:Qt5Widgets.dll
 0000:fff90000       .debug$S                   10000000     Qt5Widgets:Qt5Widgets.dll
 0000:fff90000       .debug$S                   10000000     Qt5Widgets:Qt5Widgets.dll
 0000:fff90000       .debug$S                   10000000     Qt5Widgets:Qt5Widgets.dll
 0000:fff90000       .debug$S                   10000000     Qt5Widgets:Qt5Widgets.dll
 0000:fff90000       .debug$S                   10000000     Qt5Widgets:Qt5Widgets.dll
 0000:fff90000       .debug$S                   10000000     Qt5Widgets:Qt5Widgets.dll
 0000:fff90000       .debug$S                   10000000     Qt5Widgets:Qt5Widgets.dll
 0000:fff90000       .debug$S                   10000000     Qt5Widgets:Qt5Widgets.dll
 0000:fff90000       .debug$S                   10000000     Qt5Widgets:Qt5Widgets.dll
 0000:fff90000       .debug$S                   10000000     Qt5Widgets:Qt5Widgets.dll
 0000:fff90000       .debug$S                   10000000     Qt5Widgets:Qt5Widgets.dll
 0000:fff90000       .debug$S                   10000000     Qt5Widgets:Qt5Widgets.dll
 0000:fff90000       .debug$S                   10000000     Qt5Widgets:Qt5Widgets.dll
 0000:fff90000       .debug$S                   10000000     Qt5Widgets:Qt5Widgets.dll
 0001:fffff000       __ehhandler$?_Copy@?$basic_string@DU?$char_traits@D@std@@V?$allocator@D@2@@std@@QAEXII@Z 10000000 f   moc_PhylipCmdlineTask.obj
 0000:fff90000       .debug$S                   10000000     Qt5Widgets:Qt5Widgets.dll
 0000:fff90000       .debug$S                   10000000     Qt5Widgets:Qt5Widgets.dll
 0000:fff90000       .debug$S                   10000000     Qt5Widgets:Qt5Widgets.dll
 0000:fff90000       .debug$S                   10000000     Qt5Widgets:Qt5Widgets.dll
 0000:fff90000       .debug$S                   10000000     Qt5Widgets:Qt5Widgets.dll
 0000:fff90000       .debug$S                   10000000     Qt5Widgets:Qt5Widgets.dll
 0000:fff90000       .debug$S                   10000000     Qt5Widgets:Qt5Widgets.dll
 0000:fff90000       .debug$S                   10000000     Qt5Widgets:Qt5Widgets.dll
 0000:fff90000       .debug$S                   10000000     Qt5Widgets:Qt5Widgets.dll
 0000:fff90000       .debug$S                   10000000     Qt5Widgets:Qt5Widgets.dll
 0000:fff90000       .debug$S                   10000000     Qt5Widgets:Qt5Widgets.dll
 0000:fff90000       .debug$S                   10000000     Qt5Widgets:Qt5Widgets.dll
 0000:fff90000       .debug$S                   10000000     Qt5Widgets:Qt5Widgets.dll
 0000:fff90000       .debug$S                   10000000     Qt5Widgets:Qt5Widgets.dll
 0000:fff90000       .debug$S                   10000000     Qt5Widgets:Qt5Widgets.dll
 0000:fff90000       .debug$S                   10000000     Qt5Widgets:Qt5Widgets.dll
 0000:fff90000       .debug$S                   10000000     Qt5Widgets:Qt5Widgets.dll
 0000:fff90000       .debug$S                   10000000     Qt5Widgets:Qt5Widgets.dll
 0000:fff90000       .debug$S                   10000000     Qt5Widgets:Qt5Widgets.dll
 0000:fff90000       .debug$S                   10000000     Qt5Widgets:Qt5Widgets.dll
 0000:fff90000       .debug$S                   10000000     Qt5Widgets:Qt5Widgets.dll
 0000:fff90000       .debug$S                   10000000     Qt5Widgets:Qt5Widgets.dll
 0000:fff90000       .debug$S                   10000000     Qt5Widgets:Qt5Widgets.dll
 0000:fff90000       .debug$S                   10000000     Qt5Widgets:Qt5Widgets.dll
 0002:fffbe000       __catchsym$?_Copy@?$basic_string@DU?$char_traits@D@std@@V?$allocator@D@2@@std@@QAEXII@Z$5 10000000     moc_PhylipCmdlineTask.obj
 0000:fff90000       .debug$S                   10000000     Qt5Widgets:Qt5Widgets.dll
 0000:fff90000       .debug$S                   10000000     Qt5Widgets:Qt5Widgets.dll
 0000:fff90000       .debug$S                   10000000     Qt5Widgets:Qt5Widgets.dll
 0000:fff90000       .debug$S                   10000000     Qt5Widgets:Qt5Widgets.dll
 0000:fff90000       .debug$S                   10000000     Qt5Widgets:Qt5Widgets.dll
 0000:fff90000       .debug$S                   10000000     Qt5Widgets:Qt5Widgets.dll
 0000:fff90000       .debug$S                   10000000     Qt5Widgets:Qt5Widgets.dll
 0000:fff90000       .debug$S                   10000000     Qt5Widgets:Qt5Widgets.dll
 0000:fff90000       .debug$S                   10000000     Qt5Widgets:Qt5Widgets.dll
 0000:fff90000       .debug$S                   10000000     Qt5Widgets:Qt5Widgets.dll
 0000:fff90000       .debug$S                   10000000     Qt5Widgets:Qt5Widgets.dll
 0000:fff90000       .debug$S                   10000000     Qt5Widgets:Qt5Widgets.dll
 0000:fff90000       .debug$S                   10000000     Qt5Widgets:Qt5Widgets.dll
 0000:fff90000       .debug$S                   10000000     Qt5Widgets:Qt5Widgets.dll
 0000:fff90000       .debug$S                   10000000     Qt5Widgets:Qt5Widgets.dll
 0000:fff90000       .debug$S                   10000000     Qt5Widgets:Qt5Widgets.dll
 0000:fff90000       .debug$S                   10000000     Qt5Widgets:Qt5Widgets.dll
 0000:fff90000       .debug$S                   10000000     Qt5Widgets:Qt5Widgets.dll
 0000:fff90000       .debug$S                   10000000     Qt5Widgets:Qt5Widgets.dll
 0000:fff90000       .debug$S                   10000000     Qt5Widgets:Qt5Widgets.dll
 0000:fff90000       .debug$S                   10000000     Qt5Widgets:Qt5Widgets.dll
 0000:fff90000       .debug$S                   10000000     Qt5Widgets:Qt5Widgets.dll
 0000:fff90000       .debug$S                   10000000     Qt5Widgets:Qt5Widgets.dll
 0000:fff90000       .debug$S                   10000000     Qt5Widgets:Qt5Widgets.dll
 0000:fff90000       .debug$S                   10000000     Qt5Widgets:Qt5Widgets.dll
 0000:fff90000       .debug$S                   10000000     Qt5Widgets:Qt5Widgets.dll
 0000:fff90000       .debug$S                   10000000     Qt5Widgets:Qt5Widgets.dll
 0000:fff90000       .debug$S                   10000000     Qt5Widgets:Qt5Widgets.dll
 0000:fff90000       .debug$S                   10000000     Qt5Widgets:Qt5Widgets.dll
 0000:fff90000       .debug$S                   10000000     Qt5Widgets:Qt5Widgets.dll
 0000:fff90000       .debug$S                   10000000     Qt5Widgets:Qt5Widgets.dll
 0000:fff90000       .debug$S                   10000000     Qt5Widgets:Qt5Widgets.dll
 0000:fff90000       .debug$S                   10000000     Qt5Widgets:Qt5Widgets.dll
 0000:fff90000       .debug$S                   10000000     Qt5Widgets:Qt5Widgets.dll
 0000:fff90000       .debug$S                   10000000     Qt5Widgets:Qt5Widgets.dll
 0000:fff90000       .debug$S                   10000000     Qt5Widgets:Qt5Widgets.dll
 0000:fff90000       .debug$S                   10000000     Qt5Widgets:Qt5Widgets.dll
 0000:fff90000       .debug$S                   10000000     Qt5Widgets:Qt5Widgets.dll
 0000:fff90000       .debug$S                   10000000     Qt5Widgets:Qt5Widgets.dll
 0000:fff90000       .debug$S                   10000000     Qt5Widgets:Qt5Widgets.dll
 0000:fff90000       .debug$S                   10000000     Qt5Widgets:Qt5Widgets.dll
 0002:fffbe000       ?_Generic_object$initializer$@?$_Error_objects@H@std@@2P6AXXZA 10000000     moc_PhylipCmdlineTask.obj
 0002:fffbe000       ?_Iostream_object$initializer$@?$_Error_objects@H@std@@2P6AXXZA 10000000     moc_PhylipCmdlineTask.obj
 0002:fffbe000       ?_System_object$initializer$@?$_Error_objects@H@std@@2P6AXXZA 10000000     moc_PhylipCmdlineTask.obj
 0000:fff90000       .debug$S                   10000000     Qt5Widgets:Qt5Widgets.dll
 0000:fff90000       .debug$S                   10000000     Qt5Widgets:Qt5Widgets.dll
 0000:fff90000       .debug$S                   10000000     Qt5Widgets:Qt5Widgets.dll
 0000:fff90000       .debug$S                   10000000     Qt5Widgets:Qt5Widgets.dll
 0000:fff90000       .debug$S                   10000000     Qt5Widgets:Qt5Widgets.dll
 0000:fff90000       .debug$S                   10000000     Qt5Widgets:Qt5Widgets.dll
 0000:fff90000       .debug$S                   10000000     Qt5Widgets:Qt5Widgets.dll
 0000:fff90000       .debug$S                   10000000     Qt5Widgets:Qt5Widgets.dll
 0000:fff90000       .debug$S                   10000000     Qt5Widgets:Qt5Widgets.dll
 0000:fff90000       .debug$S                   10000000     Qt5Widgets:Qt5Widgets.dll
 0000:fff90000       .debug$S                   10000000     Qt5Widgets:Qt5Widgets.dll
 0000:fff90000       .debug$S                   10000000     Qt5Widgets:Qt5Widgets.dll
 0000:fff90000       .debug$S                   10000000     Qt5Widgets:Qt5Widgets.dll
 0000:fff90000       .debug$S                   10000000     Qt5Widgets:Qt5Widgets.dll
 0000:fff90000       .debug$S                   10000000     Qt5Widgets:Qt5Widgets.dll
 0000:fff90000       .debug$S                   10000000     Qt5Widgets:Qt5Widgets.dll
 0000:fff90000       .debug$S                   10000000     Qt5Widgets:Qt5Widgets.dll
 0000:fff90000       .debug$S                   10000000     Qt5Widgets:Qt5Widgets.dll
 0000:fff90000       .debug$S                   10000000     Qt5Widgets:Qt5Widgets.dll
 0000:fff90000       .debug$S                   10000000     Qt5Widgets:Qt5Widgets.dll
 0000:fff90000       .debug$S                   10000000     Qt5Widgets:Qt5Widgets.dll
 0000:fff90000       .debug$S                   10000000     Qt5Widgets:Qt5Widgets.dll
 0000:fff90000       .debug$S                   10000000     Qt5Widgets:Qt5Widgets.dll
 0000:fff90000       .debug$S                   10000000     Qt5Widgets:Qt5Widgets.dll
 0000:fff90000       .debug$S                   10000000     Qt5Widgets:Qt5Widgets.dll
 0000:fff90000       .debug$S                   10000000     Qt5Widgets:Qt5Widgets.dll
 0000:fff90000       .debug$S                   10000000     Qt5Widgets:Qt5Widgets.dll
 0001:fffff000       __ehhandler$?_Copy@?$basic_string@DU?$char_traits@D@std@@V?$allocator@D@2@@std@@QAEXII@Z 10000000 f   moc_NeighborJoinWidget.obj
 0000:fff90000       .debug$S                   10000000     Qt5Widgets:Qt5Widgets.dll
 0000:fff90000       .debug$S                   10000000     Qt5Widgets:Qt5Widgets.dll
 0000:fff90000       .debug$S                   10000000     Qt5Widgets:Qt5Widgets.dll
 0000:fff90000       .debug$S                   10000000     Qt5Widgets:Qt5Widgets.dll
 0000:fff90000       .debug$S                   10000000     Qt5Widgets:Qt5Widgets.dll
 0000:fff90000       .debug$S                   10000000     Qt5Widgets:Qt5Widgets.dll
 0000:fff90000       .debug$S                   10000000     Qt5Widgets:Qt5Widgets.dll
 0000:fff90000       .debug$S                   10000000     Qt5Widgets:Qt5Widgets.dll
 0000:fff90000       .debug$S                   10000000     Qt5Widgets:Qt5Widgets.dll
 0000:fff90000       .debug$S                   10000000     Qt5Widgets:Qt5Widgets.dll
 0000:fff90000       .debug$S                   10000000     Qt5Widgets:Qt5Widgets.dll
 0000:fff90000       .debug$S                   10000000     Qt5Widgets:Qt5Widgets.dll
 0000:fff90000       .debug$S                   10000000     Qt5Widgets:Qt5Widgets.dll
 0000:fff90000       .debug$S                   10000000     Qt5Widgets:Qt5Widgets.dll
 0000:fff90000       .debug$S                   10000000     Qt5Widgets:Qt5Widgets.dll
 0000:fff90000       .debug$S                   10000000     Qt5Widgets:Qt5Widgets.dll
 0000:fff90000       .debug$S                   10000000     Qt5Widgets:Qt5Widgets.dll
 0000:fff90000       .debug$S                   10000000     Qt5Widgets:Qt5Widgets.dll
 0000:fff90000       .debug$S                   10000000     Qt5Widgets:Qt5Widgets.dll
 0000:fff90000       .debug$S                   10000000     Qt5Widgets:Qt5Widgets.dll
 0000:fff90000       .debug$S                   10000000     Qt5Widgets:Qt5Widgets.dll
 0000:fff90000       .debug$S                   10000000     Qt5Widgets:Qt5Widgets.dll
 0000:fff90000       .debug$S                   10000000     Qt5Widgets:Qt5Widgets.dll
 0000:fff90000       .debug$S                   10000000     Qt5Widgets:Qt5Widgets.dll
 0002:fffbe000       __catchsym$?_Copy@?$basic_string@DU?$char_traits@D@std@@V?$allocator@D@2@@std@@QAEXII@Z$5 10000000     moc_NeighborJoinWidget.obj
 0000:fff90000       .debug$S                   10000000     Qt5Widgets:Qt5Widgets.dll
 0000:fff90000       .debug$S                   10000000     Qt5Widgets:Qt5Widgets.dll
 0000:fff90000       .debug$S                   10000000     Qt5Widgets:Qt5Widgets.dll
 0000:fff90000       .debug$S                   10000000     Qt5Widgets:Qt5Widgets.dll
 0000:fff90000       .debug$S                   10000000     Qt5Widgets:Qt5Widgets.dll
 0000:fff90000       .debug$S                   10000000     Qt5Widgets:Qt5Widgets.dll
 0000:fff90000       .debug$S                   10000000     Qt5Widgets:Qt5Widgets.dll
 0000:fff90000       .debug$S                   10000000     Qt5Widgets:Qt5Widgets.dll
 0000:fff90000       .debug$S                   10000000     Qt5Widgets:Qt5Widgets.dll
 0000:fff90000       .debug$S                   10000000     Qt5Widgets:Qt5Widgets.dll
 0000:fff90000       .debug$S                   10000000     Qt5Widgets:Qt5Widgets.dll
 0000:fff90000       .debug$S                   10000000     Qt5Widgets:Qt5Widgets.dll
 0000:fff90000       .debug$S                   10000000     Qt5Widgets:Qt5Widgets.dll
 0000:fff90000       .debug$S                   10000000     Qt5Widgets:Qt5Widgets.dll
 0000:fff90000       .debug$S                   10000000     Qt5Widgets:Qt5Widgets.dll
 0000:fff90000       .debug$S                   10000000     Qt5Widgets:Qt5Widgets.dll
 0000:fff90000       .debug$S                   10000000     Qt5Widgets:Qt5Widgets.dll
 0000:fff90000       .debug$S                   10000000     Qt5Widgets:Qt5Widgets.dll
 0000:fff90000       .debug$S                   10000000     Qt5Widgets:Qt5Widgets.dll
 0000:fff90000       .debug$S                   10000000     Qt5Widgets:Qt5Widgets.dll
 0000:fff90000       .debug$S                   10000000     Qt5Widgets:Qt5Widgets.dll
 0000:fff90000       .debug$S                   10000000     Qt5Widgets:Qt5Widgets.dll
 0000:fff90000       .debug$S                   10000000     Qt5Widgets:Qt5Widgets.dll
 0000:fff90000       .debug$S                   10000000     Qt5Widgets:Qt5Widgets.dll
 0000:fff90000       .debug$S                   10000000     Qt5Widgets:Qt5Widgets.dll
 0000:fff90000       .debug$S                   10000000     Qt5Widgets:Qt5Widgets.dll
 0000:fff90000       .debug$S                   10000000     Qt5Widgets:Qt5Widgets.dll
 0000:fff90000       .debug$S                   10000000     Qt5Widgets:Qt5Widgets.dll
 0000:fff90000       .debug$S                   10000000     Qt5Widgets:Qt5Widgets.dll
 0000:fff90000       .debug$S                   10000000     Qt5Widgets:Qt5Widgets.dll
 0000:fff90000       .debug$S                   10000000     Qt5Widgets:Qt5Widgets.dll
 0000:fff90000       .debug$S                   10000000     Qt5Widgets:Qt5Widgets.dll
 0000:fff90000       .debug$S                   10000000     Qt5Widgets:Qt5Widgets.dll
 0000:fff90000       .debug$S                   10000000     Qt5Widgets:Qt5Widgets.dll
 0000:fff90000       .debug$S                   10000000     Qt5Widgets:Qt5Widgets.dll
 0000:fff90000       .debug$S                   10000000     Qt5Widgets:Qt5Widgets.dll
 0000:fff90000       .debug$S                   10000000     Qt5Widgets:Qt5Widgets.dll
 0000:fff90000       .debug$S                   10000000     Qt5Widgets:Qt5Widgets.dll
 0000:fff90000       .debug$S                   10000000     Qt5Widgets:Qt5Widgets.dll
 0000:fff90000       .debug$S                   10000000     Qt5Widgets:Qt5Widgets.dll
 0000:fff90000       .debug$S                   10000000     Qt5Widgets:Qt5Widgets.dll
 0002:fffbe000       ?_Generic_object$initializer$@?$_Error_objects@H@std@@2P6AXXZA 10000000     moc_NeighborJoinWidget.obj
 0002:fffbe000       ?_Iostream_object$initializer$@?$_Error_objects@H@std@@2P6AXXZA 10000000     moc_NeighborJoinWidget.obj
 0002:fffbe000       ?_System_object$initializer$@?$_Error_objects@H@std@@2P6AXXZA 10000000     moc_NeighborJoinWidget.obj
 0000:fff90000       .debug$S                   10000000     Qt5Widgets:Qt5Widgets.dll
 0000:fff90000       .debug$S                   10000000     Qt5Widgets:Qt5Widgets.dll
 0000:fff90000       .debug$S                   10000000     Qt5Widgets:Qt5Widgets.dll
 0000:fff90000       .debug$S                   10000000     Qt5Widgets:Qt5Widgets.dll
 0000:fff90000       .debug$S                   10000000     Qt5Widgets:Qt5Widgets.dll
 0000:fff90000       .debug$S                   10000000     Qt5Widgets:Qt5Widgets.dll
 0000:fff90000       .debug$S                   10000000     Qt5Widgets:Qt5Widgets.dll
 0000:fff90000       .debug$S                   10000000     Qt5Widgets:Qt5Widgets.dll
 0000:fff90000       .debug$S                   10000000     Qt5Widgets:Qt5Widgets.dll
 0000:fff90000       .debug$S                   10000000     Qt5Widgets:Qt5Widgets.dll
 0000:fff90000       .debug$S                   10000000     Qt5Widgets:Qt5Widgets.dll
 0000:fff90000       .debug$S                   10000000     Qt5Widgets:Qt5Widgets.dll
 0000:fff90000       .debug$S                   10000000     Qt5Widgets:Qt5Widgets.dll
 0000:fff90000       .debug$S                   10000000     Qt5Widgets:Qt5Widgets.dll
 0000:fff90000       .debug$S                   10000000     Qt5Widgets:Qt5Widgets.dll
 0000:fff90000       .debug$S                   10000000     Qt5Widgets:Qt5Widgets.dll
 0000:fff90000       .debug$S                   10000000     Qt5Widgets:Qt5Widgets.dll
 0000:fff90000       .debug$S                   10000000     Qt5Widgets:Qt5Widgets.dll
 0000:fff90000       .debug$S                   10000000     Qt5Widgets:Qt5Widgets.dll
 0000:fff90000       .debug$S                   10000000     Qt5Widgets:Qt5Widgets.dll
 0000:fff90000       .debug$S                   10000000     Qt5Widgets:Qt5Widgets.dll
 0000:fff90000       .debug$S                   10000000     Qt5Widgets:Qt5Widgets.dll
 0000:fff90000       .debug$S                   10000000     Qt5Widgets:Qt5Widgets.dll
 0000:fff90000       .debug$S                   10000000     Qt5Widgets:Qt5Widgets.dll
 0000:fff90000       .debug$S                   10000000     Qt5Widgets:Qt5Widgets.dll
 0000:fff90000       .debug$S                   10000000     Qt5Widgets:Qt5Widgets.dll
 0000:fff90000       .debug$S                   10000000     Qt5Widgets:Qt5Widgets.dll
 0000:fff90000       .debug$S                   10000000     Qt5Widgets:Qt5Widgets.dll
 0000:fff90000       .debug$S                   10000000     Qt5Widgets:Qt5Widgets.dll
 0000:fff90000       .debug$S                   10000000     Qt5Widgets:Qt5Widgets.dll
 0000:fff90000       .debug$S                   10000000     Qt5Widgets:Qt5Widgets.dll
 0000:fff90000       .debug$S                   10000000     Qt5Widgets:Qt5Widgets.dll
 0000:fff90000       .debug$S                   10000000     Qt5Widgets:Qt5Widgets.dll
 0000:fff90000       .debug$S                   10000000     Qt5Widgets:Qt5Widgets.dll
 0001:fffff000       __ehhandler$?_Copy@?$basic_string@DU?$char_traits@D@std@@V?$allocator@D@2@@std@@QAEXII@Z 10000000 f   seqboot.obj
 0000:fff90000       .debug$S                   10000000     Qt5Widgets:Qt5Widgets.dll
 0000:fff90000       .debug$S                   10000000     Qt5Widgets:Qt5Widgets.dll
 0000:fff90000       .debug$S                   10000000     Qt5Widgets:Qt5Widgets.dll
 0000:fff90000       .debug$S                   10000000     Qt5Widgets:Qt5Widgets.dll
 0000:fff90000       .debug$S                   10000000     Qt5Widgets:Qt5Widgets.dll
 0000:fff90000       .debug$S                   10000000     Qt5Widgets:Qt5Widgets.dll
 0000:fff90000       .debug$S                   10000000     Qt5Widgets:Qt5Widgets.dll
 0000:fff90000       .debug$S                   10000000     Qt5Widgets:Qt5Widgets.dll
 0000:fff90000       .debug$S                   10000000     Qt5Widgets:Qt5Widgets.dll
 0000:fff90000       .debug$S                   10000000     Qt5Widgets:Qt5Widgets.dll
 0000:fff90000       .debug$S                   10000000     U2Test:U2Test.dll
 0000:fff90000       .debug$S                   10000000     U2Test:U2Test.dll
 0000:fff90000       .debug$S                   10000000     U2Test:U2Test.dll
 0000:fff90000       .debug$S                   10000000     U2Test:U2Test.dll
 0000:fff90000       .debug$S                   10000000     U2Test:U2Test.dll
 0000:fff90000       .debug$S                   10000000     U2Test:U2Test.dll
 0000:fff90000       .debug$S                   10000000     U2Test:U2Test.dll
 0000:fff90000       .debug$S                   10000000     U2Test:U2Test.dll
 0000:fff90000       .debug$S                   10000000     U2Test:U2Test.dll
 0000:fff90000       .debug$S                   10000000     U2Test:U2Test.dll
 0000:fff90000       .debug$S                   10000000     U2Test:U2Test.dll
 0000:fff90000       .debug$S                   10000000     U2View:U2View.dll
 0000:fff90000       .debug$S                   10000000     U2View:U2View.dll
 0000:fff90000       .debug$S                   10000000     U2View:U2View.dll
 0000:fff90000       .debug$S                   10000000     U2View:U2View.dll
 0000:fff90000       .debug$S                   10000000     U2View:U2View.dll
 0000:fff90000       .debug$S                   10000000     U2View:U2View.dll
 0001:fffff000       __unwindfunclet$?reallocData@?$QVector@VMultipleSequenceAlignment@U2@@@@AAEXHHV?$QFlags@W4AllocationOption@QArrayData@@@@@Z$4 10000000 f   seqboot.obj
 0000:fff90000       .debug$S                   10000000     U2View:U2View.dll
 0001:fffff000       __unwindfunclet$?defaultConstruct@?$QVector@VMultipleSequenceAlignment@U2@@@@AAEXPAVMultipleSequenceAlignment@U2@@0@Z$0 10000000 f   seqboot.obj
 0000:fff90000       .debug$S                   10000000     U2View:U2View.dll
 0000:fff90000       .debug$S                   10000000     U2View:U2View.dll
 0000:fff90000       .debug$S                   10000000     U2View:U2View.dll
 0000:fff90000       .debug$S                   10000000     U2View:U2View.dll
 0000:fff90000       .debug$S                   10000000     U2Algorithm:U2Algorithm.dll
 0000:fff90000       .debug$S                   10000000     U2Algorithm:U2Algorithm.dll
 0002:fffbe000       __catchsym$?_Copy@?$basic_string@DU?$char_traits@D@std@@V?$allocator@D@2@@std@@QAEXII@Z$5 10000000     seqboot.obj
 0000:fff90000       .debug$S                   10000000     U2Algorithm:U2Algorithm.dll
 0000:fff90000       .debug$S                   10000000     U2Algorithm:U2Algorithm.dll
 0000:fff90000       .debug$S                   10000000     U2Algorithm:U2Algorithm.dll
 0000:fff90000       .debug$S                   10000000     U2Algorithm:U2Algorithm.dll
 0000:fff90000       .debug$S                   10000000     U2Algorithm:U2Algorithm.dll
 0000:fff90000       .debug$S                   10000000     U2Algorithm:U2Algorithm.dll
 0000:fff90000       .debug$S                   10000000     U2Algorithm:U2Algorithm.dll
 0000:fff90000       .debug$S                   10000000     U2Algorithm:U2Algorithm.dll
 0000:fff90000       .debug$S                   10000000     U2Algorithm:U2Algorithm.dll
 0000:fff90000       .debug$S                   10000000     U2Algorithm:U2Algorithm.dll
 0000:fff90000       .debug$S                   10000000     U2Algorithm:U2Algorithm.dll
 0000:fff90000       .debug$S                   10000000     U2Algorithm:U2Algorithm.dll
 0000:fff90000       .debug$S                   10000000     U2Algorithm:U2Algorithm.dll
 0000:fff90000       .debug$S                   10000000     U2Algorithm:U2Algorithm.dll
 0000:fff90000       .debug$S                   10000000     U2Algorithm:U2Algorithm.dll
 0000:fff90000       .debug$S                   10000000     U2Algorithm:U2Algorithm.dll
 0000:fff90000       .debug$S                   10000000     U2Algorithm:U2Algorithm.dll
 0000:fff90000       .debug$S                   10000000     U2Algorithm:U2Algorithm.dll
 0000:fff90000       .debug$S                   10000000     U2Algorithm:U2Algorithm.dll
 0000:fff90000       .debug$S                   10000000     U2Algorithm:U2Algorithm.dll
 0000:fff90000       .debug$S                   10000000     U2Algorithm:U2Algorithm.dll
 0000:fff90000       .debug$S                   10000000     U2Algorithm:U2Algorithm.dll
 0000:fff90000       .debug$S                   10000000     U2Core:U2Core.dll
 0000:fff90000       .debug$S                   10000000     U2Core:U2Core.dll
 0002:fffbe000       __catchsym$?reallocData@?$QVector@VMultipleSequenceAlignment@U2@@@@AAEXHHV?$QFlags@W4AllocationOption@QArrayData@@@@@Z$6 10000000     seqboot.obj
 0002:fffbe000       __ehfuncinfo$?defaultConstruct@?$QVector@VMultipleSequenceAlignment@U2@@@@AAEXPAVMultipleSequenceAlignment@U2@@0@Z 10000000     seqboot.obj
 0000:fff90000       .debug$S                   10000000     U2Core:U2Core.dll
 0000:fff90000       .debug$S                   10000000     U2Core:U2Core.dll
 0000:fff90000       .debug$S                   10000000     U2Core:U2Core.dll
 0000:fff90000       .debug$S                   10000000     U2Core:U2Core.dll
 0000:fff90000       .debug$S                   10000000     U2Core:U2Core.dll
 0000:fff90000       .debug$S                   10000000     U2Core:U2Core.dll
 0000:fff90000       .debug$S                   10000000     U2Core:U2Core.dll
 0000:fff90000       .debug$S                   10000000     U2Core:U2Core.dll
 0000:fff90000       .debug$S                   10000000     U2Core:U2Core.dll
 0000:fff90000       .debug$S                   10000000     U2Core:U2Core.dll
 0000:fff90000       .debug$S                   10000000     U2Core:U2Core.dll
 0000:fff90000       .debug$S                   10000000     U2Core:U2Core.dll
 0000:fff90000       .debug$S                   10000000     U2Core:U2Core.dll
 0000:fff90000       .debug$S                   10000000     U2Core:U2Core.dll
 0000:fff90000       .debug$S                   10000000     U2Core:U2Core.dll
 0000:fff90000       .debug$S                   10000000     U2Core:U2Core.dll
 0000:fff90000       .debug$S                   10000000     U2Core:U2Core.dll
 0000:fff90000       .debug$S                   10000000     U2Core:U2Core.dll
 0000:fff90000       .debug$S                   10000000     U2Core:U2Core.dll
 0000:fff90000       .debug$S                   10000000     U2Core:U2Core.dll
 0000:fff90000       .debug$S                   10000000     U2Core:U2Core.dll
 0000:fff90000       .debug$S                   10000000     U2Core:U2Core.dll
 0000:fff90000       .debug$S                   10000000     U2Core:U2Core.dll
 0000:fff90000       .debug$S                   10000000     U2Core:U2Core.dll
 0000:fff90000       .debug$S                   10000000     U2Core:U2Core.dll
 0000:fff90000       .debug$S                   10000000     U2Core:U2Core.dll
 0000:fff90000       .debug$S                   10000000     U2Core:U2Core.dll
 0000:fff90000       .debug$S                   10000000     U2Core:U2Core.dll
 0000:fff90000       .debug$S                   10000000     U2Core:U2Core.dll
 0000:fff90000       .debug$S                   10000000     U2Core:U2Core.dll
 0000:fff90000       .debug$S                   10000000     U2Core:U2Core.dll
 0000:fff90000       .debug$S                   10000000     U2Core:U2Core.dll
 0000:fff90000       .debug$S                   10000000     U2Core:U2Core.dll
 0000:fff90000       .debug$S                   10000000     U2Core:U2Core.dll
 0000:fff90000       .debug$S                   10000000     U2Core:U2Core.dll
 0000:fff90000       .debug$S                   10000000     U2Core:U2Core.dll
 0000:fff90000       .debug$S                   10000000     U2Core:U2Core.dll
 0000:fff90000       .debug$S                   10000000     U2Core:U2Core.dll
 0000:fff90000       .debug$S                   10000000     U2Core:U2Core.dll
 0000:fff90000       .debug$S                   10000000     U2Core:U2Core.dll
 0000:fff90000       .debug$S                   10000000     U2Core:U2Core.dll
 0000:fff90000       .debug$S                   10000000     U2Core:U2Core.dll
 0000:fff90000       .debug$S                   10000000     U2Core:U2Core.dll
 0000:fff90000       .debug$S                   10000000     U2Core:U2Core.dll
 0000:fff90000       .debug$S                   10000000     U2Core:U2Core.dll
 0000:fff90000       .debug$S                   10000000     U2Core:U2Core.dll
 0000:fff90000       .debug$S                   10000000     U2Core:U2Core.dll
 0000:fff90000       .debug$S                   10000000     U2Core:U2Core.dll
 0000:fff90000       .debug$S                   10000000     U2Core:U2Core.dll
 0000:fff90000       .debug$S                   10000000     U2Core:U2Core.dll
 0000:fff90000       .debug$S                   10000000     U2Core:U2Core.dll
 0000:fff90000       .debug$S                   10000000     U2Core:U2Core.dll
 0000:fff90000       .debug$S                   10000000     U2Core:U2Core.dll
 0000:fff90000       .debug$S                   10000000     U2Core:U2Core.dll
 0000:fff90000       .debug$S                   10000000     U2Core:U2Core.dll
 0000:fff90000       .debug$S                   10000000     U2Core:U2Core.dll
 0000:fff90000       .debug$S                   10000000     U2Core:U2Core.dll
 0000:fff90000       .debug$S                   10000000     U2Core:U2Core.dll
 0000:fff90000       .debug$S                   10000000     U2Core:U2Core.dll
 0002:fffbe000       ?_Generic_object$initializer$@?$_Error_objects@H@std@@2P6AXXZA 10000000     seqboot.obj
 0002:fffbe000       ?_Iostream_object$initializer$@?$_Error_objects@H@std@@2P6AXXZA 10000000     seqboot.obj
 0002:fffbe000       ?_System_object$initializer$@?$_Error_objects@H@std@@2P6AXXZA 10000000     seqboot.obj
 0000:fff90000       .debug$S                   10000000     U2Core:U2Core.dll
 0000:fff90000       .debug$S                   10000000     U2Core:U2Core.dll
 0000:fff90000       .debug$S                   10000000     U2Core:U2Core.dll
 0000:fff90000       .debug$S                   10000000     U2Core:U2Core.dll
 0000:fff90000       .debug$S                   10000000     U2Core:U2Core.dll
 0000:fff90000       .debug$S                   10000000     U2Core:U2Core.dll
 0000:fff90000       .debug$S                   10000000     U2Core:U2Core.dll
 0000:fff90000       .debug$S                   10000000     U2Core:U2Core.dll
 0000:fff90000       .debug$S                   10000000     U2Core:U2Core.dll
 0000:fff90000       .debug$S                   10000000     U2Core:U2Core.dll
 0000:fff90000       .debug$S                   10000000     U2Core:U2Core.dll
 0000:fff90000       .debug$S                   10000000     U2Core:U2Core.dll
 0000:fff90000       .debug$S                   10000000     U2Core:U2Core.dll
 0000:fff90000       .debug$S                   10000000     U2Core:U2Core.dll
 0000:fff90000       .debug$S                   10000000     U2Core:U2Core.dll
 0000:fff90000       .debug$S                   10000000     U2Core:U2Core.dll
 0000:fff90000       .debug$S                   10000000     U2Core:U2Core.dll
 0000:fff90000       .debug$S                   10000000     U2Core:U2Core.dll
 0000:fff90000       .debug$S                   10000000     U2Core:U2Core.dll
 0000:fff90000       .debug$S                   10000000     U2Core:U2Core.dll
 0000:fff90000       .debug$S                   10000000     U2Core:U2Core.dll
 0000:fff90000       .debug$S                   10000000     U2Core:U2Core.dll
 0000:fff90000       .debug$S                   10000000     U2Core:U2Core.dll
 0000:fff90000       .debug$S                   10000000     U2Core:U2Core.dll
 0000:fff90000       .debug$S                   10000000     U2Core:U2Core.dll
 0000:fff90000       .debug$S                   10000000     U2Core:U2Core.dll
 0000:fff90000       .debug$S                   10000000     U2Core:U2Core.dll
 0000:fff90000       .debug$S                   10000000     U2Core:U2Core.dll
 0000:fff90000       .debug$S                   10000000     U2Core:U2Core.dll
 0000:fff90000       .debug$S                   10000000     U2Core:U2Core.dll
 0000:fff90000       .debug$S                   10000000     U2Core:U2Core.dll
 0000:fff90000       .debug$S                   10000000     U2Core:U2Core.dll
 0000:fff90000       .debug$S                   10000000     U2Core:U2Core.dll
 0000:fff90000       .debug$S                   10000000     U2Core:U2Core.dll
 0000:fff90000       .debug$S                   10000000     U2Core:U2Core.dll
 0000:fff90000       .debug$S                   10000000     U2Core:U2Core.dll
 0000:fff90000       .debug$S                   10000000     U2Core:U2Core.dll
 0000:fff90000       .debug$S                   10000000     U2Core:U2Core.dll
 0000:fff90000       .debug$S                   10000000     U2Core:U2Core.dll
 0000:fff90000       .debug$S                   10000000     U2Core:U2Core.dll
 0000:fff90000       .debug$S                   10000000     U2Core:U2Core.dll
 0000:fff90000       .debug$S                   10000000     U2Core:U2Core.dll
 0000:fff90000       .debug$S                   10000000     U2Core:U2Core.dll
 0001:fffff000       __ehhandler$?_Copy@?$basic_string@DU?$char_traits@D@std@@V?$allocator@D@2@@std@@QAEXII@Z 10000000 f   protdist.obj
 0000:fff90000       .debug$S                   10000000     U2Core:U2Core.dll
 0000:fff90000       .debug$S                   10000000     U2Core:U2Core.dll
 0001:fffff000       __ehhandler$??0?$QList@VQString@@@@QAE@ABV0@@Z 10000000 f   protdist.obj
 0000:fff90000       .debug$S                   10000000     U2Core:U2Core.dll
 0000:fff90000       .debug$S                   10000000     U2Core:U2Core.dll
 0000:fff90000       .debug$S                   10000000     U2Core:U2Core.dll
 0000:fff90000       .debug$S                   10000000     U2Core:U2Core.dll
 0001:fffff000       __unwindfunclet$?append@?$QList@VQString@@@@QAEXABVQString@@@Z$7 10000000 f   protdist.obj
 0000:fff90000       .debug$S                   10000000     U2Core:U2Core.dll
 0001:fffff000       __ehhandler$?detach_helper_grow@?$QList@VQString@@@@AAEPAUNode@1@HH@Z 10000000 f   protdist.obj
 0000:fff90000       .debug$S                   10000000     U2Core:U2Core.dll
 0000:fff90000       .debug$S                   10000000     U2Core:U2Core.dll
 0000:fff90000       .debug$S                   10000000     U2Core:U2Core.dll
 0001:fffff000       __unwindfunclet$?node_construct@?$QList@VQString@@@@AAEXPAUNode@1@ABVQString@@@Z$1 10000000 f   protdist.obj
 0000:fff90000       .debug$S                   10000000     U2Core:U2Core.dll
 0000:fff90000       .debug$S                   10000000     U2Core:U2Core.dll
 0001:fffff000       __unwindfunclet$?node_copy@?$QList@VQString@@@@AAEXPAUNode@1@00@Z$5 10000000 f   protdist.obj
 0000:fff90000       .debug$S                   10000000     U2Core:U2Core.dll
 0000:fff90000       .debug$S                   10000000     U2Core:U2Core.dll
 0000:fff90000       .debug$S                   10000000     U2Core:U2Core.dll
 0000:fff90000       .debug$S                   10000000     U2Core:U2Core.dll
 0000:fff90000       .debug$S                   10000000     U2Core:U2Core.dll
 0000:fff90000       .debug$S                   10000000     U2Core:U2Core.dll
 0000:fff90000       .debug$S                   10000000     U2Core:U2Core.dll
 0000:fff90000       .debug$S                   10000000     U2Core:U2Core.dll
 0000:fff90000       .debug$S                   10000000     U2Core:U2Core.dll
 0000:fff90000       .debug$S                   10000000     U2Core:U2Core.dll
 0000:fff90000       .debug$S                   10000000     U2Core:U2Core.dll
 0000:fff90000       .debug$S                   10000000     U2Core:U2Core.dll
 0000:fff90000       .debug$S                   10000000     U2Core:U2Core.dll
 0000:fff90000       .debug$S                   10000000     U2Core:U2Core.dll
 0000:fff90000       .debug$S                   10000000     U2Core:U2Core.dll
 0000:fff90000       .debug$S                   10000000     U2Core:U2Core.dll
 0000:fff90000       .debug$S                   10000000     U2Core:U2Core.dll
 0000:fff90000       .debug$S                   10000000     U2Core:U2Core.dll
 0000:fff90000       .debug$S                   10000000     U2Core:U2Core.dll
 0001:fffff000       __unwindfunclet$?tryAcquire@MemoryLocker@U2@@QAE_N_J@Z$0 10000000 f   protdist.obj
 0000:fff90000       .debug$S                   10000000     U2Core:U2Core.dll
 0000:fff90000       .debug$S                   10000000     U2Core:U2Core.dll
 0000:fff90000       .debug$S                   10000000     U2Core:U2Core.dll
 0000:fff90000       .debug$S                   10000000     U2Core:U2Core.dll
 0000:fff90000       .debug$S                   10000000     U2Core:U2Core.dll
 0000:fff90000       .debug$S                   10000000     U2Core:U2Core.dll
 0000:fff90000       .debug$S                   10000000     U2Core:U2Core.dll
 0000:fff90000       .debug$S                   10000000     U2Core:U2Core.dll
 0000:fff90000       .debug$S                   10000000     U2Core:U2Core.dll
 0002:fffbe000       __catchsym$?_Copy@?$basic_string@DU?$char_traits@D@std@@V?$allocator@D@2@@std@@QAEXII@Z$5 10000000     protdist.obj
 0000:fff90000       .debug$S                   10000000     U2Core:U2Core.dll
 0000:fff90000       .debug$S                   10000000     U2Core:U2Core.dll
 0000:fff90000       .debug$S                   10000000     U2Core:U2Core.dll
 0002:fffbe000       __catchsym$??0?$QList@VQString@@@@QAE@ABV0@@Z$2 10000000     protdist.obj
 0000:fff90000       .debug$S                   10000000     U2Core:U2Core.dll
 0000:fff90000       .debug$S                   10000000     U2Core:U2Core.dll
 0000:fff90000       .debug$S                   10000000     U2Core:U2Core.dll
 0000:fff90000       .debug$S                   10000000     U2Core:U2Core.dll
 0002:fffbe000       __catchsym$?append@?$QList@VQString@@@@QAEXABVQString@@@Z$13 10000000     protdist.obj
 0000:fff90000       .debug$S                   10000000     U2Core:U2Core.dll
 0000:fff90000       .debug$S                   10000000     U2Core:U2Core.dll
 0000:fff90000       .debug$S                   10000000     U2Core:U2Core.dll
 0000:fff90000       .debug$S                   10000000     U2Core:U2Core.dll
 0002:fffbe000       __catchsym$?detach_helper_grow@?$QList@VQString@@@@AAEPAUNode@1@HH@Z$5 10000000     protdist.obj
 0000:fff90000       .debug$S                   10000000     U2Core:U2Core.dll
 0002:fffbe000       __unwindtable$?node_construct@?$QList@VQString@@@@AAEXPAUNode@1@ABVQString@@@Z 10000000     protdist.obj
 0000:fff90000       .debug$S                   10000000     U2Core:U2Core.dll
 0000:fff90000       .debug$S                   10000000     U2Core:U2Core.dll
 0000:fff90000       .debug$S                   10000000     U2Core:U2Core.dll
 0002:fffbe000       __catchsym$?node_copy@?$QList@VQString@@@@AAEXPAUNode@1@00@Z$6 10000000     protdist.obj
 0000:fff90000       .debug$S                   10000000     U2Core:U2Core.dll
 0000:fff90000       .debug$S                   10000000     U2Core:U2Core.dll
 0000:fff90000       .debug$S                   10000000     U2Core:U2Core.dll
 0000:fff90000       .debug$S                   10000000     U2Core:U2Core.dll
 0000:fff90000       .debug$S                   10000000     U2Core:U2Core.dll
 0000:fff90000       .debug$S                   10000000     U2Core:U2Core.dll
 0000:fff90000       .debug$S                   10000000     U2Core:U2Core.dll
 0000:fff90000       .debug$S                   10000000     U2Core:U2Core.dll
 0000:fff90000       .debug$S                   10000000     U2Core:U2Core.dll
 0000:fff90000       .debug$S                   10000000     U2Core:U2Core.dll
 0000:fff90000       .debug$S                   10000000     U2Core:U2Core.dll
 0000:fff90000       .debug$S                   10000000     U2Core:U2Core.dll
 0000:fff90000       .debug$S                   10000000     U2Core:U2Core.dll
 0000:fff90000       .debug$S                   10000000     U2Core:U2Core.dll
 0000:fff90000       .debug$S                   10000000     U2Core:U2Core.dll
 0000:fff90000       .debug$S                   10000000     U2Core:U2Core.dll
 0000:fff90000       .debug$S                   10000000     U2Core:U2Core.dll
 0000:fff90000       .debug$S                   10000000     U2Core:U2Core.dll
 0002:fffbe000       ?_System_object$initializer$@?$_Error_objects@H@std@@2P6AXXZA 10000000     NeighborJoinAdapter.obj
 0002:fffbe000       __unwindtable$?tryAcquire@MemoryLocker@U2@@QAE_N_J@Z 10000000     protdist.obj
 0002:fffbe000       ?_Iostream_object$initializer$@?$_Error_objects@H@std@@2P6AXXZA 10000000     NeighborJoinAdapter.obj
 0002:fffbe000       ?_Generic_object$initializer$@?$_Error_objects@H@std@@2P6AXXZA 10000000     NeighborJoinAdapter.obj
 0002:fffbe000       __catchsym$?reallocData@?$QVector@M@@AAEXHHV?$QFlags@W4AllocationOption@QArrayData@@@@@Z$5 10000000     NeighborJoinAdapter.obj
 0002:fffbe000       __catchsym$?reallocData@?$QVector@V?$QVector@M@@@@AAEXHHV?$QFlags@W4AllocationOption@QArrayData@@@@@Z$6 10000000     NeighborJoinAdapter.obj
 0002:fffbe000       __unwindtable$??_GMemoryLocker@U2@@UAEPAXI@Z 10000000     NeighborJoinAdapter.obj
 0002:fffbe000       __unwindtable$?release@MemoryLocker@U2@@QAEXXZ 10000000     NeighborJoinAdapter.obj
 0002:fffbe000       __unwindtable$?tryAcquire@MemoryLocker@U2@@QAE_N_J@Z 10000000     NeighborJoinAdapter.obj
 0002:fffbe000       __unwindtable$??1MemoryLocker@U2@@UAE@XZ 10000000     NeighborJoinAdapter.obj
 0002:fffbe000       __catchsym$?_Copy@?$basic_string@DU?$char_traits@D@std@@V?$allocator@D@2@@std@@QAEXII@Z$5 10000000     NeighborJoinAdapter.obj
 0001:fffff000       __ehhandler$?reallocData@?$QVector@M@@AAEXHHV?$QFlags@W4AllocationOption@QArrayData@@@@@Z 10000000 f   NeighborJoinAdapter.obj
 0001:fffff000       __unwindfunclet$?reallocData@?$QVector@V?$QVector@M@@@@AAEXHHV?$QFlags@W4AllocationOption@QArrayData@@@@@Z$4 10000000 f   NeighborJoinAdapter.obj
 0001:fffff000       __unwindfunclet$??_GMemoryLocker@U2@@UAEPAXI@Z$0 10000000 f   NeighborJoinAdapter.obj
 0001:fffff000       __unwindfunclet$?release@MemoryLocker@U2@@QAEXXZ$0 10000000 f   NeighborJoinAdapter.obj
 0001:fffff000       __unwindfunclet$?tryAcquire@MemoryLocker@U2@@QAE_N_J@Z$0 10000000 f   NeighborJoinAdapter.obj
 0001:fffff000       __unwindfunclet$??1MemoryLocker@U2@@UAE@XZ$0 10000000 f   NeighborJoinAdapter.obj
 0001:fffff000       __ehhandler$?_Copy@?$basic_string@DU?$char_traits@D@std@@V?$allocator@D@2@@std@@QAEXII@Z 10000000 f   NeighborJoinAdapter.obj
 0002:fffbe000       ?_System_object$initializer$@?$_Error_objects@H@std@@2P6AXXZA 10000000     NeighborJoinWidget.obj
 0002:fffbe000       ?_Iostream_object$initializer$@?$_Error_objects@H@std@@2P6AXXZA 10000000     NeighborJoinWidget.obj
 0002:fffbe000       ?_Generic_object$initializer$@?$_Error_objects@H@std@@2P6AXXZA 10000000     NeighborJoinWidget.obj
 0002:fffbe000       __catchsym$?node_copy@?$QList@VQString@@@@AAEXPAUNode@1@00@Z$6 10000000     NeighborJoinWidget.obj
 0002:fffbe000       __unwindtable$?node_construct@?$QList@VQString@@@@AAEXPAUNode@1@ABVQString@@@Z 10000000     NeighborJoinWidget.obj
 0002:fffbe000       __catchsym$?detach_helper_grow@?$QList@VQString@@@@AAEPAUNode@1@HH@Z$5 10000000     NeighborJoinWidget.obj
 0002:fffbe000       __catchsym$?append@?$QList@VQString@@@@QAEXABVQString@@@Z$13 10000000     NeighborJoinWidget.obj
 0002:fffbe000       __catchsym$?_Copy@?$basic_string@DU?$char_traits@D@std@@V?$allocator@D@2@@std@@QAEXII@Z$5 10000000     NeighborJoinWidget.obj
 0001:fffff000       __unwindfunclet$?node_copy@?$QList@VQString@@@@AAEXPAUNode@1@00@Z$5 10000000 f   NeighborJoinWidget.obj
 0001:fffff000       __unwindfunclet$?node_construct@?$QList@VQString@@@@AAEXPAUNode@1@ABVQString@@@Z$1 10000000 f   NeighborJoinWidget.obj
 0001:fffff000       __ehhandler$?detach_helper_grow@?$QList@VQString@@@@AAEPAUNode@1@HH@Z 10000000 f   NeighborJoinWidget.obj
 0001:fffff000       __unwindfunclet$?append@?$QList@VQString@@@@QAEXABVQString@@@Z$7 10000000 f   NeighborJoinWidget.obj
 0002:fffbe000       ?_Generic_object$initializer$@?$_Error_objects@H@std@@2P6AXXZA 10000000     protdist.obj
 0002:fffbe000       ?_Iostream_object$initializer$@?$_Error_objects@H@std@@2P6AXXZA 10000000     protdist.obj
 0002:fffbe000       ?_System_object$initializer$@?$_Error_objects@H@std@@2P6AXXZA 10000000     protdist.obj
 0001:fffff000       __ehhandler$?_Copy@?$basic_string@DU?$char_traits@D@std@@V?$allocator@D@2@@std@@QAEXII@Z 10000000 f   NeighborJoinWidget.obj
 0002:fffbe000       ?_System_object$initializer$@?$_Error_objects@H@std@@2P6AXXZA 10000000     PhylipCmdlineTask.obj
 0002:fffbe000       ?_Iostream_object$initializer$@?$_Error_objects@H@std@@2P6AXXZA 10000000     PhylipCmdlineTask.obj
 0002:fffbe000       ?_Generic_object$initializer$@?$_Error_objects@H@std@@2P6AXXZA 10000000     PhylipCmdlineTask.obj
 0002:fffbe000       __catchsym$?node_copy@?$QList@VQString@@@@AAEXPAUNode@1@00@Z$6 10000000     PhylipCmdlineTask.obj
 0002:fffbe000       __unwindtable$?node_construct@?$QList@VQString@@@@AAEXPAUNode@1@ABVQString@@@Z 10000000     PhylipCmdlineTask.obj
 0002:fffbe000       __catchsym$?detach_helper_grow@?$QList@VQString@@@@AAEPAUNode@1@HH@Z$5 10000000     PhylipCmdlineTask.obj
 0002:fffbe000       __catchsym$?append@?$QList@VQString@@@@QAEXABVQString@@@Z$13 10000000     PhylipCmdlineTask.obj
 0002:fffbe000       __catchsym$?_Copy@?$basic_string@DU?$char_traits@D@std@@V?$allocator@D@2@@std@@QAEXII@Z$5 10000000     PhylipCmdlineTask.obj
 0001:fffff000       __unwindfunclet$?node_copy@?$QList@VQString@@@@AAEXPAUNode@1@00@Z$5 10000000 f   PhylipCmdlineTask.obj
 0001:fffff000       __unwindfunclet$?node_construct@?$QList@VQString@@@@AAEXPAUNode@1@ABVQString@@@Z$1 10000000 f   PhylipCmdlineTask.obj
 0001:fffff000       __ehhandler$?detach_helper_grow@?$QList@VQString@@@@AAEPAUNode@1@HH@Z 10000000 f   PhylipCmdlineTask.obj
 0000:fff90000       .debug$S                   10000000     MSVCRT:MSVCR120.dll
 0001:fffff000       __ehhandler$?_Copy@?$basic_string@DU?$char_traits@D@std@@V?$allocator@D@2@@std@@QAEXII@Z 10000000 f   PhylipCmdlineTask.obj
 0002:fffbe000       ?_System_object$initializer$@?$_Error_objects@H@std@@2P6AXXZA 10000000     PhylipPlugin.obj
 0002:fffbe000       ?_Iostream_object$initializer$@?$_Error_objects@H@std@@2P6AXXZA 10000000     PhylipPlugin.obj
 0002:fffbe000       ?_Generic_object$initializer$@?$_Error_objects@H@std@@2P6AXXZA 10000000     PhylipPlugin.obj
 0002:fffbe000       __catchsym$?_Copy@?$basic_string@DU?$char_traits@D@std@@V?$allocator@D@2@@std@@QAEXII@Z$5 10000000     PhylipPlugin.obj
 0001:fffff000       __ehhandler$?_Copy@?$basic_string@DU?$char_traits@D@std@@V?$allocator@D@2@@std@@QAEXII@Z 10000000 f   PhylipPlugin.obj
 0002:fffbe000       ?_System_object$initializer$@?$_Error_objects@H@std@@2P6AXXZA 10000000     PhylipPluginTests.obj
 0002:fffbe000       ?_Iostream_object$initializer$@?$_Error_objects@H@std@@2P6AXXZA 10000000     PhylipPluginTests.obj
 0002:fffbe000       ?_Generic_object$initializer$@?$_Error_objects@H@std@@2P6AXXZA 10000000     PhylipPluginTests.obj
 0002:fffbe000       __catchsym$?_Copy@?$basic_string@DU?$char_traits@D@std@@V?$allocator@D@2@@std@@QAEXII@Z$5 10000000     PhylipPluginTests.obj
 0001:fffff000       __ehhandler$?_Copy@?$basic_string@DU?$char_traits@D@std@@V?$allocator@D@2@@std@@QAEXII@Z 10000000 f   PhylipPluginTests.obj
 0002:fffbe000       ?_System_object$initializer$@?$_Error_objects@H@std@@2P6AXXZA 10000000     PhylipTask.obj
 0002:fffbe000       ?_Iostream_object$initializer$@?$_Error_objects@H@std@@2P6AXXZA 10000000     PhylipTask.obj
 0002:fffbe000       ?_Generic_object$initializer$@?$_Error_objects@H@std@@2P6AXXZA 10000000     PhylipTask.obj
 0002:fffbe000       __catchsym$?_Copy@?$basic_string@DU?$char_traits@D@std@@V?$allocator@D@2@@std@@QAEXII@Z$5 10000000     PhylipTask.obj
 0001:fffff000       __ehhandler$?_Copy@?$basic_string@DU?$char_traits@D@std@@V?$allocator@D@2@@std@@QAEXII@Z 10000000 f   phylip.obj
 0001:fffff000       __ehhandler$?_Copy@?$basic_string@DU?$char_traits@D@std@@V?$allocator@D@2@@std@@QAEXII@Z 10000000 f   PhylipTask.obj
 0002:fffbe000       ?_System_object$initializer$@?$_Error_objects@H@std@@2P6AXXZA 10000000     SeqBootAdapter.obj
 0002:fffbe000       ?_Iostream_object$initializer$@?$_Error_objects@H@std@@2P6AXXZA 10000000     SeqBootAdapter.obj
 0002:fffbe000       ?_Generic_object$initializer$@?$_Error_objects@H@std@@2P6AXXZA 10000000     SeqBootAdapter.obj
 0002:fffbe000       __catchsym$?_Copy@?$basic_string@DU?$char_traits@D@std@@V?$allocator@D@2@@std@@QAEXII@Z$5 10000000     SeqBootAdapter.obj
 0001:fffff000       __ehhandler$?_Copy@?$basic_string@DU?$char_traits@D@std@@V?$allocator@D@2@@std@@QAEXII@Z 10000000 f   SeqBootAdapter.obj
 0002:fffbe000       ?_System_object$initializer$@?$_Error_objects@H@std@@2P6AXXZA 10000000     dist.obj
 0002:fffbe000       ?_Iostream_object$initializer$@?$_Error_objects@H@std@@2P6AXXZA 10000000     dist.obj
 0002:fffbe000       ?_Generic_object$initializer$@?$_Error_objects@H@std@@2P6AXXZA 10000000     dist.obj
 0002:fffbe000       __unwindtable$?tryAcquire@MemoryLocker@U2@@QAE_N_J@Z 10000000     dist.obj
 0002:fffbe000       __catchsym$?_Copy@?$basic_string@DU?$char_traits@D@std@@V?$allocator@D@2@@std@@QAEXII@Z$5 10000000     dist.obj
 0001:fffff000       __unwindfunclet$?tryAcquire@MemoryLocker@U2@@QAE_N_J@Z$0 10000000 f   dist.obj
 0001:fffff000       __ehhandler$?_Copy@?$basic_string@DU?$char_traits@D@std@@V?$allocator@D@2@@std@@QAEXII@Z 10000000 f   dist.obj
 0002:fffbe000       ?_System_object$initializer$@?$_Error_objects@H@std@@2P6AXXZA 10000000     dnadist.obj
 0002:fffbe000       ?_Iostream_object$initializer$@?$_Error_objects@H@std@@2P6AXXZA 10000000     dnadist.obj
 0002:fffbe000       ?_Generic_object$initializer$@?$_Error_objects@H@std@@2P6AXXZA 10000000     dnadist.obj
 0002:fffbe000       __unwindtable$?tryAcquire@MemoryLocker@U2@@QAE_N_J@Z 10000000     dnadist.obj
 0002:fffbe000       __catchsym$?node_copy@?$QList@VQString@@@@AAEXPAUNode@1@00@Z$6 10000000     dnadist.obj
 0002:fffbe000       __unwindtable$?node_construct@?$QList@VQString@@@@AAEXPAUNode@1@ABVQString@@@Z 10000000     dnadist.obj
 0002:fffbe000       __catchsym$?detach_helper_grow@?$QList@VQString@@@@AAEPAUNode@1@HH@Z$5 10000000     dnadist.obj
 0002:fffbe000       __catchsym$?append@?$QList@VQString@@@@QAEXABVQString@@@Z$13 10000000     dnadist.obj
 0002:fffbe000       __catchsym$??0?$QList@VQString@@@@QAE@ABV0@@Z$2 10000000     dnadist.obj
 0002:fffbe000       __catchsym$?_Copy@?$basic_string@DU?$char_traits@D@std@@V?$allocator@D@2@@std@@QAEXII@Z$5 10000000     dnadist.obj
 0001:fffff000       __unwindfunclet$?tryAcquire@MemoryLocker@U2@@QAE_N_J@Z$0 10000000 f   dnadist.obj
 0002:fffbe000       __catchsym$?_Copy@?$basic_string@DU?$char_traits@D@std@@V?$allocator@D@2@@std@@QAEXII@Z$5 10000000     phylip.obj
 0001:fffff000       __unwindfunclet$?node_copy@?$QList@VQString@@@@AAEXPAUNode@1@00@Z$5 10000000 f   dnadist.obj
 0001:fffff000       __unwindfunclet$?node_construct@?$QList@VQString@@@@AAEXPAUNode@1@ABVQString@@@Z$1 10000000 f   dnadist.obj
 0001:fffff000       __ehhandler$?detach_helper_grow@?$QList@VQString@@@@AAEPAUNode@1@HH@Z 10000000 f   dnadist.obj
 0001:fffff000       __unwindfunclet$?append@?$QList@VQString@@@@QAEXABVQString@@@Z$7 10000000 f   dnadist.obj
 0001:fffff000       __ehhandler$??0?$QList@VQString@@@@QAE@ABV0@@Z 10000000 f   dnadist.obj
 0001:fffff000       __ehhandler$?_Copy@?$basic_string@DU?$char_traits@D@std@@V?$allocator@D@2@@std@@QAEXII@Z 10000000 f   dnadist.obj
 0002:fffbe000       ?_System_object$initializer$@?$_Error_objects@H@std@@2P6AXXZA 10000000     neighbor.obj
 0002:fffbe000       ?_Iostream_object$initializer$@?$_Error_objects@H@std@@2P6AXXZA 10000000     neighbor.obj
 0002:fffbe000       ?_Generic_object$initializer$@?$_Error_objects@H@std@@2P6AXXZA 10000000     neighbor.obj
 0002:fffbe000       __catchsym$?_Copy@?$basic_string@DU?$char_traits@D@std@@V?$allocator@D@2@@std@@QAEXII@Z$5 10000000     neighbor.obj
 0001:fffff000       __ehhandler$?_Copy@?$basic_string@DU?$char_traits@D@std@@V?$allocator@D@2@@std@@QAEXII@Z 10000000 f   neighbor.obj
 0002:fffbe000       ?_System_object$initializer$@?$_Error_objects@H@std@@2P6AXXZA 10000000     phylip.obj
 0002:fffbe000       ?_Iostream_object$initializer$@?$_Error_objects@H@std@@2P6AXXZA 10000000     phylip.obj
 0002:fffbe000       ?_Generic_object$initializer$@?$_Error_objects@H@std@@2P6AXXZA 10000000     phylip.obj
 0002:fffbe008       __ehfuncinfo$?release@MemoryLocker@U2@@QAEXXZ 10000008     NeighborJoinAdapter.obj
 0002:fffbe008       __ehfuncinfo$??1MemoryLocker@U2@@UAE@XZ 10000008     NeighborJoinAdapter.obj
 0002:fffbe008       __ehfuncinfo$??_GMemoryLocker@U2@@UAEPAXI@Z 10000008     NeighborJoinAdapter.obj
 0001:fffff009       __unwindfunclet$?tryAcquire@MemoryLocker@U2@@QAE_N_J@Z$1 10000009 f   dnadist.obj
 0001:fffff009       __unwindfunclet$?tryAcquire@MemoryLocker@U2@@QAE_N_J@Z$1 10000009 f   dist.obj
 0001:fffff009       __ehhandler$?release@MemoryLocker@U2@@QAEXXZ 10000009 f   NeighborJoinAdapter.obj
 0001:fffff009       __unwindfunclet$?tryAcquire@MemoryLocker@U2@@QAE_N_J@Z$1 10000009 f   NeighborJoinAdapter.obj
 0001:fffff009       __unwindfunclet$?tryAcquire@MemoryLocker@U2@@QAE_N_J@Z$1 10000009 f   protdist.obj
 0001:fffff00c       __ehhandler$??_GMemoryLocker@U2@@UAEPAXI@Z 1000000c f   NeighborJoinAdapter.obj
 0001:fffff00c       __ehhandler$??1MemoryLocker@U2@@UAE@XZ 1000000c f   NeighborJoinAdapter.obj
 0002:fffbe010       __catchsym$?_Copy@?$basic_string@DU?$char_traits@D@std@@V?$allocator@D@2@@std@@QAEXII@Z$4 10000010     dnadist.obj
 0002:fffbe010       __catchsym$?_Copy@?$basic_string@DU?$char_traits@D@std@@V?$allocator@D@2@@std@@QAEXII@Z$4 10000010     moc_NeighborJoinWidget.obj
 0002:fffbe010       __tryblocktable$?node_copy@?$QList@VQString@@@@AAEXPAUNode@1@00@Z 10000010     dnadist.obj
 0002:fffbe010       __catchsym$?_Copy@?$basic_string@DU?$char_traits@D@std@@V?$allocator@D@2@@std@@QAEXII@Z$4 10000010     PhylipPluginTests.obj
 0002:fffbe010       __catchsym$?_Copy@?$basic_string@DU?$char_traits@D@std@@V?$allocator@D@2@@std@@QAEXII@Z$4 10000010     dist.obj
 0002:fffbe010       __catchsym$?_Copy@?$basic_string@DU?$char_traits@D@std@@V?$allocator@D@2@@std@@QAEXII@Z$4 10000010     moc_PhylipCmdlineTask.obj
 0002:fffbe010       __tryblocktable$?node_copy@?$QList@VQString@@@@AAEXPAUNode@1@00@Z 10000010     PhylipCmdlineTask.obj
 0002:fffbe010       __catchsym$?_Copy@?$basic_string@DU?$char_traits@D@std@@V?$allocator@D@2@@std@@QAEXII@Z$4 10000010     moc_PhylipPlugin.obj
 0002:fffbe010       __catchsym$?_Copy@?$basic_string@DU?$char_traits@D@std@@V?$allocator@D@2@@std@@QAEXII@Z$4 10000010     PhylipTask.obj
 0002:fffbe010       __catchsym$?detach_helper_grow@?$QList@VQString@@@@AAEPAUNode@1@HH@Z$4 10000010     dnadist.obj
 0002:fffbe010       __unwindtable$??0?$QList@VQString@@@@QAE@ABV0@@Z 10000010     dnadist.obj
 0002:fffbe010       __tryblocktable$?node_copy@?$QList@VQString@@@@AAEXPAUNode@1@00@Z 10000010     NeighborJoinWidget.obj
 0002:fffbe010       __ehfuncinfo$?node_construct@?$QList@VQString@@@@AAEXPAUNode@1@ABVQString@@@Z 10000010     dnadist.obj
 0002:fffbe010       __catchsym$?_Copy@?$basic_string@DU?$char_traits@D@std@@V?$allocator@D@2@@std@@QAEXII@Z$4 10000010     neighbor.obj
 0002:fffbe010       __catchsym$?_Copy@?$basic_string@DU?$char_traits@D@std@@V?$allocator@D@2@@std@@QAEXII@Z$4 10000010     moc_PhylipPluginTests.obj
 0002:fffbe010       __catchsym$?_Copy@?$basic_string@DU?$char_traits@D@std@@V?$allocator@D@2@@std@@QAEXII@Z$4 10000010     NeighborJoinAdapter.obj
 0002:fffbe010       __catchsym$?reallocData@?$QVector@V?$QVector@M@@@@AAEXHHV?$QFlags@W4AllocationOption@QArrayData@@@@@Z$5 10000010     NeighborJoinAdapter.obj
 0002:fffbe010       __tryblocktable$?node_copy@?$QList@VQString@@@@AAEXPAUNode@1@00@Z 10000010     protdist.obj
 0002:fffbe010       __catchsym$?_Copy@?$basic_string@DU?$char_traits@D@std@@V?$allocator@D@2@@std@@QAEXII@Z$4 10000010     seqboot.obj
 0002:fffbe010       __catchsym$?_Copy@?$basic_string@DU?$char_traits@D@std@@V?$allocator@D@2@@std@@QAEXII@Z$4 10000010     protdist.obj
 0002:fffbe010       __catchsym$?_Copy@?$basic_string@DU?$char_traits@D@std@@V?$allocator@D@2@@std@@QAEXII@Z$4 10000010     PhylipPlugin.obj
 0002:fffbe010       __catchsym$?_Copy@?$basic_string@DU?$char_traits@D@std@@V?$allocator@D@2@@std@@QAEXII@Z$4 10000010     moc_PhylipTask.obj
 0002:fffbe010       __ehfuncinfo$?node_construct@?$QList@VQString@@@@AAEXPAUNode@1@ABVQString@@@Z 10000010     NeighborJoinWidget.obj
 0002:fffbe010       __catchsym$?_Copy@?$basic_string@DU?$char_traits@D@std@@V?$allocator@D@2@@std@@QAEXII@Z$4 10000010     PhylipCmdlineTask.obj
 0002:fffbe010       __catchsym$?detach_helper_grow@?$QList@VQString@@@@AAEPAUNode@1@HH@Z$4 10000010     NeighborJoinWidget.obj
 0002:fffbe010       __catchsym$?append@?$QList@VQString@@@@QAEXABVQString@@@Z$12 10000010     dnadist.obj
 0002:fffbe010       __catchsym$?append@?$QList@VQString@@@@QAEXABVQString@@@Z$12 10000010     PhylipCmdlineTask.obj
 0002:fffbe010       __catchsym$?_Copy@?$basic_string@DU?$char_traits@D@std@@V?$allocator@D@2@@std@@QAEXII@Z$4 10000010     phylip.obj
 0002:fffbe010       __ehfuncinfo$?node_construct@?$QList@VQString@@@@AAEXPAUNode@1@ABVQString@@@Z 10000010     protdist.obj
 0002:fffbe010       __catchsym$?append@?$QList@VQString@@@@QAEXABVQString@@@Z$12 10000010     NeighborJoinWidget.obj
 0002:fffbe010       __catchsym$?detach_helper_grow@?$QList@VQString@@@@AAEPAUNode@1@HH@Z$4 10000010     PhylipCmdlineTask.obj
 0002:fffbe010       __catchsym$?_Copy@?$basic_string@DU?$char_traits@D@std@@V?$allocator@D@2@@std@@QAEXII@Z$4 10000010     NeighborJoinWidget.obj
 0002:fffbe010       __catchsym$?detach_helper_grow@?$QList@VQString@@@@AAEPAUNode@1@HH@Z$4 10000010     protdist.obj
 0002:fffbe010       __catchsym$?reallocData@?$QVector@VMultipleSequenceAlignment@U2@@@@AAEXHHV?$QFlags@W4AllocationOption@QArrayData@@@@@Z$5 10000010     seqboot.obj
 0002:fffbe010       __unwindtable$??0?$QList@VQString@@@@QAE@ABV0@@Z 10000010     protdist.obj
 0002:fffbe010       __catchsym$?_Copy@?$basic_string@DU?$char_traits@D@std@@V?$allocator@D@2@@std@@QAEXII@Z$4 10000010     SeqBootAdapter.obj
 0002:fffbe010       __ehfuncinfo$?node_construct@?$QList@VQString@@@@AAEXPAUNode@1@ABVQString@@@Z 10000010     PhylipCmdlineTask.obj
 0002:fffbe010       __catchsym$?append@?$QList@VQString@@@@QAEXABVQString@@@Z$12 10000010     protdist.obj
 0002:fffbe010       __catchsym$?reallocData@?$QVector@M@@AAEXHHV?$QFlags@W4AllocationOption@QArrayData@@@@@Z$4 10000010     NeighborJoinAdapter.obj
 0001:fffff011       __ehhandler$?reallocData@?$QVector@VMultipleSequenceAlignment@U2@@@@AAEXHHV?$QFlags@W4AllocationOption@QArrayData@@@@@Z 10000011 f   seqboot.obj
 0001:fffff011       __unwindfunclet$?append@?$QList@VQString@@@@QAEXABVQString@@@Z$11 10000011 f   PhylipCmdlineTask.obj
 0001:fffff011       __ehhandler$?node_copy@?$QList@VQString@@@@AAEXPAUNode@1@00@Z 10000011 f   dnadist.obj
 0001:fffff011       __ehhandler$?node_construct@?$QList@VQString@@@@AAEXPAUNode@1@ABVQString@@@Z 10000011 f   PhylipCmdlineTask.obj
 0001:fffff011       __unwindfunclet$?append@?$QList@VQString@@@@QAEXABVQString@@@Z$11 10000011 f   dnadist.obj
 0001:fffff011       __unwindfunclet$?append@?$QList@VQString@@@@QAEXABVQString@@@Z$11 10000011 f   protdist.obj
 0001:fffff011       __unwindfunclet$?defaultConstruct@?$QVector@VMultipleSequenceAlignment@U2@@@@AAEXPAVMultipleSequenceAlignment@U2@@0@Z$1 10000011 f   seqboot.obj
 0001:fffff011       __ehhandler$?node_copy@?$QList@VQString@@@@AAEXPAUNode@1@00@Z 10000011 f   protdist.obj
 0001:fffff011       __ehhandler$?node_construct@?$QList@VQString@@@@AAEXPAUNode@1@ABVQString@@@Z 10000011 f   NeighborJoinWidget.obj
 0001:fffff011       __ehhandler$?node_construct@?$QList@VQString@@@@AAEXPAUNode@1@ABVQString@@@Z 10000011 f   dnadist.obj
 0001:fffff011       __ehhandler$?node_construct@?$QList@VQString@@@@AAEXPAUNode@1@ABVQString@@@Z 10000011 f   protdist.obj
 0001:fffff011       __ehhandler$?node_copy@?$QList@VQString@@@@AAEXPAUNode@1@00@Z 10000011 f   PhylipCmdlineTask.obj
 0001:fffff011       __unwindfunclet$?append@?$QList@VQString@@@@QAEXABVQString@@@Z$11 10000011 f   NeighborJoinWidget.obj
 0001:fffff011       __ehhandler$?reallocData@?$QVector@V?$QVector@M@@@@AAEXHHV?$QFlags@W4AllocationOption@QArrayData@@@@@Z 10000011 f   NeighborJoinAdapter.obj
 0001:fffff011       __ehhandler$?node_copy@?$QList@VQString@@@@AAEXPAUNode@1@00@Z 10000011 f   NeighborJoinWidget.obj
 0001:fffff012       __unwindfunclet$?tryAcquire@MemoryLocker@U2@@QAE_N_J@Z$2 10000012 f   NeighborJoinAdapter.obj
 0001:fffff012       __unwindfunclet$?tryAcquire@MemoryLocker@U2@@QAE_N_J@Z$2 10000012 f   protdist.obj
 0001:fffff012       __unwindfunclet$?tryAcquire@MemoryLocker@U2@@QAE_N_J@Z$2 10000012 f   dist.obj
 0001:fffff012       __unwindfunclet$?tryAcquire@MemoryLocker@U2@@QAE_N_J@Z$2 10000012 f   dnadist.obj
 0002:fffbe018       __ehfuncinfo$?tryAcquire@MemoryLocker@U2@@QAE_N_J@Z 10000018     NeighborJoinAdapter.obj
 0002:fffbe018       __ehfuncinfo$?tryAcquire@MemoryLocker@U2@@QAE_N_J@Z 10000018     protdist.obj
 0002:fffbe018       __ehfuncinfo$?tryAcquire@MemoryLocker@U2@@QAE_N_J@Z 10000018     dist.obj
 0002:fffbe018       __ehfuncinfo$?tryAcquire@MemoryLocker@U2@@QAE_N_J@Z 10000018     dnadist.obj
 0001:fffff01b       __ehhandler$?tryAcquire@MemoryLocker@U2@@QAE_N_J@Z 1000001b f   protdist.obj
 0001:fffff01b       __ehhandler$?tryAcquire@MemoryLocker@U2@@QAE_N_J@Z 1000001b f   dist.obj
 0001:fffff01b       __ehhandler$?tryAcquire@MemoryLocker@U2@@QAE_N_J@Z 1000001b f   dnadist.obj
 0001:fffff01b       __ehhandler$?tryAcquire@MemoryLocker@U2@@QAE_N_J@Z 1000001b f   NeighborJoinAdapter.obj
 0002:fffbe020       __ehfuncinfo$?append@?$QList@VQString@@@@QAEXABVQString@@@Z 10000020     PhylipCmdlineTask.obj
 0002:fffbe020       __unwindtable$?_Copy@?$basic_string@DU?$char_traits@D@std@@V?$allocator@D@2@@std@@QAEXII@Z 10000020     moc_PhylipTask.obj
 0002:fffbe020       __unwindtable$?_Copy@?$basic_string@DU?$char_traits@D@std@@V?$allocator@D@2@@std@@QAEXII@Z 10000020     moc_PhylipPluginTests.obj
 0002:fffbe020       __ehfuncinfo$?append@?$QList@VQString@@@@QAEXABVQString@@@Z 10000020     protdist.obj
 0002:fffbe020       __unwindtable$?_Copy@?$basic_string@DU?$char_traits@D@std@@V?$allocator@D@2@@std@@QAEXII@Z 10000020     neighbor.obj
 0002:fffbe020       __ehfuncinfo$?append@?$QList@VQString@@@@QAEXABVQString@@@Z 10000020     dnadist.obj
 0002:fffbe020       __unwindtable$?detach_helper_grow@?$QList@VQString@@@@AAEPAUNode@1@HH@Z 10000020     NeighborJoinWidget.obj
 0002:fffbe020       __unwindtable$?_Copy@?$basic_string@DU?$char_traits@D@std@@V?$allocator@D@2@@std@@QAEXII@Z 10000020     dnadist.obj
 0002:fffbe020       __unwindtable$?_Copy@?$basic_string@DU?$char_traits@D@std@@V?$allocator@D@2@@std@@QAEXII@Z 10000020     PhylipCmdlineTask.obj
 0002:fffbe020       __unwindtable$?_Copy@?$basic_string@DU?$char_traits@D@std@@V?$allocator@D@2@@std@@QAEXII@Z 10000020     PhylipPlugin.obj
 0002:fffbe020       __unwindtable$?_Copy@?$basic_string@DU?$char_traits@D@std@@V?$allocator@D@2@@std@@QAEXII@Z 10000020     seqboot.obj
 0002:fffbe020       __unwindtable$?detach_helper_grow@?$QList@VQString@@@@AAEPAUNode@1@HH@Z 10000020     PhylipCmdlineTask.obj
 0002:fffbe020       __unwindtable$?_Copy@?$basic_string@DU?$char_traits@D@std@@V?$allocator@D@2@@std@@QAEXII@Z 10000020     PhylipPluginTests.obj
 0002:fffbe020       __unwindtable$?_Copy@?$basic_string@DU?$char_traits@D@std@@V?$allocator@D@2@@std@@QAEXII@Z 10000020     moc_NeighborJoinWidget.obj
 0002:fffbe020       __tryblocktable$??0?$QList@VQString@@@@QAE@ABV0@@Z 10000020     protdist.obj
 0002:fffbe020       __unwindtable$?_Copy@?$basic_string@DU?$char_traits@D@std@@V?$allocator@D@2@@std@@QAEXII@Z 10000020     PhylipTask.obj
 0002:fffbe020       __ehfuncinfo$?reallocData@?$QVector@V?$QVector@M@@@@AAEXHHV?$QFlags@W4AllocationOption@QArrayData@@@@@Z 10000020     NeighborJoinAdapter.obj
 0002:fffbe020       __ehfuncinfo$?append@?$QList@VQString@@@@QAEXABVQString@@@Z 10000020     NeighborJoinWidget.obj
 0002:fffbe020       __unwindtable$?_Copy@?$basic_string@DU?$char_traits@D@std@@V?$allocator@D@2@@std@@QAEXII@Z 10000020     SeqBootAdapter.obj
 0002:fffbe020       __unwindtable$?_Copy@?$basic_string@DU?$char_traits@D@std@@V?$allocator@D@2@@std@@QAEXII@Z 10000020     protdist.obj
 0002:fffbe020       __unwindtable$?_Copy@?$basic_string@DU?$char_traits@D@std@@V?$allocator@D@2@@std@@QAEXII@Z 10000020     dist.obj
 0002:fffbe020       __unwindtable$?_Copy@?$basic_string@DU?$char_traits@D@std@@V?$allocator@D@2@@std@@QAEXII@Z 10000020     phylip.obj
 0002:fffbe020       __unwindtable$?_Copy@?$basic_string@DU?$char_traits@D@std@@V?$allocator@D@2@@std@@QAEXII@Z 10000020     moc_PhylipPlugin.obj
 0002:fffbe020       __unwindtable$?_Copy@?$basic_string@DU?$char_traits@D@std@@V?$allocator@D@2@@std@@QAEXII@Z 10000020     NeighborJoinAdapter.obj
 0002:fffbe020       __ehfuncinfo$?reallocData@?$QVector@VMultipleSequenceAlignment@U2@@@@AAEXHHV?$QFlags@W4AllocationOption@QArrayData@@@@@Z 10000020     seqboot.obj
 0002:fffbe020       __unwindtable$?_Copy@?$basic_string@DU?$char_traits@D@std@@V?$allocator@D@2@@std@@QAEXII@Z 10000020     moc_PhylipCmdlineTask.obj
 0002:fffbe020       __unwindtable$?detach_helper_grow@?$QList@VQString@@@@AAEPAUNode@1@HH@Z 10000020     dnadist.obj
 0002:fffbe020       __unwindtable$?_Copy@?$basic_string@DU?$char_traits@D@std@@V?$allocator@D@2@@std@@QAEXII@Z 10000020     NeighborJoinWidget.obj
 0002:fffbe020       __unwindtable$?detach_helper_grow@?$QList@VQString@@@@AAEPAUNode@1@HH@Z 10000020     protdist.obj
 0002:fffbe020       __tryblocktable$??0?$QList@VQString@@@@QAE@ABV0@@Z 10000020     dnadist.obj
 0002:fffbe020       __unwindtable$?reallocData@?$QVector@M@@AAEXHHV?$QFlags@W4AllocationOption@QArrayData@@@@@Z 10000020     NeighborJoinAdapter.obj
 0001:fffff022       __ehhandler$?append@?$QList@VQString@@@@QAEXABVQString@@@Z 10000022 f   dnadist.obj
 0001:fffff022       __ehhandler$?append@?$QList@VQString@@@@QAEXABVQString@@@Z 10000022 f   NeighborJoinWidget.obj
 0001:fffff022       __ehhandler$?append@?$QList@VQString@@@@QAEXABVQString@@@Z 10000022 f   protdist.obj
 0001:fffff022       __ehhandler$?append@?$QList@VQString@@@@QAEXABVQString@@@Z 10000022 f   PhylipCmdlineTask.obj
 0002:fffbe024       __unwindtable$?defaultConstruct@?$QVector@VMultipleSequenceAlignment@U2@@@@AAEXPAVMultipleSequenceAlignment@U2@@0@Z 10000024     seqboot.obj
 0002:fffbe024       __ehfuncinfo$?node_copy@?$QList@VQString@@@@AAEXPAUNode@1@00@Z 10000024     protdist.obj
 0002:fffbe024       __ehfuncinfo$?node_copy@?$QList@VQString@@@@AAEXPAUNode@1@00@Z 10000024     dnadist.obj
 0002:fffbe024       __ehfuncinfo$?node_copy@?$QList@VQString@@@@AAEXPAUNode@1@00@Z 10000024     PhylipCmdlineTask.obj
 0002:fffbe024       __ehfuncinfo$?node_copy@?$QList@VQString@@@@AAEXPAUNode@1@00@Z 10000024     NeighborJoinWidget.obj
 0001:fffff02a       __unwindfunclet$?defaultConstruct@?$QVector@VMultipleSequenceAlignment@U2@@@@AAEXPAVMultipleSequenceAlignment@U2@@0@Z$2 1000002a f   seqboot.obj
 0002:fffbe034       __ehfuncinfo$??0?$QList@VQString@@@@QAE@ABV0@@Z 10000034     dnadist.obj
 0002:fffbe034       __ehfuncinfo$??0?$QList@VQString@@@@QAE@ABV0@@Z 10000034     protdist.obj
 0002:fffbe040       __ehfuncinfo$?_Copy@?$basic_string@DU?$char_traits@D@std@@V?$allocator@D@2@@std@@QAEXII@Z 10000040     dnadist.obj
 0002:fffbe040       __ehfuncinfo$?_Copy@?$basic_string@DU?$char_traits@D@std@@V?$allocator@D@2@@std@@QAEXII@Z 10000040     dist.obj
 0002:fffbe040       __ehfuncinfo$?detach_helper_grow@?$QList@VQString@@@@AAEPAUNode@1@HH@Z 10000040     NeighborJoinWidget.obj
 0002:fffbe040       __ehfuncinfo$?_Copy@?$basic_string@DU?$char_traits@D@std@@V?$allocator@D@2@@std@@QAEXII@Z 10000040     PhylipTask.obj
 0002:fffbe040       __ehfuncinfo$?_Copy@?$basic_string@DU?$char_traits@D@std@@V?$allocator@D@2@@std@@QAEXII@Z 10000040     protdist.obj
 0002:fffbe040       __ehfuncinfo$?_Copy@?$basic_string@DU?$char_traits@D@std@@V?$allocator@D@2@@std@@QAEXII@Z 10000040     PhylipPlugin.obj
 0002:fffbe040       __ehfuncinfo$?_Copy@?$basic_string@DU?$char_traits@D@std@@V?$allocator@D@2@@std@@QAEXII@Z 10000040     NeighborJoinAdapter.obj
 0002:fffbe040       __ehfuncinfo$?detach_helper_grow@?$QList@VQString@@@@AAEPAUNode@1@HH@Z 10000040     protdist.obj
 0002:fffbe040       __ehfuncinfo$?_Copy@?$basic_string@DU?$char_traits@D@std@@V?$allocator@D@2@@std@@QAEXII@Z 10000040     moc_PhylipPlugin.obj
 0002:fffbe040       __ehfuncinfo$?_Copy@?$basic_string@DU?$char_traits@D@std@@V?$allocator@D@2@@std@@QAEXII@Z 10000040     SeqBootAdapter.obj
 0002:fffbe040       __ehfuncinfo$?_Copy@?$basic_string@DU?$char_traits@D@std@@V?$allocator@D@2@@std@@QAEXII@Z 10000040     moc_PhylipTask.obj
 0002:fffbe040       __ehfuncinfo$?detach_helper_grow@?$QList@VQString@@@@AAEPAUNode@1@HH@Z 10000040     PhylipCmdlineTask.obj
 0002:fffbe040       __ehfuncinfo$?detach_helper_grow@?$QList@VQString@@@@AAEPAUNode@1@HH@Z 10000040     dnadist.obj
 0002:fffbe040       __ehfuncinfo$?_Copy@?$basic_string@DU?$char_traits@D@std@@V?$allocator@D@2@@std@@QAEXII@Z 10000040     NeighborJoinWidget.obj
 0002:fffbe040       __ehfuncinfo$?_Copy@?$basic_string@DU?$char_traits@D@std@@V?$allocator@D@2@@std@@QAEXII@Z 10000040     PhylipCmdlineTask.obj
 0002:fffbe040       __ehfuncinfo$?_Copy@?$basic_string@DU?$char_traits@D@std@@V?$allocator@D@2@@std@@QAEXII@Z 10000040     moc_PhylipPluginTests.obj
 0002:fffbe040       __ehfuncinfo$?_Copy@?$basic_string@DU?$char_traits@D@std@@V?$allocator@D@2@@std@@QAEXII@Z 10000040     PhylipPluginTests.obj
 0002:fffbe040       __ehfuncinfo$?_Copy@?$basic_string@DU?$char_traits@D@std@@V?$allocator@D@2@@std@@QAEXII@Z 10000040     seqboot.obj
 0002:fffbe040       __ehfuncinfo$?_Copy@?$basic_string@DU?$char_traits@D@std@@V?$allocator@D@2@@std@@QAEXII@Z 10000040     neighbor.obj
 0002:fffbe040       __ehfuncinfo$?_Copy@?$basic_string@DU?$char_traits@D@std@@V?$allocator@D@2@@std@@QAEXII@Z 10000040     moc_PhylipCmdlineTask.obj
 0002:fffbe040       __ehfuncinfo$?_Copy@?$basic_string@DU?$char_traits@D@std@@V?$allocator@D@2@@std@@QAEXII@Z 10000040     phylip.obj
 0002:fffbe040       __ehfuncinfo$?reallocData@?$QVector@M@@AAEXHHV?$QFlags@W4AllocationOption@QArrayData@@@@@Z 10000040     NeighborJoinAdapter.obj
 0002:fffbe040       __ehfuncinfo$?_Copy@?$basic_string@DU?$char_traits@D@std@@V?$allocator@D@2@@std@@QAEXII@Z 10000040     moc_NeighborJoinWidget.obj
 0002:fffbe044       __tryblocktable$?append@?$QList@VQString@@@@QAEXABVQString@@@Z 10000044     PhylipCmdlineTask.obj
 0001:fffff044       __ehhandler$?defaultConstruct@?$QVector@VMultipleSequenceAlignment@U2@@@@AAEXPAVMultipleSequenceAlignment@U2@@0@Z 10000044 f   seqboot.obj
 0002:fffbe044       __tryblocktable$?reallocData@?$QVector@VMultipleSequenceAlignment@U2@@@@AAEXHHV?$QFlags@W4AllocationOption@QArrayData@@@@@Z 10000044     seqboot.obj
 0002:fffbe044       __tryblocktable$?append@?$QList@VQString@@@@QAEXABVQString@@@Z 10000044     protdist.obj
 0002:fffbe044       __tryblocktable$?append@?$QList@VQString@@@@QAEXABVQString@@@Z 10000044     NeighborJoinWidget.obj
 0002:fffbe044       __tryblocktable$?reallocData@?$QVector@V?$QVector@M@@@@AAEXHHV?$QFlags@W4AllocationOption@QArrayData@@@@@Z 10000044     NeighborJoinAdapter.obj
 0002:fffbe044       __tryblocktable$?append@?$QList@VQString@@@@QAEXABVQString@@@Z 10000044     dnadist.obj
 0002:fffbe048       __unwindtable$?node_copy@?$QList@VQString@@@@AAEXPAUNode@1@00@Z 10000048     dnadist.obj
 0002:fffbe048       __unwindtable$?node_copy@?$QList@VQString@@@@AAEXPAUNode@1@00@Z 10000048     PhylipCmdlineTask.obj
 0002:fffbe048       __unwindtable$?node_copy@?$QList@VQString@@@@AAEXPAUNode@1@00@Z 10000048     protdist.obj
 0002:fffbe048       __unwindtable$?node_copy@?$QList@VQString@@@@AAEXPAUNode@1@00@Z 10000048     NeighborJoinWidget.obj
 0001:fffff062       __catch$?node_copy@?$QList@VQString@@@@AAEXPAUNode@1@00@Z$2 10000062 f   dnadist.obj
 0001:fffff062       __catch$?node_copy@?$QList@VQString@@@@AAEXPAUNode@1@00@Z$2 10000062 f   PhylipCmdlineTask.obj
 0001:fffff062       __catch$?node_copy@?$QList@VQString@@@@AAEXPAUNode@1@00@Z$2 10000062 f   NeighborJoinWidget.obj
 0001:fffff062       __catch$?node_copy@?$QList@VQString@@@@AAEXPAUNode@1@00@Z$2 10000062 f   protdist.obj
 0002:fffbe064       __tryblocktable$?_Copy@?$basic_string@DU?$char_traits@D@std@@V?$allocator@D@2@@std@@QAEXII@Z 10000064     dnadist.obj
 0002:fffbe064       __tryblocktable$?_Copy@?$basic_string@DU?$char_traits@D@std@@V?$allocator@D@2@@std@@QAEXII@Z 10000064     dist.obj
 0002:fffbe064       __tryblocktable$?reallocData@?$QVector@M@@AAEXHHV?$QFlags@W4AllocationOption@QArrayData@@@@@Z 10000064     NeighborJoinAdapter.obj
 0002:fffbe064       __tryblocktable$?_Copy@?$basic_string@DU?$char_traits@D@std@@V?$allocator@D@2@@std@@QAEXII@Z 10000064     neighbor.obj
 0002:fffbe064       __tryblocktable$?_Copy@?$basic_string@DU?$char_traits@D@std@@V?$allocator@D@2@@std@@QAEXII@Z 10000064     NeighborJoinAdapter.obj
 0002:fffbe064       __tryblocktable$?_Copy@?$basic_string@DU?$char_traits@D@std@@V?$allocator@D@2@@std@@QAEXII@Z 10000064     PhylipPlugin.obj
 0002:fffbe064       __tryblocktable$?detach_helper_grow@?$QList@VQString@@@@AAEPAUNode@1@HH@Z 10000064     NeighborJoinWidget.obj
 0002:fffbe064       __tryblocktable$?detach_helper_grow@?$QList@VQString@@@@AAEPAUNode@1@HH@Z 10000064     protdist.obj
 0002:fffbe064       __tryblocktable$?_Copy@?$basic_string@DU?$char_traits@D@std@@V?$allocator@D@2@@std@@QAEXII@Z 10000064     moc_PhylipTask.obj
 0002:fffbe064       __tryblocktable$?_Copy@?$basic_string@DU?$char_traits@D@std@@V?$allocator@D@2@@std@@QAEXII@Z 10000064     moc_NeighborJoinWidget.obj
 0002:fffbe064       __tryblocktable$?_Copy@?$basic_string@DU?$char_traits@D@std@@V?$allocator@D@2@@std@@QAEXII@Z 10000064     NeighborJoinWidget.obj
 0002:fffbe064       __tryblocktable$?detach_helper_grow@?$QList@VQString@@@@AAEPAUNode@1@HH@Z 10000064     dnadist.obj
 0002:fffbe064       __tryblocktable$?_Copy@?$basic_string@DU?$char_traits@D@std@@V?$allocator@D@2@@std@@QAEXII@Z 10000064     SeqBootAdapter.obj
 0002:fffbe064       __tryblocktable$?detach_helper_grow@?$QList@VQString@@@@AAEPAUNode@1@HH@Z 10000064     PhylipCmdlineTask.obj
 0002:fffbe064       __tryblocktable$?_Copy@?$basic_string@DU?$char_traits@D@std@@V?$allocator@D@2@@std@@QAEXII@Z 10000064     phylip.obj
 0002:fffbe064       __tryblocktable$?_Copy@?$basic_string@DU?$char_traits@D@std@@V?$allocator@D@2@@std@@QAEXII@Z 10000064     PhylipCmdlineTask.obj
 0002:fffbe064       __tryblocktable$?_Copy@?$basic_string@DU?$char_traits@D@std@@V?$allocator@D@2@@std@@QAEXII@Z 10000064     moc_PhylipPluginTests.obj
 0002:fffbe064       __tryblocktable$?_Copy@?$basic_string@DU?$char_traits@D@std@@V?$allocator@D@2@@std@@QAEXII@Z 10000064     seqboot.obj
 0002:fffbe064       __tryblocktable$?_Copy@?$basic_string@DU?$char_traits@D@std@@V?$allocator@D@2@@std@@QAEXII@Z 10000064     PhylipTask.obj
 0002:fffbe064       __tryblocktable$?_Copy@?$basic_string@DU?$char_traits@D@std@@V?$allocator@D@2@@std@@QAEXII@Z 10000064     PhylipPluginTests.obj
 0002:fffbe064       __tryblocktable$?_Copy@?$basic_string@DU?$char_traits@D@std@@V?$allocator@D@2@@std@@QAEXII@Z 10000064     protdist.obj
 0002:fffbe064       __tryblocktable$?_Copy@?$basic_string@DU?$char_traits@D@std@@V?$allocator@D@2@@std@@QAEXII@Z 10000064     moc_PhylipCmdlineTask.obj
 0002:fffbe064       __tryblocktable$?_Copy@?$basic_string@DU?$char_traits@D@std@@V?$allocator@D@2@@std@@QAEXII@Z 10000064     moc_PhylipPlugin.obj
 0002:fffbe06c       __unwindtable$?append@?$QList@VQString@@@@QAEXABVQString@@@Z 1000006c     dnadist.obj
 0002:fffbe06c       __unwindtable$?append@?$QList@VQString@@@@QAEXABVQString@@@Z 1000006c     NeighborJoinWidget.obj
 0002:fffbe06c       __unwindtable$?reallocData@?$QVector@VMultipleSequenceAlignment@U2@@@@AAEXHHV?$QFlags@W4AllocationOption@QArrayData@@@@@Z 1000006c     seqboot.obj
 0002:fffbe06c       __unwindtable$?append@?$QList@VQString@@@@QAEXABVQString@@@Z 1000006c     protdist.obj
 0002:fffbe06c       __unwindtable$?reallocData@?$QVector@V?$QVector@M@@@@AAEXHHV?$QFlags@W4AllocationOption@QArrayData@@@@@Z 1000006c     NeighborJoinAdapter.obj
 0002:fffbe06c       __unwindtable$?append@?$QList@VQString@@@@QAEXABVQString@@@Z 1000006c     PhylipCmdlineTask.obj
 0001:fffff07d       __catch$?append@?$QList@VQString@@@@QAEXABVQString@@@Z$0 1000007d f   dnadist.obj
 0001:fffff07d       __catch$?append@?$QList@VQString@@@@QAEXABVQString@@@Z$0 1000007d f   PhylipCmdlineTask.obj
 0001:fffff07d       __catch$?append@?$QList@VQString@@@@QAEXABVQString@@@Z$0 1000007d f   protdist.obj
 0001:fffff07d       __catch$?append@?$QList@VQString@@@@QAEXABVQString@@@Z$0 1000007d f   NeighborJoinWidget.obj
 0001:fffff096       __catch$?_Copy@?$basic_string@DU?$char_traits@D@std@@V?$allocator@D@2@@std@@QAEXII@Z$0 10000096 f   moc_PhylipTask.obj
 0001:fffff096       __catch$?_Copy@?$basic_string@DU?$char_traits@D@std@@V?$allocator@D@2@@std@@QAEXII@Z$0 10000096 f   moc_PhylipCmdlineTask.obj
 0001:fffff096       __catch$?_Copy@?$basic_string@DU?$char_traits@D@std@@V?$allocator@D@2@@std@@QAEXII@Z$0 10000096 f   seqboot.obj
 0001:fffff096       __catch$?_Copy@?$basic_string@DU?$char_traits@D@std@@V?$allocator@D@2@@std@@QAEXII@Z$0 10000096 f   moc_PhylipPluginTests.obj
 0001:fffff096       __catch$?_Copy@?$basic_string@DU?$char_traits@D@std@@V?$allocator@D@2@@std@@QAEXII@Z$0 10000096 f   protdist.obj
 0001:fffff096       __catch$?_Copy@?$basic_string@DU?$char_traits@D@std@@V?$allocator@D@2@@std@@QAEXII@Z$0 10000096 f   dist.obj
 0001:fffff096       __catch$?_Copy@?$basic_string@DU?$char_traits@D@std@@V?$allocator@D@2@@std@@QAEXII@Z$0 10000096 f   dnadist.obj
 0001:fffff096       __catch$?_Copy@?$basic_string@DU?$char_traits@D@std@@V?$allocator@D@2@@std@@QAEXII@Z$0 10000096 f   phylip.obj
 0001:fffff096       __catch$?_Copy@?$basic_string@DU?$char_traits@D@std@@V?$allocator@D@2@@std@@QAEXII@Z$0 10000096 f   PhylipTask.obj
 0001:fffff096       __catch$?_Copy@?$basic_string@DU?$char_traits@D@std@@V?$allocator@D@2@@std@@QAEXII@Z$0 10000096 f   moc_PhylipPlugin.obj
 0001:fffff096       __catch$?_Copy@?$basic_string@DU?$char_traits@D@std@@V?$allocator@D@2@@std@@QAEXII@Z$0 10000096 f   neighbor.obj
 0001:fffff096       __catch$?_Copy@?$basic_string@DU?$char_traits@D@std@@V?$allocator@D@2@@std@@QAEXII@Z$0 10000096 f   moc_NeighborJoinWidget.obj
 0001:fffff096       __catch$?_Copy@?$basic_string@DU?$char_traits@D@std@@V?$allocator@D@2@@std@@QAEXII@Z$0 10000096 f   NeighborJoinWidget.obj
 0001:fffff096       __catch$?_Copy@?$basic_string@DU?$char_traits@D@std@@V?$allocator@D@2@@std@@QAEXII@Z$0 10000096 f   PhylipPluginTests.obj
 0001:fffff096       __catch$?_Copy@?$basic_string@DU?$char_traits@D@std@@V?$allocator@D@2@@std@@QAEXII@Z$0 10000096 f   PhylipCmdlineTask.obj
 0001:fffff096       __catch$?_Copy@?$basic_string@DU?$char_traits@D@std@@V?$allocator@D@2@@std@@QAEXII@Z$0 10000096 f   PhylipPlugin.obj
 0001:fffff096       __catch$?_Copy@?$basic_string@DU?$char_traits@D@std@@V?$allocator@D@2@@std@@QAEXII@Z$0 10000096 f   NeighborJoinAdapter.obj
 0001:fffff096       __catch$?_Copy@?$basic_string@DU?$char_traits@D@std@@V?$allocator@D@2@@std@@QAEXII@Z$0 10000096 f   SeqBootAdapter.obj
 0001:fffff09e       __catch$??0?$QList@VQString@@@@QAE@ABV0@@Z$0 1000009e f   dnadist.obj
 0001:fffff09e       __catch$??0?$QList@VQString@@@@QAE@ABV0@@Z$0 1000009e f   protdist.obj
 0001:fffff0ce       __catch$?append@?$QList@VQString@@@@QAEXABVQString@@@Z$4 100000ce f   NeighborJoinWidget.obj
 0001:fffff0ce       __catch$?append@?$QList@VQString@@@@QAEXABVQString@@@Z$4 100000ce f   PhylipCmdlineTask.obj
 0001:fffff0ce       __catch$?append@?$QList@VQString@@@@QAEXABVQString@@@Z$4 100000ce f   dnadist.obj
 0001:fffff0ce       __catch$?append@?$QList@VQString@@@@QAEXABVQString@@@Z$4 100000ce f   protdist.obj
 0001:fffff0d3       __catch$?_Copy@?$basic_string@DU?$char_traits@D@std@@V?$allocator@D@2@@std@@QAEXII@Z$1 100000d3 f   neighbor.obj
 0001:fffff0d3       __catch$?_Copy@?$basic_string@DU?$char_traits@D@std@@V?$allocator@D@2@@std@@QAEXII@Z$1 100000d3 f   PhylipTask.obj
 0001:fffff0d3       __catch$?_Copy@?$basic_string@DU?$char_traits@D@std@@V?$allocator@D@2@@std@@QAEXII@Z$1 100000d3 f   moc_PhylipPlugin.obj
 0001:fffff0d3       __catch$?_Copy@?$basic_string@DU?$char_traits@D@std@@V?$allocator@D@2@@std@@QAEXII@Z$1 100000d3 f   PhylipCmdlineTask.obj
 0001:fffff0d3       __catch$?_Copy@?$basic_string@DU?$char_traits@D@std@@V?$allocator@D@2@@std@@QAEXII@Z$1 100000d3 f   phylip.obj
 0001:fffff0d3       __catch$?_Copy@?$basic_string@DU?$char_traits@D@std@@V?$allocator@D@2@@std@@QAEXII@Z$1 100000d3 f   moc_NeighborJoinWidget.obj
 0001:fffff0d3       __catch$?_Copy@?$basic_string@DU?$char_traits@D@std@@V?$allocator@D@2@@std@@QAEXII@Z$1 100000d3 f   moc_PhylipCmdlineTask.obj
 0001:fffff0d3       __catch$?_Copy@?$basic_string@DU?$char_traits@D@std@@V?$allocator@D@2@@std@@QAEXII@Z$1 100000d3 f   seqboot.obj
 0001:fffff0d3       __catch$?_Copy@?$basic_string@DU?$char_traits@D@std@@V?$allocator@D@2@@std@@QAEXII@Z$1 100000d3 f   moc_PhylipPluginTests.obj
 0001:fffff0d3       __catch$?_Copy@?$basic_string@DU?$char_traits@D@std@@V?$allocator@D@2@@std@@QAEXII@Z$1 100000d3 f   PhylipPluginTests.obj
 0001:fffff0d3       __catch$?_Copy@?$basic_string@DU?$char_traits@D@std@@V?$allocator@D@2@@std@@QAEXII@Z$1 100000d3 f   moc_PhylipTask.obj
 0001:fffff0d3       __catch$?_Copy@?$basic_string@DU?$char_traits@D@std@@V?$allocator@D@2@@std@@QAEXII@Z$1 100000d3 f   NeighborJoinWidget.obj
 0001:fffff0d3       __catch$?_Copy@?$basic_string@DU?$char_traits@D@std@@V?$allocator@D@2@@std@@QAEXII@Z$1 100000d3 f   protdist.obj
 0001:fffff0d3       __catch$?_Copy@?$basic_string@DU?$char_traits@D@std@@V?$allocator@D@2@@std@@QAEXII@Z$1 100000d3 f   NeighborJoinAdapter.obj
 0001:fffff0d3       __catch$?_Copy@?$basic_string@DU?$char_traits@D@std@@V?$allocator@D@2@@std@@QAEXII@Z$1 100000d3 f   PhylipPlugin.obj
 0001:fffff0d3       __catch$?_Copy@?$basic_string@DU?$char_traits@D@std@@V?$allocator@D@2@@std@@QAEXII@Z$1 100000d3 f   SeqBootAdapter.obj
 0001:fffff0d3       __catch$?_Copy@?$basic_string@DU?$char_traits@D@std@@V?$allocator@D@2@@std@@QAEXII@Z$1 100000d3 f   dnadist.obj
 0001:fffff0d3       __catch$?_Copy@?$basic_string@DU?$char_traits@D@std@@V?$allocator@D@2@@std@@QAEXII@Z$1 100000d3 f   dist.obj
 0001:fffff11e       __catch$?detach_helper_grow@?$QList@VQString@@@@AAEPAUNode@1@HH@Z$2 1000011e f   NeighborJoinWidget.obj
 0001:fffff11e       __catch$?detach_helper_grow@?$QList@VQString@@@@AAEPAUNode@1@HH@Z$2 1000011e f   protdist.obj
 0001:fffff11e       __catch$?detach_helper_grow@?$QList@VQString@@@@AAEPAUNode@1@HH@Z$2 1000011e f   PhylipCmdlineTask.obj
 0001:fffff11e       __catch$?detach_helper_grow@?$QList@VQString@@@@AAEPAUNode@1@HH@Z$2 1000011e f   dnadist.obj
 0001:fffff159       __catch$?detach_helper_grow@?$QList@VQString@@@@AAEPAUNode@1@HH@Z$0 10000159 f   PhylipCmdlineTask.obj
 0001:fffff159       __catch$?detach_helper_grow@?$QList@VQString@@@@AAEPAUNode@1@HH@Z$0 10000159 f   NeighborJoinWidget.obj
 0001:fffff159       __catch$?detach_helper_grow@?$QList@VQString@@@@AAEPAUNode@1@HH@Z$0 10000159 f   dnadist.obj
 0001:fffff159       __catch$?detach_helper_grow@?$QList@VQString@@@@AAEPAUNode@1@HH@Z$0 10000159 f   protdist.obj
 0001:fffff1a4       __catch$?reallocData@?$QVector@M@@AAEXHHV?$QFlags@W4AllocationOption@QArrayData@@@@@Z$0 100001a4 f   NeighborJoinAdapter.obj
 0001:fffff1b6       __catch$?reallocData@?$QVector@M@@AAEXHHV?$QFlags@W4AllocationOption@QArrayData@@@@@Z$2 100001b6 f   NeighborJoinAdapter.obj
 0001:fffff1bd       __catch$?reallocData@?$QVector@VMultipleSequenceAlignment@U2@@@@AAEXHHV?$QFlags@W4AllocationOption@QArrayData@@@@@Z$0 100001bd f   seqboot.obj
 0001:fffff1db       __catch$?reallocData@?$QVector@VMultipleSequenceAlignment@U2@@@@AAEXHHV?$QFlags@W4AllocationOption@QArrayData@@@@@Z$2 100001db f   seqboot.obj
 0001:fffff224       __catch$?reallocData@?$QVector@V?$QVector@M@@@@AAEXHHV?$QFlags@W4AllocationOption@QArrayData@@@@@Z$0 10000224 f   NeighborJoinAdapter.obj
 0001:fffff242       __catch$?reallocData@?$QVector@V?$QVector@M@@@@AAEXHHV?$QFlags@W4AllocationOption@QArrayData@@@@@Z$2 10000242 f   NeighborJoinAdapter.obj
 0001:00000000       ??__E?_Generic_object@?$_Error_objects@H@std@@2V_Generic_error_category@2@A@@YAXXZ 10001000 f   DistanceMatrix.obj
 0001:00000010       ??__E?_Iostream_object@?$_Error_objects@H@std@@2V_Iostream_error_category@2@A@@YAXXZ 10001010 f   DistanceMatrix.obj
 0001:00000020       ??__E?_System_object@?$_Error_objects@H@std@@2V_System_error_category@2@A@@YAXXZ 10001020 f   DistanceMatrix.obj
 0001:00000030       ??__EalgoLog@U2@@YAXXZ     10001030 f   DistanceMatrix.obj
 0001:000000b0       ??__EcmdLog@U2@@YAXXZ      100010b0 f   DistanceMatrix.obj
 0001:00000130       ??__EcoreLog@U2@@YAXXZ     10001130 f   DistanceMatrix.obj
 0001:000001b0       ??__EioLog@U2@@YAXXZ       100011b0 f   DistanceMatrix.obj
 0001:00000230       ??__EperfLog@U2@@YAXXZ     10001230 f   DistanceMatrix.obj
 0001:000002b0       ??__EscriptLog@U2@@YAXXZ   100012b0 f   DistanceMatrix.obj
 0001:00000330       ??__EtaskLog@U2@@YAXXZ     10001330 f   DistanceMatrix.obj
 0001:000003b0       ??__EuiLog@U2@@YAXXZ       100013b0 f   DistanceMatrix.obj
 0001:00000430       ??__EuserActLog@U2@@YAXXZ  10001430 f   DistanceMatrix.obj
 0001:000004b0       ??__E?_Generic_object@?$_Error_objects@H@std@@2V_Generic_error_category@2@A@@YAXXZ 100014b0 f   NeighborJoinAdapter.obj
 0001:000004c0       ??__E?_Iostream_object@?$_Error_objects@H@std@@2V_Iostream_error_category@2@A@@YAXXZ 100014c0 f   NeighborJoinAdapter.obj
 0001:000004d0       ??__E?_System_object@?$_Error_objects@H@std@@2V_System_error_category@2@A@@YAXXZ 100014d0 f   NeighborJoinAdapter.obj
 0001:000004e0       ??__E?runLock@NeighborJoinCalculateTreeTask@U2@@0VQMutex@@A@@YAXXZ 100014e0 f   NeighborJoinAdapter.obj
 0001:00000500       ??__EalgoLog@U2@@YAXXZ     10001500 f   NeighborJoinAdapter.obj
 0001:00000580       ??__EcmdLog@U2@@YAXXZ      10001580 f   NeighborJoinAdapter.obj
 0001:00000600       ??__EcoreLog@U2@@YAXXZ     10001600 f   NeighborJoinAdapter.obj
 0001:00000680       ??__EioLog@U2@@YAXXZ       10001680 f   NeighborJoinAdapter.obj
 0001:00000700       ??__EperfLog@U2@@YAXXZ     10001700 f   NeighborJoinAdapter.obj
 0001:00000780       ??__EscriptLog@U2@@YAXXZ   10001780 f   NeighborJoinAdapter.obj
 0001:00000800       ??__EtaskLog@U2@@YAXXZ     10001800 f   NeighborJoinAdapter.obj
 0001:00000880       ??__EuiLog@U2@@YAXXZ       10001880 f   NeighborJoinAdapter.obj
 0001:00000900       ??__EuserActLog@U2@@YAXXZ  10001900 f   NeighborJoinAdapter.obj
 0001:00000980       ??__E?M1@ConsensusModelTypes@U2@@2VQString@@A@@YAXXZ 10001980 f   NeighborJoinWidget.obj
 0001:000009a0       ??__E?MajorityRule@ConsensusModelTypes@U2@@2VQString@@A@@YAXXZ 100019a0 f   NeighborJoinWidget.obj
 0001:000009c0       ??__E?MajorityRuleExt@ConsensusModelTypes@U2@@2VQString@@A@@YAXXZ 100019c0 f   NeighborJoinWidget.obj
 0001:000009e0       ??__E?Strict@ConsensusModelTypes@U2@@2VQString@@A@@YAXXZ 100019e0 f   NeighborJoinWidget.obj
 0001:00000a00       ??__E?_Generic_object@?$_Error_objects@H@std@@2V_Generic_error_category@2@A@@YAXXZ 10001a00 f   NeighborJoinWidget.obj
 0001:00000a10       ??__E?_Iostream_object@?$_Error_objects@H@std@@2V_Iostream_error_category@2@A@@YAXXZ 10001a10 f   NeighborJoinWidget.obj
 0001:00000a20       ??__E?_System_object@?$_Error_objects@H@std@@2V_System_error_category@2@A@@YAXXZ 10001a20 f   NeighborJoinWidget.obj
 0001:00000a30       ??__EalgoLog@U2@@YAXXZ     10001a30 f   NeighborJoinWidget.obj
 0001:00000ab0       ??__EcmdLog@U2@@YAXXZ      10001ab0 f   NeighborJoinWidget.obj
 0001:00000b30       ??__EcoreLog@U2@@YAXXZ     10001b30 f   NeighborJoinWidget.obj
 0001:00000bb0       ??__EioLog@U2@@YAXXZ       10001bb0 f   NeighborJoinWidget.obj
 0001:00000c30       ??__EperfLog@U2@@YAXXZ     10001c30 f   NeighborJoinWidget.obj
 0001:00000cb0       ??__EscriptLog@U2@@YAXXZ   10001cb0 f   NeighborJoinWidget.obj
 0001:00000d30       ??__EtaskLog@U2@@YAXXZ     10001d30 f   NeighborJoinWidget.obj
 0001:00000db0       ??__EuiLog@U2@@YAXXZ       10001db0 f   NeighborJoinWidget.obj
 0001:00000e30       ??__EuserActLog@U2@@YAXXZ  10001e30 f   NeighborJoinWidget.obj
 0001:00000eb0       ??__E?ALPHA_ARG@PhylipCmdlineTask@U2@@2VQString@@B@@YAXXZ 10001eb0 f   PhylipCmdlineTask.obj
 0001:00000ed0       ??__E?BOOTSTRAP_ARG@PhylipCmdlineTask@U2@@2VQString@@B@@YAXXZ 10001ed0 f   PhylipCmdlineTask.obj
 0001:00000ef0       ??__E?CONSENSUS_ARG@PhylipCmdlineTask@U2@@2VQString@@B@@YAXXZ 10001ef0 f   PhylipCmdlineTask.obj
 0001:00000f10       ??__E?FRACTION_ARG@PhylipCmdlineTask@U2@@2VQString@@B@@YAXXZ 10001f10 f   PhylipCmdlineTask.obj
 0001:00000f30       ??__E?GAMMA_ARG@PhylipCmdlineTask@U2@@2VQString@@B@@YAXXZ 10001f30 f   PhylipCmdlineTask.obj
 0001:00000f50       ??__E?MATRIX_ARG@PhylipCmdlineTask@U2@@2VQString@@B@@YAXXZ 10001f50 f   PhylipCmdlineTask.obj
 0001:00000f70       ??__E?PHYLIP_CMDLINE@PhylipCmdlineTask@U2@@2VQString@@B@@YAXXZ 10001f70 f   PhylipCmdlineTask.obj
 0001:00000f90       ??__E?REPLICATES_ARG@PhylipCmdlineTask@U2@@2VQString@@B@@YAXXZ 10001f90 f   PhylipCmdlineTask.obj
 0001:00000fb0       ??__E?SEED_ARG@PhylipCmdlineTask@U2@@2VQString@@B@@YAXXZ 10001fb0 f   PhylipCmdlineTask.obj
 0001:00000fd0       ??__E?TT_RATIO_ARG@PhylipCmdlineTask@U2@@2VQString@@B@@YAXXZ 10001fd0 f   PhylipCmdlineTask.obj
 0001:00000ff0       ??__E?_Generic_object@?$_Error_objects@H@std@@2V_Generic_error_category@2@A@@YAXXZ 10001ff0 f   PhylipCmdlineTask.obj
 0001:00001000       ??__E?_Iostream_object@?$_Error_objects@H@std@@2V_Iostream_error_category@2@A@@YAXXZ 10002000 f   PhylipCmdlineTask.obj
 0001:00001010       ??__E?_System_object@?$_Error_objects@H@std@@2V_System_error_category@2@A@@YAXXZ 10002010 f   PhylipCmdlineTask.obj
 0001:00001020       ??__EalgoLog@U2@@YAXXZ     10002020 f   PhylipCmdlineTask.obj
 0001:000010a0       ??__EcmdLog@U2@@YAXXZ      100020a0 f   PhylipCmdlineTask.obj
 0001:00001120       ??__EcoreLog@U2@@YAXXZ     10002120 f   PhylipCmdlineTask.obj
 0001:000011a0       ??__EioLog@U2@@YAXXZ       100021a0 f   PhylipCmdlineTask.obj
 0001:00001220       ??__EperfLog@U2@@YAXXZ     10002220 f   PhylipCmdlineTask.obj
 0001:000012a0       ??__EscriptLog@U2@@YAXXZ   100022a0 f   PhylipCmdlineTask.obj
 0001:00001320       ??__EtaskLog@U2@@YAXXZ     10002320 f   PhylipCmdlineTask.obj
 0001:000013a0       ??__EuiLog@U2@@YAXXZ       100023a0 f   PhylipCmdlineTask.obj
 0001:00001420       ??__EuserActLog@U2@@YAXXZ  10002420 f   PhylipCmdlineTask.obj
 0001:000014a0       ??__E?PHYLIP_NEIGHBOUR_JOIN@PhylipPlugin@U2@@2VQString@@B@@YAXXZ 100024a0 f   PhylipPlugin.obj
 0001:000014c0       ??__E?_Generic_object@?$_Error_objects@H@std@@2V_Generic_error_category@2@A@@YAXXZ 100024c0 f   PhylipPlugin.obj
 0001:000014d0       ??__E?_Iostream_object@?$_Error_objects@H@std@@2V_Iostream_error_category@2@A@@YAXXZ 100024d0 f   PhylipPlugin.obj
 0001:000014e0       ??__E?_System_object@?$_Error_objects@H@std@@2V_System_error_category@2@A@@YAXXZ 100024e0 f   PhylipPlugin.obj
 0001:000014f0       ??__EService_DNAExport@U2@@YAXXZ 100024f0 f   PhylipPlugin.obj
 0001:00001500       ??__EService_DNAGraphPack@U2@@YAXXZ 10002500 f   PhylipPlugin.obj
 0001:00001510       ??__EService_ExternalToolSupport@U2@@YAXXZ 10002510 f   PhylipPlugin.obj
 0001:00001520       ??__EService_GUITesting@U2@@YAXXZ 10002520 f   PhylipPlugin.obj
 0001:00001530       ??__EService_MaxCoreServiceId@U2@@YAXXZ 10002530 f   PhylipPlugin.obj
 0001:00001540       ??__EService_MinCoreServiceId@U2@@YAXXZ 10002540 f   PhylipPlugin.obj
 0001:00001550       ??__EService_PluginViewer@U2@@YAXXZ 10002550 f   PhylipPlugin.obj
 0001:00001560       ??__EService_Project@U2@@YAXXZ 10002560 f   PhylipPlugin.obj
 0001:00001570       ??__EService_ProjectView@U2@@YAXXZ 10002570 f   PhylipPlugin.obj
 0001:00001580       ??__EService_QueryDesigner@U2@@YAXXZ 10002580 f   PhylipPlugin.obj
 0001:00001590       ??__EService_ScriptRegistry@U2@@YAXXZ 10002590 f   PhylipPlugin.obj
 0001:000015a0       ??__EService_TestRunner@U2@@YAXXZ 100025a0 f   PhylipPlugin.obj
 0001:000015b0       ??__EService_WorkflowDesigner@U2@@YAXXZ 100025b0 f   PhylipPlugin.obj
 0001:000015c0       ??__EalgoLog@U2@@YAXXZ     100025c0 f   PhylipPlugin.obj
 0001:00001640       ??__EcmdLog@U2@@YAXXZ      10002640 f   PhylipPlugin.obj
 0001:000016c0       ??__EcoreLog@U2@@YAXXZ     100026c0 f   PhylipPlugin.obj
 0001:00001740       ??__EioLog@U2@@YAXXZ       10002740 f   PhylipPlugin.obj
 0001:000017c0       ??__EperfLog@U2@@YAXXZ     100027c0 f   PhylipPlugin.obj
 0001:00001840       ??__EscriptLog@U2@@YAXXZ   10002840 f   PhylipPlugin.obj
 0001:000018c0       ??__EtaskLog@U2@@YAXXZ     100028c0 f   PhylipPlugin.obj
 0001:00001940       ??__EuiLog@U2@@YAXXZ       10002940 f   PhylipPlugin.obj
 0001:000019c0       ??__EuserActLog@U2@@YAXXZ  100029c0 f   PhylipPlugin.obj
 0001:00001a40       ??__E?_Generic_object@?$_Error_objects@H@std@@2V_Generic_error_category@2@A@@YAXXZ 10002a40 f   PhylipPluginTests.obj
 0001:00001a50       ??__E?_Iostream_object@?$_Error_objects@H@std@@2V_Iostream_error_category@2@A@@YAXXZ 10002a50 f   PhylipPluginTests.obj
 0001:00001a60       ??__E?_System_object@?$_Error_objects@H@std@@2V_System_error_category@2@A@@YAXXZ 10002a60 f   PhylipPluginTests.obj
 0001:00001a70       ??__EService_DNAExport@U2@@YAXXZ 10002a70 f   PhylipPluginTests.obj
 0001:00001a80       ??__EService_DNAGraphPack@U2@@YAXXZ 10002a80 f   PhylipPluginTests.obj
 0001:00001a90       ??__EService_ExternalToolSupport@U2@@YAXXZ 10002a90 f   PhylipPluginTests.obj
 0001:00001aa0       ??__EService_GUITesting@U2@@YAXXZ 10002aa0 f   PhylipPluginTests.obj
 0001:00001ab0       ??__EService_MaxCoreServiceId@U2@@YAXXZ 10002ab0 f   PhylipPluginTests.obj
 0001:00001ac0       ??__EService_MinCoreServiceId@U2@@YAXXZ 10002ac0 f   PhylipPluginTests.obj
 0001:00001ad0       ??__EService_PluginViewer@U2@@YAXXZ 10002ad0 f   PhylipPluginTests.obj
 0001:00001ae0       ??__EService_Project@U2@@YAXXZ 10002ae0 f   PhylipPluginTests.obj
 0001:00001af0       ??__EService_ProjectView@U2@@YAXXZ 10002af0 f   PhylipPluginTests.obj
 0001:00001b00       ??__EService_QueryDesigner@U2@@YAXXZ 10002b00 f   PhylipPluginTests.obj
 0001:00001b10       ??__EService_ScriptRegistry@U2@@YAXXZ 10002b10 f   PhylipPluginTests.obj
 0001:00001b20       ??__EService_TestRunner@U2@@YAXXZ 10002b20 f   PhylipPluginTests.obj
 0001:00001b30       ??__EService_WorkflowDesigner@U2@@YAXXZ 10002b30 f   PhylipPluginTests.obj
 0001:00001b40       ??__EalgoLog@U2@@YAXXZ     10002b40 f   PhylipPluginTests.obj
 0001:00001bc0       ??__EcmdLog@U2@@YAXXZ      10002bc0 f   PhylipPluginTests.obj
 0001:00001c40       ??__EcoreLog@U2@@YAXXZ     10002c40 f   PhylipPluginTests.obj
 0001:00001cc0       ??__EioLog@U2@@YAXXZ       10002cc0 f   PhylipPluginTests.obj
 0001:00001d40       ??__EperfLog@U2@@YAXXZ     10002d40 f   PhylipPluginTests.obj
 0001:00001dc0       ??__EscriptLog@U2@@YAXXZ   10002dc0 f   PhylipPluginTests.obj
 0001:00001e40       ??__EtaskLog@U2@@YAXXZ     10002e40 f   PhylipPluginTests.obj
 0001:00001ec0       ??__EuiLog@U2@@YAXXZ       10002ec0 f   PhylipPluginTests.obj
 0001:00001f40       ??__EuserActLog@U2@@YAXXZ  10002f40 f   PhylipPluginTests.obj
 0001:00001fc0       ??__E?_Generic_object@?$_Error_objects@H@std@@2V_Generic_error_category@2@A@@YAXXZ 10002fc0 f   PhylipTask.obj
 0001:00001fd0       ??__E?_Iostream_object@?$_Error_objects@H@std@@2V_Iostream_error_category@2@A@@YAXXZ 10002fd0 f   PhylipTask.obj
 0001:00001fe0       ??__E?_System_object@?$_Error_objects@H@std@@2V_System_error_category@2@A@@YAXXZ 10002fe0 f   PhylipTask.obj
 0001:00001ff0       ??__EalgoLog@U2@@YAXXZ     10002ff0 f   PhylipTask.obj
 0001:00002070       ??__EcmdLog@U2@@YAXXZ      10003070 f   PhylipTask.obj
 0001:000020f0       ??__EcoreLog@U2@@YAXXZ     100030f0 f   PhylipTask.obj
 0001:00002170       ??__EioLog@U2@@YAXXZ       10003170 f   PhylipTask.obj
 0001:000021f0       ??__EperfLog@U2@@YAXXZ     100031f0 f   PhylipTask.obj
 0001:00002270       ??__EscriptLog@U2@@YAXXZ   10003270 f   PhylipTask.obj
 0001:000022f0       ??__EtaskLog@U2@@YAXXZ     100032f0 f   PhylipTask.obj
 0001:00002370       ??__EuiLog@U2@@YAXXZ       10003370 f   PhylipTask.obj
 0001:000023f0       ??__EuserActLog@U2@@YAXXZ  100033f0 f   PhylipTask.obj
 0001:00002470       ??__E?_Generic_object@?$_Error_objects@H@std@@2V_Generic_error_category@2@A@@YAXXZ 10003470 f   SeqBootAdapter.obj
 0001:00002480       ??__E?_Iostream_object@?$_Error_objects@H@std@@2V_Iostream_error_category@2@A@@YAXXZ 10003480 f   SeqBootAdapter.obj
 0001:00002490       ??__E?_System_object@?$_Error_objects@H@std@@2V_System_error_category@2@A@@YAXXZ 10003490 f   SeqBootAdapter.obj
 0001:000024a0       ??__EalgoLog@U2@@YAXXZ     100034a0 f   SeqBootAdapter.obj
 0001:00002520       ??__EcmdLog@U2@@YAXXZ      10003520 f   SeqBootAdapter.obj
 0001:000025a0       ??__EcoreLog@U2@@YAXXZ     100035a0 f   SeqBootAdapter.obj
 0001:00002620       ??__EioLog@U2@@YAXXZ       10003620 f   SeqBootAdapter.obj
 0001:000026a0       ??__EperfLog@U2@@YAXXZ     100036a0 f   SeqBootAdapter.obj
 0001:00002720       ??__EscriptLog@U2@@YAXXZ   10003720 f   SeqBootAdapter.obj
 0001:000027a0       ??__EtaskLog@U2@@YAXXZ     100037a0 f   SeqBootAdapter.obj
 0001:00002820       ??__EuiLog@U2@@YAXXZ       10003820 f   SeqBootAdapter.obj
 0001:000028a0       ??__EuserActLog@U2@@YAXXZ  100038a0 f   SeqBootAdapter.obj
 0001:00002920       ??__E?_Generic_object@?$_Error_objects@H@std@@2V_Generic_error_category@2@A@@YAXXZ 10003920 f   dist.obj
 0001:00002930       ??__E?_Iostream_object@?$_Error_objects@H@std@@2V_Iostream_error_category@2@A@@YAXXZ 10003930 f   dist.obj
 0001:00002940       ??__E?_System_object@?$_Error_objects@H@std@@2V_System_error_category@2@A@@YAXXZ 10003940 f   dist.obj
 0001:00002950       ??__EalgoLog@U2@@YAXXZ     10003950 f   dist.obj
 0001:000029d0       ??__EcmdLog@U2@@YAXXZ      100039d0 f   dist.obj
 0001:00002a50       ??__EcoreLog@U2@@YAXXZ     10003a50 f   dist.obj
 0001:00002ad0       ??__EioLog@U2@@YAXXZ       10003ad0 f   dist.obj
 0001:00002b50       ??__EperfLog@U2@@YAXXZ     10003b50 f   dist.obj
 0001:00002bd0       ??__EscriptLog@U2@@YAXXZ   10003bd0 f   dist.obj
 0001:00002c50       ??__EtaskLog@U2@@YAXXZ     10003c50 f   dist.obj
 0001:00002cd0       ??__EuiLog@U2@@YAXXZ       10003cd0 f   dist.obj
 0001:00002d50       ??__EuserActLog@U2@@YAXXZ  10003d50 f   dist.obj
 0001:00002dd0       ??__E?F84@DNADistModelTypes@@2VQString@@A@@YAXXZ 10003dd0 f   dnadist.obj
 0001:00002df0       ??__E?JukesCantor@DNADistModelTypes@@2VQString@@A@@YAXXZ 10003df0 f   dnadist.obj
 0001:00002e10       ??__E?Kimura@DNADistModelTypes@@2VQString@@A@@YAXXZ 10003e10 f   dnadist.obj
 0001:00002e30       ??__E?LogDet@DNADistModelTypes@@2VQString@@A@@YAXXZ 10003e30 f   dnadist.obj
 0001:00002e50       ??__E?_Generic_object@?$_Error_objects@H@std@@2V_Generic_error_category@2@A@@YAXXZ 10003e50 f   dnadist.obj
 0001:00002e60       ??__E?_Iostream_object@?$_Error_objects@H@std@@2V_Iostream_error_category@2@A@@YAXXZ 10003e60 f   dnadist.obj
 0001:00002e70       ??__E?_System_object@?$_Error_objects@H@std@@2V_System_error_category@2@A@@YAXXZ 10003e70 f   dnadist.obj
 0001:00002e80       ??__EalgoLog@U2@@YAXXZ     10003e80 f   dnadist.obj
 0001:00002f00       ??__EcmdLog@U2@@YAXXZ      10003f00 f   dnadist.obj
 0001:00002f80       ??__EcoreLog@U2@@YAXXZ     10003f80 f   dnadist.obj
 0001:00003000       ??__EdnaDistSettings@@YAXXZ 10004000 f   dnadist.obj
 0001:00003020       ??__EioLog@U2@@YAXXZ       10004020 f   dnadist.obj
 0001:000030a0       ??__EperfLog@U2@@YAXXZ     100040a0 f   dnadist.obj
 0001:00003120       ??__EscriptLog@U2@@YAXXZ   10004120 f   dnadist.obj
 0001:000031a0       ??__EtaskLog@U2@@YAXXZ     100041a0 f   dnadist.obj
 0001:00003220       ??__EuiLog@U2@@YAXXZ       10004220 f   dnadist.obj
 0001:000032a0       ??__EuserActLog@U2@@YAXXZ  100042a0 f   dnadist.obj
 0001:00003320       ??__E?_Generic_object@?$_Error_objects@H@std@@2V_Generic_error_category@2@A@@YAXXZ 10004320 f   neighbor.obj
 0001:00003330       ??__E?_Iostream_object@?$_Error_objects@H@std@@2V_Iostream_error_category@2@A@@YAXXZ 10004330 f   neighbor.obj
 0001:00003340       ??__E?_System_object@?$_Error_objects@H@std@@2V_System_error_category@2@A@@YAXXZ 10004340 f   neighbor.obj
 0001:00003350       ??__EalgoLog@U2@@YAXXZ     10004350 f   neighbor.obj
 0001:000033d0       ??__EcmdLog@U2@@YAXXZ      100043d0 f   neighbor.obj
 0001:00003450       ??__EcoreLog@U2@@YAXXZ     10004450 f   neighbor.obj
 0001:000034d0       ??__EioLog@U2@@YAXXZ       100044d0 f   neighbor.obj
 0001:00003550       ??__EperfLog@U2@@YAXXZ     10004550 f   neighbor.obj
 0001:000035d0       ??__EscriptLog@U2@@YAXXZ   100045d0 f   neighbor.obj
 0001:00003650       ??__EtaskLog@U2@@YAXXZ     10004650 f   neighbor.obj
 0001:000036d0       ??__EuiLog@U2@@YAXXZ       100046d0 f   neighbor.obj
 0001:00003750       ??__EuserActLog@U2@@YAXXZ  10004750 f   neighbor.obj
 0001:000037d0       ??__E?_Generic_object@?$_Error_objects@H@std@@2V_Generic_error_category@2@A@@YAXXZ 100047d0 f   phylip.obj
 0001:000037e0       ??__E?_Iostream_object@?$_Error_objects@H@std@@2V_Iostream_error_category@2@A@@YAXXZ 100047e0 f   phylip.obj
 0001:000037f0       ??__E?_System_object@?$_Error_objects@H@std@@2V_System_error_category@2@A@@YAXXZ 100047f0 f   phylip.obj
 0001:00003800       ??__EalgoLog@U2@@YAXXZ     10004800 f   phylip.obj
 0001:00003880       ??__EcmdLog@U2@@YAXXZ      10004880 f   phylip.obj
 0001:00003900       ??__EcoreLog@U2@@YAXXZ     10004900 f   phylip.obj
 0001:00003980       ??__EioLog@U2@@YAXXZ       10004980 f   phylip.obj
 0001:00003a00       ??__EperfLog@U2@@YAXXZ     10004a00 f   phylip.obj
 0001:00003a80       ??__EscriptLog@U2@@YAXXZ   10004a80 f   phylip.obj
 0001:00003b00       ??__EtaskLog@U2@@YAXXZ     10004b00 f   phylip.obj
 0001:00003b80       ??__EuiLog@U2@@YAXXZ       10004b80 f   phylip.obj
 0001:00003c00       ??__EuserActLog@U2@@YAXXZ  10004c00 f   phylip.obj
 0001:00003c80       ??__E?JTT@ProtDistModelTypes@@2VQString@@A@@YAXXZ 10004c80 f   protdist.obj
 0001:00003ca0       ??__E?Kimura@ProtDistModelTypes@@2VQString@@A@@YAXXZ 10004ca0 f   protdist.obj
 0001:00003cc0       ??__E?PAM@ProtDistModelTypes@@2VQString@@A@@YAXXZ 10004cc0 f   protdist.obj
 0001:00003ce0       ??__E?PMB@ProtDistModelTypes@@2VQString@@A@@YAXXZ 10004ce0 f   protdist.obj
 0001:00003d00       ??__E?_Generic_object@?$_Error_objects@H@std@@2V_Generic_error_category@2@A@@YAXXZ 10004d00 f   protdist.obj
 0001:00003d10       ??__E?_Iostream_object@?$_Error_objects@H@std@@2V_Iostream_error_category@2@A@@YAXXZ 10004d10 f   protdist.obj
 0001:00003d20       ??__E?_System_object@?$_Error_objects@H@std@@2V_System_error_category@2@A@@YAXXZ 10004d20 f   protdist.obj
 0001:00003d30       ??__EalgoLog@U2@@YAXXZ     10004d30 f   protdist.obj
 0001:00003db0       ??__EcmdLog@U2@@YAXXZ      10004db0 f   protdist.obj
 0001:00003e30       ??__EcoreLog@U2@@YAXXZ     10004e30 f   protdist.obj
 0001:00003eb0       ??__EioLog@U2@@YAXXZ       10004eb0 f   protdist.obj
 0001:00003f30       ??__EperfLog@U2@@YAXXZ     10004f30 f   protdist.obj
 0001:00003fb0       ??__EscriptLog@U2@@YAXXZ   10004fb0 f   protdist.obj
 0001:00004030       ??__EtaskLog@U2@@YAXXZ     10005030 f   protdist.obj
 0001:000040b0       ??__EuiLog@U2@@YAXXZ       100050b0 f   protdist.obj
 0001:00004130       ??__EuserActLog@U2@@YAXXZ  10005130 f   protdist.obj
 0001:000041b0       ??__E?_Generic_object@?$_Error_objects@H@std@@2V_Generic_error_category@2@A@@YAXXZ 100051b0 f   seqboot.obj
 0001:000041c0       ??__E?_Iostream_object@?$_Error_objects@H@std@@2V_Iostream_error_category@2@A@@YAXXZ 100051c0 f   seqboot.obj
 0001:000041d0       ??__E?_System_object@?$_Error_objects@H@std@@2V_System_error_category@2@A@@YAXXZ 100051d0 f   seqboot.obj
 0001:000041e0       ??__EalgoLog@U2@@YAXXZ     100051e0 f   seqboot.obj
 0001:00004260       ??__EcmdLog@U2@@YAXXZ      10005260 f   seqboot.obj
 0001:000042e0       ??__EcoreLog@U2@@YAXXZ     100052e0 f   seqboot.obj
 0001:00004360       ??__EioLog@U2@@YAXXZ       10005360 f   seqboot.obj
 0001:000043e0       ??__EperfLog@U2@@YAXXZ     100053e0 f   seqboot.obj
 0001:00004460       ??__EscriptLog@U2@@YAXXZ   10005460 f   seqboot.obj
 0001:000044e0       ??__EtaskLog@U2@@YAXXZ     100054e0 f   seqboot.obj
 0001:00004560       ??__EuiLog@U2@@YAXXZ       10005560 f   seqboot.obj
 0001:000045e0       ??__EuserActLog@U2@@YAXXZ  100055e0 f   seqboot.obj
 0001:00004660       ??__E?_Generic_object@?$_Error_objects@H@std@@2V_Generic_error_category@2@A@@YAXXZ 10005660 f   moc_NeighborJoinWidget.obj
 0001:00004670       ??__E?_Iostream_object@?$_Error_objects@H@std@@2V_Iostream_error_category@2@A@@YAXXZ 10005670 f   moc_NeighborJoinWidget.obj
 0001:00004680       ??__E?_System_object@?$_Error_objects@H@std@@2V_System_error_category@2@A@@YAXXZ 10005680 f   moc_NeighborJoinWidget.obj
 0001:00004690       ??__E?staticMetaObject@NeighborJoinWidget@U2@@2UQMetaObject@@B@@YAXXZ 10005690 f   moc_NeighborJoinWidget.obj
 0001:000046a0       ??__EalgoLog@U2@@YAXXZ     100056a0 f   moc_NeighborJoinWidget.obj
 0001:00004720       ??__EcmdLog@U2@@YAXXZ      10005720 f   moc_NeighborJoinWidget.obj
 0001:000047a0       ??__EcoreLog@U2@@YAXXZ     100057a0 f   moc_NeighborJoinWidget.obj
 0001:00004820       ??__EioLog@U2@@YAXXZ       10005820 f   moc_NeighborJoinWidget.obj
 0001:000048a0       ??__EperfLog@U2@@YAXXZ     100058a0 f   moc_NeighborJoinWidget.obj
 0001:00004920       ??__EscriptLog@U2@@YAXXZ   10005920 f   moc_NeighborJoinWidget.obj
 0001:000049a0       ??__EtaskLog@U2@@YAXXZ     100059a0 f   moc_NeighborJoinWidget.obj
 0001:00004a20       ??__EuiLog@U2@@YAXXZ       10005a20 f   moc_NeighborJoinWidget.obj
 0001:00004aa0       ??__EuserActLog@U2@@YAXXZ  10005aa0 f   moc_NeighborJoinWidget.obj
 0001:00004b20       ??__E?_Generic_object@?$_Error_objects@H@std@@2V_Generic_error_category@2@A@@YAXXZ 10005b20 f   moc_PhylipCmdlineTask.obj
 0001:00004b30       ??__E?_Iostream_object@?$_Error_objects@H@std@@2V_Iostream_error_category@2@A@@YAXXZ 10005b30 f   moc_PhylipCmdlineTask.obj
 0001:00004b40       ??__E?_System_object@?$_Error_objects@H@std@@2V_System_error_category@2@A@@YAXXZ 10005b40 f   moc_PhylipCmdlineTask.obj
 0001:00004b50       ??__E?staticMetaObject@PhylipCmdlineTask@U2@@2UQMetaObject@@B@@YAXXZ 10005b50 f   moc_PhylipCmdlineTask.obj
 0001:00004b60       ??__EalgoLog@U2@@YAXXZ     10005b60 f   moc_PhylipCmdlineTask.obj
 0001:00004be0       ??__EcmdLog@U2@@YAXXZ      10005be0 f   moc_PhylipCmdlineTask.obj
 0001:00004c60       ??__EcoreLog@U2@@YAXXZ     10005c60 f   moc_PhylipCmdlineTask.obj
 0001:00004ce0       ??__EioLog@U2@@YAXXZ       10005ce0 f   moc_PhylipCmdlineTask.obj
 0001:00004d60       ??__EperfLog@U2@@YAXXZ     10005d60 f   moc_PhylipCmdlineTask.obj
 0001:00004de0       ??__EscriptLog@U2@@YAXXZ   10005de0 f   moc_PhylipCmdlineTask.obj
 0001:00004e60       ??__EtaskLog@U2@@YAXXZ     10005e60 f   moc_PhylipCmdlineTask.obj
 0001:00004ee0       ??__EuiLog@U2@@YAXXZ       10005ee0 f   moc_PhylipCmdlineTask.obj
 0001:00004f60       ??__EuserActLog@U2@@YAXXZ  10005f60 f   moc_PhylipCmdlineTask.obj
 0001:00004fe0       ??__E?_Generic_object@?$_Error_objects@H@std@@2V_Generic_error_category@2@A@@YAXXZ 10005fe0 f   moc_PhylipPlugin.obj
 0001:00004ff0       ??__E?_Iostream_object@?$_Error_objects@H@std@@2V_Iostream_error_category@2@A@@YAXXZ 10005ff0 f   moc_PhylipPlugin.obj
 0001:00005000       ??__E?_System_object@?$_Error_objects@H@std@@2V_System_error_category@2@A@@YAXXZ 10006000 f   moc_PhylipPlugin.obj
 0001:00005010       ??__E?staticMetaObject@PhylipPlugin@U2@@2UQMetaObject@@B@@YAXXZ 10006010 f   moc_PhylipPlugin.obj
 0001:00005020       ??__EService_DNAExport@U2@@YAXXZ 10006020 f   moc_PhylipPlugin.obj
 0001:00005030       ??__EService_DNAGraphPack@U2@@YAXXZ 10006030 f   moc_PhylipPlugin.obj
 0001:00005040       ??__EService_ExternalToolSupport@U2@@YAXXZ 10006040 f   moc_PhylipPlugin.obj
 0001:00005050       ??__EService_GUITesting@U2@@YAXXZ 10006050 f   moc_PhylipPlugin.obj
 0001:00005060       ??__EService_MaxCoreServiceId@U2@@YAXXZ 10006060 f   moc_PhylipPlugin.obj
 0001:00005070       ??__EService_MinCoreServiceId@U2@@YAXXZ 10006070 f   moc_PhylipPlugin.obj
 0001:00005080       ??__EService_PluginViewer@U2@@YAXXZ 10006080 f   moc_PhylipPlugin.obj
 0001:00005090       ??__EService_Project@U2@@YAXXZ 10006090 f   moc_PhylipPlugin.obj
 0001:000050a0       ??__EService_ProjectView@U2@@YAXXZ 100060a0 f   moc_PhylipPlugin.obj
 0001:000050b0       ??__EService_QueryDesigner@U2@@YAXXZ 100060b0 f   moc_PhylipPlugin.obj
 0001:000050c0       ??__EService_ScriptRegistry@U2@@YAXXZ 100060c0 f   moc_PhylipPlugin.obj
 0001:000050d0       ??__EService_TestRunner@U2@@YAXXZ 100060d0 f   moc_PhylipPlugin.obj
 0001:000050e0       ??__EService_WorkflowDesigner@U2@@YAXXZ 100060e0 f   moc_PhylipPlugin.obj
 0001:000050f0       ??__E?_Generic_object@?$_Error_objects@H@std@@2V_Generic_error_category@2@A@@YAXXZ 100060f0 f   moc_PhylipPluginTests.obj
 0001:00005100       ??__E?_Iostream_object@?$_Error_objects@H@std@@2V_Iostream_error_category@2@A@@YAXXZ 10006100 f   moc_PhylipPluginTests.obj
 0001:00005110       ??__E?_System_object@?$_Error_objects@H@std@@2V_System_error_category@2@A@@YAXXZ 10006110 f   moc_PhylipPluginTests.obj
 0001:00005120       ??__E?staticMetaObject@GTest_NeighborJoin@U2@@2UQMetaObject@@B@@YAXXZ 10006120 f   moc_PhylipPluginTests.obj
 0001:00005130       ??__EalgoLog@U2@@YAXXZ     10006130 f   moc_PhylipPluginTests.obj
 0001:000051b0       ??__EcmdLog@U2@@YAXXZ      100061b0 f   moc_PhylipPluginTests.obj
 0001:00005230       ??__EcoreLog@U2@@YAXXZ     10006230 f   moc_PhylipPluginTests.obj
 0001:000052b0       ??__EioLog@U2@@YAXXZ       100062b0 f   moc_PhylipPluginTests.obj
 0001:00005330       ??__EperfLog@U2@@YAXXZ     10006330 f   moc_PhylipPluginTests.obj
 0001:000053b0       ??__EscriptLog@U2@@YAXXZ   100063b0 f   moc_PhylipPluginTests.obj
 0001:00005430       ??__EtaskLog@U2@@YAXXZ     10006430 f   moc_PhylipPluginTests.obj
 0001:000054b0       ??__EuiLog@U2@@YAXXZ       100064b0 f   moc_PhylipPluginTests.obj
 0001:00005530       ??__EuserActLog@U2@@YAXXZ  10006530 f   moc_PhylipPluginTests.obj
 0001:000055b0       ??__E?_Generic_object@?$_Error_objects@H@std@@2V_Generic_error_category@2@A@@YAXXZ 100065b0 f   moc_PhylipTask.obj
 0001:000055c0       ??__E?_Iostream_object@?$_Error_objects@H@std@@2V_Iostream_error_category@2@A@@YAXXZ 100065c0 f   moc_PhylipTask.obj
 0001:000055d0       ??__E?_System_object@?$_Error_objects@H@std@@2V_System_error_category@2@A@@YAXXZ 100065d0 f   moc_PhylipTask.obj
 0001:000055e0       ??__E?staticMetaObject@PhylipTask@U2@@2UQMetaObject@@B@@YAXXZ 100065e0 f   moc_PhylipTask.obj
 0001:000055f0       ??__EalgoLog@U2@@YAXXZ     100065f0 f   moc_PhylipTask.obj
 0001:00005670       ??__EcmdLog@U2@@YAXXZ      10006670 f   moc_PhylipTask.obj
 0001:000056f0       ??__EcoreLog@U2@@YAXXZ     100066f0 f   moc_PhylipTask.obj
 0001:00005770       ??__EioLog@U2@@YAXXZ       10006770 f   moc_PhylipTask.obj
 0001:000057f0       ??__EperfLog@U2@@YAXXZ     100067f0 f   moc_PhylipTask.obj
 0001:00005870       ??__EscriptLog@U2@@YAXXZ   10006870 f   moc_PhylipTask.obj
 0001:000058f0       ??__EtaskLog@U2@@YAXXZ     100068f0 f   moc_PhylipTask.obj
 0001:00005970       ??__EuiLog@U2@@YAXXZ       10006970 f   moc_PhylipTask.obj
 0001:000059f0       ??__EuserActLog@U2@@YAXXZ  100069f0 f   moc_PhylipTask.obj
 0001:00005c22       __catch$??$?6U?$char_traits@D@std@@@std@@YAAAV?$basic_ostream@DU?$char_traits@D@std@@@0@AAV10@PBD@Z$0 10006c22 f i DistanceMatrix.obj
 0001:0000608e       __catch$??0?$QList@VMultipleSequenceAlignmentRow@U2@@@@QAE@ABV0@@Z$0 1000708e f i DistanceMatrix.obj
 0001:00007576       __catch$?_Copy@?$basic_string@DU?$char_traits@D@std@@V?$allocator@D@2@@std@@QAEXII@Z$0 10008576 f i DistanceMatrix.obj
 0001:000075b3       __catch$?_Copy@?$basic_string@DU?$char_traits@D@std@@V?$allocator@D@2@@std@@QAEXII@Z$1 100085b3 f i DistanceMatrix.obj
 0001:00008b35       __catch$?append@?$QList@PAVPhyBranch@U2@@@@QAEXABQAVPhyBranch@U2@@@Z$4 10009b35 f i DistanceMatrix.obj
 0001:00008bc5       __catch$?append@?$QList@PAVPhyNode@U2@@@@QAEXABQAVPhyNode@U2@@@Z$4 10009bc5 f i DistanceMatrix.obj
 0001:00008c4d       __catch$?append@?$QList@VQString@@@@QAEXABVQString@@@Z$0 10009c4d f i DistanceMatrix.obj
 0001:00008c9e       __catch$?append@?$QList@VQString@@@@QAEXABVQString@@@Z$4 10009c9e f i DistanceMatrix.obj
 0001:00009f6d       __catch$?calculateOutOfAlignment@DistanceMatrix@U2@@QAEXABVMultipleSequenceAlignment@2@ABVCreatePhyTreeSettings@2@@Z$0 1000af6d f   DistanceMatrix.obj
 0001:0000a034       $LN514                     1000b034     DistanceMatrix.obj
 0001:0000a0a0       $LN483                     1000b0a0     DistanceMatrix.obj
 0001:0000ada5       __catch$?createNode@?$QMapData@VQString@@H@@QAEPAU?$QMapNode@VQString@@H@@ABVQString@@ABHPAU2@_N@Z$2 1000bda5 f i DistanceMatrix.obj
 0001:0000b39c       __catch$?detach_helper@?$QList@PAVPhyNode@U2@@@@AAEXH@Z$0 1000c39c f i DistanceMatrix.obj
 0001:0000b4a1       __catch$?detach_helper@?$QList@VQString@@@@AAEXH@Z$0 1000c4a1 f i DistanceMatrix.obj
 0001:0000b711       __catch$?detach_helper_grow@?$QList@PAVPhyBranch@U2@@@@AAEPAUNode@1@HH@Z$0 1000c711 f i DistanceMatrix.obj
 0001:0000b711       __catch$?detach_helper_grow@?$QList@PAVPhyBranch@U2@@@@AAEPAUNode@1@HH@Z$2 1000c711 f i DistanceMatrix.obj
 0001:0000b821       __catch$?detach_helper_grow@?$QList@PAVPhyNode@U2@@@@AAEPAUNode@1@HH@Z$2 1000c821 f i DistanceMatrix.obj
 0001:0000b821       __catch$?detach_helper_grow@?$QList@PAVPhyNode@U2@@@@AAEPAUNode@1@HH@Z$0 1000c821 f i DistanceMatrix.obj
 0001:0000b95e       __catch$?detach_helper_grow@?$QList@VQString@@@@AAEPAUNode@1@HH@Z$2 1000c95e f i DistanceMatrix.obj
 0001:0000b999       __catch$?detach_helper_grow@?$QList@VQString@@@@AAEPAUNode@1@HH@Z$0 1000c999 f i DistanceMatrix.obj
 0001:0000cdc5       __catch$?node_copy@?$QList@VMultipleSequenceAlignmentRow@U2@@@@AAEXPAUNode@1@00@Z$0 1000ddc5 f i DistanceMatrix.obj
 0001:0000ce72       __catch$?node_copy@?$QList@VQString@@@@AAEXPAUNode@1@00@Z$2 1000de72 f i DistanceMatrix.obj
 0001:0000d424       __catch$?reallocData@?$QVector@M@@AAEXHHV?$QFlags@W4AllocationOption@QArrayData@@@@@Z$0 1000e424 f i DistanceMatrix.obj
 0001:0000d436       __catch$?reallocData@?$QVector@M@@AAEXHHV?$QFlags@W4AllocationOption@QArrayData@@@@@Z$2 1000e436 f i DistanceMatrix.obj
 0001:0000d6e4       __catch$?reallocData@?$QVector@V?$QVector@M@@@@AAEXHHV?$QFlags@W4AllocationOption@QArrayData@@@@@Z$0 1000e6e4 f i DistanceMatrix.obj
 0001:0000d702       __catch$?reallocData@?$QVector@V?$QVector@M@@@@AAEXHHV?$QFlags@W4AllocationOption@QArrayData@@@@@Z$2 1000e702 f i DistanceMatrix.obj
 0001:0000f8df       __catch$?run@NeighborJoinCalculateTreeTask@U2@@UAEXXZ$0 100108df f   NeighborJoinAdapter.obj
 0001:0000fa11       __catch$?run@NeighborJoinCalculateTreeTask@U2@@UAEXXZ$1 10010a11 f   NeighborJoinAdapter.obj
 0001:0000fbbe       __catch$??0?$QList@VQString@@@@QAE@ABV0@@Z$0 10010bbe f i NeighborJoinWidget.obj
 0001:0000fda0       ??R<lambda_0653c3664f4171908e49d192859671f4>@@QBE?AVQString@@XZ 10010da0 f   NeighborJoinWidget.obj
 0001:0000fdc0       ??R<lambda_0b0380af5bb2f62da28634d4824ec8ca>@@QBE?AVQString@@XZ 10010dc0 f   NeighborJoinWidget.obj
 0001:0000fde0       ??R<lambda_0b8b5ce51c46f86678041328dcb0fb05>@@QBE?AVQString@@XZ 10010de0 f   NeighborJoinWidget.obj
 0001:0000fe00       ??R<lambda_0d22fed94f2a311d9dfca95916641178>@@QBE?AVQString@@XZ 10010e00 f   NeighborJoinWidget.obj
 0001:0000fe20       ??R<lambda_14e59930e730d4459c38a093acf4d195>@@QBE?AVQString@@XZ 10010e20 f   NeighborJoinWidget.obj
 0001:0000fe40       ??R<lambda_23a54e0ab73de2509c6e5cc465bd53c9>@@QBE?AVQString@@XZ 10010e40 f   NeighborJoinWidget.obj
 0001:0000fe60       ??R<lambda_2b27d5241a7fc153d4a2a4123de53aa9>@@QBE?AVQString@@XZ 10010e60 f   NeighborJoinWidget.obj
 0001:0000fe80       ??R<lambda_2b4fc15a8fdb2e804f00ceb3bda53a64>@@QBE?AVQString@@XZ 10010e80 f   NeighborJoinWidget.obj
 0001:0000fea0       ??R<lambda_33b9794a776f12fce937feb1d38745b7>@@QBE?AVQString@@XZ 10010ea0 f   NeighborJoinWidget.obj
 0001:0000fec0       ??R<lambda_44ada46bd4b31fea57024b3ee705fbb5>@@QBE?AVQString@@XZ 10010ec0 f   NeighborJoinWidget.obj
 0001:0000fee0       ??R<lambda_47aba4f81f0235f8ea25dd5385c10da9>@@QBE?AVQString@@XZ 10010ee0 f   NeighborJoinWidget.obj
 0001:0000ff00       ??R<lambda_48eb925e0df25a63beef6f774f70e0ce>@@QBE?AVQString@@XZ 10010f00 f   NeighborJoinWidget.obj
 0001:0000ff20       ??R<lambda_4e2ee4c24f9f6f06c9235a84091eec77>@@QBE?AVQString@@XZ 10010f20 f   NeighborJoinWidget.obj
 0001:0000ff40       ??R<lambda_58398813fcf17172efc5c67a807eff6c>@@QBE?AVQString@@XZ 10010f40 f   NeighborJoinWidget.obj
 0001:0000ff60       ??R<lambda_5b8be46bdab4df2be815ada5e31bbf2e>@@QBE?AVQString@@XZ 10010f60 f   NeighborJoinWidget.obj
 0001:0000ff80       ??R<lambda_5cb97931b222ba4845c1a6793eb20d02>@@QBE?AVQString@@XZ 10010f80 f   NeighborJoinWidget.obj
 0001:0000ffa0       ??R<lambda_69ac5ad72d4d5a21717e1b3cd28fabc3>@@QBE?AVQString@@XZ 10010fa0 f   NeighborJoinWidget.obj
 0001:0000ffc0       ??R<lambda_7fcb402e3d4ced9f2dada59451304bad>@@QBE?AVQString@@XZ 10010fc0 f   NeighborJoinWidget.obj
 0001:0000ffe0       ??R<lambda_89c462f96a9772122e80910435b04d7b>@@QBE?AVQString@@XZ 10010fe0 f   NeighborJoinWidget.obj
 0001:00010000       ??R<lambda_8f99dcda7ee44bb3b2c68c37b2d63d09>@@QBE?AVQString@@XZ 10011000 f   NeighborJoinWidget.obj
 0001:00010020       ??R<lambda_992082ea6d03cf2b362a601e532562f9>@@QBE?AVQString@@XZ 10011020 f   NeighborJoinWidget.obj
 0001:00010040       ??R<lambda_9bdb903db70d78592dfa82f916e59082>@@QBE?AVQString@@XZ 10011040 f   NeighborJoinWidget.obj
 0001:00010060       ??R<lambda_9d41da171c8d767f232c43981809cb07>@@QBE?AVQString@@XZ 10011060 f   NeighborJoinWidget.obj
 0001:00010080       ??R<lambda_a240313f06a8e1d5b6e359782d131016>@@QBE?AVQString@@XZ 10011080 f   NeighborJoinWidget.obj
 0001:000100a0       ??R<lambda_a9c426da71b6bbdf1080a86813f9c2db>@@QBE?AVQString@@XZ 100110a0 f   NeighborJoinWidget.obj
 0001:000100c0       ??R<lambda_ba1cc78051bce41bc52e64c17a9c21ff>@@QBE?AVQString@@XZ 100110c0 f   NeighborJoinWidget.obj
 0001:000100e0       ??R<lambda_c5fe69c308d98b88bf0bdcb153255297>@@QBE?AVQString@@XZ 100110e0 f   NeighborJoinWidget.obj
 0001:00010100       ??R<lambda_d22a08e1c31cb8eed59da0c6f8cb4643>@@QBE?AVQString@@XZ 10011100 f   NeighborJoinWidget.obj
 0001:00010120       ??R<lambda_d5b1e7fac3396eb92e6a12b8811845a8>@@QBE?AVQString@@XZ 10011120 f   NeighborJoinWidget.obj
 0001:00010140       ??R<lambda_e1d814167b8d6739a6636789b1b459d2>@@QBE?AVQString@@XZ 10011140 f   NeighborJoinWidget.obj
 0001:00010160       ??R<lambda_e3a39c3ab834799cdee3657bb2fb9ff0>@@QBE?AVQString@@XZ 10011160 f   NeighborJoinWidget.obj
 0001:00010180       ??R<lambda_e4294879436371d98917fc7c6809dc4b>@@QBE?AVQString@@XZ 10011180 f   NeighborJoinWidget.obj
 0001:000101a0       ??R<lambda_e79d5e48dce79ac397e8108a5da31d66>@@QBE?AVQString@@XZ 100111a0 f   NeighborJoinWidget.obj
 0001:000101c0       ??R<lambda_ed8afe383a046c77d89e6b408a9bbda5>@@QBE?AVQString@@XZ 100111c0 f   NeighborJoinWidget.obj
 0001:000101e0       ??R<lambda_fe34ae2a9f494fb27c4b6c32f78f7d34>@@QBE?AVQString@@XZ 100111e0 f   NeighborJoinWidget.obj
 0001:0001361e       __catch$??0?$QList@VQByteArray@@@@QAE@ABV0@@Z$0 1001461e f i PhylipCmdlineTask.obj
 0001:00013d95       __catch$?append@?$QList@PAVGObject@U2@@@@QAEXABQAVGObject@U2@@@Z$4 10014d95 f i PhylipCmdlineTask.obj
 0001:00014741       __catch$?detach_helper@?$QList@VQByteArray@@@@AAEXH@Z$0 10015741 f i PhylipCmdlineTask.obj
 0001:00014861       __catch$?detach_helper_grow@?$QList@PAVGObject@U2@@@@AAEPAUNode@1@HH@Z$2 10015861 f i PhylipCmdlineTask.obj
 0001:00014861       __catch$?detach_helper_grow@?$QList@PAVGObject@U2@@@@AAEPAUNode@1@HH@Z$0 10015861 f i PhylipCmdlineTask.obj
 0001:00014ab2       __catch$?node_copy@?$QList@VQByteArray@@@@AAEXPAUNode@1@00@Z$2 10015ab2 f i PhylipCmdlineTask.obj
 0001:0001518e       __catch$??0?$QList@PAVXMLTestFactory@U2@@@@QAE@ABV0@@Z$0 1001618e f i PhylipPlugin.obj
 0001:00016245       __catch$?append@?$QList@PAVXMLTestFactory@U2@@@@QAEXABQAVXMLTestFactory@U2@@@Z$4 10017245 f i PhylipPluginTests.obj
 0001:0001652c       __catch$?detach_helper@?$QList@PAVGObject@U2@@@@AAEXH@Z$0 1001752c f i PhylipPluginTests.obj
 0001:00016651       __catch$?detach_helper_grow@?$QList@PAVXMLTestFactory@U2@@@@AAEPAUNode@1@HH@Z$0 10017651 f i PhylipPluginTests.obj
 0001:00016651       __catch$?detach_helper_grow@?$QList@PAVXMLTestFactory@U2@@@@AAEPAUNode@1@HH@Z$2 10017651 f i PhylipPluginTests.obj
 0001:0001859d       __catch$?reallocData@?$QVector@VMultipleSequenceAlignment@U2@@@@AAEXHHV?$QFlags@W4AllocationOption@QArrayData@@@@@Z$0 1001959d f i SeqBootAdapter.obj
 0001:000185bb       __catch$?reallocData@?$QVector@VMultipleSequenceAlignment@U2@@@@AAEXHHV?$QFlags@W4AllocationOption@QArrayData@@@@@Z$2 100195bb f i SeqBootAdapter.obj
 0001:0001a734       $LN46                      1001b734     cons.obj
 0001:0001dde0       $LN168                     1001ede0     dnadist.obj
 0001:0001de20       $LN164                     1001ee20     dnadist.obj
 0001:00022fe0       ?crash_handler@@YAXH@Z     10023fe0 f   phylip.obj
 0001:00025f2c       $LN29                      10026f2c     phylip.obj
 0001:0002b284       $LN187                     1002c284     protdist.obj
 0001:0002b2f0       $LN174                     1002c2f0     protdist.obj
 0001:0002b324       $LN188                     1002c324     protdist.obj
 0001:00030aa4       $LN159                     10031aa4     seq.obj
 0001:00030ae4       $LN156                     10031ae4     seq.obj
 0001:00030c94       $LN62                      10031c94     seq.obj
 0001:00030cdc       $LN60                      10031cdc     seq.obj
 0001:00039ba0       $$000000                   1003aba0     MSVCRT:lldiv.obj
 0001:00039cb0       $$000000                   1003acb0     MSVCRT:llmul.obj
 0001:0003a2a0       $$000000                   1003b2a0     MSVCRT:ftol3.obj
 0001:0003a66d       _pre_c_init                1003b66d f   MSVCRT:crtdll.obj
 0001:0003a8da       ___DllMainCRTStartup       1003b8da f   MSVCRT:crtdll.obj
 0001:0003aa30       $$000000                   1003ba30     MSVCRT:sehprolg4.obj
 0001:0003ab1b       ?ArrayUnwindFilter@@YAHPAU_EXCEPTION_POINTERS@@@Z 1003bb1b f   MSVCRT:ehvecdtr.obj
 0001:0003ae70       __unwindfunclet$??$?6U?$char_traits@D@std@@@std@@YAAAV?$basic_ostream@DU?$char_traits@D@std@@@0@AAV10@PBD@Z$3 1003be70 f   DistanceMatrix.obj
 0001:0003ae78       __unwindfunclet$??$?6U?$char_traits@D@std@@@std@@YAAAV?$basic_ostream@DU?$char_traits@D@std@@@0@AAV10@PBD@Z$2 1003be78 f   DistanceMatrix.obj
 0001:0003ae80       __ehhandler$??$?6U?$char_traits@D@std@@@std@@YAAAV?$basic_ostream@DU?$char_traits@D@std@@@0@AAV10@PBD@Z 1003be80 f   DistanceMatrix.obj
 0001:0003aea0       __ehhandler$??0?$QList@VMultipleSequenceAlignmentRow@U2@@@@QAE@ABV0@@Z 1003bea0 f   DistanceMatrix.obj
 0001:0003aec0       __unwindfunclet$??0DistanceMatrix@U2@@QAE@XZ$0 1003bec0 f   DistanceMatrix.obj
 0001:0003aecb       __unwindfunclet$??0DistanceMatrix@U2@@QAE@XZ$1 1003becb f   DistanceMatrix.obj
 0001:0003aed6       __unwindfunclet$??0DistanceMatrix@U2@@QAE@XZ$2 1003bed6 f   DistanceMatrix.obj
 0001:0003aee1       __unwindfunclet$??0DistanceMatrix@U2@@QAE@XZ$3 1003bee1 f   DistanceMatrix.obj
 0001:0003aeec       __unwindfunclet$??0DistanceMatrix@U2@@QAE@XZ$4 1003beec f   DistanceMatrix.obj
 0001:0003aef7       __unwindfunclet$??0DistanceMatrix@U2@@QAE@XZ$5 1003bef7 f   DistanceMatrix.obj
 0001:0003af02       __unwindfunclet$??0DistanceMatrix@U2@@QAE@XZ$6 1003bf02 f   DistanceMatrix.obj
 0001:0003af0e       __unwindfunclet$??0DistanceMatrix@U2@@QAE@XZ$7 1003bf0e f   DistanceMatrix.obj
 0001:0003af19       __unwindfunclet$??0DistanceMatrix@U2@@QAE@XZ$9 1003bf19 f   DistanceMatrix.obj
 0001:0003af25       __ehhandler$??0DistanceMatrix@U2@@QAE@XZ 1003bf25 f   DistanceMatrix.obj
 0001:0003af40       __unwindfunclet$??0MemoryLocker@U2@@QAE@HW4MemoryLockType@AppResource@1@@Z$0 1003bf40 f   DistanceMatrix.obj
 0001:0003af4c       __ehhandler$??0MemoryLocker@U2@@QAE@HW4MemoryLockType@AppResource@1@@Z 1003bf4c f   DistanceMatrix.obj
 0001:0003af70       __unwindfunclet$??0sentry@?$basic_ostream@DU?$char_traits@D@std@@@std@@QAE@AAV12@@Z$0 1003bf70 f   DistanceMatrix.obj
 0001:0003af78       __ehhandler$??0sentry@?$basic_ostream@DU?$char_traits@D@std@@@std@@QAE@AAV12@@Z 1003bf78 f   DistanceMatrix.obj
 0001:0003afa0       __unwindfunclet$??1DistanceMatrix@U2@@QAE@XZ$0 1003bfa0 f   DistanceMatrix.obj
 0001:0003afab       __unwindfunclet$??1DistanceMatrix@U2@@QAE@XZ$1 1003bfab f   DistanceMatrix.obj
 0001:0003afb6       __unwindfunclet$??1DistanceMatrix@U2@@QAE@XZ$2 1003bfb6 f   DistanceMatrix.obj
 0001:0003afc1       __unwindfunclet$??1DistanceMatrix@U2@@QAE@XZ$3 1003bfc1 f   DistanceMatrix.obj
 0001:0003afcc       __unwindfunclet$??1DistanceMatrix@U2@@QAE@XZ$4 1003bfcc f   DistanceMatrix.obj
 0001:0003afd7       __unwindfunclet$??1DistanceMatrix@U2@@QAE@XZ$5 1003bfd7 f   DistanceMatrix.obj
 0001:0003afe2       __unwindfunclet$??1DistanceMatrix@U2@@QAE@XZ$6 1003bfe2 f   DistanceMatrix.obj
 0001:0003afee       __unwindfunclet$??1DistanceMatrix@U2@@QAE@XZ$7 1003bfee f   DistanceMatrix.obj
 0001:0003aff9       __unwindfunclet$??1DistanceMatrix@U2@@QAE@XZ$9 1003bff9 f   DistanceMatrix.obj
 0001:0003b005       __unwindfunclet$??1DistanceMatrix@U2@@QAE@XZ$10 1003c005 f   DistanceMatrix.obj
 0001:0003b00e       __ehhandler$??1DistanceMatrix@U2@@QAE@XZ 1003c00e f   DistanceMatrix.obj
 0001:0003b030       __unwindfunclet$??1MemoryLocker@U2@@UAE@XZ$0 1003c030 f   DistanceMatrix.obj
 0001:0003b03c       __ehhandler$??1MemoryLocker@U2@@UAE@XZ 1003c03c f   DistanceMatrix.obj
 0001:0003b060       __unwindfunclet$??_GMemoryLocker@U2@@UAEPAXI@Z$0 1003c060 f   DistanceMatrix.obj
 0001:0003b06c       __ehhandler$??_GMemoryLocker@U2@@UAEPAXI@Z 1003c06c f   DistanceMatrix.obj
 0001:0003b090       __unwindfunclet$??__EalgoLog@U2@@YAXXZ$0 1003c090 f   DistanceMatrix.obj
 0001:0003b099       __ehhandler$??__EalgoLog@U2@@YAXXZ 1003c099 f   DistanceMatrix.obj
 0001:0003b0c0       __unwindfunclet$??__EcmdLog@U2@@YAXXZ$0 1003c0c0 f   DistanceMatrix.obj
 0001:0003b0c9       __ehhandler$??__EcmdLog@U2@@YAXXZ 1003c0c9 f   DistanceMatrix.obj
 0001:0003b0f0       __unwindfunclet$??__EcoreLog@U2@@YAXXZ$0 1003c0f0 f   DistanceMatrix.obj
 0001:0003b0f9       __ehhandler$??__EcoreLog@U2@@YAXXZ 1003c0f9 f   DistanceMatrix.obj
 0001:0003b120       __unwindfunclet$??__EioLog@U2@@YAXXZ$0 1003c120 f   DistanceMatrix.obj
 0001:0003b129       __ehhandler$??__EioLog@U2@@YAXXZ 1003c129 f   DistanceMatrix.obj
 0001:0003b150       __unwindfunclet$??__EperfLog@U2@@YAXXZ$0 1003c150 f   DistanceMatrix.obj
 0001:0003b159       __ehhandler$??__EperfLog@U2@@YAXXZ 1003c159 f   DistanceMatrix.obj
 0001:0003b180       __unwindfunclet$??__EscriptLog@U2@@YAXXZ$0 1003c180 f   DistanceMatrix.obj
 0001:0003b189       __ehhandler$??__EscriptLog@U2@@YAXXZ 1003c189 f   DistanceMatrix.obj
 0001:0003b1b0       __unwindfunclet$??__EtaskLog@U2@@YAXXZ$0 1003c1b0 f   DistanceMatrix.obj
 0001:0003b1b9       __ehhandler$??__EtaskLog@U2@@YAXXZ 1003c1b9 f   DistanceMatrix.obj
 0001:0003b1e0       __unwindfunclet$??__EuiLog@U2@@YAXXZ$0 1003c1e0 f   DistanceMatrix.obj
 0001:0003b1e9       __ehhandler$??__EuiLog@U2@@YAXXZ 1003c1e9 f   DistanceMatrix.obj
 0001:0003b210       __unwindfunclet$??__EuserActLog@U2@@YAXXZ$0 1003c210 f   DistanceMatrix.obj
 0001:0003b219       __ehhandler$??__EuserActLog@U2@@YAXXZ 1003c219 f   DistanceMatrix.obj
 0001:0003b240       __ehhandler$?_Copy@?$basic_string@DU?$char_traits@D@std@@V?$allocator@D@2@@std@@QAEXII@Z 1003c240 f   DistanceMatrix.obj
 0001:0003b260       __unwindfunclet$?addNodeToList@DistanceMatrix@U2@@CAXAAV?$QList@PAVPhyNode@U2@@@@AAV?$QMap@VQString@@H@@AAV?$QList@PAVPhyBranch@U2@@@@PAVPhyNode@2@@Z$0 1003c260 f   DistanceMatrix.obj
 0001:0003b27a       __ehhandler$?addNodeToList@DistanceMatrix@U2@@CAXAAV?$QList@PAVPhyNode@U2@@@@AAV?$QMap@VQString@@H@@AAV?$QList@PAVPhyBranch@U2@@@@PAVPhyNode@2@@Z 1003c27a f   DistanceMatrix.obj
 0001:0003b2a0       __unwindfunclet$?addPairToTree@DistanceMatrix@U2@@AAEXPAU?$QPair@HH@@@Z$0 1003c2a0 f   DistanceMatrix.obj
 0001:0003b2a9       __unwindfunclet$?addPairToTree@DistanceMatrix@U2@@AAEXPAU?$QPair@HH@@@Z$15 1003c2a9 f   DistanceMatrix.obj
 0001:0003b2b2       __unwindfunclet$?addPairToTree@DistanceMatrix@U2@@AAEXPAU?$QPair@HH@@@Z$2 1003c2b2 f   DistanceMatrix.obj
 0001:0003b2bb       __unwindfunclet$?addPairToTree@DistanceMatrix@U2@@AAEXPAU?$QPair@HH@@@Z$18 1003c2bb f   DistanceMatrix.obj
 0001:0003b2c4       __unwindfunclet$?addPairToTree@DistanceMatrix@U2@@AAEXPAU?$QPair@HH@@@Z$4 1003c2c4 f   DistanceMatrix.obj
 0001:0003b2cf       __unwindfunclet$?addPairToTree@DistanceMatrix@U2@@AAEXPAU?$QPair@HH@@@Z$5 1003c2cf f   DistanceMatrix.obj
 0001:0003b2d8       __unwindfunclet$?addPairToTree@DistanceMatrix@U2@@AAEXPAU?$QPair@HH@@@Z$7 1003c2d8 f   DistanceMatrix.obj
 0001:0003b2e1       __unwindfunclet$?addPairToTree@DistanceMatrix@U2@@AAEXPAU?$QPair@HH@@@Z$8 1003c2e1 f   DistanceMatrix.obj
 0001:0003b2e9       __unwindfunclet$?addPairToTree@DistanceMatrix@U2@@AAEXPAU?$QPair@HH@@@Z$9 1003c2e9 f   DistanceMatrix.obj
 0001:0003b2f1       __unwindfunclet$?addPairToTree@DistanceMatrix@U2@@AAEXPAU?$QPair@HH@@@Z$10 1003c2f1 f   DistanceMatrix.obj
 0001:0003b2f9       __unwindfunclet$?addPairToTree@DistanceMatrix@U2@@AAEXPAU?$QPair@HH@@@Z$11 1003c2f9 f   DistanceMatrix.obj
 0001:0003b302       __unwindfunclet$?addPairToTree@DistanceMatrix@U2@@AAEXPAU?$QPair@HH@@@Z$22 1003c302 f   DistanceMatrix.obj
 0001:0003b30b       __unwindfunclet$?addPairToTree@DistanceMatrix@U2@@AAEXPAU?$QPair@HH@@@Z$13 1003c30b f   DistanceMatrix.obj
 0001:0003b314       __unwindfunclet$?addPairToTree@DistanceMatrix@U2@@AAEXPAU?$QPair@HH@@@Z$14 1003c314 f   DistanceMatrix.obj
 0001:0003b31c       __ehhandler$?addPairToTree@DistanceMatrix@U2@@AAEXPAU?$QPair@HH@@@Z 1003c31c f   DistanceMatrix.obj
 0001:0003b340       __ehhandler$?append@?$QList@PAVPhyBranch@U2@@@@QAEXABQAVPhyBranch@U2@@@Z 1003c340 f   DistanceMatrix.obj
 0001:0003b360       __ehhandler$?append@?$QList@PAVPhyNode@U2@@@@QAEXABQAVPhyNode@U2@@@Z 1003c360 f   DistanceMatrix.obj
 0001:0003b380       __unwindfunclet$?append@?$QList@VQString@@@@QAEXABVQString@@@Z$7 1003c380 f   DistanceMatrix.obj
 0001:0003b391       __unwindfunclet$?append@?$QList@VQString@@@@QAEXABVQString@@@Z$11 1003c391 f   DistanceMatrix.obj
 0001:0003b3a2       __ehhandler$?append@?$QList@VQString@@@@QAEXABVQString@@@Z 1003c3a2 f   DistanceMatrix.obj
 0001:0003b3c0       __unwindfunclet$?append@?$QVector@V?$QVector@M@@@@QAEXABV?$QVector@M@@@Z$0 1003c3c0 f   DistanceMatrix.obj
 0001:0003b3c8       __unwindfunclet$?append@?$QVector@V?$QVector@M@@@@QAEXABV?$QVector@M@@@Z$1 1003c3c8 f   DistanceMatrix.obj
 0001:0003b3d9       __ehhandler$?append@?$QVector@V?$QVector@M@@@@QAEXABV?$QVector@M@@@Z 1003c3d9 f   DistanceMatrix.obj
 0001:0003b400       __unwindfunclet$?areTreesEqual@DistanceMatrix@U2@@CA_NPAV?$QSharedDataPointer@VPhyTreeData@U2@@@@0@Z$0 1003c400 f   DistanceMatrix.obj
 0001:0003b408       __unwindfunclet$?areTreesEqual@DistanceMatrix@U2@@CA_NPAV?$QSharedDataPointer@VPhyTreeData@U2@@@@0@Z$1 1003c408 f   DistanceMatrix.obj
 0001:0003b410       __unwindfunclet$?areTreesEqual@DistanceMatrix@U2@@CA_NPAV?$QSharedDataPointer@VPhyTreeData@U2@@@@0@Z$2 1003c410 f   DistanceMatrix.obj
 0001:0003b418       __unwindfunclet$?areTreesEqual@DistanceMatrix@U2@@CA_NPAV?$QSharedDataPointer@VPhyTreeData@U2@@@@0@Z$3 1003c418 f   DistanceMatrix.obj
 0001:0003b420       __unwindfunclet$?areTreesEqual@DistanceMatrix@U2@@CA_NPAV?$QSharedDataPointer@VPhyTreeData@U2@@@@0@Z$4 1003c420 f   DistanceMatrix.obj
 0001:0003b428       __unwindfunclet$?areTreesEqual@DistanceMatrix@U2@@CA_NPAV?$QSharedDataPointer@VPhyTreeData@U2@@@@0@Z$5 1003c428 f   DistanceMatrix.obj
 0001:0003b430       __unwindfunclet$?areTreesEqual@DistanceMatrix@U2@@CA_NPAV?$QSharedDataPointer@VPhyTreeData@U2@@@@0@Z$6 1003c430 f   DistanceMatrix.obj
 0001:0003b438       __unwindfunclet$?areTreesEqual@DistanceMatrix@U2@@CA_NPAV?$QSharedDataPointer@VPhyTreeData@U2@@@@0@Z$7 1003c438 f   DistanceMatrix.obj
 0001:0003b441       __ehhandler$?areTreesEqual@DistanceMatrix@U2@@CA_NPAV?$QSharedDataPointer@VPhyTreeData@U2@@@@0@Z 1003c441 f   DistanceMatrix.obj
 0001:0003b460       __unwindfunclet$?calculateOutOfAlignment@DistanceMatrix@U2@@QAEXABVMultipleSequenceAlignment@2@ABVCreatePhyTreeSettings@2@@Z$2 1003c460 f   DistanceMatrix.obj
 0001:0003b468       __unwindfunclet$?calculateOutOfAlignment@DistanceMatrix@U2@@QAEXABVMultipleSequenceAlignment@2@ABVCreatePhyTreeSettings@2@@Z$3 1003c468 f   DistanceMatrix.obj
 0001:0003b470       __unwindfunclet$?calculateOutOfAlignment@DistanceMatrix@U2@@QAEXABVMultipleSequenceAlignment@2@ABVCreatePhyTreeSettings@2@@Z$4 1003c470 f   DistanceMatrix.obj
 0001:0003b479       __unwindfunclet$?calculateOutOfAlignment@DistanceMatrix@U2@@QAEXABVMultipleSequenceAlignment@2@ABVCreatePhyTreeSettings@2@@Z$5 1003c479 f   DistanceMatrix.obj
 0001:0003b481       __unwindfunclet$?calculateOutOfAlignment@DistanceMatrix@U2@@QAEXABVMultipleSequenceAlignment@2@ABVCreatePhyTreeSettings@2@@Z$7 1003c481 f   DistanceMatrix.obj
 0001:0003b48a       __unwindfunclet$?calculateOutOfAlignment@DistanceMatrix@U2@@QAEXABVMultipleSequenceAlignment@2@ABVCreatePhyTreeSettings@2@@Z$6 1003c48a f   DistanceMatrix.obj
 0001:0003b493       __unwindfunclet$?calculateOutOfAlignment@DistanceMatrix@U2@@QAEXABVMultipleSequenceAlignment@2@ABVCreatePhyTreeSettings@2@@Z$8 1003c493 f   DistanceMatrix.obj
 0001:0003b49c       __unwindfunclet$?calculateOutOfAlignment@DistanceMatrix@U2@@QAEXABVMultipleSequenceAlignment@2@ABVCreatePhyTreeSettings@2@@Z$9 1003c49c f   DistanceMatrix.obj
 0001:0003b4a5       __unwindfunclet$?calculateOutOfAlignment@DistanceMatrix@U2@@QAEXABVMultipleSequenceAlignment@2@ABVCreatePhyTreeSettings@2@@Z$10 1003c4a5 f   DistanceMatrix.obj
 0001:0003b4ae       __ehhandler$?calculateOutOfAlignment@DistanceMatrix@U2@@QAEXABVMultipleSequenceAlignment@2@ABVCreatePhyTreeSettings@2@@Z 1003c4ae f   DistanceMatrix.obj
 0001:0003b4d0       __unwindfunclet$?calculateQMatrix@DistanceMatrix@U2@@AAEXXZ$0 1003c4d0 f   DistanceMatrix.obj
 0001:0003b4d8       __ehhandler$?calculateQMatrix@DistanceMatrix@U2@@AAEXXZ 1003c4d8 f   DistanceMatrix.obj
 0001:0003b500       __unwindfunclet$?clear@?$QVector@V?$QVector@M@@@@QAEXXZ$0 1003c500 f   DistanceMatrix.obj
 0001:0003b508       __ehhandler$?clear@?$QVector@V?$QVector@M@@@@QAEXXZ 1003c508 f   DistanceMatrix.obj
 0001:0003b530       __unwindfunclet$?clone@?$QSharedDataPointer@VPhyTreeData@U2@@@@IAEPAVPhyTreeData@U2@@XZ$0 1003c530 f   DistanceMatrix.obj
 0001:0003b53b       __ehhandler$?clone@?$QSharedDataPointer@VPhyTreeData@U2@@@@IAEPAVPhyTreeData@U2@@XZ 1003c53b f   DistanceMatrix.obj
 0001:0003b560       __unwindfunclet$?copyConstruct@?$QVector@V?$QVector@M@@@@AAEXPBV?$QVector@M@@0PAV2@@Z$0 1003c560 f   DistanceMatrix.obj
 0001:0003b571       __ehhandler$?copyConstruct@?$QVector@V?$QVector@M@@@@AAEXPBV?$QVector@M@@0PAV2@@Z 1003c571 f   DistanceMatrix.obj
 0001:0003b590       __unwindfunclet$?createNode@?$QMapData@VQString@@H@@QAEPAU?$QMapNode@VQString@@H@@ABVQString@@ABHPAU2@_N@Z$4 1003c590 f   DistanceMatrix.obj
 0001:0003b5a4       __ehhandler$?createNode@?$QMapData@VQString@@H@@QAEPAU?$QMapNode@VQString@@H@@ABVQString@@ABHPAU2@_N@Z 1003c5a4 f   DistanceMatrix.obj
 0001:0003b5c0       __ehhandler$?detach_helper@?$QList@PAVPhyNode@U2@@@@AAEXH@Z 1003c5c0 f   DistanceMatrix.obj
 0001:0003b5e0       __ehhandler$?detach_helper@?$QList@VQString@@@@AAEXH@Z 1003c5e0 f   DistanceMatrix.obj
 0001:0003b600       __unwindfunclet$?detach_helper@?$QSharedDataPointer@VPhyTreeData@U2@@@@AAEXXZ$0 1003c600 f   DistanceMatrix.obj
 0001:0003b60b       __ehhandler$?detach_helper@?$QSharedDataPointer@VPhyTreeData@U2@@@@AAEXXZ 1003c60b f   DistanceMatrix.obj
 0001:0003b630       __ehhandler$?detach_helper_grow@?$QList@PAVPhyBranch@U2@@@@AAEPAUNode@1@HH@Z 1003c630 f   DistanceMatrix.obj
 0001:0003b650       __ehhandler$?detach_helper_grow@?$QList@PAVPhyNode@U2@@@@AAEPAUNode@1@HH@Z 1003c650 f   DistanceMatrix.obj
 0001:0003b670       __ehhandler$?detach_helper_grow@?$QList@VQString@@@@AAEPAUNode@1@HH@Z 1003c670 f   DistanceMatrix.obj
 0001:0003b690       __unwindfunclet$?findNode@DistanceMatrix@U2@@AAEPAVPhyNode@2@PAV32@VQString@@@Z$0 1003c690 f   DistanceMatrix.obj
 0001:0003b699       __ehhandler$?findNode@DistanceMatrix@U2@@AAEPAVPhyNode@2@PAV32@VQString@@@Z 1003c699 f   DistanceMatrix.obj
 0001:0003b6c0       __unwindfunclet$?generateNodeName@DistanceMatrix@U2@@AAE?AVQString@@V3@0@Z$0 1003c6c0 f   DistanceMatrix.obj
 0001:0003b6c9       __unwindfunclet$?generateNodeName@DistanceMatrix@U2@@AAE?AVQString@@V3@0@Z$1 1003c6c9 f   DistanceMatrix.obj
 0001:0003b6d2       __unwindfunclet$?generateNodeName@DistanceMatrix@U2@@AAE?AVQString@@V3@0@Z$2 1003c6d2 f   DistanceMatrix.obj
 0001:0003b6ec       __ehhandler$?generateNodeName@DistanceMatrix@U2@@AAE?AVQString@@V3@0@Z 1003c6ec f   DistanceMatrix.obj
 0001:0003b710       __unwindfunclet$?getNewIndex@DistanceMatrix@U2@@AAEHVQString@@U?$QPair@HH@@AAV?$QMap@VQString@@H@@@Z$0 1003c710 f   DistanceMatrix.obj
 0001:0003b719       __ehhandler$?getNewIndex@DistanceMatrix@U2@@AAEHVQString@@U?$QPair@HH@@AAV?$QMap@VQString@@H@@@Z 1003c719 f   DistanceMatrix.obj
 0001:0003b740       __unwindfunclet$?getNodeByName@DistanceMatrix@U2@@AAEPAVPhyNode@2@VQString@@@Z$0 1003c740 f   DistanceMatrix.obj
 0001:0003b749       __ehhandler$?getNodeByName@DistanceMatrix@U2@@AAEPAVPhyNode@2@VQString@@@Z 1003c749 f   DistanceMatrix.obj
 0001:0003b770       __unwindfunclet$?keys@?$QMap@VQString@@H@@QBE?AV?$QList@VQString@@@@ABH@Z$0 1003c770 f   DistanceMatrix.obj
 0001:0003b789       __ehhandler$?keys@?$QMap@VQString@@H@@QBE?AV?$QList@VQString@@@@ABH@Z 1003c789 f   DistanceMatrix.obj
 0001:0003b7b0       __unwindfunclet$?keys@?$QMap@VQString@@H@@QBE?AV?$QList@VQString@@@@XZ$0 1003c7b0 f   DistanceMatrix.obj
 0001:0003b7c9       __ehhandler$?keys@?$QMap@VQString@@H@@QBE?AV?$QList@VQString@@@@XZ 1003c7c9 f   DistanceMatrix.obj
 0001:0003b7f0       __unwindfunclet$?node_construct@?$QList@VQString@@@@AAEXPAUNode@1@ABVQString@@@Z$1 1003c7f0 f   DistanceMatrix.obj
 0001:0003b801       __ehhandler$?node_construct@?$QList@VQString@@@@AAEXPAUNode@1@ABVQString@@@Z 1003c801 f   DistanceMatrix.obj
 0001:0003b820       __unwindfunclet$?node_copy@?$QList@VMultipleSequenceAlignmentRow@U2@@@@AAEXPAUNode@1@00@Z$4 1003c820 f   DistanceMatrix.obj
 0001:0003b82b       __ehhandler$?node_copy@?$QList@VMultipleSequenceAlignmentRow@U2@@@@AAEXPAUNode@1@00@Z 1003c82b f   DistanceMatrix.obj
 0001:0003b850       __unwindfunclet$?node_copy@?$QList@VQString@@@@AAEXPAUNode@1@00@Z$5 1003c850 f   DistanceMatrix.obj
 0001:0003b861       __ehhandler$?node_copy@?$QList@VQString@@@@AAEXPAUNode@1@00@Z 1003c861 f   DistanceMatrix.obj
 0001:0003b880       __unwindfunclet$?printIndex@DistanceMatrix@U2@@AAEXXZ$0 1003c880 f   DistanceMatrix.obj
 0001:0003b888       __unwindfunclet$?printIndex@DistanceMatrix@U2@@AAEXXZ$1 1003c888 f   DistanceMatrix.obj
 0001:0003b891       __ehhandler$?printIndex@DistanceMatrix@U2@@AAEXXZ 1003c891 f   DistanceMatrix.obj
 0001:0003b8b0       __unwindfunclet$?printPhyNode@DistanceMatrix@U2@@CAXPAVPhyNode@2@HAAV?$QList@PAVPhyNode@U2@@@@@Z$0 1003c8b0 f   DistanceMatrix.obj
 0001:0003b8b9       __ehhandler$?printPhyNode@DistanceMatrix@U2@@CAXPAVPhyNode@2@HAAV?$QList@PAVPhyNode@U2@@@@@Z 1003c8b9 f   DistanceMatrix.obj
 0001:0003b8e0       __ehhandler$?reallocData@?$QVector@M@@AAEXHHV?$QFlags@W4AllocationOption@QArrayData@@@@@Z 1003c8e0 f   DistanceMatrix.obj
 0001:0003b900       __unwindfunclet$?reallocData@?$QVector@V?$QVector@M@@@@AAEXHHV?$QFlags@W4AllocationOption@QArrayData@@@@@Z$4 1003c900 f   DistanceMatrix.obj
 0001:0003b911       __ehhandler$?reallocData@?$QVector@V?$QVector@M@@@@AAEXHHV?$QFlags@W4AllocationOption@QArrayData@@@@@Z 1003c911 f   DistanceMatrix.obj
 0001:0003b930       __unwindfunclet$?release@MemoryLocker@U2@@QAEXXZ$0 1003c930 f   DistanceMatrix.obj
 0001:0003b939       __ehhandler$?release@MemoryLocker@U2@@QAEXXZ 1003c939 f   DistanceMatrix.obj
 0001:0003b960       __unwindfunclet$?removeAll@?$QList@VQString@@@@QAEHABVQString@@@Z$0 1003c960 f   DistanceMatrix.obj
 0001:0003b969       __ehhandler$?removeAll@?$QList@VQString@@@@QAEHABVQString@@@Z 1003c969 f   DistanceMatrix.obj
 0001:0003b990       __unwindfunclet$?switchName@DistanceMatrix@U2@@AAEXPAVPhyNode@2@@Z$0 1003c990 f   DistanceMatrix.obj
 0001:0003b999       __unwindfunclet$?switchName@DistanceMatrix@U2@@AAEXPAVPhyNode@2@@Z$1 1003c999 f   DistanceMatrix.obj
 0001:0003b9a2       __unwindfunclet$?switchName@DistanceMatrix@U2@@AAEXPAVPhyNode@2@@Z$2 1003c9a2 f   DistanceMatrix.obj
 0001:0003b9ab       __unwindfunclet$?switchName@DistanceMatrix@U2@@AAEXPAVPhyNode@2@@Z$3 1003c9ab f   DistanceMatrix.obj
 0001:0003b9b4       __unwindfunclet$?switchName@DistanceMatrix@U2@@AAEXPAVPhyNode@2@@Z$4 1003c9b4 f   DistanceMatrix.obj
 0001:0003b9bd       __ehhandler$?switchName@DistanceMatrix@U2@@AAEXPAVPhyNode@2@@Z 1003c9bd f   DistanceMatrix.obj
 0001:0003b9e0       __unwindfunclet$?switchNamesToAllNodes@DistanceMatrix@U2@@AAEXXZ$0 1003c9e0 f   DistanceMatrix.obj
 0001:0003b9e8       __unwindfunclet$?switchNamesToAllNodes@DistanceMatrix@U2@@AAEXXZ$1 1003c9e8 f   DistanceMatrix.obj
 0001:0003b9f0       __unwindfunclet$?switchNamesToAllNodes@DistanceMatrix@U2@@AAEXXZ$2 1003c9f0 f   DistanceMatrix.obj
 0001:0003b9f8       __ehhandler$?switchNamesToAllNodes@DistanceMatrix@U2@@AAEXXZ 1003c9f8 f   DistanceMatrix.obj
 0001:0003ba20       __unwindfunclet$?tryAcquire@MemoryLocker@U2@@QAE_N_J@Z$0 1003ca20 f   DistanceMatrix.obj
 0001:0003ba29       __unwindfunclet$?tryAcquire@MemoryLocker@U2@@QAE_N_J@Z$1 1003ca29 f   DistanceMatrix.obj
 0001:0003ba32       __unwindfunclet$?tryAcquire@MemoryLocker@U2@@QAE_N_J@Z$2 1003ca32 f   DistanceMatrix.obj
 0001:0003ba3b       __ehhandler$?tryAcquire@MemoryLocker@U2@@QAE_N_J@Z 1003ca3b f   DistanceMatrix.obj
 0001:0003ba60       __unwindfunclet$?uniqueKeys@?$QMap@VQString@@H@@QBE?AV?$QList@VQString@@@@XZ$1 1003ca60 f   DistanceMatrix.obj
 0001:0003ba79       __ehhandler$?uniqueKeys@?$QMap@VQString@@H@@QBE?AV?$QList@VQString@@@@XZ 1003ca79 f   DistanceMatrix.obj
 0001:0003baa0       __unwindfunclet$??0MemoryLocker@U2@@QAE@AAVU2OpStatus@1@HW4MemoryLockType@AppResource@1@@Z$0 1003caa0 f   NeighborJoinAdapter.obj
 0001:0003baac       __ehhandler$??0MemoryLocker@U2@@QAE@AAVU2OpStatus@1@HW4MemoryLockType@AppResource@1@@Z 1003caac f   NeighborJoinAdapter.obj
 0001:0003bad0       __unwindfunclet$??0NeighborJoinCalculateTreeTask@U2@@QAE@ABVMultipleSequenceAlignment@1@ABVCreatePhyTreeSettings@1@@Z$0 1003cad0 f   NeighborJoinAdapter.obj
 0001:0003bad9       __unwindfunclet$??0NeighborJoinCalculateTreeTask@U2@@QAE@ABVMultipleSequenceAlignment@1@ABVCreatePhyTreeSettings@1@@Z$3 1003cad9 f   NeighborJoinAdapter.obj
 0001:0003bae5       __unwindfunclet$??0NeighborJoinCalculateTreeTask@U2@@QAE@ABVMultipleSequenceAlignment@1@ABVCreatePhyTreeSettings@1@@Z$1 1003cae5 f   NeighborJoinAdapter.obj
 0001:0003baf3       __unwindfunclet$??0NeighborJoinCalculateTreeTask@U2@@QAE@ABVMultipleSequenceAlignment@1@ABVCreatePhyTreeSettings@1@@Z$2 1003caf3 f   NeighborJoinAdapter.obj
 0001:0003bafc       __ehhandler$??0NeighborJoinCalculateTreeTask@U2@@QAE@ABVMultipleSequenceAlignment@1@ABVCreatePhyTreeSettings@1@@Z 1003cafc f   NeighborJoinAdapter.obj
 0001:0003bb20       __unwindfunclet$??1NeighborJoinCalculateTreeTask@U2@@UAE@XZ$0 1003cb20 f   NeighborJoinAdapter.obj
 0001:0003bb29       __unwindfunclet$??1NeighborJoinCalculateTreeTask@U2@@UAE@XZ$2 1003cb29 f   NeighborJoinAdapter.obj
 0001:0003bb35       __ehhandler$??1NeighborJoinCalculateTreeTask@U2@@UAE@XZ 1003cb35 f   NeighborJoinAdapter.obj
 0001:0003bb50       __unwindfunclet$??_GNeighborJoinCalculateTreeTask@U2@@UAEPAXI@Z$0 1003cb50 f   NeighborJoinAdapter.obj
 0001:0003bb59       __unwindfunclet$??_GNeighborJoinCalculateTreeTask@U2@@UAEPAXI@Z$2 1003cb59 f   NeighborJoinAdapter.obj
 0001:0003bb65       __ehhandler$??_GNeighborJoinCalculateTreeTask@U2@@UAEPAXI@Z 1003cb65 f   NeighborJoinAdapter.obj
 0001:0003bb80       __unwindfunclet$??__EalgoLog@U2@@YAXXZ$0 1003cb80 f   NeighborJoinAdapter.obj
 0001:0003bb89       __ehhandler$??__EalgoLog@U2@@YAXXZ 1003cb89 f   NeighborJoinAdapter.obj
 0001:0003bbb0       __unwindfunclet$??__EcmdLog@U2@@YAXXZ$0 1003cbb0 f   NeighborJoinAdapter.obj
 0001:0003bbb9       __ehhandler$??__EcmdLog@U2@@YAXXZ 1003cbb9 f   NeighborJoinAdapter.obj
 0001:0003bbe0       __unwindfunclet$??__EcoreLog@U2@@YAXXZ$0 1003cbe0 f   NeighborJoinAdapter.obj
 0001:0003bbe9       __ehhandler$??__EcoreLog@U2@@YAXXZ 1003cbe9 f   NeighborJoinAdapter.obj
 0001:0003bc10       __unwindfunclet$??__EioLog@U2@@YAXXZ$0 1003cc10 f   NeighborJoinAdapter.obj
 0001:0003bc19       __ehhandler$??__EioLog@U2@@YAXXZ 1003cc19 f   NeighborJoinAdapter.obj
 0001:0003bc40       __unwindfunclet$??__EperfLog@U2@@YAXXZ$0 1003cc40 f   NeighborJoinAdapter.obj
 0001:0003bc49       __ehhandler$??__EperfLog@U2@@YAXXZ 1003cc49 f   NeighborJoinAdapter.obj
 0001:0003bc70       __unwindfunclet$??__EscriptLog@U2@@YAXXZ$0 1003cc70 f   NeighborJoinAdapter.obj
 0001:0003bc79       __ehhandler$??__EscriptLog@U2@@YAXXZ 1003cc79 f   NeighborJoinAdapter.obj
 0001:0003bca0       __unwindfunclet$??__EtaskLog@U2@@YAXXZ$0 1003cca0 f   NeighborJoinAdapter.obj
 0001:0003bca9       __ehhandler$??__EtaskLog@U2@@YAXXZ 1003cca9 f   NeighborJoinAdapter.obj
 0001:0003bcd0       __unwindfunclet$??__EuiLog@U2@@YAXXZ$0 1003ccd0 f   NeighborJoinAdapter.obj
 0001:0003bcd9       __ehhandler$??__EuiLog@U2@@YAXXZ 1003ccd9 f   NeighborJoinAdapter.obj
 0001:0003bd00       __unwindfunclet$??__EuserActLog@U2@@YAXXZ$0 1003cd00 f   NeighborJoinAdapter.obj
 0001:0003bd09       __ehhandler$??__EuserActLog@U2@@YAXXZ 1003cd09 f   NeighborJoinAdapter.obj
 0001:0003bd30       __unwindfunclet$?createCalculatePhyTreeTask@NeighborJoinAdapter@U2@@UAEPAVTask@2@ABVMultipleSequenceAlignment@2@ABVCreatePhyTreeSettings@2@@Z$0 1003cd30 f   NeighborJoinAdapter.obj
 0001:0003bd3b       __ehhandler$?createCalculatePhyTreeTask@NeighborJoinAdapter@U2@@UAEPAVTask@2@ABVMultipleSequenceAlignment@2@ABVCreatePhyTreeSettings@2@@Z 1003cd3b f   NeighborJoinAdapter.obj
 0001:0003bd60       __unwindfunclet$?createPhyTreeFromPhylipTree@U2@@YAXABVMultipleSequenceAlignment@1@PAUnode@@NE1PAVPhyNode@1@H@Z$0 1003cd60 f   NeighborJoinAdapter.obj
 0001:0003bd6b       __unwindfunclet$?createPhyTreeFromPhylipTree@U2@@YAXABVMultipleSequenceAlignment@1@PAUnode@@NE1PAVPhyNode@1@H@Z$1 1003cd6b f   NeighborJoinAdapter.obj
 0001:0003bd74       __unwindfunclet$?createPhyTreeFromPhylipTree@U2@@YAXABVMultipleSequenceAlignment@1@PAUnode@@NE1PAVPhyNode@1@H@Z$2 1003cd74 f   NeighborJoinAdapter.obj
 0001:0003bd7d       __unwindfunclet$?createPhyTreeFromPhylipTree@U2@@YAXABVMultipleSequenceAlignment@1@PAUnode@@NE1PAVPhyNode@1@H@Z$3 1003cd7d f   NeighborJoinAdapter.obj
 0001:0003bd86       __unwindfunclet$?createPhyTreeFromPhylipTree@U2@@YAXABVMultipleSequenceAlignment@1@PAUnode@@NE1PAVPhyNode@1@H@Z$4 1003cd86 f   NeighborJoinAdapter.obj
 0001:0003bd8f       __unwindfunclet$?createPhyTreeFromPhylipTree@U2@@YAXABVMultipleSequenceAlignment@1@PAUnode@@NE1PAVPhyNode@1@H@Z$5 1003cd8f f   NeighborJoinAdapter.obj
 0001:0003bd98       __ehhandler$?createPhyTreeFromPhylipTree@U2@@YAXABVMultipleSequenceAlignment@1@PAUnode@@NE1PAVPhyNode@1@H@Z 1003cd98 f   NeighborJoinAdapter.obj
 0001:0003bdc0       __unwindfunclet$?createPhyTreeSettingsWidget@NeighborJoinAdapter@U2@@UAEPAVCreatePhyTreeWidget@2@ABVMultipleSequenceAlignment@2@PAVQWidget@@@Z$0 1003cdc0 f   NeighborJoinAdapter.obj
 0001:0003bdcb       __ehhandler$?createPhyTreeSettingsWidget@NeighborJoinAdapter@U2@@UAEPAVCreatePhyTreeWidget@2@ABVMultipleSequenceAlignment@2@PAVQWidget@@@Z 1003cdcb f   NeighborJoinAdapter.obj
 0001:0003bdf0       __unwindfunclet$?run@NeighborJoinCalculateTreeTask@U2@@UAEXXZ$3 1003cdf0 f   NeighborJoinAdapter.obj
 0001:0003bdf9       __unwindfunclet$?run@NeighborJoinCalculateTreeTask@U2@@UAEXXZ$4 1003cdf9 f   NeighborJoinAdapter.obj
 0001:0003be07       __unwindfunclet$?run@NeighborJoinCalculateTreeTask@U2@@UAEXXZ$5 1003ce07 f   NeighborJoinAdapter.obj
 0001:0003be10       __unwindfunclet$?run@NeighborJoinCalculateTreeTask@U2@@UAEXXZ$6 1003ce10 f   NeighborJoinAdapter.obj
 0001:0003be19       __unwindfunclet$?run@NeighborJoinCalculateTreeTask@U2@@UAEXXZ$7 1003ce19 f   NeighborJoinAdapter.obj
 0001:0003be25       __unwindfunclet$?run@NeighborJoinCalculateTreeTask@U2@@UAEXXZ$8 1003ce25 f   NeighborJoinAdapter.obj
 0001:0003be2d       __unwindfunclet$?run@NeighborJoinCalculateTreeTask@U2@@UAEXXZ$9 1003ce2d f   NeighborJoinAdapter.obj
 0001:0003be36       __unwindfunclet$?run@NeighborJoinCalculateTreeTask@U2@@UAEXXZ$10 1003ce36 f   NeighborJoinAdapter.obj
 0001:0003be3f       __unwindfunclet$?run@NeighborJoinCalculateTreeTask@U2@@UAEXXZ$11 1003ce3f f   NeighborJoinAdapter.obj
 0001:0003be4a       __unwindfunclet$?run@NeighborJoinCalculateTreeTask@U2@@UAEXXZ$12 1003ce4a f   NeighborJoinAdapter.obj
 0001:0003be55       __unwindfunclet$?run@NeighborJoinCalculateTreeTask@U2@@UAEXXZ$13 1003ce55 f   NeighborJoinAdapter.obj
 0001:0003be5e       __unwindfunclet$?run@NeighborJoinCalculateTreeTask@U2@@UAEXXZ$14 1003ce5e f   NeighborJoinAdapter.obj
 0001:0003be67       __unwindfunclet$?run@NeighborJoinCalculateTreeTask@U2@@UAEXXZ$15 1003ce67 f   NeighborJoinAdapter.obj
 0001:0003be70       __unwindfunclet$?run@NeighborJoinCalculateTreeTask@U2@@UAEXXZ$16 1003ce70 f   NeighborJoinAdapter.obj
 0001:0003be79       __unwindfunclet$?run@NeighborJoinCalculateTreeTask@U2@@UAEXXZ$17 1003ce79 f   NeighborJoinAdapter.obj
 0001:0003be84       __unwindfunclet$?run@NeighborJoinCalculateTreeTask@U2@@UAEXXZ$18 1003ce84 f   NeighborJoinAdapter.obj
 0001:0003be8c       __unwindfunclet$?run@NeighborJoinCalculateTreeTask@U2@@UAEXXZ$19 1003ce8c f   NeighborJoinAdapter.obj
 0001:0003be95       __unwindfunclet$?run@NeighborJoinCalculateTreeTask@U2@@UAEXXZ$20 1003ce95 f   NeighborJoinAdapter.obj
 0001:0003be9e       __unwindfunclet$?run@NeighborJoinCalculateTreeTask@U2@@UAEXXZ$21 1003ce9e f   NeighborJoinAdapter.obj
 0001:0003bea7       __unwindfunclet$?run@NeighborJoinCalculateTreeTask@U2@@UAEXXZ$22 1003cea7 f   NeighborJoinAdapter.obj
 0001:0003beb0       __unwindfunclet$?run@NeighborJoinCalculateTreeTask@U2@@UAEXXZ$23 1003ceb0 f   NeighborJoinAdapter.obj
 0001:0003beb9       __unwindfunclet$?run@NeighborJoinCalculateTreeTask@U2@@UAEXXZ$24 1003ceb9 f   NeighborJoinAdapter.obj
 0001:0003bec2       __unwindfunclet$?run@NeighborJoinCalculateTreeTask@U2@@UAEXXZ$25 1003cec2 f   NeighborJoinAdapter.obj
 0001:0003becb       __unwindfunclet$?run@NeighborJoinCalculateTreeTask@U2@@UAEXXZ$26 1003cecb f   NeighborJoinAdapter.obj
 0001:0003bed3       __unwindfunclet$?run@NeighborJoinCalculateTreeTask@U2@@UAEXXZ$27 1003ced3 f   NeighborJoinAdapter.obj
 0001:0003bedc       __unwindfunclet$?run@NeighborJoinCalculateTreeTask@U2@@UAEXXZ$28 1003cedc f   NeighborJoinAdapter.obj
 0001:0003bee4       __unwindfunclet$?run@NeighborJoinCalculateTreeTask@U2@@UAEXXZ$29 1003cee4 f   NeighborJoinAdapter.obj
 0001:0003beed       __unwindfunclet$?run@NeighborJoinCalculateTreeTask@U2@@UAEXXZ$30 1003ceed f   NeighborJoinAdapter.obj
 0001:0003bef5       __unwindfunclet$?run@NeighborJoinCalculateTreeTask@U2@@UAEXXZ$31 1003cef5 f   NeighborJoinAdapter.obj
 0001:0003befe       __unwindfunclet$?run@NeighborJoinCalculateTreeTask@U2@@UAEXXZ$32 1003cefe f   NeighborJoinAdapter.obj
 0001:0003bf06       __unwindfunclet$?run@NeighborJoinCalculateTreeTask@U2@@UAEXXZ$33 1003cf06 f   NeighborJoinAdapter.obj
 0001:0003bf11       __unwindfunclet$?run@NeighborJoinCalculateTreeTask@U2@@UAEXXZ$34 1003cf11 f   NeighborJoinAdapter.obj
 0001:0003bf1c       __unwindfunclet$?run@NeighborJoinCalculateTreeTask@U2@@UAEXXZ$35 1003cf1c f   NeighborJoinAdapter.obj
 0001:0003bf27       __unwindfunclet$?run@NeighborJoinCalculateTreeTask@U2@@UAEXXZ$36 1003cf27 f   NeighborJoinAdapter.obj
 0001:0003bf2f       __unwindfunclet$?run@NeighborJoinCalculateTreeTask@U2@@UAEXXZ$37 1003cf2f f   NeighborJoinAdapter.obj
 0001:0003bf38       __unwindfunclet$?run@NeighborJoinCalculateTreeTask@U2@@UAEXXZ$38 1003cf38 f   NeighborJoinAdapter.obj
 0001:0003bf41       __unwindfunclet$?run@NeighborJoinCalculateTreeTask@U2@@UAEXXZ$39 1003cf41 f   NeighborJoinAdapter.obj
 0001:0003bf4a       __unwindfunclet$?run@NeighborJoinCalculateTreeTask@U2@@UAEXXZ$40 1003cf4a f   NeighborJoinAdapter.obj
 0001:0003bf53       __unwindfunclet$?run@NeighborJoinCalculateTreeTask@U2@@UAEXXZ$41 1003cf53 f   NeighborJoinAdapter.obj
 0001:0003bf5c       __unwindfunclet$?run@NeighborJoinCalculateTreeTask@U2@@UAEXXZ$42 1003cf5c f   NeighborJoinAdapter.obj
 0001:0003bf67       __unwindfunclet$?run@NeighborJoinCalculateTreeTask@U2@@UAEXXZ$43 1003cf67 f   NeighborJoinAdapter.obj
 0001:0003bf72       __unwindfunclet$?run@NeighborJoinCalculateTreeTask@U2@@UAEXXZ$44 1003cf72 f   NeighborJoinAdapter.obj
 0001:0003bf7b       __unwindfunclet$?run@NeighborJoinCalculateTreeTask@U2@@UAEXXZ$45 1003cf7b f   NeighborJoinAdapter.obj
 0001:0003bf84       __unwindfunclet$?run@NeighborJoinCalculateTreeTask@U2@@UAEXXZ$46 1003cf84 f   NeighborJoinAdapter.obj
 0001:0003bf8d       __unwindfunclet$?run@NeighborJoinCalculateTreeTask@U2@@UAEXXZ$47 1003cf8d f   NeighborJoinAdapter.obj
 0001:0003bf96       __unwindfunclet$?run@NeighborJoinCalculateTreeTask@U2@@UAEXXZ$48 1003cf96 f   NeighborJoinAdapter.obj
 0001:0003bf9f       __unwindfunclet$?run@NeighborJoinCalculateTreeTask@U2@@UAEXXZ$49 1003cf9f f   NeighborJoinAdapter.obj
 0001:0003bfa8       __ehhandler$?run@NeighborJoinCalculateTreeTask@U2@@UAEXXZ 1003cfa8 f   NeighborJoinAdapter.obj
 0001:0003bfd0       __ehhandler$??0?$QList@VQString@@@@QAE@ABV0@@Z 1003cfd0 f   NeighborJoinWidget.obj
 0001:0003bff0       __unwindfunclet$??0NeighborJoinWidget@U2@@QAE@ABVMultipleSequenceAlignment@1@PAVQWidget@@@Z$0 1003cff0 f   NeighborJoinWidget.obj
 0001:0003bff9       __ehhandler$??0NeighborJoinWidget@U2@@QAE@ABVMultipleSequenceAlignment@1@PAVQWidget@@@Z 1003cff9 f   NeighborJoinWidget.obj
 0001:0003c020       __unwindfunclet$??H@YA?BVQString@@ABV0@PBD@Z$0 1003d020 f   NeighborJoinWidget.obj
 0001:0003c03a       __unwindfunclet$??H@YA?BVQString@@ABV0@PBD@Z$1 1003d03a f   NeighborJoinWidget.obj
 0001:0003c043       __ehhandler$??H@YA?BVQString@@ABV0@PBD@Z 1003d043 f   NeighborJoinWidget.obj
 0001:0003c060       __unwindfunclet$??__EalgoLog@U2@@YAXXZ$0 1003d060 f   NeighborJoinWidget.obj
 0001:0003c069       __ehhandler$??__EalgoLog@U2@@YAXXZ 1003d069 f   NeighborJoinWidget.obj
 0001:0003c090       __unwindfunclet$??__EcmdLog@U2@@YAXXZ$0 1003d090 f   NeighborJoinWidget.obj
 0001:0003c099       __ehhandler$??__EcmdLog@U2@@YAXXZ 1003d099 f   NeighborJoinWidget.obj
 0001:0003c0c0       __unwindfunclet$??__EcoreLog@U2@@YAXXZ$0 1003d0c0 f   NeighborJoinWidget.obj
 0001:0003c0c9       __ehhandler$??__EcoreLog@U2@@YAXXZ 1003d0c9 f   NeighborJoinWidget.obj
 0001:0003c0f0       __unwindfunclet$??__EioLog@U2@@YAXXZ$0 1003d0f0 f   NeighborJoinWidget.obj
 0001:0003c0f9       __ehhandler$??__EioLog@U2@@YAXXZ 1003d0f9 f   NeighborJoinWidget.obj
 0001:0003c120       __unwindfunclet$??__EperfLog@U2@@YAXXZ$0 1003d120 f   NeighborJoinWidget.obj
 0001:0003c129       __ehhandler$??__EperfLog@U2@@YAXXZ 1003d129 f   NeighborJoinWidget.obj
 0001:0003c150       __unwindfunclet$??__EscriptLog@U2@@YAXXZ$0 1003d150 f   NeighborJoinWidget.obj
 0001:0003c159       __ehhandler$??__EscriptLog@U2@@YAXXZ 1003d159 f   NeighborJoinWidget.obj
 0001:0003c180       __unwindfunclet$??__EtaskLog@U2@@YAXXZ$0 1003d180 f   NeighborJoinWidget.obj
 0001:0003c189       __ehhandler$??__EtaskLog@U2@@YAXXZ 1003d189 f   NeighborJoinWidget.obj
 0001:0003c1b0       __unwindfunclet$??__EuiLog@U2@@YAXXZ$0 1003d1b0 f   NeighborJoinWidget.obj
 0001:0003c1b9       __ehhandler$??__EuiLog@U2@@YAXXZ 1003d1b9 f   NeighborJoinWidget.obj
 0001:0003c1e0       __unwindfunclet$??__EuserActLog@U2@@YAXXZ$0 1003d1e0 f   NeighborJoinWidget.obj
 0001:0003c1e9       __ehhandler$??__EuserActLog@U2@@YAXXZ 1003d1e9 f   NeighborJoinWidget.obj
 0001:0003c210       __unwindfunclet$?checkMemoryEstimation@NeighborJoinWidget@U2@@UAE_NAAVQString@@ABVMultipleSequenceAlignment@2@ABVCreatePhyTreeSettings@2@@Z$0 1003d210 f   NeighborJoinWidget.obj
 0001:0003c219       __unwindfunclet$?checkMemoryEstimation@NeighborJoinWidget@U2@@UAE_NAAVQString@@ABVMultipleSequenceAlignment@2@ABVCreatePhyTreeSettings@2@@Z$1 1003d219 f   NeighborJoinWidget.obj
 0001:0003c222       __ehhandler$?checkMemoryEstimation@NeighborJoinWidget@U2@@UAE_NAAVQString@@ABVMultipleSequenceAlignment@2@ABVCreatePhyTreeSettings@2@@Z 1003d222 f   NeighborJoinWidget.obj
 0001:0003c240       __unwindfunclet$?checkSettings@NeighborJoinWidget@U2@@UAE_NAAVQString@@ABVCreatePhyTreeSettings@2@@Z$0 1003d240 f   NeighborJoinWidget.obj
 0001:0003c249       __ehhandler$?checkSettings@NeighborJoinWidget@U2@@UAE_NAAVQString@@ABVCreatePhyTreeSettings@2@@Z 1003d249 f   NeighborJoinWidget.obj
 0001:0003c270       __unwindfunclet$?fillSettings@NeighborJoinWidget@U2@@UAEXAAVCreatePhyTreeSettings@2@@Z$0 1003d270 f   NeighborJoinWidget.obj
 0001:0003c279       __unwindfunclet$?fillSettings@NeighborJoinWidget@U2@@UAEXAAVCreatePhyTreeSettings@2@@Z$1 1003d279 f   NeighborJoinWidget.obj
 0001:0003c282       __ehhandler$?fillSettings@NeighborJoinWidget@U2@@UAEXAAVCreatePhyTreeSettings@2@@Z 1003d282 f   NeighborJoinWidget.obj
 0001:0003c2a0       __unwindfunclet$?init@NeighborJoinWidget@U2@@AAEXABVMultipleSequenceAlignment@2@@Z$2 1003d2a0 f   NeighborJoinWidget.obj
 0001:0003c2a8       __unwindfunclet$?init@NeighborJoinWidget@U2@@AAEXABVMultipleSequenceAlignment@2@@Z$3 1003d2a8 f   NeighborJoinWidget.obj
 0001:0003c2b0       __unwindfunclet$?init@NeighborJoinWidget@U2@@AAEXABVMultipleSequenceAlignment@2@@Z$0 1003d2b0 f   NeighborJoinWidget.obj
 0001:0003c2b8       __unwindfunclet$?init@NeighborJoinWidget@U2@@AAEXABVMultipleSequenceAlignment@2@@Z$1 1003d2b8 f   NeighborJoinWidget.obj
 0001:0003c2c0       __unwindfunclet$?init@NeighborJoinWidget@U2@@AAEXABVMultipleSequenceAlignment@2@@Z$4 1003d2c0 f   NeighborJoinWidget.obj
 0001:0003c2c9       __unwindfunclet$?init@NeighborJoinWidget@U2@@AAEXABVMultipleSequenceAlignment@2@@Z$5 1003d2c9 f   NeighborJoinWidget.obj
 0001:0003c2d2       __unwindfunclet$?init@NeighborJoinWidget@U2@@AAEXABVMultipleSequenceAlignment@2@@Z$6 1003d2d2 f   NeighborJoinWidget.obj
 0001:0003c2db       __unwindfunclet$?init@NeighborJoinWidget@U2@@AAEXABVMultipleSequenceAlignment@2@@Z$7 1003d2db f   NeighborJoinWidget.obj
 0001:0003c2e4       __unwindfunclet$?init@NeighborJoinWidget@U2@@AAEXABVMultipleSequenceAlignment@2@@Z$8 1003d2e4 f   NeighborJoinWidget.obj
 0001:0003c2ed       __unwindfunclet$?init@NeighborJoinWidget@U2@@AAEXABVMultipleSequenceAlignment@2@@Z$9 1003d2ed f   NeighborJoinWidget.obj
 0001:0003c2f6       __unwindfunclet$?init@NeighborJoinWidget@U2@@AAEXABVMultipleSequenceAlignment@2@@Z$48 1003d2f6 f   NeighborJoinWidget.obj
 0001:0003c2ff       __unwindfunclet$?init@NeighborJoinWidget@U2@@AAEXABVMultipleSequenceAlignment@2@@Z$10 1003d2ff f   NeighborJoinWidget.obj
 0001:0003c308       __unwindfunclet$?init@NeighborJoinWidget@U2@@AAEXABVMultipleSequenceAlignment@2@@Z$11 1003d308 f   NeighborJoinWidget.obj
 0001:0003c311       __unwindfunclet$?init@NeighborJoinWidget@U2@@AAEXABVMultipleSequenceAlignment@2@@Z$12 1003d311 f   NeighborJoinWidget.obj
 0001:0003c31a       __unwindfunclet$?init@NeighborJoinWidget@U2@@AAEXABVMultipleSequenceAlignment@2@@Z$13 1003d31a f   NeighborJoinWidget.obj
 0001:0003c323       __unwindfunclet$?init@NeighborJoinWidget@U2@@AAEXABVMultipleSequenceAlignment@2@@Z$14 1003d323 f   NeighborJoinWidget.obj
 0001:0003c32c       __unwindfunclet$?init@NeighborJoinWidget@U2@@AAEXABVMultipleSequenceAlignment@2@@Z$15 1003d32c f   NeighborJoinWidget.obj
 0001:0003c335       __unwindfunclet$?init@NeighborJoinWidget@U2@@AAEXABVMultipleSequenceAlignment@2@@Z$16 1003d335 f   NeighborJoinWidget.obj
 0001:0003c33e       __unwindfunclet$?init@NeighborJoinWidget@U2@@AAEXABVMultipleSequenceAlignment@2@@Z$17 1003d33e f   NeighborJoinWidget.obj
 0001:0003c347       __unwindfunclet$?init@NeighborJoinWidget@U2@@AAEXABVMultipleSequenceAlignment@2@@Z$18 1003d347 f   NeighborJoinWidget.obj
 0001:0003c350       __unwindfunclet$?init@NeighborJoinWidget@U2@@AAEXABVMultipleSequenceAlignment@2@@Z$19 1003d350 f   NeighborJoinWidget.obj
 0001:0003c359       __unwindfunclet$?init@NeighborJoinWidget@U2@@AAEXABVMultipleSequenceAlignment@2@@Z$20 1003d359 f   NeighborJoinWidget.obj
 0001:0003c362       __unwindfunclet$?init@NeighborJoinWidget@U2@@AAEXABVMultipleSequenceAlignment@2@@Z$21 1003d362 f   NeighborJoinWidget.obj
 0001:0003c36b       __unwindfunclet$?init@NeighborJoinWidget@U2@@AAEXABVMultipleSequenceAlignment@2@@Z$22 1003d36b f   NeighborJoinWidget.obj
 0001:0003c373       __unwindfunclet$?init@NeighborJoinWidget@U2@@AAEXABVMultipleSequenceAlignment@2@@Z$23 1003d373 f   NeighborJoinWidget.obj
 0001:0003c37b       __unwindfunclet$?init@NeighborJoinWidget@U2@@AAEXABVMultipleSequenceAlignment@2@@Z$24 1003d37b f   NeighborJoinWidget.obj
 0001:0003c384       __unwindfunclet$?init@NeighborJoinWidget@U2@@AAEXABVMultipleSequenceAlignment@2@@Z$25 1003d384 f   NeighborJoinWidget.obj
 0001:0003c38d       __unwindfunclet$?init@NeighborJoinWidget@U2@@AAEXABVMultipleSequenceAlignment@2@@Z$26 1003d38d f   NeighborJoinWidget.obj
 0001:0003c396       __unwindfunclet$?init@NeighborJoinWidget@U2@@AAEXABVMultipleSequenceAlignment@2@@Z$27 1003d396 f   NeighborJoinWidget.obj
 0001:0003c39f       __unwindfunclet$?init@NeighborJoinWidget@U2@@AAEXABVMultipleSequenceAlignment@2@@Z$28 1003d39f f   NeighborJoinWidget.obj
 0001:0003c3a8       __unwindfunclet$?init@NeighborJoinWidget@U2@@AAEXABVMultipleSequenceAlignment@2@@Z$29 1003d3a8 f   NeighborJoinWidget.obj
 0001:0003c3b1       __unwindfunclet$?init@NeighborJoinWidget@U2@@AAEXABVMultipleSequenceAlignment@2@@Z$30 1003d3b1 f   NeighborJoinWidget.obj
 0001:0003c3ba       __unwindfunclet$?init@NeighborJoinWidget@U2@@AAEXABVMultipleSequenceAlignment@2@@Z$31 1003d3ba f   NeighborJoinWidget.obj
 0001:0003c3c3       __unwindfunclet$?init@NeighborJoinWidget@U2@@AAEXABVMultipleSequenceAlignment@2@@Z$32 1003d3c3 f   NeighborJoinWidget.obj
 0001:0003c3cc       __unwindfunclet$?init@NeighborJoinWidget@U2@@AAEXABVMultipleSequenceAlignment@2@@Z$33 1003d3cc f   NeighborJoinWidget.obj
 0001:0003c3d5       __unwindfunclet$?init@NeighborJoinWidget@U2@@AAEXABVMultipleSequenceAlignment@2@@Z$34 1003d3d5 f   NeighborJoinWidget.obj
 0001:0003c3de       __unwindfunclet$?init@NeighborJoinWidget@U2@@AAEXABVMultipleSequenceAlignment@2@@Z$35 1003d3de f   NeighborJoinWidget.obj
 0001:0003c3e7       __unwindfunclet$?init@NeighborJoinWidget@U2@@AAEXABVMultipleSequenceAlignment@2@@Z$36 1003d3e7 f   NeighborJoinWidget.obj
 0001:0003c3f0       __unwindfunclet$?init@NeighborJoinWidget@U2@@AAEXABVMultipleSequenceAlignment@2@@Z$37 1003d3f0 f   NeighborJoinWidget.obj
 0001:0003c3f9       __unwindfunclet$?init@NeighborJoinWidget@U2@@AAEXABVMultipleSequenceAlignment@2@@Z$38 1003d3f9 f   NeighborJoinWidget.obj
 0001:0003c402       __unwindfunclet$?init@NeighborJoinWidget@U2@@AAEXABVMultipleSequenceAlignment@2@@Z$39 1003d402 f   NeighborJoinWidget.obj
 0001:0003c40b       __unwindfunclet$?init@NeighborJoinWidget@U2@@AAEXABVMultipleSequenceAlignment@2@@Z$40 1003d40b f   NeighborJoinWidget.obj
 0001:0003c414       __unwindfunclet$?init@NeighborJoinWidget@U2@@AAEXABVMultipleSequenceAlignment@2@@Z$41 1003d414 f   NeighborJoinWidget.obj
 0001:0003c41d       __unwindfunclet$?init@NeighborJoinWidget@U2@@AAEXABVMultipleSequenceAlignment@2@@Z$42 1003d41d f   NeighborJoinWidget.obj
 0001:0003c426       __unwindfunclet$?init@NeighborJoinWidget@U2@@AAEXABVMultipleSequenceAlignment@2@@Z$43 1003d426 f   NeighborJoinWidget.obj
 0001:0003c42f       __unwindfunclet$?init@NeighborJoinWidget@U2@@AAEXABVMultipleSequenceAlignment@2@@Z$44 1003d42f f   NeighborJoinWidget.obj
 0001:0003c438       __unwindfunclet$?init@NeighborJoinWidget@U2@@AAEXABVMultipleSequenceAlignment@2@@Z$45 1003d438 f   NeighborJoinWidget.obj
 0001:0003c441       __unwindfunclet$?init@NeighborJoinWidget@U2@@AAEXABVMultipleSequenceAlignment@2@@Z$50 1003d441 f   NeighborJoinWidget.obj
 0001:0003c44a       __ehhandler$?init@NeighborJoinWidget@U2@@AAEXABVMultipleSequenceAlignment@2@@Z 1003d44a f   NeighborJoinWidget.obj
 0001:0003c470       __unwindfunclet$?restoreDefault@NeighborJoinWidget@U2@@UAEXXZ$0 1003d470 f   NeighborJoinWidget.obj
 0001:0003c479       __unwindfunclet$?restoreDefault@NeighborJoinWidget@U2@@UAEXXZ$1 1003d479 f   NeighborJoinWidget.obj
 0001:0003c482       __unwindfunclet$?restoreDefault@NeighborJoinWidget@U2@@UAEXXZ$2 1003d482 f   NeighborJoinWidget.obj
 0001:0003c48b       __unwindfunclet$?restoreDefault@NeighborJoinWidget@U2@@UAEXXZ$3 1003d48b f   NeighborJoinWidget.obj
 0001:0003c494       __unwindfunclet$?restoreDefault@NeighborJoinWidget@U2@@UAEXXZ$4 1003d494 f   NeighborJoinWidget.obj
 0001:0003c49d       __unwindfunclet$?restoreDefault@NeighborJoinWidget@U2@@UAEXXZ$5 1003d49d f   NeighborJoinWidget.obj
 0001:0003c4a6       __unwindfunclet$?restoreDefault@NeighborJoinWidget@U2@@UAEXXZ$6 1003d4a6 f   NeighborJoinWidget.obj
 0001:0003c4af       __unwindfunclet$?restoreDefault@NeighborJoinWidget@U2@@UAEXXZ$7 1003d4af f   NeighborJoinWidget.obj
 0001:0003c4b8       __unwindfunclet$?restoreDefault@NeighborJoinWidget@U2@@UAEXXZ$8 1003d4b8 f   NeighborJoinWidget.obj
 0001:0003c4c1       __unwindfunclet$?restoreDefault@NeighborJoinWidget@U2@@UAEXXZ$9 1003d4c1 f   NeighborJoinWidget.obj
 0001:0003c4ca       __unwindfunclet$?restoreDefault@NeighborJoinWidget@U2@@UAEXXZ$10 1003d4ca f   NeighborJoinWidget.obj
 0001:0003c4d3       __unwindfunclet$?restoreDefault@NeighborJoinWidget@U2@@UAEXXZ$11 1003d4d3 f   NeighborJoinWidget.obj
 0001:0003c4dc       __unwindfunclet$?restoreDefault@NeighborJoinWidget@U2@@UAEXXZ$12 1003d4dc f   NeighborJoinWidget.obj
 0001:0003c4e5       __unwindfunclet$?restoreDefault@NeighborJoinWidget@U2@@UAEXXZ$13 1003d4e5 f   NeighborJoinWidget.obj
 0001:0003c4ee       __unwindfunclet$?restoreDefault@NeighborJoinWidget@U2@@UAEXXZ$14 1003d4ee f   NeighborJoinWidget.obj
 0001:0003c4f7       __unwindfunclet$?restoreDefault@NeighborJoinWidget@U2@@UAEXXZ$15 1003d4f7 f   NeighborJoinWidget.obj
 0001:0003c500       __unwindfunclet$?restoreDefault@NeighborJoinWidget@U2@@UAEXXZ$16 1003d500 f   NeighborJoinWidget.obj
 0001:0003c509       __unwindfunclet$?restoreDefault@NeighborJoinWidget@U2@@UAEXXZ$17 1003d509 f   NeighborJoinWidget.obj
 0001:0003c512       __ehhandler$?restoreDefault@NeighborJoinWidget@U2@@UAEXXZ 1003d512 f   NeighborJoinWidget.obj
 0001:0003c530       __unwindfunclet$?retranslateUi@Ui_NeighborJoinWidget@@QAEXPAVQWidget@@@Z$0 1003d530 f   NeighborJoinWidget.obj
 0001:0003c539       __unwindfunclet$?retranslateUi@Ui_NeighborJoinWidget@@QAEXPAVQWidget@@@Z$1 1003d539 f   NeighborJoinWidget.obj
 0001:0003c542       __unwindfunclet$?retranslateUi@Ui_NeighborJoinWidget@@QAEXPAVQWidget@@@Z$2 1003d542 f   NeighborJoinWidget.obj
 0001:0003c54b       __unwindfunclet$?retranslateUi@Ui_NeighborJoinWidget@@QAEXPAVQWidget@@@Z$3 1003d54b f   NeighborJoinWidget.obj
 0001:0003c554       __unwindfunclet$?retranslateUi@Ui_NeighborJoinWidget@@QAEXPAVQWidget@@@Z$4 1003d554 f   NeighborJoinWidget.obj
 0001:0003c55d       __unwindfunclet$?retranslateUi@Ui_NeighborJoinWidget@@QAEXPAVQWidget@@@Z$5 1003d55d f   NeighborJoinWidget.obj
 0001:0003c566       __unwindfunclet$?retranslateUi@Ui_NeighborJoinWidget@@QAEXPAVQWidget@@@Z$6 1003d566 f   NeighborJoinWidget.obj
 0001:0003c56f       __unwindfunclet$?retranslateUi@Ui_NeighborJoinWidget@@QAEXPAVQWidget@@@Z$7 1003d56f f   NeighborJoinWidget.obj
 0001:0003c578       __unwindfunclet$?retranslateUi@Ui_NeighborJoinWidget@@QAEXPAVQWidget@@@Z$8 1003d578 f   NeighborJoinWidget.obj
 0001:0003c581       __unwindfunclet$?retranslateUi@Ui_NeighborJoinWidget@@QAEXPAVQWidget@@@Z$9 1003d581 f   NeighborJoinWidget.obj
 0001:0003c58a       __unwindfunclet$?retranslateUi@Ui_NeighborJoinWidget@@QAEXPAVQWidget@@@Z$10 1003d58a f   NeighborJoinWidget.obj
 0001:0003c593       __unwindfunclet$?retranslateUi@Ui_NeighborJoinWidget@@QAEXPAVQWidget@@@Z$11 1003d593 f   NeighborJoinWidget.obj
 0001:0003c59c       __ehhandler$?retranslateUi@Ui_NeighborJoinWidget@@QAEXPAVQWidget@@@Z 1003d59c f   NeighborJoinWidget.obj
 0001:0003c5c0       __unwindfunclet$?setupUi@Ui_NeighborJoinWidget@@QAEXPAVQWidget@@@Z$1 1003d5c0 f   NeighborJoinWidget.obj
 0001:0003c5c9       __unwindfunclet$?setupUi@Ui_NeighborJoinWidget@@QAEXPAVQWidget@@@Z$2 1003d5c9 f   NeighborJoinWidget.obj
 0001:0003c5d4       __unwindfunclet$?setupUi@Ui_NeighborJoinWidget@@QAEXPAVQWidget@@@Z$3 1003d5d4 f   NeighborJoinWidget.obj
 0001:0003c5dd       __unwindfunclet$?setupUi@Ui_NeighborJoinWidget@@QAEXPAVQWidget@@@Z$4 1003d5dd f   NeighborJoinWidget.obj
 0001:0003c5e8       __unwindfunclet$?setupUi@Ui_NeighborJoinWidget@@QAEXPAVQWidget@@@Z$5 1003d5e8 f   NeighborJoinWidget.obj
 0001:0003c5f1       __unwindfunclet$?setupUi@Ui_NeighborJoinWidget@@QAEXPAVQWidget@@@Z$6 1003d5f1 f   NeighborJoinWidget.obj
 0001:0003c5fc       __unwindfunclet$?setupUi@Ui_NeighborJoinWidget@@QAEXPAVQWidget@@@Z$7 1003d5fc f   NeighborJoinWidget.obj
 0001:0003c605       __unwindfunclet$?setupUi@Ui_NeighborJoinWidget@@QAEXPAVQWidget@@@Z$8 1003d605 f   NeighborJoinWidget.obj
 0001:0003c610       __unwindfunclet$?setupUi@Ui_NeighborJoinWidget@@QAEXPAVQWidget@@@Z$9 1003d610 f   NeighborJoinWidget.obj
 0001:0003c619       __unwindfunclet$?setupUi@Ui_NeighborJoinWidget@@QAEXPAVQWidget@@@Z$10 1003d619 f   NeighborJoinWidget.obj
 0001:0003c624       __unwindfunclet$?setupUi@Ui_NeighborJoinWidget@@QAEXPAVQWidget@@@Z$11 1003d624 f   NeighborJoinWidget.obj
 0001:0003c62d       __unwindfunclet$?setupUi@Ui_NeighborJoinWidget@@QAEXPAVQWidget@@@Z$12 1003d62d f   NeighborJoinWidget.obj
 0001:0003c638       __unwindfunclet$?setupUi@Ui_NeighborJoinWidget@@QAEXPAVQWidget@@@Z$13 1003d638 f   NeighborJoinWidget.obj
 0001:0003c641       __unwindfunclet$?setupUi@Ui_NeighborJoinWidget@@QAEXPAVQWidget@@@Z$14 1003d641 f   NeighborJoinWidget.obj
 0001:0003c64c       __unwindfunclet$?setupUi@Ui_NeighborJoinWidget@@QAEXPAVQWidget@@@Z$15 1003d64c f   NeighborJoinWidget.obj
 0001:0003c655       __unwindfunclet$?setupUi@Ui_NeighborJoinWidget@@QAEXPAVQWidget@@@Z$16 1003d655 f   NeighborJoinWidget.obj
 0001:0003c660       __unwindfunclet$?setupUi@Ui_NeighborJoinWidget@@QAEXPAVQWidget@@@Z$17 1003d660 f   NeighborJoinWidget.obj
 0001:0003c669       __unwindfunclet$?setupUi@Ui_NeighborJoinWidget@@QAEXPAVQWidget@@@Z$18 1003d669 f   NeighborJoinWidget.obj
 0001:0003c674       __unwindfunclet$?setupUi@Ui_NeighborJoinWidget@@QAEXPAVQWidget@@@Z$19 1003d674 f   NeighborJoinWidget.obj
 0001:0003c67d       __unwindfunclet$?setupUi@Ui_NeighborJoinWidget@@QAEXPAVQWidget@@@Z$20 1003d67d f   NeighborJoinWidget.obj
 0001:0003c688       __unwindfunclet$?setupUi@Ui_NeighborJoinWidget@@QAEXPAVQWidget@@@Z$21 1003d688 f   NeighborJoinWidget.obj
 0001:0003c691       __unwindfunclet$?setupUi@Ui_NeighborJoinWidget@@QAEXPAVQWidget@@@Z$22 1003d691 f   NeighborJoinWidget.obj
 0001:0003c69c       __unwindfunclet$?setupUi@Ui_NeighborJoinWidget@@QAEXPAVQWidget@@@Z$23 1003d69c f   NeighborJoinWidget.obj
 0001:0003c6a5       __unwindfunclet$?setupUi@Ui_NeighborJoinWidget@@QAEXPAVQWidget@@@Z$24 1003d6a5 f   NeighborJoinWidget.obj
 0001:0003c6b0       __unwindfunclet$?setupUi@Ui_NeighborJoinWidget@@QAEXPAVQWidget@@@Z$25 1003d6b0 f   NeighborJoinWidget.obj
 0001:0003c6b9       __unwindfunclet$?setupUi@Ui_NeighborJoinWidget@@QAEXPAVQWidget@@@Z$26 1003d6b9 f   NeighborJoinWidget.obj
 0001:0003c6c4       __unwindfunclet$?setupUi@Ui_NeighborJoinWidget@@QAEXPAVQWidget@@@Z$27 1003d6c4 f   NeighborJoinWidget.obj
 0001:0003c6cd       __unwindfunclet$?setupUi@Ui_NeighborJoinWidget@@QAEXPAVQWidget@@@Z$28 1003d6cd f   NeighborJoinWidget.obj
 0001:0003c6d8       __unwindfunclet$?setupUi@Ui_NeighborJoinWidget@@QAEXPAVQWidget@@@Z$29 1003d6d8 f   NeighborJoinWidget.obj
 0001:0003c6e1       __unwindfunclet$?setupUi@Ui_NeighborJoinWidget@@QAEXPAVQWidget@@@Z$30 1003d6e1 f   NeighborJoinWidget.obj
 0001:0003c6ec       __unwindfunclet$?setupUi@Ui_NeighborJoinWidget@@QAEXPAVQWidget@@@Z$31 1003d6ec f   NeighborJoinWidget.obj
 0001:0003c6f5       __unwindfunclet$?setupUi@Ui_NeighborJoinWidget@@QAEXPAVQWidget@@@Z$32 1003d6f5 f   NeighborJoinWidget.obj
 0001:0003c700       __unwindfunclet$?setupUi@Ui_NeighborJoinWidget@@QAEXPAVQWidget@@@Z$33 1003d700 f   NeighborJoinWidget.obj
 0001:0003c709       __unwindfunclet$?setupUi@Ui_NeighborJoinWidget@@QAEXPAVQWidget@@@Z$34 1003d709 f   NeighborJoinWidget.obj
 0001:0003c714       __unwindfunclet$?setupUi@Ui_NeighborJoinWidget@@QAEXPAVQWidget@@@Z$35 1003d714 f   NeighborJoinWidget.obj
 0001:0003c71d       __unwindfunclet$?setupUi@Ui_NeighborJoinWidget@@QAEXPAVQWidget@@@Z$36 1003d71d f   NeighborJoinWidget.obj
 0001:0003c728       __unwindfunclet$?setupUi@Ui_NeighborJoinWidget@@QAEXPAVQWidget@@@Z$37 1003d728 f   NeighborJoinWidget.obj
 0001:0003c731       __unwindfunclet$?setupUi@Ui_NeighborJoinWidget@@QAEXPAVQWidget@@@Z$38 1003d731 f   NeighborJoinWidget.obj
 0001:0003c73c       __unwindfunclet$?setupUi@Ui_NeighborJoinWidget@@QAEXPAVQWidget@@@Z$39 1003d73c f   NeighborJoinWidget.obj
 0001:0003c745       __unwindfunclet$?setupUi@Ui_NeighborJoinWidget@@QAEXPAVQWidget@@@Z$40 1003d745 f   NeighborJoinWidget.obj
 0001:0003c750       __unwindfunclet$?setupUi@Ui_NeighborJoinWidget@@QAEXPAVQWidget@@@Z$41 1003d750 f   NeighborJoinWidget.obj
 0001:0003c759       __unwindfunclet$?setupUi@Ui_NeighborJoinWidget@@QAEXPAVQWidget@@@Z$42 1003d759 f   NeighborJoinWidget.obj
 0001:0003c764       __unwindfunclet$?setupUi@Ui_NeighborJoinWidget@@QAEXPAVQWidget@@@Z$43 1003d764 f   NeighborJoinWidget.obj
 0001:0003c76d       __unwindfunclet$?setupUi@Ui_NeighborJoinWidget@@QAEXPAVQWidget@@@Z$44 1003d76d f   NeighborJoinWidget.obj
 0001:0003c778       __unwindfunclet$?setupUi@Ui_NeighborJoinWidget@@QAEXPAVQWidget@@@Z$45 1003d778 f   NeighborJoinWidget.obj
 0001:0003c781       __unwindfunclet$?setupUi@Ui_NeighborJoinWidget@@QAEXPAVQWidget@@@Z$46 1003d781 f   NeighborJoinWidget.obj
 0001:0003c78c       __unwindfunclet$?setupUi@Ui_NeighborJoinWidget@@QAEXPAVQWidget@@@Z$47 1003d78c f   NeighborJoinWidget.obj
 0001:0003c795       __unwindfunclet$?setupUi@Ui_NeighborJoinWidget@@QAEXPAVQWidget@@@Z$48 1003d795 f   NeighborJoinWidget.obj
 0001:0003c7a0       __unwindfunclet$?setupUi@Ui_NeighborJoinWidget@@QAEXPAVQWidget@@@Z$49 1003d7a0 f   NeighborJoinWidget.obj
 0001:0003c7a9       __unwindfunclet$?setupUi@Ui_NeighborJoinWidget@@QAEXPAVQWidget@@@Z$50 1003d7a9 f   NeighborJoinWidget.obj
 0001:0003c7b4       __unwindfunclet$?setupUi@Ui_NeighborJoinWidget@@QAEXPAVQWidget@@@Z$51 1003d7b4 f   NeighborJoinWidget.obj
 0001:0003c7bd       __unwindfunclet$?setupUi@Ui_NeighborJoinWidget@@QAEXPAVQWidget@@@Z$52 1003d7bd f   NeighborJoinWidget.obj
 0001:0003c7c8       __unwindfunclet$?setupUi@Ui_NeighborJoinWidget@@QAEXPAVQWidget@@@Z$53 1003d7c8 f   NeighborJoinWidget.obj
 0001:0003c7d1       __unwindfunclet$?setupUi@Ui_NeighborJoinWidget@@QAEXPAVQWidget@@@Z$54 1003d7d1 f   NeighborJoinWidget.obj
 0001:0003c7dc       __unwindfunclet$?setupUi@Ui_NeighborJoinWidget@@QAEXPAVQWidget@@@Z$55 1003d7dc f   NeighborJoinWidget.obj
 0001:0003c7e5       __unwindfunclet$?setupUi@Ui_NeighborJoinWidget@@QAEXPAVQWidget@@@Z$56 1003d7e5 f   NeighborJoinWidget.obj
 0001:0003c7f0       __unwindfunclet$?setupUi@Ui_NeighborJoinWidget@@QAEXPAVQWidget@@@Z$57 1003d7f0 f   NeighborJoinWidget.obj
 0001:0003c7f9       __unwindfunclet$?setupUi@Ui_NeighborJoinWidget@@QAEXPAVQWidget@@@Z$58 1003d7f9 f   NeighborJoinWidget.obj
 0001:0003c804       __unwindfunclet$?setupUi@Ui_NeighborJoinWidget@@QAEXPAVQWidget@@@Z$59 1003d804 f   NeighborJoinWidget.obj
 0001:0003c80d       __unwindfunclet$?setupUi@Ui_NeighborJoinWidget@@QAEXPAVQWidget@@@Z$60 1003d80d f   NeighborJoinWidget.obj
 0001:0003c818       __unwindfunclet$?setupUi@Ui_NeighborJoinWidget@@QAEXPAVQWidget@@@Z$61 1003d818 f   NeighborJoinWidget.obj
 0001:0003c821       __unwindfunclet$?setupUi@Ui_NeighborJoinWidget@@QAEXPAVQWidget@@@Z$62 1003d821 f   NeighborJoinWidget.obj
 0001:0003c82c       __unwindfunclet$?setupUi@Ui_NeighborJoinWidget@@QAEXPAVQWidget@@@Z$63 1003d82c f   NeighborJoinWidget.obj
 0001:0003c835       __unwindfunclet$?setupUi@Ui_NeighborJoinWidget@@QAEXPAVQWidget@@@Z$64 1003d835 f   NeighborJoinWidget.obj
 0001:0003c840       __unwindfunclet$?setupUi@Ui_NeighborJoinWidget@@QAEXPAVQWidget@@@Z$65 1003d840 f   NeighborJoinWidget.obj
 0001:0003c849       __unwindfunclet$?setupUi@Ui_NeighborJoinWidget@@QAEXPAVQWidget@@@Z$66 1003d849 f   NeighborJoinWidget.obj
 0001:0003c854       __unwindfunclet$?setupUi@Ui_NeighborJoinWidget@@QAEXPAVQWidget@@@Z$67 1003d854 f   NeighborJoinWidget.obj
 0001:0003c85d       __unwindfunclet$?setupUi@Ui_NeighborJoinWidget@@QAEXPAVQWidget@@@Z$68 1003d85d f   NeighborJoinWidget.obj
 0001:0003c868       __unwindfunclet$?setupUi@Ui_NeighborJoinWidget@@QAEXPAVQWidget@@@Z$69 1003d868 f   NeighborJoinWidget.obj
 0001:0003c871       __unwindfunclet$?setupUi@Ui_NeighborJoinWidget@@QAEXPAVQWidget@@@Z$70 1003d871 f   NeighborJoinWidget.obj
 0001:0003c87c       __unwindfunclet$?setupUi@Ui_NeighborJoinWidget@@QAEXPAVQWidget@@@Z$71 1003d87c f   NeighborJoinWidget.obj
 0001:0003c885       __unwindfunclet$?setupUi@Ui_NeighborJoinWidget@@QAEXPAVQWidget@@@Z$72 1003d885 f   NeighborJoinWidget.obj
 0001:0003c890       __unwindfunclet$?setupUi@Ui_NeighborJoinWidget@@QAEXPAVQWidget@@@Z$73 1003d890 f   NeighborJoinWidget.obj
 0001:0003c899       __unwindfunclet$?setupUi@Ui_NeighborJoinWidget@@QAEXPAVQWidget@@@Z$74 1003d899 f   NeighborJoinWidget.obj
 0001:0003c8a4       __unwindfunclet$?setupUi@Ui_NeighborJoinWidget@@QAEXPAVQWidget@@@Z$75 1003d8a4 f   NeighborJoinWidget.obj
 0001:0003c8ad       __ehhandler$?setupUi@Ui_NeighborJoinWidget@@QAEXPAVQWidget@@@Z 1003d8ad f   NeighborJoinWidget.obj
 0001:0003c8d0       __unwindfunclet$?storeSettings@NeighborJoinWidget@U2@@UAEXXZ$0 1003d8d0 f   NeighborJoinWidget.obj
 0001:0003c8d9       __unwindfunclet$?storeSettings@NeighborJoinWidget@U2@@UAEXXZ$1 1003d8d9 f   NeighborJoinWidget.obj
 0001:0003c8e2       __unwindfunclet$?storeSettings@NeighborJoinWidget@U2@@UAEXXZ$2 1003d8e2 f   NeighborJoinWidget.obj
 0001:0003c8eb       __unwindfunclet$?storeSettings@NeighborJoinWidget@U2@@UAEXXZ$3 1003d8eb f   NeighborJoinWidget.obj
 0001:0003c8f4       __unwindfunclet$?storeSettings@NeighborJoinWidget@U2@@UAEXXZ$4 1003d8f4 f   NeighborJoinWidget.obj
 0001:0003c8fd       __unwindfunclet$?storeSettings@NeighborJoinWidget@U2@@UAEXXZ$5 1003d8fd f   NeighborJoinWidget.obj
 0001:0003c906       __unwindfunclet$?storeSettings@NeighborJoinWidget@U2@@UAEXXZ$6 1003d906 f   NeighborJoinWidget.obj
 0001:0003c90f       __unwindfunclet$?storeSettings@NeighborJoinWidget@U2@@UAEXXZ$7 1003d90f f   NeighborJoinWidget.obj
 0001:0003c918       __unwindfunclet$?storeSettings@NeighborJoinWidget@U2@@UAEXXZ$8 1003d918 f   NeighborJoinWidget.obj
 0001:0003c921       __unwindfunclet$?storeSettings@NeighborJoinWidget@U2@@UAEXXZ$9 1003d921 f   NeighborJoinWidget.obj
 0001:0003c92a       __unwindfunclet$?storeSettings@NeighborJoinWidget@U2@@UAEXXZ$10 1003d92a f   NeighborJoinWidget.obj
 0001:0003c933       __unwindfunclet$?storeSettings@NeighborJoinWidget@U2@@UAEXXZ$11 1003d933 f   NeighborJoinWidget.obj
 0001:0003c93c       __unwindfunclet$?storeSettings@NeighborJoinWidget@U2@@UAEXXZ$12 1003d93c f   NeighborJoinWidget.obj
 0001:0003c945       __unwindfunclet$?storeSettings@NeighborJoinWidget@U2@@UAEXXZ$13 1003d945 f   NeighborJoinWidget.obj
 0001:0003c94e       __unwindfunclet$?storeSettings@NeighborJoinWidget@U2@@UAEXXZ$14 1003d94e f   NeighborJoinWidget.obj
 0001:0003c957       __unwindfunclet$?storeSettings@NeighborJoinWidget@U2@@UAEXXZ$15 1003d957 f   NeighborJoinWidget.obj
 0001:0003c960       __unwindfunclet$?storeSettings@NeighborJoinWidget@U2@@UAEXXZ$16 1003d960 f   NeighborJoinWidget.obj
 0001:0003c969       __unwindfunclet$?storeSettings@NeighborJoinWidget@U2@@UAEXXZ$17 1003d969 f   NeighborJoinWidget.obj
 0001:0003c972       __unwindfunclet$?storeSettings@NeighborJoinWidget@U2@@UAEXXZ$18 1003d972 f   NeighborJoinWidget.obj
 0001:0003c97b       __unwindfunclet$?storeSettings@NeighborJoinWidget@U2@@UAEXXZ$19 1003d97b f   NeighborJoinWidget.obj
 0001:0003c984       __unwindfunclet$?storeSettings@NeighborJoinWidget@U2@@UAEXXZ$20 1003d984 f   NeighborJoinWidget.obj
 0001:0003c98d       __unwindfunclet$?storeSettings@NeighborJoinWidget@U2@@UAEXXZ$21 1003d98d f   NeighborJoinWidget.obj
 0001:0003c996       __unwindfunclet$?storeSettings@NeighborJoinWidget@U2@@UAEXXZ$22 1003d996 f   NeighborJoinWidget.obj
 0001:0003c99f       __unwindfunclet$?storeSettings@NeighborJoinWidget@U2@@UAEXXZ$23 1003d99f f   NeighborJoinWidget.obj
 0001:0003c9a8       __unwindfunclet$?storeSettings@NeighborJoinWidget@U2@@UAEXXZ$24 1003d9a8 f   NeighborJoinWidget.obj
 0001:0003c9b1       __unwindfunclet$?storeSettings@NeighborJoinWidget@U2@@UAEXXZ$25 1003d9b1 f   NeighborJoinWidget.obj
 0001:0003c9ba       __unwindfunclet$?storeSettings@NeighborJoinWidget@U2@@UAEXXZ$26 1003d9ba f   NeighborJoinWidget.obj
 0001:0003c9c3       __unwindfunclet$?storeSettings@NeighborJoinWidget@U2@@UAEXXZ$27 1003d9c3 f   NeighborJoinWidget.obj
 0001:0003c9cc       __unwindfunclet$?storeSettings@NeighborJoinWidget@U2@@UAEXXZ$28 1003d9cc f   NeighborJoinWidget.obj
 0001:0003c9d5       __ehhandler$?storeSettings@NeighborJoinWidget@U2@@UAEXXZ 1003d9d5 f   NeighborJoinWidget.obj
 0001:0003c9f0       __unwindfunclet$??0?$QHashNode@VQString@@V1@@@QAE@ABVQString@@0IPAU0@@Z$0 1003d9f0 f   PhylipCmdlineTask.obj
 0001:0003c9fc       __ehhandler$??0?$QHashNode@VQString@@V1@@@QAE@ABVQString@@0IPAU0@@Z 1003d9fc f   PhylipCmdlineTask.obj
 0001:0003ca20       __ehhandler$??0?$QList@VQByteArray@@@@QAE@ABV0@@Z 1003da20 f   PhylipCmdlineTask.obj
 0001:0003ca40       __unwindfunclet$??0PhylipCmdlineTask@U2@@QAE@ABVMultipleSequenceAlignment@1@ABVCreatePhyTreeSettings@1@@Z$0 1003da40 f   PhylipCmdlineTask.obj
 0001:0003ca49       __unwindfunclet$??0PhylipCmdlineTask@U2@@QAE@ABVMultipleSequenceAlignment@1@ABVCreatePhyTreeSettings@1@@Z$1 1003da49 f   PhylipCmdlineTask.obj
 0001:0003ca58       __unwindfunclet$??0PhylipCmdlineTask@U2@@QAE@ABVMultipleSequenceAlignment@1@ABVCreatePhyTreeSettings@1@@Z$2 1003da58 f   PhylipCmdlineTask.obj
 0001:0003ca61       __unwindfunclet$??0PhylipCmdlineTask@U2@@QAE@ABVMultipleSequenceAlignment@1@ABVCreatePhyTreeSettings@1@@Z$3 1003da61 f   PhylipCmdlineTask.obj
 0001:0003ca6a       __unwindfunclet$??0PhylipCmdlineTask@U2@@QAE@ABVMultipleSequenceAlignment@1@ABVCreatePhyTreeSettings@1@@Z$4 1003da6a f   PhylipCmdlineTask.obj
 0001:0003ca79       __unwindfunclet$??0PhylipCmdlineTask@U2@@QAE@ABVMultipleSequenceAlignment@1@ABVCreatePhyTreeSettings@1@@Z$5 1003da79 f   PhylipCmdlineTask.obj
 0001:0003ca82       __ehhandler$??0PhylipCmdlineTask@U2@@QAE@ABVMultipleSequenceAlignment@1@ABVCreatePhyTreeSettings@1@@Z 1003da82 f   PhylipCmdlineTask.obj
 0001:0003caa0       __unwindfunclet$??1?$QHashNode@VQString@@V1@@@QAE@XZ$0 1003daa0 f   PhylipCmdlineTask.obj
 0001:0003caac       __ehhandler$??1?$QHashNode@VQString@@V1@@@QAE@XZ 1003daac f   PhylipCmdlineTask.obj
 0001:0003cad0       __unwindfunclet$??1PhylipCmdlineTask@U2@@UAE@XZ$0 1003dad0 f   PhylipCmdlineTask.obj
 0001:0003cad9       __unwindfunclet$??1PhylipCmdlineTask@U2@@UAE@XZ$1 1003dad9 f   PhylipCmdlineTask.obj
 0001:0003cae8       __unwindfunclet$??1PhylipCmdlineTask@U2@@UAE@XZ$2 1003dae8 f   PhylipCmdlineTask.obj
 0001:0003caf7       __ehhandler$??1PhylipCmdlineTask@U2@@UAE@XZ 1003daf7 f   PhylipCmdlineTask.obj
 0001:0003cb20       __unwindfunclet$??A?$QHash@VQString@@V1@@@QAEAAVQString@@ABV1@@Z$0 1003db20 f   PhylipCmdlineTask.obj
 0001:0003cb29       __ehhandler$??A?$QHash@VQString@@V1@@@QAEAAVQString@@ABV1@@Z 1003db29 f   PhylipCmdlineTask.obj
 0001:0003cb50       __unwindfunclet$??H@YA?BVQString@@PBDABV0@@Z$0 1003db50 f   PhylipCmdlineTask.obj
 0001:0003cb6a       __ehhandler$??H@YA?BVQString@@PBDABV0@@Z 1003db6a f   PhylipCmdlineTask.obj
 0001:0003cb90       __unwindfunclet$??_G?$QHashNode@VQString@@V1@@@QAEPAXI@Z$0 1003db90 f   PhylipCmdlineTask.obj
 0001:0003cb9c       __ehhandler$??_G?$QHashNode@VQString@@V1@@@QAEPAXI@Z 1003db9c f   PhylipCmdlineTask.obj
 0001:0003cbc0       __unwindfunclet$??_GPhylipCmdlineTask@U2@@UAEPAXI@Z$0 1003dbc0 f   PhylipCmdlineTask.obj
 0001:0003cbc9       __unwindfunclet$??_GPhylipCmdlineTask@U2@@UAEPAXI@Z$1 1003dbc9 f   PhylipCmdlineTask.obj
 0001:0003cbd8       __unwindfunclet$??_GPhylipCmdlineTask@U2@@UAEPAXI@Z$2 1003dbd8 f   PhylipCmdlineTask.obj
 0001:0003cbe7       __ehhandler$??_GPhylipCmdlineTask@U2@@UAEPAXI@Z 1003dbe7 f   PhylipCmdlineTask.obj
 0001:0003cc10       __unwindfunclet$??__EalgoLog@U2@@YAXXZ$0 1003dc10 f   PhylipCmdlineTask.obj
 0001:0003cc19       __ehhandler$??__EalgoLog@U2@@YAXXZ 1003dc19 f   PhylipCmdlineTask.obj
 0001:0003cc40       __unwindfunclet$??__EcmdLog@U2@@YAXXZ$0 1003dc40 f   PhylipCmdlineTask.obj
 0001:0003cc49       __ehhandler$??__EcmdLog@U2@@YAXXZ 1003dc49 f   PhylipCmdlineTask.obj
 0001:0003cc70       __unwindfunclet$??__EcoreLog@U2@@YAXXZ$0 1003dc70 f   PhylipCmdlineTask.obj
 0001:0003cc79       __ehhandler$??__EcoreLog@U2@@YAXXZ 1003dc79 f   PhylipCmdlineTask.obj
 0001:0003cca0       __unwindfunclet$??__EioLog@U2@@YAXXZ$0 1003dca0 f   PhylipCmdlineTask.obj
 0001:0003cca9       __ehhandler$??__EioLog@U2@@YAXXZ 1003dca9 f   PhylipCmdlineTask.obj
 0001:0003ccd0       __unwindfunclet$??__EperfLog@U2@@YAXXZ$0 1003dcd0 f   PhylipCmdlineTask.obj
 0001:0003ccd9       __ehhandler$??__EperfLog@U2@@YAXXZ 1003dcd9 f   PhylipCmdlineTask.obj
 0001:0003cd00       __unwindfunclet$??__EscriptLog@U2@@YAXXZ$0 1003dd00 f   PhylipCmdlineTask.obj
 0001:0003cd09       __ehhandler$??__EscriptLog@U2@@YAXXZ 1003dd09 f   PhylipCmdlineTask.obj
 0001:0003cd30       __unwindfunclet$??__EtaskLog@U2@@YAXXZ$0 1003dd30 f   PhylipCmdlineTask.obj
 0001:0003cd39       __ehhandler$??__EtaskLog@U2@@YAXXZ 1003dd39 f   PhylipCmdlineTask.obj
 0001:0003cd60       __unwindfunclet$??__EuiLog@U2@@YAXXZ$0 1003dd60 f   PhylipCmdlineTask.obj
 0001:0003cd69       __ehhandler$??__EuiLog@U2@@YAXXZ 1003dd69 f   PhylipCmdlineTask.obj
 0001:0003cd90       __unwindfunclet$??__EuserActLog@U2@@YAXXZ$0 1003dd90 f   PhylipCmdlineTask.obj
 0001:0003cd99       __ehhandler$??__EuserActLog@U2@@YAXXZ 1003dd99 f   PhylipCmdlineTask.obj
 0001:0003cdc0       __ehhandler$?append@?$QList@PAVGObject@U2@@@@QAEXABQAVGObject@U2@@@Z 1003ddc0 f   PhylipCmdlineTask.obj
 0001:0003cde0       __unwindfunclet$?createCmdlineTask@PhylipCmdlineTask@U2@@AAEXXZ$0 1003dde0 f   PhylipCmdlineTask.obj
 0001:0003cde9       __unwindfunclet$?createCmdlineTask@PhylipCmdlineTask@U2@@AAEXXZ$1 1003dde9 f   PhylipCmdlineTask.obj
 0001:0003cdf2       __unwindfunclet$?createCmdlineTask@PhylipCmdlineTask@U2@@AAEXXZ$2 1003ddf2 f   PhylipCmdlineTask.obj
 0001:0003cdfb       __unwindfunclet$?createCmdlineTask@PhylipCmdlineTask@U2@@AAEXXZ$3 1003ddfb f   PhylipCmdlineTask.obj
 0001:0003ce04       __unwindfunclet$?createCmdlineTask@PhylipCmdlineTask@U2@@AAEXXZ$4 1003de04 f   PhylipCmdlineTask.obj
 0001:0003ce0d       __unwindfunclet$?createCmdlineTask@PhylipCmdlineTask@U2@@AAEXXZ$5 1003de0d f   PhylipCmdlineTask.obj
 0001:0003ce16       __unwindfunclet$?createCmdlineTask@PhylipCmdlineTask@U2@@AAEXXZ$6 1003de16 f   PhylipCmdlineTask.obj
 0001:0003ce1f       __unwindfunclet$?createCmdlineTask@PhylipCmdlineTask@U2@@AAEXXZ$7 1003de1f f   PhylipCmdlineTask.obj
 0001:0003ce28       __unwindfunclet$?createCmdlineTask@PhylipCmdlineTask@U2@@AAEXXZ$8 1003de28 f   PhylipCmdlineTask.obj
 0001:0003ce31       __unwindfunclet$?createCmdlineTask@PhylipCmdlineTask@U2@@AAEXXZ$9 1003de31 f   PhylipCmdlineTask.obj
 0001:0003ce3a       __unwindfunclet$?createCmdlineTask@PhylipCmdlineTask@U2@@AAEXXZ$10 1003de3a f   PhylipCmdlineTask.obj
 0001:0003ce43       __unwindfunclet$?createCmdlineTask@PhylipCmdlineTask@U2@@AAEXXZ$11 1003de43 f   PhylipCmdlineTask.obj
 0001:0003ce4c       __unwindfunclet$?createCmdlineTask@PhylipCmdlineTask@U2@@AAEXXZ$12 1003de4c f   PhylipCmdlineTask.obj
 0001:0003ce55       __unwindfunclet$?createCmdlineTask@PhylipCmdlineTask@U2@@AAEXXZ$13 1003de55 f   PhylipCmdlineTask.obj
 0001:0003ce5e       __unwindfunclet$?createCmdlineTask@PhylipCmdlineTask@U2@@AAEXXZ$14 1003de5e f   PhylipCmdlineTask.obj
 0001:0003ce67       __unwindfunclet$?createCmdlineTask@PhylipCmdlineTask@U2@@AAEXXZ$15 1003de67 f   PhylipCmdlineTask.obj
 0001:0003ce70       __unwindfunclet$?createCmdlineTask@PhylipCmdlineTask@U2@@AAEXXZ$16 1003de70 f   PhylipCmdlineTask.obj
 0001:0003ce79       __unwindfunclet$?createCmdlineTask@PhylipCmdlineTask@U2@@AAEXXZ$17 1003de79 f   PhylipCmdlineTask.obj
 0001:0003ce82       __unwindfunclet$?createCmdlineTask@PhylipCmdlineTask@U2@@AAEXXZ$18 1003de82 f   PhylipCmdlineTask.obj
 0001:0003ce8b       __unwindfunclet$?createCmdlineTask@PhylipCmdlineTask@U2@@AAEXXZ$19 1003de8b f   PhylipCmdlineTask.obj
 0001:0003ce94       __unwindfunclet$?createCmdlineTask@PhylipCmdlineTask@U2@@AAEXXZ$20 1003de94 f   PhylipCmdlineTask.obj
 0001:0003ce9d       __unwindfunclet$?createCmdlineTask@PhylipCmdlineTask@U2@@AAEXXZ$21 1003de9d f   PhylipCmdlineTask.obj
 0001:0003cea6       __unwindfunclet$?createCmdlineTask@PhylipCmdlineTask@U2@@AAEXXZ$22 1003dea6 f   PhylipCmdlineTask.obj
 0001:0003ceb1       __ehhandler$?createCmdlineTask@PhylipCmdlineTask@U2@@AAEXXZ 1003deb1 f   PhylipCmdlineTask.obj
 0001:0003ced0       __unwindfunclet$?createNode@?$QHash@VQString@@V1@@@AAEPAU?$QHashNode@VQString@@V1@@@IABVQString@@0PAPAU2@@Z$0 1003ded0 f   PhylipCmdlineTask.obj
 0001:0003cee1       __unwindfunclet$?createNode@?$QHash@VQString@@V1@@@AAEPAU?$QHashNode@VQString@@V1@@@IABVQString@@0PAPAU2@@Z$1 1003dee1 f   PhylipCmdlineTask.obj
 0001:0003ceed       __ehhandler$?createNode@?$QHash@VQString@@V1@@@AAEPAU?$QHashNode@VQString@@V1@@@IABVQString@@0PAPAU2@@Z 1003deed f   PhylipCmdlineTask.obj
 0001:0003cf10       __unwindfunclet$?deleteNode2@?$QHash@VQString@@V1@@@CAXPAUNode@QHashData@@@Z$0 1003df10 f   PhylipCmdlineTask.obj
 0001:0003cf1c       __ehhandler$?deleteNode2@?$QHash@VQString@@V1@@@CAXPAUNode@QHashData@@@Z 1003df1c f   PhylipCmdlineTask.obj
 0001:0003cf40       __ehhandler$?detach_helper@?$QList@VQByteArray@@@@AAEXH@Z 1003df40 f   PhylipCmdlineTask.obj
 0001:0003cf60       __ehhandler$?detach_helper_grow@?$QList@PAVGObject@U2@@@@AAEPAUNode@1@HH@Z 1003df60 f   PhylipCmdlineTask.obj
 0001:0003cf80       __unwindfunclet$?duplicateNode@?$QHash@VQString@@V1@@@CAXPAUNode@QHashData@@PAX@Z$0 1003df80 f   PhylipCmdlineTask.obj
 0001:0003cf91       __unwindfunclet$?duplicateNode@?$QHash@VQString@@V1@@@CAXPAUNode@QHashData@@PAX@Z$1 1003df91 f   PhylipCmdlineTask.obj
 0001:0003cf9d       __ehhandler$?duplicateNode@?$QHash@VQString@@V1@@@CAXPAUNode@QHashData@@PAX@Z 1003df9d f   PhylipCmdlineTask.obj
 0001:0003cfc0       __unwindfunclet$?node_copy@?$QList@VQByteArray@@@@AAEXPAUNode@1@00@Z$5 1003dfc0 f   PhylipCmdlineTask.obj
 0001:0003cfd1       __ehhandler$?node_copy@?$QList@VQByteArray@@@@AAEXPAUNode@1@00@Z 1003dfd1 f   PhylipCmdlineTask.obj
 0001:0003d000       __unwindfunclet$?prepareTempDbi@PhylipCmdlineTask@U2@@AAEXXZ$0 1003e000 f   PhylipCmdlineTask.obj
 0001:0003d009       __unwindfunclet$?prepareTempDbi@PhylipCmdlineTask@U2@@AAEXXZ$1 1003e009 f   PhylipCmdlineTask.obj
 0001:0003d012       __unwindfunclet$?prepareTempDbi@PhylipCmdlineTask@U2@@AAEXXZ$2 1003e012 f   PhylipCmdlineTask.obj
 0001:0003d01b       __unwindfunclet$?prepareTempDbi@PhylipCmdlineTask@U2@@AAEXXZ$3 1003e01b f   PhylipCmdlineTask.obj
 0001:0003d024       __unwindfunclet$?prepareTempDbi@PhylipCmdlineTask@U2@@AAEXXZ$4 1003e024 f   PhylipCmdlineTask.obj
 0001:0003d02d       __unwindfunclet$?prepareTempDbi@PhylipCmdlineTask@U2@@AAEXXZ$5 1003e02d f   PhylipCmdlineTask.obj
 0001:0003d036       __unwindfunclet$?prepareTempDbi@PhylipCmdlineTask@U2@@AAEXXZ$6 1003e036 f   PhylipCmdlineTask.obj
 0001:0003d03f       __unwindfunclet$?prepareTempDbi@PhylipCmdlineTask@U2@@AAEXXZ$7 1003e03f f   PhylipCmdlineTask.obj
 0001:0003d047       __ehhandler$?prepareTempDbi@PhylipCmdlineTask@U2@@AAEXXZ 1003e047 f   PhylipCmdlineTask.obj
 0001:0003d070       __unwindfunclet$?report@PhylipCmdlineTask@U2@@UAE?AW4ReportResult@Task@2@XZ$0 1003e070 f   PhylipCmdlineTask.obj
 0001:0003d078       __unwindfunclet$?report@PhylipCmdlineTask@U2@@UAE?AW4ReportResult@Task@2@XZ$1 1003e078 f   PhylipCmdlineTask.obj
 0001:0003d081       __unwindfunclet$?report@PhylipCmdlineTask@U2@@UAE?AW4ReportResult@Task@2@XZ$2 1003e081 f   PhylipCmdlineTask.obj
 0001:0003d08c       __unwindfunclet$?report@PhylipCmdlineTask@U2@@UAE?AW4ReportResult@Task@2@XZ$3 1003e08c f   PhylipCmdlineTask.obj
 0001:0003d0a6       __unwindfunclet$?report@PhylipCmdlineTask@U2@@UAE?AW4ReportResult@Task@2@XZ$4 1003e0a6 f   PhylipCmdlineTask.obj
 0001:0003d0bf       __unwindfunclet$?report@PhylipCmdlineTask@U2@@UAE?AW4ReportResult@Task@2@XZ$5 1003e0bf f   PhylipCmdlineTask.obj
 0001:0003d0d9       __ehhandler$?report@PhylipCmdlineTask@U2@@UAE?AW4ReportResult@Task@2@XZ 1003e0d9 f   PhylipCmdlineTask.obj
 0001:0003d100       __ehhandler$??0?$QList@PAVXMLTestFactory@U2@@@@QAE@ABV0@@Z 1003e100 f   PhylipPlugin.obj
 0001:0003d120       __unwindfunclet$??0PhylipPlugin@U2@@QAE@XZ$0 1003e120 f   PhylipPlugin.obj
 0001:0003d129       __unwindfunclet$??0PhylipPlugin@U2@@QAE@XZ$1 1003e129 f   PhylipPlugin.obj
 0001:0003d132       __unwindfunclet$??0PhylipPlugin@U2@@QAE@XZ$2 1003e132 f   PhylipPlugin.obj
 0001:0003d13b       __unwindfunclet$??0PhylipPlugin@U2@@QAE@XZ$3 1003e13b f   PhylipPlugin.obj
 0001:0003d144       __unwindfunclet$??0PhylipPlugin@U2@@QAE@XZ$4 1003e144 f   PhylipPlugin.obj
 0001:0003d14f       __unwindfunclet$??0PhylipPlugin@U2@@QAE@XZ$6 1003e14f f   PhylipPlugin.obj
 0001:0003d157       __ehhandler$??0PhylipPlugin@U2@@QAE@XZ 1003e157 f   PhylipPlugin.obj
 0001:0003d180       __unwindfunclet$??1?$GAutoDeleteList@VXMLTestFactory@U2@@@U2@@UAE@XZ$0 1003e180 f   PhylipPlugin.obj
 0001:0003d189       __unwindfunclet$??1?$GAutoDeleteList@VXMLTestFactory@U2@@@U2@@UAE@XZ$1 1003e189 f   PhylipPlugin.obj
 0001:0003d194       __ehhandler$??1?$GAutoDeleteList@VXMLTestFactory@U2@@@U2@@UAE@XZ 1003e194 f   PhylipPlugin.obj
 0001:0003d1b0       __unwindfunclet$??__EalgoLog@U2@@YAXXZ$0 1003e1b0 f   PhylipPlugin.obj
 0001:0003d1b9       __ehhandler$??__EalgoLog@U2@@YAXXZ 1003e1b9 f   PhylipPlugin.obj
 0001:0003d1e0       __unwindfunclet$??__EcmdLog@U2@@YAXXZ$0 1003e1e0 f   PhylipPlugin.obj
 0001:0003d1e9       __ehhandler$??__EcmdLog@U2@@YAXXZ 1003e1e9 f   PhylipPlugin.obj
 0001:0003d210       __unwindfunclet$??__EcoreLog@U2@@YAXXZ$0 1003e210 f   PhylipPlugin.obj
 0001:0003d219       __ehhandler$??__EcoreLog@U2@@YAXXZ 1003e219 f   PhylipPlugin.obj
 0001:0003d240       __unwindfunclet$??__EioLog@U2@@YAXXZ$0 1003e240 f   PhylipPlugin.obj
 0001:0003d249       __ehhandler$??__EioLog@U2@@YAXXZ 1003e249 f   PhylipPlugin.obj
 0001:0003d270       __unwindfunclet$??__EperfLog@U2@@YAXXZ$0 1003e270 f   PhylipPlugin.obj
 0001:0003d279       __ehhandler$??__EperfLog@U2@@YAXXZ 1003e279 f   PhylipPlugin.obj
 0001:0003d2a0       __unwindfunclet$??__EscriptLog@U2@@YAXXZ$0 1003e2a0 f   PhylipPlugin.obj
 0001:0003d2a9       __ehhandler$??__EscriptLog@U2@@YAXXZ 1003e2a9 f   PhylipPlugin.obj
 0001:0003d2d0       __unwindfunclet$??__EtaskLog@U2@@YAXXZ$0 1003e2d0 f   PhylipPlugin.obj
 0001:0003d2d9       __ehhandler$??__EtaskLog@U2@@YAXXZ 1003e2d9 f   PhylipPlugin.obj
 0001:0003d300       __unwindfunclet$??__EuiLog@U2@@YAXXZ$0 1003e300 f   PhylipPlugin.obj
 0001:0003d309       __ehhandler$??__EuiLog@U2@@YAXXZ 1003e309 f   PhylipPlugin.obj
 0001:0003d330       __unwindfunclet$??__EuserActLog@U2@@YAXXZ$0 1003e330 f   PhylipPlugin.obj
 0001:0003d339       __ehhandler$??__EuserActLog@U2@@YAXXZ 1003e339 f   PhylipPlugin.obj
 0001:0003d360       __unwindfunclet$?fetchSettings@?A0xabc90af7@U2@@YA?AVCreatePhyTreeSettings@2@XZ$0 1003e360 f   PhylipPlugin.obj
 0001:0003d37a       __unwindfunclet$?fetchSettings@?A0xabc90af7@U2@@YA?AVCreatePhyTreeSettings@2@XZ$1 1003e37a f   PhylipPlugin.obj
 0001:0003d383       __unwindfunclet$?fetchSettings@?A0xabc90af7@U2@@YA?AVCreatePhyTreeSettings@2@XZ$2 1003e383 f   PhylipPlugin.obj
 0001:0003d38c       __unwindfunclet$?fetchSettings@?A0xabc90af7@U2@@YA?AVCreatePhyTreeSettings@2@XZ$3 1003e38c f   PhylipPlugin.obj
 0001:0003d395       __unwindfunclet$?fetchSettings@?A0xabc90af7@U2@@YA?AVCreatePhyTreeSettings@2@XZ$4 1003e395 f   PhylipPlugin.obj
 0001:0003d39e       __unwindfunclet$?fetchSettings@?A0xabc90af7@U2@@YA?AVCreatePhyTreeSettings@2@XZ$5 1003e39e f   PhylipPlugin.obj
 0001:0003d3a7       __unwindfunclet$?fetchSettings@?A0xabc90af7@U2@@YA?AVCreatePhyTreeSettings@2@XZ$6 1003e3a7 f   PhylipPlugin.obj
 0001:0003d3b0       __unwindfunclet$?fetchSettings@?A0xabc90af7@U2@@YA?AVCreatePhyTreeSettings@2@XZ$7 1003e3b0 f   PhylipPlugin.obj
 0001:0003d3b9       __unwindfunclet$?fetchSettings@?A0xabc90af7@U2@@YA?AVCreatePhyTreeSettings@2@XZ$8 1003e3b9 f   PhylipPlugin.obj
 0001:0003d3c2       __unwindfunclet$?fetchSettings@?A0xabc90af7@U2@@YA?AVCreatePhyTreeSettings@2@XZ$9 1003e3c2 f   PhylipPlugin.obj
 0001:0003d3cb       __ehhandler$?fetchSettings@?A0xabc90af7@U2@@YA?AVCreatePhyTreeSettings@2@XZ 1003e3cb f   PhylipPlugin.obj
 0001:0003d3f0       __unwindfunclet$?processCmdlineOptions@PhylipPlugin@U2@@AAEXXZ$0 1003e3f0 f   PhylipPlugin.obj
 0001:0003d3fc       __unwindfunclet$?processCmdlineOptions@PhylipPlugin@U2@@AAEXXZ$1 1003e3fc f   PhylipPlugin.obj
 0001:0003d405       __unwindfunclet$?processCmdlineOptions@PhylipPlugin@U2@@AAEXXZ$2 1003e405 f   PhylipPlugin.obj
 0001:0003d40e       __unwindfunclet$?processCmdlineOptions@PhylipPlugin@U2@@AAEXXZ$3 1003e40e f   PhylipPlugin.obj
 0001:0003d417       __unwindfunclet$?processCmdlineOptions@PhylipPlugin@U2@@AAEXXZ$4 1003e417 f   PhylipPlugin.obj
 0001:0003d420       __unwindfunclet$?processCmdlineOptions@PhylipPlugin@U2@@AAEXXZ$5 1003e420 f   PhylipPlugin.obj
 0001:0003d429       __unwindfunclet$?processCmdlineOptions@PhylipPlugin@U2@@AAEXXZ$6 1003e429 f   PhylipPlugin.obj
 0001:0003d432       __unwindfunclet$?processCmdlineOptions@PhylipPlugin@U2@@AAEXXZ$7 1003e432 f   PhylipPlugin.obj
 0001:0003d43b       __unwindfunclet$?processCmdlineOptions@PhylipPlugin@U2@@AAEXXZ$8 1003e43b f   PhylipPlugin.obj
 0001:0003d446       __unwindfunclet$?processCmdlineOptions@PhylipPlugin@U2@@AAEXXZ$9 1003e446 f   PhylipPlugin.obj
 0001:0003d460       __unwindfunclet$?processCmdlineOptions@PhylipPlugin@U2@@AAEXXZ$10 1003e460 f   PhylipPlugin.obj
 0001:0003d46b       __ehhandler$?processCmdlineOptions@PhylipPlugin@U2@@AAEXXZ 1003e46b f   PhylipPlugin.obj
 0001:0003d490       __unwindfunclet$??0GTest_NeighborJoin@U2@@QAE@PAVXMLTestFormat@1@ABVQString@@PAVGTest@1@PBVGTestEnvironment@1@ABV?$QList@PAVGTest@U2@@@@ABVQDomElement@@@Z$0 1003e490 f   PhylipPluginTests.obj
 0001:0003d499       __unwindfunclet$??0GTest_NeighborJoin@U2@@QAE@PAVXMLTestFormat@1@ABVQString@@PAVGTest@1@PBVGTestEnvironment@1@ABV?$QList@PAVGTest@U2@@@@ABVQDomElement@@@Z$1 1003e499 f   PhylipPluginTests.obj
 0001:0003d4a8       __unwindfunclet$??0GTest_NeighborJoin@U2@@QAE@PAVXMLTestFormat@1@ABVQString@@PAVGTest@1@PBVGTestEnvironment@1@ABV?$QList@PAVGTest@U2@@@@ABVQDomElement@@@Z$2 1003e4a8 f   PhylipPluginTests.obj
 0001:0003d4b7       __ehhandler$??0GTest_NeighborJoin@U2@@QAE@PAVXMLTestFormat@1@ABVQString@@PAVGTest@1@PBVGTestEnvironment@1@ABV?$QList@PAVGTest@U2@@@@ABVQDomElement@@@Z 1003e4b7 f   PhylipPluginTests.obj
 0001:0003d4e0       __unwindfunclet$??0GTest_NeighborJoinFactory@GTest_NeighborJoin@U2@@QAE@XZ$0 1003e4e0 f   PhylipPluginTests.obj
 0001:0003d4e9       __unwindfunclet$??0GTest_NeighborJoinFactory@GTest_NeighborJoin@U2@@QAE@XZ$1 1003e4e9 f   PhylipPluginTests.obj
 0001:0003d4f2       __ehhandler$??0GTest_NeighborJoinFactory@GTest_NeighborJoin@U2@@QAE@XZ 1003e4f2 f   PhylipPluginTests.obj
 0001:0003d510       __unwindfunclet$??1GTest_NeighborJoin@U2@@UAE@XZ$0 1003e510 f   PhylipPluginTests.obj
 0001:0003d519       __unwindfunclet$??1GTest_NeighborJoin@U2@@UAE@XZ$1 1003e519 f   PhylipPluginTests.obj
 0001:0003d528       __ehhandler$??1GTest_NeighborJoin@U2@@UAE@XZ 1003e528 f   PhylipPluginTests.obj
 0001:0003d550       __unwindfunclet$??_GGTest_NeighborJoin@U2@@UAEPAXI@Z$0 1003e550 f   PhylipPluginTests.obj
 0001:0003d559       __unwindfunclet$??_GGTest_NeighborJoin@U2@@UAEPAXI@Z$1 1003e559 f   PhylipPluginTests.obj
 0001:0003d568       __ehhandler$??_GGTest_NeighborJoin@U2@@UAEPAXI@Z 1003e568 f   PhylipPluginTests.obj
 0001:0003d590       __unwindfunclet$??__EalgoLog@U2@@YAXXZ$0 1003e590 f   PhylipPluginTests.obj
 0001:0003d599       __ehhandler$??__EalgoLog@U2@@YAXXZ 1003e599 f   PhylipPluginTests.obj
 0001:0003d5c0       __unwindfunclet$??__EcmdLog@U2@@YAXXZ$0 1003e5c0 f   PhylipPluginTests.obj
 0001:0003d5c9       __ehhandler$??__EcmdLog@U2@@YAXXZ 1003e5c9 f   PhylipPluginTests.obj
 0001:0003d5f0       __unwindfunclet$??__EcoreLog@U2@@YAXXZ$0 1003e5f0 f   PhylipPluginTests.obj
 0001:0003d5f9       __ehhandler$??__EcoreLog@U2@@YAXXZ 1003e5f9 f   PhylipPluginTests.obj
 0001:0003d620       __unwindfunclet$??__EioLog@U2@@YAXXZ$0 1003e620 f   PhylipPluginTests.obj
 0001:0003d629       __ehhandler$??__EioLog@U2@@YAXXZ 1003e629 f   PhylipPluginTests.obj
 0001:0003d650       __unwindfunclet$??__EperfLog@U2@@YAXXZ$0 1003e650 f   PhylipPluginTests.obj
 0001:0003d659       __ehhandler$??__EperfLog@U2@@YAXXZ 1003e659 f   PhylipPluginTests.obj
 0001:0003d680       __unwindfunclet$??__EscriptLog@U2@@YAXXZ$0 1003e680 f   PhylipPluginTests.obj
 0001:0003d689       __ehhandler$??__EscriptLog@U2@@YAXXZ 1003e689 f   PhylipPluginTests.obj
 0001:0003d6b0       __unwindfunclet$??__EtaskLog@U2@@YAXXZ$0 1003e6b0 f   PhylipPluginTests.obj
 0001:0003d6b9       __ehhandler$??__EtaskLog@U2@@YAXXZ 1003e6b9 f   PhylipPluginTests.obj
 0001:0003d6e0       __unwindfunclet$??__EuiLog@U2@@YAXXZ$0 1003e6e0 f   PhylipPluginTests.obj
 0001:0003d6e9       __ehhandler$??__EuiLog@U2@@YAXXZ 1003e6e9 f   PhylipPluginTests.obj
 0001:0003d710       __unwindfunclet$??__EuserActLog@U2@@YAXXZ$0 1003e710 f   PhylipPluginTests.obj
 0001:0003d719       __ehhandler$??__EuserActLog@U2@@YAXXZ 1003e719 f   PhylipPluginTests.obj
 0001:0003d740       __ehhandler$?append@?$QList@PAVXMLTestFactory@U2@@@@QAEXABQAVXMLTestFactory@U2@@@Z 1003e740 f   PhylipPluginTests.obj
 0001:0003d760       __unwindfunclet$?createFactory@GTest_NeighborJoin@U2@@SAPAVXMLTestFactory@2@XZ$0 1003e760 f   PhylipPluginTests.obj
 0001:0003d76b       __unwindfunclet$?createFactory@GTest_NeighborJoin@U2@@SAPAVXMLTestFactory@2@XZ$1 1003e76b f   PhylipPluginTests.obj
 0001:0003d774       __unwindfunclet$?createFactory@GTest_NeighborJoin@U2@@SAPAVXMLTestFactory@2@XZ$2 1003e774 f   PhylipPluginTests.obj
 0001:0003d77d       __ehhandler$?createFactory@GTest_NeighborJoin@U2@@SAPAVXMLTestFactory@2@XZ 1003e77d f   PhylipPluginTests.obj
 0001:0003d7a0       __unwindfunclet$?createTest@GTest_NeighborJoinFactory@GTest_NeighborJoin@U2@@UAEPAVGTest@3@PAVXMLTestFormat@3@ABVQString@@PAV43@PBVGTestEnvironment@3@ABV?$QList@PAVGTest@U2@@@@ABVQDomElement@@@Z$0 1003e7a0 f   PhylipPluginTests.obj
 0001:0003d7ab       __unwindfunclet$?createTest@GTest_NeighborJoinFactory@GTest_NeighborJoin@U2@@UAEPAVGTest@3@PAVXMLTestFormat@3@ABVQString@@PAV43@PBVGTestEnvironment@3@ABV?$QList@PAVGTest@U2@@@@ABVQDomElement@@@Z$1 1003e7ab f   PhylipPluginTests.obj
 0001:0003d7b4       __unwindfunclet$?createTest@GTest_NeighborJoinFactory@GTest_NeighborJoin@U2@@UAEPAVGTest@3@PAVXMLTestFormat@3@ABVQString@@PAV43@PBVGTestEnvironment@3@ABV?$QList@PAVGTest@U2@@@@ABVQDomElement@@@Z$2 1003e7b4 f   PhylipPluginTests.obj
 0001:0003d7c3       __unwindfunclet$?createTest@GTest_NeighborJoinFactory@GTest_NeighborJoin@U2@@UAEPAVGTest@3@PAVXMLTestFormat@3@ABVQString@@PAV43@PBVGTestEnvironment@3@ABV?$QList@PAVGTest@U2@@@@ABVQDomElement@@@Z$3 1003e7c3 f   PhylipPluginTests.obj
 0001:0003d7d2       __ehhandler$?createTest@GTest_NeighborJoinFactory@GTest_NeighborJoin@U2@@UAEPAVGTest@3@PAVXMLTestFormat@3@ABVQString@@PAV43@PBVGTestEnvironment@3@ABV?$QList@PAVGTest@U2@@@@ABVQDomElement@@@Z 1003e7d2 f   PhylipPluginTests.obj
 0001:0003d7f0       __unwindfunclet$?createTestFactories@PhylipPluginTests@U2@@SA?AV?$QList@PAVXMLTestFactory@U2@@@@XZ$0 1003e7f0 f   PhylipPluginTests.obj
 0001:0003d809       __ehhandler$?createTestFactories@PhylipPluginTests@U2@@SA?AV?$QList@PAVXMLTestFactory@U2@@@@XZ 1003e809 f   PhylipPluginTests.obj
 0001:0003d830       __ehhandler$?detach_helper@?$QList@PAVGObject@U2@@@@AAEXH@Z 1003e830 f   PhylipPluginTests.obj
 0001:0003d850       __ehhandler$?detach_helper_grow@?$QList@PAVXMLTestFactory@U2@@@@AAEPAUNode@1@HH@Z 1003e850 f   PhylipPluginTests.obj
 0001:0003d870       __unwindfunclet$?init@GTest_NeighborJoin@U2@@QAEXPAVXMLTestFormat@2@ABVQDomElement@@@Z$0 1003e870 f   PhylipPluginTests.obj
 0001:0003d879       __unwindfunclet$?init@GTest_NeighborJoin@U2@@QAEXPAVXMLTestFormat@2@ABVQDomElement@@@Z$1 1003e879 f   PhylipPluginTests.obj
 0001:0003d882       __unwindfunclet$?init@GTest_NeighborJoin@U2@@QAEXPAVXMLTestFormat@2@ABVQDomElement@@@Z$2 1003e882 f   PhylipPluginTests.obj
 0001:0003d88b       __unwindfunclet$?init@GTest_NeighborJoin@U2@@QAEXPAVXMLTestFormat@2@ABVQDomElement@@@Z$3 1003e88b f   PhylipPluginTests.obj
 0001:0003d894       __unwindfunclet$?init@GTest_NeighborJoin@U2@@QAEXPAVXMLTestFormat@2@ABVQDomElement@@@Z$4 1003e894 f   PhylipPluginTests.obj
 0001:0003d89d       __unwindfunclet$?init@GTest_NeighborJoin@U2@@QAEXPAVXMLTestFormat@2@ABVQDomElement@@@Z$5 1003e89d f   PhylipPluginTests.obj
 0001:0003d8a6       __unwindfunclet$?init@GTest_NeighborJoin@U2@@QAEXPAVXMLTestFormat@2@ABVQDomElement@@@Z$6 1003e8a6 f   PhylipPluginTests.obj
 0001:0003d8af       __unwindfunclet$?init@GTest_NeighborJoin@U2@@QAEXPAVXMLTestFormat@2@ABVQDomElement@@@Z$7 1003e8af f   PhylipPluginTests.obj
 0001:0003d8b8       __unwindfunclet$?init@GTest_NeighborJoin@U2@@QAEXPAVXMLTestFormat@2@ABVQDomElement@@@Z$8 1003e8b8 f   PhylipPluginTests.obj
 0001:0003d8c1       __unwindfunclet$?init@GTest_NeighborJoin@U2@@QAEXPAVXMLTestFormat@2@ABVQDomElement@@@Z$9 1003e8c1 f   PhylipPluginTests.obj
 0001:0003d8ca       __unwindfunclet$?init@GTest_NeighborJoin@U2@@QAEXPAVXMLTestFormat@2@ABVQDomElement@@@Z$10 1003e8ca f   PhylipPluginTests.obj
 0001:0003d8d3       __ehhandler$?init@GTest_NeighborJoin@U2@@QAEXPAVXMLTestFormat@2@ABVQDomElement@@@Z 1003e8d3 f   PhylipPluginTests.obj
 0001:0003d8f0       __unwindfunclet$?prepare@GTest_NeighborJoin@U2@@UAEXXZ$0 1003e8f0 f   PhylipPluginTests.obj
 0001:0003d8f9       __unwindfunclet$?prepare@GTest_NeighborJoin@U2@@UAEXXZ$1 1003e8f9 f   PhylipPluginTests.obj
 0001:0003d902       __unwindfunclet$?prepare@GTest_NeighborJoin@U2@@UAEXXZ$3 1003e902 f   PhylipPluginTests.obj
 0001:0003d90a       __unwindfunclet$?prepare@GTest_NeighborJoin@U2@@UAEXXZ$4 1003e90a f   PhylipPluginTests.obj
 0001:0003d913       __unwindfunclet$?prepare@GTest_NeighborJoin@U2@@UAEXXZ$5 1003e913 f   PhylipPluginTests.obj
 0001:0003d91c       __unwindfunclet$?prepare@GTest_NeighborJoin@U2@@UAEXXZ$6 1003e91c f   PhylipPluginTests.obj
 0001:0003d925       __unwindfunclet$?prepare@GTest_NeighborJoin@U2@@UAEXXZ$7 1003e925 f   PhylipPluginTests.obj
 0001:0003d92e       __unwindfunclet$?prepare@GTest_NeighborJoin@U2@@UAEXXZ$8 1003e92e f   PhylipPluginTests.obj
 0001:0003d937       __unwindfunclet$?prepare@GTest_NeighborJoin@U2@@UAEXXZ$9 1003e937 f   PhylipPluginTests.obj
 0001:0003d940       __unwindfunclet$?prepare@GTest_NeighborJoin@U2@@UAEXXZ$10 1003e940 f   PhylipPluginTests.obj
 0001:0003d949       __unwindfunclet$?prepare@GTest_NeighborJoin@U2@@UAEXXZ$12 1003e949 f   PhylipPluginTests.obj
 0001:0003d951       __unwindfunclet$?prepare@GTest_NeighborJoin@U2@@UAEXXZ$13 1003e951 f   PhylipPluginTests.obj
 0001:0003d95a       __unwindfunclet$?prepare@GTest_NeighborJoin@U2@@UAEXXZ$14 1003e95a f   PhylipPluginTests.obj
 0001:0003d963       __unwindfunclet$?prepare@GTest_NeighborJoin@U2@@UAEXXZ$15 1003e963 f   PhylipPluginTests.obj
 0001:0003d96c       __unwindfunclet$?prepare@GTest_NeighborJoin@U2@@UAEXXZ$16 1003e96c f   PhylipPluginTests.obj
 0001:0003d975       __unwindfunclet$?prepare@GTest_NeighborJoin@U2@@UAEXXZ$17 1003e975 f   PhylipPluginTests.obj
 0001:0003d97e       __unwindfunclet$?prepare@GTest_NeighborJoin@U2@@UAEXXZ$18 1003e97e f   PhylipPluginTests.obj
 0001:0003d98a       __unwindfunclet$?prepare@GTest_NeighborJoin@U2@@UAEXXZ$19 1003e98a f   PhylipPluginTests.obj
 0001:0003d995       __unwindfunclet$?prepare@GTest_NeighborJoin@U2@@UAEXXZ$20 1003e995 f   PhylipPluginTests.obj
 0001:0003d9af       __ehhandler$?prepare@GTest_NeighborJoin@U2@@UAEXXZ 1003e9af f   PhylipPluginTests.obj
 0001:0003d9d0       __unwindfunclet$?report@GTest_NeighborJoin@U2@@UAE?AW4ReportResult@Task@2@XZ$0 1003e9d0 f   PhylipPluginTests.obj
 0001:0003d9d8       __unwindfunclet$?report@GTest_NeighborJoin@U2@@UAE?AW4ReportResult@Task@2@XZ$1 1003e9d8 f   PhylipPluginTests.obj
 0001:0003d9e1       __unwindfunclet$?report@GTest_NeighborJoin@U2@@UAE?AW4ReportResult@Task@2@XZ$2 1003e9e1 f   PhylipPluginTests.obj
 0001:0003d9ea       __ehhandler$?report@GTest_NeighborJoin@U2@@UAE?AW4ReportResult@Task@2@XZ 1003e9ea f   PhylipPluginTests.obj
 0001:0003da10       __unwindfunclet$??0PhylipTask@U2@@QAE@ABVU2EntityRef@1@ABVU2DbiRef@1@ABVCreatePhyTreeSettings@1@@Z$0 1003ea10 f   PhylipTask.obj
 0001:0003da19       __unwindfunclet$??0PhylipTask@U2@@QAE@ABVU2EntityRef@1@ABVU2DbiRef@1@ABVCreatePhyTreeSettings@1@@Z$1 1003ea19 f   PhylipTask.obj
 0001:0003da22       __unwindfunclet$??0PhylipTask@U2@@QAE@ABVU2EntityRef@1@ABVU2DbiRef@1@ABVCreatePhyTreeSettings@1@@Z$2 1003ea22 f   PhylipTask.obj
 0001:0003da31       __unwindfunclet$??0PhylipTask@U2@@QAE@ABVU2EntityRef@1@ABVU2DbiRef@1@ABVCreatePhyTreeSettings@1@@Z$3 1003ea31 f   PhylipTask.obj
 0001:0003da40       __ehhandler$??0PhylipTask@U2@@QAE@ABVU2EntityRef@1@ABVU2DbiRef@1@ABVCreatePhyTreeSettings@1@@Z 1003ea40 f   PhylipTask.obj
 0001:0003da60       __unwindfunclet$??1PhylipTask@U2@@UAE@XZ$0 1003ea60 f   PhylipTask.obj
 0001:0003da69       __unwindfunclet$??1PhylipTask@U2@@UAE@XZ$1 1003ea69 f   PhylipTask.obj
 0001:0003da78       __unwindfunclet$??1PhylipTask@U2@@UAE@XZ$2 1003ea78 f   PhylipTask.obj
 0001:0003da87       __ehhandler$??1PhylipTask@U2@@UAE@XZ 1003ea87 f   PhylipTask.obj
 0001:0003dab0       __unwindfunclet$??_GPhylipTask@U2@@UAEPAXI@Z$0 1003eab0 f   PhylipTask.obj
 0001:0003dab9       __unwindfunclet$??_GPhylipTask@U2@@UAEPAXI@Z$1 1003eab9 f   PhylipTask.obj
 0001:0003dac8       __unwindfunclet$??_GPhylipTask@U2@@UAEPAXI@Z$2 1003eac8 f   PhylipTask.obj
 0001:0003dad7       __ehhandler$??_GPhylipTask@U2@@UAEPAXI@Z 1003ead7 f   PhylipTask.obj
 0001:0003db00       __unwindfunclet$??__EalgoLog@U2@@YAXXZ$0 1003eb00 f   PhylipTask.obj
 0001:0003db09       __ehhandler$??__EalgoLog@U2@@YAXXZ 1003eb09 f   PhylipTask.obj
 0001:0003db30       __unwindfunclet$??__EcmdLog@U2@@YAXXZ$0 1003eb30 f   PhylipTask.obj
 0001:0003db39       __ehhandler$??__EcmdLog@U2@@YAXXZ 1003eb39 f   PhylipTask.obj
 0001:0003db60       __unwindfunclet$??__EcoreLog@U2@@YAXXZ$0 1003eb60 f   PhylipTask.obj
 0001:0003db69       __ehhandler$??__EcoreLog@U2@@YAXXZ 1003eb69 f   PhylipTask.obj
 0001:0003db90       __unwindfunclet$??__EioLog@U2@@YAXXZ$0 1003eb90 f   PhylipTask.obj
 0001:0003db99       __ehhandler$??__EioLog@U2@@YAXXZ 1003eb99 f   PhylipTask.obj
 0001:0003dbc0       __unwindfunclet$??__EperfLog@U2@@YAXXZ$0 1003ebc0 f   PhylipTask.obj
 0001:0003dbc9       __ehhandler$??__EperfLog@U2@@YAXXZ 1003ebc9 f   PhylipTask.obj
 0001:0003dbf0       __unwindfunclet$??__EscriptLog@U2@@YAXXZ$0 1003ebf0 f   PhylipTask.obj
 0001:0003dbf9       __ehhandler$??__EscriptLog@U2@@YAXXZ 1003ebf9 f   PhylipTask.obj
 0001:0003dc20       __unwindfunclet$??__EtaskLog@U2@@YAXXZ$0 1003ec20 f   PhylipTask.obj
 0001:0003dc29       __ehhandler$??__EtaskLog@U2@@YAXXZ 1003ec29 f   PhylipTask.obj
 0001:0003dc50       __unwindfunclet$??__EuiLog@U2@@YAXXZ$0 1003ec50 f   PhylipTask.obj
 0001:0003dc59       __ehhandler$??__EuiLog@U2@@YAXXZ 1003ec59 f   PhylipTask.obj
 0001:0003dc80       __unwindfunclet$??__EuserActLog@U2@@YAXXZ$0 1003ec80 f   PhylipTask.obj
 0001:0003dc89       __ehhandler$??__EuserActLog@U2@@YAXXZ 1003ec89 f   PhylipTask.obj
 0001:0003dcb0       __unwindfunclet$?prepare@PhylipTask@U2@@UAEXXZ$0 1003ecb0 f   PhylipTask.obj
 0001:0003dcbb       __unwindfunclet$?prepare@PhylipTask@U2@@UAEXXZ$1 1003ecbb f   PhylipTask.obj
 0001:0003dcd5       __unwindfunclet$?prepare@PhylipTask@U2@@UAEXXZ$2 1003ecd5 f   PhylipTask.obj
 0001:0003dcee       __unwindfunclet$?prepare@PhylipTask@U2@@UAEXXZ$3 1003ecee f   PhylipTask.obj
 0001:0003dd08       __unwindfunclet$?prepare@PhylipTask@U2@@UAEXXZ$4 1003ed08 f   PhylipTask.obj
 0001:0003dd22       __unwindfunclet$?prepare@PhylipTask@U2@@UAEXXZ$5 1003ed22 f   PhylipTask.obj
 0001:0003dd3b       __unwindfunclet$?prepare@PhylipTask@U2@@UAEXXZ$6 1003ed3b f   PhylipTask.obj
 0001:0003dd46       __unwindfunclet$?prepare@PhylipTask@U2@@UAEXXZ$7 1003ed46 f   PhylipTask.obj
 0001:0003dd60       __ehhandler$?prepare@PhylipTask@U2@@UAEXXZ 1003ed60 f   PhylipTask.obj
 0001:0003dd80       __unwindfunclet$?report@PhylipTask@U2@@UAE?AW4ReportResult@Task@2@XZ$0 1003ed80 f   PhylipTask.obj
 0001:0003dd89       __ehhandler$?report@PhylipTask@U2@@UAE?AW4ReportResult@Task@2@XZ 1003ed89 f   PhylipTask.obj
 0001:0003ddb0       __unwindfunclet$?saveTree@PhylipTask@U2@@AAE?AVQByteArray@@XZ$0 1003edb0 f   PhylipTask.obj
 0001:0003ddb9       __unwindfunclet$?saveTree@PhylipTask@U2@@AAE?AVQByteArray@@XZ$1 1003edb9 f   PhylipTask.obj
 0001:0003ddc1       __unwindfunclet$?saveTree@PhylipTask@U2@@AAE?AVQByteArray@@XZ$2 1003edc1 f   PhylipTask.obj
 0001:0003ddc9       __unwindfunclet$?saveTree@PhylipTask@U2@@AAE?AVQByteArray@@XZ$3 1003edc9 f   PhylipTask.obj
 0001:0003dde3       __unwindfunclet$?saveTree@PhylipTask@U2@@AAE?AVQByteArray@@XZ$4 1003ede3 f   PhylipTask.obj
 0001:0003ddec       __ehhandler$?saveTree@PhylipTask@U2@@AAE?AVQByteArray@@XZ 1003edec f   PhylipTask.obj
 0001:0003de10       __unwindfunclet$??0SeqBoot@U2@@QAE@XZ$0 1003ee10 f   SeqBootAdapter.obj
 0001:0003de18       __unwindfunclet$??0SeqBoot@U2@@QAE@XZ$1 1003ee18 f   SeqBootAdapter.obj
 0001:0003de21       __unwindfunclet$??0SeqBoot@U2@@QAE@XZ$2 1003ee21 f   SeqBootAdapter.obj
 0001:0003de2a       __ehhandler$??0SeqBoot@U2@@QAE@XZ 1003ee2a f   SeqBootAdapter.obj
 0001:0003de50       __unwindfunclet$??1SeqBoot@U2@@QAE@XZ$0 1003ee50 f   SeqBootAdapter.obj
 0001:0003de59       __unwindfunclet$??1SeqBoot@U2@@QAE@XZ$1 1003ee59 f   SeqBootAdapter.obj
 0001:0003de64       __ehhandler$??1SeqBoot@U2@@QAE@XZ 1003ee64 f   SeqBootAdapter.obj
 0001:0003de80       __unwindfunclet$??__EalgoLog@U2@@YAXXZ$0 1003ee80 f   SeqBootAdapter.obj
 0001:0003de89       __ehhandler$??__EalgoLog@U2@@YAXXZ 1003ee89 f   SeqBootAdapter.obj
 0001:0003deb0       __unwindfunclet$??__EcmdLog@U2@@YAXXZ$0 1003eeb0 f   SeqBootAdapter.obj
 0001:0003deb9       __ehhandler$??__EcmdLog@U2@@YAXXZ 1003eeb9 f   SeqBootAdapter.obj
 0001:0003dee0       __unwindfunclet$??__EcoreLog@U2@@YAXXZ$0 1003eee0 f   SeqBootAdapter.obj
 0001:0003dee9       __ehhandler$??__EcoreLog@U2@@YAXXZ 1003eee9 f   SeqBootAdapter.obj
 0001:0003df10       __unwindfunclet$??__EioLog@U2@@YAXXZ$0 1003ef10 f   SeqBootAdapter.obj
 0001:0003df19       __ehhandler$??__EioLog@U2@@YAXXZ 1003ef19 f   SeqBootAdapter.obj
 0001:0003df40       __unwindfunclet$??__EperfLog@U2@@YAXXZ$0 1003ef40 f   SeqBootAdapter.obj
 0001:0003df49       __ehhandler$??__EperfLog@U2@@YAXXZ 1003ef49 f   SeqBootAdapter.obj
 0001:0003df70       __unwindfunclet$??__EscriptLog@U2@@YAXXZ$0 1003ef70 f   SeqBootAdapter.obj
 0001:0003df79       __ehhandler$??__EscriptLog@U2@@YAXXZ 1003ef79 f   SeqBootAdapter.obj
 0001:0003dfa0       __unwindfunclet$??__EtaskLog@U2@@YAXXZ$0 1003efa0 f   SeqBootAdapter.obj
 0001:0003dfa9       __ehhandler$??__EtaskLog@U2@@YAXXZ 1003efa9 f   SeqBootAdapter.obj
 0001:0003dfd0       __unwindfunclet$??__EuiLog@U2@@YAXXZ$0 1003efd0 f   SeqBootAdapter.obj
 0001:0003dfd9       __ehhandler$??__EuiLog@U2@@YAXXZ 1003efd9 f   SeqBootAdapter.obj
 0001:0003e000       __unwindfunclet$??__EuserActLog@U2@@YAXXZ$0 1003f000 f   SeqBootAdapter.obj
 0001:0003e009       __ehhandler$??__EuserActLog@U2@@YAXXZ 1003f009 f   SeqBootAdapter.obj
 0001:0003e030       __unwindfunclet$?clear@?$QVector@VMultipleSequenceAlignment@U2@@@@QAEXXZ$0 1003f030 f   SeqBootAdapter.obj
 0001:0003e038       __ehhandler$?clear@?$QVector@VMultipleSequenceAlignment@U2@@@@QAEXXZ 1003f038 f   SeqBootAdapter.obj
 0001:0003e060       __unwindfunclet$?copyConstruct@?$QVector@VMultipleSequenceAlignment@U2@@@@AAEXPBVMultipleSequenceAlignment@U2@@0PAV23@@Z$0 1003f060 f   SeqBootAdapter.obj
 0001:0003e071       __ehhandler$?copyConstruct@?$QVector@VMultipleSequenceAlignment@U2@@@@AAEXPBVMultipleSequenceAlignment@U2@@0PAV23@@Z 1003f071 f   SeqBootAdapter.obj
 0001:0003e090       __unwindfunclet$?defaultConstruct@?$QVector@VMultipleSequenceAlignment@U2@@@@AAEXPAVMultipleSequenceAlignment@U2@@0@Z$0 1003f090 f   SeqBootAdapter.obj
 0001:0003e0a1       __unwindfunclet$?defaultConstruct@?$QVector@VMultipleSequenceAlignment@U2@@@@AAEXPAVMultipleSequenceAlignment@U2@@0@Z$1 1003f0a1 f   SeqBootAdapter.obj
 0001:0003e0ba       __unwindfunclet$?defaultConstruct@?$QVector@VMultipleSequenceAlignment@U2@@@@AAEXPAVMultipleSequenceAlignment@U2@@0@Z$2 1003f0ba f   SeqBootAdapter.obj
 0001:0003e0d4       __ehhandler$?defaultConstruct@?$QVector@VMultipleSequenceAlignment@U2@@@@AAEXPAVMultipleSequenceAlignment@U2@@0@Z 1003f0d4 f   SeqBootAdapter.obj
 0001:0003e0f0       __unwindfunclet$?generateSequencesFromAlignment@SeqBoot@U2@@QAEXABVMultipleSequenceAlignment@2@ABVCreatePhyTreeSettings@2@@Z$0 1003f0f0 f   SeqBootAdapter.obj
 0001:0003e0f9       __ehhandler$?generateSequencesFromAlignment@SeqBoot@U2@@QAEXABVMultipleSequenceAlignment@2@ABVCreatePhyTreeSettings@2@@Z 1003f0f9 f   SeqBootAdapter.obj
 0001:0003e120       __unwindfunclet$?getTmpFileTemplate@SeqBoot@U2@@QAE?AVQString@@XZ$0 1003f120 f   SeqBootAdapter.obj
 0001:0003e129       __unwindfunclet$?getTmpFileTemplate@SeqBoot@U2@@QAE?AVQString@@XZ$1 1003f129 f   SeqBootAdapter.obj
 0001:0003e132       __unwindfunclet$?getTmpFileTemplate@SeqBoot@U2@@QAE?AVQString@@XZ$2 1003f132 f   SeqBootAdapter.obj
 0001:0003e13b       __unwindfunclet$?getTmpFileTemplate@SeqBoot@U2@@QAE?AVQString@@XZ$4 1003f13b f   SeqBootAdapter.obj
 0001:0003e155       __ehhandler$?getTmpFileTemplate@SeqBoot@U2@@QAE?AVQString@@XZ 1003f155 f   SeqBootAdapter.obj
 0001:0003e170       __unwindfunclet$?initGenerSeq@SeqBoot@U2@@QAEXHHH@Z$0 1003f170 f   SeqBootAdapter.obj
 0001:0003e178       __unwindfunclet$?initGenerSeq@SeqBoot@U2@@QAEXHHH@Z$2 1003f178 f   SeqBootAdapter.obj
 0001:0003e180       __unwindfunclet$?initGenerSeq@SeqBoot@U2@@QAEXHHH@Z$3 1003f180 f   SeqBootAdapter.obj
 0001:0003e189       __unwindfunclet$?initGenerSeq@SeqBoot@U2@@QAEXHHH@Z$4 1003f189 f   SeqBootAdapter.obj
 0001:0003e192       __unwindfunclet$?initGenerSeq@SeqBoot@U2@@QAEXHHH@Z$5 1003f192 f   SeqBootAdapter.obj
 0001:0003e19b       __ehhandler$?initGenerSeq@SeqBoot@U2@@QAEXHHH@Z 1003f19b f   SeqBootAdapter.obj
 0001:0003e1c0       __unwindfunclet$?reallocData@?$QVector@VMultipleSequenceAlignment@U2@@@@AAEXHHV?$QFlags@W4AllocationOption@QArrayData@@@@@Z$4 1003f1c0 f   SeqBootAdapter.obj
 0001:0003e1d1       __ehhandler$?reallocData@?$QVector@VMultipleSequenceAlignment@U2@@@@AAEXHHV?$QFlags@W4AllocationOption@QArrayData@@@@@Z 1003f1d1 f   SeqBootAdapter.obj
 0001:0003e1f0       __unwindfunclet$??__EalgoLog@U2@@YAXXZ$0 1003f1f0 f   dist.obj
 0001:0003e1f9       __ehhandler$??__EalgoLog@U2@@YAXXZ 1003f1f9 f   dist.obj
 0001:0003e220       __unwindfunclet$??__EcmdLog@U2@@YAXXZ$0 1003f220 f   dist.obj
 0001:0003e229       __ehhandler$??__EcmdLog@U2@@YAXXZ 1003f229 f   dist.obj
 0001:0003e250       __unwindfunclet$??__EcoreLog@U2@@YAXXZ$0 1003f250 f   dist.obj
 0001:0003e259       __ehhandler$??__EcoreLog@U2@@YAXXZ 1003f259 f   dist.obj
 0001:0003e280       __unwindfunclet$??__EioLog@U2@@YAXXZ$0 1003f280 f   dist.obj
 0001:0003e289       __ehhandler$??__EioLog@U2@@YAXXZ 1003f289 f   dist.obj
 0001:0003e2b0       __unwindfunclet$??__EperfLog@U2@@YAXXZ$0 1003f2b0 f   dist.obj
 0001:0003e2b9       __ehhandler$??__EperfLog@U2@@YAXXZ 1003f2b9 f   dist.obj
 0001:0003e2e0       __unwindfunclet$??__EscriptLog@U2@@YAXXZ$0 1003f2e0 f   dist.obj
 0001:0003e2e9       __ehhandler$??__EscriptLog@U2@@YAXXZ 1003f2e9 f   dist.obj
 0001:0003e310       __unwindfunclet$??__EtaskLog@U2@@YAXXZ$0 1003f310 f   dist.obj
 0001:0003e319       __ehhandler$??__EtaskLog@U2@@YAXXZ 1003f319 f   dist.obj
 0001:0003e340       __unwindfunclet$??__EuiLog@U2@@YAXXZ$0 1003f340 f   dist.obj
 0001:0003e349       __ehhandler$??__EuiLog@U2@@YAXXZ 1003f349 f   dist.obj
 0001:0003e370       __unwindfunclet$??__EuserActLog@U2@@YAXXZ$0 1003f370 f   dist.obj
 0001:0003e379       __ehhandler$??__EuserActLog@U2@@YAXXZ 1003f379 f   dist.obj
 0001:0003e3a0       __unwindfunclet$?dist_treeout@@YAXPAUnode@@PAJNE0@Z$0 1003f3a0 f   dist.obj
 0001:0003e3a9       __unwindfunclet$?dist_treeout@@YAXPAUnode@@PAJNE0@Z$1 1003f3a9 f   dist.obj
 0001:0003e3b2       __ehhandler$?dist_treeout@@YAXPAUnode@@PAJNE0@Z 1003f3b2 f   dist.obj
 0001:0003e3e0       __unwindfunclet$?treeoutr@@YAXPAUnode@@PAJPAUtree@@@Z$0 1003f3e0 f   dist.obj
 0001:0003e3e9       __unwindfunclet$?treeoutr@@YAXPAUnode@@PAJPAUtree@@@Z$1 1003f3e9 f   dist.obj
 0001:0003e3f2       __ehhandler$?treeoutr@@YAXPAUnode@@PAJPAUtree@@@Z 1003f3f2 f   dist.obj
 0001:0003e420       __unwindfunclet$??__EalgoLog@U2@@YAXXZ$0 1003f420 f   dnadist.obj
 0001:0003e429       __ehhandler$??__EalgoLog@U2@@YAXXZ 1003f429 f   dnadist.obj
 0001:0003e450       __unwindfunclet$??__EcmdLog@U2@@YAXXZ$0 1003f450 f   dnadist.obj
 0001:0003e459       __ehhandler$??__EcmdLog@U2@@YAXXZ 1003f459 f   dnadist.obj
 0001:0003e480       __unwindfunclet$??__EcoreLog@U2@@YAXXZ$0 1003f480 f   dnadist.obj
 0001:0003e489       __ehhandler$??__EcoreLog@U2@@YAXXZ 1003f489 f   dnadist.obj
 0001:0003e4b0       __unwindfunclet$??__EioLog@U2@@YAXXZ$0 1003f4b0 f   dnadist.obj
 0001:0003e4b9       __ehhandler$??__EioLog@U2@@YAXXZ 1003f4b9 f   dnadist.obj
 0001:0003e4e0       __unwindfunclet$??__EperfLog@U2@@YAXXZ$0 1003f4e0 f   dnadist.obj
 0001:0003e4e9       __ehhandler$??__EperfLog@U2@@YAXXZ 1003f4e9 f   dnadist.obj
 0001:0003e510       __unwindfunclet$??__EscriptLog@U2@@YAXXZ$0 1003f510 f   dnadist.obj
 0001:0003e519       __ehhandler$??__EscriptLog@U2@@YAXXZ 1003f519 f   dnadist.obj
 0001:0003e540       __unwindfunclet$??__EtaskLog@U2@@YAXXZ$0 1003f540 f   dnadist.obj
 0001:0003e549       __ehhandler$??__EtaskLog@U2@@YAXXZ 1003f549 f   dnadist.obj
 0001:0003e570       __unwindfunclet$??__EuiLog@U2@@YAXXZ$0 1003f570 f   dnadist.obj
 0001:0003e579       __ehhandler$??__EuiLog@U2@@YAXXZ 1003f579 f   dnadist.obj
 0001:0003e5a0       __unwindfunclet$??__EuserActLog@U2@@YAXXZ$0 1003f5a0 f   dnadist.obj
 0001:0003e5a9       __ehhandler$??__EuserActLog@U2@@YAXXZ 1003f5a9 f   dnadist.obj
 0001:0003e5d0       __unwindfunclet$?getoptions@@YAXXZ$0 1003f5d0 f   dnadist.obj
 0001:0003e5d9       __ehhandler$?getoptions@@YAXXZ 1003f5d9 f   dnadist.obj
 0001:0003e600       __unwindfunclet$??__EalgoLog@U2@@YAXXZ$0 1003f600 f   neighbor.obj
 0001:0003e609       __ehhandler$??__EalgoLog@U2@@YAXXZ 1003f609 f   neighbor.obj
 0001:0003e630       __unwindfunclet$??__EcmdLog@U2@@YAXXZ$0 1003f630 f   neighbor.obj
 0001:0003e639       __ehhandler$??__EcmdLog@U2@@YAXXZ 1003f639 f   neighbor.obj
 0001:0003e660       __unwindfunclet$??__EcoreLog@U2@@YAXXZ$0 1003f660 f   neighbor.obj
 0001:0003e669       __ehhandler$??__EcoreLog@U2@@YAXXZ 1003f669 f   neighbor.obj
 0001:0003e690       __unwindfunclet$??__EioLog@U2@@YAXXZ$0 1003f690 f   neighbor.obj
 0001:0003e699       __ehhandler$??__EioLog@U2@@YAXXZ 1003f699 f   neighbor.obj
 0001:0003e6c0       __unwindfunclet$??__EperfLog@U2@@YAXXZ$0 1003f6c0 f   neighbor.obj
 0001:0003e6c9       __ehhandler$??__EperfLog@U2@@YAXXZ 1003f6c9 f   neighbor.obj
 0001:0003e6f0       __unwindfunclet$??__EscriptLog@U2@@YAXXZ$0 1003f6f0 f   neighbor.obj
 0001:0003e6f9       __ehhandler$??__EscriptLog@U2@@YAXXZ 1003f6f9 f   neighbor.obj
 0001:0003e720       __unwindfunclet$??__EtaskLog@U2@@YAXXZ$0 1003f720 f   neighbor.obj
 0001:0003e729       __ehhandler$??__EtaskLog@U2@@YAXXZ 1003f729 f   neighbor.obj
 0001:0003e750       __unwindfunclet$??__EuiLog@U2@@YAXXZ$0 1003f750 f   neighbor.obj
 0001:0003e759       __ehhandler$??__EuiLog@U2@@YAXXZ 1003f759 f   neighbor.obj
 0001:0003e780       __unwindfunclet$??__EuserActLog@U2@@YAXXZ$0 1003f780 f   neighbor.obj
 0001:0003e789       __ehhandler$??__EuserActLog@U2@@YAXXZ 1003f789 f   neighbor.obj
 0001:0003e7b0       __unwindfunclet$??__EalgoLog@U2@@YAXXZ$0 1003f7b0 f   phylip.obj
 0001:0003e7b9       __ehhandler$??__EalgoLog@U2@@YAXXZ 1003f7b9 f   phylip.obj
 0001:0003e7e0       __unwindfunclet$??__EcmdLog@U2@@YAXXZ$0 1003f7e0 f   phylip.obj
 0001:0003e7e9       __ehhandler$??__EcmdLog@U2@@YAXXZ 1003f7e9 f   phylip.obj
 0001:0003e810       __unwindfunclet$??__EcoreLog@U2@@YAXXZ$0 1003f810 f   phylip.obj
 0001:0003e819       __ehhandler$??__EcoreLog@U2@@YAXXZ 1003f819 f   phylip.obj
 0001:0003e840       __unwindfunclet$??__EioLog@U2@@YAXXZ$0 1003f840 f   phylip.obj
 0001:0003e849       __ehhandler$??__EioLog@U2@@YAXXZ 1003f849 f   phylip.obj
 0001:0003e870       __unwindfunclet$??__EperfLog@U2@@YAXXZ$0 1003f870 f   phylip.obj
 0001:0003e879       __ehhandler$??__EperfLog@U2@@YAXXZ 1003f879 f   phylip.obj
 0001:0003e8a0       __unwindfunclet$??__EscriptLog@U2@@YAXXZ$0 1003f8a0 f   phylip.obj
 0001:0003e8a9       __ehhandler$??__EscriptLog@U2@@YAXXZ 1003f8a9 f   phylip.obj
 0001:0003e8d0       __unwindfunclet$??__EtaskLog@U2@@YAXXZ$0 1003f8d0 f   phylip.obj
 0001:0003e8d9       __ehhandler$??__EtaskLog@U2@@YAXXZ 1003f8d9 f   phylip.obj
 0001:0003e900       __unwindfunclet$??__EuiLog@U2@@YAXXZ$0 1003f900 f   phylip.obj
 0001:0003e909       __ehhandler$??__EuiLog@U2@@YAXXZ 1003f909 f   phylip.obj
 0001:0003e930       __unwindfunclet$??__EuserActLog@U2@@YAXXZ$0 1003f930 f   phylip.obj
 0001:0003e939       __ehhandler$??__EuserActLog@U2@@YAXXZ 1003f939 f   phylip.obj
 0001:0003e960       __unwindfunclet$??__EalgoLog@U2@@YAXXZ$0 1003f960 f   protdist.obj
 0001:0003e969       __ehhandler$??__EalgoLog@U2@@YAXXZ 1003f969 f   protdist.obj
 0001:0003e990       __unwindfunclet$??__EcmdLog@U2@@YAXXZ$0 1003f990 f   protdist.obj
 0001:0003e999       __ehhandler$??__EcmdLog@U2@@YAXXZ 1003f999 f   protdist.obj
 0001:0003e9c0       __unwindfunclet$??__EcoreLog@U2@@YAXXZ$0 1003f9c0 f   protdist.obj
 0001:0003e9c9       __ehhandler$??__EcoreLog@U2@@YAXXZ 1003f9c9 f   protdist.obj
 0001:0003e9f0       __unwindfunclet$??__EioLog@U2@@YAXXZ$0 1003f9f0 f   protdist.obj
 0001:0003e9f9       __ehhandler$??__EioLog@U2@@YAXXZ 1003f9f9 f   protdist.obj
 0001:0003ea20       __unwindfunclet$??__EperfLog@U2@@YAXXZ$0 1003fa20 f   protdist.obj
 0001:0003ea29       __ehhandler$??__EperfLog@U2@@YAXXZ 1003fa29 f   protdist.obj
 0001:0003ea50       __unwindfunclet$??__EscriptLog@U2@@YAXXZ$0 1003fa50 f   protdist.obj
 0001:0003ea59       __ehhandler$??__EscriptLog@U2@@YAXXZ 1003fa59 f   protdist.obj
 0001:0003ea80       __unwindfunclet$??__EtaskLog@U2@@YAXXZ$0 1003fa80 f   protdist.obj
 0001:0003ea89       __ehhandler$??__EtaskLog@U2@@YAXXZ 1003fa89 f   protdist.obj
 0001:0003eab0       __unwindfunclet$??__EuiLog@U2@@YAXXZ$0 1003fab0 f   protdist.obj
 0001:0003eab9       __ehhandler$??__EuiLog@U2@@YAXXZ 1003fab9 f   protdist.obj
 0001:0003eae0       __unwindfunclet$??__EuserActLog@U2@@YAXXZ$0 1003fae0 f   protdist.obj
 0001:0003eae9       __ehhandler$??__EuserActLog@U2@@YAXXZ 1003fae9 f   protdist.obj
 0001:0003eb10       __unwindfunclet$??__EalgoLog@U2@@YAXXZ$0 1003fb10 f   seqboot.obj
 0001:0003eb19       __ehhandler$??__EalgoLog@U2@@YAXXZ 1003fb19 f   seqboot.obj
 0001:0003eb40       __unwindfunclet$??__EcmdLog@U2@@YAXXZ$0 1003fb40 f   seqboot.obj
 0001:0003eb49       __ehhandler$??__EcmdLog@U2@@YAXXZ 1003fb49 f   seqboot.obj
 0001:0003eb70       __unwindfunclet$??__EcoreLog@U2@@YAXXZ$0 1003fb70 f   seqboot.obj
 0001:0003eb79       __ehhandler$??__EcoreLog@U2@@YAXXZ 1003fb79 f   seqboot.obj
 0001:0003eba0       __unwindfunclet$??__EioLog@U2@@YAXXZ$0 1003fba0 f   seqboot.obj
 0001:0003eba9       __ehhandler$??__EioLog@U2@@YAXXZ 1003fba9 f   seqboot.obj
 0001:0003ebd0       __unwindfunclet$??__EperfLog@U2@@YAXXZ$0 1003fbd0 f   seqboot.obj
 0001:0003ebd9       __ehhandler$??__EperfLog@U2@@YAXXZ 1003fbd9 f   seqboot.obj
 0001:0003ec00       __unwindfunclet$??__EscriptLog@U2@@YAXXZ$0 1003fc00 f   seqboot.obj
 0001:0003ec09       __ehhandler$??__EscriptLog@U2@@YAXXZ 1003fc09 f   seqboot.obj
 0001:0003ec30       __unwindfunclet$??__EtaskLog@U2@@YAXXZ$0 1003fc30 f   seqboot.obj
 0001:0003ec39       __ehhandler$??__EtaskLog@U2@@YAXXZ 1003fc39 f   seqboot.obj
 0001:0003ec60       __unwindfunclet$??__EuiLog@U2@@YAXXZ$0 1003fc60 f   seqboot.obj
 0001:0003ec69       __ehhandler$??__EuiLog@U2@@YAXXZ 1003fc69 f   seqboot.obj
 0001:0003ec90       __unwindfunclet$??__EuserActLog@U2@@YAXXZ$0 1003fc90 f   seqboot.obj
 0001:0003ec99       __ehhandler$??__EuserActLog@U2@@YAXXZ 1003fc99 f   seqboot.obj
 0001:0003ecc0       __unwindfunclet$?writedata@@YAXAAV?$QVector@VMultipleSequenceAlignment@U2@@@@HABVMultipleSequenceAlignment@U2@@@Z$0 1003fcc0 f   seqboot.obj
 0001:0003ecc9       __unwindfunclet$?writedata@@YAXAAV?$QVector@VMultipleSequenceAlignment@U2@@@@HABVMultipleSequenceAlignment@U2@@@Z$1 1003fcc9 f   seqboot.obj
 0001:0003ecd2       __unwindfunclet$?writedata@@YAXAAV?$QVector@VMultipleSequenceAlignment@U2@@@@HABVMultipleSequenceAlignment@U2@@@Z$2 1003fcd2 f   seqboot.obj
 0001:0003ecdb       __ehhandler$?writedata@@YAXAAV?$QVector@VMultipleSequenceAlignment@U2@@@@HABVMultipleSequenceAlignment@U2@@@Z 1003fcdb f   seqboot.obj
 0001:0003ed00       __unwindfunclet$??__EalgoLog@U2@@YAXXZ$0 1003fd00 f   moc_NeighborJoinWidget.obj
 0001:0003ed09       __ehhandler$??__EalgoLog@U2@@YAXXZ 1003fd09 f   moc_NeighborJoinWidget.obj
 0001:0003ed30       __unwindfunclet$??__EcmdLog@U2@@YAXXZ$0 1003fd30 f   moc_NeighborJoinWidget.obj
 0001:0003ed39       __ehhandler$??__EcmdLog@U2@@YAXXZ 1003fd39 f   moc_NeighborJoinWidget.obj
 0001:0003ed60       __unwindfunclet$??__EcoreLog@U2@@YAXXZ$0 1003fd60 f   moc_NeighborJoinWidget.obj
 0001:0003ed69       __ehhandler$??__EcoreLog@U2@@YAXXZ 1003fd69 f   moc_NeighborJoinWidget.obj
 0001:0003ed90       __unwindfunclet$??__EioLog@U2@@YAXXZ$0 1003fd90 f   moc_NeighborJoinWidget.obj
 0001:0003ed99       __ehhandler$??__EioLog@U2@@YAXXZ 1003fd99 f   moc_NeighborJoinWidget.obj
 0001:0003edc0       __unwindfunclet$??__EperfLog@U2@@YAXXZ$0 1003fdc0 f   moc_NeighborJoinWidget.obj
 0001:0003edc9       __ehhandler$??__EperfLog@U2@@YAXXZ 1003fdc9 f   moc_NeighborJoinWidget.obj
 0001:0003edf0       __unwindfunclet$??__EscriptLog@U2@@YAXXZ$0 1003fdf0 f   moc_NeighborJoinWidget.obj
 0001:0003edf9       __ehhandler$??__EscriptLog@U2@@YAXXZ 1003fdf9 f   moc_NeighborJoinWidget.obj
 0001:0003ee20       __unwindfunclet$??__EtaskLog@U2@@YAXXZ$0 1003fe20 f   moc_NeighborJoinWidget.obj
 0001:0003ee29       __ehhandler$??__EtaskLog@U2@@YAXXZ 1003fe29 f   moc_NeighborJoinWidget.obj
 0001:0003ee50       __unwindfunclet$??__EuiLog@U2@@YAXXZ$0 1003fe50 f   moc_NeighborJoinWidget.obj
 0001:0003ee59       __ehhandler$??__EuiLog@U2@@YAXXZ 1003fe59 f   moc_NeighborJoinWidget.obj
 0001:0003ee80       __unwindfunclet$??__EuserActLog@U2@@YAXXZ$0 1003fe80 f   moc_NeighborJoinWidget.obj
 0001:0003ee89       __ehhandler$??__EuserActLog@U2@@YAXXZ 1003fe89 f   moc_NeighborJoinWidget.obj
 0001:0003eeb0       __unwindfunclet$??__EalgoLog@U2@@YAXXZ$0 1003feb0 f   moc_PhylipCmdlineTask.obj
 0001:0003eeb9       __ehhandler$??__EalgoLog@U2@@YAXXZ 1003feb9 f   moc_PhylipCmdlineTask.obj
 0001:0003eee0       __unwindfunclet$??__EcmdLog@U2@@YAXXZ$0 1003fee0 f   moc_PhylipCmdlineTask.obj
 0001:0003eee9       __ehhandler$??__EcmdLog@U2@@YAXXZ 1003fee9 f   moc_PhylipCmdlineTask.obj
 0001:0003ef10       __unwindfunclet$??__EcoreLog@U2@@YAXXZ$0 1003ff10 f   moc_PhylipCmdlineTask.obj
 0001:0003ef19       __ehhandler$??__EcoreLog@U2@@YAXXZ 1003ff19 f   moc_PhylipCmdlineTask.obj
 0001:0003ef40       __unwindfunclet$??__EioLog@U2@@YAXXZ$0 1003ff40 f   moc_PhylipCmdlineTask.obj
 0001:0003ef49       __ehhandler$??__EioLog@U2@@YAXXZ 1003ff49 f   moc_PhylipCmdlineTask.obj
 0001:0003ef70       __unwindfunclet$??__EperfLog@U2@@YAXXZ$0 1003ff70 f   moc_PhylipCmdlineTask.obj
 0001:0003ef79       __ehhandler$??__EperfLog@U2@@YAXXZ 1003ff79 f   moc_PhylipCmdlineTask.obj
 0001:0003efa0       __unwindfunclet$??__EscriptLog@U2@@YAXXZ$0 1003ffa0 f   moc_PhylipCmdlineTask.obj
 0001:0003efa9       __ehhandler$??__EscriptLog@U2@@YAXXZ 1003ffa9 f   moc_PhylipCmdlineTask.obj
 0001:0003efd0       __unwindfunclet$??__EtaskLog@U2@@YAXXZ$0 1003ffd0 f   moc_PhylipCmdlineTask.obj
 0001:0003efd9       __ehhandler$??__EtaskLog@U2@@YAXXZ 1003ffd9 f   moc_PhylipCmdlineTask.obj
 0001:0003f000       __unwindfunclet$??__EuiLog@U2@@YAXXZ$0 10040000 f   moc_PhylipCmdlineTask.obj
 0001:0003f009       __ehhandler$??__EuiLog@U2@@YAXXZ 10040009 f   moc_PhylipCmdlineTask.obj
 0001:0003f030       __unwindfunclet$??__EuserActLog@U2@@YAXXZ$0 10040030 f   moc_PhylipCmdlineTask.obj
 0001:0003f039       __ehhandler$??__EuserActLog@U2@@YAXXZ 10040039 f   moc_PhylipCmdlineTask.obj
 0001:0003f060       __unwindfunclet$??__EalgoLog@U2@@YAXXZ$0 10040060 f   moc_PhylipPluginTests.obj
 0001:0003f069       __ehhandler$??__EalgoLog@U2@@YAXXZ 10040069 f   moc_PhylipPluginTests.obj
 0001:0003f090       __unwindfunclet$??__EcmdLog@U2@@YAXXZ$0 10040090 f   moc_PhylipPluginTests.obj
 0001:0003f099       __ehhandler$??__EcmdLog@U2@@YAXXZ 10040099 f   moc_PhylipPluginTests.obj
 0001:0003f0c0       __unwindfunclet$??__EcoreLog@U2@@YAXXZ$0 100400c0 f   moc_PhylipPluginTests.obj
 0001:0003f0c9       __ehhandler$??__EcoreLog@U2@@YAXXZ 100400c9 f   moc_PhylipPluginTests.obj
 0001:0003f0f0       __unwindfunclet$??__EioLog@U2@@YAXXZ$0 100400f0 f   moc_PhylipPluginTests.obj
 0001:0003f0f9       __ehhandler$??__EioLog@U2@@YAXXZ 100400f9 f   moc_PhylipPluginTests.obj
 0001:0003f120       __unwindfunclet$??__EperfLog@U2@@YAXXZ$0 10040120 f   moc_PhylipPluginTests.obj
 0001:0003f129       __ehhandler$??__EperfLog@U2@@YAXXZ 10040129 f   moc_PhylipPluginTests.obj
 0001:0003f150       __unwindfunclet$??__EscriptLog@U2@@YAXXZ$0 10040150 f   moc_PhylipPluginTests.obj
 0001:0003f159       __ehhandler$??__EscriptLog@U2@@YAXXZ 10040159 f   moc_PhylipPluginTests.obj
 0001:0003f180       __unwindfunclet$??__EtaskLog@U2@@YAXXZ$0 10040180 f   moc_PhylipPluginTests.obj
 0001:0003f189       __ehhandler$??__EtaskLog@U2@@YAXXZ 10040189 f   moc_PhylipPluginTests.obj
 0001:0003f1b0       __unwindfunclet$??__EuiLog@U2@@YAXXZ$0 100401b0 f   moc_PhylipPluginTests.obj
 0001:0003f1b9       __ehhandler$??__EuiLog@U2@@YAXXZ 100401b9 f   moc_PhylipPluginTests.obj
 0001:0003f1e0       __unwindfunclet$??__EuserActLog@U2@@YAXXZ$0 100401e0 f   moc_PhylipPluginTests.obj
 0001:0003f1e9       __ehhandler$??__EuserActLog@U2@@YAXXZ 100401e9 f   moc_PhylipPluginTests.obj
 0001:0003f210       __unwindfunclet$??__EalgoLog@U2@@YAXXZ$0 10040210 f   moc_PhylipTask.obj
 0001:0003f219       __ehhandler$??__EalgoLog@U2@@YAXXZ 10040219 f   moc_PhylipTask.obj
 0001:0003f240       __unwindfunclet$??__EcmdLog@U2@@YAXXZ$0 10040240 f   moc_PhylipTask.obj
 0001:0003f249       __ehhandler$??__EcmdLog@U2@@YAXXZ 10040249 f   moc_PhylipTask.obj
 0001:0003f270       __unwindfunclet$??__EcoreLog@U2@@YAXXZ$0 10040270 f   moc_PhylipTask.obj
 0001:0003f279       __ehhandler$??__EcoreLog@U2@@YAXXZ 10040279 f   moc_PhylipTask.obj
 0001:0003f2a0       __unwindfunclet$??__EioLog@U2@@YAXXZ$0 100402a0 f   moc_PhylipTask.obj
 0001:0003f2a9       __ehhandler$??__EioLog@U2@@YAXXZ 100402a9 f   moc_PhylipTask.obj
 0001:0003f2d0       __unwindfunclet$??__EperfLog@U2@@YAXXZ$0 100402d0 f   moc_PhylipTask.obj
 0001:0003f2d9       __ehhandler$??__EperfLog@U2@@YAXXZ 100402d9 f   moc_PhylipTask.obj
 0001:0003f300       __unwindfunclet$??__EscriptLog@U2@@YAXXZ$0 10040300 f   moc_PhylipTask.obj
 0001:0003f309       __ehhandler$??__EscriptLog@U2@@YAXXZ 10040309 f   moc_PhylipTask.obj
 0001:0003f330       __unwindfunclet$??__EtaskLog@U2@@YAXXZ$0 10040330 f   moc_PhylipTask.obj
 0001:0003f339       __ehhandler$??__EtaskLog@U2@@YAXXZ 10040339 f   moc_PhylipTask.obj
 0001:0003f360       __unwindfunclet$??__EuiLog@U2@@YAXXZ$0 10040360 f   moc_PhylipTask.obj
 0001:0003f369       __ehhandler$??__EuiLog@U2@@YAXXZ 10040369 f   moc_PhylipTask.obj
 0001:0003f390       __unwindfunclet$??__EuserActLog@U2@@YAXXZ$0 10040390 f   moc_PhylipTask.obj
 0001:0003f399       __ehhandler$??__EuserActLog@U2@@YAXXZ 10040399 f   moc_PhylipTask.obj
 0001:0003f3c0       ??__F?_Generic_object@?$_Error_objects@H@std@@2V_Generic_error_category@2@A@@YAXXZ 100403c0 f   DistanceMatrix.obj
 0001:0003f3d0       ??__F?_Iostream_object@?$_Error_objects@H@std@@2V_Iostream_error_category@2@A@@YAXXZ 100403d0 f   DistanceMatrix.obj
 0001:0003f3e0       ??__F?_System_object@?$_Error_objects@H@std@@2V_System_error_category@2@A@@YAXXZ 100403e0 f   DistanceMatrix.obj
 0001:0003f3f0       ??__FalgoLog@U2@@YAXXZ     100403f0 f   DistanceMatrix.obj
 0001:0003f400       ??__FcmdLog@U2@@YAXXZ      10040400 f   DistanceMatrix.obj
 0001:0003f410       ??__FcoreLog@U2@@YAXXZ     10040410 f   DistanceMatrix.obj
 0001:0003f420       ??__FioLog@U2@@YAXXZ       10040420 f   DistanceMatrix.obj
 0001:0003f430       ??__FperfLog@U2@@YAXXZ     10040430 f   DistanceMatrix.obj
 0001:0003f440       ??__FscriptLog@U2@@YAXXZ   10040440 f   DistanceMatrix.obj
 0001:0003f450       ??__FtaskLog@U2@@YAXXZ     10040450 f   DistanceMatrix.obj
 0001:0003f460       ??__FuiLog@U2@@YAXXZ       10040460 f   DistanceMatrix.obj
 0001:0003f470       ??__FuserActLog@U2@@YAXXZ  10040470 f   DistanceMatrix.obj
 0001:0003f480       ??__F?_Generic_object@?$_Error_objects@H@std@@2V_Generic_error_category@2@A@@YAXXZ 10040480 f   NeighborJoinAdapter.obj
 0001:0003f490       ??__F?_Iostream_object@?$_Error_objects@H@std@@2V_Iostream_error_category@2@A@@YAXXZ 10040490 f   NeighborJoinAdapter.obj
 0001:0003f4a0       ??__F?_System_object@?$_Error_objects@H@std@@2V_System_error_category@2@A@@YAXXZ 100404a0 f   NeighborJoinAdapter.obj
 0001:0003f4b0       ??__F?runLock@NeighborJoinCalculateTreeTask@U2@@0VQMutex@@A@@YAXXZ 100404b0 f   NeighborJoinAdapter.obj
 0001:0003f4c0       ??__FalgoLog@U2@@YAXXZ     100404c0 f   NeighborJoinAdapter.obj
 0001:0003f4d0       ??__FcmdLog@U2@@YAXXZ      100404d0 f   NeighborJoinAdapter.obj
 0001:0003f4e0       ??__FcoreLog@U2@@YAXXZ     100404e0 f   NeighborJoinAdapter.obj
 0001:0003f4f0       ??__Fcvar@?1??run@NeighborJoinCalculateTreeTask@U2@@UAEXXZ@YAXXZ 100404f0 f   NeighborJoinAdapter.obj
 0001:0003f500       ??__FioLog@U2@@YAXXZ       10040500 f   NeighborJoinAdapter.obj
 0001:0003f510       ??__FperfLog@U2@@YAXXZ     10040510 f   NeighborJoinAdapter.obj
 0001:0003f520       ??__FscriptLog@U2@@YAXXZ   10040520 f   NeighborJoinAdapter.obj
 0001:0003f530       ??__FtaskLog@U2@@YAXXZ     10040530 f   NeighborJoinAdapter.obj
 0001:0003f540       ??__FuiLog@U2@@YAXXZ       10040540 f   NeighborJoinAdapter.obj
 0001:0003f550       ??__FuserActLog@U2@@YAXXZ  10040550 f   NeighborJoinAdapter.obj
 0001:0003f560       ??__F?M1@ConsensusModelTypes@U2@@2VQString@@A@@YAXXZ 10040560 f   NeighborJoinWidget.obj
 0001:0003f570       ??__F?MajorityRule@ConsensusModelTypes@U2@@2VQString@@A@@YAXXZ 10040570 f   NeighborJoinWidget.obj
 0001:0003f580       ??__F?MajorityRuleExt@ConsensusModelTypes@U2@@2VQString@@A@@YAXXZ 10040580 f   NeighborJoinWidget.obj
 0001:0003f590       ??__F?Strict@ConsensusModelTypes@U2@@2VQString@@A@@YAXXZ 10040590 f   NeighborJoinWidget.obj
 0001:0003f5a0       ??__F?_Generic_object@?$_Error_objects@H@std@@2V_Generic_error_category@2@A@@YAXXZ 100405a0 f   NeighborJoinWidget.obj
 0001:0003f5b0       ??__F?_Iostream_object@?$_Error_objects@H@std@@2V_Iostream_error_category@2@A@@YAXXZ 100405b0 f   NeighborJoinWidget.obj
 0001:0003f5c0       ??__F?_System_object@?$_Error_objects@H@std@@2V_System_error_category@2@A@@YAXXZ 100405c0 f   NeighborJoinWidget.obj
 0001:0003f5d0       ??__FalgoLog@U2@@YAXXZ     100405d0 f   NeighborJoinWidget.obj
 0001:0003f5e0       ??__FcmdLog@U2@@YAXXZ      100405e0 f   NeighborJoinWidget.obj
 0001:0003f5f0       ??__FcoreLog@U2@@YAXXZ     100405f0 f   NeighborJoinWidget.obj
 0001:0003f600       ??__FioLog@U2@@YAXXZ       10040600 f   NeighborJoinWidget.obj
 0001:0003f610       ??__Flist@?1??getConsensusModelTypes@ConsensusModelTypes@U2@@SA?AV?$QList@VQString@@@@XZ@YAXXZ 10040610 f   NeighborJoinWidget.obj
 0001:0003f620       ??__FperfLog@U2@@YAXXZ     10040620 f   NeighborJoinWidget.obj
 0001:0003f630       ??__FscriptLog@U2@@YAXXZ   10040630 f   NeighborJoinWidget.obj
 0001:0003f640       ??__FtaskLog@U2@@YAXXZ     10040640 f   NeighborJoinWidget.obj
 0001:0003f650       ??__FuiLog@U2@@YAXXZ       10040650 f   NeighborJoinWidget.obj
 0001:0003f660       ??__FuserActLog@U2@@YAXXZ  10040660 f   NeighborJoinWidget.obj
 0001:0003f670       ??__F?ALPHA_ARG@PhylipCmdlineTask@U2@@2VQString@@B@@YAXXZ 10040670 f   PhylipCmdlineTask.obj
 0001:0003f680       ??__F?BOOTSTRAP_ARG@PhylipCmdlineTask@U2@@2VQString@@B@@YAXXZ 10040680 f   PhylipCmdlineTask.obj
 0001:0003f690       ??__F?CONSENSUS_ARG@PhylipCmdlineTask@U2@@2VQString@@B@@YAXXZ 10040690 f   PhylipCmdlineTask.obj
 0001:0003f6a0       ??__F?FRACTION_ARG@PhylipCmdlineTask@U2@@2VQString@@B@@YAXXZ 100406a0 f   PhylipCmdlineTask.obj
 0001:0003f6b0       ??__F?GAMMA_ARG@PhylipCmdlineTask@U2@@2VQString@@B@@YAXXZ 100406b0 f   PhylipCmdlineTask.obj
 0001:0003f6c0       ??__F?MATRIX_ARG@PhylipCmdlineTask@U2@@2VQString@@B@@YAXXZ 100406c0 f   PhylipCmdlineTask.obj
 0001:0003f6d0       ??__F?PHYLIP_CMDLINE@PhylipCmdlineTask@U2@@2VQString@@B@@YAXXZ 100406d0 f   PhylipCmdlineTask.obj
 0001:0003f6e0       ??__F?REPLICATES_ARG@PhylipCmdlineTask@U2@@2VQString@@B@@YAXXZ 100406e0 f   PhylipCmdlineTask.obj
 0001:0003f6f0       ??__F?SEED_ARG@PhylipCmdlineTask@U2@@2VQString@@B@@YAXXZ 100406f0 f   PhylipCmdlineTask.obj
 0001:0003f700       ??__F?TT_RATIO_ARG@PhylipCmdlineTask@U2@@2VQString@@B@@YAXXZ 10040700 f   PhylipCmdlineTask.obj
 0001:0003f710       ??__F?_Generic_object@?$_Error_objects@H@std@@2V_Generic_error_category@2@A@@YAXXZ 10040710 f   PhylipCmdlineTask.obj
 0001:0003f720       ??__F?_Iostream_object@?$_Error_objects@H@std@@2V_Iostream_error_category@2@A@@YAXXZ 10040720 f   PhylipCmdlineTask.obj
 0001:0003f730       ??__F?_System_object@?$_Error_objects@H@std@@2V_System_error_category@2@A@@YAXXZ 10040730 f   PhylipCmdlineTask.obj
 0001:0003f740       ??__FalgoLog@U2@@YAXXZ     10040740 f   PhylipCmdlineTask.obj
 0001:0003f750       ??__FcmdLog@U2@@YAXXZ      10040750 f   PhylipCmdlineTask.obj
 0001:0003f760       ??__FcoreLog@U2@@YAXXZ     10040760 f   PhylipCmdlineTask.obj
 0001:0003f770       ??__FioLog@U2@@YAXXZ       10040770 f   PhylipCmdlineTask.obj
 0001:0003f780       ??__FperfLog@U2@@YAXXZ     10040780 f   PhylipCmdlineTask.obj
 0001:0003f790       ??__FscriptLog@U2@@YAXXZ   10040790 f   PhylipCmdlineTask.obj
 0001:0003f7a0       ??__FtaskLog@U2@@YAXXZ     100407a0 f   PhylipCmdlineTask.obj
 0001:0003f7b0       ??__FuiLog@U2@@YAXXZ       100407b0 f   PhylipCmdlineTask.obj
 0001:0003f7c0       ??__FuserActLog@U2@@YAXXZ  100407c0 f   PhylipCmdlineTask.obj
 0001:0003f7d0       ??__F?PHYLIP_NEIGHBOUR_JOIN@PhylipPlugin@U2@@2VQString@@B@@YAXXZ 100407d0 f   PhylipPlugin.obj
 0001:0003f7e0       ??__F?_Generic_object@?$_Error_objects@H@std@@2V_Generic_error_category@2@A@@YAXXZ 100407e0 f   PhylipPlugin.obj
 0001:0003f7f0       ??__F?_Iostream_object@?$_Error_objects@H@std@@2V_Iostream_error_category@2@A@@YAXXZ 100407f0 f   PhylipPlugin.obj
 0001:0003f800       ??__F?_System_object@?$_Error_objects@H@std@@2V_System_error_category@2@A@@YAXXZ 10040800 f   PhylipPlugin.obj
 0001:0003f810       ??__FService_DNAExport@U2@@YAXXZ 10040810 f   PhylipPlugin.obj
 0001:0003f820       ??__FService_DNAGraphPack@U2@@YAXXZ 10040820 f   PhylipPlugin.obj
 0001:0003f830       ??__FService_ExternalToolSupport@U2@@YAXXZ 10040830 f   PhylipPlugin.obj
 0001:0003f840       ??__FService_GUITesting@U2@@YAXXZ 10040840 f   PhylipPlugin.obj
 0001:0003f850       ??__FService_MaxCoreServiceId@U2@@YAXXZ 10040850 f   PhylipPlugin.obj
 0001:0003f860       ??__FService_MinCoreServiceId@U2@@YAXXZ 10040860 f   PhylipPlugin.obj
 0001:0003f870       ??__FService_PluginViewer@U2@@YAXXZ 10040870 f   PhylipPlugin.obj
 0001:0003f880       ??__FService_Project@U2@@YAXXZ 10040880 f   PhylipPlugin.obj
 0001:0003f890       ??__FService_ProjectView@U2@@YAXXZ 10040890 f   PhylipPlugin.obj
 0001:0003f8a0       ??__FService_QueryDesigner@U2@@YAXXZ 100408a0 f   PhylipPlugin.obj
 0001:0003f8b0       ??__FService_ScriptRegistry@U2@@YAXXZ 100408b0 f   PhylipPlugin.obj
 0001:0003f8c0       ??__FService_TestRunner@U2@@YAXXZ 100408c0 f   PhylipPlugin.obj
 0001:0003f8d0       ??__FService_WorkflowDesigner@U2@@YAXXZ 100408d0 f   PhylipPlugin.obj
 0001:0003f8e0       ??__FalgoLog@U2@@YAXXZ     100408e0 f   PhylipPlugin.obj
 0001:0003f8f0       ??__FcmdLog@U2@@YAXXZ      100408f0 f   PhylipPlugin.obj
 0001:0003f900       ??__FcoreLog@U2@@YAXXZ     10040900 f   PhylipPlugin.obj
 0001:0003f910       ??__FioLog@U2@@YAXXZ       10040910 f   PhylipPlugin.obj
 0001:0003f920       ??__FperfLog@U2@@YAXXZ     10040920 f   PhylipPlugin.obj
 0001:0003f930       ??__FscriptLog@U2@@YAXXZ   10040930 f   PhylipPlugin.obj
 0001:0003f940       ??__FtaskLog@U2@@YAXXZ     10040940 f   PhylipPlugin.obj
 0001:0003f950       ??__FuiLog@U2@@YAXXZ       10040950 f   PhylipPlugin.obj
 0001:0003f960       ??__FuserActLog@U2@@YAXXZ  10040960 f   PhylipPlugin.obj
 0001:0003f970       ??__F?_Generic_object@?$_Error_objects@H@std@@2V_Generic_error_category@2@A@@YAXXZ 10040970 f   PhylipPluginTests.obj
 0001:0003f980       ??__F?_Iostream_object@?$_Error_objects@H@std@@2V_Iostream_error_category@2@A@@YAXXZ 10040980 f   PhylipPluginTests.obj
 0001:0003f990       ??__F?_System_object@?$_Error_objects@H@std@@2V_System_error_category@2@A@@YAXXZ 10040990 f   PhylipPluginTests.obj
 0001:0003f9a0       ??__FService_DNAExport@U2@@YAXXZ 100409a0 f   PhylipPluginTests.obj
 0001:0003f9b0       ??__FService_DNAGraphPack@U2@@YAXXZ 100409b0 f   PhylipPluginTests.obj
 0001:0003f9c0       ??__FService_ExternalToolSupport@U2@@YAXXZ 100409c0 f   PhylipPluginTests.obj
 0001:0003f9d0       ??__FService_GUITesting@U2@@YAXXZ 100409d0 f   PhylipPluginTests.obj
 0001:0003f9e0       ??__FService_MaxCoreServiceId@U2@@YAXXZ 100409e0 f   PhylipPluginTests.obj
 0001:0003f9f0       ??__FService_MinCoreServiceId@U2@@YAXXZ 100409f0 f   PhylipPluginTests.obj
 0001:0003fa00       ??__FService_PluginViewer@U2@@YAXXZ 10040a00 f   PhylipPluginTests.obj
 0001:0003fa10       ??__FService_Project@U2@@YAXXZ 10040a10 f   PhylipPluginTests.obj
 0001:0003fa20       ??__FService_ProjectView@U2@@YAXXZ 10040a20 f   PhylipPluginTests.obj
 0001:0003fa30       ??__FService_QueryDesigner@U2@@YAXXZ 10040a30 f   PhylipPluginTests.obj
 0001:0003fa40       ??__FService_ScriptRegistry@U2@@YAXXZ 10040a40 f   PhylipPluginTests.obj
 0001:0003fa50       ??__FService_TestRunner@U2@@YAXXZ 10040a50 f   PhylipPluginTests.obj
 0001:0003fa60       ??__FService_WorkflowDesigner@U2@@YAXXZ 10040a60 f   PhylipPluginTests.obj
 0001:0003fa70       ??__FalgoLog@U2@@YAXXZ     10040a70 f   PhylipPluginTests.obj
 0001:0003fa80       ??__FcmdLog@U2@@YAXXZ      10040a80 f   PhylipPluginTests.obj
 0001:0003fa90       ??__FcoreLog@U2@@YAXXZ     10040a90 f   PhylipPluginTests.obj
 0001:0003faa0       ??__FioLog@U2@@YAXXZ       10040aa0 f   PhylipPluginTests.obj
 0001:0003fab0       ??__FperfLog@U2@@YAXXZ     10040ab0 f   PhylipPluginTests.obj
 0001:0003fac0       ??__FscriptLog@U2@@YAXXZ   10040ac0 f   PhylipPluginTests.obj
 0001:0003fad0       ??__FtaskLog@U2@@YAXXZ     10040ad0 f   PhylipPluginTests.obj
 0001:0003fae0       ??__FuiLog@U2@@YAXXZ       10040ae0 f   PhylipPluginTests.obj
 0001:0003faf0       ??__FuserActLog@U2@@YAXXZ  10040af0 f   PhylipPluginTests.obj
 0001:0003fb00       ??__F?_Generic_object@?$_Error_objects@H@std@@2V_Generic_error_category@2@A@@YAXXZ 10040b00 f   PhylipTask.obj
 0001:0003fb10       ??__F?_Iostream_object@?$_Error_objects@H@std@@2V_Iostream_error_category@2@A@@YAXXZ 10040b10 f   PhylipTask.obj
 0001:0003fb20       ??__F?_System_object@?$_Error_objects@H@std@@2V_System_error_category@2@A@@YAXXZ 10040b20 f   PhylipTask.obj
 0001:0003fb30       ??__FalgoLog@U2@@YAXXZ     10040b30 f   PhylipTask.obj
 0001:0003fb40       ??__FcmdLog@U2@@YAXXZ      10040b40 f   PhylipTask.obj
 0001:0003fb50       ??__FcoreLog@U2@@YAXXZ     10040b50 f   PhylipTask.obj
 0001:0003fb60       ??__FioLog@U2@@YAXXZ       10040b60 f   PhylipTask.obj
 0001:0003fb70       ??__FperfLog@U2@@YAXXZ     10040b70 f   PhylipTask.obj
 0001:0003fb80       ??__FscriptLog@U2@@YAXXZ   10040b80 f   PhylipTask.obj
 0001:0003fb90       ??__FtaskLog@U2@@YAXXZ     10040b90 f   PhylipTask.obj
 0001:0003fba0       ??__FuiLog@U2@@YAXXZ       10040ba0 f   PhylipTask.obj
 0001:0003fbb0       ??__FuserActLog@U2@@YAXXZ  10040bb0 f   PhylipTask.obj
 0001:0003fbc0       ??__F?_Generic_object@?$_Error_objects@H@std@@2V_Generic_error_category@2@A@@YAXXZ 10040bc0 f   SeqBootAdapter.obj
 0001:0003fbd0       ??__F?_Iostream_object@?$_Error_objects@H@std@@2V_Iostream_error_category@2@A@@YAXXZ 10040bd0 f   SeqBootAdapter.obj
 0001:0003fbe0       ??__F?_System_object@?$_Error_objects@H@std@@2V_System_error_category@2@A@@YAXXZ 10040be0 f   SeqBootAdapter.obj
 0001:0003fbf0       ??__FalgoLog@U2@@YAXXZ     10040bf0 f   SeqBootAdapter.obj
 0001:0003fc00       ??__FcmdLog@U2@@YAXXZ      10040c00 f   SeqBootAdapter.obj
 0001:0003fc10       ??__FcoreLog@U2@@YAXXZ     10040c10 f   SeqBootAdapter.obj
 0001:0003fc20       ??__FioLog@U2@@YAXXZ       10040c20 f   SeqBootAdapter.obj
 0001:0003fc30       ??__FperfLog@U2@@YAXXZ     10040c30 f   SeqBootAdapter.obj
 0001:0003fc40       ??__FscriptLog@U2@@YAXXZ   10040c40 f   SeqBootAdapter.obj
 0001:0003fc50       ??__FtaskLog@U2@@YAXXZ     10040c50 f   SeqBootAdapter.obj
 0001:0003fc60       ??__FuiLog@U2@@YAXXZ       10040c60 f   SeqBootAdapter.obj
 0001:0003fc70       ??__FuserActLog@U2@@YAXXZ  10040c70 f   SeqBootAdapter.obj
 0001:0003fc80       ??__F?_Generic_object@?$_Error_objects@H@std@@2V_Generic_error_category@2@A@@YAXXZ 10040c80 f   dist.obj
 0001:0003fc90       ??__F?_Iostream_object@?$_Error_objects@H@std@@2V_Iostream_error_category@2@A@@YAXXZ 10040c90 f   dist.obj
 0001:0003fca0       ??__F?_System_object@?$_Error_objects@H@std@@2V_System_error_category@2@A@@YAXXZ 10040ca0 f   dist.obj
 0001:0003fcb0       ??__FalgoLog@U2@@YAXXZ     10040cb0 f   dist.obj
 0001:0003fcc0       ??__FcmdLog@U2@@YAXXZ      10040cc0 f   dist.obj
 0001:0003fcd0       ??__FcoreLog@U2@@YAXXZ     10040cd0 f   dist.obj
 0001:0003fce0       ??__FioLog@U2@@YAXXZ       10040ce0 f   dist.obj
 0001:0003fcf0       ??__FperfLog@U2@@YAXXZ     10040cf0 f   dist.obj
 0001:0003fd00       ??__FscriptLog@U2@@YAXXZ   10040d00 f   dist.obj
 0001:0003fd10       ??__FtaskLog@U2@@YAXXZ     10040d10 f   dist.obj
 0001:0003fd20       ??__FuiLog@U2@@YAXXZ       10040d20 f   dist.obj
 0001:0003fd30       ??__FuserActLog@U2@@YAXXZ  10040d30 f   dist.obj
 0001:0003fd40       ??__F?F84@DNADistModelTypes@@2VQString@@A@@YAXXZ 10040d40 f   dnadist.obj
 0001:0003fd50       ??__F?JukesCantor@DNADistModelTypes@@2VQString@@A@@YAXXZ 10040d50 f   dnadist.obj
 0001:0003fd60       ??__F?Kimura@DNADistModelTypes@@2VQString@@A@@YAXXZ 10040d60 f   dnadist.obj
 0001:0003fd70       ??__F?LogDet@DNADistModelTypes@@2VQString@@A@@YAXXZ 10040d70 f   dnadist.obj
 0001:0003fd80       ??__F?_Generic_object@?$_Error_objects@H@std@@2V_Generic_error_category@2@A@@YAXXZ 10040d80 f   dnadist.obj
 0001:0003fd90       ??__F?_Iostream_object@?$_Error_objects@H@std@@2V_Iostream_error_category@2@A@@YAXXZ 10040d90 f   dnadist.obj
 0001:0003fda0       ??__F?_System_object@?$_Error_objects@H@std@@2V_System_error_category@2@A@@YAXXZ 10040da0 f   dnadist.obj
 0001:0003fdb0       ??__FalgoLog@U2@@YAXXZ     10040db0 f   dnadist.obj
 0001:0003fdc0       ??__FcmdLog@U2@@YAXXZ      10040dc0 f   dnadist.obj
 0001:0003fdd0       ??__FcoreLog@U2@@YAXXZ     10040dd0 f   dnadist.obj
 0001:0003fde0       ??__FdnaDistSettings@@YAXXZ 10040de0 f   dnadist.obj
 0001:0003fdf0       ??__FioLog@U2@@YAXXZ       10040df0 f   dnadist.obj
 0001:0003fe00       ??__Flist@?1??getDNADistModelTypes@DNADistModelTypes@@SA?AV?$QList@VQString@@@@XZ@YAXXZ 10040e00 f   dnadist.obj
 0001:0003fe10       ??__FperfLog@U2@@YAXXZ     10040e10 f   dnadist.obj
 0001:0003fe20       ??__FscriptLog@U2@@YAXXZ   10040e20 f   dnadist.obj
 0001:0003fe30       ??__FtaskLog@U2@@YAXXZ     10040e30 f   dnadist.obj
 0001:0003fe40       ??__FuiLog@U2@@YAXXZ       10040e40 f   dnadist.obj
 0001:0003fe50       ??__FuserActLog@U2@@YAXXZ  10040e50 f   dnadist.obj
 0001:0003fe60       ??__F?_Generic_object@?$_Error_objects@H@std@@2V_Generic_error_category@2@A@@YAXXZ 10040e60 f   neighbor.obj
 0001:0003fe70       ??__F?_Iostream_object@?$_Error_objects@H@std@@2V_Iostream_error_category@2@A@@YAXXZ 10040e70 f   neighbor.obj
 0001:0003fe80       ??__F?_System_object@?$_Error_objects@H@std@@2V_System_error_category@2@A@@YAXXZ 10040e80 f   neighbor.obj
 0001:0003fe90       ??__FalgoLog@U2@@YAXXZ     10040e90 f   neighbor.obj
 0001:0003fea0       ??__FcmdLog@U2@@YAXXZ      10040ea0 f   neighbor.obj
 0001:0003feb0       ??__FcoreLog@U2@@YAXXZ     10040eb0 f   neighbor.obj
 0001:0003fec0       ??__FioLog@U2@@YAXXZ       10040ec0 f   neighbor.obj
 0001:0003fed0       ??__FperfLog@U2@@YAXXZ     10040ed0 f   neighbor.obj
 0001:0003fee0       ??__FscriptLog@U2@@YAXXZ   10040ee0 f   neighbor.obj
 0001:0003fef0       ??__FtaskLog@U2@@YAXXZ     10040ef0 f   neighbor.obj
 0001:0003ff00       ??__FuiLog@U2@@YAXXZ       10040f00 f   neighbor.obj
 0001:0003ff10       ??__FuserActLog@U2@@YAXXZ  10040f10 f   neighbor.obj
 0001:0003ff20       ??__F?_Generic_object@?$_Error_objects@H@std@@2V_Generic_error_category@2@A@@YAXXZ 10040f20 f   phylip.obj
 0001:0003ff30       ??__F?_Iostream_object@?$_Error_objects@H@std@@2V_Iostream_error_category@2@A@@YAXXZ 10040f30 f   phylip.obj
 0001:0003ff40       ??__F?_System_object@?$_Error_objects@H@std@@2V_System_error_category@2@A@@YAXXZ 10040f40 f   phylip.obj
 0001:0003ff50       ??__FalgoLog@U2@@YAXXZ     10040f50 f   phylip.obj
 0001:0003ff60       ??__FcmdLog@U2@@YAXXZ      10040f60 f   phylip.obj
 0001:0003ff70       ??__FcoreLog@U2@@YAXXZ     10040f70 f   phylip.obj
 0001:0003ff80       ??__FioLog@U2@@YAXXZ       10040f80 f   phylip.obj
 0001:0003ff90       ??__FperfLog@U2@@YAXXZ     10040f90 f   phylip.obj
 0001:0003ffa0       ??__FscriptLog@U2@@YAXXZ   10040fa0 f   phylip.obj
 0001:0003ffb0       ??__FtaskLog@U2@@YAXXZ     10040fb0 f   phylip.obj
 0001:0003ffc0       ??__FuiLog@U2@@YAXXZ       10040fc0 f   phylip.obj
 0001:0003ffd0       ??__FuserActLog@U2@@YAXXZ  10040fd0 f   phylip.obj
 0001:0003ffe0       ??__F?JTT@ProtDistModelTypes@@2VQString@@A@@YAXXZ 10040fe0 f   protdist.obj
 0001:0003fff0       ??__F?Kimura@ProtDistModelTypes@@2VQString@@A@@YAXXZ 10040ff0 f   protdist.obj
 0001:00040000       ??__F?PAM@ProtDistModelTypes@@2VQString@@A@@YAXXZ 10041000 f   protdist.obj
 0001:00040010       ??__F?PMB@ProtDistModelTypes@@2VQString@@A@@YAXXZ 10041010 f   protdist.obj
 0001:00040020       ??__F?_Generic_object@?$_Error_objects@H@std@@2V_Generic_error_category@2@A@@YAXXZ 10041020 f   protdist.obj
 0001:00040030       ??__F?_Iostream_object@?$_Error_objects@H@std@@2V_Iostream_error_category@2@A@@YAXXZ 10041030 f   protdist.obj
 0001:00040040       ??__F?_System_object@?$_Error_objects@H@std@@2V_System_error_category@2@A@@YAXXZ 10041040 f   protdist.obj
 0001:00040050       ??__FalgoLog@U2@@YAXXZ     10041050 f   protdist.obj
 0001:00040060       ??__FcmdLog@U2@@YAXXZ      10041060 f   protdist.obj
 0001:00040070       ??__FcoreLog@U2@@YAXXZ     10041070 f   protdist.obj
 0001:00040080       ??__FioLog@U2@@YAXXZ       10041080 f   protdist.obj
 0001:00040090       ??__Flist@?1??getProtDistModelTypes@ProtDistModelTypes@@SA?AV?$QList@VQString@@@@XZ@YAXXZ 10041090 f   protdist.obj
 0001:000400a0       ??__FperfLog@U2@@YAXXZ     100410a0 f   protdist.obj
 0001:000400b0       ??__FscriptLog@U2@@YAXXZ   100410b0 f   protdist.obj
 0001:000400c0       ??__FtaskLog@U2@@YAXXZ     100410c0 f   protdist.obj
 0001:000400d0       ??__FuiLog@U2@@YAXXZ       100410d0 f   protdist.obj
 0001:000400e0       ??__FuserActLog@U2@@YAXXZ  100410e0 f   protdist.obj
 0001:000400f0       ??__F?_Generic_object@?$_Error_objects@H@std@@2V_Generic_error_category@2@A@@YAXXZ 100410f0 f   seqboot.obj
 0001:00040100       ??__F?_Iostream_object@?$_Error_objects@H@std@@2V_Iostream_error_category@2@A@@YAXXZ 10041100 f   seqboot.obj
 0001:00040110       ??__F?_System_object@?$_Error_objects@H@std@@2V_System_error_category@2@A@@YAXXZ 10041110 f   seqboot.obj
 0001:00040120       ??__FalgoLog@U2@@YAXXZ     10041120 f   seqboot.obj
 0001:00040130       ??__FcmdLog@U2@@YAXXZ      10041130 f   seqboot.obj
 0001:00040140       ??__FcoreLog@U2@@YAXXZ     10041140 f   seqboot.obj
 0001:00040150       ??__FioLog@U2@@YAXXZ       10041150 f   seqboot.obj
 0001:00040160       ??__FperfLog@U2@@YAXXZ     10041160 f   seqboot.obj
 0001:00040170       ??__FscriptLog@U2@@YAXXZ   10041170 f   seqboot.obj
 0001:00040180       ??__FtaskLog@U2@@YAXXZ     10041180 f   seqboot.obj
 0001:00040190       ??__FuiLog@U2@@YAXXZ       10041190 f   seqboot.obj
 0001:000401a0       ??__FuserActLog@U2@@YAXXZ  100411a0 f   seqboot.obj
 0001:000401b0       ??__F?_Generic_object@?$_Error_objects@H@std@@2V_Generic_error_category@2@A@@YAXXZ 100411b0 f   moc_NeighborJoinWidget.obj
 0001:000401c0       ??__F?_Iostream_object@?$_Error_objects@H@std@@2V_Iostream_error_category@2@A@@YAXXZ 100411c0 f   moc_NeighborJoinWidget.obj
 0001:000401d0       ??__F?_System_object@?$_Error_objects@H@std@@2V_System_error_category@2@A@@YAXXZ 100411d0 f   moc_NeighborJoinWidget.obj
 0001:000401e0       ??__FalgoLog@U2@@YAXXZ     100411e0 f   moc_NeighborJoinWidget.obj
 0001:000401f0       ??__FcmdLog@U2@@YAXXZ      100411f0 f   moc_NeighborJoinWidget.obj
 0001:00040200       ??__FcoreLog@U2@@YAXXZ     10041200 f   moc_NeighborJoinWidget.obj
 0001:00040210       ??__FioLog@U2@@YAXXZ       10041210 f   moc_NeighborJoinWidget.obj
 0001:00040220       ??__FperfLog@U2@@YAXXZ     10041220 f   moc_NeighborJoinWidget.obj
 0001:00040230       ??__FscriptLog@U2@@YAXXZ   10041230 f   moc_NeighborJoinWidget.obj
 0001:00040240       ??__FtaskLog@U2@@YAXXZ     10041240 f   moc_NeighborJoinWidget.obj
 0001:00040250       ??__FuiLog@U2@@YAXXZ       10041250 f   moc_NeighborJoinWidget.obj
 0001:00040260       ??__FuserActLog@U2@@YAXXZ  10041260 f   moc_NeighborJoinWidget.obj
 0001:00040270       ??__F?_Generic_object@?$_Error_objects@H@std@@2V_Generic_error_category@2@A@@YAXXZ 10041270 f   moc_PhylipCmdlineTask.obj
 0001:00040280       ??__F?_Iostream_object@?$_Error_objects@H@std@@2V_Iostream_error_category@2@A@@YAXXZ 10041280 f   moc_PhylipCmdlineTask.obj
 0001:00040290       ??__F?_System_object@?$_Error_objects@H@std@@2V_System_error_category@2@A@@YAXXZ 10041290 f   moc_PhylipCmdlineTask.obj
 0001:000402a0       ??__FalgoLog@U2@@YAXXZ     100412a0 f   moc_PhylipCmdlineTask.obj
 0001:000402b0       ??__FcmdLog@U2@@YAXXZ      100412b0 f   moc_PhylipCmdlineTask.obj
 0001:000402c0       ??__FcoreLog@U2@@YAXXZ     100412c0 f   moc_PhylipCmdlineTask.obj
 0001:000402d0       ??__FioLog@U2@@YAXXZ       100412d0 f   moc_PhylipCmdlineTask.obj
 0001:000402e0       ??__FperfLog@U2@@YAXXZ     100412e0 f   moc_PhylipCmdlineTask.obj
 0001:000402f0       ??__FscriptLog@U2@@YAXXZ   100412f0 f   moc_PhylipCmdlineTask.obj
 0001:00040300       ??__FtaskLog@U2@@YAXXZ     10041300 f   moc_PhylipCmdlineTask.obj
 0001:00040310       ??__FuiLog@U2@@YAXXZ       10041310 f   moc_PhylipCmdlineTask.obj
 0001:00040320       ??__FuserActLog@U2@@YAXXZ  10041320 f   moc_PhylipCmdlineTask.obj
 0001:00040330       ??__F?_Generic_object@?$_Error_objects@H@std@@2V_Generic_error_category@2@A@@YAXXZ 10041330 f   moc_PhylipPlugin.obj
 0001:00040340       ??__F?_Iostream_object@?$_Error_objects@H@std@@2V_Iostream_error_category@2@A@@YAXXZ 10041340 f   moc_PhylipPlugin.obj
 0001:00040350       ??__F?_System_object@?$_Error_objects@H@std@@2V_System_error_category@2@A@@YAXXZ 10041350 f   moc_PhylipPlugin.obj
 0001:00040360       ??__FService_DNAExport@U2@@YAXXZ 10041360 f   moc_PhylipPlugin.obj
 0001:00040370       ??__FService_DNAGraphPack@U2@@YAXXZ 10041370 f   moc_PhylipPlugin.obj
 0001:00040380       ??__FService_ExternalToolSupport@U2@@YAXXZ 10041380 f   moc_PhylipPlugin.obj
 0001:00040390       ??__FService_GUITesting@U2@@YAXXZ 10041390 f   moc_PhylipPlugin.obj
 0001:000403a0       ??__FService_MaxCoreServiceId@U2@@YAXXZ 100413a0 f   moc_PhylipPlugin.obj
 0001:000403b0       ??__FService_MinCoreServiceId@U2@@YAXXZ 100413b0 f   moc_PhylipPlugin.obj
 0001:000403c0       ??__FService_PluginViewer@U2@@YAXXZ 100413c0 f   moc_PhylipPlugin.obj
 0001:000403d0       ??__FService_Project@U2@@YAXXZ 100413d0 f   moc_PhylipPlugin.obj
 0001:000403e0       ??__FService_ProjectView@U2@@YAXXZ 100413e0 f   moc_PhylipPlugin.obj
 0001:000403f0       ??__FService_QueryDesigner@U2@@YAXXZ 100413f0 f   moc_PhylipPlugin.obj
 0001:00040400       ??__FService_ScriptRegistry@U2@@YAXXZ 10041400 f   moc_PhylipPlugin.obj
 0001:00040410       ??__FService_TestRunner@U2@@YAXXZ 10041410 f   moc_PhylipPlugin.obj
 0001:00040420       ??__FService_WorkflowDesigner@U2@@YAXXZ 10041420 f   moc_PhylipPlugin.obj
 0001:00040430       ??__F?_Generic_object@?$_Error_objects@H@std@@2V_Generic_error_category@2@A@@YAXXZ 10041430 f   moc_PhylipPluginTests.obj
 0001:00040440       ??__F?_Iostream_object@?$_Error_objects@H@std@@2V_Iostream_error_category@2@A@@YAXXZ 10041440 f   moc_PhylipPluginTests.obj
 0001:00040450       ??__F?_System_object@?$_Error_objects@H@std@@2V_System_error_category@2@A@@YAXXZ 10041450 f   moc_PhylipPluginTests.obj
 0001:00040460       ??__FalgoLog@U2@@YAXXZ     10041460 f   moc_PhylipPluginTests.obj
 0001:00040470       ??__FcmdLog@U2@@YAXXZ      10041470 f   moc_PhylipPluginTests.obj
 0001:00040480       ??__FcoreLog@U2@@YAXXZ     10041480 f   moc_PhylipPluginTests.obj
 0001:00040490       ??__FioLog@U2@@YAXXZ       10041490 f   moc_PhylipPluginTests.obj
 0001:000404a0       ??__FperfLog@U2@@YAXXZ     100414a0 f   moc_PhylipPluginTests.obj
 0001:000404b0       ??__FscriptLog@U2@@YAXXZ   100414b0 f   moc_PhylipPluginTests.obj
 0001:000404c0       ??__FtaskLog@U2@@YAXXZ     100414c0 f   moc_PhylipPluginTests.obj
 0001:000404d0       ??__FuiLog@U2@@YAXXZ       100414d0 f   moc_PhylipPluginTests.obj
 0001:000404e0       ??__FuserActLog@U2@@YAXXZ  100414e0 f   moc_PhylipPluginTests.obj
 0001:000404f0       ??__F?_Generic_object@?$_Error_objects@H@std@@2V_Generic_error_category@2@A@@YAXXZ 100414f0 f   moc_PhylipTask.obj
 0001:00040500       ??__F?_Iostream_object@?$_Error_objects@H@std@@2V_Iostream_error_category@2@A@@YAXXZ 10041500 f   moc_PhylipTask.obj
 0001:00040510       ??__F?_System_object@?$_Error_objects@H@std@@2V_System_error_category@2@A@@YAXXZ 10041510 f   moc_PhylipTask.obj
 0001:00040520       ??__FalgoLog@U2@@YAXXZ     10041520 f   moc_PhylipTask.obj
 0001:00040530       ??__FcmdLog@U2@@YAXXZ      10041530 f   moc_PhylipTask.obj
 0001:00040540       ??__FcoreLog@U2@@YAXXZ     10041540 f   moc_PhylipTask.obj
 0001:00040550       ??__FioLog@U2@@YAXXZ       10041550 f   moc_PhylipTask.obj
 0001:00040560       ??__FperfLog@U2@@YAXXZ     10041560 f   moc_PhylipTask.obj
 0001:00040570       ??__FscriptLog@U2@@YAXXZ   10041570 f   moc_PhylipTask.obj
 0001:00040580       ??__FtaskLog@U2@@YAXXZ     10041580 f   moc_PhylipTask.obj
 0001:00040590       ??__FuiLog@U2@@YAXXZ       10041590 f   moc_PhylipTask.obj
 0001:000405a0       ??__FuserActLog@U2@@YAXXZ  100415a0 f   moc_PhylipTask.obj
 0002:00000b54       _algoLog$initializer$      10042b54     DistanceMatrix.obj
 0002:00000b58       _cmdLog$initializer$       10042b58     DistanceMatrix.obj
 0002:00000b5c       _coreLog$initializer$      10042b5c     DistanceMatrix.obj
 0002:00000b60       _ioLog$initializer$        10042b60     DistanceMatrix.obj
 0002:00000b64       _perfLog$initializer$      10042b64     DistanceMatrix.obj
 0002:00000b68       _scriptLog$initializer$    10042b68     DistanceMatrix.obj
 0002:00000b6c       _taskLog$initializer$      10042b6c     DistanceMatrix.obj
 0002:00000b70       _uiLog$initializer$        10042b70     DistanceMatrix.obj
 0002:00000b74       _userActLog$initializer$   10042b74     DistanceMatrix.obj
 0002:00000b78       ?_Generic_object$initializer$@?$_Error_objects@H@std@@2P6AXXZA 10042b78     DistanceMatrix.obj
 0002:00000b7c       ?_Iostream_object$initializer$@?$_Error_objects@H@std@@2P6AXXZA 10042b7c     DistanceMatrix.obj
 0002:00000b80       ?_System_object$initializer$@?$_Error_objects@H@std@@2P6AXXZA 10042b80     DistanceMatrix.obj
 0002:00000b84       _algoLog$initializer$      10042b84     NeighborJoinAdapter.obj
 0002:00000b88       _cmdLog$initializer$       10042b88     NeighborJoinAdapter.obj
 0002:00000b8c       _coreLog$initializer$      10042b8c     NeighborJoinAdapter.obj
 0002:00000b90       _ioLog$initializer$        10042b90     NeighborJoinAdapter.obj
 0002:00000b94       _perfLog$initializer$      10042b94     NeighborJoinAdapter.obj
 0002:00000b98       _scriptLog$initializer$    10042b98     NeighborJoinAdapter.obj
 0002:00000b9c       _taskLog$initializer$      10042b9c     NeighborJoinAdapter.obj
 0002:00000ba0       _uiLog$initializer$        10042ba0     NeighborJoinAdapter.obj
 0002:00000ba4       _userActLog$initializer$   10042ba4     NeighborJoinAdapter.obj
 0002:00000ba8       ?runLock$initializer$@NeighborJoinCalculateTreeTask@U2@@0P6AXXZA 10042ba8     NeighborJoinAdapter.obj
 0002:00000bac       _algoLog$initializer$      10042bac     NeighborJoinWidget.obj
 0002:00000bb0       _cmdLog$initializer$       10042bb0     NeighborJoinWidget.obj
 0002:00000bb4       _coreLog$initializer$      10042bb4     NeighborJoinWidget.obj
 0002:00000bb8       _ioLog$initializer$        10042bb8     NeighborJoinWidget.obj
 0002:00000bbc       _perfLog$initializer$      10042bbc     NeighborJoinWidget.obj
 0002:00000bc0       _scriptLog$initializer$    10042bc0     NeighborJoinWidget.obj
 0002:00000bc4       _taskLog$initializer$      10042bc4     NeighborJoinWidget.obj
 0002:00000bc8       _uiLog$initializer$        10042bc8     NeighborJoinWidget.obj
 0002:00000bcc       _userActLog$initializer$   10042bcc     NeighborJoinWidget.obj
 0002:00000bd0       ?M1$initializer$@ConsensusModelTypes@U2@@2P6AXXZA 10042bd0     NeighborJoinWidget.obj
 0002:00000bd4       ?Strict$initializer$@ConsensusModelTypes@U2@@2P6AXXZA 10042bd4     NeighborJoinWidget.obj
 0002:00000bd8       ?MajorityRuleExt$initializer$@ConsensusModelTypes@U2@@2P6AXXZA 10042bd8     NeighborJoinWidget.obj
 0002:00000bdc       ?MajorityRule$initializer$@ConsensusModelTypes@U2@@2P6AXXZA 10042bdc     NeighborJoinWidget.obj
 0002:00000be0       _algoLog$initializer$      10042be0     PhylipCmdlineTask.obj
 0002:00000be4       _cmdLog$initializer$       10042be4     PhylipCmdlineTask.obj
 0002:00000be8       _coreLog$initializer$      10042be8     PhylipCmdlineTask.obj
 0002:00000bec       _ioLog$initializer$        10042bec     PhylipCmdlineTask.obj
 0002:00000bf0       _perfLog$initializer$      10042bf0     PhylipCmdlineTask.obj
 0002:00000bf4       _scriptLog$initializer$    10042bf4     PhylipCmdlineTask.obj
 0002:00000bf8       _taskLog$initializer$      10042bf8     PhylipCmdlineTask.obj
 0002:00000bfc       _uiLog$initializer$        10042bfc     PhylipCmdlineTask.obj
 0002:00000c00       _userActLog$initializer$   10042c00     PhylipCmdlineTask.obj
 0002:00000c04       ?PHYLIP_CMDLINE$initializer$@PhylipCmdlineTask@U2@@2P6AXXZA 10042c04     PhylipCmdlineTask.obj
 0002:00000c08       ?MATRIX_ARG$initializer$@PhylipCmdlineTask@U2@@2P6AXXZA 10042c08     PhylipCmdlineTask.obj
 0002:00000c0c       ?GAMMA_ARG$initializer$@PhylipCmdlineTask@U2@@2P6AXXZA 10042c0c     PhylipCmdlineTask.obj
 0002:00000c10       ?ALPHA_ARG$initializer$@PhylipCmdlineTask@U2@@2P6AXXZA 10042c10     PhylipCmdlineTask.obj
 0002:00000c14       ?TT_RATIO_ARG$initializer$@PhylipCmdlineTask@U2@@2P6AXXZA 10042c14     PhylipCmdlineTask.obj
 0002:00000c18       ?BOOTSTRAP_ARG$initializer$@PhylipCmdlineTask@U2@@2P6AXXZA 10042c18     PhylipCmdlineTask.obj
 0002:00000c1c       ?REPLICATES_ARG$initializer$@PhylipCmdlineTask@U2@@2P6AXXZA 10042c1c     PhylipCmdlineTask.obj
 0002:00000c20       ?SEED_ARG$initializer$@PhylipCmdlineTask@U2@@2P6AXXZA 10042c20     PhylipCmdlineTask.obj
 0002:00000c24       ?FRACTION_ARG$initializer$@PhylipCmdlineTask@U2@@2P6AXXZA 10042c24     PhylipCmdlineTask.obj
 0002:00000c28       ?CONSENSUS_ARG$initializer$@PhylipCmdlineTask@U2@@2P6AXXZA 10042c28     PhylipCmdlineTask.obj
 0002:00000c2c       _algoLog$initializer$      10042c2c     PhylipPlugin.obj
 0002:00000c30       _cmdLog$initializer$       10042c30     PhylipPlugin.obj
 0002:00000c34       _coreLog$initializer$      10042c34     PhylipPlugin.obj
 0002:00000c38       _ioLog$initializer$        10042c38     PhylipPlugin.obj
 0002:00000c3c       _perfLog$initializer$      10042c3c     PhylipPlugin.obj
 0002:00000c40       _scriptLog$initializer$    10042c40     PhylipPlugin.obj
 0002:00000c44       _taskLog$initializer$      10042c44     PhylipPlugin.obj
 0002:00000c48       _uiLog$initializer$        10042c48     PhylipPlugin.obj
 0002:00000c4c       _userActLog$initializer$   10042c4c     PhylipPlugin.obj
 0002:00000c50       _Service_PluginViewer$initializer$ 10042c50     PhylipPlugin.obj
 0002:00000c54       _Service_Project$initializer$ 10042c54     PhylipPlugin.obj
 0002:00000c58       _Service_ProjectView$initializer$ 10042c58     PhylipPlugin.obj
 0002:00000c5c       _Service_DNAGraphPack$initializer$ 10042c5c     PhylipPlugin.obj
 0002:00000c60       _Service_DNAExport$initializer$ 10042c60     PhylipPlugin.obj
 0002:00000c64       _Service_TestRunner$initializer$ 10042c64     PhylipPlugin.obj
 0002:00000c68       _Service_ScriptRegistry$initializer$ 10042c68     PhylipPlugin.obj
 0002:00000c6c       _Service_ExternalToolSupport$initializer$ 10042c6c     PhylipPlugin.obj
 0002:00000c70       _Service_GUITesting$initializer$ 10042c70     PhylipPlugin.obj
 0002:00000c74       _Service_WorkflowDesigner$initializer$ 10042c74     PhylipPlugin.obj
 0002:00000c78       _Service_QueryDesigner$initializer$ 10042c78     PhylipPlugin.obj
 0002:00000c7c       _Service_MinCoreServiceId$initializer$ 10042c7c     PhylipPlugin.obj
 0002:00000c80       _Service_MaxCoreServiceId$initializer$ 10042c80     PhylipPlugin.obj
 0002:00000c84       ?PHYLIP_NEIGHBOUR_JOIN$initializer$@PhylipPlugin@U2@@2P6AXXZA 10042c84     PhylipPlugin.obj
 0002:00000c88       _Service_PluginViewer$initializer$ 10042c88     PhylipPluginTests.obj
 0002:00000c8c       _Service_Project$initializer$ 10042c8c     PhylipPluginTests.obj
 0002:00000c90       _Service_ProjectView$initializer$ 10042c90     PhylipPluginTests.obj
 0002:00000c94       _Service_DNAGraphPack$initializer$ 10042c94     PhylipPluginTests.obj
 0002:00000c98       _Service_DNAExport$initializer$ 10042c98     PhylipPluginTests.obj
 0002:00000c9c       _Service_TestRunner$initializer$ 10042c9c     PhylipPluginTests.obj
 0002:00000ca0       _Service_ScriptRegistry$initializer$ 10042ca0     PhylipPluginTests.obj
 0002:00000ca4       _Service_ExternalToolSupport$initializer$ 10042ca4     PhylipPluginTests.obj
 0002:00000ca8       _Service_GUITesting$initializer$ 10042ca8     PhylipPluginTests.obj
 0002:00000cac       _Service_WorkflowDesigner$initializer$ 10042cac     PhylipPluginTests.obj
 0002:00000cb0       _Service_QueryDesigner$initializer$ 10042cb0     PhylipPluginTests.obj
 0002:00000cb4       _Service_MinCoreServiceId$initializer$ 10042cb4     PhylipPluginTests.obj
 0002:00000cb8       _Service_MaxCoreServiceId$initializer$ 10042cb8     PhylipPluginTests.obj
 0002:00000cbc       _algoLog$initializer$      10042cbc     PhylipPluginTests.obj
 0002:00000cc0       _cmdLog$initializer$       10042cc0     PhylipPluginTests.obj
 0002:00000cc4       _coreLog$initializer$      10042cc4     PhylipPluginTests.obj
 0002:00000cc8       _ioLog$initializer$        10042cc8     PhylipPluginTests.obj
 0002:00000ccc       _perfLog$initializer$      10042ccc     PhylipPluginTests.obj
 0002:00000cd0       _scriptLog$initializer$    10042cd0     PhylipPluginTests.obj
 0002:00000cd4       _taskLog$initializer$      10042cd4     PhylipPluginTests.obj
 0002:00000cd8       _uiLog$initializer$        10042cd8     PhylipPluginTests.obj
 0002:00000cdc       _userActLog$initializer$   10042cdc     PhylipPluginTests.obj
 0002:00000ce0       _algoLog$initializer$      10042ce0     PhylipTask.obj
 0002:00000ce4       _cmdLog$initializer$       10042ce4     PhylipTask.obj
 0002:00000ce8       _coreLog$initializer$      10042ce8     PhylipTask.obj
 0002:00000cec       _ioLog$initializer$        10042cec     PhylipTask.obj
 0002:00000cf0       _perfLog$initializer$      10042cf0     PhylipTask.obj
 0002:00000cf4       _scriptLog$initializer$    10042cf4     PhylipTask.obj
 0002:00000cf8       _taskLog$initializer$      10042cf8     PhylipTask.obj
 0002:00000cfc       _uiLog$initializer$        10042cfc     PhylipTask.obj
 0002:00000d00       _userActLog$initializer$   10042d00     PhylipTask.obj
 0002:00000d04       _algoLog$initializer$      10042d04     SeqBootAdapter.obj
 0002:00000d08       _cmdLog$initializer$       10042d08     SeqBootAdapter.obj
 0002:00000d0c       _coreLog$initializer$      10042d0c     SeqBootAdapter.obj
 0002:00000d10       _ioLog$initializer$        10042d10     SeqBootAdapter.obj
 0002:00000d14       _perfLog$initializer$      10042d14     SeqBootAdapter.obj
 0002:00000d18       _scriptLog$initializer$    10042d18     SeqBootAdapter.obj
 0002:00000d1c       _taskLog$initializer$      10042d1c     SeqBootAdapter.obj
 0002:00000d20       _uiLog$initializer$        10042d20     SeqBootAdapter.obj
 0002:00000d24       _userActLog$initializer$   10042d24     SeqBootAdapter.obj
 0002:00000d28       _algoLog$initializer$      10042d28     dist.obj
 0002:00000d2c       _cmdLog$initializer$       10042d2c     dist.obj
 0002:00000d30       _coreLog$initializer$      10042d30     dist.obj
 0002:00000d34       _ioLog$initializer$        10042d34     dist.obj
 0002:00000d38       _perfLog$initializer$      10042d38     dist.obj
 0002:00000d3c       _scriptLog$initializer$    10042d3c     dist.obj
 0002:00000d40       _taskLog$initializer$      10042d40     dist.obj
 0002:00000d44       _uiLog$initializer$        10042d44     dist.obj
 0002:00000d48       _userActLog$initializer$   10042d48     dist.obj
 0002:00000d4c       _algoLog$initializer$      10042d4c     dnadist.obj
 0002:00000d50       _cmdLog$initializer$       10042d50     dnadist.obj
 0002:00000d54       _coreLog$initializer$      10042d54     dnadist.obj
 0002:00000d58       _ioLog$initializer$        10042d58     dnadist.obj
 0002:00000d5c       _perfLog$initializer$      10042d5c     dnadist.obj
 0002:00000d60       _scriptLog$initializer$    10042d60     dnadist.obj
 0002:00000d64       _taskLog$initializer$      10042d64     dnadist.obj
 0002:00000d68       _uiLog$initializer$        10042d68     dnadist.obj
 0002:00000d6c       _userActLog$initializer$   10042d6c     dnadist.obj
 0002:00000d70       ?F84$initializer$@DNADistModelTypes@@2P6AXXZA 10042d70     dnadist.obj
 0002:00000d74       ?Kimura$initializer$@DNADistModelTypes@@2P6AXXZA 10042d74     dnadist.obj
 0002:00000d78       ?JukesCantor$initializer$@DNADistModelTypes@@2P6AXXZA 10042d78     dnadist.obj
 0002:00000d7c       ?LogDet$initializer$@DNADistModelTypes@@2P6AXXZA 10042d7c     dnadist.obj
 0002:00000d80       _dnaDistSettings$initializer$ 10042d80     dnadist.obj
 0002:00000d84       _algoLog$initializer$      10042d84     neighbor.obj
 0002:00000d88       _cmdLog$initializer$       10042d88     neighbor.obj
 0002:00000d8c       _coreLog$initializer$      10042d8c     neighbor.obj
 0002:00000d90       _ioLog$initializer$        10042d90     neighbor.obj
 0002:00000d94       _perfLog$initializer$      10042d94     neighbor.obj
 0002:00000d98       _scriptLog$initializer$    10042d98     neighbor.obj
 0002:00000d9c       _taskLog$initializer$      10042d9c     neighbor.obj
 0002:00000da0       _uiLog$initializer$        10042da0     neighbor.obj
 0002:00000da4       _userActLog$initializer$   10042da4     neighbor.obj
 0002:00000da8       _algoLog$initializer$      10042da8     phylip.obj
 0002:00000dac       _cmdLog$initializer$       10042dac     phylip.obj
 0002:00000db0       _coreLog$initializer$      10042db0     phylip.obj
 0002:00000db4       _ioLog$initializer$        10042db4     phylip.obj
 0002:00000db8       _perfLog$initializer$      10042db8     phylip.obj
 0002:00000dbc       _scriptLog$initializer$    10042dbc     phylip.obj
 0002:00000dc0       _taskLog$initializer$      10042dc0     phylip.obj
 0002:00000dc4       _uiLog$initializer$        10042dc4     phylip.obj
 0002:00000dc8       _userActLog$initializer$   10042dc8     phylip.obj
 0002:00000dcc       _algoLog$initializer$      10042dcc     protdist.obj
 0002:00000dd0       _cmdLog$initializer$       10042dd0     protdist.obj
 0002:00000dd4       _coreLog$initializer$      10042dd4     protdist.obj
 0002:00000dd8       _ioLog$initializer$        10042dd8     protdist.obj
 0002:00000ddc       _perfLog$initializer$      10042ddc     protdist.obj
 0002:00000de0       _scriptLog$initializer$    10042de0     protdist.obj
 0002:00000de4       _taskLog$initializer$      10042de4     protdist.obj
 0002:00000de8       _uiLog$initializer$        10042de8     protdist.obj
 0002:00000dec       _userActLog$initializer$   10042dec     protdist.obj
 0002:00000df0       ?JTT$initializer$@ProtDistModelTypes@@2P6AXXZA 10042df0     protdist.obj
 0002:00000df4       ?PMB$initializer$@ProtDistModelTypes@@2P6AXXZA 10042df4     protdist.obj
 0002:00000df8       ?PAM$initializer$@ProtDistModelTypes@@2P6AXXZA 10042df8     protdist.obj
 0002:00000dfc       ?Kimura$initializer$@ProtDistModelTypes@@2P6AXXZA 10042dfc     protdist.obj
 0002:00000e00       _algoLog$initializer$      10042e00     seqboot.obj
 0002:00000e04       _cmdLog$initializer$       10042e04     seqboot.obj
 0002:00000e08       _coreLog$initializer$      10042e08     seqboot.obj
 0002:00000e0c       _ioLog$initializer$        10042e0c     seqboot.obj
 0002:00000e10       _perfLog$initializer$      10042e10     seqboot.obj
 0002:00000e14       _scriptLog$initializer$    10042e14     seqboot.obj
 0002:00000e18       _taskLog$initializer$      10042e18     seqboot.obj
 0002:00000e1c       _uiLog$initializer$        10042e1c     seqboot.obj
 0002:00000e20       _userActLog$initializer$   10042e20     seqboot.obj
 0002:00000e24       _algoLog$initializer$      10042e24     moc_NeighborJoinWidget.obj
 0002:00000e28       _cmdLog$initializer$       10042e28     moc_NeighborJoinWidget.obj
 0002:00000e2c       _coreLog$initializer$      10042e2c     moc_NeighborJoinWidget.obj
 0002:00000e30       _ioLog$initializer$        10042e30     moc_NeighborJoinWidget.obj
 0002:00000e34       _perfLog$initializer$      10042e34     moc_NeighborJoinWidget.obj
 0002:00000e38       _scriptLog$initializer$    10042e38     moc_NeighborJoinWidget.obj
 0002:00000e3c       _taskLog$initializer$      10042e3c     moc_NeighborJoinWidget.obj
 0002:00000e40       _uiLog$initializer$        10042e40     moc_NeighborJoinWidget.obj
 0002:00000e44       _userActLog$initializer$   10042e44     moc_NeighborJoinWidget.obj
 0002:00000e48       ?staticMetaObject$initializer$@NeighborJoinWidget@U2@@2P6AXXZA 10042e48     moc_NeighborJoinWidget.obj
 0002:00000e4c       _algoLog$initializer$      10042e4c     moc_PhylipCmdlineTask.obj
 0002:00000e50       _cmdLog$initializer$       10042e50     moc_PhylipCmdlineTask.obj
 0002:00000e54       _coreLog$initializer$      10042e54     moc_PhylipCmdlineTask.obj
 0002:00000e58       _ioLog$initializer$        10042e58     moc_PhylipCmdlineTask.obj
 0002:00000e5c       _perfLog$initializer$      10042e5c     moc_PhylipCmdlineTask.obj
 0002:00000e60       _scriptLog$initializer$    10042e60     moc_PhylipCmdlineTask.obj
 0002:00000e64       _taskLog$initializer$      10042e64     moc_PhylipCmdlineTask.obj
 0002:00000e68       _uiLog$initializer$        10042e68     moc_PhylipCmdlineTask.obj
 0002:00000e6c       _userActLog$initializer$   10042e6c     moc_PhylipCmdlineTask.obj
 0002:00000e70       ?staticMetaObject$initializer$@PhylipCmdlineTask@U2@@2P6AXXZA 10042e70     moc_PhylipCmdlineTask.obj
 0002:00000e74       _Service_PluginViewer$initializer$ 10042e74     moc_PhylipPlugin.obj
 0002:00000e78       _Service_Project$initializer$ 10042e78     moc_PhylipPlugin.obj
 0002:00000e7c       _Service_ProjectView$initializer$ 10042e7c     moc_PhylipPlugin.obj
 0002:00000e80       _Service_DNAGraphPack$initializer$ 10042e80     moc_PhylipPlugin.obj
 0002:00000e84       _Service_DNAExport$initializer$ 10042e84     moc_PhylipPlugin.obj
 0002:00000e88       _Service_TestRunner$initializer$ 10042e88     moc_PhylipPlugin.obj
 0002:00000e8c       _Service_ScriptRegistry$initializer$ 10042e8c     moc_PhylipPlugin.obj
 0002:00000e90       _Service_ExternalToolSupport$initializer$ 10042e90     moc_PhylipPlugin.obj
 0002:00000e94       _Service_GUITesting$initializer$ 10042e94     moc_PhylipPlugin.obj
 0002:00000e98       _Service_WorkflowDesigner$initializer$ 10042e98     moc_PhylipPlugin.obj
 0002:00000e9c       _Service_QueryDesigner$initializer$ 10042e9c     moc_PhylipPlugin.obj
 0002:00000ea0       _Service_MinCoreServiceId$initializer$ 10042ea0     moc_PhylipPlugin.obj
 0002:00000ea4       _Service_MaxCoreServiceId$initializer$ 10042ea4     moc_PhylipPlugin.obj
 0002:00000ea8       ?staticMetaObject$initializer$@PhylipPlugin@U2@@2P6AXXZA 10042ea8     moc_PhylipPlugin.obj
 0002:00000eac       _algoLog$initializer$      10042eac     moc_PhylipPluginTests.obj
 0002:00000eb0       _cmdLog$initializer$       10042eb0     moc_PhylipPluginTests.obj
 0002:00000eb4       _coreLog$initializer$      10042eb4     moc_PhylipPluginTests.obj
 0002:00000eb8       _ioLog$initializer$        10042eb8     moc_PhylipPluginTests.obj
 0002:00000ebc       _perfLog$initializer$      10042ebc     moc_PhylipPluginTests.obj
 0002:00000ec0       _scriptLog$initializer$    10042ec0     moc_PhylipPluginTests.obj
 0002:00000ec4       _taskLog$initializer$      10042ec4     moc_PhylipPluginTests.obj
 0002:00000ec8       _uiLog$initializer$        10042ec8     moc_PhylipPluginTests.obj
 0002:00000ecc       _userActLog$initializer$   10042ecc     moc_PhylipPluginTests.obj
 0002:00000ed0       ?staticMetaObject$initializer$@GTest_NeighborJoin@U2@@2P6AXXZA 10042ed0     moc_PhylipPluginTests.obj
 0002:00000ed4       _algoLog$initializer$      10042ed4     moc_PhylipTask.obj
 0002:00000ed8       _cmdLog$initializer$       10042ed8     moc_PhylipTask.obj
 0002:00000edc       _coreLog$initializer$      10042edc     moc_PhylipTask.obj
 0002:00000ee0       _ioLog$initializer$        10042ee0     moc_PhylipTask.obj
 0002:00000ee4       _perfLog$initializer$      10042ee4     moc_PhylipTask.obj
 0002:00000ee8       _scriptLog$initializer$    10042ee8     moc_PhylipTask.obj
 0002:00000eec       _taskLog$initializer$      10042eec     moc_PhylipTask.obj
 0002:00000ef0       _uiLog$initializer$        10042ef0     moc_PhylipTask.obj
 0002:00000ef4       _userActLog$initializer$   10042ef4     moc_PhylipTask.obj
 0002:00000ef8       ?staticMetaObject$initializer$@PhylipTask@U2@@2P6AXXZA 10042ef8     moc_PhylipTask.obj
 0002:00000f04       _pcinit                    10042f04     MSVCRT:crtdll.obj
 0002:00000f08       _pinit                     10042f08     MSVCRT:atonexit.obj
 0002:00000f0c       _pinit                     10042f0c     MSVCRT:cpu_disp.obj
 0002:00001278       ?badSymbols@?1??replacePhylipRestrictedSymbols@U2@@YAXAAVQByteArray@@@Z@4QBDB 10043278     NeighborJoinAdapter.obj
 0002:00001e78       ?qstring_literal@?6???R<lambda_0b0380af5bb2f62da28634d4824ec8ca>@@QBE?AVQString@@XZ@4U?$QStaticStringData@$0BC@@@B 10043e78     NeighborJoinWidget.obj
 0002:00001eb0       ?qstring_literal@?7???R<lambda_33b9794a776f12fce937feb1d38745b7>@@QBE?AVQString@@XZ@4U?$QStaticStringData@$0O@@@B 10043eb0     NeighborJoinWidget.obj
 0002:00001ee0       ?qstring_literal@?8???R<lambda_d22a08e1c31cb8eed59da0c6f8cb4643>@@QBE?AVQString@@XZ@4U?$QStaticStringData@$08@@B 10043ee0     NeighborJoinWidget.obj
 0002:00001f04       ?qstring_literal@?9???R<lambda_992082ea6d03cf2b362a601e532562f9>@@QBE?AVQString@@XZ@4U?$QStaticStringData@$0BB@@@B 10043f04     NeighborJoinWidget.obj
 0002:00001f38       ?qstring_literal@?L@???R<lambda_0d22fed94f2a311d9dfca95916641178>@@QBE?AVQString@@XZ@4U?$QStaticStringData@$0BA@@@B 10043f38     NeighborJoinWidget.obj
 0002:00001f6c       ?qstring_literal@?M@???R<lambda_48eb925e0df25a63beef6f774f70e0ce>@@QBE?AVQString@@XZ@4U?$QStaticStringData@$0L@@@B 10043f6c     NeighborJoinWidget.obj
 0002:00001f94       ?qstring_literal@?N@???R<lambda_23a54e0ab73de2509c6e5cc465bd53c9>@@QBE?AVQString@@XZ@4U?$QStaticStringData@$07@@B 10043f94     NeighborJoinWidget.obj
 0002:00001fb8       ?qstring_literal@?O@???R<lambda_9d41da171c8d767f232c43981809cb07>@@QBE?AVQString@@XZ@4U?$QStaticStringData@$06@@B 10043fb8     NeighborJoinWidget.obj
 0002:00001fd8       ?qstring_literal@?P@???R<lambda_a9c426da71b6bbdf1080a86813f9c2db>@@QBE?AVQString@@XZ@4U?$QStaticStringData@$0BB@@@B 10043fd8     NeighborJoinWidget.obj
 0002:0000200c       ?qstring_literal@?BA@???R<lambda_ba1cc78051bce41bc52e64c17a9c21ff>@@QBE?AVQString@@XZ@4U?$QStaticStringData@$0O@@@B 1004400c     NeighborJoinWidget.obj
 0002:0000203c       ?qstring_literal@?BB@???R<lambda_fe34ae2a9f494fb27c4b6c32f78f7d34>@@QBE?AVQString@@XZ@4U?$QStaticStringData@$06@@B 1004403c     NeighborJoinWidget.obj
 0002:0000205c       ?qstring_literal@?BC@???R<lambda_47aba4f81f0235f8ea25dd5385c10da9>@@QBE?AVQString@@XZ@4U?$QStaticStringData@$07@@B 1004405c     NeighborJoinWidget.obj
 0002:00002080       ?qstring_literal@?BD@???R<lambda_e4294879436371d98917fc7c6809dc4b>@@QBE?AVQString@@XZ@4U?$QStaticStringData@$0BA@@@B 10044080     NeighborJoinWidget.obj
 0002:000020b4       ?qstring_literal@?BE@???R<lambda_7fcb402e3d4ced9f2dada59451304bad>@@QBE?AVQString@@XZ@4U?$QStaticStringData@$0N@@@B 100440b4     NeighborJoinWidget.obj
 0002:000020e0       ?qstring_literal@?BF@???R<lambda_9bdb903db70d78592dfa82f916e59082>@@QBE?AVQString@@XZ@4U?$QStaticStringData@$0BG@@@B 100440e0     NeighborJoinWidget.obj
 0002:00002120       ?qstring_literal@?BG@???R<lambda_69ac5ad72d4d5a21717e1b3cd28fabc3>@@QBE?AVQString@@XZ@4U?$QStaticStringData@$0M@@@B 10044120     NeighborJoinWidget.obj
 0002:0000214c       ?qstring_literal@?BH@???R<lambda_4e2ee4c24f9f6f06c9235a84091eec77>@@QBE?AVQString@@XZ@4U?$QStaticStringData@$0BA@@@B 1004414c     NeighborJoinWidget.obj
 0002:00002180       ?qstring_literal@?BI@???R<lambda_a240313f06a8e1d5b6e359782d131016>@@QBE?AVQString@@XZ@4U?$QStaticStringData@$0BG@@@B 10044180     NeighborJoinWidget.obj
 0002:000021c0       ?qstring_literal@?BJ@???R<lambda_2b4fc15a8fdb2e804f00ceb3bda53a64>@@QBE?AVQString@@XZ@4U?$QStaticStringData@$0BJ@@@B 100441c0     NeighborJoinWidget.obj
 0002:00002204       ?qstring_literal@?BK@???R<lambda_0b8b5ce51c46f86678041328dcb0fb05>@@QBE?AVQString@@XZ@4U?$QStaticStringData@$0BA@@@B 10044204     NeighborJoinWidget.obj
 0002:00002238       ?qstring_literal@?BL@???R<lambda_8f99dcda7ee44bb3b2c68c37b2d63d09>@@QBE?AVQString@@XZ@4U?$QStaticStringData@$0BG@@@B 10044238     NeighborJoinWidget.obj
 0002:00002278       ?qstring_literal@?BM@???R<lambda_89c462f96a9772122e80910435b04d7b>@@QBE?AVQString@@XZ@4U?$QStaticStringData@$0BD@@@B 10044278     NeighborJoinWidget.obj
 0002:000022b0       ?qstring_literal@?BN@???R<lambda_5cb97931b222ba4845c1a6793eb20d02>@@QBE?AVQString@@XZ@4U?$QStaticStringData@$0BC@@@B 100442b0     NeighborJoinWidget.obj
 0002:000022e8       ?qstring_literal@?BO@???R<lambda_d5b1e7fac3396eb92e6a12b8811845a8>@@QBE?AVQString@@XZ@4U?$QStaticStringData@$09@@B 100442e8     NeighborJoinWidget.obj
 0002:00002310       ?qstring_literal@?BP@???R<lambda_c5fe69c308d98b88bf0bdcb153255297>@@QBE?AVQString@@XZ@4U?$QStaticStringData@$06@@B 10044310     NeighborJoinWidget.obj
 0002:00002330       ?qstring_literal@?CA@???R<lambda_ed8afe383a046c77d89e6b408a9bbda5>@@QBE?AVQString@@XZ@4U?$QStaticStringData@$05@@B 10044330     NeighborJoinWidget.obj
 0002:00002350       ?qstring_literal@?CB@???R<lambda_14e59930e730d4459c38a093acf4d195>@@QBE?AVQString@@XZ@4U?$QStaticStringData@$0BD@@@B 10044350     NeighborJoinWidget.obj
 0002:00002388       ?qstring_literal@?CC@???R<lambda_e79d5e48dce79ac397e8108a5da31d66>@@QBE?AVQString@@XZ@4U?$QStaticStringData@$0BA@@@B 10044388     NeighborJoinWidget.obj
 0002:000023bc       ?qstring_literal@?CD@???R<lambda_44ada46bd4b31fea57024b3ee705fbb5>@@QBE?AVQString@@XZ@4U?$QStaticStringData@$0P@@@B 100443bc     NeighborJoinWidget.obj
 0002:000023ec       ?qstring_literal@?CE@???R<lambda_5b8be46bdab4df2be815ada5e31bbf2e>@@QBE?AVQString@@XZ@4U?$QStaticStringData@$0O@@@B 100443ec     NeighborJoinWidget.obj
 0002:0000241c       ?qstring_literal@?CF@???R<lambda_58398813fcf17172efc5c67a807eff6c>@@QBE?AVQString@@XZ@4U?$QStaticStringData@$0L@@@B 1004441c     NeighborJoinWidget.obj
 0002:00002444       ?qstring_literal@?CG@???R<lambda_e3a39c3ab834799cdee3657bb2fb9ff0>@@QBE?AVQString@@XZ@4U?$QStaticStringData@$09@@B 10044444     NeighborJoinWidget.obj
 0002:0000246c       ?qstring_literal@?CH@???R<lambda_0653c3664f4171908e49d192859671f4>@@QBE?AVQString@@XZ@4U?$QStaticStringData@$0BB@@@B 1004446c     NeighborJoinWidget.obj
 0002:000024a0       ?qstring_literal@?CI@???R<lambda_e1d814167b8d6739a6636789b1b459d2>@@QBE?AVQString@@XZ@4U?$QStaticStringData@$0BA@@@B 100444a0     NeighborJoinWidget.obj
 0002:000024d4       ?qstring_literal@?CJ@???R<lambda_2b27d5241a7fc153d4a2a4123de53aa9>@@QBE?AVQString@@XZ@4U?$QStaticStringData@$0O@@@B 100444d4     NeighborJoinWidget.obj
 0002:00006380       _qt_meta_stringdata_U2__NeighborJoinWidget 10048380     moc_NeighborJoinWidget.obj
 0002:00006450       _qt_meta_data_U2__NeighborJoinWidget 10048450     moc_NeighborJoinWidget.obj
 0002:000064e4       _qt_meta_stringdata_U2__PhylipCmdlineTask 100484e4     moc_PhylipCmdlineTask.obj
 0002:0000650c       _qt_meta_data_U2__PhylipCmdlineTask 1004850c     moc_PhylipCmdlineTask.obj
 0002:00006548       _qt_meta_stringdata_U2__PhylipPlugin 10048548     moc_PhylipPlugin.obj
 0002:0000656c       _qt_meta_data_U2__PhylipPlugin 1004856c     moc_PhylipPlugin.obj
 0002:000065a8       _qt_meta_stringdata_U2__GTest_NeighborJoin 100485a8     moc_PhylipPluginTests.obj
 0002:000065d0       _qt_meta_data_U2__GTest_NeighborJoin 100485d0     moc_PhylipPluginTests.obj
 0002:0000660c       _qt_meta_stringdata_U2__PhylipTask 1004860c     moc_PhylipTask.obj
 0002:0000662c       _qt_meta_data_U2__PhylipTask 1004862c     moc_PhylipTask.obj
 0002:00006674       _GS_ExceptionPointers      10048674     MSVCRT:gs_report.obj
 0002:00006680       _Int32ToUInt32             10048680     MSVCRT:ftol3.obj
 0002:00006690       _MantissaMask              10048690     MSVCRT:ftol3.obj
 0002:00006698       _IntegerBit                10048698     MSVCRT:ftol3.obj
 0002:000066a0       _SignBit64                 100486a0     MSVCRT:ftol3.obj
 0002:000066a8       _MinFP64                   100486a8     MSVCRT:ftol3.obj
 0002:000066b0       _MinInt64                  100486b0     MSVCRT:ftol3.obj
 0002:000066b8       _MaxInt64                  100486b8     MSVCRT:ftol3.obj
 0002:000066c0       _MaxUInt64                 100486c0     MSVCRT:ftol3.obj
 0002:000066c8       _MaxFP32                   100486c8     MSVCRT:ftol3.obj
 0002:000066d0       _MinFP32                   100486d0     MSVCRT:ftol3.obj
 0002:000066d8       _MinSubInexact             100486d8     MSVCRT:ftol3.obj
 0002:000066e0       _FpExcptTable              100486e0     MSVCRT:ftol3.obj
 0002:000066f0       _i1075                     100486f0     MSVCRT:ftol3.obj
 0002:000066f4       _i1087                     100486f4     MSVCRT:ftol3.obj
 0002:000066f8       _x0800                     100486f8     MSVCRT:ftol3.obj
 0002:000066fc       _x17FF                     100486fc     MSVCRT:ftol3.obj
 0002:00006700       _CWMask                    10048700     MSVCRT:ftol3.obj
 0002:00007f28       __catchsym$?_Copy@?$basic_string@DU?$char_traits@D@std@@V?$allocator@D@2@@std@@QAEXII@Z$5 10049f28     DistanceMatrix.obj
 0002:00007f38       __catchsym$?_Copy@?$basic_string@DU?$char_traits@D@std@@V?$allocator@D@2@@std@@QAEXII@Z$4 10049f38     DistanceMatrix.obj
 0002:00007f48       __unwindtable$?_Copy@?$basic_string@DU?$char_traits@D@std@@V?$allocator@D@2@@std@@QAEXII@Z 10049f48     DistanceMatrix.obj
 0002:00007f68       __ehfuncinfo$?_Copy@?$basic_string@DU?$char_traits@D@std@@V?$allocator@D@2@@std@@QAEXII@Z 10049f68     DistanceMatrix.obj
 0002:00007f8c       __tryblocktable$?_Copy@?$basic_string@DU?$char_traits@D@std@@V?$allocator@D@2@@std@@QAEXII@Z 10049f8c     DistanceMatrix.obj
 0002:00007fb4       __catchsym$?append@?$QList@VQString@@@@QAEXABVQString@@@Z$13 10049fb4     DistanceMatrix.obj
 0002:00007fc4       __catchsym$?append@?$QList@VQString@@@@QAEXABVQString@@@Z$12 10049fc4     DistanceMatrix.obj
 0002:00007fd4       __ehfuncinfo$?append@?$QList@VQString@@@@QAEXABVQString@@@Z 10049fd4     DistanceMatrix.obj
 0002:00007ff8       __tryblocktable$?append@?$QList@VQString@@@@QAEXABVQString@@@Z 10049ff8     DistanceMatrix.obj
 0002:00008020       __unwindtable$?append@?$QList@VQString@@@@QAEXABVQString@@@Z 1004a020     DistanceMatrix.obj
 0002:00008080       __unwindtable$?removeAll@?$QList@VQString@@@@QAEHABVQString@@@Z 1004a080     DistanceMatrix.obj
 0002:00008088       __ehfuncinfo$?removeAll@?$QList@VQString@@@@QAEHABVQString@@@Z 1004a088     DistanceMatrix.obj
 0002:000080ac       __catchsym$?detach_helper_grow@?$QList@VQString@@@@AAEPAUNode@1@HH@Z$5 1004a0ac     DistanceMatrix.obj
 0002:000080bc       __catchsym$?detach_helper_grow@?$QList@VQString@@@@AAEPAUNode@1@HH@Z$4 1004a0bc     DistanceMatrix.obj
 0002:000080cc       __unwindtable$?detach_helper_grow@?$QList@VQString@@@@AAEPAUNode@1@HH@Z 1004a0cc     DistanceMatrix.obj
 0002:000080ec       __ehfuncinfo$?detach_helper_grow@?$QList@VQString@@@@AAEPAUNode@1@HH@Z 1004a0ec     DistanceMatrix.obj
 0002:00008110       __tryblocktable$?detach_helper_grow@?$QList@VQString@@@@AAEPAUNode@1@HH@Z 1004a110     DistanceMatrix.obj
 0002:00008138       __catchsym$?detach_helper@?$QList@VQString@@@@AAEXH@Z$2 1004a138     DistanceMatrix.obj
 0002:00008148       __unwindtable$?detach_helper@?$QList@VQString@@@@AAEXH@Z 1004a148     DistanceMatrix.obj
 0002:00008158       __tryblocktable$?detach_helper@?$QList@VQString@@@@AAEXH@Z 1004a158     DistanceMatrix.obj
 0002:0000816c       __ehfuncinfo$?detach_helper@?$QList@VQString@@@@AAEXH@Z 1004a16c     DistanceMatrix.obj
 0002:00008190       __unwindtable$?node_construct@?$QList@VQString@@@@AAEXPAUNode@1@ABVQString@@@Z 1004a190     DistanceMatrix.obj
 0002:000081a0       __ehfuncinfo$?node_construct@?$QList@VQString@@@@AAEXPAUNode@1@ABVQString@@@Z 1004a1a0     DistanceMatrix.obj
 0002:000081c4       __catchsym$?node_copy@?$QList@VQString@@@@AAEXPAUNode@1@00@Z$6 1004a1c4     DistanceMatrix.obj
 0002:000081d4       __tryblocktable$?node_copy@?$QList@VQString@@@@AAEXPAUNode@1@00@Z 1004a1d4     DistanceMatrix.obj
 0002:000081e8       __ehfuncinfo$?node_copy@?$QList@VQString@@@@AAEXPAUNode@1@00@Z 1004a1e8     DistanceMatrix.obj
 0002:0000820c       __unwindtable$?node_copy@?$QList@VQString@@@@AAEXPAUNode@1@00@Z 1004a20c     DistanceMatrix.obj
 0002:0000823c       __unwindtable$??__EalgoLog@U2@@YAXXZ 1004a23c     DistanceMatrix.obj
 0002:00008244       __ehfuncinfo$??__EalgoLog@U2@@YAXXZ 1004a244     DistanceMatrix.obj
 0002:00008268       __unwindtable$??__EcmdLog@U2@@YAXXZ 1004a268     DistanceMatrix.obj
 0002:00008270       __ehfuncinfo$??__EcmdLog@U2@@YAXXZ 1004a270     DistanceMatrix.obj
 0002:00008294       __unwindtable$??__EcoreLog@U2@@YAXXZ 1004a294     DistanceMatrix.obj
 0002:0000829c       __ehfuncinfo$??__EcoreLog@U2@@YAXXZ 1004a29c     DistanceMatrix.obj
 0002:000082c0       __unwindtable$??__EioLog@U2@@YAXXZ 1004a2c0     DistanceMatrix.obj
 0002:000082c8       __ehfuncinfo$??__EioLog@U2@@YAXXZ 1004a2c8     DistanceMatrix.obj
 0002:000082ec       __unwindtable$??__EperfLog@U2@@YAXXZ 1004a2ec     DistanceMatrix.obj
 0002:000082f4       __ehfuncinfo$??__EperfLog@U2@@YAXXZ 1004a2f4     DistanceMatrix.obj
 0002:00008318       __unwindtable$??__EscriptLog@U2@@YAXXZ 1004a318     DistanceMatrix.obj
 0002:00008320       __ehfuncinfo$??__EscriptLog@U2@@YAXXZ 1004a320     DistanceMatrix.obj
 0002:00008344       __unwindtable$??__EtaskLog@U2@@YAXXZ 1004a344     DistanceMatrix.obj
 0002:0000834c       __ehfuncinfo$??__EtaskLog@U2@@YAXXZ 1004a34c     DistanceMatrix.obj
 0002:00008370       __unwindtable$??__EuiLog@U2@@YAXXZ 1004a370     DistanceMatrix.obj
 0002:00008378       __ehfuncinfo$??__EuiLog@U2@@YAXXZ 1004a378     DistanceMatrix.obj
 0002:0000839c       __unwindtable$??__EuserActLog@U2@@YAXXZ 1004a39c     DistanceMatrix.obj
 0002:000083a4       __ehfuncinfo$??__EuserActLog@U2@@YAXXZ 1004a3a4     DistanceMatrix.obj
 0002:000083c8       __unwindtable$??0MemoryLocker@U2@@QAE@HW4MemoryLockType@AppResource@1@@Z 1004a3c8     DistanceMatrix.obj
 0002:000083d0       __ehfuncinfo$??0MemoryLocker@U2@@QAE@HW4MemoryLockType@AppResource@1@@Z 1004a3d0     DistanceMatrix.obj
 0002:000083f4       __unwindtable$??1MemoryLocker@U2@@UAE@XZ 1004a3f4     DistanceMatrix.obj
 0002:000083fc       __ehfuncinfo$??1MemoryLocker@U2@@UAE@XZ 1004a3fc     DistanceMatrix.obj
 0002:00008420       __unwindtable$?tryAcquire@MemoryLocker@U2@@QAE_N_J@Z 1004a420     DistanceMatrix.obj
 0002:00008438       __ehfuncinfo$?tryAcquire@MemoryLocker@U2@@QAE_N_J@Z 1004a438     DistanceMatrix.obj
 0002:0000845c       __unwindtable$?release@MemoryLocker@U2@@QAEXXZ 1004a45c     DistanceMatrix.obj
 0002:00008464       __ehfuncinfo$?release@MemoryLocker@U2@@QAEXXZ 1004a464     DistanceMatrix.obj
 0002:00008488       __unwindtable$??_GMemoryLocker@U2@@UAEPAXI@Z 1004a488     DistanceMatrix.obj
 0002:00008490       __ehfuncinfo$??_GMemoryLocker@U2@@UAEPAXI@Z 1004a490     DistanceMatrix.obj
 0002:000084b4       __catchsym$??0?$QList@VMultipleSequenceAlignmentRow@U2@@@@QAE@ABV0@@Z$2 1004a4b4     DistanceMatrix.obj
 0002:000084c4       __unwindtable$??0?$QList@VMultipleSequenceAlignmentRow@U2@@@@QAE@ABV0@@Z 1004a4c4     DistanceMatrix.obj
 0002:000084d4       __tryblocktable$??0?$QList@VMultipleSequenceAlignmentRow@U2@@@@QAE@ABV0@@Z 1004a4d4     DistanceMatrix.obj
 0002:000084e8       __ehfuncinfo$??0?$QList@VMultipleSequenceAlignmentRow@U2@@@@QAE@ABV0@@Z 1004a4e8     DistanceMatrix.obj
 0002:0000850c       __catchsym$?node_copy@?$QList@VMultipleSequenceAlignmentRow@U2@@@@AAEXPAUNode@1@00@Z$6 1004a50c     DistanceMatrix.obj
 0002:0000851c       __tryblocktable$?node_copy@?$QList@VMultipleSequenceAlignmentRow@U2@@@@AAEXPAUNode@1@00@Z 1004a51c     DistanceMatrix.obj
 0002:00008530       __ehfuncinfo$?node_copy@?$QList@VMultipleSequenceAlignmentRow@U2@@@@AAEXPAUNode@1@00@Z 1004a530     DistanceMatrix.obj
 0002:00008554       __unwindtable$?node_copy@?$QList@VMultipleSequenceAlignmentRow@U2@@@@AAEXPAUNode@1@00@Z 1004a554     DistanceMatrix.obj
 0002:00008584       __catchsym$?append@?$QList@PAVPhyBranch@U2@@@@QAEXABQAVPhyBranch@U2@@@Z$6 1004a584     DistanceMatrix.obj
 0002:00008594       __tryblocktable$?append@?$QList@PAVPhyBranch@U2@@@@QAEXABQAVPhyBranch@U2@@@Z 1004a594     DistanceMatrix.obj
 0002:000085a8       __ehfuncinfo$?append@?$QList@PAVPhyBranch@U2@@@@QAEXABQAVPhyBranch@U2@@@Z 1004a5a8     DistanceMatrix.obj
 0002:000085cc       __unwindtable$?append@?$QList@PAVPhyBranch@U2@@@@QAEXABQAVPhyBranch@U2@@@Z 1004a5cc     DistanceMatrix.obj
 0002:000085fc       __catchsym$?detach_helper_grow@?$QList@PAVPhyBranch@U2@@@@AAEPAUNode@1@HH@Z$5 1004a5fc     DistanceMatrix.obj
 0002:0000860c       __catchsym$?detach_helper_grow@?$QList@PAVPhyBranch@U2@@@@AAEPAUNode@1@HH@Z$4 1004a60c     DistanceMatrix.obj
 0002:0000861c       __unwindtable$?detach_helper_grow@?$QList@PAVPhyBranch@U2@@@@AAEPAUNode@1@HH@Z 1004a61c     DistanceMatrix.obj
 0002:0000863c       __ehfuncinfo$?detach_helper_grow@?$QList@PAVPhyBranch@U2@@@@AAEPAUNode@1@HH@Z 1004a63c     DistanceMatrix.obj
 0002:00008660       __tryblocktable$?detach_helper_grow@?$QList@PAVPhyBranch@U2@@@@AAEPAUNode@1@HH@Z 1004a660     DistanceMatrix.obj
 0002:00008688       __unwindtable$?uniqueKeys@?$QMap@VQString@@H@@QBE?AV?$QList@VQString@@@@XZ 1004a688     DistanceMatrix.obj
 0002:00008690       __ehfuncinfo$?uniqueKeys@?$QMap@VQString@@H@@QBE?AV?$QList@VQString@@@@XZ 1004a690     DistanceMatrix.obj
 0002:000086b4       __unwindtable$?keys@?$QMap@VQString@@H@@QBE?AV?$QList@VQString@@@@XZ 1004a6b4     DistanceMatrix.obj
 0002:000086bc       __ehfuncinfo$?keys@?$QMap@VQString@@H@@QBE?AV?$QList@VQString@@@@XZ 1004a6bc     DistanceMatrix.obj
 0002:000086e0       __unwindtable$?keys@?$QMap@VQString@@H@@QBE?AV?$QList@VQString@@@@ABH@Z 1004a6e0     DistanceMatrix.obj
 0002:000086e8       __ehfuncinfo$?keys@?$QMap@VQString@@H@@QBE?AV?$QList@VQString@@@@ABH@Z 1004a6e8     DistanceMatrix.obj
 0002:0000870c       __unwindtable$?clear@?$QVector@V?$QVector@M@@@@QAEXXZ 1004a70c     DistanceMatrix.obj
 0002:00008714       __ehfuncinfo$?clear@?$QVector@V?$QVector@M@@@@QAEXXZ 1004a714     DistanceMatrix.obj
 0002:00008738       __unwindtable$?append@?$QVector@V?$QVector@M@@@@QAEXABV?$QVector@M@@@Z 1004a738     DistanceMatrix.obj
 0002:00008748       __ehfuncinfo$?append@?$QVector@V?$QVector@M@@@@QAEXABV?$QVector@M@@@Z 1004a748     DistanceMatrix.obj
 0002:0000876c       __catchsym$?reallocData@?$QVector@V?$QVector@M@@@@AAEXHHV?$QFlags@W4AllocationOption@QArrayData@@@@@Z$6 1004a76c     DistanceMatrix.obj
 0002:0000877c       __catchsym$?reallocData@?$QVector@V?$QVector@M@@@@AAEXHHV?$QFlags@W4AllocationOption@QArrayData@@@@@Z$5 1004a77c     DistanceMatrix.obj
 0002:0000878c       __ehfuncinfo$?reallocData@?$QVector@V?$QVector@M@@@@AAEXHHV?$QFlags@W4AllocationOption@QArrayData@@@@@Z 1004a78c     DistanceMatrix.obj
 0002:000087b0       __tryblocktable$?reallocData@?$QVector@V?$QVector@M@@@@AAEXHHV?$QFlags@W4AllocationOption@QArrayData@@@@@Z 1004a7b0     DistanceMatrix.obj
 0002:000087d8       __unwindtable$?reallocData@?$QVector@V?$QVector@M@@@@AAEXHHV?$QFlags@W4AllocationOption@QArrayData@@@@@Z 1004a7d8     DistanceMatrix.obj
 0002:00008800       __unwindtable$?copyConstruct@?$QVector@V?$QVector@M@@@@AAEXPBV?$QVector@M@@0PAV2@@Z 1004a800     DistanceMatrix.obj
 0002:00008808       __ehfuncinfo$?copyConstruct@?$QVector@V?$QVector@M@@@@AAEXPBV?$QVector@M@@0PAV2@@Z 1004a808     DistanceMatrix.obj
 0002:0000882c       __catchsym$?append@?$QList@PAVPhyNode@U2@@@@QAEXABQAVPhyNode@U2@@@Z$6 1004a82c     DistanceMatrix.obj
 0002:0000883c       __tryblocktable$?append@?$QList@PAVPhyNode@U2@@@@QAEXABQAVPhyNode@U2@@@Z 1004a83c     DistanceMatrix.obj
 0002:00008850       __ehfuncinfo$?append@?$QList@PAVPhyNode@U2@@@@QAEXABQAVPhyNode@U2@@@Z 1004a850     DistanceMatrix.obj
 0002:00008874       __unwindtable$?append@?$QList@PAVPhyNode@U2@@@@QAEXABQAVPhyNode@U2@@@Z 1004a874     DistanceMatrix.obj
 0002:000088a4       __catchsym$?detach_helper_grow@?$QList@PAVPhyNode@U2@@@@AAEPAUNode@1@HH@Z$5 1004a8a4     DistanceMatrix.obj
 0002:000088b4       __catchsym$?detach_helper_grow@?$QList@PAVPhyNode@U2@@@@AAEPAUNode@1@HH@Z$4 1004a8b4     DistanceMatrix.obj
 0002:000088c4       __unwindtable$?detach_helper_grow@?$QList@PAVPhyNode@U2@@@@AAEPAUNode@1@HH@Z 1004a8c4     DistanceMatrix.obj
 0002:000088e4       __ehfuncinfo$?detach_helper_grow@?$QList@PAVPhyNode@U2@@@@AAEPAUNode@1@HH@Z 1004a8e4     DistanceMatrix.obj
 0002:00008908       __tryblocktable$?detach_helper_grow@?$QList@PAVPhyNode@U2@@@@AAEPAUNode@1@HH@Z 1004a908     DistanceMatrix.obj
 0002:00008930       __catchsym$?detach_helper@?$QList@PAVPhyNode@U2@@@@AAEXH@Z$2 1004a930     DistanceMatrix.obj
 0002:00008940       __unwindtable$?detach_helper@?$QList@PAVPhyNode@U2@@@@AAEXH@Z 1004a940     DistanceMatrix.obj
 0002:00008950       __tryblocktable$?detach_helper@?$QList@PAVPhyNode@U2@@@@AAEXH@Z 1004a950     DistanceMatrix.obj
 0002:00008964       __ehfuncinfo$?detach_helper@?$QList@PAVPhyNode@U2@@@@AAEXH@Z 1004a964     DistanceMatrix.obj
 0002:00008988       __ehfuncinfo$??0DistanceMatrix@U2@@QAE@XZ 1004a988     DistanceMatrix.obj
 0002:000089ac       __unwindtable$??0DistanceMatrix@U2@@QAE@XZ 1004a9ac     DistanceMatrix.obj
 0002:000089f4       __ehfuncinfo$??1DistanceMatrix@U2@@QAE@XZ 1004a9f4     DistanceMatrix.obj
 0002:00008a18       __unwindtable$??1DistanceMatrix@U2@@QAE@XZ 1004aa18     DistanceMatrix.obj
 0002:00008a68       __catchsym$?calculateOutOfAlignment@DistanceMatrix@U2@@QAEXABVMultipleSequenceAlignment@2@ABVCreatePhyTreeSettings@2@@Z$15 1004aa68     DistanceMatrix.obj
 0002:00008a78       __tryblocktable$?calculateOutOfAlignment@DistanceMatrix@U2@@QAEXABVMultipleSequenceAlignment@2@ABVCreatePhyTreeSettings@2@@Z 1004aa78     DistanceMatrix.obj
 0002:00008a8c       __ehfuncinfo$?calculateOutOfAlignment@DistanceMatrix@U2@@QAEXABVMultipleSequenceAlignment@2@ABVCreatePhyTreeSettings@2@@Z 1004aa8c     DistanceMatrix.obj
 0002:00008ab0       __unwindtable$?calculateOutOfAlignment@DistanceMatrix@U2@@QAEXABVMultipleSequenceAlignment@2@ABVCreatePhyTreeSettings@2@@Z 1004aab0     DistanceMatrix.obj
 0002:00008b10       __unwindtable$?calculateQMatrix@DistanceMatrix@U2@@AAEXXZ 1004ab10     DistanceMatrix.obj
 0002:00008b18       __ehfuncinfo$?calculateQMatrix@DistanceMatrix@U2@@AAEXXZ 1004ab18     DistanceMatrix.obj
 0002:00008b3c       __ehfuncinfo$?addPairToTree@DistanceMatrix@U2@@AAEXPAU?$QPair@HH@@@Z 1004ab3c     DistanceMatrix.obj
 0002:00008b60       __unwindtable$?addPairToTree@DistanceMatrix@U2@@AAEXPAU?$QPair@HH@@@Z 1004ab60     DistanceMatrix.obj
 0002:00008bd0       __unwindtable$?getNodeByName@DistanceMatrix@U2@@AAEPAVPhyNode@2@VQString@@@Z 1004abd0     DistanceMatrix.obj
 0002:00008bd8       __ehfuncinfo$?getNodeByName@DistanceMatrix@U2@@AAEPAVPhyNode@2@VQString@@@Z 1004abd8     DistanceMatrix.obj
 0002:00008bfc       __unwindtable$?findNode@DistanceMatrix@U2@@AAEPAVPhyNode@2@PAV32@VQString@@@Z 1004abfc     DistanceMatrix.obj
 0002:00008c04       __ehfuncinfo$?findNode@DistanceMatrix@U2@@AAEPAVPhyNode@2@PAV32@VQString@@@Z 1004ac04     DistanceMatrix.obj
 0002:00008c28       __unwindtable$?generateNodeName@DistanceMatrix@U2@@AAE?AVQString@@V3@0@Z 1004ac28     DistanceMatrix.obj
 0002:00008c40       __ehfuncinfo$?generateNodeName@DistanceMatrix@U2@@AAE?AVQString@@V3@0@Z 1004ac40     DistanceMatrix.obj
 0002:00008c64       __unwindtable$?printPhyNode@DistanceMatrix@U2@@CAXPAVPhyNode@2@HAAV?$QList@PAVPhyNode@U2@@@@@Z 1004ac64     DistanceMatrix.obj
 0002:00008c6c       __ehfuncinfo$?printPhyNode@DistanceMatrix@U2@@CAXPAVPhyNode@2@HAAV?$QList@PAVPhyNode@U2@@@@@Z 1004ac6c     DistanceMatrix.obj
 0002:00008c90       __unwindtable$?printIndex@DistanceMatrix@U2@@AAEXXZ 1004ac90     DistanceMatrix.obj
 0002:00008ca0       __ehfuncinfo$?printIndex@DistanceMatrix@U2@@AAEXXZ 1004aca0     DistanceMatrix.obj
 0002:00008cc4       __unwindtable$?getNewIndex@DistanceMatrix@U2@@AAEHVQString@@U?$QPair@HH@@AAV?$QMap@VQString@@H@@@Z 1004acc4     DistanceMatrix.obj
 0002:00008ccc       __ehfuncinfo$?getNewIndex@DistanceMatrix@U2@@AAEHVQString@@U?$QPair@HH@@AAV?$QMap@VQString@@H@@@Z 1004accc     DistanceMatrix.obj
 0002:00008cf0       __ehfuncinfo$?areTreesEqual@DistanceMatrix@U2@@CA_NPAV?$QSharedDataPointer@VPhyTreeData@U2@@@@0@Z 1004acf0     DistanceMatrix.obj
 0002:00008d14       __unwindtable$?areTreesEqual@DistanceMatrix@U2@@CA_NPAV?$QSharedDataPointer@VPhyTreeData@U2@@@@0@Z 1004ad14     DistanceMatrix.obj
 0002:00008d54       __unwindtable$?addNodeToList@DistanceMatrix@U2@@CAXAAV?$QList@PAVPhyNode@U2@@@@AAV?$QMap@VQString@@H@@AAV?$QList@PAVPhyBranch@U2@@@@PAVPhyNode@2@@Z 1004ad54     DistanceMatrix.obj
 0002:00008d5c       __ehfuncinfo$?addNodeToList@DistanceMatrix@U2@@CAXAAV?$QList@PAVPhyNode@U2@@@@AAV?$QMap@VQString@@H@@AAV?$QList@PAVPhyBranch@U2@@@@PAVPhyNode@2@@Z 1004ad5c     DistanceMatrix.obj
 0002:00008d80       __ehfuncinfo$?switchName@DistanceMatrix@U2@@AAEXPAVPhyNode@2@@Z 1004ad80     DistanceMatrix.obj
 0002:00008da4       __unwindtable$?switchName@DistanceMatrix@U2@@AAEXPAVPhyNode@2@@Z 1004ada4     DistanceMatrix.obj
 0002:00008dcc       __unwindtable$?switchNamesToAllNodes@DistanceMatrix@U2@@AAEXXZ 1004adcc     DistanceMatrix.obj
 0002:00008de4       __ehfuncinfo$?switchNamesToAllNodes@DistanceMatrix@U2@@AAEXXZ 1004ade4     DistanceMatrix.obj
 0002:00008e08       __catchsym$?reallocData@?$QVector@M@@AAEXHHV?$QFlags@W4AllocationOption@QArrayData@@@@@Z$5 1004ae08     DistanceMatrix.obj
 0002:00008e18       __catchsym$?reallocData@?$QVector@M@@AAEXHHV?$QFlags@W4AllocationOption@QArrayData@@@@@Z$4 1004ae18     DistanceMatrix.obj
 0002:00008e28       __unwindtable$?reallocData@?$QVector@M@@AAEXHHV?$QFlags@W4AllocationOption@QArrayData@@@@@Z 1004ae28     DistanceMatrix.obj
 0002:00008e48       __ehfuncinfo$?reallocData@?$QVector@M@@AAEXHHV?$QFlags@W4AllocationOption@QArrayData@@@@@Z 1004ae48     DistanceMatrix.obj
 0002:00008e6c       __tryblocktable$?reallocData@?$QVector@M@@AAEXHHV?$QFlags@W4AllocationOption@QArrayData@@@@@Z 1004ae6c     DistanceMatrix.obj
 0002:00008e94       __catchsym$??$?6U?$char_traits@D@std@@@std@@YAAAV?$basic_ostream@DU?$char_traits@D@std@@@0@AAV10@PBD@Z$4 1004ae94     DistanceMatrix.obj
 0002:00008ea4       __tryblocktable$??$?6U?$char_traits@D@std@@@std@@YAAAV?$basic_ostream@DU?$char_traits@D@std@@@0@AAV10@PBD@Z 1004aea4     DistanceMatrix.obj
 0002:00008eb8       __unwindtable$??$?6U?$char_traits@D@std@@@std@@YAAAV?$basic_ostream@DU?$char_traits@D@std@@@0@AAV10@PBD@Z 1004aeb8     DistanceMatrix.obj
 0002:00008ed8       __ehfuncinfo$??$?6U?$char_traits@D@std@@@std@@YAAAV?$basic_ostream@DU?$char_traits@D@std@@@0@AAV10@PBD@Z 1004aed8     DistanceMatrix.obj
 0002:00008efc       __unwindtable$?clone@?$QSharedDataPointer@VPhyTreeData@U2@@@@IAEPAVPhyTreeData@U2@@XZ 1004aefc     DistanceMatrix.obj
 0002:00008f04       __ehfuncinfo$?clone@?$QSharedDataPointer@VPhyTreeData@U2@@@@IAEPAVPhyTreeData@U2@@XZ 1004af04     DistanceMatrix.obj
 0002:00008f28       __unwindtable$?detach_helper@?$QSharedDataPointer@VPhyTreeData@U2@@@@AAEXXZ 1004af28     DistanceMatrix.obj
 0002:00008f30       __ehfuncinfo$?detach_helper@?$QSharedDataPointer@VPhyTreeData@U2@@@@AAEXXZ 1004af30     DistanceMatrix.obj
 0002:00008f54       __unwindtable$??0sentry@?$basic_ostream@DU?$char_traits@D@std@@@std@@QAE@AAV12@@Z 1004af54     DistanceMatrix.obj
 0002:00008f5c       __ehfuncinfo$??0sentry@?$basic_ostream@DU?$char_traits@D@std@@@std@@QAE@AAV12@@Z 1004af5c     DistanceMatrix.obj
 0002:00008f80       __catchsym$?createNode@?$QMapData@VQString@@H@@QAEPAU?$QMapNode@VQString@@H@@ABVQString@@ABHPAU2@_N@Z$5 1004af80     DistanceMatrix.obj
 0002:00008f90       __tryblocktable$?createNode@?$QMapData@VQString@@H@@QAEPAU?$QMapNode@VQString@@H@@ABVQString@@ABHPAU2@_N@Z 1004af90     DistanceMatrix.obj
 0002:00008fa4       __ehfuncinfo$?createNode@?$QMapData@VQString@@H@@QAEPAU?$QMapNode@VQString@@H@@ABVQString@@ABHPAU2@_N@Z 1004afa4     DistanceMatrix.obj
 0002:00008fc8       __unwindtable$?createNode@?$QMapData@VQString@@H@@QAEPAU?$QMapNode@VQString@@H@@ABVQString@@ABHPAU2@_N@Z 1004afc8     DistanceMatrix.obj
 0002:00008ff0       __unwindtable$??__EalgoLog@U2@@YAXXZ 1004aff0     NeighborJoinAdapter.obj
 0002:00008ff8       __ehfuncinfo$??__EalgoLog@U2@@YAXXZ 1004aff8     NeighborJoinAdapter.obj
 0002:0000901c       __unwindtable$??__EcmdLog@U2@@YAXXZ 1004b01c     NeighborJoinAdapter.obj
 0002:00009024       __ehfuncinfo$??__EcmdLog@U2@@YAXXZ 1004b024     NeighborJoinAdapter.obj
 0002:00009048       __unwindtable$??__EcoreLog@U2@@YAXXZ 1004b048     NeighborJoinAdapter.obj
 0002:00009050       __ehfuncinfo$??__EcoreLog@U2@@YAXXZ 1004b050     NeighborJoinAdapter.obj
 0002:00009074       __unwindtable$??__EioLog@U2@@YAXXZ 1004b074     NeighborJoinAdapter.obj
 0002:0000907c       __ehfuncinfo$??__EioLog@U2@@YAXXZ 1004b07c     NeighborJoinAdapter.obj
 0002:000090a0       __unwindtable$??__EperfLog@U2@@YAXXZ 1004b0a0     NeighborJoinAdapter.obj
 0002:000090a8       __ehfuncinfo$??__EperfLog@U2@@YAXXZ 1004b0a8     NeighborJoinAdapter.obj
 0002:000090cc       __unwindtable$??__EscriptLog@U2@@YAXXZ 1004b0cc     NeighborJoinAdapter.obj
 0002:000090d4       __ehfuncinfo$??__EscriptLog@U2@@YAXXZ 1004b0d4     NeighborJoinAdapter.obj
 0002:000090f8       __unwindtable$??__EtaskLog@U2@@YAXXZ 1004b0f8     NeighborJoinAdapter.obj
 0002:00009100       __ehfuncinfo$??__EtaskLog@U2@@YAXXZ 1004b100     NeighborJoinAdapter.obj
 0002:00009124       __unwindtable$??__EuiLog@U2@@YAXXZ 1004b124     NeighborJoinAdapter.obj
 0002:0000912c       __ehfuncinfo$??__EuiLog@U2@@YAXXZ 1004b12c     NeighborJoinAdapter.obj
 0002:00009150       __unwindtable$??__EuserActLog@U2@@YAXXZ 1004b150     NeighborJoinAdapter.obj
 0002:00009158       __ehfuncinfo$??__EuserActLog@U2@@YAXXZ 1004b158     NeighborJoinAdapter.obj
 0002:0000917c       __unwindtable$??0MemoryLocker@U2@@QAE@AAVU2OpStatus@1@HW4MemoryLockType@AppResource@1@@Z 1004b17c     NeighborJoinAdapter.obj
 0002:00009184       __ehfuncinfo$??0MemoryLocker@U2@@QAE@AAVU2OpStatus@1@HW4MemoryLockType@AppResource@1@@Z 1004b184     NeighborJoinAdapter.obj
 0002:000091a8       __unwindtable$?createCalculatePhyTreeTask@NeighborJoinAdapter@U2@@UAEPAVTask@2@ABVMultipleSequenceAlignment@2@ABVCreatePhyTreeSettings@2@@Z 1004b1a8     NeighborJoinAdapter.obj
 0002:000091b0       __ehfuncinfo$?createCalculatePhyTreeTask@NeighborJoinAdapter@U2@@UAEPAVTask@2@ABVMultipleSequenceAlignment@2@ABVCreatePhyTreeSettings@2@@Z 1004b1b0     NeighborJoinAdapter.obj
 0002:000091d4       __unwindtable$?createPhyTreeSettingsWidget@NeighborJoinAdapter@U2@@UAEPAVCreatePhyTreeWidget@2@ABVMultipleSequenceAlignment@2@PAVQWidget@@@Z 1004b1d4     NeighborJoinAdapter.obj
 0002:000091dc       __ehfuncinfo$?createPhyTreeSettingsWidget@NeighborJoinAdapter@U2@@UAEPAVCreatePhyTreeWidget@2@ABVMultipleSequenceAlignment@2@PAVQWidget@@@Z 1004b1dc     NeighborJoinAdapter.obj
 0002:00009200       __unwindtable$??0NeighborJoinCalculateTreeTask@U2@@QAE@ABVMultipleSequenceAlignment@1@ABVCreatePhyTreeSettings@1@@Z 1004b200     NeighborJoinAdapter.obj
 0002:00009220       __ehfuncinfo$??0NeighborJoinCalculateTreeTask@U2@@QAE@ABVMultipleSequenceAlignment@1@ABVCreatePhyTreeSettings@1@@Z 1004b220     NeighborJoinAdapter.obj
 0002:00009244       __tryblocktable$?run@NeighborJoinCalculateTreeTask@U2@@UAEXXZ 1004b244     NeighborJoinAdapter.obj
 0002:00009258       __catchsym$?run@NeighborJoinCalculateTreeTask@U2@@UAEXXZ$52 1004b258     NeighborJoinAdapter.obj
 0002:00009278       __ehfuncinfo$?run@NeighborJoinCalculateTreeTask@U2@@UAEXXZ 1004b278     NeighborJoinAdapter.obj
 0002:0000929c       __unwindtable$?run@NeighborJoinCalculateTreeTask@U2@@UAEXXZ 1004b29c     NeighborJoinAdapter.obj
 0002:00009434       __unwindtable$??1NeighborJoinCalculateTreeTask@U2@@UAE@XZ 1004b434     NeighborJoinAdapter.obj
 0002:00009444       __ehfuncinfo$??1NeighborJoinCalculateTreeTask@U2@@UAE@XZ 1004b444     NeighborJoinAdapter.obj
 0002:00009468       __unwindtable$??_GNeighborJoinCalculateTreeTask@U2@@UAEPAXI@Z 1004b468     NeighborJoinAdapter.obj
 0002:00009478       __ehfuncinfo$??_GNeighborJoinCalculateTreeTask@U2@@UAEPAXI@Z 1004b478     NeighborJoinAdapter.obj
 0002:0000949c       __ehfuncinfo$?createPhyTreeFromPhylipTree@U2@@YAXABVMultipleSequenceAlignment@1@PAUnode@@NE1PAVPhyNode@1@H@Z 1004b49c     NeighborJoinAdapter.obj
 0002:000094c0       __unwindtable$?createPhyTreeFromPhylipTree@U2@@YAXABVMultipleSequenceAlignment@1@PAUnode@@NE1PAVPhyNode@1@H@Z 1004b4c0     NeighborJoinAdapter.obj
 0002:000094f0       __unwindtable$??H@YA?BVQString@@ABV0@PBD@Z 1004b4f0     NeighborJoinWidget.obj
 0002:00009500       __ehfuncinfo$??H@YA?BVQString@@ABV0@PBD@Z 1004b500     NeighborJoinWidget.obj
 0002:00009524       __catchsym$??0?$QList@VQString@@@@QAE@ABV0@@Z$2 1004b524     NeighborJoinWidget.obj
 0002:00009534       __unwindtable$??0?$QList@VQString@@@@QAE@ABV0@@Z 1004b534     NeighborJoinWidget.obj
 0002:00009544       __tryblocktable$??0?$QList@VQString@@@@QAE@ABV0@@Z 1004b544     NeighborJoinWidget.obj
 0002:00009558       __ehfuncinfo$??0?$QList@VQString@@@@QAE@ABV0@@Z 1004b558     NeighborJoinWidget.obj
 0002:0000957c       __unwindtable$??__EalgoLog@U2@@YAXXZ 1004b57c     NeighborJoinWidget.obj
 0002:00009584       __ehfuncinfo$??__EalgoLog@U2@@YAXXZ 1004b584     NeighborJoinWidget.obj
 0002:000095a8       __unwindtable$??__EcmdLog@U2@@YAXXZ 1004b5a8     NeighborJoinWidget.obj
 0002:000095b0       __ehfuncinfo$??__EcmdLog@U2@@YAXXZ 1004b5b0     NeighborJoinWidget.obj
 0002:000095d4       __unwindtable$??__EcoreLog@U2@@YAXXZ 1004b5d4     NeighborJoinWidget.obj
 0002:000095dc       __ehfuncinfo$??__EcoreLog@U2@@YAXXZ 1004b5dc     NeighborJoinWidget.obj
 0002:00009600       __unwindtable$??__EioLog@U2@@YAXXZ 1004b600     NeighborJoinWidget.obj
 0002:00009608       __ehfuncinfo$??__EioLog@U2@@YAXXZ 1004b608     NeighborJoinWidget.obj
 0002:0000962c       __unwindtable$??__EperfLog@U2@@YAXXZ 1004b62c     NeighborJoinWidget.obj
 0002:00009634       __ehfuncinfo$??__EperfLog@U2@@YAXXZ 1004b634     NeighborJoinWidget.obj
 0002:00009658       __unwindtable$??__EscriptLog@U2@@YAXXZ 1004b658     NeighborJoinWidget.obj
 0002:00009660       __ehfuncinfo$??__EscriptLog@U2@@YAXXZ 1004b660     NeighborJoinWidget.obj
 0002:00009684       __unwindtable$??__EtaskLog@U2@@YAXXZ 1004b684     NeighborJoinWidget.obj
 0002:0000968c       __ehfuncinfo$??__EtaskLog@U2@@YAXXZ 1004b68c     NeighborJoinWidget.obj
 0002:000096b0       __unwindtable$??__EuiLog@U2@@YAXXZ 1004b6b0     NeighborJoinWidget.obj
 0002:000096b8       __ehfuncinfo$??__EuiLog@U2@@YAXXZ 1004b6b8     NeighborJoinWidget.obj
 0002:000096dc       __unwindtable$??__EuserActLog@U2@@YAXXZ 1004b6dc     NeighborJoinWidget.obj
 0002:000096e4       __ehfuncinfo$??__EuserActLog@U2@@YAXXZ 1004b6e4     NeighborJoinWidget.obj
 0002:00009708       __ehfuncinfo$?setupUi@Ui_NeighborJoinWidget@@QAEXPAVQWidget@@@Z 1004b708     NeighborJoinWidget.obj
 0002:0000972c       __unwindtable$?setupUi@Ui_NeighborJoinWidget@@QAEXPAVQWidget@@@Z 1004b72c     NeighborJoinWidget.obj
 0002:00009984       __ehfuncinfo$?retranslateUi@Ui_NeighborJoinWidget@@QAEXPAVQWidget@@@Z 1004b984     NeighborJoinWidget.obj
 0002:000099a8       __unwindtable$?retranslateUi@Ui_NeighborJoinWidget@@QAEXPAVQWidget@@@Z 1004b9a8     NeighborJoinWidget.obj
 0002:00009a08       __unwindtable$??0NeighborJoinWidget@U2@@QAE@ABVMultipleSequenceAlignment@1@PAVQWidget@@@Z 1004ba08     NeighborJoinWidget.obj
 0002:00009a10       __ehfuncinfo$??0NeighborJoinWidget@U2@@QAE@ABVMultipleSequenceAlignment@1@PAVQWidget@@@Z 1004ba10     NeighborJoinWidget.obj
 0002:00009a34       __unwindtable$?fillSettings@NeighborJoinWidget@U2@@UAEXAAVCreatePhyTreeSettings@2@@Z 1004ba34     NeighborJoinWidget.obj
 0002:00009a44       __ehfuncinfo$?fillSettings@NeighborJoinWidget@U2@@UAEXAAVCreatePhyTreeSettings@2@@Z 1004ba44     NeighborJoinWidget.obj
 0002:00009a68       __ehfuncinfo$?storeSettings@NeighborJoinWidget@U2@@UAEXXZ 1004ba68     NeighborJoinWidget.obj
 0002:00009a8c       __unwindtable$?storeSettings@NeighborJoinWidget@U2@@UAEXXZ 1004ba8c     NeighborJoinWidget.obj
 0002:00009b74       __ehfuncinfo$?restoreDefault@NeighborJoinWidget@U2@@UAEXXZ 1004bb74     NeighborJoinWidget.obj
 0002:00009b98       __unwindtable$?restoreDefault@NeighborJoinWidget@U2@@UAEXXZ 1004bb98     NeighborJoinWidget.obj
 0002:00009c28       __unwindtable$?checkMemoryEstimation@NeighborJoinWidget@U2@@UAE_NAAVQString@@ABVMultipleSequenceAlignment@2@ABVCreatePhyTreeSettings@2@@Z 1004bc28     NeighborJoinWidget.obj
 0002:00009c38       __ehfuncinfo$?checkMemoryEstimation@NeighborJoinWidget@U2@@UAE_NAAVQString@@ABVMultipleSequenceAlignment@2@ABVCreatePhyTreeSettings@2@@Z 1004bc38     NeighborJoinWidget.obj
 0002:00009c5c       __unwindtable$?checkSettings@NeighborJoinWidget@U2@@UAE_NAAVQString@@ABVCreatePhyTreeSettings@2@@Z 1004bc5c     NeighborJoinWidget.obj
 0002:00009c64       __ehfuncinfo$?checkSettings@NeighborJoinWidget@U2@@UAE_NAAVQString@@ABVCreatePhyTreeSettings@2@@Z 1004bc64     NeighborJoinWidget.obj
 0002:00009c88       __ehfuncinfo$?init@NeighborJoinWidget@U2@@AAEXABVMultipleSequenceAlignment@2@@Z 1004bc88     NeighborJoinWidget.obj
 0002:00009cac       __unwindtable$?init@NeighborJoinWidget@U2@@AAEXABVMultipleSequenceAlignment@2@@Z 1004bcac     NeighborJoinWidget.obj
 0002:00009e7c       __unwindtable$??H@YA?BVQString@@PBDABV0@@Z 1004be7c     PhylipCmdlineTask.obj
 0002:00009e84       __ehfuncinfo$??H@YA?BVQString@@PBDABV0@@Z 1004be84     PhylipCmdlineTask.obj
 0002:00009ea8       __catchsym$??0?$QList@VQByteArray@@@@QAE@ABV0@@Z$2 1004bea8     PhylipCmdlineTask.obj
 0002:00009eb8       __unwindtable$??0?$QList@VQByteArray@@@@QAE@ABV0@@Z 1004beb8     PhylipCmdlineTask.obj
 0002:00009ec8       __tryblocktable$??0?$QList@VQByteArray@@@@QAE@ABV0@@Z 1004bec8     PhylipCmdlineTask.obj
 0002:00009edc       __ehfuncinfo$??0?$QList@VQByteArray@@@@QAE@ABV0@@Z 1004bedc     PhylipCmdlineTask.obj
 0002:00009f00       __catchsym$?detach_helper@?$QList@VQByteArray@@@@AAEXH@Z$2 1004bf00     PhylipCmdlineTask.obj
 0002:00009f10       __unwindtable$?detach_helper@?$QList@VQByteArray@@@@AAEXH@Z 1004bf10     PhylipCmdlineTask.obj
 0002:00009f20       __tryblocktable$?detach_helper@?$QList@VQByteArray@@@@AAEXH@Z 1004bf20     PhylipCmdlineTask.obj
 0002:00009f34       __ehfuncinfo$?detach_helper@?$QList@VQByteArray@@@@AAEXH@Z 1004bf34     PhylipCmdlineTask.obj
 0002:00009f58       __catchsym$?node_copy@?$QList@VQByteArray@@@@AAEXPAUNode@1@00@Z$6 1004bf58     PhylipCmdlineTask.obj
 0002:00009f68       __tryblocktable$?node_copy@?$QList@VQByteArray@@@@AAEXPAUNode@1@00@Z 1004bf68     PhylipCmdlineTask.obj
 0002:00009f7c       __ehfuncinfo$?node_copy@?$QList@VQByteArray@@@@AAEXPAUNode@1@00@Z 1004bf7c     PhylipCmdlineTask.obj
 0002:00009fa0       __unwindtable$?node_copy@?$QList@VQByteArray@@@@AAEXPAUNode@1@00@Z 1004bfa0     PhylipCmdlineTask.obj
 0002:00009fd0       __unwindtable$??__EalgoLog@U2@@YAXXZ 1004bfd0     PhylipCmdlineTask.obj
 0002:00009fd8       __ehfuncinfo$??__EalgoLog@U2@@YAXXZ 1004bfd8     PhylipCmdlineTask.obj
 0002:00009ffc       __unwindtable$??__EcmdLog@U2@@YAXXZ 1004bffc     PhylipCmdlineTask.obj
 0002:0000a004       __ehfuncinfo$??__EcmdLog@U2@@YAXXZ 1004c004     PhylipCmdlineTask.obj
 0002:0000a028       __unwindtable$??__EcoreLog@U2@@YAXXZ 1004c028     PhylipCmdlineTask.obj
 0002:0000a030       __ehfuncinfo$??__EcoreLog@U2@@YAXXZ 1004c030     PhylipCmdlineTask.obj
 0002:0000a054       __unwindtable$??__EioLog@U2@@YAXXZ 1004c054     PhylipCmdlineTask.obj
 0002:0000a05c       __ehfuncinfo$??__EioLog@U2@@YAXXZ 1004c05c     PhylipCmdlineTask.obj
 0002:0000a080       __unwindtable$??__EperfLog@U2@@YAXXZ 1004c080     PhylipCmdlineTask.obj
 0002:0000a088       __ehfuncinfo$??__EperfLog@U2@@YAXXZ 1004c088     PhylipCmdlineTask.obj
 0002:0000a0ac       __unwindtable$??__EscriptLog@U2@@YAXXZ 1004c0ac     PhylipCmdlineTask.obj
 0002:0000a0b4       __ehfuncinfo$??__EscriptLog@U2@@YAXXZ 1004c0b4     PhylipCmdlineTask.obj
 0002:0000a0d8       __unwindtable$??__EtaskLog@U2@@YAXXZ 1004c0d8     PhylipCmdlineTask.obj
 0002:0000a0e0       __ehfuncinfo$??__EtaskLog@U2@@YAXXZ 1004c0e0     PhylipCmdlineTask.obj
 0002:0000a104       __unwindtable$??__EuiLog@U2@@YAXXZ 1004c104     PhylipCmdlineTask.obj
 0002:0000a10c       __ehfuncinfo$??__EuiLog@U2@@YAXXZ 1004c10c     PhylipCmdlineTask.obj
 0002:0000a130       __unwindtable$??__EuserActLog@U2@@YAXXZ 1004c130     PhylipCmdlineTask.obj
 0002:0000a138       __ehfuncinfo$??__EuserActLog@U2@@YAXXZ 1004c138     PhylipCmdlineTask.obj
 0002:0000a15c       __catchsym$?append@?$QList@PAVGObject@U2@@@@QAEXABQAVGObject@U2@@@Z$6 1004c15c     PhylipCmdlineTask.obj
 0002:0000a16c       __tryblocktable$?append@?$QList@PAVGObject@U2@@@@QAEXABQAVGObject@U2@@@Z 1004c16c     PhylipCmdlineTask.obj
 0002:0000a180       __ehfuncinfo$?append@?$QList@PAVGObject@U2@@@@QAEXABQAVGObject@U2@@@Z 1004c180     PhylipCmdlineTask.obj
 0002:0000a1a4       __unwindtable$?append@?$QList@PAVGObject@U2@@@@QAEXABQAVGObject@U2@@@Z 1004c1a4     PhylipCmdlineTask.obj
 0002:0000a1d4       __catchsym$?detach_helper_grow@?$QList@PAVGObject@U2@@@@AAEPAUNode@1@HH@Z$5 1004c1d4     PhylipCmdlineTask.obj
 0002:0000a1e4       __catchsym$?detach_helper_grow@?$QList@PAVGObject@U2@@@@AAEPAUNode@1@HH@Z$4 1004c1e4     PhylipCmdlineTask.obj
 0002:0000a1f4       __unwindtable$?detach_helper_grow@?$QList@PAVGObject@U2@@@@AAEPAUNode@1@HH@Z 1004c1f4     PhylipCmdlineTask.obj
 0002:0000a214       __ehfuncinfo$?detach_helper_grow@?$QList@PAVGObject@U2@@@@AAEPAUNode@1@HH@Z 1004c214     PhylipCmdlineTask.obj
 0002:0000a238       __tryblocktable$?detach_helper_grow@?$QList@PAVGObject@U2@@@@AAEPAUNode@1@HH@Z 1004c238     PhylipCmdlineTask.obj
 0002:0000a260       __unwindtable$??A?$QHash@VQString@@V1@@@QAEAAVQString@@ABV1@@Z 1004c260     PhylipCmdlineTask.obj
 0002:0000a268       __ehfuncinfo$??A?$QHash@VQString@@V1@@@QAEAAVQString@@ABV1@@Z 1004c268     PhylipCmdlineTask.obj
 0002:0000a28c       __unwindtable$?createNode@?$QHash@VQString@@V1@@@AAEPAU?$QHashNode@VQString@@V1@@@IABVQString@@0PAPAU2@@Z 1004c28c     PhylipCmdlineTask.obj
 0002:0000a29c       __ehfuncinfo$?createNode@?$QHash@VQString@@V1@@@AAEPAU?$QHashNode@VQString@@V1@@@IABVQString@@0PAPAU2@@Z 1004c29c     PhylipCmdlineTask.obj
 0002:0000a2c0       __unwindtable$?deleteNode2@?$QHash@VQString@@V1@@@CAXPAUNode@QHashData@@@Z 1004c2c0     PhylipCmdlineTask.obj
 0002:0000a2c8       __ehfuncinfo$?deleteNode2@?$QHash@VQString@@V1@@@CAXPAUNode@QHashData@@@Z 1004c2c8     PhylipCmdlineTask.obj
 0002:0000a2ec       __unwindtable$?duplicateNode@?$QHash@VQString@@V1@@@CAXPAUNode@QHashData@@PAX@Z 1004c2ec     PhylipCmdlineTask.obj
 0002:0000a2fc       __ehfuncinfo$?duplicateNode@?$QHash@VQString@@V1@@@CAXPAUNode@QHashData@@PAX@Z 1004c2fc     PhylipCmdlineTask.obj
 0002:0000a320       __ehfuncinfo$??0PhylipCmdlineTask@U2@@QAE@ABVMultipleSequenceAlignment@1@ABVCreatePhyTreeSettings@1@@Z 1004c320     PhylipCmdlineTask.obj
 0002:0000a344       __unwindtable$??0PhylipCmdlineTask@U2@@QAE@ABVMultipleSequenceAlignment@1@ABVCreatePhyTreeSettings@1@@Z 1004c344     PhylipCmdlineTask.obj
 0002:0000a384       __unwindtable$??1PhylipCmdlineTask@U2@@UAE@XZ 1004c384     PhylipCmdlineTask.obj
 0002:0000a39c       __ehfuncinfo$??1PhylipCmdlineTask@U2@@UAE@XZ 1004c39c     PhylipCmdlineTask.obj
 0002:0000a3c0       __ehfuncinfo$?report@PhylipCmdlineTask@U2@@UAE?AW4ReportResult@Task@2@XZ 1004c3c0     PhylipCmdlineTask.obj
 0002:0000a3e4       __unwindtable$?report@PhylipCmdlineTask@U2@@UAE?AW4ReportResult@Task@2@XZ 1004c3e4     PhylipCmdlineTask.obj
 0002:0000a42c       __ehfuncinfo$?createCmdlineTask@PhylipCmdlineTask@U2@@AAEXXZ 1004c42c     PhylipCmdlineTask.obj
 0002:0000a450       __unwindtable$?createCmdlineTask@PhylipCmdlineTask@U2@@AAEXXZ 1004c450     PhylipCmdlineTask.obj
 0002:0000a508       __ehfuncinfo$?prepareTempDbi@PhylipCmdlineTask@U2@@AAEXXZ 1004c508     PhylipCmdlineTask.obj
 0002:0000a52c       __unwindtable$?prepareTempDbi@PhylipCmdlineTask@U2@@AAEXXZ 1004c52c     PhylipCmdlineTask.obj
 0002:0000a574       __unwindtable$??_GPhylipCmdlineTask@U2@@UAEPAXI@Z 1004c574     PhylipCmdlineTask.obj
 0002:0000a58c       __ehfuncinfo$??_GPhylipCmdlineTask@U2@@UAEPAXI@Z 1004c58c     PhylipCmdlineTask.obj
 0002:0000a5b0       __unwindtable$??0?$QHashNode@VQString@@V1@@@QAE@ABVQString@@0IPAU0@@Z 1004c5b0     PhylipCmdlineTask.obj
 0002:0000a5b8       __ehfuncinfo$??0?$QHashNode@VQString@@V1@@@QAE@ABVQString@@0IPAU0@@Z 1004c5b8     PhylipCmdlineTask.obj
 0002:0000a5dc       __unwindtable$??1?$QHashNode@VQString@@V1@@@QAE@XZ 1004c5dc     PhylipCmdlineTask.obj
 0002:0000a5e4       __ehfuncinfo$??1?$QHashNode@VQString@@V1@@@QAE@XZ 1004c5e4     PhylipCmdlineTask.obj
 0002:0000a608       __unwindtable$??_G?$QHashNode@VQString@@V1@@@QAEPAXI@Z 1004c608     PhylipCmdlineTask.obj
 0002:0000a610       __ehfuncinfo$??_G?$QHashNode@VQString@@V1@@@QAEPAXI@Z 1004c610     PhylipCmdlineTask.obj
 0002:0000a634       __unwindtable$??__EalgoLog@U2@@YAXXZ 1004c634     PhylipPlugin.obj
 0002:0000a63c       __ehfuncinfo$??__EalgoLog@U2@@YAXXZ 1004c63c     PhylipPlugin.obj
 0002:0000a660       __unwindtable$??__EcmdLog@U2@@YAXXZ 1004c660     PhylipPlugin.obj
 0002:0000a668       __ehfuncinfo$??__EcmdLog@U2@@YAXXZ 1004c668     PhylipPlugin.obj
 0002:0000a68c       __unwindtable$??__EcoreLog@U2@@YAXXZ 1004c68c     PhylipPlugin.obj
 0002:0000a694       __ehfuncinfo$??__EcoreLog@U2@@YAXXZ 1004c694     PhylipPlugin.obj
 0002:0000a6b8       __unwindtable$??__EioLog@U2@@YAXXZ 1004c6b8     PhylipPlugin.obj
 0002:0000a6c0       __ehfuncinfo$??__EioLog@U2@@YAXXZ 1004c6c0     PhylipPlugin.obj
 0002:0000a6e4       __unwindtable$??__EperfLog@U2@@YAXXZ 1004c6e4     PhylipPlugin.obj
 0002:0000a6ec       __ehfuncinfo$??__EperfLog@U2@@YAXXZ 1004c6ec     PhylipPlugin.obj
 0002:0000a710       __unwindtable$??__EscriptLog@U2@@YAXXZ 1004c710     PhylipPlugin.obj
 0002:0000a718       __ehfuncinfo$??__EscriptLog@U2@@YAXXZ 1004c718     PhylipPlugin.obj
 0002:0000a73c       __unwindtable$??__EtaskLog@U2@@YAXXZ 1004c73c     PhylipPlugin.obj
 0002:0000a744       __ehfuncinfo$??__EtaskLog@U2@@YAXXZ 1004c744     PhylipPlugin.obj
 0002:0000a768       __unwindtable$??__EuiLog@U2@@YAXXZ 1004c768     PhylipPlugin.obj
 0002:0000a770       __ehfuncinfo$??__EuiLog@U2@@YAXXZ 1004c770     PhylipPlugin.obj
 0002:0000a794       __unwindtable$??__EuserActLog@U2@@YAXXZ 1004c794     PhylipPlugin.obj
 0002:0000a79c       __ehfuncinfo$??__EuserActLog@U2@@YAXXZ 1004c79c     PhylipPlugin.obj
 0002:0000a7c0       __ehfuncinfo$??0PhylipPlugin@U2@@QAE@XZ 1004c7c0     PhylipPlugin.obj
 0002:0000a7e4       __unwindtable$??0PhylipPlugin@U2@@QAE@XZ 1004c7e4     PhylipPlugin.obj
 0002:0000a824       __ehfuncinfo$?processCmdlineOptions@PhylipPlugin@U2@@AAEXXZ 1004c824     PhylipPlugin.obj
 0002:0000a848       __unwindtable$?processCmdlineOptions@PhylipPlugin@U2@@AAEXXZ 1004c848     PhylipPlugin.obj
 0002:0000a8a8       __unwindtable$??1?$GAutoDeleteList@VXMLTestFactory@U2@@@U2@@UAE@XZ 1004c8a8     PhylipPlugin.obj
 0002:0000a8b8       __ehfuncinfo$??1?$GAutoDeleteList@VXMLTestFactory@U2@@@U2@@UAE@XZ 1004c8b8     PhylipPlugin.obj
 0002:0000a8dc       __catchsym$??0?$QList@PAVXMLTestFactory@U2@@@@QAE@ABV0@@Z$2 1004c8dc     PhylipPlugin.obj
 0002:0000a8ec       __unwindtable$??0?$QList@PAVXMLTestFactory@U2@@@@QAE@ABV0@@Z 1004c8ec     PhylipPlugin.obj
 0002:0000a8fc       __tryblocktable$??0?$QList@PAVXMLTestFactory@U2@@@@QAE@ABV0@@Z 1004c8fc     PhylipPlugin.obj
 0002:0000a910       __ehfuncinfo$??0?$QList@PAVXMLTestFactory@U2@@@@QAE@ABV0@@Z 1004c910     PhylipPlugin.obj
 0002:0000a934       __ehfuncinfo$?fetchSettings@?A0xabc90af7@U2@@YA?AVCreatePhyTreeSettings@2@XZ 1004c934     PhylipPlugin.obj
 0002:0000a958       __unwindtable$?fetchSettings@?A0xabc90af7@U2@@YA?AVCreatePhyTreeSettings@2@XZ 1004c958     PhylipPlugin.obj
 0002:0000a9a8       __catchsym$?detach_helper@?$QList@PAVGObject@U2@@@@AAEXH@Z$2 1004c9a8     PhylipPluginTests.obj
 0002:0000a9b8       __unwindtable$?detach_helper@?$QList@PAVGObject@U2@@@@AAEXH@Z 1004c9b8     PhylipPluginTests.obj
 0002:0000a9c8       __tryblocktable$?detach_helper@?$QList@PAVGObject@U2@@@@AAEXH@Z 1004c9c8     PhylipPluginTests.obj
 0002:0000a9dc       __ehfuncinfo$?detach_helper@?$QList@PAVGObject@U2@@@@AAEXH@Z 1004c9dc     PhylipPluginTests.obj
 0002:0000aa00       __unwindtable$??__EalgoLog@U2@@YAXXZ 1004ca00     PhylipPluginTests.obj
 0002:0000aa08       __ehfuncinfo$??__EalgoLog@U2@@YAXXZ 1004ca08     PhylipPluginTests.obj
 0002:0000aa2c       __unwindtable$??__EcmdLog@U2@@YAXXZ 1004ca2c     PhylipPluginTests.obj
 0002:0000aa34       __ehfuncinfo$??__EcmdLog@U2@@YAXXZ 1004ca34     PhylipPluginTests.obj
 0002:0000aa58       __unwindtable$??__EcoreLog@U2@@YAXXZ 1004ca58     PhylipPluginTests.obj
 0002:0000aa60       __ehfuncinfo$??__EcoreLog@U2@@YAXXZ 1004ca60     PhylipPluginTests.obj
 0002:0000aa84       __unwindtable$??__EioLog@U2@@YAXXZ 1004ca84     PhylipPluginTests.obj
 0002:0000aa8c       __ehfuncinfo$??__EioLog@U2@@YAXXZ 1004ca8c     PhylipPluginTests.obj
 0002:0000aab0       __unwindtable$??__EperfLog@U2@@YAXXZ 1004cab0     PhylipPluginTests.obj
 0002:0000aab8       __ehfuncinfo$??__EperfLog@U2@@YAXXZ 1004cab8     PhylipPluginTests.obj
 0002:0000aadc       __unwindtable$??__EscriptLog@U2@@YAXXZ 1004cadc     PhylipPluginTests.obj
 0002:0000aae4       __ehfuncinfo$??__EscriptLog@U2@@YAXXZ 1004cae4     PhylipPluginTests.obj
 0002:0000ab08       __unwindtable$??__EtaskLog@U2@@YAXXZ 1004cb08     PhylipPluginTests.obj
 0002:0000ab10       __ehfuncinfo$??__EtaskLog@U2@@YAXXZ 1004cb10     PhylipPluginTests.obj
 0002:0000ab34       __unwindtable$??__EuiLog@U2@@YAXXZ 1004cb34     PhylipPluginTests.obj
 0002:0000ab3c       __ehfuncinfo$??__EuiLog@U2@@YAXXZ 1004cb3c     PhylipPluginTests.obj
 0002:0000ab60       __unwindtable$??__EuserActLog@U2@@YAXXZ 1004cb60     PhylipPluginTests.obj
 0002:0000ab68       __ehfuncinfo$??__EuserActLog@U2@@YAXXZ 1004cb68     PhylipPluginTests.obj
 0002:0000ab8c       __unwindtable$??0GTest_NeighborJoin@U2@@QAE@PAVXMLTestFormat@1@ABVQString@@PAVGTest@1@PBVGTestEnvironment@1@ABV?$QList@PAVGTest@U2@@@@ABVQDomElement@@@Z 1004cb8c     PhylipPluginTests.obj
 0002:0000aba4       __ehfuncinfo$??0GTest_NeighborJoin@U2@@QAE@PAVXMLTestFormat@1@ABVQString@@PAVGTest@1@PBVGTestEnvironment@1@ABV?$QList@PAVGTest@U2@@@@ABVQDomElement@@@Z 1004cba4     PhylipPluginTests.obj
 0002:0000abc8       __ehfuncinfo$?init@GTest_NeighborJoin@U2@@QAEXPAVXMLTestFormat@2@ABVQDomElement@@@Z 1004cbc8     PhylipPluginTests.obj
 0002:0000abec       __unwindtable$?init@GTest_NeighborJoin@U2@@QAEXPAVXMLTestFormat@2@ABVQDomElement@@@Z 1004cbec     PhylipPluginTests.obj
 0002:0000ac44       __unwindtable$??0GTest_NeighborJoinFactory@GTest_NeighborJoin@U2@@QAE@XZ 1004cc44     PhylipPluginTests.obj
 0002:0000ac5c       __ehfuncinfo$??0GTest_NeighborJoinFactory@GTest_NeighborJoin@U2@@QAE@XZ 1004cc5c     PhylipPluginTests.obj
 0002:0000ac80       __unwindtable$?createTest@GTest_NeighborJoinFactory@GTest_NeighborJoin@U2@@UAEPAVGTest@3@PAVXMLTestFormat@3@ABVQString@@PAV43@PBVGTestEnvironment@3@ABV?$QList@PAVGTest@U2@@@@ABVQDomElement@@@Z 1004cc80     PhylipPluginTests.obj
 0002:0000aca0       __ehfuncinfo$?createTest@GTest_NeighborJoinFactory@GTest_NeighborJoin@U2@@UAEPAVGTest@3@PAVXMLTestFormat@3@ABVQString@@PAV43@PBVGTestEnvironment@3@ABV?$QList@PAVGTest@U2@@@@ABVQDomElement@@@Z 1004cca0     PhylipPluginTests.obj
 0002:0000acc4       __unwindtable$?createFactory@GTest_NeighborJoin@U2@@SAPAVXMLTestFactory@2@XZ 1004ccc4     PhylipPluginTests.obj
 0002:0000ace4       __ehfuncinfo$?createFactory@GTest_NeighborJoin@U2@@SAPAVXMLTestFactory@2@XZ 1004cce4     PhylipPluginTests.obj
 0002:0000ad08       __ehfuncinfo$?prepare@GTest_NeighborJoin@U2@@UAEXXZ 1004cd08     PhylipPluginTests.obj
 0002:0000ad2c       __unwindtable$?prepare@GTest_NeighborJoin@U2@@UAEXXZ 1004cd2c     PhylipPluginTests.obj
 0002:0000adcc       __unwindtable$?report@GTest_NeighborJoin@U2@@UAE?AW4ReportResult@Task@2@XZ 1004cdcc     PhylipPluginTests.obj
 0002:0000ade4       __ehfuncinfo$?report@GTest_NeighborJoin@U2@@UAE?AW4ReportResult@Task@2@XZ 1004cde4     PhylipPluginTests.obj
 0002:0000ae08       __unwindtable$??1GTest_NeighborJoin@U2@@UAE@XZ 1004ce08     PhylipPluginTests.obj
 0002:0000ae18       __ehfuncinfo$??1GTest_NeighborJoin@U2@@UAE@XZ 1004ce18     PhylipPluginTests.obj
 0002:0000ae3c       __unwindtable$??_GGTest_NeighborJoin@U2@@UAEPAXI@Z 1004ce3c     PhylipPluginTests.obj
 0002:0000ae4c       __ehfuncinfo$??_GGTest_NeighborJoin@U2@@UAEPAXI@Z 1004ce4c     PhylipPluginTests.obj
 0002:0000ae70       __unwindtable$?createTestFactories@PhylipPluginTests@U2@@SA?AV?$QList@PAVXMLTestFactory@U2@@@@XZ 1004ce70     PhylipPluginTests.obj
 0002:0000ae78       __ehfuncinfo$?createTestFactories@PhylipPluginTests@U2@@SA?AV?$QList@PAVXMLTestFactory@U2@@@@XZ 1004ce78     PhylipPluginTests.obj
 0002:0000ae9c       __catchsym$?append@?$QList@PAVXMLTestFactory@U2@@@@QAEXABQAVXMLTestFactory@U2@@@Z$6 1004ce9c     PhylipPluginTests.obj
 0002:0000aeac       __tryblocktable$?append@?$QList@PAVXMLTestFactory@U2@@@@QAEXABQAVXMLTestFactory@U2@@@Z 1004ceac     PhylipPluginTests.obj
 0002:0000aec0       __ehfuncinfo$?append@?$QList@PAVXMLTestFactory@U2@@@@QAEXABQAVXMLTestFactory@U2@@@Z 1004cec0     PhylipPluginTests.obj
 0002:0000aee4       __unwindtable$?append@?$QList@PAVXMLTestFactory@U2@@@@QAEXABQAVXMLTestFactory@U2@@@Z 1004cee4     PhylipPluginTests.obj
 0002:0000af14       __catchsym$?detach_helper_grow@?$QList@PAVXMLTestFactory@U2@@@@AAEPAUNode@1@HH@Z$5 1004cf14     PhylipPluginTests.obj
 0002:0000af24       __catchsym$?detach_helper_grow@?$QList@PAVXMLTestFactory@U2@@@@AAEPAUNode@1@HH@Z$4 1004cf24     PhylipPluginTests.obj
 0002:0000af34       __unwindtable$?detach_helper_grow@?$QList@PAVXMLTestFactory@U2@@@@AAEPAUNode@1@HH@Z 1004cf34     PhylipPluginTests.obj
 0002:0000af54       __ehfuncinfo$?detach_helper_grow@?$QList@PAVXMLTestFactory@U2@@@@AAEPAUNode@1@HH@Z 1004cf54     PhylipPluginTests.obj
 0002:0000af78       __tryblocktable$?detach_helper_grow@?$QList@PAVXMLTestFactory@U2@@@@AAEPAUNode@1@HH@Z 1004cf78     PhylipPluginTests.obj
 0002:0000afa0       __unwindtable$??__EalgoLog@U2@@YAXXZ 1004cfa0     PhylipTask.obj
 0002:0000afa8       __ehfuncinfo$??__EalgoLog@U2@@YAXXZ 1004cfa8     PhylipTask.obj
 0002:0000afcc       __unwindtable$??__EcmdLog@U2@@YAXXZ 1004cfcc     PhylipTask.obj
 0002:0000afd4       __ehfuncinfo$??__EcmdLog@U2@@YAXXZ 1004cfd4     PhylipTask.obj
 0002:0000aff8       __unwindtable$??__EcoreLog@U2@@YAXXZ 1004cff8     PhylipTask.obj
 0002:0000b000       __ehfuncinfo$??__EcoreLog@U2@@YAXXZ 1004d000     PhylipTask.obj
 0002:0000b024       __unwindtable$??__EioLog@U2@@YAXXZ 1004d024     PhylipTask.obj
 0002:0000b02c       __ehfuncinfo$??__EioLog@U2@@YAXXZ 1004d02c     PhylipTask.obj
 0002:0000b050       __unwindtable$??__EperfLog@U2@@YAXXZ 1004d050     PhylipTask.obj
 0002:0000b058       __ehfuncinfo$??__EperfLog@U2@@YAXXZ 1004d058     PhylipTask.obj
 0002:0000b07c       __unwindtable$??__EscriptLog@U2@@YAXXZ 1004d07c     PhylipTask.obj
 0002:0000b084       __ehfuncinfo$??__EscriptLog@U2@@YAXXZ 1004d084     PhylipTask.obj
 0002:0000b0a8       __unwindtable$??__EtaskLog@U2@@YAXXZ 1004d0a8     PhylipTask.obj
 0002:0000b0b0       __ehfuncinfo$??__EtaskLog@U2@@YAXXZ 1004d0b0     PhylipTask.obj
 0002:0000b0d4       __unwindtable$??__EuiLog@U2@@YAXXZ 1004d0d4     PhylipTask.obj
 0002:0000b0dc       __ehfuncinfo$??__EuiLog@U2@@YAXXZ 1004d0dc     PhylipTask.obj
 0002:0000b100       __unwindtable$??__EuserActLog@U2@@YAXXZ 1004d100     PhylipTask.obj
 0002:0000b108       __ehfuncinfo$??__EuserActLog@U2@@YAXXZ 1004d108     PhylipTask.obj
 0002:0000b12c       __ehfuncinfo$??0PhylipTask@U2@@QAE@ABVU2EntityRef@1@ABVU2DbiRef@1@ABVCreatePhyTreeSettings@1@@Z 1004d12c     PhylipTask.obj
 0002:0000b150       __unwindtable$??0PhylipTask@U2@@QAE@ABVU2EntityRef@1@ABVU2DbiRef@1@ABVCreatePhyTreeSettings@1@@Z 1004d150     PhylipTask.obj
 0002:0000b178       __ehfuncinfo$?prepare@PhylipTask@U2@@UAEXXZ 1004d178     PhylipTask.obj
 0002:0000b19c       __unwindtable$?prepare@PhylipTask@U2@@UAEXXZ 1004d19c     PhylipTask.obj
 0002:0000b20c       __unwindtable$?report@PhylipTask@U2@@UAE?AW4ReportResult@Task@2@XZ 1004d20c     PhylipTask.obj
 0002:0000b214       __ehfuncinfo$?report@PhylipTask@U2@@UAE?AW4ReportResult@Task@2@XZ 1004d214     PhylipTask.obj
 0002:0000b238       __ehfuncinfo$?saveTree@PhylipTask@U2@@AAE?AVQByteArray@@XZ 1004d238     PhylipTask.obj
 0002:0000b25c       __unwindtable$?saveTree@PhylipTask@U2@@AAE?AVQByteArray@@XZ 1004d25c     PhylipTask.obj
 0002:0000b284       __unwindtable$??1PhylipTask@U2@@UAE@XZ 1004d284     PhylipTask.obj
 0002:0000b29c       __ehfuncinfo$??1PhylipTask@U2@@UAE@XZ 1004d29c     PhylipTask.obj
 0002:0000b2c0       __unwindtable$??_GPhylipTask@U2@@UAEPAXI@Z 1004d2c0     PhylipTask.obj
 0002:0000b2d8       __ehfuncinfo$??_GPhylipTask@U2@@UAEPAXI@Z 1004d2d8     PhylipTask.obj
 0002:0000b2fc       __unwindtable$??__EalgoLog@U2@@YAXXZ 1004d2fc     SeqBootAdapter.obj
 0002:0000b304       __ehfuncinfo$??__EalgoLog@U2@@YAXXZ 1004d304     SeqBootAdapter.obj
 0002:0000b328       __unwindtable$??__EcmdLog@U2@@YAXXZ 1004d328     SeqBootAdapter.obj
 0002:0000b330       __ehfuncinfo$??__EcmdLog@U2@@YAXXZ 1004d330     SeqBootAdapter.obj
 0002:0000b354       __unwindtable$??__EcoreLog@U2@@YAXXZ 1004d354     SeqBootAdapter.obj
 0002:0000b35c       __ehfuncinfo$??__EcoreLog@U2@@YAXXZ 1004d35c     SeqBootAdapter.obj
 0002:0000b380       __unwindtable$??__EioLog@U2@@YAXXZ 1004d380     SeqBootAdapter.obj
 0002:0000b388       __ehfuncinfo$??__EioLog@U2@@YAXXZ 1004d388     SeqBootAdapter.obj
 0002:0000b3ac       __unwindtable$??__EperfLog@U2@@YAXXZ 1004d3ac     SeqBootAdapter.obj
 0002:0000b3b4       __ehfuncinfo$??__EperfLog@U2@@YAXXZ 1004d3b4     SeqBootAdapter.obj
 0002:0000b3d8       __unwindtable$??__EscriptLog@U2@@YAXXZ 1004d3d8     SeqBootAdapter.obj
 0002:0000b3e0       __ehfuncinfo$??__EscriptLog@U2@@YAXXZ 1004d3e0     SeqBootAdapter.obj
 0002:0000b404       __unwindtable$??__EtaskLog@U2@@YAXXZ 1004d404     SeqBootAdapter.obj
 0002:0000b40c       __ehfuncinfo$??__EtaskLog@U2@@YAXXZ 1004d40c     SeqBootAdapter.obj
 0002:0000b430       __unwindtable$??__EuiLog@U2@@YAXXZ 1004d430     SeqBootAdapter.obj
 0002:0000b438       __ehfuncinfo$??__EuiLog@U2@@YAXXZ 1004d438     SeqBootAdapter.obj
 0002:0000b45c       __unwindtable$??__EuserActLog@U2@@YAXXZ 1004d45c     SeqBootAdapter.obj
 0002:0000b464       __ehfuncinfo$??__EuserActLog@U2@@YAXXZ 1004d464     SeqBootAdapter.obj
 0002:0000b488       __unwindtable$?clear@?$QVector@VMultipleSequenceAlignment@U2@@@@QAEXXZ 1004d488     SeqBootAdapter.obj
 0002:0000b490       __ehfuncinfo$?clear@?$QVector@VMultipleSequenceAlignment@U2@@@@QAEXXZ 1004d490     SeqBootAdapter.obj
 0002:0000b4b4       __catchsym$?reallocData@?$QVector@VMultipleSequenceAlignment@U2@@@@AAEXHHV?$QFlags@W4AllocationOption@QArrayData@@@@@Z$6 1004d4b4     SeqBootAdapter.obj
 0002:0000b4c4       __catchsym$?reallocData@?$QVector@VMultipleSequenceAlignment@U2@@@@AAEXHHV?$QFlags@W4AllocationOption@QArrayData@@@@@Z$5 1004d4c4     SeqBootAdapter.obj
 0002:0000b4d4       __ehfuncinfo$?reallocData@?$QVector@VMultipleSequenceAlignment@U2@@@@AAEXHHV?$QFlags@W4AllocationOption@QArrayData@@@@@Z 1004d4d4     SeqBootAdapter.obj
 0002:0000b4f8       __tryblocktable$?reallocData@?$QVector@VMultipleSequenceAlignment@U2@@@@AAEXHHV?$QFlags@W4AllocationOption@QArrayData@@@@@Z 1004d4f8     SeqBootAdapter.obj
 0002:0000b520       __unwindtable$?reallocData@?$QVector@VMultipleSequenceAlignment@U2@@@@AAEXHHV?$QFlags@W4AllocationOption@QArrayData@@@@@Z 1004d520     SeqBootAdapter.obj
 0002:0000b548       __ehfuncinfo$?defaultConstruct@?$QVector@VMultipleSequenceAlignment@U2@@@@AAEXPAVMultipleSequenceAlignment@U2@@0@Z 1004d548     SeqBootAdapter.obj
 0002:0000b56c       __unwindtable$?defaultConstruct@?$QVector@VMultipleSequenceAlignment@U2@@@@AAEXPAVMultipleSequenceAlignment@U2@@0@Z 1004d56c     SeqBootAdapter.obj
 0002:0000b594       __unwindtable$?copyConstruct@?$QVector@VMultipleSequenceAlignment@U2@@@@AAEXPBVMultipleSequenceAlignment@U2@@0PAV23@@Z 1004d594     SeqBootAdapter.obj
 0002:0000b59c       __ehfuncinfo$?copyConstruct@?$QVector@VMultipleSequenceAlignment@U2@@@@AAEXPBVMultipleSequenceAlignment@U2@@0PAV23@@Z 1004d59c     SeqBootAdapter.obj
 0002:0000b5c0       __ehfuncinfo$?getTmpFileTemplate@SeqBoot@U2@@QAE?AVQString@@XZ 1004d5c0     SeqBootAdapter.obj
 0002:0000b5e4       __unwindtable$?getTmpFileTemplate@SeqBoot@U2@@QAE?AVQString@@XZ 1004d5e4     SeqBootAdapter.obj
 0002:0000b60c       __unwindtable$?generateSequencesFromAlignment@SeqBoot@U2@@QAEXABVMultipleSequenceAlignment@2@ABVCreatePhyTreeSettings@2@@Z 1004d60c     SeqBootAdapter.obj
 0002:0000b614       __ehfuncinfo$?generateSequencesFromAlignment@SeqBoot@U2@@QAEXABVMultipleSequenceAlignment@2@ABVCreatePhyTreeSettings@2@@Z 1004d614     SeqBootAdapter.obj
 0002:0000b638       __ehfuncinfo$?initGenerSeq@SeqBoot@U2@@QAEXHHH@Z 1004d638     SeqBootAdapter.obj
 0002:0000b65c       __unwindtable$?initGenerSeq@SeqBoot@U2@@QAEXHHH@Z 1004d65c     SeqBootAdapter.obj
 0002:0000b684       __ehfuncinfo$??0SeqBoot@U2@@QAE@XZ 1004d684     SeqBootAdapter.obj
 0002:0000b6a8       __unwindtable$??0SeqBoot@U2@@QAE@XZ 1004d6a8     SeqBootAdapter.obj
 0002:0000b6d0       __unwindtable$??1SeqBoot@U2@@QAE@XZ 1004d6d0     SeqBootAdapter.obj
 0002:0000b6e0       __ehfuncinfo$??1SeqBoot@U2@@QAE@XZ 1004d6e0     SeqBootAdapter.obj
 0002:0000b704       __unwindtable$??__EalgoLog@U2@@YAXXZ 1004d704     dist.obj
 0002:0000b70c       __ehfuncinfo$??__EalgoLog@U2@@YAXXZ 1004d70c     dist.obj
 0002:0000b730       __unwindtable$??__EcmdLog@U2@@YAXXZ 1004d730     dist.obj
 0002:0000b738       __ehfuncinfo$??__EcmdLog@U2@@YAXXZ 1004d738     dist.obj
 0002:0000b75c       __unwindtable$??__EcoreLog@U2@@YAXXZ 1004d75c     dist.obj
 0002:0000b764       __ehfuncinfo$??__EcoreLog@U2@@YAXXZ 1004d764     dist.obj
 0002:0000b788       __unwindtable$??__EioLog@U2@@YAXXZ 1004d788     dist.obj
 0002:0000b790       __ehfuncinfo$??__EioLog@U2@@YAXXZ 1004d790     dist.obj
 0002:0000b7b4       __unwindtable$??__EperfLog@U2@@YAXXZ 1004d7b4     dist.obj
 0002:0000b7bc       __ehfuncinfo$??__EperfLog@U2@@YAXXZ 1004d7bc     dist.obj
 0002:0000b7e0       __unwindtable$??__EscriptLog@U2@@YAXXZ 1004d7e0     dist.obj
 0002:0000b7e8       __ehfuncinfo$??__EscriptLog@U2@@YAXXZ 1004d7e8     dist.obj
 0002:0000b80c       __unwindtable$??__EtaskLog@U2@@YAXXZ 1004d80c     dist.obj
 0002:0000b814       __ehfuncinfo$??__EtaskLog@U2@@YAXXZ 1004d814     dist.obj
 0002:0000b838       __unwindtable$??__EuiLog@U2@@YAXXZ 1004d838     dist.obj
 0002:0000b840       __ehfuncinfo$??__EuiLog@U2@@YAXXZ 1004d840     dist.obj
 0002:0000b864       __unwindtable$??__EuserActLog@U2@@YAXXZ 1004d864     dist.obj
 0002:0000b86c       __ehfuncinfo$??__EuserActLog@U2@@YAXXZ 1004d86c     dist.obj
 0002:0000b890       __unwindtable$?treeoutr@@YAXPAUnode@@PAJPAUtree@@@Z 1004d890     dist.obj
 0002:0000b8a8       __ehfuncinfo$?treeoutr@@YAXPAUnode@@PAJPAUtree@@@Z 1004d8a8     dist.obj
 0002:0000b8cc       __unwindtable$?dist_treeout@@YAXPAUnode@@PAJNE0@Z 1004d8cc     dist.obj
 0002:0000b8e4       __ehfuncinfo$?dist_treeout@@YAXPAUnode@@PAJNE0@Z 1004d8e4     dist.obj
 0002:0000b908       __unwindtable$??__EalgoLog@U2@@YAXXZ 1004d908     dnadist.obj
 0002:0000b910       __ehfuncinfo$??__EalgoLog@U2@@YAXXZ 1004d910     dnadist.obj
 0002:0000b934       __unwindtable$??__EcmdLog@U2@@YAXXZ 1004d934     dnadist.obj
 0002:0000b93c       __ehfuncinfo$??__EcmdLog@U2@@YAXXZ 1004d93c     dnadist.obj
 0002:0000b960       __unwindtable$??__EcoreLog@U2@@YAXXZ 1004d960     dnadist.obj
 0002:0000b968       __ehfuncinfo$??__EcoreLog@U2@@YAXXZ 1004d968     dnadist.obj
 0002:0000b98c       __unwindtable$??__EioLog@U2@@YAXXZ 1004d98c     dnadist.obj
 0002:0000b994       __ehfuncinfo$??__EioLog@U2@@YAXXZ 1004d994     dnadist.obj
 0002:0000b9b8       __unwindtable$??__EperfLog@U2@@YAXXZ 1004d9b8     dnadist.obj
 0002:0000b9c0       __ehfuncinfo$??__EperfLog@U2@@YAXXZ 1004d9c0     dnadist.obj
 0002:0000b9e4       __unwindtable$??__EscriptLog@U2@@YAXXZ 1004d9e4     dnadist.obj
 0002:0000b9ec       __ehfuncinfo$??__EscriptLog@U2@@YAXXZ 1004d9ec     dnadist.obj
 0002:0000ba10       __unwindtable$??__EtaskLog@U2@@YAXXZ 1004da10     dnadist.obj
 0002:0000ba18       __ehfuncinfo$??__EtaskLog@U2@@YAXXZ 1004da18     dnadist.obj
 0002:0000ba3c       __unwindtable$??__EuiLog@U2@@YAXXZ 1004da3c     dnadist.obj
 0002:0000ba44       __ehfuncinfo$??__EuiLog@U2@@YAXXZ 1004da44     dnadist.obj
 0002:0000ba68       __unwindtable$??__EuserActLog@U2@@YAXXZ 1004da68     dnadist.obj
 0002:0000ba70       __ehfuncinfo$??__EuserActLog@U2@@YAXXZ 1004da70     dnadist.obj
 0002:0000ba94       __unwindtable$?getoptions@@YAXXZ 1004da94     dnadist.obj
 0002:0000ba9c       __ehfuncinfo$?getoptions@@YAXXZ 1004da9c     dnadist.obj
 0002:0000bac0       __unwindtable$??__EalgoLog@U2@@YAXXZ 1004dac0     neighbor.obj
 0002:0000bac8       __ehfuncinfo$??__EalgoLog@U2@@YAXXZ 1004dac8     neighbor.obj
 0002:0000baec       __unwindtable$??__EcmdLog@U2@@YAXXZ 1004daec     neighbor.obj
 0002:0000baf4       __ehfuncinfo$??__EcmdLog@U2@@YAXXZ 1004daf4     neighbor.obj
 0002:0000bb18       __unwindtable$??__EcoreLog@U2@@YAXXZ 1004db18     neighbor.obj
 0002:0000bb20       __ehfuncinfo$??__EcoreLog@U2@@YAXXZ 1004db20     neighbor.obj
 0002:0000bb44       __unwindtable$??__EioLog@U2@@YAXXZ 1004db44     neighbor.obj
 0002:0000bb4c       __ehfuncinfo$??__EioLog@U2@@YAXXZ 1004db4c     neighbor.obj
 0002:0000bb70       __unwindtable$??__EperfLog@U2@@YAXXZ 1004db70     neighbor.obj
 0002:0000bb78       __ehfuncinfo$??__EperfLog@U2@@YAXXZ 1004db78     neighbor.obj
 0002:0000bb9c       __unwindtable$??__EscriptLog@U2@@YAXXZ 1004db9c     neighbor.obj
 0002:0000bba4       __ehfuncinfo$??__EscriptLog@U2@@YAXXZ 1004dba4     neighbor.obj
 0002:0000bbc8       __unwindtable$??__EtaskLog@U2@@YAXXZ 1004dbc8     neighbor.obj
 0002:0000bbd0       __ehfuncinfo$??__EtaskLog@U2@@YAXXZ 1004dbd0     neighbor.obj
 0002:0000bbf4       __unwindtable$??__EuiLog@U2@@YAXXZ 1004dbf4     neighbor.obj
 0002:0000bbfc       __ehfuncinfo$??__EuiLog@U2@@YAXXZ 1004dbfc     neighbor.obj
 0002:0000bc20       __unwindtable$??__EuserActLog@U2@@YAXXZ 1004dc20     neighbor.obj
 0002:0000bc28       __ehfuncinfo$??__EuserActLog@U2@@YAXXZ 1004dc28     neighbor.obj
 0002:0000bc4c       __unwindtable$??__EalgoLog@U2@@YAXXZ 1004dc4c     phylip.obj
 0002:0000bc54       __ehfuncinfo$??__EalgoLog@U2@@YAXXZ 1004dc54     phylip.obj
 0002:0000bc78       __unwindtable$??__EcmdLog@U2@@YAXXZ 1004dc78     phylip.obj
 0002:0000bc80       __ehfuncinfo$??__EcmdLog@U2@@YAXXZ 1004dc80     phylip.obj
 0002:0000bca4       __unwindtable$??__EcoreLog@U2@@YAXXZ 1004dca4     phylip.obj
 0002:0000bcac       __ehfuncinfo$??__EcoreLog@U2@@YAXXZ 1004dcac     phylip.obj
 0002:0000bcd0       __unwindtable$??__EioLog@U2@@YAXXZ 1004dcd0     phylip.obj
 0002:0000bcd8       __ehfuncinfo$??__EioLog@U2@@YAXXZ 1004dcd8     phylip.obj
 0002:0000bcfc       __unwindtable$??__EperfLog@U2@@YAXXZ 1004dcfc     phylip.obj
 0002:0000bd04       __ehfuncinfo$??__EperfLog@U2@@YAXXZ 1004dd04     phylip.obj
 0002:0000bd28       __unwindtable$??__EscriptLog@U2@@YAXXZ 1004dd28     phylip.obj
 0002:0000bd30       __ehfuncinfo$??__EscriptLog@U2@@YAXXZ 1004dd30     phylip.obj
 0002:0000bd54       __unwindtable$??__EtaskLog@U2@@YAXXZ 1004dd54     phylip.obj
 0002:0000bd5c       __ehfuncinfo$??__EtaskLog@U2@@YAXXZ 1004dd5c     phylip.obj
 0002:0000bd80       __unwindtable$??__EuiLog@U2@@YAXXZ 1004dd80     phylip.obj
 0002:0000bd88       __ehfuncinfo$??__EuiLog@U2@@YAXXZ 1004dd88     phylip.obj
 0002:0000bdac       __unwindtable$??__EuserActLog@U2@@YAXXZ 1004ddac     phylip.obj
 0002:0000bdb4       __ehfuncinfo$??__EuserActLog@U2@@YAXXZ 1004ddb4     phylip.obj
 0002:0000be2c       __unwindtable$??__EalgoLog@U2@@YAXXZ 1004de2c     protdist.obj
 0002:0000be34       __ehfuncinfo$??__EalgoLog@U2@@YAXXZ 1004de34     protdist.obj
 0002:0000be58       __unwindtable$??__EcmdLog@U2@@YAXXZ 1004de58     protdist.obj
 0002:0000be60       __ehfuncinfo$??__EcmdLog@U2@@YAXXZ 1004de60     protdist.obj
 0002:0000be84       __unwindtable$??__EcoreLog@U2@@YAXXZ 1004de84     protdist.obj
 0002:0000be8c       __ehfuncinfo$??__EcoreLog@U2@@YAXXZ 1004de8c     protdist.obj
 0002:0000beb0       __unwindtable$??__EioLog@U2@@YAXXZ 1004deb0     protdist.obj
 0002:0000beb8       __ehfuncinfo$??__EioLog@U2@@YAXXZ 1004deb8     protdist.obj
 0002:0000bedc       __unwindtable$??__EperfLog@U2@@YAXXZ 1004dedc     protdist.obj
 0002:0000bee4       __ehfuncinfo$??__EperfLog@U2@@YAXXZ 1004dee4     protdist.obj
 0002:0000bf08       __unwindtable$??__EscriptLog@U2@@YAXXZ 1004df08     protdist.obj
 0002:0000bf10       __ehfuncinfo$??__EscriptLog@U2@@YAXXZ 1004df10     protdist.obj
 0002:0000bf34       __unwindtable$??__EtaskLog@U2@@YAXXZ 1004df34     protdist.obj
 0002:0000bf3c       __ehfuncinfo$??__EtaskLog@U2@@YAXXZ 1004df3c     protdist.obj
 0002:0000bf60       __unwindtable$??__EuiLog@U2@@YAXXZ 1004df60     protdist.obj
 0002:0000bf68       __ehfuncinfo$??__EuiLog@U2@@YAXXZ 1004df68     protdist.obj
 0002:0000bf8c       __unwindtable$??__EuserActLog@U2@@YAXXZ 1004df8c     protdist.obj
 0002:0000bf94       __ehfuncinfo$??__EuserActLog@U2@@YAXXZ 1004df94     protdist.obj
 0002:0000bfb8       __unwindtable$??__EalgoLog@U2@@YAXXZ 1004dfb8     seqboot.obj
 0002:0000bfc0       __ehfuncinfo$??__EalgoLog@U2@@YAXXZ 1004dfc0     seqboot.obj
 0002:0000bfe4       __unwindtable$??__EcmdLog@U2@@YAXXZ 1004dfe4     seqboot.obj
 0002:0000bfec       __ehfuncinfo$??__EcmdLog@U2@@YAXXZ 1004dfec     seqboot.obj
 0002:0000c010       __unwindtable$??__EcoreLog@U2@@YAXXZ 1004e010     seqboot.obj
 0002:0000c018       __ehfuncinfo$??__EcoreLog@U2@@YAXXZ 1004e018     seqboot.obj
 0002:0000c03c       __unwindtable$??__EioLog@U2@@YAXXZ 1004e03c     seqboot.obj
 0002:0000c044       __ehfuncinfo$??__EioLog@U2@@YAXXZ 1004e044     seqboot.obj
 0002:0000c068       __unwindtable$??__EperfLog@U2@@YAXXZ 1004e068     seqboot.obj
 0002:0000c070       __ehfuncinfo$??__EperfLog@U2@@YAXXZ 1004e070     seqboot.obj
 0002:0000c094       __unwindtable$??__EscriptLog@U2@@YAXXZ 1004e094     seqboot.obj
 0002:0000c09c       __ehfuncinfo$??__EscriptLog@U2@@YAXXZ 1004e09c     seqboot.obj
 0002:0000c0c0       __unwindtable$??__EtaskLog@U2@@YAXXZ 1004e0c0     seqboot.obj
 0002:0000c0c8       __ehfuncinfo$??__EtaskLog@U2@@YAXXZ 1004e0c8     seqboot.obj
 0002:0000c0ec       __unwindtable$??__EuiLog@U2@@YAXXZ 1004e0ec     seqboot.obj
 0002:0000c0f4       __ehfuncinfo$??__EuiLog@U2@@YAXXZ 1004e0f4     seqboot.obj
 0002:0000c118       __unwindtable$??__EuserActLog@U2@@YAXXZ 1004e118     seqboot.obj
 0002:0000c120       __ehfuncinfo$??__EuserActLog@U2@@YAXXZ 1004e120     seqboot.obj
 0002:0000c144       __unwindtable$?writedata@@YAXAAV?$QVector@VMultipleSequenceAlignment@U2@@@@HABVMultipleSequenceAlignment@U2@@@Z 1004e144     seqboot.obj
 0002:0000c15c       __ehfuncinfo$?writedata@@YAXAAV?$QVector@VMultipleSequenceAlignment@U2@@@@HABVMultipleSequenceAlignment@U2@@@Z 1004e15c     seqboot.obj
 0002:0000c180       __unwindtable$??__EalgoLog@U2@@YAXXZ 1004e180     moc_NeighborJoinWidget.obj
 0002:0000c188       __ehfuncinfo$??__EalgoLog@U2@@YAXXZ 1004e188     moc_NeighborJoinWidget.obj
 0002:0000c1ac       __unwindtable$??__EcmdLog@U2@@YAXXZ 1004e1ac     moc_NeighborJoinWidget.obj
 0002:0000c1b4       __ehfuncinfo$??__EcmdLog@U2@@YAXXZ 1004e1b4     moc_NeighborJoinWidget.obj
 0002:0000c1d8       __unwindtable$??__EcoreLog@U2@@YAXXZ 1004e1d8     moc_NeighborJoinWidget.obj
 0002:0000c1e0       __ehfuncinfo$??__EcoreLog@U2@@YAXXZ 1004e1e0     moc_NeighborJoinWidget.obj
 0002:0000c204       __unwindtable$??__EioLog@U2@@YAXXZ 1004e204     moc_NeighborJoinWidget.obj
 0002:0000c20c       __ehfuncinfo$??__EioLog@U2@@YAXXZ 1004e20c     moc_NeighborJoinWidget.obj
 0002:0000c230       __unwindtable$??__EperfLog@U2@@YAXXZ 1004e230     moc_NeighborJoinWidget.obj
 0002:0000c238       __ehfuncinfo$??__EperfLog@U2@@YAXXZ 1004e238     moc_NeighborJoinWidget.obj
 0002:0000c25c       __unwindtable$??__EscriptLog@U2@@YAXXZ 1004e25c     moc_NeighborJoinWidget.obj
 0002:0000c264       __ehfuncinfo$??__EscriptLog@U2@@YAXXZ 1004e264     moc_NeighborJoinWidget.obj
 0002:0000c288       __unwindtable$??__EtaskLog@U2@@YAXXZ 1004e288     moc_NeighborJoinWidget.obj
 0002:0000c290       __ehfuncinfo$??__EtaskLog@U2@@YAXXZ 1004e290     moc_NeighborJoinWidget.obj
 0002:0000c2b4       __unwindtable$??__EuiLog@U2@@YAXXZ 1004e2b4     moc_NeighborJoinWidget.obj
 0002:0000c2bc       __ehfuncinfo$??__EuiLog@U2@@YAXXZ 1004e2bc     moc_NeighborJoinWidget.obj
 0002:0000c2e0       __unwindtable$??__EuserActLog@U2@@YAXXZ 1004e2e0     moc_NeighborJoinWidget.obj
 0002:0000c2e8       __ehfuncinfo$??__EuserActLog@U2@@YAXXZ 1004e2e8     moc_NeighborJoinWidget.obj
 0002:0000c30c       __unwindtable$??__EalgoLog@U2@@YAXXZ 1004e30c     moc_PhylipCmdlineTask.obj
 0002:0000c314       __ehfuncinfo$??__EalgoLog@U2@@YAXXZ 1004e314     moc_PhylipCmdlineTask.obj
 0002:0000c338       __unwindtable$??__EcmdLog@U2@@YAXXZ 1004e338     moc_PhylipCmdlineTask.obj
 0002:0000c340       __ehfuncinfo$??__EcmdLog@U2@@YAXXZ 1004e340     moc_PhylipCmdlineTask.obj
 0002:0000c364       __unwindtable$??__EcoreLog@U2@@YAXXZ 1004e364     moc_PhylipCmdlineTask.obj
 0002:0000c36c       __ehfuncinfo$??__EcoreLog@U2@@YAXXZ 1004e36c     moc_PhylipCmdlineTask.obj
 0002:0000c390       __unwindtable$??__EioLog@U2@@YAXXZ 1004e390     moc_PhylipCmdlineTask.obj
 0002:0000c398       __ehfuncinfo$??__EioLog@U2@@YAXXZ 1004e398     moc_PhylipCmdlineTask.obj
 0002:0000c3bc       __unwindtable$??__EperfLog@U2@@YAXXZ 1004e3bc     moc_PhylipCmdlineTask.obj
 0002:0000c3c4       __ehfuncinfo$??__EperfLog@U2@@YAXXZ 1004e3c4     moc_PhylipCmdlineTask.obj
 0002:0000c3e8       __unwindtable$??__EscriptLog@U2@@YAXXZ 1004e3e8     moc_PhylipCmdlineTask.obj
 0002:0000c3f0       __ehfuncinfo$??__EscriptLog@U2@@YAXXZ 1004e3f0     moc_PhylipCmdlineTask.obj
 0002:0000c414       __unwindtable$??__EtaskLog@U2@@YAXXZ 1004e414     moc_PhylipCmdlineTask.obj
 0002:0000c41c       __ehfuncinfo$??__EtaskLog@U2@@YAXXZ 1004e41c     moc_PhylipCmdlineTask.obj
 0002:0000c440       __unwindtable$??__EuiLog@U2@@YAXXZ 1004e440     moc_PhylipCmdlineTask.obj
 0002:0000c448       __ehfuncinfo$??__EuiLog@U2@@YAXXZ 1004e448     moc_PhylipCmdlineTask.obj
 0002:0000c46c       __unwindtable$??__EuserActLog@U2@@YAXXZ 1004e46c     moc_PhylipCmdlineTask.obj
 0002:0000c474       __ehfuncinfo$??__EuserActLog@U2@@YAXXZ 1004e474     moc_PhylipCmdlineTask.obj
 0002:0000c498       __unwindtable$??__EalgoLog@U2@@YAXXZ 1004e498     moc_PhylipPluginTests.obj
 0002:0000c4a0       __ehfuncinfo$??__EalgoLog@U2@@YAXXZ 1004e4a0     moc_PhylipPluginTests.obj
 0002:0000c4c4       __unwindtable$??__EcmdLog@U2@@YAXXZ 1004e4c4     moc_PhylipPluginTests.obj
 0002:0000c4cc       __ehfuncinfo$??__EcmdLog@U2@@YAXXZ 1004e4cc     moc_PhylipPluginTests.obj
 0002:0000c4f0       __unwindtable$??__EcoreLog@U2@@YAXXZ 1004e4f0     moc_PhylipPluginTests.obj
 0002:0000c4f8       __ehfuncinfo$??__EcoreLog@U2@@YAXXZ 1004e4f8     moc_PhylipPluginTests.obj
 0002:0000c51c       __unwindtable$??__EioLog@U2@@YAXXZ 1004e51c     moc_PhylipPluginTests.obj
 0002:0000c524       __ehfuncinfo$??__EioLog@U2@@YAXXZ 1004e524     moc_PhylipPluginTests.obj
 0002:0000c548       __unwindtable$??__EperfLog@U2@@YAXXZ 1004e548     moc_PhylipPluginTests.obj
 0002:0000c550       __ehfuncinfo$??__EperfLog@U2@@YAXXZ 1004e550     moc_PhylipPluginTests.obj
 0002:0000c574       __unwindtable$??__EscriptLog@U2@@YAXXZ 1004e574     moc_PhylipPluginTests.obj
 0002:0000c57c       __ehfuncinfo$??__EscriptLog@U2@@YAXXZ 1004e57c     moc_PhylipPluginTests.obj
 0002:0000c5a0       __unwindtable$??__EtaskLog@U2@@YAXXZ 1004e5a0     moc_PhylipPluginTests.obj
 0002:0000c5a8       __ehfuncinfo$??__EtaskLog@U2@@YAXXZ 1004e5a8     moc_PhylipPluginTests.obj
 0002:0000c5cc       __unwindtable$??__EuiLog@U2@@YAXXZ 1004e5cc     moc_PhylipPluginTests.obj
 0002:0000c5d4       __ehfuncinfo$??__EuiLog@U2@@YAXXZ 1004e5d4     moc_PhylipPluginTests.obj
 0002:0000c5f8       __unwindtable$??__EuserActLog@U2@@YAXXZ 1004e5f8     moc_PhylipPluginTests.obj
 0002:0000c600       __ehfuncinfo$??__EuserActLog@U2@@YAXXZ 1004e600     moc_PhylipPluginTests.obj
 0002:0000c624       __unwindtable$??__EalgoLog@U2@@YAXXZ 1004e624     moc_PhylipTask.obj
 0002:0000c62c       __ehfuncinfo$??__EalgoLog@U2@@YAXXZ 1004e62c     moc_PhylipTask.obj
 0002:0000c650       __unwindtable$??__EcmdLog@U2@@YAXXZ 1004e650     moc_PhylipTask.obj
 0002:0000c658       __ehfuncinfo$??__EcmdLog@U2@@YAXXZ 1004e658     moc_PhylipTask.obj
 0002:0000c67c       __unwindtable$??__EcoreLog@U2@@YAXXZ 1004e67c     moc_PhylipTask.obj
 0002:0000c684       __ehfuncinfo$??__EcoreLog@U2@@YAXXZ 1004e684     moc_PhylipTask.obj
 0002:0000c6a8       __unwindtable$??__EioLog@U2@@YAXXZ 1004e6a8     moc_PhylipTask.obj
 0002:0000c6b0       __ehfuncinfo$??__EioLog@U2@@YAXXZ 1004e6b0     moc_PhylipTask.obj
 0002:0000c6d4       __unwindtable$??__EperfLog@U2@@YAXXZ 1004e6d4     moc_PhylipTask.obj
 0002:0000c6dc       __ehfuncinfo$??__EperfLog@U2@@YAXXZ 1004e6dc     moc_PhylipTask.obj
 0002:0000c700       __unwindtable$??__EscriptLog@U2@@YAXXZ 1004e700     moc_PhylipTask.obj
 0002:0000c708       __ehfuncinfo$??__EscriptLog@U2@@YAXXZ 1004e708     moc_PhylipTask.obj
 0002:0000c72c       __unwindtable$??__EtaskLog@U2@@YAXXZ 1004e72c     moc_PhylipTask.obj
 0002:0000c734       __ehfuncinfo$??__EtaskLog@U2@@YAXXZ 1004e734     moc_PhylipTask.obj
 0002:0000c758       __unwindtable$??__EuiLog@U2@@YAXXZ 1004e758     moc_PhylipTask.obj
 0002:0000c760       __ehfuncinfo$??__EuiLog@U2@@YAXXZ 1004e760     moc_PhylipTask.obj
 0002:0000c784       __unwindtable$??__EuserActLog@U2@@YAXXZ 1004e784     moc_PhylipTask.obj
 0002:0000c78c       __ehfuncinfo$??__EuserActLog@U2@@YAXXZ 1004e78c     moc_PhylipTask.obj
 0002:0000c7b0       __sehtable$__onexit        1004e7b0     MSVCRT:atonexit.obj
 0002:0000c7d0       __sehtable$___DllMainCRTStartup 1004e7d0     MSVCRT:crtdll.obj
 0002:0000c7f8       __sehtable$??_M@YGXPAXIHP6EX0@Z@Z 1004e7f8     MSVCRT:ehvecdtr.obj
 0002:0000c818       __sehtable$?__ArrayUnwind@@YGXPAXIHP6EX0@Z@Z 1004e818     MSVCRT:ehvecdtr.obj
 0002:0000c838       __sehtable$__IsNonwritableInCurrentImage 1004e838     MSVCRT:pesect.obj
 0002:0000c860       .edata                     1004e860     phylip.exp
 0002:0000c888       rgpv                       1004e888     phylip.exp
 0002:0000c88c       rgszName                   1004e88c     phylip.exp
 0002:0000c890       rgwOrd                     1004e890     phylip.exp
 0002:0000c892       szName                     1004e892     phylip.exp
 0002:0000c89d       $N00001                    1004e89d     phylip.exp
 0002:0000fcc0       .idata$6                   10051cc0     U2Core:U2Core.dll
 0002:000102b4       .idata$6                   100522b4     U2Algorithm:U2Algorithm.dll
 0002:000105b0       .idata$6                   100525b0     U2View:U2View.dll
 0002:00010814       .idata$6                   10052814     U2Test:U2Test.dll
 0002:000139d4       .idata$6                   100559d4     Qt5Widgets:Qt5Widgets.dll
 0002:00013a16       .idata$6                   10055a16     Qt5Xml:Qt5Xml.dll
 0002:00014a4e       .idata$6                   10056a4e     Qt5Core:Qt5Core.dll
 0002:00014afa       .idata$6                   10056afa     kernel32:KERNEL32.dll
 0002:00014e92       .idata$6                   10056e92     msvcprt:MSVCP120.dll
 0002:00015110       .idata$6                   10057110     MSVCRT:MSVCR120.dll
 0003:00000000       _jtteigs                   10058000     DistanceMatrix.obj
 0003:000000a0       _jttprobs                  100580a0     DistanceMatrix.obj
 0003:00000d20       _pmbeigs                   10058d20     DistanceMatrix.obj
 0003:00000dc0       _pmbprobs                  10058dc0     DistanceMatrix.obj
 0003:00001a40       _pameigs                   10059a40     DistanceMatrix.obj
 0003:00001ae0       _pamprobs                  10059ae0     DistanceMatrix.obj
 0003:00002770       _jtteigs                   1005a770     NeighborJoinAdapter.obj
 0003:00002810       _jttprobs                  1005a810     NeighborJoinAdapter.obj
 0003:00003490       _pmbeigs                   1005b490     NeighborJoinAdapter.obj
 0003:00003530       _pmbprobs                  1005b530     NeighborJoinAdapter.obj
 0003:000041b0       _pameigs                   1005c1b0     NeighborJoinAdapter.obj
 0003:00004250       _pamprobs                  1005c250     NeighborJoinAdapter.obj
 0003:00004ed0       _regular                   1005ced0     NeighborJoinAdapter.obj
 0003:00004ed1       _progress                  1005ced1     NeighborJoinAdapter.obj
 0003:00004ed8       _fracsample                1005ced8     NeighborJoinAdapter.obj
 0003:00004ee0       ?sz@?1??replacePhylipRestrictedSymbols@U2@@YAXAAVQByteArray@@@Z@4HA 1005cee0     NeighborJoinAdapter.obj
 0003:00004ee8       _jtteigs                   1005cee8     NeighborJoinWidget.obj
 0003:00004f88       _jttprobs                  1005cf88     NeighborJoinWidget.obj
 0003:00005c08       _pmbeigs                   1005dc08     NeighborJoinWidget.obj
 0003:00005ca8       _pmbprobs                  1005dca8     NeighborJoinWidget.obj
 0003:00006928       _pameigs                   1005e928     NeighborJoinWidget.obj
 0003:000069c8       _pamprobs                  1005e9c8     NeighborJoinWidget.obj
 0003:00007648       _Service_PluginViewer      1005f648     PhylipPlugin.obj
 0003:00007650       _Service_Project           1005f650     PhylipPlugin.obj
 0003:00007658       _Service_ProjectView       1005f658     PhylipPlugin.obj
 0003:00007660       _Service_DNAGraphPack      1005f660     PhylipPlugin.obj
 0003:00007668       _Service_DNAExport         1005f668     PhylipPlugin.obj
 0003:00007670       _Service_TestRunner        1005f670     PhylipPlugin.obj
 0003:00007678       _Service_ScriptRegistry    1005f678     PhylipPlugin.obj
 0003:00007680       _Service_ExternalToolSupport 1005f680     PhylipPlugin.obj
 0003:00007688       _Service_GUITesting        1005f688     PhylipPlugin.obj
 0003:00007690       _Service_WorkflowDesigner  1005f690     PhylipPlugin.obj
 0003:00007698       _Service_QueryDesigner     1005f698     PhylipPlugin.obj
 0003:000076a0       _Service_MinCoreServiceId  1005f6a0     PhylipPlugin.obj
 0003:000076a8       _Service_MaxCoreServiceId  1005f6a8     PhylipPlugin.obj
 0003:000076b0       _Service_PluginViewer      1005f6b0     PhylipPluginTests.obj
 0003:000076b8       _Service_Project           1005f6b8     PhylipPluginTests.obj
 0003:000076c0       _Service_ProjectView       1005f6c0     PhylipPluginTests.obj
 0003:000076c8       _Service_DNAGraphPack      1005f6c8     PhylipPluginTests.obj
 0003:000076d0       _Service_DNAExport         1005f6d0     PhylipPluginTests.obj
 0003:000076d8       _Service_TestRunner        1005f6d8     PhylipPluginTests.obj
 0003:000076e0       _Service_ScriptRegistry    1005f6e0     PhylipPluginTests.obj
 0003:000076e8       _Service_ExternalToolSupport 1005f6e8     PhylipPluginTests.obj
 0003:000076f0       _Service_GUITesting        1005f6f0     PhylipPluginTests.obj
 0003:000076f8       _Service_WorkflowDesigner  1005f6f8     PhylipPluginTests.obj
 0003:00007700       _Service_QueryDesigner     1005f700     PhylipPluginTests.obj
 0003:00007708       _Service_MinCoreServiceId  1005f708     PhylipPluginTests.obj
 0003:00007710       _Service_MaxCoreServiceId  1005f710     PhylipPluginTests.obj
 0003:00007718       _regular                   1005f718     SeqBootAdapter.obj
 0003:00007719       _progress                  1005f719     SeqBootAdapter.obj
 0003:00007720       _fracsample                1005f720     SeqBootAdapter.obj
 0003:00007728       _jtteigs                   1005f728     protdist.obj
 0003:000077c8       _jttprobs                  1005f7c8     protdist.obj
 0003:00008448       _pmbeigs                   10060448     protdist.obj
 0003:000084e8       _pmbprobs                  100604e8     protdist.obj
 0003:00009168       _pameigs                   10061168     protdist.obj
 0003:00009208       _pamprobs                  10061208     protdist.obj
 0003:00009e88       _regular                   10061e88     seqboot.obj
 0003:00009e89       _progress                  10061e89     seqboot.obj
 0003:00009e90       _fracsample                10061e90     seqboot.obj
 0003:00009ec8       _Service_PluginViewer      10061ec8     moc_PhylipPlugin.obj
 0003:00009ed0       _Service_Project           10061ed0     moc_PhylipPlugin.obj
 0003:00009ed8       _Service_ProjectView       10061ed8     moc_PhylipPlugin.obj
 0003:00009ee0       _Service_DNAGraphPack      10061ee0     moc_PhylipPlugin.obj
 0003:00009ee8       _Service_DNAExport         10061ee8     moc_PhylipPlugin.obj
 0003:00009ef0       _Service_TestRunner        10061ef0     moc_PhylipPlugin.obj
 0003:00009ef8       _Service_ScriptRegistry    10061ef8     moc_PhylipPlugin.obj
 0003:00009f00       _Service_ExternalToolSupport 10061f00     moc_PhylipPlugin.obj
 0003:00009f08       _Service_GUITesting        10061f08     moc_PhylipPlugin.obj
 0003:00009f10       _Service_WorkflowDesigner  10061f10     moc_PhylipPlugin.obj
 0003:00009f18       _Service_QueryDesigner     10061f18     moc_PhylipPlugin.obj
 0003:00009f20       _Service_MinCoreServiceId  10061f20     moc_PhylipPlugin.obj
 0003:00009f28       _Service_MaxCoreServiceId  10061f28     moc_PhylipPlugin.obj
 0003:0000a838       __Tuple_alloc              10062838     DistanceMatrix.obj
 0003:0000a839       _ignore                    10062839     DistanceMatrix.obj
 0003:0000a83a       _allocator_arg             1006283a     DistanceMatrix.obj
 0003:0000a83b       _piecewise_construct       1006283b     DistanceMatrix.obj
 0003:0000a83c       _taskLog                   1006283c     DistanceMatrix.obj
 0003:0000a844       _algoLog                   10062844     DistanceMatrix.obj
 0003:0000a84c       _userActLog                1006284c     DistanceMatrix.obj
 0003:0000a854       _ioLog                     10062854     DistanceMatrix.obj
 0003:0000a85c       _coreLog                   1006285c     DistanceMatrix.obj
 0003:0000a864       _uiLog                     10062864     DistanceMatrix.obj
 0003:0000a86c       _scriptLog                 1006286c     DistanceMatrix.obj
 0003:0000a874       _perfLog                   10062874     DistanceMatrix.obj
 0003:0000a87c       _cmdLog                    1006287c     DistanceMatrix.obj
 0003:0000a88c       _factors                   1006288c     NeighborJoinAdapter.obj
 0003:0000a88d       _xml                       1006288d     NeighborJoinAdapter.obj
 0003:0000a88e       _nexus                     1006288e     NeighborJoinAdapter.obj
 0003:0000a88f       _weights                   1006288f     NeighborJoinAdapter.obj
 0003:0000a890       _categories                10062890     NeighborJoinAdapter.obj
 0003:0000a891       _justwts                   10062891     NeighborJoinAdapter.obj
 0003:0000a894       _nodef                     10062894     NeighborJoinAdapter.obj
 0003:0000a898       __Tuple_alloc              10062898     NeighborJoinAdapter.obj
 0003:0000a899       _ignore                    10062899     NeighborJoinAdapter.obj
 0003:0000a89a       _allocator_arg             1006289a     NeighborJoinAdapter.obj
 0003:0000a89b       _piecewise_construct       1006289b     NeighborJoinAdapter.obj
 0003:0000a89c       _taskLog                   1006289c     NeighborJoinAdapter.obj
 0003:0000a8a4       _algoLog                   100628a4     NeighborJoinAdapter.obj
 0003:0000a8ac       _userActLog                100628ac     NeighborJoinAdapter.obj
 0003:0000a8b4       _ioLog                     100628b4     NeighborJoinAdapter.obj
 0003:0000a8bc       _coreLog                   100628bc     NeighborJoinAdapter.obj
 0003:0000a8c4       _uiLog                     100628c4     NeighborJoinAdapter.obj
 0003:0000a8cc       _scriptLog                 100628cc     NeighborJoinAdapter.obj
 0003:0000a8d8       _perfLog                   100628d8     NeighborJoinAdapter.obj
 0003:0000a8e0       _cmdLog                    100628e0     NeighborJoinAdapter.obj
 0003:0000a8e8       ?counter@?9??createPhyTreeFromPhylipTree@U2@@YAXABVMultipleSequenceAlignment@2@PAUnode@@NE1PAVPhyNode@2@H@Z@4HA 100628e8     NeighborJoinAdapter.obj
 0003:0000a8f0       ?cvar@?1??run@NeighborJoinCalculateTreeTask@U2@@UAEXXZ@4VGReportableCounter@3@A 100628f0     NeighborJoinAdapter.obj
 0003:0000a918       ?$S1@?1??run@NeighborJoinCalculateTreeTask@U2@@UAEXXZ@4IA 10062918     NeighborJoinAdapter.obj
 0003:0000a91c       __Tuple_alloc              1006291c     NeighborJoinWidget.obj
 0003:0000a91d       _ignore                    1006291d     NeighborJoinWidget.obj
 0003:0000a91e       _allocator_arg             1006291e     NeighborJoinWidget.obj
 0003:0000a91f       _piecewise_construct       1006291f     NeighborJoinWidget.obj
 0003:0000a920       _taskLog                   10062920     NeighborJoinWidget.obj
 0003:0000a928       _algoLog                   10062928     NeighborJoinWidget.obj
 0003:0000a930       _userActLog                10062930     NeighborJoinWidget.obj
 0003:0000a938       _ioLog                     10062938     NeighborJoinWidget.obj
 0003:0000a940       _coreLog                   10062940     NeighborJoinWidget.obj
 0003:0000a94c       _uiLog                     1006294c     NeighborJoinWidget.obj
 0003:0000a954       _scriptLog                 10062954     NeighborJoinWidget.obj
 0003:0000a95c       _perfLog                   1006295c     NeighborJoinWidget.obj
 0003:0000a964       _cmdLog                    10062964     NeighborJoinWidget.obj
 0003:0000a978       ?list@?1??getConsensusModelTypes@ConsensusModelTypes@U2@@SA?AV?$QList@VQString@@@@XZ@4V4@A 10062978     NeighborJoinWidget.obj
 0003:0000a97c       ?$S1@?1??getConsensusModelTypes@ConsensusModelTypes@U2@@SA?AV?$QList@VQString@@@@XZ@4IA 1006297c     NeighborJoinWidget.obj
 0003:0000a980       __Tuple_alloc              10062980     PhylipCmdlineTask.obj
 0003:0000a981       _ignore                    10062981     PhylipCmdlineTask.obj
 0003:0000a982       _allocator_arg             10062982     PhylipCmdlineTask.obj
 0003:0000a983       _piecewise_construct       10062983     PhylipCmdlineTask.obj
 0003:0000a984       _taskLog                   10062984     PhylipCmdlineTask.obj
 0003:0000a98c       _algoLog                   1006298c     PhylipCmdlineTask.obj
 0003:0000a998       _userActLog                10062998     PhylipCmdlineTask.obj
 0003:0000a9a0       _ioLog                     100629a0     PhylipCmdlineTask.obj
 0003:0000a9b0       _coreLog                   100629b0     PhylipCmdlineTask.obj
 0003:0000a9c0       _uiLog                     100629c0     PhylipCmdlineTask.obj
 0003:0000a9c8       _scriptLog                 100629c8     PhylipCmdlineTask.obj
 0003:0000a9d0       _perfLog                   100629d0     PhylipCmdlineTask.obj
 0003:0000a9d8       _cmdLog                    100629d8     PhylipCmdlineTask.obj
 0003:0000a9f4       __Tuple_alloc              100629f4     PhylipPlugin.obj
 0003:0000a9f5       _ignore                    100629f5     PhylipPlugin.obj
 0003:0000a9f6       _allocator_arg             100629f6     PhylipPlugin.obj
 0003:0000a9f7       _piecewise_construct       100629f7     PhylipPlugin.obj
 0003:0000a9f8       _taskLog                   100629f8     PhylipPlugin.obj
 0003:0000aa00       _algoLog                   10062a00     PhylipPlugin.obj
 0003:0000aa08       _userActLog                10062a08     PhylipPlugin.obj
 0003:0000aa10       _ioLog                     10062a10     PhylipPlugin.obj
 0003:0000aa18       _coreLog                   10062a18     PhylipPlugin.obj
 0003:0000aa20       _uiLog                     10062a20     PhylipPlugin.obj
 0003:0000aa28       _scriptLog                 10062a28     PhylipPlugin.obj
 0003:0000aa30       _perfLog                   10062a30     PhylipPlugin.obj
 0003:0000aa3c       _cmdLog                    10062a3c     PhylipPlugin.obj
 0003:0000aa44       __Tuple_alloc              10062a44     PhylipPluginTests.obj
 0003:0000aa45       _ignore                    10062a45     PhylipPluginTests.obj
 0003:0000aa46       _allocator_arg             10062a46     PhylipPluginTests.obj
 0003:0000aa47       _piecewise_construct       10062a47     PhylipPluginTests.obj
 0003:0000aa48       _taskLog                   10062a48     PhylipPluginTests.obj
 0003:0000aa50       _algoLog                   10062a50     PhylipPluginTests.obj
 0003:0000aa58       _userActLog                10062a58     PhylipPluginTests.obj
 0003:0000aa60       _ioLog                     10062a60     PhylipPluginTests.obj
 0003:0000aa68       _coreLog                   10062a68     PhylipPluginTests.obj
 0003:0000aa70       _uiLog                     10062a70     PhylipPluginTests.obj
 0003:0000aa78       _scriptLog                 10062a78     PhylipPluginTests.obj
 0003:0000aa80       _perfLog                   10062a80     PhylipPluginTests.obj
 0003:0000aa88       _cmdLog                    10062a88     PhylipPluginTests.obj
 0003:0000aa90       __Tuple_alloc              10062a90     PhylipTask.obj
 0003:0000aa91       _ignore                    10062a91     PhylipTask.obj
 0003:0000aa92       _allocator_arg             10062a92     PhylipTask.obj
 0003:0000aa93       _piecewise_construct       10062a93     PhylipTask.obj
 0003:0000aa94       _taskLog                   10062a94     PhylipTask.obj
 0003:0000aa9c       _algoLog                   10062a9c     PhylipTask.obj
 0003:0000aaa4       _userActLog                10062aa4     PhylipTask.obj
 0003:0000aaac       _ioLog                     10062aac     PhylipTask.obj
 0003:0000aab4       _coreLog                   10062ab4     PhylipTask.obj
 0003:0000aabc       _uiLog                     10062abc     PhylipTask.obj
 0003:0000aac4       _scriptLog                 10062ac4     PhylipTask.obj
 0003:0000aacc       _perfLog                   10062acc     PhylipTask.obj
 0003:0000aad4       _cmdLog                    10062ad4     PhylipTask.obj
 0003:0000aadc       _factors                   10062adc     SeqBootAdapter.obj
 0003:0000aadd       _xml                       10062add     SeqBootAdapter.obj
 0003:0000aade       _nexus                     10062ade     SeqBootAdapter.obj
 0003:0000aadf       _weights                   10062adf     SeqBootAdapter.obj
 0003:0000aae0       _categories                10062ae0     SeqBootAdapter.obj
 0003:0000aae1       _justwts                   10062ae1     SeqBootAdapter.obj
 0003:0000aae4       _nodef                     10062ae4     SeqBootAdapter.obj
 0003:0000aae8       __Tuple_alloc              10062ae8     SeqBootAdapter.obj
 0003:0000aae9       _ignore                    10062ae9     SeqBootAdapter.obj
 0003:0000aaea       _allocator_arg             10062aea     SeqBootAdapter.obj
 0003:0000aaeb       _piecewise_construct       10062aeb     SeqBootAdapter.obj
 0003:0000aaec       _taskLog                   10062aec     SeqBootAdapter.obj
 0003:0000aaf4       _algoLog                   10062af4     SeqBootAdapter.obj
 0003:0000aafc       _userActLog                10062afc     SeqBootAdapter.obj
 0003:0000ab04       _ioLog                     10062b04     SeqBootAdapter.obj
 0003:0000ab0c       _coreLog                   10062b0c     SeqBootAdapter.obj
 0003:0000ab14       _uiLog                     10062b14     SeqBootAdapter.obj
 0003:0000ab1c       _scriptLog                 10062b1c     SeqBootAdapter.obj
 0003:0000ab24       _perfLog                   10062b24     SeqBootAdapter.obj
 0003:0000ab2c       _cmdLog                    10062b2c     SeqBootAdapter.obj
 0003:0000abc0       __Tuple_alloc              10062bc0     dist.obj
 0003:0000abc1       _ignore                    10062bc1     dist.obj
 0003:0000abc2       _allocator_arg             10062bc2     dist.obj
 0003:0000abc3       _piecewise_construct       10062bc3     dist.obj
 0003:0000abc4       _taskLog                   10062bc4     dist.obj
 0003:0000abcc       _algoLog                   10062bcc     dist.obj
 0003:0000abd4       _userActLog                10062bd4     dist.obj
 0003:0000abdc       _ioLog                     10062bdc     dist.obj
 0003:0000abe4       _coreLog                   10062be4     dist.obj
 0003:0000abec       _uiLog                     10062bec     dist.obj
 0003:0000abf4       _scriptLog                 10062bf4     dist.obj
 0003:0000abfc       _perfLog                   10062bfc     dist.obj
 0003:0000ac04       _cmdLog                    10062c04     dist.obj
 0003:0000b248       __Tuple_alloc              10063248     dnadist.obj
 0003:0000b249       _ignore                    10063249     dnadist.obj
 0003:0000b24a       _allocator_arg             1006324a     dnadist.obj
 0003:0000b24b       _piecewise_construct       1006324b     dnadist.obj
 0003:0000b250       _taskLog                   10063250     dnadist.obj
 0003:0000b258       _algoLog                   10063258     dnadist.obj
 0003:0000b260       _userActLog                10063260     dnadist.obj
 0003:0000b268       _ioLog                     10063268     dnadist.obj
 0003:0000b270       _coreLog                   10063270     dnadist.obj
 0003:0000b278       _uiLog                     10063278     dnadist.obj
 0003:0000b280       _scriptLog                 10063280     dnadist.obj
 0003:0000b288       _perfLog                   10063288     dnadist.obj
 0003:0000b290       _dnaDistSettings           10063290     dnadist.obj
 0003:0000b2f0       _cmdLog                    100632f0     dnadist.obj
 0003:0000b2fc       ?list@?1??getDNADistModelTypes@DNADistModelTypes@@SA?AV?$QList@VQString@@@@XZ@4V3@A 100632fc     dnadist.obj
 0003:0000b300       ?$S1@?1??getDNADistModelTypes@DNADistModelTypes@@SA?AV?$QList@VQString@@@@XZ@4IA 10063300     dnadist.obj
 0003:0000b308       __Tuple_alloc              10063308     neighbor.obj
 0003:0000b309       _ignore                    10063309     neighbor.obj
 0003:0000b30a       _allocator_arg             1006330a     neighbor.obj
 0003:0000b30b       _piecewise_construct       1006330b     neighbor.obj
 0003:0000b30c       _taskLog                   1006330c     neighbor.obj
 0003:0000b314       _algoLog                   10063314     neighbor.obj
 0003:0000b31c       _userActLog                1006331c     neighbor.obj
 0003:0000b324       _ioLog                     10063324     neighbor.obj
 0003:0000b32c       _coreLog                   1006332c     neighbor.obj
 0003:0000b334       _uiLog                     10063334     neighbor.obj
 0003:0000b33c       _scriptLog                 1006333c     neighbor.obj
 0003:0000b344       _perfLog                   10063344     neighbor.obj
 0003:0000b34c       _cmdLog                    1006334c     neighbor.obj
 0003:0000b354       _nonodes2                  10063354     neighbor.obj
 0003:0000b358       _outfilename               10063358     neighbor.obj
 0003:0000b420       _outtreename               10063420     neighbor.obj
 0003:0000b4e8       _outgrno                   100634e8     neighbor.obj
 0003:0000b4ec       _col                       100634ec     neighbor.obj
 0003:0000b4f0       _datasets                  100634f0     neighbor.obj
 0003:0000b4f4       _ith                       100634f4     neighbor.obj
 0003:0000b4f8       _x                         100634f8     neighbor.obj
 0003:0000b4fc       _reps                      100634fc     neighbor.obj
 0003:0000b500       _jumble                    10063500     neighbor.obj
 0003:0000b501       _lower                     10063501     neighbor.obj
 0003:0000b502       _upper                     10063502     neighbor.obj
 0003:0000b503       _outgropt                  10063503     neighbor.obj
 0003:0000b504       _replicates                10063504     neighbor.obj
 0003:0000b505       _trout                     10063505     neighbor.obj
 0003:0000b506       _printdata                 10063506     neighbor.obj
 0003:0000b507       _progress                  10063507     neighbor.obj
 0003:0000b508       _treeprint                 10063508     neighbor.obj
 0003:0000b509       _mulsets                   10063509     neighbor.obj
 0003:0000b50a       _njoin                     1006350a     neighbor.obj
 0003:0000b510       _curtree                   10063510     neighbor.obj
 0003:0000b538       _seed                      10063538     neighbor.obj
 0003:0000b550       _enterorder                10063550     neighbor.obj
 0003:0000b554       _cluster                   10063554     neighbor.obj
 0003:0000b578       _ts                        10063578     phylip.obj
 0003:0000b57c       _isBootstrap               1006357c     phylip.obj
 0003:0000b5b4       __Tuple_alloc              100635b4     phylip.obj
 0003:0000b5b5       _ignore                    100635b5     phylip.obj
 0003:0000b5b6       _allocator_arg             100635b6     phylip.obj
 0003:0000b5b7       _piecewise_construct       100635b7     phylip.obj
 0003:0000b5b8       _taskLog                   100635b8     phylip.obj
 0003:0000b5c0       _algoLog                   100635c0     phylip.obj
 0003:0000b5c8       _userActLog                100635c8     phylip.obj
 0003:0000b5d0       _ioLog                     100635d0     phylip.obj
 0003:0000b5d8       _coreLog                   100635d8     phylip.obj
 0003:0000b5e0       _uiLog                     100635e0     phylip.obj
 0003:0000b5e8       _scriptLog                 100635e8     phylip.obj
 0003:0000b5f0       _perfLog                   100635f0     phylip.obj
 0003:0000b5f8       _cmdLog                    100635f8     phylip.obj
 0003:0000d268       __Tuple_alloc              10065268     protdist.obj
 0003:0000d269       _ignore                    10065269     protdist.obj
 0003:0000d26a       _allocator_arg             1006526a     protdist.obj
 0003:0000d26b       _piecewise_construct       1006526b     protdist.obj
 0003:0000d26c       _taskLog                   1006526c     protdist.obj
 0003:0000d274       _algoLog                   10065274     protdist.obj
 0003:0000d27c       _userActLog                1006527c     protdist.obj
 0003:0000d284       _ioLog                     10065284     protdist.obj
 0003:0000d28c       _coreLog                   1006528c     protdist.obj
 0003:0000d294       _uiLog                     10065294     protdist.obj
 0003:0000d29c       _scriptLog                 1006529c     protdist.obj
 0003:0000d2a8       _perfLog                   100652a8     protdist.obj
 0003:0000d2b8       _cmdLog                    100652b8     protdist.obj
 0003:0000d2c4       ?list@?1??getProtDistModelTypes@ProtDistModelTypes@@SA?AV?$QList@VQString@@@@XZ@4V3@A 100652c4     protdist.obj
 0003:0000d2c8       ?$S1@?1??getProtDistModelTypes@ProtDistModelTypes@@SA?AV?$QList@VQString@@@@XZ@4IA 100652c8     protdist.obj
 0003:0000d300       _factors                   10065300     seqboot.obj
 0003:0000d301       _xml                       10065301     seqboot.obj
 0003:0000d302       _nexus                     10065302     seqboot.obj
 0003:0000d303       _weights                   10065303     seqboot.obj
 0003:0000d304       _categories                10065304     seqboot.obj
 0003:0000d305       _justwts                   10065305     seqboot.obj
 0003:0000d344       _nodef                     10065344     seqboot.obj
 0003:0000d380       __Tuple_alloc              10065380     seqboot.obj
 0003:0000d381       _ignore                    10065381     seqboot.obj
 0003:0000d382       _allocator_arg             10065382     seqboot.obj
 0003:0000d383       _piecewise_construct       10065383     seqboot.obj
 0003:0000d384       _taskLog                   10065384     seqboot.obj
 0003:0000d38c       _algoLog                   1006538c     seqboot.obj
 0003:0000d394       _userActLog                10065394     seqboot.obj
 0003:0000d39c       _ioLog                     1006539c     seqboot.obj
 0003:0000d3a4       _coreLog                   100653a4     seqboot.obj
 0003:0000d3ac       _uiLog                     100653ac     seqboot.obj
 0003:0000d3b4       _scriptLog                 100653b4     seqboot.obj
 0003:0000d3bc       _perfLog                   100653bc     seqboot.obj
 0003:0000d3c4       _cmdLog                    100653c4     seqboot.obj
 0003:0000d3cc       _bootstrap                 100653cc     seqboot.obj
 0003:0000d3cd       _jackknife                 100653cd     seqboot.obj
 0003:0000d3ce       _permute                   100653ce     seqboot.obj
 0003:0000d3cf       _ild                       100653cf     seqboot.obj
 0003:0000d3d0       _lockhart                  100653d0     seqboot.obj
 0003:0000d3d1       _rewrite                   100653d1     seqboot.obj
 0003:0000d3d2       _enzymes                   100653d2     seqboot.obj
 0003:0000d3d3       _all                       100653d3     seqboot.obj
 0003:0000d3d4       _mixture                   100653d4     seqboot.obj
 0003:0000d3d5       _ancvar                    100653d5     seqboot.obj
 0003:0000d3d6       _firstrep                  100653d6     seqboot.obj
 0003:0000d3d8       _outcatfile                100653d8     seqboot.obj
 0003:0000d3dc       _outweightfile             100653dc     seqboot.obj
 0003:0000d3e0       _outmixfile                100653e0     seqboot.obj
 0003:0000d3e4       _outancfile                100653e4     seqboot.obj
 0003:0000d3e8       _outfactfile               100653e8     seqboot.obj
 0003:0000d3ec       _data                      100653ec     seqboot.obj
 0003:0000d3f0       _outfilename               100653f0     seqboot.obj
 0003:0000d4b8       _catfilename               100654b8     seqboot.obj
 0003:0000d580       _outcatfilename            10065580     seqboot.obj
 0003:0000d648       _weightfilename            10065648     seqboot.obj
 0003:0000d710       _outweightfilename         10065710     seqboot.obj
 0003:0000d7d8       _mixfilename               100657d8     seqboot.obj
 0003:0000d8a0       _outmixfilename            100658a0     seqboot.obj
 0003:0000d968       _ancfilename               10065968     seqboot.obj
 0003:0000da30       _outancfilename            10065a30     seqboot.obj
 0003:0000daf8       _factfilename              10065af8     seqboot.obj
 0003:0000dbc0       _outfactfilename           10065bc0     seqboot.obj
 0003:0000dc88       _seq                       10065c88     seqboot.obj
 0003:0000dc8c       _oldweight                 10065c8c     seqboot.obj
 0003:0000dc90       _where                     10065c90     seqboot.obj
 0003:0000dc94       _how_many                  10065c94     seqboot.obj
 0003:0000dc98       _mixdata                   10065c98     seqboot.obj
 0003:0000dc9c       _ancdata                   10065c9c     seqboot.obj
 0003:0000dca0       ?curnewergroups@?1??allocnewer@@YAXJJ@Z@4JA 10065ca0     seqboot.obj
 0003:0000dca4       ?curnewersites@?1??allocnewer@@YAXJJ@Z@4JA 10065ca4     seqboot.obj
 0003:0000dca8       __Tuple_alloc              10065ca8     moc_NeighborJoinWidget.obj
 0003:0000dca9       _ignore                    10065ca9     moc_NeighborJoinWidget.obj
 0003:0000dcaa       _allocator_arg             10065caa     moc_NeighborJoinWidget.obj
 0003:0000dcab       _piecewise_construct       10065cab     moc_NeighborJoinWidget.obj
 0003:0000dcac       _taskLog                   10065cac     moc_NeighborJoinWidget.obj
 0003:0000dcb4       _algoLog                   10065cb4     moc_NeighborJoinWidget.obj
 0003:0000dcbc       _userActLog                10065cbc     moc_NeighborJoinWidget.obj
 0003:0000dcc4       _ioLog                     10065cc4     moc_NeighborJoinWidget.obj
 0003:0000dccc       _coreLog                   10065ccc     moc_NeighborJoinWidget.obj
 0003:0000dcd4       _uiLog                     10065cd4     moc_NeighborJoinWidget.obj
 0003:0000dcdc       _scriptLog                 10065cdc     moc_NeighborJoinWidget.obj
 0003:0000dce4       _perfLog                   10065ce4     moc_NeighborJoinWidget.obj
 0003:0000dcec       _cmdLog                    10065cec     moc_NeighborJoinWidget.obj
 0003:0000dcf4       __Tuple_alloc              10065cf4     moc_PhylipCmdlineTask.obj
 0003:0000dcf5       _ignore                    10065cf5     moc_PhylipCmdlineTask.obj
 0003:0000dcf6       _allocator_arg             10065cf6     moc_PhylipCmdlineTask.obj
 0003:0000dcf7       _piecewise_construct       10065cf7     moc_PhylipCmdlineTask.obj
 0003:0000dcf8       _taskLog                   10065cf8     moc_PhylipCmdlineTask.obj
 0003:0000dd00       _algoLog                   10065d00     moc_PhylipCmdlineTask.obj
 0003:0000dd08       _userActLog                10065d08     moc_PhylipCmdlineTask.obj
 0003:0000dd10       _ioLog                     10065d10     moc_PhylipCmdlineTask.obj
 0003:0000dd18       _coreLog                   10065d18     moc_PhylipCmdlineTask.obj
 0003:0000dd20       _uiLog                     10065d20     moc_PhylipCmdlineTask.obj
 0003:0000dd28       _scriptLog                 10065d28     moc_PhylipCmdlineTask.obj
 0003:0000dd30       _perfLog                   10065d30     moc_PhylipCmdlineTask.obj
 0003:0000dd38       _cmdLog                    10065d38     moc_PhylipCmdlineTask.obj
 0003:0000dd40       __Tuple_alloc              10065d40     moc_PhylipPlugin.obj
 0003:0000dd41       _ignore                    10065d41     moc_PhylipPlugin.obj
 0003:0000dd42       _allocator_arg             10065d42     moc_PhylipPlugin.obj
 0003:0000dd43       _piecewise_construct       10065d43     moc_PhylipPlugin.obj
 0003:0000dd44       __Tuple_alloc              10065d44     moc_PhylipPluginTests.obj
 0003:0000dd45       _ignore                    10065d45     moc_PhylipPluginTests.obj
 0003:0000dd46       _allocator_arg             10065d46     moc_PhylipPluginTests.obj
 0003:0000dd47       _piecewise_construct       10065d47     moc_PhylipPluginTests.obj
 0003:0000dd48       _taskLog                   10065d48     moc_PhylipPluginTests.obj
 0003:0000dd50       _algoLog                   10065d50     moc_PhylipPluginTests.obj
 0003:0000dd58       _userActLog                10065d58     moc_PhylipPluginTests.obj
 0003:0000dd60       _ioLog                     10065d60     moc_PhylipPluginTests.obj
 0003:0000dd68       _coreLog                   10065d68     moc_PhylipPluginTests.obj
 0003:0000dd70       _uiLog                     10065d70     moc_PhylipPluginTests.obj
 0003:0000dd78       _scriptLog                 10065d78     moc_PhylipPluginTests.obj
 0003:0000dd80       _perfLog                   10065d80     moc_PhylipPluginTests.obj
 0003:0000dd88       _cmdLog                    10065d88     moc_PhylipPluginTests.obj
 0003:0000dd90       __Tuple_alloc              10065d90     moc_PhylipTask.obj
 0003:0000dd91       _ignore                    10065d91     moc_PhylipTask.obj
 0003:0000dd92       _allocator_arg             10065d92     moc_PhylipTask.obj
 0003:0000dd93       _piecewise_construct       10065d93     moc_PhylipTask.obj
 0003:0000dd94       _taskLog                   10065d94     moc_PhylipTask.obj
 0003:0000dd9c       _algoLog                   10065d9c     moc_PhylipTask.obj
 0003:0000dda4       _userActLog                10065da4     moc_PhylipTask.obj
 0003:0000ddac       _ioLog                     10065dac     moc_PhylipTask.obj
 0003:0000ddb4       _coreLog                   10065db4     moc_PhylipTask.obj
 0003:0000ddbc       _uiLog                     10065dbc     moc_PhylipTask.obj
 0003:0000ddc4       _scriptLog                 10065dc4     moc_PhylipTask.obj
 0003:0000ddcc       _perfLog                   10065dcc     moc_PhylipTask.obj
 0003:0000ddd4       _cmdLog                    10065dd4     moc_PhylipTask.obj
 0003:0000dde0       _GS_ExceptionRecord        10065de0     MSVCRT:gs_report.obj
 0003:0000de30       _GS_ContextRecord          10065e30     MSVCRT:gs_report.obj
 0003:0000e0fc       _DebuggerWasPresent        100660fc     MSVCRT:gs_report.obj
 0003:0000e108       ___proc_attached           10066108     MSVCRT:crtdll.obj
 0004:00000060       $R000000                   10067060     * linker generated manifest res *

 Exports

  ordinal    name

        1    _ugene_plugin_init
               exported name: ugene_plugin_init
